 config_alm_bncs_output

 Timestamp is 614c80e0 (Thu Sep 23 13:28:00 2021)

 Preferred load address is 10000000

 Start         Length     Name                   Class
 0001:00000000 00000134H .text$di                CODE
 0001:00000140 00017b2cH .text$mn                CODE
 0001:00017c70 0000433dH .text$x                 CODE
 0001:0001bfb0 0000008fH .text$yd                CODE
 0002:00000000 0000135cH .idata$5                DATA
 0002:0000135c 00000004H .CRT$XCA                DATA
 0002:00001360 00000024H .CRT$XCU                DATA
 0002:00001384 00000004H .CRT$XCZ                DATA
 0002:00001388 00000004H .CRT$XIA                DATA
 0002:0000138c 00000004H .CRT$XIAA               DATA
 0002:00001390 00000004H .CRT$XIC                DATA
 0002:00001394 00000004H .CRT$XIZ                DATA
 0002:00001398 00008008H .rdata                  DATA
 0002:000093a0 00001a58H .rdata$r                DATA
 0002:0000adf8 00000004H .rtc$IAA                DATA
 0002:0000adfc 00000004H .rtc$IZZ                DATA
 0002:0000ae00 00000004H .rtc$TAA                DATA
 0002:0000ae04 00000004H .rtc$TZZ                DATA
 0002:0000ae08 000041acH .xdata$x                DATA
 0002:0000efc0 0000006aH .edata                  DATA
 0002:0000f02c 00000078H .idata$2                DATA
 0002:0000f0a4 00000014H .idata$3                DATA
 0002:0000f0b8 0000135cH .idata$4                DATA
 0002:00010414 0000c8daH .idata$6                DATA
 0003:00000000 00000174H .data                   DATA
 0003:00000174 00000844H .data$r                 DATA
 0003:000009b8 00000454H .bss                    DATA
 0004:00000000 000000a0H .rsrc$01                DATA
 0004:000000a0 00000620H .rsrc$02                DATA

  Address         Publics by Value              Rva+Base       Lib:Object

 0000:00000000       __except_list              00000000     <absolute>
 0000:00000000       ___guard_flags             00000000     <absolute>
 0000:00000000       ___safe_se_handler_count   00000000     <absolute>
 0000:00000000       ___guard_fids_table        00000000     <absolute>
 0000:00000000       ___safe_se_handler_table   00000000     <absolute>
 0000:00000000       ___guard_fids_count        00000000     <absolute>
 0000:00009876       __ldused                   00009876     <absolute>
 0000:00009876       __fltused                  00009876     <absolute>
 0000:00000000       ___ImageBase               10000000     <linker-defined>
 0001:00000140       ??0?$QGuardedPtr@VQPopupMenu@@@@QAE@XZ 10001140 f i alm_bncs_output.obj
 0001:00000140       ??0?$QGuardedPtr@VQDockWindow@@@@QAE@XZ 10001140 f i alm_bncs_output.obj
 0001:00000181       ??0?$QMap@VQString@@W4ESection@@@@QAE@XZ 10001181 f i alm_bncs_output.obj
 0001:000001b4       ??0?$QMapNode@VQString@@W4ESection@@@@QAE@ABU0@@Z 100011b4 f i alm_bncs_output.obj
 0001:000001f2       ??0?$QMapNode@VQString@@W4ESection@@@@QAE@ABVQString@@@Z 100011f2 f i alm_bncs_output.obj
 0001:00000226       ??0?$QMapPrivate@VQString@@W4ESection@@@@QAE@PBV0@@Z 10001226 f i alm_bncs_output.obj
 0001:000002d8       ??0?$QMapPrivate@VQString@@W4ESection@@@@QAE@XZ 100012d8 f i alm_bncs_output.obj
 0001:00000334       ??0FileLoad_BncsSystem@alm_bncs_output@@QAE@PAV1@@Z 10001334 f   alm_bncs_output.obj
 0001:000003a5       ??0alm_bncs_output@@QAE@ABVQString@@00@Z 100013a5 f   alm_bncs_output.obj
 0001:00001000       ??0config_plugin_base@@QAE@ABVQString@@00@Z 10002000 f i alm_bncs_output.obj
 0001:0000108d       ??1?$QDictIterator@VdevTemplate@@@@QAE@XZ 1000208d f i alm_bncs_output.obj
 0001:00001093       ??1?$QGuardedPtr@VQPopupMenu@@@@QAE@XZ 10002093 f i alm_bncs_output.obj
 0001:00001093       ??1?$QGuardedPtr@VQDockWindow@@@@QAE@XZ 10002093 f i alm_bncs_output.obj
 0001:00001098       ??1?$QMap@VQString@@W4ESection@@@@QAE@XZ 10002098 f i alm_bncs_output.obj
 0001:000010b5       ??1?$QMapPrivate@VQString@@W4ESection@@@@QAE@XZ 100020b5 f i alm_bncs_output.obj
 0001:000010d6       ??1?$QPtrList@VQPopupMenu@@@@UAE@XZ 100020d6 f i alm_bncs_output.obj
 0001:00001109       ??1?$QPtrList@VcOutputFile@@@@UAE@XZ 10002109 f i alm_bncs_output.obj
 0001:0000113c       ??1FileLoad_BncsSystem@alm_bncs_output@@UAE@XZ 1000213c f   alm_bncs_output.obj
 0001:00001175       ??1IDomDoc@@UAE@XZ         10002175 f i alm_bncs_output.obj
 0001:0000117c       ??1QDockWindowList@@UAE@XZ 1000217c f i alm_bncs_output.obj
 0001:000011c5       ??1QPopupMenuList@@UAE@XZ  100021c5 f i alm_bncs_output.obj
 0001:000011f7       ??1alm_bncs_output@@UAE@XZ 100021f7 f   alm_bncs_output.obj
 0001:0000139e       ??1config_plugin_base@@UAE@XZ 1000239e f i alm_bncs_output.obj
 0001:000013f8       ??4?$QGuardedPtr@VQDockWindow@@@@QAEAAV0@PAVQDockWindow@@@Z 100023f8 f i alm_bncs_output.obj
 0001:000013f8       ??4?$QGuardedPtr@VQPopupMenu@@@@QAEAAV0@PAVQPopupMenu@@@Z 100023f8 f i alm_bncs_output.obj
 0001:00001456       ??_ECAlm_sys_select@@WCI@AEPAXI@Z 10002456 f i alm_bncs_output.obj
 0001:0000145e       ??_EQBoxLayout@@WCI@AEPAXI@Z 1000245e f i alm_bncs_output.obj
 0001:00001466       ??_EQDockWindow@@WCI@AEPAXI@Z 10002466 f i alm_bncs_output.obj
 0001:0000146e       ??_EQListView@@WCI@AEPAXI@Z 1000246e f i alm_bncs_output.obj
 0001:00001476       ??_EQPopupMenu@@WCI@AEPAXI@Z 10002476 f i alm_bncs_output.obj
 0001:0000147e       ??_EQPopupMenu@@WIM@AEPAXI@Z 1000247e f i alm_bncs_output.obj
 0001:00001489       ??_EQTabWidget@@WCI@AEPAXI@Z 10002489 f i alm_bncs_output.obj
 0001:00001491       ??_EQToolBar@@WCI@AEPAXI@Z 10002491 f i alm_bncs_output.obj
 0001:00001499       ??_EQWidget@@WCI@AEPAXI@Z  10002499 f i alm_bncs_output.obj
 0001:000014a1       ??_Ealm_bncs_output@@WCI@AEPAXI@Z 100024a1 f i alm_bncs_output.obj
 0001:000014a9       ??_Ealm_bncs_output@@WHI@AEPAXI@Z 100024a9 f i alm_bncs_output.obj
 0001:000014b1       ??_Econfig_plugin_base@@WCI@AEPAXI@Z 100024b1 f i alm_bncs_output.obj
 0001:000014b9       ??_E?$QPtrList@VQPopupMenu@@@@UAEPAXI@Z 100024b9 f i alm_bncs_output.obj
 0001:000014b9       ??_G?$QPtrList@VQPopupMenu@@@@UAEPAXI@Z 100024b9 f i alm_bncs_output.obj
 0001:000014d8       ??_E?$QPtrList@VcOutputFile@@@@UAEPAXI@Z 100024d8 f i alm_bncs_output.obj
 0001:000014d8       ??_G?$QPtrList@VcOutputFile@@@@UAEPAXI@Z 100024d8 f i alm_bncs_output.obj
 0001:000014f7       ??_GCAlm_sys_select@@UAEPAXI@Z 100024f7 f i alm_bncs_output.obj
 0001:000014f7       ??_ECAlm_sys_select@@UAEPAXI@Z 100024f7 f i alm_bncs_output.obj
 0001:00001517       ??_GFileLoad_BncsSystem@alm_bncs_output@@UAEPAXI@Z 10002517 f i alm_bncs_output.obj
 0001:00001517       ??_EFileLoad_BncsSystem@alm_bncs_output@@UAEPAXI@Z 10002517 f i alm_bncs_output.obj
 0001:00001536       ??_EIDomDoc@@UAEPAXI@Z     10002536 f i alm_bncs_output.obj
 0001:00001536       ??_GIDomDoc@@UAEPAXI@Z     10002536 f i alm_bncs_output.obj
 0001:00001556       ??_EQAction@@UAEPAXI@Z     10002556 f i alm_bncs_output.obj
 0001:00001556       ??_GQAction@@UAEPAXI@Z     10002556 f i alm_bncs_output.obj
 0001:00001576       ??_GQBoxLayout@@UAEPAXI@Z  10002576 f i alm_bncs_output.obj
 0001:00001576       ??_EQBoxLayout@@UAEPAXI@Z  10002576 f i alm_bncs_output.obj
 0001:00001596       ??_EQDockWindow@@UAEPAXI@Z 10002596 f i alm_bncs_output.obj
 0001:00001596       ??_GQDockWindow@@UAEPAXI@Z 10002596 f i alm_bncs_output.obj
 0001:000015b6       ??_EQDockWindowList@@UAEPAXI@Z 100025b6 f i alm_bncs_output.obj
 0001:000015b6       ??_GQDockWindowList@@UAEPAXI@Z 100025b6 f i alm_bncs_output.obj
 0001:000015d5       ??_GQGuardedPtrPrivate@@UAEPAXI@Z 100025d5 f i alm_bncs_output.obj
 0001:000015d5       ??_EQGuardedPtrPrivate@@UAEPAXI@Z 100025d5 f i alm_bncs_output.obj
 0001:000015f5       ??_GQListView@@UAEPAXI@Z   100025f5 f i alm_bncs_output.obj
 0001:000015f5       ??_EQListView@@UAEPAXI@Z   100025f5 f i alm_bncs_output.obj
 0001:00001615       ??_GQListViewItem@@UAEPAXI@Z 10002615 f i alm_bncs_output.obj
 0001:00001615       ??_EQListViewItem@@UAEPAXI@Z 10002615 f i alm_bncs_output.obj
 0001:00001635       ??_EQPopupMenu@@UAEPAXI@Z  10002635 f i alm_bncs_output.obj
 0001:00001635       ??_GQPopupMenu@@UAEPAXI@Z  10002635 f i alm_bncs_output.obj
 0001:00001655       ??_EQPopupMenuList@@UAEPAXI@Z 10002655 f i alm_bncs_output.obj
 0001:00001655       ??_GQPopupMenuList@@UAEPAXI@Z 10002655 f i alm_bncs_output.obj
 0001:00001674       ??_GQTabWidget@@UAEPAXI@Z  10002674 f i alm_bncs_output.obj
 0001:00001674       ??_EQTabWidget@@UAEPAXI@Z  10002674 f i alm_bncs_output.obj
 0001:00001694       ??_GQToolBar@@UAEPAXI@Z    10002694 f i alm_bncs_output.obj
 0001:00001694       ??_EQToolBar@@UAEPAXI@Z    10002694 f i alm_bncs_output.obj
 0001:000016b4       ??_EQWidget@@UAEPAXI@Z     100026b4 f i alm_bncs_output.obj
 0001:000016b4       ??_GQWidget@@UAEPAXI@Z     100026b4 f i alm_bncs_output.obj
 0001:000016d4       ??_Ealm_bncs_output@@UAEPAXI@Z 100026d4 f i alm_bncs_output.obj
 0001:000016d4       ??_Galm_bncs_output@@UAEPAXI@Z 100026d4 f i alm_bncs_output.obj
 0001:000016f3       ??_Econfig_plugin_base@@UAEPAXI@Z 100026f3 f i alm_bncs_output.obj
 0001:000016f3       ??_Gconfig_plugin_base@@UAEPAXI@Z 100026f3 f i alm_bncs_output.obj
 0001:00001712       ??_GdevTemplate@@UAEPAXI@Z 10002712 f i alm_bncs_output.obj
 0001:00001712       ??_EdevTemplate@@UAEPAXI@Z 10002712 f i alm_bncs_output.obj
 0001:00001731       ?EditProcess@alm_bncs_output@@QAEXXZ 10002731 f   alm_bncs_output.obj
 0001:000017fe       ?GetBncsSystem@alm_bncs_output@@UBEPAVDocument_BncsSystem@@XZ 100027fe f   alm_bncs_output.obj
 0001:00001805       ?GetLaunch@alm_bncs_output@@UBEPAVDocument_Launch@@XZ 10002805 f   alm_bncs_output.obj
 0001:00001805       ?GetDeviceDescriptions@alm_bncs_output@@UBEPAVDocumentSet_DeviceDescription@@XZ 10002805 f   alm_bncs_output.obj
 0001:00001805       ?GetComplexSpecs@alm_bncs_output@@UBEPAVDocumentSet_ComplexSpec@@XZ 10002805 f   alm_bncs_output.obj
 0001:00001805       ?GetDevicetypes@alm_bncs_output@@UBEPAVDocument_Devicetypes@@XZ 10002805 f   alm_bncs_output.obj
 0001:00001805       ?GetInstances@alm_bncs_output@@UBEPAVDocument_Instances@@XZ 10002805 f   alm_bncs_output.obj
 0001:00001808       ?about@alm_bncs_output@@UAE?AVQString@@XZ 10002808 f   alm_bncs_output.obj
 0001:0000185c       ?about@config_plugin_base@@UAE?AVQString@@XZ 1000285c f i alm_bncs_output.obj
 0001:000018b2       ?activate@alm_bncs_output@@UAEX_N@Z 100028b2 f   alm_bncs_output.obj
 0001:00001a8a       ?allocateCfgFileName@alm_bncs_output@@AAEXAAVQString@@0@Z 10002a8a f   alm_bncs_output.obj
 0001:00001c38       ?allocateModuleName@alm_bncs_output@@AAEXAAVQString@@@Z 10002c38 f   alm_bncs_output.obj
 0001:00001d05       ?apply@alm_bncs_output@@UAEXXZ 10002d05 f   alm_bncs_output.obj
 0001:00001eb8       ?apply@config_plugin_base@@UAEXXZ 10002eb8 f i alm_bncs_output.obj
 0001:00001eb9       ?applyTemplates@alm_bncs_output@@QAEXXZ 10002eb9 f   alm_bncs_output.obj
 0001:0000238e       ?changeDevType@alm_bncs_output@@AAEXABVQString@@0@Z 1000338e f   alm_bncs_output.obj
 0001:0000248a       ?changeDevTypeDevicetypes@alm_bncs_output@@AAEXABVQString@@0@Z 1000348a f   alm_bncs_output.obj
 0001:00002bc6       ?changeDevTypeInstances@alm_bncs_output@@AAEXABVQString@@0@Z 10003bc6 f   alm_bncs_output.obj
 0001:000034bb       ?clear@?$QMapPrivate@VQString@@W4ESection@@@@QAEXPAU?$QMapNode@VQString@@W4ESection@@@@@Z 100044bb f i alm_bncs_output.obj
 0001:000034f3       ?clear@?$QMapPrivate@VQString@@W4ESection@@@@QAEXXZ 100044f3 f i alm_bncs_output.obj
 0001:00003530       ?clear@?$QPtrList@VDirLoad@@@@UAEXXZ 10004530 f i config_alarm_utilities:Loaders.obj
 0001:00003530       ?clear@?$QPtrList@VcOutputFile@@@@UAEXXZ 10004530 f i alm_bncs_output.obj
 0001:00003530       ?clear@?$QPtrList@VFileLoad@@@@UAEXXZ 10004530 f i config_alarm_utilities:Loaders.obj
 0001:00003530       ?clear@?$QPtrList@VQPopupMenu@@@@UAEXXZ 10004530 f i alm_bncs_output.obj
 0001:00003536       ?closeEvent@alm_bncs_output@@UAEXPAVQCloseEvent@@@Z 10004536 f   alm_bncs_output.obj
 0001:000036e1       ?closeEvent@config_plugin_base@@UAEXPAVQCloseEvent@@@Z 100046e1 f i alm_bncs_output.obj
 0001:000036ef       ?copy@?$QMapPrivate@VQString@@W4ESection@@@@QAEPAU?$QMapNode@VQString@@W4ESection@@@@PAU2@@Z 100046ef f i alm_bncs_output.obj
 0001:00003780       ?count@?$QPtrList@VDirLoad@@@@UBEIXZ 10004780 f i config_alarm_utilities:Loaders.obj
 0001:00003780       ?count@?$QPtrList@VQPopupMenu@@@@UBEIXZ 10004780 f i alm_bncs_output.obj
 0001:00003780       ?count@?$QPtrList@VFileLoad@@@@UBEIXZ 10004780 f i config_alarm_utilities:Loaders.obj
 0001:00003780       ?count@?$QPtrList@VcOutputFile@@@@UBEIXZ 10004780 f i alm_bncs_output.obj
 0001:00003784       ?createEmptyDomDoc@alm_bncs_output@@EBEXABVQString@@0AAVQDomDocument@@@Z 10004784 f   alm_bncs_output.obj
 0001:000038dc       ?currentKey@?$QDictIterator@VdevTemplate@@@@QBE?AVQString@@XZ 100048dc f i alm_bncs_output.obj
 0001:000038f6       ?dec@?$QMapIterator@VQString@@W4ESection@@@@AAEHXZ 100048f6 f i alm_bncs_output.obj
 0001:00003935       ?deleteAndLockDevDescs@alm_bncs_output@@AAEXABVQString@@0@Z 10004935 f   alm_bncs_output.obj
 0001:00003eef       ?deleteItem@?$QPtrList@VQPopupMenu@@@@EAEXPAX@Z 10004eef f i alm_bncs_output.obj
 0001:00003f0a       ?deleteItem@?$QDict@VdevTemplate@@@@EAEXPAX@Z 10004f0a f i devTemplate.obj
 0001:00003f0a       ?deleteItem@?$QPtrList@VcOutputFile@@@@EAEXPAX@Z 10004f0a f i alm_bncs_output.obj
 0001:00003f24       ?deref@?$QGuardedPtr@VQPopupMenu@@@@AAEXXZ 10004f24 f i alm_bncs_output.obj
 0001:00003f24       ?deref@?$QGuardedPtr@VQDockWindow@@@@AAEXXZ 10004f24 f i alm_bncs_output.obj
 0001:00003f39       ?detachInternal@?$QMap@VQString@@W4ESection@@@@AAEXXZ 10004f39 f i alm_bncs_output.obj
 0001:00003f70       ?doDone@alm_bncs_output@@AAEXPAVresponse@@@Z 10004f70 f   alm_bncs_output.obj
 0001:0000433a       ?doDownloadRead@alm_bncs_output@@AAEXPAVresponse@@@Z 1000533a f   alm_bncs_output.obj
 0001:000049bf       ?enableControls@alm_bncs_output@@AAEXXZ 100059bf f   alm_bncs_output.obj
 0001:00004b00       ?ensureFolderExists@alm_bncs_output@@AAE_NABVQString@@@Z 10005b00 f   alm_bncs_output.obj
 0001:00004c40       ?extractParam@alm_bncs_output@@AAE?AVQString@@ABV2@0PA_N@Z 10005c40 f   alm_bncs_output.obj
 0001:00004e1b       ?fileListContextMenu@alm_bncs_output@@QAEXPAVQListViewItem@@ABVQPoint@@H@Z 10005e1b f   alm_bncs_output.obj
 0001:00004e36       ?find@?$QMap@VQString@@W4ESection@@@@QAE?AV?$QMapIterator@VQString@@W4ESection@@@@ABVQString@@@Z 10005e36 f i alm_bncs_output.obj
 0001:00004e62       ?find@?$QMapPrivate@VQString@@W4ESection@@@@QBE?AV?$QMapConstIterator@VQString@@W4ESection@@@@ABVQString@@@Z 10005e62 f i alm_bncs_output.obj
 0001:00004ec0       ?getKey@config_plugin_base@@QAE?AVQString@@XZ 10005ec0 f i alm_bncs_output.obj
 0001:00004ede       ?inc@?$QMapConstIterator@VQString@@H@@AAEHXZ 10005ede f i alm_bncs_output.obj
 0001:00004ede       ?inc@?$QMapIterator@VQString@@V1@@@AAEHXZ 10005ede f i alm_bncs_output.obj
 0001:00004ede       ?inc@?$QMapIterator@VQString@@H@@AAEHXZ 10005ede f i alm_bncs_output.obj
 0001:00004f0f       ?insert@?$QMap@VQString@@W4ESection@@@@QAE?AV?$QMapIterator@VQString@@W4ESection@@@@ABVQString@@ABW4ESection@@_N@Z 10005f0f f i alm_bncs_output.obj
 0001:00004f54       ?insert@?$QMapPrivate@VQString@@W4ESection@@@@QAE?AV?$QMapIterator@VQString@@W4ESection@@@@PAUQMapNodeBase@@0ABVQString@@@Z 10005f54 f i alm_bncs_output.obj
 0001:00004ffd       ?insertModifiedInstances@alm_bncs_output@@AAE?AVQString@@PAV?$QDictIterator@VdevTemplate@@@@ABV2@11@Z 10005ffd f   alm_bncs_output.obj
 0001:00005415       ?insertSingle@?$QMapPrivate@VQString@@W4ESection@@@@QAE?AV?$QMapIterator@VQString@@W4ESection@@@@ABVQString@@@Z 10006415 f i alm_bncs_output.obj
 0001:000054a2       ?isDirty@alm_bncs_output@@UAE_NXZ 100064a2 f   alm_bncs_output.obj
 0001:000054a9       ?validate@config_plugin_base@@UAE_NXZ 100064a9 f i alm_bncs_output.obj
 0001:000054a9       ?isDirty@config_plugin_base@@UAE_NXZ 100064a9 f i alm_bncs_output.obj
 0001:000054ac       ?load@FileLoad_BncsSystem@alm_bncs_output@@UAEXABVQString@@@Z 100064ac f   alm_bncs_output.obj
 0001:000054d2       ?loadFile@alm_bncs_output@@AAE_NABVQString@@@Z 100064d2 f   alm_bncs_output.obj
 0001:00005de7       ?loadProcesses@alm_bncs_output@@AAE_NABVQString@@@Z 10006de7 f   alm_bncs_output.obj
 0001:000062ba       ?loadTemplates@alm_bncs_output@@AAEXABVQStringList@@ABV?$QMap@VQString@@V1@@@@Z 100072ba f   alm_bncs_output.obj
 0001:000066db       ?lockDevDesc@alm_bncs_output@@AAEXABVQString@@@Z 100076db f   alm_bncs_output.obj
 0001:0000677e       ?manageTemplate@alm_bncs_output@@QAEXXZ 1000777e f   alm_bncs_output.obj
 0001:00006b66       ?markDirty@alm_bncs_output@@QAEXXZ 10007b66 f   alm_bncs_output.obj
 0001:00006bd9       ?menuDeleteFile@alm_bncs_output@@QAEXXZ 10007bd9 f   alm_bncs_output.obj
 0001:00006d6b       ?menuDuplicateFile@alm_bncs_output@@QAEXXZ 10007d6b f   alm_bncs_output.obj
 0001:000070dd       ?menuNewFile@alm_bncs_output@@QAEXXZ 100080dd f   alm_bncs_output.obj
 0001:0000712f       ?menuRename@alm_bncs_output@@QAEXXZ 1000812f f   alm_bncs_output.obj
 0001:00007149       ?menus@alm_bncs_output@@UAE?AVQPopupMenuList@@XZ 10008149 f   alm_bncs_output.obj
 0001:00007196       ?menus@config_plugin_base@@UAE?AVQPopupMenuList@@XZ 10008196 f i alm_bncs_output.obj
 0001:000071b9       ?metaObject@alm_bncs_output@@UBEPAVQMetaObject@@XZ 100081b9 f i alm_bncs_output.obj
 0001:000071be       ?navigate@alm_bncs_output@@UAEXABVQString@@0@Z 100081be f   alm_bncs_output.obj
 0001:00007584       ?navigate@config_plugin_base@@UAEXABVQString@@0@Z 10008584 f i alm_bncs_output.obj
 0001:00007587       ?newFile@alm_bncs_output@@AAEXABVQString@@@Z 10008587 f   alm_bncs_output.obj
 0001:000079b1       ?renameModule@alm_bncs_output@@QAEXPAVQListViewItem@@HABVQString@@@Z 100089b1 f   alm_bncs_output.obj
 0001:00007be1       ?reply@alm_bncs_output@@UAEXPAVresponse@@@Z 10008be1 f   alm_bncs_output.obj
 0001:00007cb0       ?replyDownload@alm_bncs_output@@AAEXPAVresponse@@@Z 10008cb0 f   alm_bncs_output.obj
 0001:00007d99       ?replyLock@alm_bncs_output@@AAEXPAVresponse@@@Z 10008d99 f   alm_bncs_output.obj
 0001:000080b5       ?replyUpload@alm_bncs_output@@AAEXPAVresponse@@@Z 100090b5 f   alm_bncs_output.obj
 0001:0000813b       ?resizeEvent@alm_bncs_output@@UAEXPAVQResizeEvent@@@Z 1000913b f   alm_bncs_output.obj
 0001:00008170       ?saveFile@alm_bncs_output@@AAE_NQAVcOutputFile@@_N1@Z 10009170 f   alm_bncs_output.obj
 0001:0000869d       ?saveTemplates@alm_bncs_output@@AAEXPBVcOutputFile@@_NAAVQString@@2@Z 1000969d f   alm_bncs_output.obj
 0001:00008b97       ?selectFile@alm_bncs_output@@QAEXPAVQListViewItem@@@Z 10009b97 f   alm_bncs_output.obj
 0001:00008dd4       ?selectSystem@alm_bncs_output@@IAEXABVQString@@@Z 10009dd4 f   alm_bncs_output.obj
 0001:00009091       ?sendCommand@alm_bncs_output@@UAEXABVQString@@0@Z 1000a091 f   alm_bncs_output.obj
 0001:000090d2       ?setBncsSystemValues@alm_bncs_output@@AAEXXZ 1000a0d2 f   alm_bncs_output.obj
 0001:00009102       ?showLockedDevDescFileList@alm_bncs_output@@AAEXXZ 1000a102 f   alm_bncs_output.obj
 0001:00009214       ?toolbars@alm_bncs_output@@UAE?AVQDockWindowList@@XZ 1000a214 f   alm_bncs_output.obj
 0001:0000926f       ?toolbars@config_plugin_base@@UAE?AVQDockWindowList@@XZ 1000a26f f i alm_bncs_output.obj
 0001:00009292       ?updateFileList@alm_bncs_output@@AAEXXZ 1000a292 f   alm_bncs_output.obj
 0001:00009c43       ?writeDefaultDevicetypesFile@alm_bncs_output@@AAEXXZ 1000ac43 f   alm_bncs_output.obj
 0001:0000a036       ?writeDevDescFile@alm_bncs_output@@AAEXQBVcOutputFile@@_N@Z 1000b036 f   alm_bncs_output.obj
 0001:0000a76f       ?writeDeviceTypesFile@alm_bncs_output@@AAE_NQBVcOutputFile@@@Z 1000b76f f   alm_bncs_output.obj
 0001:0000b23e       ?writeDomDoc@alm_bncs_output@@EBEXAAVQDomDocument@@ABVQString@@@Z 1000c23e f   alm_bncs_output.obj
 0001:0000b387       ?writeEmptyDevicetypesFile@alm_bncs_output@@AAEXABVQString@@@Z 1000c387 f   alm_bncs_output.obj
 0001:0000b556       ?writeEmptyInstancesFile@alm_bncs_output@@AAEXABVQString@@@Z 1000c556 f   alm_bncs_output.obj
 0001:0000b799       ?writeInstances@alm_bncs_output@@AAE_NXZ 1000c799 f   alm_bncs_output.obj
 0001:0000c316       ?writeNewInstanceFile@alm_bncs_output@@AAEXXZ 1000d316 f   alm_bncs_output.obj
 0001:0000ca57       ??0autoNumberDialog@@QAE@PAVQWidget@@PBD_NI@Z 1000da57 f   autonumberdialogimpl.obj
 0001:0000ca82       ??1autoNumberDialog@@UAE@XZ 1000da82 f   autonumberdialogimpl.obj
 0001:0000ca94       ??_EautoNumberDialog@@WCI@AEPAXI@Z 1000da94 f i autonumberdialogimpl.obj
 0001:0000ca9c       ??_EautoNumberDialog@@UAEPAXI@Z 1000da9c f i autonumberdialogimpl.obj
 0001:0000ca9c       ??_GautoNumberDialog@@UAEPAXI@Z 1000da9c f i autonumberdialogimpl.obj
 0001:0000cabb       ?metaObject@autoNumberDialog@@UBEPAVQMetaObject@@XZ 1000dabb f i autonumberdialogimpl.obj
 0001:0000cac0       ??0cOutputFile@@QAE@ABVQString@@00@Z 1000dac0 f   cOutputFile.obj
 0001:0000cb11       ??0cOutputFile@@QAE@XZ     1000db11 f   cOutputFile.obj
 0001:0000cb5d       ??1cOutputFile@@UAE@XZ     1000db5d f   cOutputFile.obj
 0001:0000cba4       ??_EcOutputFile@@UAEPAXI@Z 1000dba4 f i cOutputFile.obj
 0001:0000cba4       ??_GcOutputFile@@UAEPAXI@Z 1000dba4 f i cOutputFile.obj
 0001:0000cbc3       ??0TemplateList@@QAE@XZ    1000dbc3 f   devTemplate.obj
 0001:0000cbe2       ??0devTemplate@@QAE@ABVQString@@@Z 1000dbe2 f   devTemplate.obj
 0001:0000ce12       ??1?$QDict@VdevTemplate@@@@UAE@XZ 1000de12 f i devTemplate.obj
 0001:0000ce45       ??1TemplateList@@UAE@XZ    1000de45 f   devTemplate.obj
 0001:0000ce50       ??1devTemplate@@UAE@XZ     1000de50 f   devTemplate.obj
 0001:0000cea4       ??_E?$QDict@VdevTemplate@@@@UAEPAXI@Z 1000dea4 f i devTemplate.obj
 0001:0000cea4       ??_G?$QDict@VdevTemplate@@@@UAEPAXI@Z 1000dea4 f i devTemplate.obj
 0001:0000cec3       ??_ETemplateList@@UAEPAXI@Z 1000dec3 f i devTemplate.obj
 0001:0000cec3       ??_GTemplateList@@UAEPAXI@Z 1000dec3 f i devTemplate.obj
 0001:0000cee8       ?clear@?$QDict@VdevTemplate@@@@UAEXXZ 1000dee8 f i devTemplate.obj
 0001:0000ceee       ?getName@devTemplate@@QBE?AVQString@@XZ 1000deee f   devTemplate.obj
 0001:0000cf0c       ?loadDevDesc@devTemplate@@QAE_NABVQString@@0@Z 1000df0c f   devTemplate.obj
 0001:0000d2a2       ?saveFile@devTemplate@@QBE_NABVQString@@0QBVIDomDoc@@QAVIGetDocuments@@@Z 1000e2a2 f   devTemplate.obj
 0001:0000d683       ??$_Allocate@H@std@@YAPAHIPAH@Z 1000e683 f i dialogimpl.obj
 0001:0000d6b0       ??$_Fill_n@PAHIH@std@@YAPAHPAHIABH@Z 1000e6b0 f i dialogimpl.obj
 0001:0000d6d0       ??$_Uninit_move@PAHPAHU?$_Wrap_alloc@V?$allocator@H@std@@@std@@@std@@YAPAHPAH00AAU?$_Wrap_alloc@V?$allocator@H@std@@@0@@Z 1000e6d0 f i dialogimpl.obj
 0001:0000d6f2       ??0dialog@@QAE@PAVIGetDocuments@@PAVQWidget@@PBDI@Z 1000e6f2 f   dialogimpl.obj
 0001:0000dc6e       ??1?$vector@HV?$allocator@H@std@@@std@@QAE@XZ 1000ec6e f i dialogimpl.obj
 0001:0000dc73       ??1dialog@@UAE@XZ          1000ec73 f   dialogimpl.obj
 0001:0000dd05       ??_Edialog@@WCI@AEPAXI@Z   1000ed05 f i dialogimpl.obj
 0001:0000dd0d       ??_Edialog@@UAEPAXI@Z      1000ed0d f i dialogimpl.obj
 0001:0000dd0d       ??_Gdialog@@UAEPAXI@Z      1000ed0d f i dialogimpl.obj
 0001:0000dd2c       ?_Grow_to@?$vector@HV?$allocator@H@std@@@std@@IBEII@Z 1000ed2c f i dialogimpl.obj
 0001:0000dd59       ?_Reallocate@?$vector@HV?$allocator@H@std@@@std@@IAEXI@Z 1000ed59 f i dialogimpl.obj
 0001:0000ddaf       ?_Reserve@?$vector@HV?$allocator@H@std@@@std@@IAEXI@Z 1000edaf f i dialogimpl.obj
 0001:0000ddfa       ?_Tidy@?$vector@HV?$allocator@H@std@@@std@@IAEXXZ 1000edfa f i dialogimpl.obj
 0001:0000de19       ?autoNumber@dialog@@QAEXXZ 1000ee19 f   dialogimpl.obj
 0001:0000e1dd       ?changeSelection@dialog@@QAEXXZ 1000f1dd f   dialogimpl.obj
 0001:0000e2cc       ?checkForDuplicates@dialog@@QAE_NXZ 1000f2cc f   dialogimpl.obj
 0001:0000e4dd       ?clearAllSlots@dialog@@QAEXXZ 1000f4dd f   dialogimpl.obj
 0001:0000e5c5       ?clearSelectableSlots@dialog@@QAEXXZ 1000f5c5 f   dialogimpl.obj
 0001:0000e6c7       ?clearSelectedSlots@dialog@@QAEXXZ 1000f6c7 f   dialogimpl.obj
 0001:0000e7b9       ?clearSlots@dialog@@QAEXXZ 1000f7b9 f   dialogimpl.obj
 0001:0000e9a4       ?clipboardDataChange@dialog@@QAEXXZ 1000f9a4 f   dialogimpl.obj
 0001:0000eafc       ?copyData@dialog@@QAEXXZ   1000fafc f   dialogimpl.obj
 0001:0000ec35       ?itemChanged@dialog@@QAEXABVQString@@@Z 1000fc35 f   dialogimpl.obj
 0001:0000ec3d       ?itemDoubleClicked@dialog@@QAEXPAVQListViewItem@@@Z 1000fc3d f   dialogimpl.obj
 0001:0000ec62       ?metaObject@dialog@@UBEPAVQMetaObject@@XZ 1000fc62 f i dialogimpl.obj
 0001:0000ec67       ?moveProcDown@dialog@@QAEXXZ 1000fc67 f   dialogimpl.obj
 0001:0000ecda       ?moveProcUp@dialog@@QAEXXZ 1000fcda f   dialogimpl.obj
 0001:0000ed4d       ?pasteData@dialog@@QAEXXZ  1000fd4d f   dialogimpl.obj
 0001:0000f12a       ?reSort@dialog@@QAEXH@Z    1001012a f   dialogimpl.obj
 0001:0000f16b       ?resize@?$vector@HV?$allocator@H@std@@@std@@QAEXIABH@Z 1001016b f i dialogimpl.obj
 0001:0000f1f7       ?selectProc@dialog@@QAEXPAVQListViewItem@@@Z 100101f7 f   dialogimpl.obj
 0001:0000f274       ?setBncsSystemValues@dialog@@QAEXXZ 10010274 f   dialogimpl.obj
 0001:0000f2c0       ?slotChange@dialog@@QAEXPAVQListViewItem@@HABVQString@@@Z 100102c0 f   dialogimpl.obj
 0001:0000f427       ??0manage_tempBase@@QAE@PAVQWidget@@PBD_NI@Z 10010427 f   manage_temp.obj
 0001:000102e4       ??1manage_tempBase@@UAE@XZ 100112e4 f   manage_temp.obj
 0001:000102f7       ??_EQComboBox@@WCI@AEPAXI@Z 100112f7 f i manage_temp.obj
 0001:000102ff       ??_EQGridLayout@@WCI@AEPAXI@Z 100112ff f i manage_temp.obj
 0001:00010307       ??_EQHBoxLayout@@WCI@AEPAXI@Z 10011307 f i manage_temp.obj
 0001:0001030f       ??_EQLabel@@WCI@AEPAXI@Z   1001130f f i manage_temp.obj
 0001:00010317       ??_EQLineEdit@@WCI@AEPAXI@Z 10011317 f i manage_temp.obj
 0001:0001031f       ??_EQPushButton@@WCI@AEPAXI@Z 1001131f f i manage_temp.obj
 0001:00010327       ??_EQSpinBox@@WCI@AEPAXI@Z 10011327 f i manage_temp.obj
 0001:0001032f       ??_EQSpinBox@@WGM@AEPAXI@Z 1001132f f i manage_temp.obj
 0001:00010337       ??_EQTable@@WCI@AEPAXI@Z   10011337 f i manage_temp.obj
 0001:0001033f       ??_EQVBoxLayout@@WCI@AEPAXI@Z 1001133f f i manage_temp.obj
 0001:00010347       ??_Emanage_tempBase@@WCI@AEPAXI@Z 10011347 f i manage_temp.obj
 0001:0001034f       ??_GQComboBox@@UAEPAXI@Z   1001134f f i manage_temp.obj
 0001:0001034f       ??_EQComboBox@@UAEPAXI@Z   1001134f f i manage_temp.obj
 0001:0001036f       ??_EQGridLayout@@UAEPAXI@Z 1001136f f i manage_temp.obj
 0001:0001036f       ??_GQGridLayout@@UAEPAXI@Z 1001136f f i manage_temp.obj
 0001:0001038f       ??_EQHBoxLayout@@UAEPAXI@Z 1001138f f i manage_temp.obj
 0001:0001038f       ??_GQHBoxLayout@@UAEPAXI@Z 1001138f f i manage_temp.obj
 0001:000103af       ??_GQLabel@@UAEPAXI@Z      100113af f i manage_temp.obj
 0001:000103af       ??_EQLabel@@UAEPAXI@Z      100113af f i manage_temp.obj
 0001:000103cf       ??_GQLineEdit@@UAEPAXI@Z   100113cf f i manage_temp.obj
 0001:000103cf       ??_EQLineEdit@@UAEPAXI@Z   100113cf f i manage_temp.obj
 0001:000103ef       ??_GQPushButton@@UAEPAXI@Z 100113ef f i manage_temp.obj
 0001:000103ef       ??_EQPushButton@@UAEPAXI@Z 100113ef f i manage_temp.obj
 0001:0001040f       ??_EQSpacerItem@@UAEPAXI@Z 1001140f f i manage_temp.obj
 0001:0001040f       ??_GQSpacerItem@@UAEPAXI@Z 1001140f f i manage_temp.obj
 0001:0001042f       ??_GQSpinBox@@UAEPAXI@Z    1001142f f i manage_temp.obj
 0001:0001042f       ??_EQSpinBox@@UAEPAXI@Z    1001142f f i manage_temp.obj
 0001:0001044f       ??_GQTable@@UAEPAXI@Z      1001144f f i manage_temp.obj
 0001:0001044f       ??_EQTable@@UAEPAXI@Z      1001144f f i manage_temp.obj
 0001:0001046f       ??_GQVBoxLayout@@UAEPAXI@Z 1001146f f i manage_temp.obj
 0001:0001046f       ??_EQVBoxLayout@@UAEPAXI@Z 1001146f f i manage_temp.obj
 0001:0001048f       ??_Emanage_tempBase@@UAEPAXI@Z 1001148f f i manage_temp.obj
 0001:0001048f       ??_Gmanage_tempBase@@UAEPAXI@Z 1001148f f i manage_temp.obj
 0001:000104ae       ?languageChange@manage_tempBase@@MAEXXZ 100114ae f   manage_temp.obj
 0001:000109cf       ?metaObject@manage_tempBase@@UBEPAVQMetaObject@@XZ 100119cf f i manage_temp.obj
 0001:000109d4       ??0manage_temp@@QAE@ABVQStringList@@QBVTemplateList@@QAVIGetDocuments@@PAVQWidget@@PBD_NI@Z 100119d4 f   manage_tempimpl.obj
 0001:00010ce2       ??1manage_temp@@UAE@XZ     10011ce2 f   manage_tempimpl.obj
 0001:00010e42       ??4devTemplate@@QAEAAV0@ABV0@@Z 10011e42 f i manage_tempimpl.obj
 0001:00010e94       ??_Emanage_temp@@WCI@AEPAXI@Z 10011e94 f i manage_tempimpl.obj
 0001:00010e9c       ??_EQCheckTableItem@@UAEPAXI@Z 10011e9c f i manage_tempimpl.obj
 0001:00010e9c       ??_GQCheckTableItem@@UAEPAXI@Z 10011e9c f i manage_tempimpl.obj
 0001:00010ebc       ??_Emanage_temp@@UAEPAXI@Z 10011ebc f i manage_tempimpl.obj
 0001:00010ebc       ??_Gmanage_temp@@UAEPAXI@Z 10011ebc f i manage_tempimpl.obj
 0001:00010edb       ?autoNumberSlots@manage_temp@@QAEXXZ 10011edb f   manage_tempimpl.obj
 0001:00010fb6       ?changePrefix@manage_temp@@QAEXABVQString@@@Z 10011fb6 f   manage_tempimpl.obj
 0001:000111c2       ?changeTab@manage_temp@@QAEXPAVQWidget@@@Z 100121c2 f   manage_tempimpl.obj
 0001:000111e6       ?clearSlots@manage_temp@@QAEXXZ 100121e6 f   manage_tempimpl.obj
 0001:000112b2       ?getTemplates@manage_temp@@QAEXQAVTemplateList@@@Z 100122b2 f   manage_tempimpl.obj
 0001:0001136f       ?itemDoubleClicked@manage_temp@@QAEXPAVQListViewItem@@@Z 1001236f f   manage_tempimpl.obj
 0001:00011384       ?loadTemplates@manage_temp@@AAEXABVQStringList@@QBVTemplateList@@@Z 10012384 f   manage_tempimpl.obj
 0001:00011566       ?metaObject@manage_temp@@UBEPAVQMetaObject@@XZ 10012566 f i manage_tempimpl.obj
 0001:0001156b       ?newTemplate@manage_temp@@QAEXXZ 1001256b f   manage_tempimpl.obj
 0001:0001178d       ?saveCurrentTemplate@manage_temp@@QAEXXZ 1001278d f   manage_tempimpl.obj
 0001:0001193f       ?selectAllInstances@manage_temp@@QAEXXZ 1001293f f   manage_tempimpl.obj
 0001:00011949       ?selectSelectedInstances@manage_temp@@QAEXXZ 10012949 f   manage_tempimpl.obj
 0001:00011953       ?selectTemplate@manage_temp@@QAEXABVQString@@@Z 10012953 f   manage_tempimpl.obj
 0001:00011aa7       ?setSelection@manage_temp@@AAEX_N0@Z 10012aa7 f   manage_tempimpl.obj
 0001:00011b1f       ?slotChange@manage_temp@@QAEXPAVQListViewItem@@HABVQString@@@Z 10012b1f f   manage_tempimpl.obj
 0001:00011b22       ?unselectAllInstances@manage_temp@@QAEXXZ 10012b22 f   manage_tempimpl.obj
 0001:00011b2c       ?unselectSelectedInstances@manage_temp@@QAEXXZ 10012b2c f   manage_tempimpl.obj
 0001:00011b36       ?updateInstanceDisplay@manage_temp@@AAEXXZ 10012b36 f   manage_tempimpl.obj
 0001:00011ead       ?className@manage_tempBase@@UBEPBDXZ 10012ead f   moc_manage_temp.obj
 0001:00011eb3       ?qt_cast@manage_tempBase@@UAEPAXPBD@Z 10012eb3 f   moc_manage_temp.obj
 0001:00011ee1       ?qt_invoke@manage_tempBase@@UAE_NHPAUQUObject@@@Z 10012ee1 f   moc_manage_temp.obj
 0001:00011f13       ?qt_property@manage_tempBase@@UAE_NHHPAVQVariant@@@Z 10012f13 f   moc_manage_temp.obj
 0001:00011f13       ?qt_property@autoNumberDialogBase@@UAE_NHHPAVQVariant@@@Z 10012f13 f   moc_autonumberdialog.obj
 0001:00011f1d       ?staticMetaObject@manage_tempBase@@SAPAVQMetaObject@@XZ 10012f1d f   moc_manage_temp.obj
 0001:00011f67       ?tr@manage_tempBase@@SA?AVQString@@PBD0@Z 10012f67 f   moc_manage_temp.obj
 0001:00011faa       ?className@manage_temp@@UBEPBDXZ 10012faa f   moc_manage_tempimpl.obj
 0001:00011fb0       ?qt_cast@manage_temp@@UAEPAXPBD@Z 10012fb0 f   moc_manage_tempimpl.obj
 0001:00011fdd       ?qt_invoke@manage_temp@@UAE_NHPAUQUObject@@@Z 10012fdd f   moc_manage_tempimpl.obj
 0001:00012105       ?qt_property@manage_temp@@UAE_NHHPAVQVariant@@@Z 10013105 f   moc_manage_tempimpl.obj
 0001:00012105       ?qt_property@autoNumberDialog@@UAE_NHHPAVQVariant@@@Z 10013105 f   moc_autonumberdialogimpl.obj
 0001:0001210e       ?staticMetaObject@manage_temp@@SAPAVQMetaObject@@XZ 1001310e f   moc_manage_tempimpl.obj
 0001:0001227b       ??_Eplugindesc@@UAEPAXI@Z  1001327b f i plugindesc.obj
 0001:0001227b       ??_Gconfig_plugin_desc_base@@UAEPAXI@Z 1001327b f i plugindesc.obj
 0001:0001227b       ??_Econfig_plugin_desc_base@@UAEPAXI@Z 1001327b f i plugindesc.obj
 0001:0001227b       ??_Gplugindesc@@UAEPAXI@Z  1001327b f i plugindesc.obj
 0001:0001229b       ?create@plugindesc@@UAEPAVconfig_plugin_base@@ABVQString@@00@Z 1001329b f   plugindesc.obj
 0001:000122d6       ?keys@plugindesc@@UAE?AVQStringList@@ABVQString@@0@Z 100132d6 f   plugindesc.obj
 0001:00012331       ?pixmap@plugindesc@@UAE?AVQPixmap@@ABVQString@@@Z 10013331 f   plugindesc.obj
 0001:00012350       _load_bncs_config_plugin_desc 10013350 f   plugindesc.obj
 0001:00012366       ??0processItem@@QAE@PAVQListView@@VQString@@1@Z 10013366 f   processItem.obj
 0001:00012443       ??1processItem@@UAE@XZ     10013443 f   processItem.obj
 0001:0001244f       ??_GprocessItem@@UAEPAXI@Z 1001344f f i processItem.obj
 0001:0001244f       ??_EprocessItem@@UAEPAXI@Z 1001344f f i processItem.obj
 0001:0001246e       ?compare@processItem@@UBEHPAVQListViewItem@@H_N@Z 1001346e f   processItem.obj
 0001:00012590       ?paintCell@processItem@@UAEXPAVQPainter@@ABVQColorGroup@@HHH@Z 10013590 f   processItem.obj
 0001:0001262c       ??0autoNumberDialogBase@@QAE@PAVQWidget@@PBD_NI@Z 1001362c f   autonumberdialog.obj
 0001:00012d88       ??1autoNumberDialogBase@@UAE@XZ 10013d88 f   autonumberdialog.obj
 0001:00012d9b       ??_EQButtonGroup@@WCI@AEPAXI@Z 10013d9b f i autonumberdialog.obj
 0001:00012da3       ??_EQGroupBox@@WCI@AEPAXI@Z 10013da3 f i autonumberdialog.obj
 0001:00012dab       ??_EQRadioButton@@WCI@AEPAXI@Z 10013dab f i autonumberdialog.obj
 0001:00012db3       ??_EautoNumberDialogBase@@WCI@AEPAXI@Z 10013db3 f i autonumberdialog.obj
 0001:00012dbb       ??_EQButtonGroup@@UAEPAXI@Z 10013dbb f i autonumberdialog.obj
 0001:00012dbb       ??_GQButtonGroup@@UAEPAXI@Z 10013dbb f i autonumberdialog.obj
 0001:00012ddb       ??_GQGroupBox@@UAEPAXI@Z   10013ddb f i autonumberdialog.obj
 0001:00012ddb       ??_EQGroupBox@@UAEPAXI@Z   10013ddb f i autonumberdialog.obj
 0001:00012dfb       ??_GQRadioButton@@UAEPAXI@Z 10013dfb f i autonumberdialog.obj
 0001:00012dfb       ??_EQRadioButton@@UAEPAXI@Z 10013dfb f i autonumberdialog.obj
 0001:00012e1b       ??_EautoNumberDialogBase@@UAEPAXI@Z 10013e1b f i autonumberdialog.obj
 0001:00012e1b       ??_GautoNumberDialogBase@@UAEPAXI@Z 10013e1b f i autonumberdialog.obj
 0001:00012e3a       ?languageChange@autoNumberDialogBase@@MAEXXZ 10013e3a f   autonumberdialog.obj
 0001:00013100       ?metaObject@autoNumberDialogBase@@UBEPAVQMetaObject@@XZ 10014100 f i autonumberdialog.obj
 0001:00013105       ??0dialogBase@@QAE@PAVQWidget@@PBDI@Z 10014105 f   dialog.obj
 0001:00013ae9       ??1dialogBase@@UAE@XZ      10014ae9 f   dialog.obj
 0001:00013afc       ??_EdialogBase@@WCI@AEPAXI@Z 10014afc f i dialog.obj
 0001:00013b04       ??_GdialogBase@@UAEPAXI@Z  10014b04 f i dialog.obj
 0001:00013b04       ??_EdialogBase@@UAEPAXI@Z  10014b04 f i dialog.obj
 0001:00013b23       ?languageChange@dialogBase@@MAEXXZ 10014b23 f   dialog.obj
 0001:000142e3       ?metaObject@dialogBase@@UBEPAVQMetaObject@@XZ 100152e3 f i dialog.obj
 0001:000142e8       ?className@alm_bncs_output@@UBEPBDXZ 100152e8 f   moc_alm_bncs_output.obj
 0001:000142ee       ?command@alm_bncs_output@@IAEXVQString@@0@Z 100152ee f   moc_alm_bncs_output.obj
 0001:000143ae       ?qt_cast@alm_bncs_output@@UAEPAXPBD@Z 100153ae f   moc_alm_bncs_output.obj
 0001:00014435       ?qt_emit@alm_bncs_output@@UAE_NHPAUQUObject@@@Z 10015435 f   moc_alm_bncs_output.obj
 0001:00014499       ?qt_invoke@alm_bncs_output@@UAE_NHPAUQUObject@@@Z 10015499 f   moc_alm_bncs_output.obj
 0001:00014619       ?staticMetaObject@alm_bncs_output@@SAPAVQMetaObject@@XZ 10015619 f   moc_alm_bncs_output.obj
 0001:00014820       ?className@autoNumberDialogBase@@UBEPBDXZ 10015820 f   moc_autonumberdialog.obj
 0001:00014826       ?qt_cast@autoNumberDialogBase@@UAEPAXPBD@Z 10015826 f   moc_autonumberdialog.obj
 0001:00014854       ?qt_emit@autoNumberDialogBase@@UAE_NHPAUQUObject@@@Z 10015854 f   moc_autonumberdialog.obj
 0001:00014854       ?qt_emit@manage_tempBase@@UAE_NHPAUQUObject@@@Z 10015854 f   moc_manage_temp.obj
 0001:0001485e       ?qt_invoke@autoNumberDialogBase@@UAE_NHPAUQUObject@@@Z 1001585e f   moc_autonumberdialog.obj
 0001:00014890       ?staticMetaObject@autoNumberDialogBase@@SAPAVQMetaObject@@XZ 10015890 f   moc_autonumberdialog.obj
 0001:000148da       ?tr@autoNumberDialogBase@@SA?AVQString@@PBD0@Z 100158da f   moc_autonumberdialog.obj
 0001:0001491d       ?className@autoNumberDialog@@UBEPBDXZ 1001591d f   moc_autonumberdialogimpl.obj
 0001:00014923       ?qt_cast@autoNumberDialog@@UAEPAXPBD@Z 10015923 f   moc_autonumberdialogimpl.obj
 0001:00014950       ?qt_emit@autoNumberDialog@@UAE_NHPAUQUObject@@@Z 10015950 f   moc_autonumberdialogimpl.obj
 0001:00014950       ?qt_emit@manage_temp@@UAE_NHPAUQUObject@@@Z 10015950 f   moc_manage_tempimpl.obj
 0001:00014959       ?qt_invoke@autoNumberDialog@@UAE_NHPAUQUObject@@@Z 10015959 f   moc_autonumberdialogimpl.obj
 0001:00014962       ?staticMetaObject@autoNumberDialog@@SAPAVQMetaObject@@XZ 10015962 f   moc_autonumberdialogimpl.obj
 0001:000149a6       ?className@dialogBase@@UBEPBDXZ 100159a6 f   moc_dialog.obj
 0001:000149ac       ?qt_cast@dialogBase@@UAEPAXPBD@Z 100159ac f   moc_dialog.obj
 0001:000149da       ?qt_emit@dialogBase@@UAE_NHPAUQUObject@@@Z 100159da f   moc_dialog.obj
 0001:000149e4       ?qt_invoke@dialogBase@@UAE_NHPAUQUObject@@@Z 100159e4 f   moc_dialog.obj
 0001:00014a16       ?qt_property@dialogBase@@UAE_NHHPAVQVariant@@@Z 10015a16 f   moc_dialog.obj
 0001:00014a16       ?qt_property@alm_bncs_output@@UAE_NHHPAVQVariant@@@Z 10015a16 f   moc_alm_bncs_output.obj
 0001:00014a20       ?staticMetaObject@dialogBase@@SAPAVQMetaObject@@XZ 10015a20 f   moc_dialog.obj
 0001:00014a6a       ?tr@dialogBase@@SA?AVQString@@PBD0@Z 10015a6a f   moc_dialog.obj
 0001:00014aad       ?className@dialog@@UBEPBDXZ 10015aad f   moc_dialogimpl.obj
 0001:00014ab3       ?itemsChanged@dialog@@IAEXXZ 10015ab3 f   moc_dialogimpl.obj
 0001:00014ac8       ?qt_cast@dialog@@UAEPAXPBD@Z 10015ac8 f   moc_dialogimpl.obj
 0001:00014af5       ?qt_emit@dialog@@UAE_NHPAUQUObject@@@Z 10015af5 f   moc_dialogimpl.obj
 0001:00014b23       ?qt_invoke@dialog@@UAE_NHPAUQUObject@@@Z 10015b23 f   moc_dialogimpl.obj
 0001:00014cc7       ?qt_property@dialog@@UAE_NHHPAVQVariant@@@Z 10015cc7 f   moc_dialogimpl.obj
 0001:00014cd0       ?staticMetaObject@dialog@@SAPAVQMetaObject@@XZ 10015cd0 f   moc_dialogimpl.obj
 0001:00014e52       ?setName@QWidget@@UAEXPBD@Z 10015e52 f   qt-mt323:qt-mt323.dll
 0001:00014e58       ?acceptDrop@QListViewItem@@UBE_NPBVQMimeSource@@@Z 10015e58 f   qt-mt323:qt-mt323.dll
 0001:00014e5e       ?activate@QListViewItem@@MAEXXZ 10015e5e f   qt-mt323:qt-mt323.dll
 0001:00014e64       ?activateItemAt@QPopupMenu@@UAEXH@Z 10015e64 f   qt-mt323:qt-mt323.dll
 0001:00014e6a       ?addChild@QScrollView@@UAEXPAVQWidget@@HH@Z 10015e6a f   qt-mt323:qt-mt323.dll
 0001:00014e70       ?addColumn@QListView@@UAEHABVQIconSet@@ABVQString@@H@Z 10015e70 f   qt-mt323:qt-mt323.dll
 0001:00014e76       ?addColumn@QListView@@UAEHABVQString@@H@Z 10015e76 f   qt-mt323:qt-mt323.dll
 0001:00014e7c       ?addItem@QBoxLayout@@UAEXPAVQLayoutItem@@@Z 10015e7c f   qt-mt323:qt-mt323.dll
 0001:00014e82       ?addTab@QTabWidget@@UAEXPAVQWidget@@ABVQIconSet@@ABVQString@@@Z 10015e82 f   qt-mt323:qt-mt323.dll
 0001:00014e88       ?addTab@QTabWidget@@UAEXPAVQWidget@@ABVQString@@@Z 10015e88 f   qt-mt323:qt-mt323.dll
 0001:00014e8e       ?addTab@QTabWidget@@UAEXPAVQWidget@@PAVQTab@@@Z 10015e8e f   qt-mt323:qt-mt323.dll
 0001:00014e94       ?addTo@QAction@@UAE_NPAVQWidget@@@Z 10015e94 f   qt-mt323:qt-mt323.dll
 0001:00014e9a       ?addedTo@QAction@@MAEXHPAVQPopupMenu@@@Z 10015e9a f   qt-mt323:qt-mt323.dll
 0001:00014ea0       ?addedTo@QAction@@MAEXPAVQWidget@@0@Z 10015ea0 f   qt-mt323:qt-mt323.dll
 0001:00014ea6       ?adjustSize@QWidget@@UAEXXZ 10015ea6 f   qt-mt323:qt-mt323.dll
 0001:00014eac       ?cancelRename@QListViewItem@@MAEXH@Z 10015eac f   qt-mt323:qt-mt323.dll
 0001:00014eb2       ?checkConnectArgs@QObject@@MAE_NPBDPBV1@0@Z 10015eb2 f   qt-mt323:qt-mt323.dll
 0001:00014eb8       ?childEvent@QLayout@@MAEXPAVQChildEvent@@@Z 10015eb8 f   qt-mt323:qt-mt323.dll
 0001:00014ebe       ?childEvent@QObject@@MAEXPAVQChildEvent@@@Z 10015ebe f   qt-mt323:qt-mt323.dll
 0001:00014ec4       ?className@QAction@@UBEPBDXZ 10015ec4 f   qt-mt323:qt-mt323.dll
 0001:00014eca       ?className@QBoxLayout@@UBEPBDXZ 10015eca f   qt-mt323:qt-mt323.dll
 0001:00014ed0       ?className@QDockWindow@@UBEPBDXZ 10015ed0 f   qt-mt323:qt-mt323.dll
 0001:00014ed6       ?className@QGuardedPtrPrivate@@UBEPBDXZ 10015ed6 f   qt-mt323:qt-mt323.dll
 0001:00014edc       ?className@QListView@@UBEPBDXZ 10015edc f   qt-mt323:qt-mt323.dll
 0001:00014ee2       ?className@QPopupMenu@@UBEPBDXZ 10015ee2 f   qt-mt323:qt-mt323.dll
 0001:00014ee8       ?className@QTabWidget@@UBEPBDXZ 10015ee8 f   qt-mt323:qt-mt323.dll
 0001:00014eee       ?className@QToolBar@@UBEPBDXZ 10015eee f   qt-mt323:qt-mt323.dll
 0001:00014ef4       ?className@QWidget@@UBEPBDXZ 10015ef4 f   qt-mt323:qt-mt323.dll
 0001:00014efa       ?clear@?$QPtrList@VQDockWindow@@@@UAEXXZ 10015efa f   qt-mt323:qt-mt323.dll
 0001:00014f00       ?clear@QListView@@UAEXXZ   10015f00 f   qt-mt323:qt-mt323.dll
 0001:00014f06       ?clear@QToolBar@@UAEXXZ    10015f06 f   qt-mt323:qt-mt323.dll
 0001:00014f0c       ?clearSelection@QListView@@UAEXXZ 10015f0c f   qt-mt323:qt-mt323.dll
 0001:00014f12       ?close@QWidget@@UAE_N_N@Z  10015f12 f   qt-mt323:qt-mt323.dll
 0001:00014f18       ?closeEvent@QPopupMenu@@MAEXPAVQCloseEvent@@@Z 10015f18 f   qt-mt323:qt-mt323.dll
 0001:00014f1e       ?closeEvent@QWidget@@MAEXPAVQCloseEvent@@@Z 10015f1e f   qt-mt323:qt-mt323.dll
 0001:00014f24       ?cmd@QPaintDevice@@MAE_NHPAVQPainter@@PATQPDevCmdParam@@@Z 10015f24 f   qt-mt323:qt-mt323.dll
 0001:00014f2a       ?compare@QListViewItem@@UBEHPAV1@H_N@Z 10015f2a f   qt-mt323:qt-mt323.dll
 0001:00014f30       ?compareItems@QGList@@MAEHPAX0@Z 10015f30 f   qt-mt323:qt-mt323.dll
 0001:00014f36       ?connectNotify@QObject@@MAEXPBD@Z 10015f36 f   qt-mt323:qt-mt323.dll
 0001:00014f3c       ?contentsContextMenuEvent@QListView@@MAEXPAVQContextMenuEvent@@@Z 10015f3c f   qt-mt323:qt-mt323.dll
 0001:00014f42       ?contentsDragEnterEvent@QListView@@MAEXPAVQDragEnterEvent@@@Z 10015f42 f   qt-mt323:qt-mt323.dll
 0001:00014f48       ?contentsDragLeaveEvent@QListView@@MAEXPAVQDragLeaveEvent@@@Z 10015f48 f   qt-mt323:qt-mt323.dll
 0001:00014f4e       ?contentsDragMoveEvent@QListView@@MAEXPAVQDragMoveEvent@@@Z 10015f4e f   qt-mt323:qt-mt323.dll
 0001:00014f54       ?contentsDropEvent@QListView@@MAEXPAVQDropEvent@@@Z 10015f54 f   qt-mt323:qt-mt323.dll
 0001:00014f5a       ?contentsMouseDoubleClickEvent@QListView@@MAEXPAVQMouseEvent@@@Z 10015f5a f   qt-mt323:qt-mt323.dll
 0001:00014f60       ?contentsMouseMoveEvent@QListView@@MAEXPAVQMouseEvent@@@Z 10015f60 f   qt-mt323:qt-mt323.dll
 0001:00014f66       ?contentsMousePressEvent@QListView@@MAEXPAVQMouseEvent@@@Z 10015f66 f   qt-mt323:qt-mt323.dll
 0001:00014f6c       ?contentsMouseReleaseEvent@QListView@@MAEXPAVQMouseEvent@@@Z 10015f6c f   qt-mt323:qt-mt323.dll
 0001:00014f72       ?contentsWheelEvent@QScrollView@@MAEXPAVQWheelEvent@@@Z 10015f72 f   qt-mt323:qt-mt323.dll
 0001:00014f78       ?contextMenuEvent@QDockWindow@@MAEXPAVQContextMenuEvent@@@Z 10015f78 f   qt-mt323:qt-mt323.dll
 0001:00014f7e       ?contextMenuEvent@QScrollView@@MAEXPAVQContextMenuEvent@@@Z 10015f7e f   qt-mt323:qt-mt323.dll
 0001:00014f84       ?contextMenuEvent@QWidget@@MAEXPAVQContextMenuEvent@@@Z 10015f84 f   qt-mt323:qt-mt323.dll
 0001:00014f8a       ?count@?$QPtrList@VQDockWindow@@@@UBEIXZ 10015f8a f   qt-mt323:qt-mt323.dll
 0001:00014f90       ?create@QWidget@@MAEXPAUHWND__@@_N1@Z 10015f90 f   qt-mt323:qt-mt323.dll
 0001:00014f96       ?customEvent@QObject@@MAEXPAVQCustomEvent@@@Z 10015f96 f   qt-mt323:qt-mt323.dll
 0001:00014f9c       ?customWhatsThis@QPopupMenu@@UBE_NXZ 10015f9c f   qt-mt323:qt-mt323.dll
 0001:00014fa2       ?customWhatsThis@QWidget@@UBE_NXZ 10015fa2 f   qt-mt323:qt-mt323.dll
 0001:00014fa8       ?deleteItem@?$QPtrList@VQDockWindow@@@@EAEXPAX@Z 10015fa8 f   qt-mt323:qt-mt323.dll
 0001:00014fae       ?destroy@QWidget@@MAEX_N0@Z 10015fae f   qt-mt323:qt-mt323.dll
 0001:00014fb4       ?disconnectNotify@QObject@@MAEXPBD@Z 10015fb4 f   qt-mt323:qt-mt323.dll
 0001:00014fba       ?dock@QDockWindow@@UAEXXZ  10015fba f   qt-mt323:qt-mt323.dll
 0001:00014fc0       ?dragEnterEvent@QWidget@@MAEXPAVQDragEnterEvent@@@Z 10015fc0 f   qt-mt323:qt-mt323.dll
 0001:00014fc6       ?dragEntered@QListViewItem@@MAEXXZ 10015fc6 f   qt-mt323:qt-mt323.dll
 0001:00014fcc       ?dragLeaveEvent@QWidget@@MAEXPAVQDragLeaveEvent@@@Z 10015fcc f   qt-mt323:qt-mt323.dll
 0001:00014fd2       ?dragLeft@QListViewItem@@MAEXXZ 10015fd2 f   qt-mt323:qt-mt323.dll
 0001:00014fd8       ?dragMoveEvent@QWidget@@MAEXPAVQDragMoveEvent@@@Z 10015fd8 f   qt-mt323:qt-mt323.dll
 0001:00014fde       ?dragObject@QListView@@MAEPAVQDragObject@@XZ 10015fde f   qt-mt323:qt-mt323.dll
 0001:00014fe4       ?drawContents@QDockWindow@@MAEXPAVQPainter@@@Z 10015fe4 f   qt-mt323:qt-mt323.dll
 0001:00014fea       ?drawContents@QFrame@@MAEXPAVQPainter@@@Z 10015fea f   qt-mt323:qt-mt323.dll
 0001:00014ff0       ?drawContents@QPopupMenu@@MAEXPAVQPainter@@@Z 10015ff0 f   qt-mt323:qt-mt323.dll
 0001:00014ff6       ?drawContents@QScrollView@@EAEXPAVQPainter@@@Z 10015ff6 f   qt-mt323:qt-mt323.dll
 0001:00014ffe       ?drawContents@QScrollView@@MAEXPAVQPainter@@HHHH@Z 10015ffe f   qt-mt323:qt-mt323.dll
 0001:00015004       ?drawContentsOffset@QListView@@MAEXPAVQPainter@@HHHHHH@Z 10016004 f   qt-mt323:qt-mt323.dll
 0001:0001500a       ?drawFrame@QDockWindow@@MAEXPAVQPainter@@@Z 1001600a f   qt-mt323:qt-mt323.dll
 0001:00015010       ?drawFrame@QFrame@@MAEXPAVQPainter@@@Z 10016010 f   qt-mt323:qt-mt323.dll
 0001:00015016       ?dropEvent@QWidget@@MAEXPAVQDropEvent@@@Z 10016016 f   qt-mt323:qt-mt323.dll
 0001:0001501c       ?dropped@QListViewItem@@MAEXPAVQDropEvent@@@Z 1001601c f   qt-mt323:qt-mt323.dll
 0001:00015022       ?enabledChange@QPopupMenu@@MAEX_N@Z 10016022 f   qt-mt323:qt-mt323.dll
 0001:00015028       ?enabledChange@QWidget@@MAEX_N@Z 10016028 f   qt-mt323:qt-mt323.dll
 0001:0001502e       ?enforceSortOrder@QListViewItem@@MBEXXZ 1001602e f   qt-mt323:qt-mt323.dll
 0001:00015034       ?enterEvent@QWidget@@MAEXPAVQEvent@@@Z 10016034 f   qt-mt323:qt-mt323.dll
 0001:0001503a       ?event@QDockWindow@@MAE_NPAVQEvent@@@Z 1001603a f   qt-mt323:qt-mt323.dll
 0001:00015040       ?event@QObject@@UAE_NPAVQEvent@@@Z 10016040 f   qt-mt323:qt-mt323.dll
 0001:00015046       ?event@QToolBar@@UAE_NPAVQEvent@@@Z 10016046 f   qt-mt323:qt-mt323.dll
 0001:0001504c       ?event@QWidget@@MAE_NPAVQEvent@@@Z 1001604c f   qt-mt323:qt-mt323.dll
 0001:00015052       ?eventFilter@QDockWindow@@UAE_NPAVQObject@@PAVQEvent@@@Z 10016052 f   qt-mt323:qt-mt323.dll
 0001:00015058       ?eventFilter@QLayout@@MAE_NPAVQObject@@PAVQEvent@@@Z 10016058 f   qt-mt323:qt-mt323.dll
 0001:0001505e       ?eventFilter@QListView@@UAE_NPAVQObject@@PAVQEvent@@@Z 1001605e f   qt-mt323:qt-mt323.dll
 0001:00015064       ?eventFilter@QObject@@UAE_NPAV1@PAVQEvent@@@Z 10016064 f   qt-mt323:qt-mt323.dll
 0001:0001506a       ?eventFilter@QTabWidget@@MAE_NPAVQObject@@PAVQEvent@@@Z 1001606a f   qt-mt323:qt-mt323.dll
 0001:00015070       ?expanding@QBoxLayout@@UBE?AW4ExpandData@QSizePolicy@@XZ 10016070 f   qt-mt323:qt-mt323.dll
 0001:00015076       ?focusInEvent@QListView@@MAEXPAVQFocusEvent@@@Z 10016076 f   qt-mt323:qt-mt323.dll
 0001:0001507c       ?focusInEvent@QPopupMenu@@MAEXPAVQFocusEvent@@@Z 1001607c f   qt-mt323:qt-mt323.dll
 0001:00015082       ?focusInEvent@QWidget@@MAEXPAVQFocusEvent@@@Z 10016082 f   qt-mt323:qt-mt323.dll
 0001:00015088       ?focusNextPrevChild@QPopupMenu@@MAE_N_N@Z 10016088 f   qt-mt323:qt-mt323.dll
 0001:0001508e       ?focusNextPrevChild@QScrollView@@MAE_N_N@Z 1001608e f   qt-mt323:qt-mt323.dll
 0001:00015094       ?focusNextPrevChild@QWidget@@MAE_N_N@Z 10016094 f   qt-mt323:qt-mt323.dll
 0001:0001509a       ?focusOutEvent@QListView@@MAEXPAVQFocusEvent@@@Z 1001609a f   qt-mt323:qt-mt323.dll
 0001:000150a0       ?focusOutEvent@QPopupMenu@@MAEXPAVQFocusEvent@@@Z 100160a0 f   qt-mt323:qt-mt323.dll
 0001:000150a6       ?focusOutEvent@QWidget@@MAEXPAVQFocusEvent@@@Z 100160a6 f   qt-mt323:qt-mt323.dll
 0001:000150ac       ?fontChange@QScrollView@@MAEXABVQFont@@@Z 100160ac f   qt-mt323:qt-mt323.dll
 0001:000150b2       ?fontChange@QWidget@@MAEXABVQFont@@@Z 100160b2 f   qt-mt323:qt-mt323.dll
 0001:000150b8       ?fontInf@QPaintDevice@@MBEHPAVQFont@@H@Z 100160b8 f   qt-mt323:qt-mt323.dll
 0001:000150be       ?fontMet@QPaintDevice@@MBEHPAVQFont@@HPBDH@Z 100160be f   qt-mt323:qt-mt323.dll
 0001:000150c4       ?frameChanged@QFrame@@MAEXXZ 100160c4 f   qt-mt323:qt-mt323.dll
 0001:000150ca       ?frameChanged@QHBox@@MAEXXZ 100160ca f   qt-mt323:qt-mt323.dll
 0001:000150d0       ?frameChanged@QPopupMenu@@EAEXXZ 100160d0 f   qt-mt323:qt-mt323.dll
 0001:000150d6       ?frameChanged@QScrollView@@MAEXXZ 100160d6 f   qt-mt323:qt-mt323.dll
 0001:000150dc       ?geometry@QLayout@@UBE?AVQRect@@XZ 100160dc f   qt-mt323:qt-mt323.dll
 0001:000150e2       ?handle@QPaintDevice@@UBEPAUHDC__@@XZ 100160e2 f   qt-mt323:qt-mt323.dll
 0001:000150e8       ?hasHeightForWidth@QBoxLayout@@UBE_NXZ 100160e8 f   qt-mt323:qt-mt323.dll
 0001:000150ee       ?heightForWidth@QBoxLayout@@UBEHH@Z 100160ee f   qt-mt323:qt-mt323.dll
 0001:000150f4       ?heightForWidth@QWidget@@UBEHH@Z 100160f4 f   qt-mt323:qt-mt323.dll
 0001:000150fa       ?hide@QPopupMenu@@UAEXXZ   100160fa f   qt-mt323:qt-mt323.dll
 0001:00015100       ?hide@QToolBar@@UAEXXZ     10016100 f   qt-mt323:qt-mt323.dll
 0001:00015106       ?hide@QWidget@@UAEXXZ      10016106 f   qt-mt323:qt-mt323.dll
 0001:0001510c       ?hideEvent@QDockWindow@@MAEXPAVQHideEvent@@@Z 1001610c f   qt-mt323:qt-mt323.dll
 0001:00015112       ?hideEvent@QWidget@@MAEXPAVQHideEvent@@@Z 10016112 f   qt-mt323:qt-mt323.dll
 0001:00015118       ?imComposeEvent@QWidget@@MAEXPAVQIMEvent@@@Z 10016118 f   qt-mt323:qt-mt323.dll
 0001:0001511e       ?imEndEvent@QWidget@@MAEXPAVQIMEvent@@@Z 1001611e f   qt-mt323:qt-mt323.dll
 0001:00015124       ?imStartEvent@QWidget@@MAEXPAVQIMEvent@@@Z 10016124 f   qt-mt323:qt-mt323.dll
 0001:0001512a       ?insertChild@QObject@@UAEXPAV1@@Z 1001612a f   qt-mt323:qt-mt323.dll
 0001:00015130       ?insertItem@QListView@@UAEXPAVQListViewItem@@@Z 10016130 f   qt-mt323:qt-mt323.dll
 0001:00015136       ?insertItem@QListViewItem@@UAEXPAV1@@Z 10016136 f   qt-mt323:qt-mt323.dll
 0001:0001513c       ?insertTab@QTabWidget@@UAEXPAVQWidget@@ABVQIconSet@@ABVQString@@H@Z 1001613c f   qt-mt323:qt-mt323.dll
 0001:00015142       ?insertTab@QTabWidget@@UAEXPAVQWidget@@ABVQString@@H@Z 10016142 f   qt-mt323:qt-mt323.dll
 0001:00015148       ?insertTab@QTabWidget@@UAEXPAVQWidget@@PAVQTab@@H@Z 10016148 f   qt-mt323:qt-mt323.dll
 0001:0001514e       ?invalidate@QBoxLayout@@UAEXXZ 1001614e f   qt-mt323:qt-mt323.dll
 0001:00015154       ?invalidateHeight@QListViewItem@@UAEXXZ 10016154 f   qt-mt323:qt-mt323.dll
 0001:0001515a       ?invertSelection@QListView@@UAEXXZ 1001615a f   qt-mt323:qt-mt323.dll
 0001:00015160       ?isEmpty@QLayout@@UBE_NXZ  10016160 f   qt-mt323:qt-mt323.dll
 0001:00015166       ?iterator@QBoxLayout@@UAE?AVQLayoutIterator@@XZ 10016166 f   qt-mt323:qt-mt323.dll
 0001:0001516c       ?key@QListViewItem@@UBE?AVQString@@H_N@Z 1001616c f   qt-mt323:qt-mt323.dll
 0001:00015172       ?keyPressEvent@QListView@@MAEXPAVQKeyEvent@@@Z 10016172 f   qt-mt323:qt-mt323.dll
 0001:00015178       ?keyPressEvent@QPopupMenu@@MAEXPAVQKeyEvent@@@Z 10016178 f   qt-mt323:qt-mt323.dll
 0001:0001517e       ?keyPressEvent@QWidget@@MAEXPAVQKeyEvent@@@Z 1001617e f   qt-mt323:qt-mt323.dll
 0001:00015184       ?keyReleaseEvent@QWidget@@MAEXPAVQKeyEvent@@@Z 10016184 f   qt-mt323:qt-mt323.dll
 0001:0001518a       ?layout@QLayout@@UAEPAV1@XZ 1001618a f   qt-mt323:qt-mt323.dll
 0001:00015190       ?leaveEvent@QPopupMenu@@MAEXPAVQEvent@@@Z 10016190 f   qt-mt323:qt-mt323.dll
 0001:00015196       ?leaveEvent@QWidget@@MAEXPAVQEvent@@@Z 10016196 f   qt-mt323:qt-mt323.dll
 0001:0001519c       ?maximumSize@QBoxLayout@@UBE?AVQSize@@XZ 1001619c f   qt-mt323:qt-mt323.dll
 0001:000151a2       ?menuContentsChanged@QPopupMenu@@EAEXXZ 100161a2 f   qt-mt323:qt-mt323.dll
 0001:000151a8       ?menuDelPopup@QPopupMenu@@EAEXPAV1@@Z 100161a8 f   qt-mt323:qt-mt323.dll
 0001:000151ae       ?menuInsPopup@QPopupMenu@@EAEXPAV1@@Z 100161ae f   qt-mt323:qt-mt323.dll
 0001:000151b4       ?menuStateChanged@QPopupMenu@@EAEXXZ 100161b4 f   qt-mt323:qt-mt323.dll
 0001:000151ba       ?metaObject@QAction@@UBEPAVQMetaObject@@XZ 100161ba f   qt-mt323:qt-mt323.dll
 0001:000151c0       ?metaObject@QBoxLayout@@UBEPAVQMetaObject@@XZ 100161c0 f   qt-mt323:qt-mt323.dll
 0001:000151c6       ?metaObject@QDockWindow@@UBEPAVQMetaObject@@XZ 100161c6 f   qt-mt323:qt-mt323.dll
 0001:000151cc       ?metaObject@QGuardedPtrPrivate@@UBEPAVQMetaObject@@XZ 100161cc f   qt-mt323:qt-mt323.dll
 0001:000151d2       ?metaObject@QListView@@UBEPAVQMetaObject@@XZ 100161d2 f   qt-mt323:qt-mt323.dll
 0001:000151d8       ?metaObject@QPopupMenu@@UBEPAVQMetaObject@@XZ 100161d8 f   qt-mt323:qt-mt323.dll
 0001:000151de       ?metaObject@QTabWidget@@UBEPAVQMetaObject@@XZ 100161de f   qt-mt323:qt-mt323.dll
 0001:000151e4       ?metaObject@QToolBar@@UBEPAVQMetaObject@@XZ 100161e4 f   qt-mt323:qt-mt323.dll
 0001:000151ea       ?metaObject@QWidget@@UBEPAVQMetaObject@@XZ 100161ea f   qt-mt323:qt-mt323.dll
 0001:000151f0       ?metric@QWidget@@MBEHH@Z   100161f0 f   qt-mt323:qt-mt323.dll
 0001:000151f6       ?minimumSize@QBoxLayout@@UBE?AVQSize@@XZ 100161f6 f   qt-mt323:qt-mt323.dll
 0001:000151fc       ?minimumSizeHint@QDockWindow@@UBE?AVQSize@@XZ 100161fc f   qt-mt323:qt-mt323.dll
 0001:00015202       ?minimumSizeHint@QListView@@UBE?AVQSize@@XZ 10016202 f   qt-mt323:qt-mt323.dll
 0001:00015208       ?minimumSizeHint@QTabWidget@@UBE?AVQSize@@XZ 10016208 f   qt-mt323:qt-mt323.dll
 0001:0001520e       ?minimumSizeHint@QToolBar@@UBE?AVQSize@@XZ 1001620e f   qt-mt323:qt-mt323.dll
 0001:00015214       ?minimumSizeHint@QWidget@@UBE?AVQSize@@XZ 10016214 f   qt-mt323:qt-mt323.dll
 0001:0001521a       ?mouseDoubleClickEvent@QScrollView@@MAEXPAVQMouseEvent@@@Z 1001621a f   qt-mt323:qt-mt323.dll
 0001:00015220       ?mouseDoubleClickEvent@QWidget@@MAEXPAVQMouseEvent@@@Z 10016220 f   qt-mt323:qt-mt323.dll
 0001:00015226       ?mouseMoveEvent@QPopupMenu@@MAEXPAVQMouseEvent@@@Z 10016226 f   qt-mt323:qt-mt323.dll
 0001:0001522c       ?mouseMoveEvent@QScrollView@@MAEXPAVQMouseEvent@@@Z 1001622c f   qt-mt323:qt-mt323.dll
 0001:00015232       ?mouseMoveEvent@QWidget@@MAEXPAVQMouseEvent@@@Z 10016232 f   qt-mt323:qt-mt323.dll
 0001:00015238       ?mousePressEvent@QPopupMenu@@MAEXPAVQMouseEvent@@@Z 10016238 f   qt-mt323:qt-mt323.dll
 0001:0001523e       ?mousePressEvent@QScrollView@@MAEXPAVQMouseEvent@@@Z 1001623e f   qt-mt323:qt-mt323.dll
 0001:00015244       ?mousePressEvent@QWidget@@MAEXPAVQMouseEvent@@@Z 10016244 f   qt-mt323:qt-mt323.dll
 0001:0001524a       ?mouseReleaseEvent@QPopupMenu@@MAEXPAVQMouseEvent@@@Z 1001624a f   qt-mt323:qt-mt323.dll
 0001:00015250       ?mouseReleaseEvent@QScrollView@@MAEXPAVQMouseEvent@@@Z 10016250 f   qt-mt323:qt-mt323.dll
 0001:00015256       ?mouseReleaseEvent@QWidget@@MAEXPAVQMouseEvent@@@Z 10016256 f   qt-mt323:qt-mt323.dll
 0001:0001525c       ?move@QWidget@@UAEXHH@Z    1001625c f   qt-mt323:qt-mt323.dll
 0001:00015262       ?moveChild@QScrollView@@UAEXPAVQWidget@@HH@Z 10016262 f   qt-mt323:qt-mt323.dll
 0001:00015268       ?moveEvent@QWidget@@MAEXPAVQMoveEvent@@@Z 10016268 f   qt-mt323:qt-mt323.dll
 0001:0001526e       ?newItem@QPtrCollection@@MAEPAXPAX@Z 1001626e f   qt-mt323:qt-mt323.dll
 0001:00015274       ?okRename@QListViewItem@@MAEXH@Z 10016274 f   qt-mt323:qt-mt323.dll
 0001:0001527a       ?paintBranches@QListViewItem@@UAEXPAVQPainter@@ABVQColorGroup@@HHH@Z 1001627a f   qt-mt323:qt-mt323.dll
 0001:00015280       ?paintCell@QListViewItem@@UAEXPAVQPainter@@ABVQColorGroup@@HHH@Z 10016280 f   qt-mt323:qt-mt323.dll
 0001:00015286       ?paintEmptyArea@QListView@@MAEXPAVQPainter@@ABVQRect@@@Z 10016286 f   qt-mt323:qt-mt323.dll
 0001:0001528c       ?paintEvent@QFrame@@MAEXPAVQPaintEvent@@@Z 1001628c f   qt-mt323:qt-mt323.dll
 0001:00015292       ?paintEvent@QPopupMenu@@MAEXPAVQPaintEvent@@@Z 10016292 f   qt-mt323:qt-mt323.dll
 0001:00015298       ?paintEvent@QWidget@@MAEXPAVQPaintEvent@@@Z 10016298 f   qt-mt323:qt-mt323.dll
 0001:0001529e       ?paintFocus@QListViewItem@@UAEXPAVQPainter@@ABVQColorGroup@@ABVQRect@@@Z 1001629e f   qt-mt323:qt-mt323.dll
 0001:000152a4       ?paletteChange@QWidget@@MAEXABVQPalette@@@Z 100162a4 f   qt-mt323:qt-mt323.dll
 0001:000152aa       ?pixmap@QListViewItem@@UBEPBVQPixmap@@H@Z 100162aa f   qt-mt323:qt-mt323.dll
 0001:000152b0       ?polish@QWidget@@UAEXXZ    100162b0 f   qt-mt323:qt-mt323.dll
 0001:000152b6       ?property@QObject@@UBE?AVQVariant@@PBD@Z 100162b6 f   qt-mt323:qt-mt323.dll
 0001:000152bc       ?qt_cast@QAction@@UAEPAXPBD@Z 100162bc f   qt-mt323:qt-mt323.dll
 0001:000152c2       ?qt_cast@QBoxLayout@@UAEPAXPBD@Z 100162c2 f   qt-mt323:qt-mt323.dll
 0001:000152c8       ?qt_cast@QDockWindow@@UAEPAXPBD@Z 100162c8 f   qt-mt323:qt-mt323.dll
 0001:000152ce       ?qt_cast@QGuardedPtrPrivate@@UAEPAXPBD@Z 100162ce f   qt-mt323:qt-mt323.dll
 0001:000152d4       ?qt_cast@QListView@@UAEPAXPBD@Z 100162d4 f   qt-mt323:qt-mt323.dll
 0001:000152da       ?qt_cast@QPopupMenu@@UAEPAXPBD@Z 100162da f   qt-mt323:qt-mt323.dll
 0001:000152e0       ?qt_cast@QTabWidget@@UAEPAXPBD@Z 100162e0 f   qt-mt323:qt-mt323.dll
 0001:000152e6       ?qt_cast@QToolBar@@UAEPAXPBD@Z 100162e6 f   qt-mt323:qt-mt323.dll
 0001:000152ec       ?qt_cast@QWidget@@UAEPAXPBD@Z 100162ec f   qt-mt323:qt-mt323.dll
 0001:000152f2       ?qt_emit@QAction@@UAE_NHPAUQUObject@@@Z 100162f2 f   qt-mt323:qt-mt323.dll
 0001:000152f8       ?qt_emit@QBoxLayout@@UAE_NHPAUQUObject@@@Z 100162f8 f   qt-mt323:qt-mt323.dll
 0001:000152fe       ?qt_emit@QDockWindow@@UAE_NHPAUQUObject@@@Z 100162fe f   qt-mt323:qt-mt323.dll
 0001:00015304       ?qt_emit@QGuardedPtrPrivate@@UAE_NHPAUQUObject@@@Z 10016304 f   qt-mt323:qt-mt323.dll
 0001:0001530a       ?qt_emit@QListView@@UAE_NHPAUQUObject@@@Z 1001630a f   qt-mt323:qt-mt323.dll
 0001:00015310       ?qt_emit@QPopupMenu@@UAE_NHPAUQUObject@@@Z 10016310 f   qt-mt323:qt-mt323.dll
 0001:00015316       ?qt_emit@QTabWidget@@UAE_NHPAUQUObject@@@Z 10016316 f   qt-mt323:qt-mt323.dll
 0001:0001531c       ?qt_emit@QToolBar@@UAE_NHPAUQUObject@@@Z 1001631c f   qt-mt323:qt-mt323.dll
 0001:00015322       ?qt_emit@QWidget@@UAE_NHPAUQUObject@@@Z 10016322 f   qt-mt323:qt-mt323.dll
 0001:00015328       ?qt_invoke@QAction@@UAE_NHPAUQUObject@@@Z 10016328 f   qt-mt323:qt-mt323.dll
 0001:0001532e       ?qt_invoke@QBoxLayout@@UAE_NHPAUQUObject@@@Z 1001632e f   qt-mt323:qt-mt323.dll
 0001:00015334       ?qt_invoke@QDockWindow@@UAE_NHPAUQUObject@@@Z 10016334 f   qt-mt323:qt-mt323.dll
 0001:0001533a       ?qt_invoke@QGuardedPtrPrivate@@UAE_NHPAUQUObject@@@Z 1001633a f   qt-mt323:qt-mt323.dll
 0001:00015340       ?qt_invoke@QListView@@UAE_NHPAUQUObject@@@Z 10016340 f   qt-mt323:qt-mt323.dll
 0001:00015346       ?qt_invoke@QPopupMenu@@UAE_NHPAUQUObject@@@Z 10016346 f   qt-mt323:qt-mt323.dll
 0001:0001534c       ?qt_invoke@QTabWidget@@UAE_NHPAUQUObject@@@Z 1001634c f   qt-mt323:qt-mt323.dll
 0001:00015352       ?qt_invoke@QToolBar@@UAE_NHPAUQUObject@@@Z 10016352 f   qt-mt323:qt-mt323.dll
 0001:00015358       ?qt_invoke@QWidget@@UAE_NHPAUQUObject@@@Z 10016358 f   qt-mt323:qt-mt323.dll
 0001:0001535e       ?qt_property@QAction@@UAE_NHHPAVQVariant@@@Z 1001635e f   qt-mt323:qt-mt323.dll
 0001:00015364       ?qt_property@QBoxLayout@@UAE_NHHPAVQVariant@@@Z 10016364 f   qt-mt323:qt-mt323.dll
 0001:0001536a       ?qt_property@QDockWindow@@UAE_NHHPAVQVariant@@@Z 1001636a f   qt-mt323:qt-mt323.dll
 0001:00015370       ?qt_property@QGuardedPtrPrivate@@UAE_NHHPAVQVariant@@@Z 10016370 f   qt-mt323:qt-mt323.dll
 0001:00015376       ?qt_property@QListView@@UAE_NHHPAVQVariant@@@Z 10016376 f   qt-mt323:qt-mt323.dll
 0001:0001537c       ?qt_property@QPopupMenu@@UAE_NHHPAVQVariant@@@Z 1001637c f   qt-mt323:qt-mt323.dll
 0001:00015382       ?qt_property@QTabWidget@@UAE_NHHPAVQVariant@@@Z 10016382 f   qt-mt323:qt-mt323.dll
 0001:00015388       ?qt_property@QToolBar@@UAE_NHHPAVQVariant@@@Z 10016388 f   qt-mt323:qt-mt323.dll
 0001:0001538e       ?qt_property@QWidget@@UAE_NHHPAVQVariant@@@Z 1001638e f   qt-mt323:qt-mt323.dll
 0001:00015394       ?read@QGList@@MAEAAVQDataStream@@AAV2@AAPAX@Z 10016394 f   qt-mt323:qt-mt323.dll
 0001:0001539a       ?removeChild@QObject@@UAEXPAV1@@Z 1001639a f   qt-mt323:qt-mt323.dll
 0001:000153a0       ?removeChild@QScrollView@@UAEXPAVQObject@@@Z 100163a0 f   qt-mt323:qt-mt323.dll
 0001:000153a6       ?removeColumn@QListView@@UAEXH@Z 100163a6 f   qt-mt323:qt-mt323.dll
 0001:000153ac       ?removeFrom@QAction@@UAE_NPAVQWidget@@@Z 100163ac f   qt-mt323:qt-mt323.dll
 0001:000153b2       ?removeItem@QListView@@UAEXPAVQListViewItem@@@Z 100163b2 f   qt-mt323:qt-mt323.dll
 0001:000153b8       ?removeItem@QListViewItem@@UAEXPAV1@@Z 100163b8 f   qt-mt323:qt-mt323.dll
 0001:000153be       ?removePage@QTabWidget@@UAEXPAVQWidget@@@Z 100163be f   qt-mt323:qt-mt323.dll
 0001:000153c4       ?reparent@QWidget@@UAEXPAV1@IABVQPoint@@_N@Z 100163c4 f   qt-mt323:qt-mt323.dll
 0001:000153ca       ?resize@QScrollView@@UAEXHH@Z 100163ca f   qt-mt323:qt-mt323.dll
 0001:000153d0       ?resize@QWidget@@UAEXHH@Z  100163d0 f   qt-mt323:qt-mt323.dll
 0001:000153d6       ?resizeContents@QScrollView@@UAEXHH@Z 100163d6 f   qt-mt323:qt-mt323.dll
 0001:000153dc       ?resizeEvent@QDockWindow@@MAEXPAVQResizeEvent@@@Z 100163dc f   qt-mt323:qt-mt323.dll
 0001:000153e2       ?resizeEvent@QFrame@@MAEXPAVQResizeEvent@@@Z 100163e2 f   qt-mt323:qt-mt323.dll
 0001:000153e8       ?resizeEvent@QListView@@MAEXPAVQResizeEvent@@@Z 100163e8 f   qt-mt323:qt-mt323.dll
 0001:000153ee       ?resizeEvent@QTabWidget@@MAEXPAVQResizeEvent@@@Z 100163ee f   qt-mt323:qt-mt323.dll
 0001:000153f4       ?resizeEvent@QToolBar@@MAEXPAVQResizeEvent@@@Z 100163f4 f   qt-mt323:qt-mt323.dll
 0001:000153fa       ?resizeEvent@QWidget@@MAEXPAVQResizeEvent@@@Z 100163fa f   qt-mt323:qt-mt323.dll
 0001:00015400       ?resolution@QPaintDevice@@UBEHXZ 10016400 f   qt-mt323:qt-mt323.dll
 0001:00015406       ?rtti@QListViewItem@@UBEHXZ 10016406 f   qt-mt323:qt-mt323.dll
 0001:0001540c       ?selectAll@QListView@@UAEX_N@Z 1001640c f   qt-mt323:qt-mt323.dll
 0001:00015412       ?setAccel@QAction@@UAEXABVQKeySequence@@@Z 10016412 f   qt-mt323:qt-mt323.dll
 0001:00015418       ?setAcceptDrops@QWidget@@UAEX_N@Z 10016418 f   qt-mt323:qt-mt323.dll
 0001:0001541e       ?setActiveItem@QPopupMenu@@UAEXH@Z 1001641e f   qt-mt323:qt-mt323.dll
 0001:00015424       ?setActiveWindow@QWidget@@UAEXXZ 10016424 f   qt-mt323:qt-mt323.dll
 0001:0001542a       ?setAlignment@QLayoutItem@@UAEXH@Z 1001642a f   qt-mt323:qt-mt323.dll
 0001:00015430       ?setAllColumnsShowFocus@QListView@@UAEX_N@Z 10016430 f   qt-mt323:qt-mt323.dll
 0001:00015436       ?setAutoAdd@QLayout@@UAEX_N@Z 10016436 f   qt-mt323:qt-mt323.dll
 0001:0001543c       ?setAutoMask@QWidget@@UAEX_N@Z 1001643c f   qt-mt323:qt-mt323.dll
 0001:00015442       ?setBackgroundColor@QWidget@@UAEXABVQColor@@@Z 10016442 f   qt-mt323:qt-mt323.dll
 0001:00015448       ?setBackgroundMode@QWidget@@UAEXW4BackgroundMode@Qt@@@Z 10016448 f   qt-mt323:qt-mt323.dll
 0001:0001544e       ?setBackgroundOrigin@QWidget@@UAEXW4BackgroundOrigin@1@@Z 1001644e f   qt-mt323:qt-mt323.dll
 0001:00015454       ?setBackgroundPixmap@QWidget@@UAEXABVQPixmap@@@Z 10016454 f   qt-mt323:qt-mt323.dll
 0001:0001545a       ?setCaption@QDockWindow@@UAEXABVQString@@@Z 1001645a f   qt-mt323:qt-mt323.dll
 0001:00015460       ?setCaption@QWidget@@UAEXABVQString@@@Z 10016460 f   qt-mt323:qt-mt323.dll
 0001:00015466       ?setCheckable@QPopupMenu@@UAEX_N@Z 10016466 f   qt-mt323:qt-mt323.dll
 0001:0001546c       ?setCloseMode@QDockWindow@@UAEXH@Z 1001646c f   qt-mt323:qt-mt323.dll
 0001:00015472       ?setColumnAlignment@QListView@@UAEXHH@Z 10016472 f   qt-mt323:qt-mt323.dll
 0001:00015478       ?setColumnText@QListView@@UAEXHABVQIconSet@@ABVQString@@@Z 10016478 f   qt-mt323:qt-mt323.dll
 0001:0001547e       ?setColumnText@QListView@@UAEXHABVQString@@@Z 1001647e f   qt-mt323:qt-mt323.dll
 0001:00015484       ?setColumnWidth@QListView@@UAEXHH@Z 10016484 f   qt-mt323:qt-mt323.dll
 0001:0001548a       ?setColumnWidthMode@QListView@@UAEXHW4WidthMode@1@@Z 1001648a f   qt-mt323:qt-mt323.dll
 0001:00015490       ?setContentsPos@QListView@@UAEXHH@Z 10016490 f   qt-mt323:qt-mt323.dll
 0001:00015496       ?setCornerWidget@QScrollView@@UAEXPAVQWidget@@@Z 10016496 f   qt-mt323:qt-mt323.dll
 0001:0001549c       ?setCurrentItem@QListView@@UAEXPAVQListViewItem@@@Z 1001649c f   qt-mt323:qt-mt323.dll
 0001:000154a2       ?setCursor@QWidget@@UAEXABVQCursor@@@Z 100164a2 f   qt-mt323:qt-mt323.dll
 0001:000154a8       ?setDefaultRenameAction@QListView@@UAEXW4RenameAction@1@@Z 100164a8 f   qt-mt323:qt-mt323.dll
 0001:000154ae       ?setDragAutoScroll@QScrollView@@UAEX_N@Z 100164ae f   qt-mt323:qt-mt323.dll
 0001:000154b4       ?setDragEnabled@QListViewItem@@UAEX_N@Z 100164b4 f   qt-mt323:qt-mt323.dll
 0001:000154ba       ?setDropEnabled@QListViewItem@@UAEX_N@Z 100164ba f   qt-mt323:qt-mt323.dll
 0001:000154c0       ?setEnabled@QAction@@UAEX_N@Z 100164c0 f   qt-mt323:qt-mt323.dll
 0001:000154c6       ?setEnabled@QListViewItem@@UAEX_N@Z 100164c6 f   qt-mt323:qt-mt323.dll
 0001:000154cc       ?setEnabled@QScrollView@@UAEX_N@Z 100164cc f   qt-mt323:qt-mt323.dll
 0001:000154d2       ?setEnabled@QWidget@@UAEX_N@Z 100164d2 f   qt-mt323:qt-mt323.dll
 0001:000154d8       ?setEraseColor@QWidget@@UAEXABVQColor@@@Z 100164d8 f   qt-mt323:qt-mt323.dll
 0001:000154de       ?setErasePixmap@QWidget@@UAEXABVQPixmap@@@Z 100164de f   qt-mt323:qt-mt323.dll
 0001:000154e4       ?setExpandable@QListViewItem@@UAEX_N@Z 100164e4 f   qt-mt323:qt-mt323.dll
 0001:000154ea       ?setFirstItemActive@QPopupMenu@@EAEXXZ 100164ea f   qt-mt323:qt-mt323.dll
 0001:000154f0       ?setFixedExtentHeight@QDockWindow@@UAEXH@Z 100164f0 f   qt-mt323:qt-mt323.dll
 0001:000154f6       ?setFixedExtentWidth@QDockWindow@@UAEXH@Z 100164f6 f   qt-mt323:qt-mt323.dll
 0001:000154fc       ?setFocus@QWidget@@UAEXXZ  100164fc f   qt-mt323:qt-mt323.dll
 0001:00015502       ?setFocusPolicy@QWidget@@UAEXW4FocusPolicy@1@@Z 10016502 f   qt-mt323:qt-mt323.dll
 0001:00015508       ?setFocusProxy@QWidget@@UAEXPAV1@@Z 10016508 f   qt-mt323:qt-mt323.dll
 0001:0001550e       ?setFont@QListView@@UAEXABVQFont@@@Z 1001650e f   qt-mt323:qt-mt323.dll
 0001:00015514       ?setFont@QPopupMenu@@UAEXABVQFont@@@Z 10016514 f   qt-mt323:qt-mt323.dll
 0001:0001551a       ?setFont@QWidget@@UAEXABVQFont@@@Z 1001651a f   qt-mt323:qt-mt323.dll
 0001:00015520       ?setFrameRect@QFrame@@UAEXABVQRect@@@Z 10016520 f   qt-mt323:qt-mt323.dll
 0001:00015526       ?setFrameStyle@QFrame@@UAEXH@Z 10016526 f   qt-mt323:qt-mt323.dll
 0001:0001552c       ?setGeometry@QBoxLayout@@UAEXABVQRect@@@Z 1001652c f   qt-mt323:qt-mt323.dll
 0001:00015532       ?setGeometry@QWidget@@UAEXABVQRect@@@Z 10016532 f   qt-mt323:qt-mt323.dll
 0001:00015538       ?setGeometry@QWidget@@UAEXHHHH@Z 10016538 f   qt-mt323:qt-mt323.dll
 0001:0001553e       ?setHBarGeometry@QScrollView@@MAEXAAVQScrollBar@@HHHH@Z 1001653e f   qt-mt323:qt-mt323.dll
 0001:00015544       ?setHScrollBarMode@QScrollView@@UAEXW4ScrollBarMode@1@@Z 10016544 f   qt-mt323:qt-mt323.dll
 0001:0001554a       ?setHeight@QListViewItem@@MAEXH@Z 1001654a f   qt-mt323:qt-mt323.dll
 0001:00015550       ?setHorizontallyStretchable@QDockWindow@@UAEX_N@Z 10016550 f   qt-mt323:qt-mt323.dll
 0001:00015556       ?setIcon@QWidget@@UAEXABVQPixmap@@@Z 10016556 f   qt-mt323:qt-mt323.dll
 0001:0001555c       ?setIconSet@QAction@@UAEXABVQIconSet@@@Z 1001655c f   qt-mt323:qt-mt323.dll
 0001:00015562       ?setIconText@QWidget@@UAEXABVQString@@@Z 10016562 f   qt-mt323:qt-mt323.dll
 0001:00015568       ?setId@QMenuData@@UAEXHH@Z 10016568 f   qt-mt323:qt-mt323.dll
 0001:0001556e       ?setItemMargin@QListView@@UAEXH@Z 1001656e f   qt-mt323:qt-mt323.dll
 0001:00015574       ?setKeyCompression@QWidget@@MAEX_N@Z 10016574 f   qt-mt323:qt-mt323.dll
 0001:0001557a       ?setLabel@QToolBar@@UAEXABVQString@@@Z 1001657a f   qt-mt323:qt-mt323.dll
 0001:00015580       ?setLineWidth@QFrame@@UAEXH@Z 10016580 f   qt-mt323:qt-mt323.dll
 0001:00015586       ?setMargin@QFrame@@UAEXH@Z 10016586 f   qt-mt323:qt-mt323.dll
 0001:0001558c       ?setMargin@QLayout@@UAEXH@Z 1001658c f   qt-mt323:qt-mt323.dll
 0001:00015592       ?setMargins@QScrollView@@MAEXHHHH@Z 10016592 f   qt-mt323:qt-mt323.dll
 0001:00015598       ?setMask@QWidget@@UAEXABVQBitmap@@@Z 10016598 f   qt-mt323:qt-mt323.dll
 0001:0001559e       ?setMask@QWidget@@UAEXABVQRegion@@@Z 1001659e f   qt-mt323:qt-mt323.dll
 0001:000155a4       ?setMaximumSize@QWidget@@UAEXHH@Z 100165a4 f   qt-mt323:qt-mt323.dll
 0001:000155aa       ?setMenuBar@QLayout@@UAEXPAVQMenuBar@@@Z 100165aa f   qt-mt323:qt-mt323.dll
 0001:000155b0       ?setMenuText@QAction@@UAEXABVQString@@@Z 100165b0 f   qt-mt323:qt-mt323.dll
 0001:000155b6       ?setMicroFocusHint@QWidget@@MAEXHHHH_NPAVQFont@@@Z 100165b6 f   qt-mt323:qt-mt323.dll
 0001:000155bc       ?setMidLineWidth@QFrame@@UAEXH@Z 100165bc f   qt-mt323:qt-mt323.dll
 0001:000155c2       ?setMinimumSize@QToolBar@@UAEXHH@Z 100165c2 f   qt-mt323:qt-mt323.dll
 0001:000155c8       ?setMinimumSize@QWidget@@UAEXHH@Z 100165c8 f   qt-mt323:qt-mt323.dll
 0001:000155ce       ?setMouseTracking@QWidget@@UAEX_N@Z 100165ce f   qt-mt323:qt-mt323.dll
 0001:000155d4       ?setMovingEnabled@QDockWindow@@UAEX_N@Z 100165d4 f   qt-mt323:qt-mt323.dll
 0001:000155da       ?setMultiLinesEnabled@QListViewItem@@UAEX_N@Z 100165da f   qt-mt323:qt-mt323.dll
 0001:000155e0       ?setMultiSelection@QListView@@UAEX_N@Z 100165e0 f   qt-mt323:qt-mt323.dll
 0001:000155e6       ?setName@QObject@@UAEXPBD@Z 100165e6 f   qt-mt323:qt-mt323.dll
 0001:000155ec       ?setNewLine@QDockWindow@@UAEX_N@Z 100165ec f   qt-mt323:qt-mt323.dll
 0001:000155f2       ?setOffset@QDockWindow@@UAEXH@Z 100165f2 f   qt-mt323:qt-mt323.dll
 0001:000155f8       ?setOn@QAction@@UAEX_N@Z   100165f8 f   qt-mt323:qt-mt323.dll
 0001:000155fe       ?setOpaqueMoving@QDockWindow@@UAEX_N@Z 100165fe f   qt-mt323:qt-mt323.dll
 0001:00015604       ?setOpen@QListView@@UAEXPAVQListViewItem@@_N@Z 10016604 f   qt-mt323:qt-mt323.dll
 0001:0001560a       ?setOpen@QListViewItem@@UAEX_N@Z 1001660a f   qt-mt323:qt-mt323.dll
 0001:00015610       ?setOrientation@QDockWindow@@UAEXW4Orientation@Qt@@@Z 10016610 f   qt-mt323:qt-mt323.dll
 0001:00015616       ?setOrientation@QToolBar@@UAEXW4Orientation@Qt@@@Z 10016616 f   qt-mt323:qt-mt323.dll
 0001:0001561c       ?setPalette@QListView@@UAEXABVQPalette@@@Z 1001661c f   qt-mt323:qt-mt323.dll
 0001:00015622       ?setPalette@QWidget@@UAEXABVQPalette@@@Z 10016622 f   qt-mt323:qt-mt323.dll
 0001:00015628       ?setPaletteBackgroundColor@QWidget@@UAEXABVQColor@@@Z 10016628 f   qt-mt323:qt-mt323.dll
 0001:0001562e       ?setPaletteBackgroundPixmap@QWidget@@UAEXABVQPixmap@@@Z 1001662e f   qt-mt323:qt-mt323.dll
 0001:00015634       ?setPixmap@QListViewItem@@UAEXHABVQPixmap@@@Z 10016634 f   qt-mt323:qt-mt323.dll
 0001:0001563a       ?setProperty@QObject@@UAE_NPBDABVQVariant@@@Z 1001663a f   qt-mt323:qt-mt323.dll
 0001:00015640       ?setRenameEnabled@QListViewItem@@UAEXH_N@Z 10016640 f   qt-mt323:qt-mt323.dll
 0001:00015646       ?setResizeEnabled@QDockWindow@@UAEX_N@Z 10016646 f   qt-mt323:qt-mt323.dll
 0001:0001564c       ?setResizeMode@QListView@@UAEXW4ResizeMode@1@@Z 1001664c f   qt-mt323:qt-mt323.dll
 0001:00015652       ?setResizePolicy@QScrollView@@UAEXW4ResizePolicy@1@@Z 10016652 f   qt-mt323:qt-mt323.dll
 0001:00015658       ?setResolution@QPaintDevice@@UAEXH@Z 10016658 f   qt-mt323:qt-mt323.dll
 0001:0001565e       ?setRootIsDecorated@QListView@@UAEX_N@Z 1001665e f   qt-mt323:qt-mt323.dll
 0001:00015664       ?setSelectable@QListViewItem@@UAEX_N@Z 10016664 f   qt-mt323:qt-mt323.dll
 0001:0001566a       ?setSelected@QListView@@UAEXPAVQListViewItem@@_N@Z 1001666a f   qt-mt323:qt-mt323.dll
 0001:00015670       ?setSelected@QListViewItem@@UAEX_N@Z 10016670 f   qt-mt323:qt-mt323.dll
 0001:00015676       ?setShowSortIndicator@QListView@@UAEX_N@Z 10016676 f   qt-mt323:qt-mt323.dll
 0001:0001567c       ?setShowToolTips@QListView@@UAEX_N@Z 1001667c f   qt-mt323:qt-mt323.dll
 0001:00015682       ?setSizeIncrement@QWidget@@UAEXHH@Z 10016682 f   qt-mt323:qt-mt323.dll
 0001:00015688       ?setSizePolicy@QWidget@@UAEXVQSizePolicy@@@Z 10016688 f   qt-mt323:qt-mt323.dll
 0001:0001568e       ?setSorting@QListView@@UAEXH_N@Z 1001668e f   qt-mt323:qt-mt323.dll
 0001:00015694       ?setSpacing@QLayout@@UAEXH@Z 10016694 f   qt-mt323:qt-mt323.dll
 0001:0001569a       ?setStatusTip@QAction@@UAEXABVQString@@@Z 1001669a f   qt-mt323:qt-mt323.dll
 0001:000156a0       ?setStretchableWidget@QToolBar@@UAEXPAVQWidget@@@Z 100166a0 f   qt-mt323:qt-mt323.dll
 0001:000156a6       ?setText@QAction@@UAEXABVQString@@@Z 100166a6 f   qt-mt323:qt-mt323.dll
 0001:000156ac       ?setText@QListViewItem@@UAEXHABVQString@@@Z 100166ac f   qt-mt323:qt-mt323.dll
 0001:000156b2       ?setToggleAction@QAction@@UAEX_N@Z 100166b2 f   qt-mt323:qt-mt323.dll
 0001:000156b8       ?setToolTip@QAction@@UAEXABVQString@@@Z 100166b8 f   qt-mt323:qt-mt323.dll
 0001:000156be       ?setTreeStepSize@QListView@@UAEXH@Z 100166be f   qt-mt323:qt-mt323.dll
 0001:000156c4       ?setUpdatesEnabled@QWidget@@UAEX_N@Z 100166c4 f   qt-mt323:qt-mt323.dll
 0001:000156ca       ?setVBarGeometry@QScrollView@@MAEXAAVQScrollBar@@HHHH@Z 100166ca f   qt-mt323:qt-mt323.dll
 0001:000156d0       ?setVScrollBarMode@QScrollView@@UAEXW4ScrollBarMode@1@@Z 100166d0 f   qt-mt323:qt-mt323.dll
 0001:000156d6       ?setVerticallyStretchable@QDockWindow@@UAEX_N@Z 100166d6 f   qt-mt323:qt-mt323.dll
 0001:000156dc       ?setWFlags@QWidget@@MAEXI@Z 100166dc f   qt-mt323:qt-mt323.dll
 0001:000156e2       ?setWState@QWidget@@MAEXI@Z 100166e2 f   qt-mt323:qt-mt323.dll
 0001:000156e8       ?setWhatsThis@QAction@@UAEXABVQString@@@Z 100166e8 f   qt-mt323:qt-mt323.dll
 0001:000156ee       ?setWidget@QDockWindow@@UAEXPAVQWidget@@@Z 100166ee f   qt-mt323:qt-mt323.dll
 0001:000156f4       ?setup@QListViewItem@@UAEXXZ 100166f4 f   qt-mt323:qt-mt323.dll
 0001:000156fa       ?show@QListView@@UAEXXZ    100166fa f   qt-mt323:qt-mt323.dll
 0001:00015700       ?show@QPopupMenu@@UAEXXZ   10016700 f   qt-mt323:qt-mt323.dll
 0001:00015706       ?show@QToolBar@@UAEXXZ     10016706 f   qt-mt323:qt-mt323.dll
 0001:0001570c       ?show@QWidget@@UAEXXZ      1001670c f   qt-mt323:qt-mt323.dll
 0001:00015712       ?showEvent@QDockWindow@@MAEXPAVQShowEvent@@@Z 10016712 f   qt-mt323:qt-mt323.dll
 0001:00015718       ?showEvent@QListView@@MAEXPAVQShowEvent@@@Z 10016718 f   qt-mt323:qt-mt323.dll
 0001:0001571e       ?showEvent@QTabWidget@@MAEXPAVQShowEvent@@@Z 1001671e f   qt-mt323:qt-mt323.dll
 0001:00015724       ?showEvent@QWidget@@MAEXPAVQShowEvent@@@Z 10016724 f   qt-mt323:qt-mt323.dll
 0001:0001572a       ?showMaximized@QWidget@@UAEXXZ 1001672a f   qt-mt323:qt-mt323.dll
 0001:00015730       ?showMinimized@QWidget@@UAEXXZ 10016730 f   qt-mt323:qt-mt323.dll
 0001:00015736       ?showNormal@QWidget@@UAEXXZ 10016736 f   qt-mt323:qt-mt323.dll
 0001:0001573c       ?showPage@QTabWidget@@UAEXPAVQWidget@@@Z 1001673c f   qt-mt323:qt-mt323.dll
 0001:00015742       ?sizeHint@QBoxLayout@@UBE?AVQSize@@XZ 10016742 f   qt-mt323:qt-mt323.dll
 0001:00015748       ?sizeHint@QDockWindow@@UBE?AVQSize@@XZ 10016748 f   qt-mt323:qt-mt323.dll
 0001:0001574e       ?sizeHint@QHBox@@UBE?AVQSize@@XZ 1001674e f   qt-mt323:qt-mt323.dll
 0001:00015754       ?sizeHint@QListView@@UBE?AVQSize@@XZ 10016754 f   qt-mt323:qt-mt323.dll
 0001:0001575a       ?sizeHint@QPopupMenu@@UBE?AVQSize@@XZ 1001675a f   qt-mt323:qt-mt323.dll
 0001:00015760       ?sizeHint@QTabWidget@@UBE?AVQSize@@XZ 10016760 f   qt-mt323:qt-mt323.dll
 0001:00015766       ?sizeHint@QWidget@@UBE?AVQSize@@XZ 10016766 f   qt-mt323:qt-mt323.dll
 0001:0001576c       ?sizePolicy@QWidget@@UBE?AVQSizePolicy@@XZ 1001676c f   qt-mt323:qt-mt323.dll
 0001:00015772       ?sort@QListView@@UAEXXZ    10016772 f   qt-mt323:qt-mt323.dll
 0001:00015778       ?sort@QListViewItem@@UAEXXZ 10016778 f   qt-mt323:qt-mt323.dll
 0001:0001577e       ?sortChildItems@QListViewItem@@UAEXH_N@Z 1001677e f   qt-mt323:qt-mt323.dll
 0001:00015784       ?spacerItem@QLayoutItem@@UAEPAVQSpacerItem@@XZ 10016784 f   qt-mt323:qt-mt323.dll
 0001:0001578a       ?startDrag@QListView@@MAEXXZ 1001678a f   qt-mt323:qt-mt323.dll
 0001:00015790       ?startRename@QListViewItem@@UAEXH@Z 10016790 f   qt-mt323:qt-mt323.dll
 0001:00015796       ?styleChange@QFrame@@MAEXAAVQStyle@@@Z 10016796 f   qt-mt323:qt-mt323.dll
 0001:0001579c       ?styleChange@QListView@@MAEXAAVQStyle@@@Z 1001679c f   qt-mt323:qt-mt323.dll
 0001:000157a2       ?styleChange@QPopupMenu@@MAEXAAVQStyle@@@Z 100167a2 f   qt-mt323:qt-mt323.dll
 0001:000157a8       ?styleChange@QTabWidget@@MAEXAAVQStyle@@@Z 100167a8 f   qt-mt323:qt-mt323.dll
 0001:000157ae       ?styleChange@QToolBar@@MAEXAAVQStyle@@@Z 100167ae f   qt-mt323:qt-mt323.dll
 0001:000157b4       ?styleChange@QWidget@@MAEXAAVQStyle@@@Z 100167b4 f   qt-mt323:qt-mt323.dll
 0001:000157ba       ?tabletEvent@QWidget@@MAEXPAVQTabletEvent@@@Z 100167ba f   qt-mt323:qt-mt323.dll
 0001:000157c0       ?takeItem@QListView@@UAEXPAVQListViewItem@@@Z 100167c0 f   qt-mt323:qt-mt323.dll
 0001:000157c6       ?takeItem@QListViewItem@@UAEXPAV1@@Z 100167c6 f   qt-mt323:qt-mt323.dll
 0001:000157cc       ?text@QListViewItem@@UBE?AVQString@@H@Z 100167cc f   qt-mt323:qt-mt323.dll
 0001:000157d2       ?timerEvent@QObject@@MAEXPAVQTimerEvent@@@Z 100167d2 f   qt-mt323:qt-mt323.dll
 0001:000157d8       ?timerEvent@QPopupMenu@@MAEXPAVQTimerEvent@@@Z 100167d8 f   qt-mt323:qt-mt323.dll
 0001:000157de       ?undock@QDockWindow@@UAEXPAVQWidget@@@Z 100167de f   qt-mt323:qt-mt323.dll
 0001:000157e4       ?undock@QDockWindow@@UAEXXZ 100167e4 f   qt-mt323:qt-mt323.dll
 0001:000157ea       ?unsetCursor@QWidget@@UAEXXZ 100167ea f   qt-mt323:qt-mt323.dll
 0001:000157f0       ?updateItem@QPopupMenu@@UAEXH@Z 100167f0 f   qt-mt323:qt-mt323.dll
 0001:000157f6       ?updateMask@QTabWidget@@MAEXXZ 100167f6 f   qt-mt323:qt-mt323.dll
 0001:000157fc       ?updateMask@QWidget@@MAEXXZ 100167fc f   qt-mt323:qt-mt323.dll
 0001:00015802       ?viewportContextMenuEvent@QScrollView@@MAEXPAVQContextMenuEvent@@@Z 10016802 f   qt-mt323:qt-mt323.dll
 0001:00015808       ?viewportDragEnterEvent@QScrollView@@MAEXPAVQDragEnterEvent@@@Z 10016808 f   qt-mt323:qt-mt323.dll
 0001:0001580e       ?viewportDragLeaveEvent@QScrollView@@MAEXPAVQDragLeaveEvent@@@Z 1001680e f   qt-mt323:qt-mt323.dll
 0001:00015814       ?viewportDragMoveEvent@QScrollView@@MAEXPAVQDragMoveEvent@@@Z 10016814 f   qt-mt323:qt-mt323.dll
 0001:0001581a       ?viewportDropEvent@QScrollView@@MAEXPAVQDropEvent@@@Z 1001681a f   qt-mt323:qt-mt323.dll
 0001:00015820       ?viewportMouseDoubleClickEvent@QScrollView@@MAEXPAVQMouseEvent@@@Z 10016820 f   qt-mt323:qt-mt323.dll
 0001:00015826       ?viewportMouseMoveEvent@QScrollView@@MAEXPAVQMouseEvent@@@Z 10016826 f   qt-mt323:qt-mt323.dll
 0001:0001582c       ?viewportMousePressEvent@QScrollView@@MAEXPAVQMouseEvent@@@Z 1001682c f   qt-mt323:qt-mt323.dll
 0001:00015832       ?viewportMouseReleaseEvent@QScrollView@@MAEXPAVQMouseEvent@@@Z 10016832 f   qt-mt323:qt-mt323.dll
 0001:00015838       ?viewportPaintEvent@QScrollView@@MAEXPAVQPaintEvent@@@Z 10016838 f   qt-mt323:qt-mt323.dll
 0001:0001583e       ?viewportResizeEvent@QListView@@MAEXPAVQResizeEvent@@@Z 1001683e f   qt-mt323:qt-mt323.dll
 0001:00015844       ?viewportWheelEvent@QScrollView@@MAEXPAVQWheelEvent@@@Z 10016844 f   qt-mt323:qt-mt323.dll
 0001:0001584a       ?wheelEvent@QScrollView@@MAEXPAVQWheelEvent@@@Z 1001684a f   qt-mt323:qt-mt323.dll
 0001:00015850       ?wheelEvent@QWidget@@MAEXPAVQWheelEvent@@@Z 10016850 f   qt-mt323:qt-mt323.dll
 0001:00015856       ?widget@QLayoutItem@@UAEPAVQWidget@@XZ 10016856 f   qt-mt323:qt-mt323.dll
 0001:0001585c       ?width@QListViewItem@@UBEHABVQFontMetrics@@PBVQListView@@H@Z 1001685c f   qt-mt323:qt-mt323.dll
 0001:00015862       ?winEvent@QWidget@@MAE_NPAUtagMSG@@@Z 10016862 f   qt-mt323:qt-mt323.dll
 0001:00015868       ?windowActivationChange@QListView@@MAEX_N@Z 10016868 f   qt-mt323:qt-mt323.dll
 0001:0001586e       ?windowActivationChange@QWidget@@MAEX_N@Z 1001686e f   qt-mt323:qt-mt323.dll
 0001:00015874       ?write@QGList@@MBEAAVQDataStream@@AAV2@PAX@Z 10016874 f   qt-mt323:qt-mt323.dll
 0001:0001587a       ?accept@QDialog@@MAEXXZ    1001687a f   qt-mt323:qt-mt323.dll
 0001:00015880       ?closeEvent@QDialog@@MAEXPAVQCloseEvent@@@Z 10016880 f   qt-mt323:qt-mt323.dll
 0001:00015886       ?contextMenuEvent@QDialog@@MAEXPAVQContextMenuEvent@@@Z 10016886 f   qt-mt323:qt-mt323.dll
 0001:0001588c       ?done@QDialog@@MAEXH@Z     1001688c f   qt-mt323:qt-mt323.dll
 0001:00015892       ?eventFilter@QDialog@@MAE_NPAVQObject@@PAVQEvent@@@Z 10016892 f   qt-mt323:qt-mt323.dll
 0001:00015898       ?hide@QDialog@@UAEXXZ      10016898 f   qt-mt323:qt-mt323.dll
 0001:0001589e       ?keyPressEvent@QDialog@@MAEXPAVQKeyEvent@@@Z 1001689e f   qt-mt323:qt-mt323.dll
 0001:000158a4       ?minimumSizeHint@QDialog@@UBE?AVQSize@@XZ 100168a4 f   qt-mt323:qt-mt323.dll
 0001:000158aa       ?move@QDialog@@UAEXHH@Z    100168aa f   qt-mt323:qt-mt323.dll
 0001:000158b0       ?reject@QDialog@@MAEXXZ    100168b0 f   qt-mt323:qt-mt323.dll
 0001:000158b6       ?resize@QDialog@@UAEXHH@Z  100168b6 f   qt-mt323:qt-mt323.dll
 0001:000158bc       ?resizeEvent@QDialog@@MAEXPAVQResizeEvent@@@Z 100168bc f   qt-mt323:qt-mt323.dll
 0001:000158c2       ?setGeometry@QDialog@@UAEXABVQRect@@@Z 100168c2 f   qt-mt323:qt-mt323.dll
 0001:000158c8       ?setGeometry@QDialog@@UAEXHHHH@Z 100168c8 f   qt-mt323:qt-mt323.dll
 0001:000158ce       ?show@QDialog@@UAEXXZ      100168ce f   qt-mt323:qt-mt323.dll
 0001:000158d4       ?sizeHint@QDialog@@UBE?AVQSize@@XZ 100168d4 f   qt-mt323:qt-mt323.dll
 0001:000158da       ?read@QGDict@@MAEAAVQDataStream@@AAV2@AAPAX@Z 100168da f   qt-mt323:qt-mt323.dll
 0001:000158e0       ?write@QGDict@@MBEAAVQDataStream@@AAV2@PAX@Z 100168e0 f   qt-mt323:qt-mt323.dll
 0001:000158e6       ?activateNextCell@QTable@@MAEXXZ 100168e6 f   qt-mt323:qt-mt323.dll
 0001:000158ec       ?addItem@QGridLayout@@UAEXPAVQLayoutItem@@@Z 100168ec f   qt-mt323:qt-mt323.dll
 0001:000158f2       ?addSelection@QTable@@UAEHABVQTableSelection@@@Z 100168f2 f   qt-mt323:qt-mt323.dll
 0001:000158f8       ?adjustColumn@QTable@@UAEXH@Z 100168f8 f   qt-mt323:qt-mt323.dll
 0001:000158fe       ?adjustRow@QTable@@UAEXH@Z 100168fe f   qt-mt323:qt-mt323.dll
 0001:00015904       ?beginEdit@QTable@@MAEPAVQWidget@@HH_N@Z 10016904 f   qt-mt323:qt-mt323.dll
 0001:0001590a       ?cellGeometry@QTable@@UBE?AVQRect@@HH@Z 1001690a f   qt-mt323:qt-mt323.dll
 0001:00015910       ?cellRect@QTable@@UBE?AVQRect@@HH@Z 10016910 f   qt-mt323:qt-mt323.dll
 0001:00015916       ?cellWidget@QTable@@UBEPAVQWidget@@HH@Z 10016916 f   qt-mt323:qt-mt323.dll
 0001:0001591c       ?className@QComboBox@@UBEPBDXZ 1001691c f   qt-mt323:qt-mt323.dll
 0001:00015922       ?className@QGridLayout@@UBEPBDXZ 10016922 f   qt-mt323:qt-mt323.dll
 0001:00015928       ?className@QHBoxLayout@@UBEPBDXZ 10016928 f   qt-mt323:qt-mt323.dll
 0001:0001592e       ?className@QLabel@@UBEPBDXZ 1001692e f   qt-mt323:qt-mt323.dll
 0001:00015934       ?className@QLineEdit@@UBEPBDXZ 10016934 f   qt-mt323:qt-mt323.dll
 0001:0001593a       ?className@QPushButton@@UBEPBDXZ 1001693a f   qt-mt323:qt-mt323.dll
 0001:00015940       ?className@QSpinBox@@UBEPBDXZ 10016940 f   qt-mt323:qt-mt323.dll
 0001:00015946       ?className@QTable@@UBEPBDXZ 10016946 f   qt-mt323:qt-mt323.dll
 0001:0001594c       ?className@QVBoxLayout@@UBEPBDXZ 1001694c f   qt-mt323:qt-mt323.dll
 0001:00015952       ?cleanText@QSpinBox@@UBE?AVQString@@XZ 10016952 f   qt-mt323:qt-mt323.dll
 0001:00015958       ?clear@QLineEdit@@UAEXXZ   10016958 f   qt-mt323:qt-mt323.dll
 0001:0001595e       ?clearCell@QTable@@UAEXHH@Z 1001695e f   qt-mt323:qt-mt323.dll
 0001:00015964       ?clearCellWidget@QTable@@UAEXHH@Z 10016964 f   qt-mt323:qt-mt323.dll
 0001:0001596a       ?clearValidator@QLineEdit@@UAEXXZ 1001696a f   qt-mt323:qt-mt323.dll
 0001:00015970       ?columnAt@QTable@@UBEHH@Z  10016970 f   qt-mt323:qt-mt323.dll
 0001:00015976       ?columnClicked@QTable@@MAEXH@Z 10016976 f   qt-mt323:qt-mt323.dll
 0001:0001597c       ?columnIndexChanged@QTable@@MAEXHHH@Z 1001697c f   qt-mt323:qt-mt323.dll
 0001:00015982       ?columnPos@QTable@@UBEHH@Z 10016982 f   qt-mt323:qt-mt323.dll
 0001:00015988       ?columnWidth@QTable@@UBEHH@Z 10016988 f   qt-mt323:qt-mt323.dll
 0001:0001598e       ?columnWidthChanged@QTable@@MAEXH@Z 1001698e f   qt-mt323:qt-mt323.dll
 0001:00015994       ?contentsContextMenuEvent@QTable@@MAEXPAVQContextMenuEvent@@@Z 10016994 f   qt-mt323:qt-mt323.dll
 0001:0001599a       ?contentsDragEnterEvent@QTable@@MAEXPAVQDragEnterEvent@@@Z 1001699a f   qt-mt323:qt-mt323.dll
 0001:000159a0       ?contentsDragLeaveEvent@QTable@@MAEXPAVQDragLeaveEvent@@@Z 100169a0 f   qt-mt323:qt-mt323.dll
 0001:000159a6       ?contentsDragMoveEvent@QTable@@MAEXPAVQDragMoveEvent@@@Z 100169a6 f   qt-mt323:qt-mt323.dll
 0001:000159ac       ?contentsDropEvent@QTable@@MAEXPAVQDropEvent@@@Z 100169ac f   qt-mt323:qt-mt323.dll
 0001:000159b2       ?contentsMouseDoubleClickEvent@QTable@@MAEXPAVQMouseEvent@@@Z 100169b2 f   qt-mt323:qt-mt323.dll
 0001:000159b8       ?contentsMouseMoveEvent@QTable@@MAEXPAVQMouseEvent@@@Z 100169b8 f   qt-mt323:qt-mt323.dll
 0001:000159be       ?contentsMousePressEvent@QTable@@MAEXPAVQMouseEvent@@@Z 100169be f   qt-mt323:qt-mt323.dll
 0001:000159c4       ?contentsMouseReleaseEvent@QTable@@MAEXPAVQMouseEvent@@@Z 100169c4 f   qt-mt323:qt-mt323.dll
 0001:000159ca       ?contextMenuEvent@QLineEdit@@MAEXPAVQContextMenuEvent@@@Z 100169ca f   qt-mt323:qt-mt323.dll
 0001:000159d0       ?copy@QLineEdit@@UBEXXZ    100169d0 f   qt-mt323:qt-mt323.dll
 0001:000159d6       ?createEditor@QTable@@MBEPAVQWidget@@HH_N@Z 100169d6 f   qt-mt323:qt-mt323.dll
 0001:000159dc       ?createPopupMenu@QLineEdit@@MAEPAVQPopupMenu@@XZ 100169dc f   qt-mt323:qt-mt323.dll
 0001:000159e2       ?currentSelection@QTable@@UBEHXZ 100169e2 f   qt-mt323:qt-mt323.dll
 0001:000159e8       ?cut@QLineEdit@@UAEXXZ     100169e8 f   qt-mt323:qt-mt323.dll
 0001:000159ee       ?deselect@QLineEdit@@UAEXXZ 100169ee f   qt-mt323:qt-mt323.dll
 0001:000159f4       ?dragEnterEvent@QLineEdit@@MAEXPAVQDragEnterEvent@@@Z 100169f4 f   qt-mt323:qt-mt323.dll
 0001:000159fa       ?dragLeaveEvent@QLineEdit@@MAEXPAVQDragLeaveEvent@@@Z 100169fa f   qt-mt323:qt-mt323.dll
 0001:00015a00       ?dragMoveEvent@QLineEdit@@MAEXPAVQDragMoveEvent@@@Z 10016a00 f   qt-mt323:qt-mt323.dll
 0001:00015a06       ?dragObject@QTable@@MAEPAVQDragObject@@XZ 10016a06 f   qt-mt323:qt-mt323.dll
 0001:00015a0c       ?drawButton@QPushButton@@MAEXPAVQPainter@@@Z 10016a0c f   qt-mt323:qt-mt323.dll
 0001:00015a12       ?drawButtonLabel@QPushButton@@MAEXPAVQPainter@@@Z 10016a12 f   qt-mt323:qt-mt323.dll
 0001:00015a18       ?drawContents@QLabel@@MAEXPAVQPainter@@@Z 10016a18 f   qt-mt323:qt-mt323.dll
 0001:00015a1e       ?drawContents@QLineEdit@@MAEXPAVQPainter@@@Z 10016a1e f   qt-mt323:qt-mt323.dll
 0001:00015a24       ?drawContents@QTable@@EAEXPAVQPainter@@@Z 10016a24 f   qt-mt323:qt-mt323.dll
 0001:00015a2a       ?drawContents@QTable@@MAEXPAVQPainter@@HHHH@Z 10016a2a f   qt-mt323:qt-mt323.dll
 0001:00015a30       ?drawContentsOffset@QScrollView@@MAEXPAVQPainter@@HHHHHH@Z 10016a30 f   qt-mt323:qt-mt323.dll
 0001:00015a36       ?dropEvent@QLineEdit@@MAEXPAVQDropEvent@@@Z 10016a36 f   qt-mt323:qt-mt323.dll
 0001:00015a3c       ?editCell@QTable@@UAEXHH_N@Z 10016a3c f   qt-mt323:qt-mt323.dll
 0001:00015a42       ?enabledChange@QButton@@MAEX_N@Z 10016a42 f   qt-mt323:qt-mt323.dll
 0001:00015a48       ?endEdit@QTable@@MAEXHH_N0@Z 10016a48 f   qt-mt323:qt-mt323.dll
 0001:00015a4e       ?event@QLineEdit@@MAE_NPAVQEvent@@@Z 10016a4e f   qt-mt323:qt-mt323.dll
 0001:00015a54       ?eventFilter@QComboBox@@UAE_NPAVQObject@@PAVQEvent@@@Z 10016a54 f   qt-mt323:qt-mt323.dll
 0001:00015a5a       ?eventFilter@QSpinBox@@MAE_NPAVQObject@@PAVQEvent@@@Z 10016a5a f   qt-mt323:qt-mt323.dll
 0001:00015a60       ?eventFilter@QTable@@UAE_NPAVQObject@@PAVQEvent@@@Z 10016a60 f   qt-mt323:qt-mt323.dll
 0001:00015a66       ?expanding@QGridLayout@@UBE?AW4ExpandData@QSizePolicy@@XZ 10016a66 f   qt-mt323:qt-mt323.dll
 0001:00015a6c       ?expanding@QSpacerItem@@UBE?AW4ExpandData@QSizePolicy@@XZ 10016a6c f   qt-mt323:qt-mt323.dll
 0001:00015a72       ?focusInEvent@QComboBox@@MAEXPAVQFocusEvent@@@Z 10016a72 f   qt-mt323:qt-mt323.dll
 0001:00015a78       ?focusInEvent@QLineEdit@@MAEXPAVQFocusEvent@@@Z 10016a78 f   qt-mt323:qt-mt323.dll
 0001:00015a7e       ?focusInEvent@QPushButton@@MAEXPAVQFocusEvent@@@Z 10016a7e f   qt-mt323:qt-mt323.dll
 0001:00015a84       ?focusInEvent@QTable@@MAEXPAVQFocusEvent@@@Z 10016a84 f   qt-mt323:qt-mt323.dll
 0001:00015a8a       ?focusOutEvent@QComboBox@@MAEXPAVQFocusEvent@@@Z 10016a8a f   qt-mt323:qt-mt323.dll
 0001:00015a90       ?focusOutEvent@QLineEdit@@MAEXPAVQFocusEvent@@@Z 10016a90 f   qt-mt323:qt-mt323.dll
 0001:00015a96       ?focusOutEvent@QPushButton@@MAEXPAVQFocusEvent@@@Z 10016a96 f   qt-mt323:qt-mt323.dll
 0001:00015a9c       ?focusOutEvent@QTable@@MAEXPAVQFocusEvent@@@Z 10016a9c f   qt-mt323:qt-mt323.dll
 0001:00015aa2       ?fontChange@QLabel@@MAEXABVQFont@@@Z 10016aa2 f   qt-mt323:qt-mt323.dll
 0001:00015aa8       ?geometry@QSpacerItem@@UBE?AVQRect@@XZ 10016aa8 f   qt-mt323:qt-mt323.dll
 0001:00015aae       ?hasHeightForWidth@QGridLayout@@UBE_NXZ 10016aae f   qt-mt323:qt-mt323.dll
 0001:00015ab4       ?hasHeightForWidth@QLayoutItem@@UBE_NXZ 10016ab4 f   qt-mt323:qt-mt323.dll
 0001:00015aba       ?heightForWidth@QGridLayout@@UBEHH@Z 10016aba f   qt-mt323:qt-mt323.dll
 0001:00015ac0       ?heightForWidth@QLabel@@UBEHH@Z 10016ac0 f   qt-mt323:qt-mt323.dll
 0001:00015ac6       ?heightForWidth@QLayoutItem@@UBEHH@Z 10016ac6 f   qt-mt323:qt-mt323.dll
 0001:00015acc       ?hideColumn@QTable@@UAEXH@Z 10016acc f   qt-mt323:qt-mt323.dll
 0001:00015ad2       ?hideRow@QTable@@UAEXH@Z   10016ad2 f   qt-mt323:qt-mt323.dll
 0001:00015ad8       ?hitButton@QButton@@MBE_NABVQPoint@@@Z 10016ad8 f   qt-mt323:qt-mt323.dll
 0001:00015ade       ?imComposeEvent@QLineEdit@@MAEXPAVQIMEvent@@@Z 10016ade f   qt-mt323:qt-mt323.dll
 0001:00015ae4       ?imEndEvent@QLineEdit@@MAEXPAVQIMEvent@@@Z 10016ae4 f   qt-mt323:qt-mt323.dll
 0001:00015aea       ?imStartEvent@QLineEdit@@MAEXPAVQIMEvent@@@Z 10016aea f   qt-mt323:qt-mt323.dll
 0001:00015af0       ?insert@QLineEdit@@UAEXABVQString@@@Z 10016af0 f   qt-mt323:qt-mt323.dll
 0001:00015af6       ?insertColumns@QTable@@UAEXHH@Z 10016af6 f   qt-mt323:qt-mt323.dll
 0001:00015afc       ?insertRows@QTable@@UAEXHH@Z 10016afc f   qt-mt323:qt-mt323.dll
 0001:00015b02       ?insertWidget@QTable@@MAEXHHPAVQWidget@@@Z 10016b02 f   qt-mt323:qt-mt323.dll
 0001:00015b08       ?interpretText@QSpinBox@@MAEXXZ 10016b08 f   qt-mt323:qt-mt323.dll
 0001:00015b0e       ?invalidate@QGridLayout@@UAEXXZ 10016b0e f   qt-mt323:qt-mt323.dll
 0001:00015b14       ?invalidate@QLayoutItem@@UAEXXZ 10016b14 f   qt-mt323:qt-mt323.dll
 0001:00015b1a       ?isEmpty@QSpacerItem@@UBE_NXZ 10016b1a f   qt-mt323:qt-mt323.dll
 0001:00015b20       ?item@QTable@@UBEPAVQTableItem@@HH@Z 10016b20 f   qt-mt323:qt-mt323.dll
 0001:00015b26       ?iterator@QGridLayout@@UAE?AVQLayoutIterator@@XZ 10016b26 f   qt-mt323:qt-mt323.dll
 0001:00015b2c       ?iterator@QLayoutItem@@UAE?AVQLayoutIterator@@XZ 10016b2c f   qt-mt323:qt-mt323.dll
 0001:00015b32       ?keyPressEvent@QButton@@MAEXPAVQKeyEvent@@@Z 10016b32 f   qt-mt323:qt-mt323.dll
 0001:00015b38       ?keyPressEvent@QComboBox@@MAEXPAVQKeyEvent@@@Z 10016b38 f   qt-mt323:qt-mt323.dll
 0001:00015b3e       ?keyPressEvent@QLineEdit@@MAEXPAVQKeyEvent@@@Z 10016b3e f   qt-mt323:qt-mt323.dll
 0001:00015b44       ?keyPressEvent@QTable@@MAEXPAVQKeyEvent@@@Z 10016b44 f   qt-mt323:qt-mt323.dll
 0001:00015b4a       ?keyReleaseEvent@QButton@@MAEXPAVQKeyEvent@@@Z 10016b4a f   qt-mt323:qt-mt323.dll
 0001:00015b50       ?layout@QLayoutItem@@UAEPAVQLayout@@XZ 10016b50 f   qt-mt323:qt-mt323.dll
 0001:00015b56       ?leaveEvent@QSpinBox@@MAEXPAVQEvent@@@Z 10016b56 f   qt-mt323:qt-mt323.dll
 0001:00015b5c       ?mapTextToValue@QSpinBox@@MAEHPA_N@Z 10016b5c f   qt-mt323:qt-mt323.dll
 0001:00015b62       ?mapValueToText@QSpinBox@@MAE?AVQString@@H@Z 10016b62 f   qt-mt323:qt-mt323.dll
 0001:00015b68       ?maximumSize@QGridLayout@@UBE?AVQSize@@XZ 10016b68 f   qt-mt323:qt-mt323.dll
 0001:00015b6e       ?maximumSize@QSpacerItem@@UBE?AVQSize@@XZ 10016b6e f   qt-mt323:qt-mt323.dll
 0001:00015b74       ?metaObject@QComboBox@@UBEPAVQMetaObject@@XZ 10016b74 f   qt-mt323:qt-mt323.dll
 0001:00015b7a       ?metaObject@QGridLayout@@UBEPAVQMetaObject@@XZ 10016b7a f   qt-mt323:qt-mt323.dll
 0001:00015b80       ?metaObject@QHBoxLayout@@UBEPAVQMetaObject@@XZ 10016b80 f   qt-mt323:qt-mt323.dll
 0001:00015b86       ?metaObject@QLabel@@UBEPAVQMetaObject@@XZ 10016b86 f   qt-mt323:qt-mt323.dll
 0001:00015b8c       ?metaObject@QLineEdit@@UBEPAVQMetaObject@@XZ 10016b8c f   qt-mt323:qt-mt323.dll
 0001:00015b92       ?metaObject@QPushButton@@UBEPAVQMetaObject@@XZ 10016b92 f   qt-mt323:qt-mt323.dll
 0001:00015b98       ?metaObject@QSpinBox@@UBEPAVQMetaObject@@XZ 10016b98 f   qt-mt323:qt-mt323.dll
 0001:00015b9e       ?metaObject@QTable@@UBEPAVQMetaObject@@XZ 10016b9e f   qt-mt323:qt-mt323.dll
 0001:00015ba4       ?metaObject@QVBoxLayout@@UBEPAVQMetaObject@@XZ 10016ba4 f   qt-mt323:qt-mt323.dll
 0001:00015baa       ?minimumSize@QGridLayout@@UBE?AVQSize@@XZ 10016baa f   qt-mt323:qt-mt323.dll
 0001:00015bb0       ?minimumSize@QSpacerItem@@UBE?AVQSize@@XZ 10016bb0 f   qt-mt323:qt-mt323.dll
 0001:00015bb6       ?minimumSizeHint@QLabel@@UBE?AVQSize@@XZ 10016bb6 f   qt-mt323:qt-mt323.dll
 0001:00015bbc       ?minimumSizeHint@QLineEdit@@UBE?AVQSize@@XZ 10016bbc f   qt-mt323:qt-mt323.dll
 0001:00015bc2       ?minimumSizeHint@QScrollView@@UBE?AVQSize@@XZ 10016bc2 f   qt-mt323:qt-mt323.dll
 0001:00015bc8       ?minimumSizeHint@QSpinBox@@UBE?AVQSize@@XZ 10016bc8 f   qt-mt323:qt-mt323.dll
 0001:00015bce       ?mouseDoubleClickEvent@QComboBox@@MAEXPAVQMouseEvent@@@Z 10016bce f   qt-mt323:qt-mt323.dll
 0001:00015bd4       ?mouseDoubleClickEvent@QLineEdit@@MAEXPAVQMouseEvent@@@Z 10016bd4 f   qt-mt323:qt-mt323.dll
 0001:00015bda       ?mouseMoveEvent@QButton@@MAEXPAVQMouseEvent@@@Z 10016bda f   qt-mt323:qt-mt323.dll
 0001:00015be0       ?mouseMoveEvent@QComboBox@@MAEXPAVQMouseEvent@@@Z 10016be0 f   qt-mt323:qt-mt323.dll
 0001:00015be6       ?mouseMoveEvent@QLineEdit@@MAEXPAVQMouseEvent@@@Z 10016be6 f   qt-mt323:qt-mt323.dll
 0001:00015bec       ?mousePressEvent@QButton@@MAEXPAVQMouseEvent@@@Z 10016bec f   qt-mt323:qt-mt323.dll
 0001:00015bf2       ?mousePressEvent@QComboBox@@MAEXPAVQMouseEvent@@@Z 10016bf2 f   qt-mt323:qt-mt323.dll
 0001:00015bf8       ?mousePressEvent@QLineEdit@@MAEXPAVQMouseEvent@@@Z 10016bf8 f   qt-mt323:qt-mt323.dll
 0001:00015bfe       ?mouseReleaseEvent@QButton@@MAEXPAVQMouseEvent@@@Z 10016bfe f   qt-mt323:qt-mt323.dll
 0001:00015c04       ?mouseReleaseEvent@QComboBox@@MAEXPAVQMouseEvent@@@Z 10016c04 f   qt-mt323:qt-mt323.dll
 0001:00015c0a       ?mouseReleaseEvent@QLineEdit@@MAEXPAVQMouseEvent@@@Z 10016c0a f   qt-mt323:qt-mt323.dll
 0001:00015c10       ?move@QPushButton@@UAEXHH@Z 10016c10 f   qt-mt323:qt-mt323.dll
 0001:00015c16       ?numCols@QTable@@UBEHXZ    10016c16 f   qt-mt323:qt-mt323.dll
 0001:00015c1c       ?numRows@QTable@@UBEHXZ    10016c1c f   qt-mt323:qt-mt323.dll
 0001:00015c22       ?paintCell@QTable@@UAEXPAVQPainter@@HHABVQRect@@_N@Z 10016c22 f   qt-mt323:qt-mt323.dll
 0001:00015c28       ?paintCell@QTable@@UAEXPAVQPainter@@HHABVQRect@@_NABVQColorGroup@@@Z 10016c28 f   qt-mt323:qt-mt323.dll
 0001:00015c2e       ?paintEmptyArea@QTable@@MAEXPAVQPainter@@HHHH@Z 10016c2e f   qt-mt323:qt-mt323.dll
 0001:00015c34       ?paintEvent@QButton@@MAEXPAVQPaintEvent@@@Z 10016c34 f   qt-mt323:qt-mt323.dll
 0001:00015c3a       ?paintEvent@QComboBox@@MAEXPAVQPaintEvent@@@Z 10016c3a f   qt-mt323:qt-mt323.dll
 0001:00015c40       ?paintEvent@QTable@@MAEXPAVQPaintEvent@@@Z 10016c40 f   qt-mt323:qt-mt323.dll
 0001:00015c46       ?paintFocus@QTable@@UAEXPAVQPainter@@ABVQRect@@@Z 10016c46 f   qt-mt323:qt-mt323.dll
 0001:00015c4c       ?paste@QLineEdit@@UAEXXZ   10016c4c f   qt-mt323:qt-mt323.dll
 0001:00015c52       ?pixmap@QTable@@UBE?AVQPixmap@@HH@Z 10016c52 f   qt-mt323:qt-mt323.dll
 0001:00015c58       ?popup@QComboBox@@UAEXXZ   10016c58 f   qt-mt323:qt-mt323.dll
 0001:00015c5e       ?prefix@QSpinBox@@UBE?AVQString@@XZ 10016c5e f   qt-mt323:qt-mt323.dll
 0001:00015c64       ?qt_cast@QComboBox@@UAEPAXPBD@Z 10016c64 f   qt-mt323:qt-mt323.dll
 0001:00015c6a       ?qt_cast@QGridLayout@@UAEPAXPBD@Z 10016c6a f   qt-mt323:qt-mt323.dll
 0001:00015c70       ?qt_cast@QHBoxLayout@@UAEPAXPBD@Z 10016c70 f   qt-mt323:qt-mt323.dll
 0001:00015c76       ?qt_cast@QLabel@@UAEPAXPBD@Z 10016c76 f   qt-mt323:qt-mt323.dll
 0001:00015c7c       ?qt_cast@QLineEdit@@UAEPAXPBD@Z 10016c7c f   qt-mt323:qt-mt323.dll
 0001:00015c82       ?qt_cast@QPushButton@@UAEPAXPBD@Z 10016c82 f   qt-mt323:qt-mt323.dll
 0001:00015c88       ?qt_cast@QSpinBox@@UAEPAXPBD@Z 10016c88 f   qt-mt323:qt-mt323.dll
 0001:00015c8e       ?qt_cast@QTable@@UAEPAXPBD@Z 10016c8e f   qt-mt323:qt-mt323.dll
 0001:00015c94       ?qt_cast@QVBoxLayout@@UAEPAXPBD@Z 10016c94 f   qt-mt323:qt-mt323.dll
 0001:00015c9a       ?qt_emit@QComboBox@@UAE_NHPAUQUObject@@@Z 10016c9a f   qt-mt323:qt-mt323.dll
 0001:00015ca0       ?qt_emit@QGridLayout@@UAE_NHPAUQUObject@@@Z 10016ca0 f   qt-mt323:qt-mt323.dll
 0001:00015ca6       ?qt_emit@QHBoxLayout@@UAE_NHPAUQUObject@@@Z 10016ca6 f   qt-mt323:qt-mt323.dll
 0001:00015cac       ?qt_emit@QLabel@@UAE_NHPAUQUObject@@@Z 10016cac f   qt-mt323:qt-mt323.dll
 0001:00015cb2       ?qt_emit@QLineEdit@@UAE_NHPAUQUObject@@@Z 10016cb2 f   qt-mt323:qt-mt323.dll
 0001:00015cb8       ?qt_emit@QPushButton@@UAE_NHPAUQUObject@@@Z 10016cb8 f   qt-mt323:qt-mt323.dll
 0001:00015cbe       ?qt_emit@QSpinBox@@UAE_NHPAUQUObject@@@Z 10016cbe f   qt-mt323:qt-mt323.dll
 0001:00015cc4       ?qt_emit@QTable@@UAE_NHPAUQUObject@@@Z 10016cc4 f   qt-mt323:qt-mt323.dll
 0001:00015cca       ?qt_emit@QVBoxLayout@@UAE_NHPAUQUObject@@@Z 10016cca f   qt-mt323:qt-mt323.dll
 0001:00015cd0       ?qt_invoke@QComboBox@@UAE_NHPAUQUObject@@@Z 10016cd0 f   qt-mt323:qt-mt323.dll
 0001:00015cd6       ?qt_invoke@QGridLayout@@UAE_NHPAUQUObject@@@Z 10016cd6 f   qt-mt323:qt-mt323.dll
 0001:00015cdc       ?qt_invoke@QHBoxLayout@@UAE_NHPAUQUObject@@@Z 10016cdc f   qt-mt323:qt-mt323.dll
 0001:00015ce2       ?qt_invoke@QLabel@@UAE_NHPAUQUObject@@@Z 10016ce2 f   qt-mt323:qt-mt323.dll
 0001:00015ce8       ?qt_invoke@QLineEdit@@UAE_NHPAUQUObject@@@Z 10016ce8 f   qt-mt323:qt-mt323.dll
 0001:00015cee       ?qt_invoke@QPushButton@@UAE_NHPAUQUObject@@@Z 10016cee f   qt-mt323:qt-mt323.dll
 0001:00015cf4       ?qt_invoke@QSpinBox@@UAE_NHPAUQUObject@@@Z 10016cf4 f   qt-mt323:qt-mt323.dll
 0001:00015cfa       ?qt_invoke@QTable@@UAE_NHPAUQUObject@@@Z 10016cfa f   qt-mt323:qt-mt323.dll
 0001:00015d00       ?qt_invoke@QVBoxLayout@@UAE_NHPAUQUObject@@@Z 10016d00 f   qt-mt323:qt-mt323.dll
 0001:00015d06       ?qt_property@QComboBox@@UAE_NHHPAVQVariant@@@Z 10016d06 f   qt-mt323:qt-mt323.dll
 0001:00015d0c       ?qt_property@QGridLayout@@UAE_NHHPAVQVariant@@@Z 10016d0c f   qt-mt323:qt-mt323.dll
 0001:00015d12       ?qt_property@QHBoxLayout@@UAE_NHHPAVQVariant@@@Z 10016d12 f   qt-mt323:qt-mt323.dll
 0001:00015d18       ?qt_property@QLabel@@UAE_NHHPAVQVariant@@@Z 10016d18 f   qt-mt323:qt-mt323.dll
 0001:00015d1e       ?qt_property@QLineEdit@@UAE_NHHPAVQVariant@@@Z 10016d1e f   qt-mt323:qt-mt323.dll
 0001:00015d24       ?qt_property@QPushButton@@UAE_NHHPAVQVariant@@@Z 10016d24 f   qt-mt323:qt-mt323.dll
 0001:00015d2a       ?qt_property@QSpinBox@@UAE_NHHPAVQVariant@@@Z 10016d2a f   qt-mt323:qt-mt323.dll
 0001:00015d30       ?qt_property@QTable@@UAE_NHHPAVQVariant@@@Z 10016d30 f   qt-mt323:qt-mt323.dll
 0001:00015d36       ?qt_property@QVBoxLayout@@UAE_NHHPAVQVariant@@@Z 10016d36 f   qt-mt323:qt-mt323.dll
 0001:00015d3c       ?rangeChange@QSpinBox@@MAEXXZ 10016d3c f   qt-mt323:qt-mt323.dll
 0001:00015d42       ?redo@QLineEdit@@UAEXXZ    10016d42 f   qt-mt323:qt-mt323.dll
 0001:00015d48       ?removeColumn@QTable@@UAEXH@Z 10016d48 f   qt-mt323:qt-mt323.dll
 0001:00015d4e       ?removeColumns@QTable@@UAEXABV?$QMemArray@H@@@Z 10016d4e f   qt-mt323:qt-mt323.dll
 0001:00015d54       ?removeRow@QTable@@UAEXH@Z 10016d54 f   qt-mt323:qt-mt323.dll
 0001:00015d5a       ?removeRows@QTable@@UAEXABV?$QMemArray@H@@@Z 10016d5a f   qt-mt323:qt-mt323.dll
 0001:00015d60       ?removeSelection@QTable@@UAEXABVQTableSelection@@@Z 10016d60 f   qt-mt323:qt-mt323.dll
 0001:00015d66       ?removeSelection@QTable@@UAEXH@Z 10016d66 f   qt-mt323:qt-mt323.dll
 0001:00015d6c       ?resize@QPushButton@@UAEXHH@Z 10016d6c f   qt-mt323:qt-mt323.dll
 0001:00015d72       ?resizeData@QTable@@MAEXH@Z 10016d72 f   qt-mt323:qt-mt323.dll
 0001:00015d78       ?resizeEvent@QComboBox@@MAEXPAVQResizeEvent@@@Z 10016d78 f   qt-mt323:qt-mt323.dll
 0001:00015d7e       ?resizeEvent@QLabel@@MAEXPAVQResizeEvent@@@Z 10016d7e f   qt-mt323:qt-mt323.dll
 0001:00015d84       ?resizeEvent@QLineEdit@@MAEXPAVQResizeEvent@@@Z 10016d84 f   qt-mt323:qt-mt323.dll
 0001:00015d8a       ?resizeEvent@QPushButton@@MAEXPAVQResizeEvent@@@Z 10016d8a f   qt-mt323:qt-mt323.dll
 0001:00015d90       ?resizeEvent@QScrollView@@MAEXPAVQResizeEvent@@@Z 10016d90 f   qt-mt323:qt-mt323.dll
 0001:00015d96       ?resizeEvent@QSpinBox@@MAEXPAVQResizeEvent@@@Z 10016d96 f   qt-mt323:qt-mt323.dll
 0001:00015d9c       ?rowAt@QTable@@UBEHH@Z     10016d9c f   qt-mt323:qt-mt323.dll
 0001:00015da2       ?rowHeight@QTable@@UBEHH@Z 10016da2 f   qt-mt323:qt-mt323.dll
 0001:00015da8       ?rowHeightChanged@QTable@@MAEXH@Z 10016da8 f   qt-mt323:qt-mt323.dll
 0001:00015dae       ?rowIndexChanged@QTable@@MAEXHHH@Z 10016dae f   qt-mt323:qt-mt323.dll
 0001:00015db4       ?rowPos@QTable@@UBEHH@Z    10016db4 f   qt-mt323:qt-mt323.dll
 0001:00015dba       ?selectAll@QLineEdit@@UAEXXZ 10016dba f   qt-mt323:qt-mt323.dll
 0001:00015dc0       ?selectAll@QSpinBox@@UAEXXZ 10016dc0 f   qt-mt323:qt-mt323.dll
 0001:00015dc6       ?setAccel@QButton@@UAEXABVQKeySequence@@@Z 10016dc6 f   qt-mt323:qt-mt323.dll
 0001:00015dcc       ?setAlignment@QLabel@@UAEXH@Z 10016dcc f   qt-mt323:qt-mt323.dll
 0001:00015dd2       ?setAlignment@QLineEdit@@UAEXH@Z 10016dd2 f   qt-mt323:qt-mt323.dll
 0001:00015dd8       ?setAutoCompletion@QComboBox@@UAEX_N@Z 10016dd8 f   qt-mt323:qt-mt323.dll
 0001:00015dde       ?setAutoDefault@QPushButton@@UAEX_N@Z 10016dde f   qt-mt323:qt-mt323.dll
 0001:00015de4       ?setAutoRepeat@QButton@@UAEX_N@Z 10016de4 f   qt-mt323:qt-mt323.dll
 0001:00015dea       ?setAutoResize@QComboBox@@UAEX_N@Z 10016dea f   qt-mt323:qt-mt323.dll
 0001:00015df0       ?setAutoResize@QLabel@@UAEX_N@Z 10016df0 f   qt-mt323:qt-mt323.dll
 0001:00015df6       ?setBuddy@QLabel@@UAEXPAVQWidget@@@Z 10016df6 f   qt-mt323:qt-mt323.dll
 0001:00015dfc       ?setButtonSymbols@QSpinBox@@UAEXW4ButtonSymbols@1@@Z 10016dfc f   qt-mt323:qt-mt323.dll
 0001:00015e02       ?setCellContentFromEditor@QTable@@MAEXHH@Z 10016e02 f   qt-mt323:qt-mt323.dll
 0001:00015e08       ?setCellWidget@QTable@@UAEXHHPAVQWidget@@@Z 10016e08 f   qt-mt323:qt-mt323.dll
 0001:00015e0e       ?setColStretch@QGridLayout@@UAEXHH@Z 10016e0e f   qt-mt323:qt-mt323.dll
 0001:00015e14       ?setColumnMovingEnabled@QTable@@UAEX_N@Z 10016e14 f   qt-mt323:qt-mt323.dll
 0001:00015e1a       ?setColumnReadOnly@QTable@@UAEXH_N@Z 10016e1a f   qt-mt323:qt-mt323.dll
 0001:00015e20       ?setColumnStretchable@QTable@@UAEXH_N@Z 10016e20 f   qt-mt323:qt-mt323.dll
 0001:00015e26       ?setColumnWidth@QTable@@UAEXHH@Z 10016e26 f   qt-mt323:qt-mt323.dll
 0001:00015e2c       ?setContentsPos@QScrollView@@UAEXHH@Z 10016e2c f   qt-mt323:qt-mt323.dll
 0001:00015e32       ?setCurrentCell@QTable@@UAEXHH@Z 10016e32 f   qt-mt323:qt-mt323.dll
 0001:00015e38       ?setCurrentItem@QComboBox@@UAEXH@Z 10016e38 f   qt-mt323:qt-mt323.dll
 0001:00015e3e       ?setCurrentText@QComboBox@@UAEXABVQString@@@Z 10016e3e f   qt-mt323:qt-mt323.dll
 0001:00015e44       ?setCursorPosition@QLineEdit@@UAEXH@Z 10016e44 f   qt-mt323:qt-mt323.dll
 0001:00015e4a       ?setDefault@QPushButton@@UAEX_N@Z 10016e4a f   qt-mt323:qt-mt323.dll
 0001:00015e50       ?setDown@QButton@@UAEX_N@Z 10016e50 f   qt-mt323:qt-mt323.dll
 0001:00015e56       ?setDragEnabled@QLineEdit@@UAEX_N@Z 10016e56 f   qt-mt323:qt-mt323.dll
 0001:00015e5c       ?setDragEnabled@QTable@@UAEX_N@Z 10016e5c f   qt-mt323:qt-mt323.dll
 0001:00015e62       ?setEchoMode@QLineEdit@@UAEXW4EchoMode@1@@Z 10016e62 f   qt-mt323:qt-mt323.dll
 0001:00015e68       ?setEditText@QComboBox@@UAEXABVQString@@@Z 10016e68 f   qt-mt323:qt-mt323.dll
 0001:00015e6e       ?setEnabled@QComboBox@@UAEX_N@Z 10016e6e f   qt-mt323:qt-mt323.dll
 0001:00015e74       ?setEnabled@QSpinBox@@UAEX_N@Z 10016e74 f   qt-mt323:qt-mt323.dll
 0001:00015e7a       ?setEnabled@QTable@@UAEX_N@Z 10016e7a f   qt-mt323:qt-mt323.dll
 0001:00015e80       ?setFocusStyle@QTable@@UAEXW4FocusStyle@1@@Z 10016e80 f   qt-mt323:qt-mt323.dll
 0001:00015e86       ?setFont@QComboBox@@UAEXABVQFont@@@Z 10016e86 f   qt-mt323:qt-mt323.dll
 0001:00015e8c       ?setFont@QLabel@@UAEXABVQFont@@@Z 10016e8c f   qt-mt323:qt-mt323.dll
 0001:00015e92       ?setFont@QLineEdit@@UAEXABVQFont@@@Z 10016e92 f   qt-mt323:qt-mt323.dll
 0001:00015e98       ?setFrame@QLineEdit@@UAEX_N@Z 10016e98 f   qt-mt323:qt-mt323.dll
 0001:00015e9e       ?setGeometry@QGridLayout@@UAEXABVQRect@@@Z 10016e9e f   qt-mt323:qt-mt323.dll
 0001:00015ea4       ?setGeometry@QPushButton@@UAEXABVQRect@@@Z 10016ea4 f   qt-mt323:qt-mt323.dll
 0001:00015eaa       ?setGeometry@QPushButton@@UAEXHHHH@Z 10016eaa f   qt-mt323:qt-mt323.dll
 0001:00015eb0       ?setGeometry@QSpacerItem@@UAEXABVQRect@@@Z 10016eb0 f   qt-mt323:qt-mt323.dll
 0001:00015eb6       ?setGroup@QButton@@EAEXPAVQButtonGroup@@@Z 10016eb6 f   qt-mt323:qt-mt323.dll
 0001:00015ebc       ?setInsertionPolicy@QComboBox@@UAEXW4Policy@1@@Z 10016ebc f   qt-mt323:qt-mt323.dll
 0001:00015ec2       ?setIsMenuButton@QPushButton@@UAEX_N@Z 10016ec2 f   qt-mt323:qt-mt323.dll
 0001:00015ec8       ?setItem@QTable@@UAEXHHPAVQTableItem@@@Z 10016ec8 f   qt-mt323:qt-mt323.dll
 0001:00015ece       ?setLeftMargin@QTable@@UAEXH@Z 10016ece f   qt-mt323:qt-mt323.dll
 0001:00015ed4       ?setLineEdit@QComboBox@@UAEXPAVQLineEdit@@@Z 10016ed4 f   qt-mt323:qt-mt323.dll
 0001:00015eda       ?setListBox@QComboBox@@UAEXPAVQListBox@@@Z 10016eda f   qt-mt323:qt-mt323.dll
 0001:00015ee0       ?setMaxCount@QComboBox@@UAEXH@Z 10016ee0 f   qt-mt323:qt-mt323.dll
 0001:00015ee6       ?setMaxLength@QLineEdit@@UAEXH@Z 10016ee6 f   qt-mt323:qt-mt323.dll
 0001:00015eec       ?setMovie@QLabel@@UAEXABVQMovie@@@Z 10016eec f   qt-mt323:qt-mt323.dll
 0001:00015ef2       ?setNum@QLabel@@UAEXH@Z    10016ef2 f   qt-mt323:qt-mt323.dll
 0001:00015ef8       ?setNum@QLabel@@UAEXN@Z    10016ef8 f   qt-mt323:qt-mt323.dll
 0001:00015efe       ?setNumCols@QTable@@UAEXH@Z 10016efe f   qt-mt323:qt-mt323.dll
 0001:00015f04       ?setNumRows@QTable@@UAEXH@Z 10016f04 f   qt-mt323:qt-mt323.dll
 0001:00015f0a       ?setOn@QPushButton@@UAEX_N@Z 10016f0a f   qt-mt323:qt-mt323.dll
 0001:00015f10       ?setPalette@QComboBox@@UAEXABVQPalette@@@Z 10016f10 f   qt-mt323:qt-mt323.dll
 0001:00015f16       ?setPalette@QLineEdit@@UAEXABVQPalette@@@Z 10016f16 f   qt-mt323:qt-mt323.dll
 0001:00015f1c       ?setPicture@QLabel@@UAEXABVQPicture@@@Z 10016f1c f   qt-mt323:qt-mt323.dll
 0001:00015f22       ?setPixmap@QButton@@UAEXABVQPixmap@@@Z 10016f22 f   qt-mt323:qt-mt323.dll
 0001:00015f28       ?setPixmap@QLabel@@UAEXABVQPixmap@@@Z 10016f28 f   qt-mt323:qt-mt323.dll
 0001:00015f2e       ?setPixmap@QTable@@UAEXHHABVQPixmap@@@Z 10016f2e f   qt-mt323:qt-mt323.dll
 0001:00015f34       ?setPrefix@QSpinBox@@UAEXABVQString@@@Z 10016f34 f   qt-mt323:qt-mt323.dll
 0001:00015f3a       ?setReadOnly@QLineEdit@@UAEX_N@Z 10016f3a f   qt-mt323:qt-mt323.dll
 0001:00015f40       ?setReadOnly@QTable@@UAEX_N@Z 10016f40 f   qt-mt323:qt-mt323.dll
 0001:00015f46       ?setRowHeight@QTable@@UAEXHH@Z 10016f46 f   qt-mt323:qt-mt323.dll
 0001:00015f4c       ?setRowMovingEnabled@QTable@@UAEX_N@Z 10016f4c f   qt-mt323:qt-mt323.dll
 0001:00015f52       ?setRowReadOnly@QTable@@UAEXH_N@Z 10016f52 f   qt-mt323:qt-mt323.dll
 0001:00015f58       ?setRowStretch@QGridLayout@@UAEXHH@Z 10016f58 f   qt-mt323:qt-mt323.dll
 0001:00015f5e       ?setRowStretchable@QTable@@UAEXH_N@Z 10016f5e f   qt-mt323:qt-mt323.dll
 0001:00015f64       ?setSelection@QLineEdit@@UAEXHH@Z 10016f64 f   qt-mt323:qt-mt323.dll
 0001:00015f6a       ?setSelectionMode@QTable@@UAEXW4SelectionMode@1@@Z 10016f6a f   qt-mt323:qt-mt323.dll
 0001:00015f70       ?setShowGrid@QTable@@UAEX_N@Z 10016f70 f   qt-mt323:qt-mt323.dll
 0001:00015f76       ?setSizeLimit@QComboBox@@UAEXH@Z 10016f76 f   qt-mt323:qt-mt323.dll
 0001:00015f7c       ?setSorting@QTable@@UAEX_N@Z 10016f7c f   qt-mt323:qt-mt323.dll
 0001:00015f82       ?setSpecialValueText@QSpinBox@@UAEXABVQString@@@Z 10016f82 f   qt-mt323:qt-mt323.dll
 0001:00015f88       ?setState@QButton@@MAEXW4ToggleState@1@@Z 10016f88 f   qt-mt323:qt-mt323.dll
 0001:00015f8e       ?setSuffix@QSpinBox@@UAEXABVQString@@@Z 10016f8e f   qt-mt323:qt-mt323.dll
 0001:00015f94       ?setText@QButton@@UAEXABVQString@@@Z 10016f94 f   qt-mt323:qt-mt323.dll
 0001:00015f9a       ?setText@QLabel@@UAEXABVQString@@@Z 10016f9a f   qt-mt323:qt-mt323.dll
 0001:00015fa0       ?setText@QLineEdit@@UAEXABVQString@@@Z 10016fa0 f   qt-mt323:qt-mt323.dll
 0001:00015fa6       ?setText@QTable@@UAEXHHABVQString@@@Z 10016fa6 f   qt-mt323:qt-mt323.dll
 0001:00015fac       ?setToggleType@QButton@@MAEXW4ToggleType@1@@Z 10016fac f   qt-mt323:qt-mt323.dll
 0001:00015fb2       ?setTopMargin@QTable@@UAEXH@Z 10016fb2 f   qt-mt323:qt-mt323.dll
 0001:00015fb8       ?setValidator@QComboBox@@UAEXPBVQValidator@@@Z 10016fb8 f   qt-mt323:qt-mt323.dll
 0001:00015fbe       ?setValidator@QLineEdit@@UAEXPBVQValidator@@@Z 10016fbe f   qt-mt323:qt-mt323.dll
 0001:00015fc4       ?setValidator@QSpinBox@@UAEXPBVQValidator@@@Z 10016fc4 f   qt-mt323:qt-mt323.dll
 0001:00015fca       ?setValue@QSpinBox@@UAEXH@Z 10016fca f   qt-mt323:qt-mt323.dll
 0001:00015fd0       ?setWrapping@QSpinBox@@UAEX_N@Z 10016fd0 f   qt-mt323:qt-mt323.dll
 0001:00015fd6       ?show@QScrollView@@UAEXXZ  10016fd6 f   qt-mt323:qt-mt323.dll
 0001:00015fdc       ?showColumn@QTable@@UAEXH@Z 10016fdc f   qt-mt323:qt-mt323.dll
 0001:00015fe2       ?showEvent@QTable@@MAEXPAVQShowEvent@@@Z 10016fe2 f   qt-mt323:qt-mt323.dll
 0001:00015fe8       ?showRow@QTable@@UAEXH@Z   10016fe8 f   qt-mt323:qt-mt323.dll
 0001:00015fee       ?sizeHint@QComboBox@@UBE?AVQSize@@XZ 10016fee f   qt-mt323:qt-mt323.dll
 0001:00015ff4       ?sizeHint@QGridLayout@@UBE?AVQSize@@XZ 10016ff4 f   qt-mt323:qt-mt323.dll
 0001:00015ffa       ?sizeHint@QLabel@@UBE?AVQSize@@XZ 10016ffa f   qt-mt323:qt-mt323.dll
 0001:00016000       ?sizeHint@QLineEdit@@UBE?AVQSize@@XZ 10017000 f   qt-mt323:qt-mt323.dll
 0001:00016006       ?sizeHint@QPushButton@@UBE?AVQSize@@XZ 10017006 f   qt-mt323:qt-mt323.dll
 0001:0001600c       ?sizeHint@QSpacerItem@@UBE?AVQSize@@XZ 1001700c f   qt-mt323:qt-mt323.dll
 0001:00016012       ?sizeHint@QSpinBox@@UBE?AVQSize@@XZ 10017012 f   qt-mt323:qt-mt323.dll
 0001:00016018       ?sizeHint@QTable@@UBE?AVQSize@@XZ 10017018 f   qt-mt323:qt-mt323.dll
 0001:0001601e       ?sortColumn@QTable@@UAEXH_N0@Z 1001701e f   qt-mt323:qt-mt323.dll
 0001:00016024       ?spacerItem@QSpacerItem@@UAEPAV1@XZ 10017024 f   qt-mt323:qt-mt323.dll
 0001:0001602a       ?startDrag@QTable@@MAEXXZ  1001702a f   qt-mt323:qt-mt323.dll
 0001:00016030       ?stepChange@QRangeControl@@MAEXXZ 10017030 f   qt-mt323:qt-mt323.dll
 0001:00016036       ?stepDown@QSpinBox@@UAEXXZ 10017036 f   qt-mt323:qt-mt323.dll
 0001:0001603c       ?stepUp@QSpinBox@@UAEXXZ   1001703c f   qt-mt323:qt-mt323.dll
 0001:00016042       ?styleChange@QComboBox@@MAEXAAVQStyle@@@Z 10017042 f   qt-mt323:qt-mt323.dll
 0001:00016048       ?styleChange@QScrollView@@UAEXAAVQStyle@@@Z 10017048 f   qt-mt323:qt-mt323.dll
 0001:0001604e       ?styleChange@QSpinBox@@MAEXAAVQStyle@@@Z 1001704e f   qt-mt323:qt-mt323.dll
 0001:00016054       ?suffix@QSpinBox@@UBE?AVQString@@XZ 10017054 f   qt-mt323:qt-mt323.dll
 0001:0001605a       ?swapCells@QTable@@UAEXHHHH@Z 1001705a f   qt-mt323:qt-mt323.dll
 0001:00016060       ?swapColumns@QTable@@UAEXHH_N@Z 10017060 f   qt-mt323:qt-mt323.dll
 0001:00016066       ?swapRows@QTable@@UAEXHH_N@Z 10017066 f   qt-mt323:qt-mt323.dll
 0001:0001606c       ?takeItem@QTable@@UAEXPAVQTableItem@@@Z 1001706c f   qt-mt323:qt-mt323.dll
 0001:00016072       ?text@QTable@@UBE?AVQString@@HH@Z 10017072 f   qt-mt323:qt-mt323.dll
 0001:00016078       ?undo@QLineEdit@@UAEXXZ    10017078 f   qt-mt323:qt-mt323.dll
 0001:0001607e       ?updateDisplay@QSpinBox@@MAEXXZ 1001707e f   qt-mt323:qt-mt323.dll
 0001:00016084       ?updateMask@QComboBox@@MAEXXZ 10017084 f   qt-mt323:qt-mt323.dll
 0001:0001608a       ?updateMask@QPushButton@@MAEXXZ 1001708a f   qt-mt323:qt-mt323.dll
 0001:00016090       ?valueChange@QSpinBox@@MAEXXZ 10017090 f   qt-mt323:qt-mt323.dll
 0001:00016096       ?viewportResizeEvent@QTable@@MAEXPAVQResizeEvent@@@Z 10017096 f   qt-mt323:qt-mt323.dll
 0001:0001609c       ?wheelEvent@QComboBox@@MAEXPAVQWheelEvent@@@Z 1001709c f   qt-mt323:qt-mt323.dll
 0001:000160a2       ?wheelEvent@QSpinBox@@MAEXPAVQWheelEvent@@@Z 100170a2 f   qt-mt323:qt-mt323.dll
 0001:000160a8       ?windowActivationChange@QLineEdit@@MAEX_N@Z 100170a8 f   qt-mt323:qt-mt323.dll
 0001:000160ae       ?windowActivationChange@QTable@@MAEX_N@Z 100170ae f   qt-mt323:qt-mt323.dll
 0001:000160b4       ?alignment@QTableItem@@UBEHXZ 100170b4 f   qt-mt323:qt-mt323.dll
 0001:000160ba       ?createEditor@QCheckTableItem@@UBEPAVQWidget@@XZ 100170ba f   qt-mt323:qt-mt323.dll
 0001:000160c0       ?key@QTableItem@@UBE?AVQString@@XZ 100170c0 f   qt-mt323:qt-mt323.dll
 0001:000160c6       ?paint@QCheckTableItem@@UAEXPAVQPainter@@ABVQColorGroup@@ABVQRect@@_N@Z 100170c6 f   qt-mt323:qt-mt323.dll
 0001:000160cc       ?pixmap@QTableItem@@UBE?AVQPixmap@@XZ 100170cc f   qt-mt323:qt-mt323.dll
 0001:000160d2       ?rtti@QCheckTableItem@@UBEHXZ 100170d2 f   qt-mt323:qt-mt323.dll
 0001:000160d8       ?setChecked@QCheckTableItem@@UAEX_N@Z 100170d8 f   qt-mt323:qt-mt323.dll
 0001:000160de       ?setCol@QTableItem@@UAEXH@Z 100170de f   qt-mt323:qt-mt323.dll
 0001:000160e4       ?setContentFromEditor@QCheckTableItem@@UAEXPAVQWidget@@@Z 100170e4 f   qt-mt323:qt-mt323.dll
 0001:000160ea       ?setEnabled@QTableItem@@UAEX_N@Z 100170ea f   qt-mt323:qt-mt323.dll
 0001:000160f0       ?setPixmap@QTableItem@@UAEXABVQPixmap@@@Z 100170f0 f   qt-mt323:qt-mt323.dll
 0001:000160f6       ?setReplaceable@QTableItem@@UAEX_N@Z 100170f6 f   qt-mt323:qt-mt323.dll
 0001:000160fc       ?setRow@QTableItem@@UAEXH@Z 100170fc f   qt-mt323:qt-mt323.dll
 0001:00016102       ?setSpan@QTableItem@@UAEXHH@Z 10017102 f   qt-mt323:qt-mt323.dll
 0001:00016108       ?setText@QCheckTableItem@@UAEXABVQString@@@Z 10017108 f   qt-mt323:qt-mt323.dll
 0001:0001610e       ?setWordWrap@QTableItem@@UAEX_N@Z 1001710e f   qt-mt323:qt-mt323.dll
 0001:00016114       ?sizeHint@QCheckTableItem@@UBE?AVQSize@@XZ 10017114 f   qt-mt323:qt-mt323.dll
 0001:0001611a       ?text@QTableItem@@UBE?AVQString@@XZ 1001711a f   qt-mt323:qt-mt323.dll
 0001:00016120       ?childEvent@QGroupBox@@MAEXPAVQChildEvent@@@Z 10017120 f   qt-mt323:qt-mt323.dll
 0001:00016126       ?className@QButtonGroup@@UBEPBDXZ 10017126 f   qt-mt323:qt-mt323.dll
 0001:0001612c       ?className@QGroupBox@@UBEPBDXZ 1001712c f   qt-mt323:qt-mt323.dll
 0001:00016132       ?className@QRadioButton@@UBEPBDXZ 10017132 f   qt-mt323:qt-mt323.dll
 0001:00016138       ?drawButton@QRadioButton@@MAEXPAVQPainter@@@Z 10017138 f   qt-mt323:qt-mt323.dll
 0001:0001613e       ?drawButtonLabel@QRadioButton@@MAEXPAVQPainter@@@Z 1001713e f   qt-mt323:qt-mt323.dll
 0001:00016144       ?event@QButtonGroup@@MAE_NPAVQEvent@@@Z 10017144 f   qt-mt323:qt-mt323.dll
 0001:0001614a       ?event@QGroupBox@@MAE_NPAVQEvent@@@Z 1001714a f   qt-mt323:qt-mt323.dll
 0001:00016150       ?focusInEvent@QButton@@MAEXPAVQFocusEvent@@@Z 10017150 f   qt-mt323:qt-mt323.dll
 0001:00016156       ?focusInEvent@QGroupBox@@MAEXPAVQFocusEvent@@@Z 10017156 f   qt-mt323:qt-mt323.dll
 0001:0001615c       ?focusOutEvent@QButton@@MAEXPAVQFocusEvent@@@Z 1001715c f   qt-mt323:qt-mt323.dll
 0001:00016162       ?fontChange@QGroupBox@@MAEXABVQFont@@@Z 10017162 f   qt-mt323:qt-mt323.dll
 0001:00016168       ?hitButton@QRadioButton@@MBE_NABVQPoint@@@Z 10017168 f   qt-mt323:qt-mt323.dll
 0001:0001616e       ?metaObject@QButtonGroup@@UBEPAVQMetaObject@@XZ 1001716e f   qt-mt323:qt-mt323.dll
 0001:00016174       ?metaObject@QGroupBox@@UBEPAVQMetaObject@@XZ 10017174 f   qt-mt323:qt-mt323.dll
 0001:0001617a       ?metaObject@QRadioButton@@UBEPAVQMetaObject@@XZ 1001717a f   qt-mt323:qt-mt323.dll
 0001:00016180       ?moveFocus@QButtonGroup@@UAEXH@Z 10017180 f   qt-mt323:qt-mt323.dll
 0001:00016186       ?paintEvent@QGroupBox@@MAEXPAVQPaintEvent@@@Z 10017186 f   qt-mt323:qt-mt323.dll
 0001:0001618c       ?qt_cast@QButtonGroup@@UAEPAXPBD@Z 1001718c f   qt-mt323:qt-mt323.dll
 0001:00016192       ?qt_cast@QGroupBox@@UAEPAXPBD@Z 10017192 f   qt-mt323:qt-mt323.dll
 0001:00016198       ?qt_cast@QRadioButton@@UAEPAXPBD@Z 10017198 f   qt-mt323:qt-mt323.dll
 0001:0001619e       ?qt_emit@QButtonGroup@@UAE_NHPAUQUObject@@@Z 1001719e f   qt-mt323:qt-mt323.dll
 0001:000161a4       ?qt_emit@QGroupBox@@UAE_NHPAUQUObject@@@Z 100171a4 f   qt-mt323:qt-mt323.dll
 0001:000161aa       ?qt_emit@QRadioButton@@UAE_NHPAUQUObject@@@Z 100171aa f   qt-mt323:qt-mt323.dll
 0001:000161b0       ?qt_invoke@QButtonGroup@@UAE_NHPAUQUObject@@@Z 100171b0 f   qt-mt323:qt-mt323.dll
 0001:000161b6       ?qt_invoke@QGroupBox@@UAE_NHPAUQUObject@@@Z 100171b6 f   qt-mt323:qt-mt323.dll
 0001:000161bc       ?qt_invoke@QRadioButton@@UAE_NHPAUQUObject@@@Z 100171bc f   qt-mt323:qt-mt323.dll
 0001:000161c2       ?qt_property@QButtonGroup@@UAE_NHHPAVQVariant@@@Z 100171c2 f   qt-mt323:qt-mt323.dll
 0001:000161c8       ?qt_property@QGroupBox@@UAE_NHHPAVQVariant@@@Z 100171c8 f   qt-mt323:qt-mt323.dll
 0001:000161ce       ?qt_property@QRadioButton@@UAE_NHHPAVQVariant@@@Z 100171ce f   qt-mt323:qt-mt323.dll
 0001:000161d4       ?resizeEvent@QGroupBox@@MAEXPAVQResizeEvent@@@Z 100171d4 f   qt-mt323:qt-mt323.dll
 0001:000161da       ?resizeEvent@QRadioButton@@MAEXPAVQResizeEvent@@@Z 100171da f   qt-mt323:qt-mt323.dll
 0001:000161e0       ?setAlignment@QGroupBox@@UAEXH@Z 100171e0 f   qt-mt323:qt-mt323.dll
 0001:000161e6       ?setButton@QButtonGroup@@UAEXH@Z 100171e6 f   qt-mt323:qt-mt323.dll
 0001:000161ec       ?setChecked@QRadioButton@@UAEX_N@Z 100171ec f   qt-mt323:qt-mt323.dll
 0001:000161f2       ?setColumnLayout@QGroupBox@@UAEXHW4Orientation@Qt@@@Z 100171f2 f   qt-mt323:qt-mt323.dll
 0001:000161f8       ?setEnabled@QGroupBox@@UAEX_N@Z 100171f8 f   qt-mt323:qt-mt323.dll
 0001:000161fe       ?setExclusive@QButtonGroup@@UAEX_N@Z 100171fe f   qt-mt323:qt-mt323.dll
 0001:00016204       ?setRadioButtonExclusive@QButtonGroup@@UAEX_N@Z 10017204 f   qt-mt323:qt-mt323.dll
 0001:0001620a       ?setTitle@QGroupBox@@UAEXABVQString@@@Z 1001720a f   qt-mt323:qt-mt323.dll
 0001:00016210       ?sizeHint@QGroupBox@@UBE?AVQSize@@XZ 10017210 f   qt-mt323:qt-mt323.dll
 0001:00016216       ?sizeHint@QRadioButton@@UBE?AVQSize@@XZ 10017216 f   qt-mt323:qt-mt323.dll
 0001:0001621c       ?updateMask@QRadioButton@@MAEXXZ 1001721c f   qt-mt323:qt-mt323.dll
 0001:00016222       ?loadState@cfg_Settings@@SA?AVQString@@ABV2@@Z 10017222 f   cfg_widgets001:cfg_Settings.obj
 0001:000162b4       ?loadState@cfg_Settings@@SAXAAVQPoint@@AAVQSize@@AA_NABVQString@@@Z 100172b4 f   cfg_widgets001:cfg_Settings.obj
 0001:000163ad       ?loadState@cfg_Settings@@SAXQAVQListView@@ABVQString@@@Z 100173ad f   cfg_widgets001:cfg_Settings.obj
 0001:000164aa       ?loadState@cfg_Settings@@SAXQAVQTable@@ABVQString@@@Z 100174aa f   cfg_widgets001:cfg_Settings.obj
 0001:00016597       ?saveState@cfg_Settings@@SAXABVQPoint@@ABVQSize@@AB_NABVQString@@@Z 10017597 f   cfg_widgets001:cfg_Settings.obj
 0001:000166b1       ?saveState@cfg_Settings@@SAXABVQString@@0@Z 100176b1 f   cfg_widgets001:cfg_Settings.obj
 0001:0001672d       ?saveState@cfg_Settings@@SAXQBVQListView@@ABVQString@@@Z 1001772d f   cfg_widgets001:cfg_Settings.obj
 0001:00016805       ?saveState@cfg_Settings@@SAXQBVQTable@@ABVQString@@@Z 10017805 f   cfg_widgets001:cfg_Settings.obj
 0001:000168e4       ?className@CAlm_sys_select@@UBEPBDXZ 100178e4 f   alm_sys_select:alm_sys_select.dll
 0001:000168ea       ?metaObject@CAlm_sys_select@@UBEPAVQMetaObject@@XZ 100178ea f   alm_sys_select:alm_sys_select.dll
 0001:000168f0       ?qt_cast@CAlm_sys_select@@UAEPAXPBD@Z 100178f0 f   alm_sys_select:alm_sys_select.dll
 0001:000168f6       ?qt_emit@CAlm_sys_select@@UAE_NHPAUQUObject@@@Z 100178f6 f   alm_sys_select:alm_sys_select.dll
 0001:000168fc       ?qt_invoke@CAlm_sys_select@@UAE_NHPAUQUObject@@@Z 100178fc f   alm_sys_select:alm_sys_select.dll
 0001:00016902       ?qt_property@CAlm_sys_select@@UAE_NHHPAVQVariant@@@Z 10017902 f   alm_sys_select:alm_sys_select.dll
 0001:00016910       ??0Document@@QAE@ABVQString@@@Z 10017910 f   config_alarm_utilities:Document.obj
 0001:00016930       ??0Document_BncsSystem@@QAE@XZ 10017930 f   config_alarm_utilities:Document.obj
 0001:000169c0       ??1Document@@UAE@XZ        100179c0 f   config_alarm_utilities:Document.obj
 0001:000169d0       ??1Document_BncsSystem@@UAE@XZ 100179d0 f   config_alarm_utilities:Document.obj
 0001:000169e0       ??_GDocument@@UAEPAXI@Z    100179e0 f i config_alarm_utilities:Document.obj
 0001:000169e0       ??_EDocument@@UAEPAXI@Z    100179e0 f i config_alarm_utilities:Document.obj
 0001:00016a10       ??_EDocument_BncsSystem@@UAEPAXI@Z 10017a10 f i config_alarm_utilities:Document.obj
 0001:00016a10       ??_GDocument_BncsSystem@@UAEPAXI@Z 10017a10 f i config_alarm_utilities:Document.obj
 0001:00016a40       ?getMaxDevice@Document_BncsSystem@@QBEHXZ 10017a40 f   config_alarm_utilities:Document.obj
 0001:00016a50       ?getMaxSlot@Document_BncsSystem@@QBEHXZ 10017a50 f   config_alarm_utilities:Document.obj
 0001:00016a60       ?count@?$QDict@VdevTemplate@@@@UBEIXZ 10017a60 f   devTemplate.obj
 0001:00016a60       ?getMaxWorkstation@Document_BncsSystem@@QBEHXZ 10017a60 f   config_alarm_utilities:Document.obj
 0001:00016a70       ?load@Document_BncsSystem@@QAE_NXZ 10017a70 f   config_alarm_utilities:Document.obj
 0001:00016b70       ??0FileLoad@@IAE@ABVQString@@@Z 10017b70 f   config_alarm_utilities:Loaders.obj
 0001:00016be0       ??0Loaders@@QAE@XZ         10017be0 f   config_alarm_utilities:Loaders.obj
 0001:00016c60       ??1?$QPtrList@VDirLoad@@@@UAE@XZ 10017c60 f i config_alarm_utilities:Loaders.obj
 0001:00016cc0       ??1?$QPtrList@VFileLoad@@@@UAE@XZ 10017cc0 f i config_alarm_utilities:Loaders.obj
 0001:00016d20       ??1FileLoad@@UAE@XZ        10017d20 f   config_alarm_utilities:Loaders.obj
 0001:00016d80       ??1Loaders@@UAE@XZ         10017d80 f   config_alarm_utilities:Loaders.obj
 0001:00016e30       ??_E?$QPtrList@VDirLoad@@@@UAEPAXI@Z 10017e30 f i config_alarm_utilities:Loaders.obj
 0001:00016e30       ??_G?$QPtrList@VDirLoad@@@@UAEPAXI@Z 10017e30 f i config_alarm_utilities:Loaders.obj
 0001:00016ea0       ??_G?$QPtrList@VFileLoad@@@@UAEPAXI@Z 10017ea0 f i config_alarm_utilities:Loaders.obj
 0001:00016ea0       ??_E?$QPtrList@VFileLoad@@@@UAEPAXI@Z 10017ea0 f i config_alarm_utilities:Loaders.obj
 0001:00016f10       ??_GFileLoad@@UAEPAXI@Z    10017f10 f i config_alarm_utilities:Loaders.obj
 0001:00016f10       ??_EFileLoad@@UAEPAXI@Z    10017f10 f i config_alarm_utilities:Loaders.obj
 0001:00016f40       ??_GLoaders@@UAEPAXI@Z     10017f40 f i config_alarm_utilities:Loaders.obj
 0001:00016f40       ??_ELoaders@@UAEPAXI@Z     10017f40 f i config_alarm_utilities:Loaders.obj
 0001:00016f70       ?append@Loaders@@QAEXPAVFileLoad@@@Z 10017f70 f   config_alarm_utilities:Loaders.obj
 0001:00016f80       ?deleteItem@?$QPtrList@VFileLoad@@@@EAEXPAX@Z 10017f80 f i config_alarm_utilities:Loaders.obj
 0001:00016f80       ?deleteItem@?$QPtrList@VDirLoad@@@@EAEXPAX@Z 10017f80 f i config_alarm_utilities:Loaders.obj
 0001:00016fa0       ?fileName@FileLoad@@QBE?AVQString@@XZ 10017fa0 f   config_alarm_utilities:Loaders.obj
 0001:00016fd0       ?got@FileLoad@@QBE_NXZ     10017fd0 f   config_alarm_utilities:Loaders.obj
 0001:00016fe0       ?lock@FileLoad@@UAEXABVQString@@@Z 10017fe0 f   config_alarm_utilities:Loaders.obj
 0001:00016fe0       ?activate@config_plugin_base@@UAEX_N@Z 10017fe0 f   alm_bncs_output.obj
 0001:00016fe0       ?reply@config_plugin_base@@UAEXPAVresponse@@@Z 10017fe0 f   alm_bncs_output.obj
 0001:00016ff0       ?matches@FileLoad@@QAE_NABVQString@@@Z 10017ff0 f   config_alarm_utilities:Loaders.obj
 0001:000170a0       ?request@FileLoad@@QAEXPAVISendCommand@@@Z 100180a0 f   config_alarm_utilities:Loaders.obj
 0001:00017130       ?resetNameRead@FileLoad@@QAEXABVQString@@@Z 10018130 f   config_alarm_utilities:Loaders.obj
 0001:00017140       ?setGot@FileLoad@@QAEXXZ   10018140 f   config_alarm_utilities:Loaders.obj
 0001:00017146       __purecall                 10018146 f   MSVCRT:MSVCR120.dll
 0001:0001714c       ??2@YAPAXI@Z               1001814c f   MSVCRT:MSVCR120.dll
 0001:00017152       ??3@YAXPAX@Z               10018152 f   MSVCRT:MSVCR120.dll
 0001:00017158       ___atonexitinit            10018158 f   MSVCRT:atonexit.obj
 0001:00017194       __onexit                   10018194 f   MSVCRT:atonexit.obj
 0001:0001723d       _atexit                    1001823d f   MSVCRT:atonexit.obj
 0001:00017252       @__security_check_cookie@4 10018252 f   MSVCRT:secchk.obj
 0001:00017261       __EH_epilog3               10018261 f   MSVCRT:ehprolg3.obj
 0001:00017275       __EH_epilog3_GS            10018275 f   MSVCRT:ehprolg3.obj
 0001:00017284       __EH_prolog3               10018284 f   MSVCRT:ehprolg3.obj
 0001:000172b7       __EH_prolog3_GS            100182b7 f   MSVCRT:ehprolg3.obj
 0001:000172ee       ___CxxFrameHandler3        100182ee f   MSVCRT:MSVCR120.dll
 0001:000172f4       ??_Etype_info@@UAEPAXI@Z   100182f4 f i MSVCRT:ti_inst.obj
 0001:00017340       ??_L@YGXPAXIHP6EX0@Z1@Z    10018340 f   MSVCRT:ehvecctr.obj
 0001:000173a2       ??_M@YGXPAXIHP6EX0@Z@Z     100183a2 f   MSVCRT:ehvecdtr.obj
 0001:00017411       ?__ArrayUnwind@@YGXPAXIHP6EX0@Z@Z 10018411 f   MSVCRT:ehvecdtr.obj
 0001:000174bb       __CRT_INIT@12              100184bb f   MSVCRT:crtdll.obj
 0001:000176b2       __DllMainCRTStartup@12     100186b2 f   MSVCRT:crtdll.obj
 0001:00017808       __lock                     10018808 f   MSVCRT:MSVCR120.dll
 0001:0001780e       __unlock                   1001880e f   MSVCRT:MSVCR120.dll
 0001:00017814       ___dllonexit               10018814 f   MSVCRT:MSVCR120.dll
 0001:00017820       __SEH_prolog4              10018820 f   MSVCRT:sehprolg4.obj
 0001:00017865       __SEH_epilog4              10018865 f   MSVCRT:sehprolg4.obj
 0001:00017879       __except_handler4          10018879 f   MSVCRT:chandler4gs.obj
 0001:0001789c       ___raise_securityfailure   1001889c f   MSVCRT:gs_report.obj
 0001:000178d9       ___report_gsfailure        100188d9 f   MSVCRT:gs_report.obj
 0001:000179d4       ??1type_info@@UAE@XZ       100189d4 f   MSVCRT:MSVCR120.dll
 0001:000179da       ?terminate@@YAXXZ          100189da f   MSVCRT:MSVCR120.dll
 0001:000179e0       ___CppXcptFilter           100189e0 f   MSVCRT:MSVCR120.dll
 0001:000179e6       __amsg_exit                100189e6 f   MSVCRT:MSVCR120.dll
 0001:000179f0       __FindPESection            100189f0 f   MSVCRT:pesect.obj
 0001:00017a40       __IsNonwritableInCurrentImage 10018a40 f   MSVCRT:pesect.obj
 0001:00017b00       __ValidateImageBase        10018b00 f   MSVCRT:pesect.obj
 0001:00017b31       ___security_init_cookie    10018b31 f   MSVCRT:gs_support.obj
 0001:00017bcd       _DllMain@12                10018bcd f   MSVCRT:dllmain.obj
 0001:00017bef       __RTC_Initialize           10018bef f   MSVCRT:initsect.obj
 0001:00017c0f       __RTC_Terminate            10018c0f f   MSVCRT:initsect.obj
 0001:00017c30       __initterm                 10018c30 f   MSVCRT:MSVCR120.dll
 0001:00017c36       __initterm_e               10018c36 f   MSVCRT:MSVCR120.dll
 0001:00017c3c       ___clean_type_info_names   10018c3c f   MSVCRT:tncleanup.obj
 0001:00017c48       __except_handler4_common   10018c48 f   MSVCRT:MSVCR120.dll
 0001:00017c4e       __crt_debugger_hook        10018c4e f   MSVCRT:MSVCR120.dll
 0001:00017c54       ___crtUnhandledException   10018c54 f   MSVCRT:MSVCR120.dll
 0001:00017c5a       ___crtTerminateProcess     10018c5a f   MSVCRT:MSVCR120.dll
 0001:00017c60       ___clean_type_info_names_internal 10018c60 f   MSVCRT:MSVCR120.dll
 0001:00017c66       _IsProcessorFeaturePresent@4 10018c66 f   kernel32:KERNEL32.dll
 0002:00000000       __imp__DisableThreadLibraryCalls@4 1001e000     kernel32:KERNEL32.dll
 0002:00000004       __imp__GetSystemTimeAsFileTime@4 1001e004     kernel32:KERNEL32.dll
 0002:00000008       __imp__GetCurrentThreadId@0 1001e008     kernel32:KERNEL32.dll
 0002:0000000c       __imp__GetCurrentProcessId@0 1001e00c     kernel32:KERNEL32.dll
 0002:00000010       __imp__QueryPerformanceCounter@4 1001e010     kernel32:KERNEL32.dll
 0002:00000014       __imp__IsProcessorFeaturePresent@4 1001e014     kernel32:KERNEL32.dll
 0002:00000018       __imp__IsDebuggerPresent@0 1001e018     kernel32:KERNEL32.dll
 0002:0000001c       __imp__DecodePointer@4     1001e01c     kernel32:KERNEL32.dll
 0002:00000020       __imp__EncodePointer@4     1001e020     kernel32:KERNEL32.dll
 0002:00000024       __imp__GetPrivateProfileStringA@24 1001e024     kernel32:KERNEL32.dll
 0002:00000028       \177KERNEL32_NULL_THUNK_DATA 1001e028     kernel32:KERNEL32.dll
 0002:0000002c       __imp_?_Xlength_error@std@@YAXPBD@Z 1001e02c     msvcprt:MSVCP120.dll
 0002:00000030       __imp_?_Xbad_alloc@std@@YAXXZ 1001e030     msvcprt:MSVCP120.dll
 0002:00000034       \177MSVCP120_NULL_THUNK_DATA 1001e034     msvcprt:MSVCP120.dll
 0002:00000038       __imp___crt_debugger_hook  1001e038     MSVCRT:MSVCR120.dll
 0002:0000003c       __imp___except_handler4_common 1001e03c     MSVCRT:MSVCR120.dll
 0002:00000040       __imp___initterm_e         1001e040     MSVCRT:MSVCR120.dll
 0002:00000044       __imp___initterm           1001e044     MSVCRT:MSVCR120.dll
 0002:00000048       __imp___malloc_crt         1001e048     MSVCRT:MSVCR120.dll
 0002:0000004c       __imp__free                1001e04c     MSVCRT:MSVCR120.dll
 0002:00000050       __imp____crtUnhandledException 1001e050     MSVCRT:MSVCR120.dll
 0002:00000054       __imp____CppXcptFilter     1001e054     MSVCRT:MSVCR120.dll
 0002:00000058       __imp_?terminate@@YAXXZ    1001e058     MSVCRT:MSVCR120.dll
 0002:0000005c       __imp_??1type_info@@UAE@XZ 1001e05c     MSVCRT:MSVCR120.dll
 0002:00000060       __imp___onexit             1001e060     MSVCRT:MSVCR120.dll
 0002:00000064       __imp____crtTerminateProcess 1001e064     MSVCRT:MSVCR120.dll
 0002:00000068       __imp___calloc_crt         1001e068     MSVCRT:MSVCR120.dll
 0002:0000006c       __imp___unlock             1001e06c     MSVCRT:MSVCR120.dll
 0002:00000070       __imp___lock               1001e070     MSVCRT:MSVCR120.dll
 0002:00000074       __imp__memmove             1001e074     MSVCRT:MSVCR120.dll
 0002:00000078       __imp____CxxFrameHandler3  1001e078     MSVCRT:MSVCR120.dll
 0002:0000007c       __imp__atoi                1001e07c     MSVCRT:MSVCR120.dll
 0002:00000080       __imp_??3@YAXPAX@Z         1001e080     MSVCRT:MSVCR120.dll
 0002:00000084       __imp_??2@YAPAXI@Z         1001e084     MSVCRT:MSVCR120.dll
 0002:00000088       __imp___purecall           1001e088     MSVCRT:MSVCR120.dll
 0002:0000008c       __imp____dllonexit         1001e08c     MSVCRT:MSVCR120.dll
 0002:00000090       __imp____clean_type_info_names_internal 1001e090     MSVCRT:MSVCR120.dll
 0002:00000094       __imp___amsg_exit          1001e094     MSVCRT:MSVCR120.dll
 0002:00000098       \177MSVCR120_NULL_THUNK_DATA 1001e098     MSVCRT:MSVCR120.dll
 0002:0000009c       __imp_?metaObject@CAlm_sys_select@@UBEPAVQMetaObject@@XZ 1001e09c     alm_sys_select:alm_sys_select.dll
 0002:000000a0       __imp_?qt_property@CAlm_sys_select@@UAE_NHHPAVQVariant@@@Z 1001e0a0     alm_sys_select:alm_sys_select.dll
 0002:000000a4       __imp_?qt_invoke@CAlm_sys_select@@UAE_NHPAUQUObject@@@Z 1001e0a4     alm_sys_select:alm_sys_select.dll
 0002:000000a8       __imp_?qt_emit@CAlm_sys_select@@UAE_NHPAUQUObject@@@Z 1001e0a8     alm_sys_select:alm_sys_select.dll
 0002:000000ac       __imp_?qt_cast@CAlm_sys_select@@UAEPAXPBD@Z 1001e0ac     alm_sys_select:alm_sys_select.dll
 0002:000000b0       __imp_?getSystemName@CAlm_sys_select@@QAE?AVQString@@XZ 1001e0b0     alm_sys_select:alm_sys_select.dll
 0002:000000b4       __imp_?className@CAlm_sys_select@@UBEPBDXZ 1001e0b4     alm_sys_select:alm_sys_select.dll
 0002:000000b8       __imp_??1CAlm_sys_select@@UAE@XZ 1001e0b8     alm_sys_select:alm_sys_select.dll
 0002:000000bc       __imp_??0CAlm_sys_select@@QAE@PAVQWidget@@PBD@Z 1001e0bc     alm_sys_select:alm_sys_select.dll
 0002:000000c0       __imp_?setSystemNames@CAlm_sys_select@@QAE_NVQString@@@Z 1001e0c0     alm_sys_select:alm_sys_select.dll
 0002:000000c4       \177alm_sys_select_NULL_THUNK_DATA 1001e0c4     alm_sys_select:alm_sys_select.dll
 0002:000000c8       __imp_?fnConfig_icons@@YAPAPBDPBD@Z 1001e0c8     config_icons:config_icons.dll
 0002:000000cc       \177config_icons_NULL_THUNK_DATA 1001e0cc     config_icons:config_icons.dll
 0002:000000d0       __imp_?setDevice@QTextStream@@QAEXPAVQIODevice@@@Z 1001e0d0     qt-mt323:qt-mt323.dll
 0002:000000d4       __imp_?atEnd@QTextStream@@QBE_NXZ 1001e0d4     qt-mt323:qt-mt323.dll
 0002:000000d8       __imp_??6QTextStream@@QAEAAV0@PBD@Z 1001e0d8     qt-mt323:qt-mt323.dll
 0002:000000dc       __imp_??6QTextStream@@QAEAAV0@ABVQString@@@Z 1001e0dc     qt-mt323:qt-mt323.dll
 0002:000000e0       __imp_?readLine@QTextStream@@QAE?AVQString@@XZ 1001e0e0     qt-mt323:qt-mt323.dll
 0002:000000e4       __imp_?begin@?$QValueList@VQString@@@@QAE?AV?$QValueListIterator@VQString@@@@XZ 1001e0e4     qt-mt323:qt-mt323.dll
 0002:000000e8       __imp_?begin@?$QValueList@VQString@@@@QBE?AV?$QValueListConstIterator@VQString@@@@XZ 1001e0e8     qt-mt323:qt-mt323.dll
 0002:000000ec       __imp_?end@?$QValueList@VQString@@@@QBE?AV?$QValueListConstIterator@VQString@@@@XZ 1001e0ec     qt-mt323:qt-mt323.dll
 0002:000000f0       __imp_?remove@?$QValueList@VQString@@@@QAEIABVQString@@@Z 1001e0f0     qt-mt323:qt-mt323.dll
 0002:000000f4       __imp_?clear@?$QValueList@VQString@@@@QAEXXZ 1001e0f4     qt-mt323:qt-mt323.dll
 0002:000000f8       __imp_?append@?$QValueList@VQString@@@@QAE?AV?$QValueListIterator@VQString@@@@ABVQString@@@Z 1001e0f8     qt-mt323:qt-mt323.dll
 0002:000000fc       __imp_??A?$QValueList@VQString@@@@QAEAAVQString@@I@Z 1001e0fc     qt-mt323:qt-mt323.dll
 0002:00000100       __imp_?contains@?$QValueList@VQString@@@@QBEIABVQString@@@Z 1001e100     qt-mt323:qt-mt323.dll
 0002:00000104       __imp_?detach@?$QValueList@VQString@@@@IAEXXZ 1001e104     qt-mt323:qt-mt323.dll
 0002:00000108       __imp_?detachInternal@?$QValueList@VQString@@@@AAEXXZ 1001e108     qt-mt323:qt-mt323.dll
 0002:0000010c       __imp_?rebalance@QMapPrivateBase@@QAEXPAUQMapNodeBase@@AAPAU2@@Z 1001e10c     qt-mt323:qt-mt323.dll
 0002:00000110       __imp_??0?$QMap@VQString@@V1@@@QAE@XZ 1001e110     qt-mt323:qt-mt323.dll
 0002:00000114       __imp_??1?$QMap@VQString@@V1@@@QAE@XZ 1001e114     qt-mt323:qt-mt323.dll
 0002:00000118       __imp_?begin@?$QMap@VQString@@V1@@@QAE?AV?$QMapIterator@VQString@@V1@@@XZ 1001e118     qt-mt323:qt-mt323.dll
 0002:0000011c       __imp_?end@?$QMap@VQString@@V1@@@QAE?AV?$QMapIterator@VQString@@V1@@@XZ 1001e11c     qt-mt323:qt-mt323.dll
 0002:00000120       __imp_?end@?$QMap@VQString@@V1@@@QBE?AV?$QMapConstIterator@VQString@@V1@@@XZ 1001e120     qt-mt323:qt-mt323.dll
 0002:00000124       __imp_?erase@?$QMap@VQString@@V1@@@QAEXV?$QMapIterator@VQString@@V1@@@@Z 1001e124     qt-mt323:qt-mt323.dll
 0002:00000128       __imp_?find@?$QMap@VQString@@V1@@@QAE?AV?$QMapIterator@VQString@@V1@@@ABVQString@@@Z 1001e128     qt-mt323:qt-mt323.dll
 0002:0000012c       __imp_?find@?$QMap@VQString@@V1@@@QBE?AV?$QMapConstIterator@VQString@@V1@@@ABVQString@@@Z 1001e12c     qt-mt323:qt-mt323.dll
 0002:00000130       __imp_?insert@?$QMap@VQString@@V1@@@QAE?AV?$QMapIterator@VQString@@V1@@@ABVQString@@0_N@Z 1001e130     qt-mt323:qt-mt323.dll
 0002:00000134       __imp_??1?$QMap@VQString@@H@@QAE@XZ 1001e134     qt-mt323:qt-mt323.dll
 0002:00000138       __imp_?begin@?$QMap@VQString@@H@@QAE?AV?$QMapIterator@VQString@@H@@XZ 1001e138     qt-mt323:qt-mt323.dll
 0002:0000013c       __imp_?end@?$QMap@VQString@@H@@QAE?AV?$QMapIterator@VQString@@H@@XZ 1001e13c     qt-mt323:qt-mt323.dll
 0002:00000140       __imp_?connect@QObject@@SA_NPBV1@PBD01@Z 1001e140     qt-mt323:qt-mt323.dll
 0002:00000144       __imp_??0QStringList@@QAE@XZ 1001e144     qt-mt323:qt-mt323.dll
 0002:00000148       __imp_??0QStringList@@QAE@ABV0@@Z 1001e148     qt-mt323:qt-mt323.dll
 0002:0000014c       __imp_?split@QStringList@@SA?AV1@ABVQString@@0_N@Z 1001e14c     qt-mt323:qt-mt323.dll
 0002:00000150       __imp_?join@QStringList@@QBE?AVQString@@ABV2@@Z 1001e150     qt-mt323:qt-mt323.dll
 0002:00000154       __imp_??1QStringList@@QAE@XZ 1001e154     qt-mt323:qt-mt323.dll
 0002:00000158       __imp_??4QStringList@@QAEAAV0@ABV0@@Z 1001e158     qt-mt323:qt-mt323.dll
 0002:0000015c       __imp_??0QWidget@@QAE@PAV0@PBDI@Z 1001e15c     qt-mt323:qt-mt323.dll
 0002:00000160       __imp_??1QWidget@@UAE@XZ   1001e160     qt-mt323:qt-mt323.dll
 0002:00000164       __imp_?setName@QWidget@@UAEXPBD@Z 1001e164     qt-mt323:qt-mt323.dll
 0002:00000168       __imp_?rect@QWidget@@QBE?AVQRect@@XZ 1001e168     qt-mt323:qt-mt323.dll
 0002:0000016c       __imp_?exec@QDialog@@QAEHXZ 1001e16c     qt-mt323:qt-mt323.dll
 0002:00000170       __imp_?information@QMessageBox@@SAHPAVQWidget@@ABVQString@@1111HH@Z 1001e170     qt-mt323:qt-mt323.dll
 0002:00000174       __imp_?warning@QMessageBox@@SAHPAVQWidget@@ABVQString@@1111HH@Z 1001e174     qt-mt323:qt-mt323.dll
 0002:00000178       __imp_?critical@QMessageBox@@SAHPAVQWidget@@ABVQString@@1111HH@Z 1001e178     qt-mt323:qt-mt323.dll
 0002:0000017c       __imp_??0QPixmap@@QAE@QAPBD@Z 1001e17c     qt-mt323:qt-mt323.dll
 0002:00000180       __imp_??1QPixmap@@UAE@XZ   1001e180     qt-mt323:qt-mt323.dll
 0002:00000184       __imp_??0QIconSet@@QAE@ABVQPixmap@@W4Size@0@@Z 1001e184     qt-mt323:qt-mt323.dll
 0002:00000188       __imp_??1QIconSet@@UAE@XZ  1001e188     qt-mt323:qt-mt323.dll
 0002:0000018c       __imp_??0QKeySequence@@QAE@H@Z 1001e18c     qt-mt323:qt-mt323.dll
 0002:00000190       __imp_??0QAction@@QAE@ABVQString@@ABVQIconSet@@0VQKeySequence@@PAVQObject@@PBD_N@Z 1001e190     qt-mt323:qt-mt323.dll
 0002:00000194       __imp_??1QAction@@UAE@XZ   1001e194     qt-mt323:qt-mt323.dll
 0002:00000198       __imp_??0QDockWindow@@QAE@W4Place@0@PAVQWidget@@PBDI@Z 1001e198     qt-mt323:qt-mt323.dll
 0002:0000019c       __imp_??1QDockWindow@@UAE@XZ 1001e19c     qt-mt323:qt-mt323.dll
 0002:000001a0       __imp_??1?$QPtrList@VQDockWindow@@@@UAE@XZ 1001e1a0     qt-mt323:qt-mt323.dll
 0002:000001a4       __imp_??0QToolBar@@QAE@PAVQMainWindow@@PBD@Z 1001e1a4     qt-mt323:qt-mt323.dll
 0002:000001a8       __imp_??1QToolBar@@UAE@XZ  1001e1a8     qt-mt323:qt-mt323.dll
 0002:000001ac       __imp_?text@QSpinBox@@QBE?AVQString@@XZ 1001e1ac     qt-mt323:qt-mt323.dll
 0002:000001b0       __imp_??0QListViewItem@@QAE@PAVQListView@@VQString@@1111111@Z 1001e1b0     qt-mt323:qt-mt323.dll
 0002:000001b4       __imp_??1QListViewItem@@UAE@XZ 1001e1b4     qt-mt323:qt-mt323.dll
 0002:000001b8       __imp_??0QListView@@QAE@PAVQWidget@@PBDI@Z 1001e1b8     qt-mt323:qt-mt323.dll
 0002:000001bc       __imp_??1QListView@@UAE@XZ 1001e1bc     qt-mt323:qt-mt323.dll
 0002:000001c0       __imp_?selectedItem@QListView@@QBEPAVQListViewItem@@XZ 1001e1c0     qt-mt323:qt-mt323.dll
 0002:000001c4       __imp_?currentItem@QListView@@QBEPAVQListViewItem@@XZ 1001e1c4     qt-mt323:qt-mt323.dll
 0002:000001c8       __imp_?firstChild@QListView@@QBEPAVQListViewItem@@XZ 1001e1c8     qt-mt323:qt-mt323.dll
 0002:000001cc       __imp_?findItem@QListView@@QBEPAVQListViewItem@@ABVQString@@HI@Z 1001e1cc     qt-mt323:qt-mt323.dll
 0002:000001d0       __imp_?triggerUpdate@QListView@@QAEXXZ 1001e1d0     qt-mt323:qt-mt323.dll
 0002:000001d4       __imp_??0QFile@@QAE@ABVQString@@@Z 1001e1d4     qt-mt323:qt-mt323.dll
 0002:000001d8       __imp_??1QFile@@UAE@XZ     1001e1d8     qt-mt323:qt-mt323.dll
 0002:000001dc       __imp_?name@QFile@@QBE?AVQString@@XZ 1001e1dc     qt-mt323:qt-mt323.dll
 0002:000001e0       __imp_?exists@QFile@@QBE_NXZ 1001e1e0     qt-mt323:qt-mt323.dll
 0002:000001e4       __imp_?exists@QFile@@SA_NABVQString@@@Z 1001e1e4     qt-mt323:qt-mt323.dll
 0002:000001e8       __imp_?remove@QFile@@QAE_NXZ 1001e1e8     qt-mt323:qt-mt323.dll
 0002:000001ec       __imp_?open@QFile@@UAE_NH@Z 1001e1ec     qt-mt323:qt-mt323.dll
 0002:000001f0       __imp_?close@QFile@@UAEXXZ 1001e1f0     qt-mt323:qt-mt323.dll
 0002:000001f4       __imp_?errorString@QFile@@QBE?AVQString@@XZ 1001e1f4     qt-mt323:qt-mt323.dll
 0002:000001f8       __imp_?secsTo@QTime@@QBEHABV1@@Z 1001e1f8     qt-mt323:qt-mt323.dll
 0002:000001fc       __imp_?msecsTo@QTime@@QBEHABV1@@Z 1001e1fc     qt-mt323:qt-mt323.dll
 0002:00000200       __imp_?currentTime@QTime@@SA?AV1@XZ 1001e200     qt-mt323:qt-mt323.dll
 0002:00000204       __imp_??8QDateTime@@QBE_NABV0@@Z 1001e204     qt-mt323:qt-mt323.dll
 0002:00000208       __imp_??9QDateTime@@QBE_NABV0@@Z 1001e208     qt-mt323:qt-mt323.dll
 0002:0000020c       __imp_??0QFileInfo@@QAE@XZ 1001e20c     qt-mt323:qt-mt323.dll
 0002:00000210       __imp_??0QFileInfo@@QAE@ABVQString@@@Z 1001e210     qt-mt323:qt-mt323.dll
 0002:00000214       __imp_??1QFileInfo@@QAE@XZ 1001e214     qt-mt323:qt-mt323.dll
 0002:00000218       __imp_?setFile@QFileInfo@@QAEXABVQString@@@Z 1001e218     qt-mt323:qt-mt323.dll
 0002:0000021c       __imp_?exists@QFileInfo@@QBE_NXZ 1001e21c     qt-mt323:qt-mt323.dll
 0002:00000220       __imp_?isFile@QFileInfo@@QBE_NXZ 1001e220     qt-mt323:qt-mt323.dll
 0002:00000224       __imp_?lastModified@QFileInfo@@QBE?AVQDateTime@@XZ 1001e224     qt-mt323:qt-mt323.dll
 0002:00000228       __imp_??0QTabWidget@@QAE@PAVQWidget@@PBDI@Z 1001e228     qt-mt323:qt-mt323.dll
 0002:0000022c       __imp_??1QTabWidget@@UAE@XZ 1001e22c     qt-mt323:qt-mt323.dll
 0002:00000230       __imp_??0QDir@@QAE@XZ      1001e230     qt-mt323:qt-mt323.dll
 0002:00000234       __imp_??0QDir@@QAE@ABVQString@@0HH@Z 1001e234     qt-mt323:qt-mt323.dll
 0002:00000238       __imp_??1QDir@@UAE@XZ      1001e238     qt-mt323:qt-mt323.dll
 0002:0000023c       __imp_?setPath@QDir@@UAEXABVQString@@@Z 1001e23c     qt-mt323:qt-mt323.dll
 0002:00000240       __imp_?entryList@QDir@@UBE?AVQStringList@@HH@Z 1001e240     qt-mt323:qt-mt323.dll
 0002:00000244       __imp_?mkdir@QDir@@UBE_NABVQString@@_N@Z 1001e244     qt-mt323:qt-mt323.dll
 0002:00000248       __imp_?exists@QDir@@UBE_NXZ 1001e248     qt-mt323:qt-mt323.dll
 0002:0000024c       __imp_?add@QLayout@@QAEXPAVQWidget@@@Z 1001e24c     qt-mt323:qt-mt323.dll
 0002:00000250       __imp_??0QBoxLayout@@QAE@PAVQWidget@@W4Direction@0@HHPBD@Z 1001e250     qt-mt323:qt-mt323.dll
 0002:00000254       __imp_??1QBoxLayout@@UAE@XZ 1001e254     qt-mt323:qt-mt323.dll
 0002:00000258       __imp_??0QRegExp@@QAE@ABVQString@@_N1@Z 1001e258     qt-mt323:qt-mt323.dll
 0002:0000025c       __imp_??1QRegExp@@QAE@XZ   1001e25c     qt-mt323:qt-mt323.dll
 0002:00000260       __imp_?search@QRegExp@@QBEHABVQString@@H@Z 1001e260     qt-mt323:qt-mt323.dll
 0002:00000264       __imp_??0QDomImplementation@@QAE@XZ 1001e264     qt-mt323:qt-mt323.dll
 0002:00000268       __imp_??1QDomImplementation@@UAE@XZ 1001e268     qt-mt323:qt-mt323.dll
 0002:0000026c       __imp_?createDocumentType@QDomImplementation@@UAE?AVQDomDocumentType@@ABVQString@@00@Z 1001e26c     qt-mt323:qt-mt323.dll
 0002:00000270       __imp_??1QDomNode@@UAE@XZ  1001e270     qt-mt323:qt-mt323.dll
 0002:00000274       __imp_?appendChild@QDomNode@@UAE?AV1@ABV1@@Z 1001e274     qt-mt323:qt-mt323.dll
 0002:00000278       __imp_?save@QDomNode@@QBEXAAVQTextStream@@H@Z 1001e278     qt-mt323:qt-mt323.dll
 0002:0000027c       __imp_??1QDomDocumentType@@UAE@XZ 1001e27c     qt-mt323:qt-mt323.dll
 0002:00000280       __imp_??0QDomDocument@@QAE@XZ 1001e280     qt-mt323:qt-mt323.dll
 0002:00000284       __imp_??0QDomDocument@@QAE@ABVQDomDocumentType@@@Z 1001e284     qt-mt323:qt-mt323.dll
 0002:00000288       __imp_??4QDomDocument@@QAEAAV0@ABV0@@Z 1001e288     qt-mt323:qt-mt323.dll
 0002:0000028c       __imp_??1QDomDocument@@UAE@XZ 1001e28c     qt-mt323:qt-mt323.dll
 0002:00000290       __imp_?createElement@QDomDocument@@QAE?AVQDomElement@@ABVQString@@@Z 1001e290     qt-mt323:qt-mt323.dll
 0002:00000294       __imp_?createProcessingInstruction@QDomDocument@@QAE?AVQDomProcessingInstruction@@ABVQString@@0@Z 1001e294     qt-mt323:qt-mt323.dll
 0002:00000298       __imp_?documentElement@QDomDocument@@QBE?AVQDomElement@@XZ 1001e298     qt-mt323:qt-mt323.dll
 0002:0000029c       __imp_?toString@QDomDocument@@QBE?AVQString@@XZ 1001e29c     qt-mt323:qt-mt323.dll
 0002:000002a0       __imp_??1QDomElement@@UAE@XZ 1001e2a0     qt-mt323:qt-mt323.dll
 0002:000002a4       __imp_?setAttribute@QDomElement@@QAEXABVQString@@0@Z 1001e2a4     qt-mt323:qt-mt323.dll
 0002:000002a8       __imp_??1QDomProcessingInstruction@@UAE@XZ 1001e2a8     qt-mt323:qt-mt323.dll
 0002:000002ac       __imp_?codecForName@QTextCodec@@SAPAV1@PBDH@Z 1001e2ac     qt-mt323:qt-mt323.dll
 0002:000002b0       __imp_?fromUnicode@QTextCodec@@QBE?AVQCString@@ABVQString@@@Z 1001e2b0     qt-mt323:qt-mt323.dll
 0002:000002b4       __imp_??0QGuardedPtrPrivate@@QAE@PAVQObject@@@Z 1001e2b4     qt-mt323:qt-mt323.dll
 0002:000002b8       __imp_??1QGuardedPtrPrivate@@UAE@XZ 1001e2b8     qt-mt323:qt-mt323.dll
 0002:000002bc       __imp_?reconnect@QGuardedPtrPrivate@@QAEXPAVQObject@@@Z 1001e2bc     qt-mt323:qt-mt323.dll
 0002:000002c0       __imp_?look_string@QGDict@@QAEPAXABVQString@@PAXH@Z 1001e2c0     qt-mt323:qt-mt323.dll
 0002:000002c4       __imp_?remove_string@QGDict@@IAE_NABVQString@@PAX@Z 1001e2c4     qt-mt323:qt-mt323.dll
 0002:000002c8       __imp_??0QGDictIterator@@QAE@ABVQGDict@@@Z 1001e2c8     qt-mt323:qt-mt323.dll
 0002:000002cc       __imp_??1QGDictIterator@@QAE@XZ 1001e2cc     qt-mt323:qt-mt323.dll
 0002:000002d0       __imp_?toFirst@QGDictIterator@@QAEPAXXZ 1001e2d0     qt-mt323:qt-mt323.dll
 0002:000002d4       __imp_?get@QGDictIterator@@QBEPAXXZ 1001e2d4     qt-mt323:qt-mt323.dll
 0002:000002d8       __imp_?getKeyString@QGDictIterator@@QBE?AVQString@@XZ 1001e2d8     qt-mt323:qt-mt323.dll
 0002:000002dc       __imp_??EQGDictIterator@@QAEPAXXZ 1001e2dc     qt-mt323:qt-mt323.dll
 0002:000002e0       __imp_??0QPopupMenu@@QAE@PAVQWidget@@PBD@Z 1001e2e0     qt-mt323:qt-mt323.dll
 0002:000002e4       __imp_??1QPopupMenu@@UAE@XZ 1001e2e4     qt-mt323:qt-mt323.dll
 0002:000002e8       __imp_?exec@QPopupMenu@@QAEHABVQPoint@@H@Z 1001e2e8     qt-mt323:qt-mt323.dll
 0002:000002ec       __imp_?acceptDrop@QListViewItem@@UBE_NPBVQMimeSource@@@Z 1001e2ec     qt-mt323:qt-mt323.dll
 0002:000002f0       __imp_?activate@QListViewItem@@MAEXXZ 1001e2f0     qt-mt323:qt-mt323.dll
 0002:000002f4       __imp_?activateItemAt@QPopupMenu@@UAEXH@Z 1001e2f4     qt-mt323:qt-mt323.dll
 0002:000002f8       __imp_?addChild@QScrollView@@UAEXPAVQWidget@@HH@Z 1001e2f8     qt-mt323:qt-mt323.dll
 0002:000002fc       __imp_?addColumn@QListView@@UAEHABVQIconSet@@ABVQString@@H@Z 1001e2fc     qt-mt323:qt-mt323.dll
 0002:00000300       __imp_?addColumn@QListView@@UAEHABVQString@@H@Z 1001e300     qt-mt323:qt-mt323.dll
 0002:00000304       __imp_?addItem@QBoxLayout@@UAEXPAVQLayoutItem@@@Z 1001e304     qt-mt323:qt-mt323.dll
 0002:00000308       __imp_?addTab@QTabWidget@@UAEXPAVQWidget@@ABVQIconSet@@ABVQString@@@Z 1001e308     qt-mt323:qt-mt323.dll
 0002:0000030c       __imp_?addTab@QTabWidget@@UAEXPAVQWidget@@ABVQString@@@Z 1001e30c     qt-mt323:qt-mt323.dll
 0002:00000310       __imp_?addTab@QTabWidget@@UAEXPAVQWidget@@PAVQTab@@@Z 1001e310     qt-mt323:qt-mt323.dll
 0002:00000314       __imp_?addTo@QAction@@UAE_NPAVQWidget@@@Z 1001e314     qt-mt323:qt-mt323.dll
 0002:00000318       __imp_?addedTo@QAction@@MAEXHPAVQPopupMenu@@@Z 1001e318     qt-mt323:qt-mt323.dll
 0002:0000031c       __imp_?addedTo@QAction@@MAEXPAVQWidget@@0@Z 1001e31c     qt-mt323:qt-mt323.dll
 0002:00000320       __imp_?adjustSize@QWidget@@UAEXXZ 1001e320     qt-mt323:qt-mt323.dll
 0002:00000324       __imp_?cancelRename@QListViewItem@@MAEXH@Z 1001e324     qt-mt323:qt-mt323.dll
 0002:00000328       __imp_?checkConnectArgs@QObject@@MAE_NPBDPBV1@0@Z 1001e328     qt-mt323:qt-mt323.dll
 0002:0000032c       __imp_?childEvent@QLayout@@MAEXPAVQChildEvent@@@Z 1001e32c     qt-mt323:qt-mt323.dll
 0002:00000330       __imp_?childEvent@QObject@@MAEXPAVQChildEvent@@@Z 1001e330     qt-mt323:qt-mt323.dll
 0002:00000334       __imp_?className@QAction@@UBEPBDXZ 1001e334     qt-mt323:qt-mt323.dll
 0002:00000338       __imp_?className@QBoxLayout@@UBEPBDXZ 1001e338     qt-mt323:qt-mt323.dll
 0002:0000033c       __imp_?className@QDockWindow@@UBEPBDXZ 1001e33c     qt-mt323:qt-mt323.dll
 0002:00000340       __imp_?className@QGuardedPtrPrivate@@UBEPBDXZ 1001e340     qt-mt323:qt-mt323.dll
 0002:00000344       __imp_?className@QListView@@UBEPBDXZ 1001e344     qt-mt323:qt-mt323.dll
 0002:00000348       __imp_?className@QPopupMenu@@UBEPBDXZ 1001e348     qt-mt323:qt-mt323.dll
 0002:0000034c       __imp_?className@QTabWidget@@UBEPBDXZ 1001e34c     qt-mt323:qt-mt323.dll
 0002:00000350       __imp_?className@QToolBar@@UBEPBDXZ 1001e350     qt-mt323:qt-mt323.dll
 0002:00000354       __imp_?className@QWidget@@UBEPBDXZ 1001e354     qt-mt323:qt-mt323.dll
 0002:00000358       __imp_?clear@?$QPtrList@VQDockWindow@@@@UAEXXZ 1001e358     qt-mt323:qt-mt323.dll
 0002:0000035c       __imp_?clear@QListView@@UAEXXZ 1001e35c     qt-mt323:qt-mt323.dll
 0002:00000360       __imp_?clear@QToolBar@@UAEXXZ 1001e360     qt-mt323:qt-mt323.dll
 0002:00000364       __imp_?clearSelection@QListView@@UAEXXZ 1001e364     qt-mt323:qt-mt323.dll
 0002:00000368       __imp_?close@QWidget@@UAE_N_N@Z 1001e368     qt-mt323:qt-mt323.dll
 0002:0000036c       __imp_?closeEvent@QPopupMenu@@MAEXPAVQCloseEvent@@@Z 1001e36c     qt-mt323:qt-mt323.dll
 0002:00000370       __imp_?closeEvent@QWidget@@MAEXPAVQCloseEvent@@@Z 1001e370     qt-mt323:qt-mt323.dll
 0002:00000374       __imp_?cmd@QPaintDevice@@MAE_NHPAVQPainter@@PATQPDevCmdParam@@@Z 1001e374     qt-mt323:qt-mt323.dll
 0002:00000378       __imp_?compare@QListViewItem@@UBEHPAV1@H_N@Z 1001e378     qt-mt323:qt-mt323.dll
 0002:0000037c       __imp_?compareItems@QGList@@MAEHPAX0@Z 1001e37c     qt-mt323:qt-mt323.dll
 0002:00000380       __imp_?connectNotify@QObject@@MAEXPBD@Z 1001e380     qt-mt323:qt-mt323.dll
 0002:00000384       __imp_?contentsContextMenuEvent@QListView@@MAEXPAVQContextMenuEvent@@@Z 1001e384     qt-mt323:qt-mt323.dll
 0002:00000388       __imp_?contentsDragEnterEvent@QListView@@MAEXPAVQDragEnterEvent@@@Z 1001e388     qt-mt323:qt-mt323.dll
 0002:0000038c       __imp_?contentsDragLeaveEvent@QListView@@MAEXPAVQDragLeaveEvent@@@Z 1001e38c     qt-mt323:qt-mt323.dll
 0002:00000390       __imp_?contentsDragMoveEvent@QListView@@MAEXPAVQDragMoveEvent@@@Z 1001e390     qt-mt323:qt-mt323.dll
 0002:00000394       __imp_?contentsDropEvent@QListView@@MAEXPAVQDropEvent@@@Z 1001e394     qt-mt323:qt-mt323.dll
 0002:00000398       __imp_?contentsMouseDoubleClickEvent@QListView@@MAEXPAVQMouseEvent@@@Z 1001e398     qt-mt323:qt-mt323.dll
 0002:0000039c       __imp_?contentsMouseMoveEvent@QListView@@MAEXPAVQMouseEvent@@@Z 1001e39c     qt-mt323:qt-mt323.dll
 0002:000003a0       __imp_?contentsMousePressEvent@QListView@@MAEXPAVQMouseEvent@@@Z 1001e3a0     qt-mt323:qt-mt323.dll
 0002:000003a4       __imp_?contentsMouseReleaseEvent@QListView@@MAEXPAVQMouseEvent@@@Z 1001e3a4     qt-mt323:qt-mt323.dll
 0002:000003a8       __imp_?contentsWheelEvent@QScrollView@@MAEXPAVQWheelEvent@@@Z 1001e3a8     qt-mt323:qt-mt323.dll
 0002:000003ac       __imp_?contextMenuEvent@QDockWindow@@MAEXPAVQContextMenuEvent@@@Z 1001e3ac     qt-mt323:qt-mt323.dll
 0002:000003b0       __imp_?contextMenuEvent@QScrollView@@MAEXPAVQContextMenuEvent@@@Z 1001e3b0     qt-mt323:qt-mt323.dll
 0002:000003b4       __imp_?contextMenuEvent@QWidget@@MAEXPAVQContextMenuEvent@@@Z 1001e3b4     qt-mt323:qt-mt323.dll
 0002:000003b8       __imp_?count@?$QPtrList@VQDockWindow@@@@UBEIXZ 1001e3b8     qt-mt323:qt-mt323.dll
 0002:000003bc       __imp_?create@QWidget@@MAEXPAUHWND__@@_N1@Z 1001e3bc     qt-mt323:qt-mt323.dll
 0002:000003c0       __imp_?customEvent@QObject@@MAEXPAVQCustomEvent@@@Z 1001e3c0     qt-mt323:qt-mt323.dll
 0002:000003c4       __imp_?customWhatsThis@QPopupMenu@@UBE_NXZ 1001e3c4     qt-mt323:qt-mt323.dll
 0002:000003c8       __imp_?customWhatsThis@QWidget@@UBE_NXZ 1001e3c8     qt-mt323:qt-mt323.dll
 0002:000003cc       __imp_?deleteItem@?$QPtrList@VQDockWindow@@@@EAEXPAX@Z 1001e3cc     qt-mt323:qt-mt323.dll
 0002:000003d0       __imp_?destroy@QWidget@@MAEX_N0@Z 1001e3d0     qt-mt323:qt-mt323.dll
 0002:000003d4       __imp_?disconnectNotify@QObject@@MAEXPBD@Z 1001e3d4     qt-mt323:qt-mt323.dll
 0002:000003d8       __imp_?dock@QDockWindow@@UAEXXZ 1001e3d8     qt-mt323:qt-mt323.dll
 0002:000003dc       __imp_?dragEnterEvent@QWidget@@MAEXPAVQDragEnterEvent@@@Z 1001e3dc     qt-mt323:qt-mt323.dll
 0002:000003e0       __imp_?dragEntered@QListViewItem@@MAEXXZ 1001e3e0     qt-mt323:qt-mt323.dll
 0002:000003e4       __imp_?dragLeaveEvent@QWidget@@MAEXPAVQDragLeaveEvent@@@Z 1001e3e4     qt-mt323:qt-mt323.dll
 0002:000003e8       __imp_?dragLeft@QListViewItem@@MAEXXZ 1001e3e8     qt-mt323:qt-mt323.dll
 0002:000003ec       __imp_?dragMoveEvent@QWidget@@MAEXPAVQDragMoveEvent@@@Z 1001e3ec     qt-mt323:qt-mt323.dll
 0002:000003f0       __imp_?dragObject@QListView@@MAEPAVQDragObject@@XZ 1001e3f0     qt-mt323:qt-mt323.dll
 0002:000003f4       __imp_?drawContents@QDockWindow@@MAEXPAVQPainter@@@Z 1001e3f4     qt-mt323:qt-mt323.dll
 0002:000003f8       __imp_?drawContents@QFrame@@MAEXPAVQPainter@@@Z 1001e3f8     qt-mt323:qt-mt323.dll
 0002:000003fc       __imp_?drawContents@QPopupMenu@@MAEXPAVQPainter@@@Z 1001e3fc     qt-mt323:qt-mt323.dll
 0002:00000400       __imp_?drawContents@QScrollView@@EAEXPAVQPainter@@@Z 1001e400     qt-mt323:qt-mt323.dll
 0002:00000404       __imp_?drawContents@QScrollView@@MAEXPAVQPainter@@HHHH@Z 1001e404     qt-mt323:qt-mt323.dll
 0002:00000408       __imp_?drawContentsOffset@QListView@@MAEXPAVQPainter@@HHHHHH@Z 1001e408     qt-mt323:qt-mt323.dll
 0002:0000040c       __imp_?drawFrame@QDockWindow@@MAEXPAVQPainter@@@Z 1001e40c     qt-mt323:qt-mt323.dll
 0002:00000410       __imp_?drawFrame@QFrame@@MAEXPAVQPainter@@@Z 1001e410     qt-mt323:qt-mt323.dll
 0002:00000414       __imp_?dropEvent@QWidget@@MAEXPAVQDropEvent@@@Z 1001e414     qt-mt323:qt-mt323.dll
 0002:00000418       __imp_?dropped@QListViewItem@@MAEXPAVQDropEvent@@@Z 1001e418     qt-mt323:qt-mt323.dll
 0002:0000041c       __imp_?enabledChange@QPopupMenu@@MAEX_N@Z 1001e41c     qt-mt323:qt-mt323.dll
 0002:00000420       __imp_?enabledChange@QWidget@@MAEX_N@Z 1001e420     qt-mt323:qt-mt323.dll
 0002:00000424       __imp_?enforceSortOrder@QListViewItem@@MBEXXZ 1001e424     qt-mt323:qt-mt323.dll
 0002:00000428       __imp_?enterEvent@QWidget@@MAEXPAVQEvent@@@Z 1001e428     qt-mt323:qt-mt323.dll
 0002:0000042c       __imp_?event@QDockWindow@@MAE_NPAVQEvent@@@Z 1001e42c     qt-mt323:qt-mt323.dll
 0002:00000430       __imp_?event@QObject@@UAE_NPAVQEvent@@@Z 1001e430     qt-mt323:qt-mt323.dll
 0002:00000434       __imp_?event@QToolBar@@UAE_NPAVQEvent@@@Z 1001e434     qt-mt323:qt-mt323.dll
 0002:00000438       __imp_?event@QWidget@@MAE_NPAVQEvent@@@Z 1001e438     qt-mt323:qt-mt323.dll
 0002:0000043c       __imp_?eventFilter@QDockWindow@@UAE_NPAVQObject@@PAVQEvent@@@Z 1001e43c     qt-mt323:qt-mt323.dll
 0002:00000440       __imp_?eventFilter@QLayout@@MAE_NPAVQObject@@PAVQEvent@@@Z 1001e440     qt-mt323:qt-mt323.dll
 0002:00000444       __imp_?eventFilter@QListView@@UAE_NPAVQObject@@PAVQEvent@@@Z 1001e444     qt-mt323:qt-mt323.dll
 0002:00000448       __imp_?eventFilter@QObject@@UAE_NPAV1@PAVQEvent@@@Z 1001e448     qt-mt323:qt-mt323.dll
 0002:0000044c       __imp_?eventFilter@QTabWidget@@MAE_NPAVQObject@@PAVQEvent@@@Z 1001e44c     qt-mt323:qt-mt323.dll
 0002:00000450       __imp_?expanding@QBoxLayout@@UBE?AW4ExpandData@QSizePolicy@@XZ 1001e450     qt-mt323:qt-mt323.dll
 0002:00000454       __imp_?focusInEvent@QListView@@MAEXPAVQFocusEvent@@@Z 1001e454     qt-mt323:qt-mt323.dll
 0002:00000458       __imp_?focusInEvent@QPopupMenu@@MAEXPAVQFocusEvent@@@Z 1001e458     qt-mt323:qt-mt323.dll
 0002:0000045c       __imp_?focusInEvent@QWidget@@MAEXPAVQFocusEvent@@@Z 1001e45c     qt-mt323:qt-mt323.dll
 0002:00000460       __imp_?focusNextPrevChild@QPopupMenu@@MAE_N_N@Z 1001e460     qt-mt323:qt-mt323.dll
 0002:00000464       __imp_?focusNextPrevChild@QScrollView@@MAE_N_N@Z 1001e464     qt-mt323:qt-mt323.dll
 0002:00000468       __imp_?focusNextPrevChild@QWidget@@MAE_N_N@Z 1001e468     qt-mt323:qt-mt323.dll
 0002:0000046c       __imp_?focusOutEvent@QListView@@MAEXPAVQFocusEvent@@@Z 1001e46c     qt-mt323:qt-mt323.dll
 0002:00000470       __imp_?focusOutEvent@QPopupMenu@@MAEXPAVQFocusEvent@@@Z 1001e470     qt-mt323:qt-mt323.dll
 0002:00000474       __imp_?focusOutEvent@QWidget@@MAEXPAVQFocusEvent@@@Z 1001e474     qt-mt323:qt-mt323.dll
 0002:00000478       __imp_?fontChange@QScrollView@@MAEXABVQFont@@@Z 1001e478     qt-mt323:qt-mt323.dll
 0002:0000047c       __imp_?fontChange@QWidget@@MAEXABVQFont@@@Z 1001e47c     qt-mt323:qt-mt323.dll
 0002:00000480       __imp_?fontInf@QPaintDevice@@MBEHPAVQFont@@H@Z 1001e480     qt-mt323:qt-mt323.dll
 0002:00000484       __imp_?fontMet@QPaintDevice@@MBEHPAVQFont@@HPBDH@Z 1001e484     qt-mt323:qt-mt323.dll
 0002:00000488       __imp_?frameChanged@QFrame@@MAEXXZ 1001e488     qt-mt323:qt-mt323.dll
 0002:0000048c       __imp_?frameChanged@QHBox@@MAEXXZ 1001e48c     qt-mt323:qt-mt323.dll
 0002:00000490       __imp_?frameChanged@QPopupMenu@@EAEXXZ 1001e490     qt-mt323:qt-mt323.dll
 0002:00000494       __imp_?frameChanged@QScrollView@@MAEXXZ 1001e494     qt-mt323:qt-mt323.dll
 0002:00000498       __imp_?geometry@QLayout@@UBE?AVQRect@@XZ 1001e498     qt-mt323:qt-mt323.dll
 0002:0000049c       __imp_?handle@QPaintDevice@@UBEPAUHDC__@@XZ 1001e49c     qt-mt323:qt-mt323.dll
 0002:000004a0       __imp_?hasHeightForWidth@QBoxLayout@@UBE_NXZ 1001e4a0     qt-mt323:qt-mt323.dll
 0002:000004a4       __imp_?heightForWidth@QBoxLayout@@UBEHH@Z 1001e4a4     qt-mt323:qt-mt323.dll
 0002:000004a8       __imp_?heightForWidth@QWidget@@UBEHH@Z 1001e4a8     qt-mt323:qt-mt323.dll
 0002:000004ac       __imp_?hide@QPopupMenu@@UAEXXZ 1001e4ac     qt-mt323:qt-mt323.dll
 0002:000004b0       __imp_?hide@QToolBar@@UAEXXZ 1001e4b0     qt-mt323:qt-mt323.dll
 0002:000004b4       __imp_?hide@QWidget@@UAEXXZ 1001e4b4     qt-mt323:qt-mt323.dll
 0002:000004b8       __imp_?hideEvent@QDockWindow@@MAEXPAVQHideEvent@@@Z 1001e4b8     qt-mt323:qt-mt323.dll
 0002:000004bc       __imp_?hideEvent@QWidget@@MAEXPAVQHideEvent@@@Z 1001e4bc     qt-mt323:qt-mt323.dll
 0002:000004c0       __imp_?imComposeEvent@QWidget@@MAEXPAVQIMEvent@@@Z 1001e4c0     qt-mt323:qt-mt323.dll
 0002:000004c4       __imp_?imEndEvent@QWidget@@MAEXPAVQIMEvent@@@Z 1001e4c4     qt-mt323:qt-mt323.dll
 0002:000004c8       __imp_?imStartEvent@QWidget@@MAEXPAVQIMEvent@@@Z 1001e4c8     qt-mt323:qt-mt323.dll
 0002:000004cc       __imp_?insertChild@QObject@@UAEXPAV1@@Z 1001e4cc     qt-mt323:qt-mt323.dll
 0002:000004d0       __imp_?insertItem@QListView@@UAEXPAVQListViewItem@@@Z 1001e4d0     qt-mt323:qt-mt323.dll
 0002:000004d4       __imp_?insertItem@QListViewItem@@UAEXPAV1@@Z 1001e4d4     qt-mt323:qt-mt323.dll
 0002:000004d8       __imp_?insertTab@QTabWidget@@UAEXPAVQWidget@@ABVQIconSet@@ABVQString@@H@Z 1001e4d8     qt-mt323:qt-mt323.dll
 0002:000004dc       __imp_?insertTab@QTabWidget@@UAEXPAVQWidget@@ABVQString@@H@Z 1001e4dc     qt-mt323:qt-mt323.dll
 0002:000004e0       __imp_?insertTab@QTabWidget@@UAEXPAVQWidget@@PAVQTab@@H@Z 1001e4e0     qt-mt323:qt-mt323.dll
 0002:000004e4       __imp_?invalidate@QBoxLayout@@UAEXXZ 1001e4e4     qt-mt323:qt-mt323.dll
 0002:000004e8       __imp_?invalidateHeight@QListViewItem@@UAEXXZ 1001e4e8     qt-mt323:qt-mt323.dll
 0002:000004ec       __imp_?invertSelection@QListView@@UAEXXZ 1001e4ec     qt-mt323:qt-mt323.dll
 0002:000004f0       __imp_?isEmpty@QLayout@@UBE_NXZ 1001e4f0     qt-mt323:qt-mt323.dll
 0002:000004f4       __imp_?iterator@QBoxLayout@@UAE?AVQLayoutIterator@@XZ 1001e4f4     qt-mt323:qt-mt323.dll
 0002:000004f8       __imp_?key@QListViewItem@@UBE?AVQString@@H_N@Z 1001e4f8     qt-mt323:qt-mt323.dll
 0002:000004fc       __imp_?keyPressEvent@QListView@@MAEXPAVQKeyEvent@@@Z 1001e4fc     qt-mt323:qt-mt323.dll
 0002:00000500       __imp_?keyPressEvent@QPopupMenu@@MAEXPAVQKeyEvent@@@Z 1001e500     qt-mt323:qt-mt323.dll
 0002:00000504       __imp_?keyPressEvent@QWidget@@MAEXPAVQKeyEvent@@@Z 1001e504     qt-mt323:qt-mt323.dll
 0002:00000508       __imp_?keyReleaseEvent@QWidget@@MAEXPAVQKeyEvent@@@Z 1001e508     qt-mt323:qt-mt323.dll
 0002:0000050c       __imp_?layout@QLayout@@UAEPAV1@XZ 1001e50c     qt-mt323:qt-mt323.dll
 0002:00000510       __imp_?leaveEvent@QPopupMenu@@MAEXPAVQEvent@@@Z 1001e510     qt-mt323:qt-mt323.dll
 0002:00000514       __imp_?leaveEvent@QWidget@@MAEXPAVQEvent@@@Z 1001e514     qt-mt323:qt-mt323.dll
 0002:00000518       __imp_?maximumSize@QBoxLayout@@UBE?AVQSize@@XZ 1001e518     qt-mt323:qt-mt323.dll
 0002:0000051c       __imp_?menuContentsChanged@QPopupMenu@@EAEXXZ 1001e51c     qt-mt323:qt-mt323.dll
 0002:00000520       __imp_?menuDelPopup@QPopupMenu@@EAEXPAV1@@Z 1001e520     qt-mt323:qt-mt323.dll
 0002:00000524       __imp_?menuInsPopup@QPopupMenu@@EAEXPAV1@@Z 1001e524     qt-mt323:qt-mt323.dll
 0002:00000528       __imp_?menuStateChanged@QPopupMenu@@EAEXXZ 1001e528     qt-mt323:qt-mt323.dll
 0002:0000052c       __imp_?metaObject@QAction@@UBEPAVQMetaObject@@XZ 1001e52c     qt-mt323:qt-mt323.dll
 0002:00000530       __imp_?metaObject@QBoxLayout@@UBEPAVQMetaObject@@XZ 1001e530     qt-mt323:qt-mt323.dll
 0002:00000534       __imp_?metaObject@QDockWindow@@UBEPAVQMetaObject@@XZ 1001e534     qt-mt323:qt-mt323.dll
 0002:00000538       __imp_?metaObject@QGuardedPtrPrivate@@UBEPAVQMetaObject@@XZ 1001e538     qt-mt323:qt-mt323.dll
 0002:0000053c       __imp_?metaObject@QListView@@UBEPAVQMetaObject@@XZ 1001e53c     qt-mt323:qt-mt323.dll
 0002:00000540       __imp_?metaObject@QPopupMenu@@UBEPAVQMetaObject@@XZ 1001e540     qt-mt323:qt-mt323.dll
 0002:00000544       __imp_?metaObject@QTabWidget@@UBEPAVQMetaObject@@XZ 1001e544     qt-mt323:qt-mt323.dll
 0002:00000548       __imp_?metaObject@QToolBar@@UBEPAVQMetaObject@@XZ 1001e548     qt-mt323:qt-mt323.dll
 0002:0000054c       __imp_?metaObject@QWidget@@UBEPAVQMetaObject@@XZ 1001e54c     qt-mt323:qt-mt323.dll
 0002:00000550       __imp_?metric@QWidget@@MBEHH@Z 1001e550     qt-mt323:qt-mt323.dll
 0002:00000554       __imp_?minimumSize@QBoxLayout@@UBE?AVQSize@@XZ 1001e554     qt-mt323:qt-mt323.dll
 0002:00000558       __imp_?minimumSizeHint@QDockWindow@@UBE?AVQSize@@XZ 1001e558     qt-mt323:qt-mt323.dll
 0002:0000055c       __imp_?minimumSizeHint@QListView@@UBE?AVQSize@@XZ 1001e55c     qt-mt323:qt-mt323.dll
 0002:00000560       __imp_?minimumSizeHint@QTabWidget@@UBE?AVQSize@@XZ 1001e560     qt-mt323:qt-mt323.dll
 0002:00000564       __imp_?minimumSizeHint@QToolBar@@UBE?AVQSize@@XZ 1001e564     qt-mt323:qt-mt323.dll
 0002:00000568       __imp_?minimumSizeHint@QWidget@@UBE?AVQSize@@XZ 1001e568     qt-mt323:qt-mt323.dll
 0002:0000056c       __imp_?mouseDoubleClickEvent@QScrollView@@MAEXPAVQMouseEvent@@@Z 1001e56c     qt-mt323:qt-mt323.dll
 0002:00000570       __imp_?mouseDoubleClickEvent@QWidget@@MAEXPAVQMouseEvent@@@Z 1001e570     qt-mt323:qt-mt323.dll
 0002:00000574       __imp_?mouseMoveEvent@QPopupMenu@@MAEXPAVQMouseEvent@@@Z 1001e574     qt-mt323:qt-mt323.dll
 0002:00000578       __imp_?mouseMoveEvent@QScrollView@@MAEXPAVQMouseEvent@@@Z 1001e578     qt-mt323:qt-mt323.dll
 0002:0000057c       __imp_?mouseMoveEvent@QWidget@@MAEXPAVQMouseEvent@@@Z 1001e57c     qt-mt323:qt-mt323.dll
 0002:00000580       __imp_?mousePressEvent@QPopupMenu@@MAEXPAVQMouseEvent@@@Z 1001e580     qt-mt323:qt-mt323.dll
 0002:00000584       __imp_?mousePressEvent@QScrollView@@MAEXPAVQMouseEvent@@@Z 1001e584     qt-mt323:qt-mt323.dll
 0002:00000588       __imp_?mousePressEvent@QWidget@@MAEXPAVQMouseEvent@@@Z 1001e588     qt-mt323:qt-mt323.dll
 0002:0000058c       __imp_?mouseReleaseEvent@QPopupMenu@@MAEXPAVQMouseEvent@@@Z 1001e58c     qt-mt323:qt-mt323.dll
 0002:00000590       __imp_?mouseReleaseEvent@QScrollView@@MAEXPAVQMouseEvent@@@Z 1001e590     qt-mt323:qt-mt323.dll
 0002:00000594       __imp_?mouseReleaseEvent@QWidget@@MAEXPAVQMouseEvent@@@Z 1001e594     qt-mt323:qt-mt323.dll
 0002:00000598       __imp_?move@QWidget@@UAEXHH@Z 1001e598     qt-mt323:qt-mt323.dll
 0002:0000059c       __imp_?moveChild@QScrollView@@UAEXPAVQWidget@@HH@Z 1001e59c     qt-mt323:qt-mt323.dll
 0002:000005a0       __imp_?moveEvent@QWidget@@MAEXPAVQMoveEvent@@@Z 1001e5a0     qt-mt323:qt-mt323.dll
 0002:000005a4       __imp_?newItem@QPtrCollection@@MAEPAXPAX@Z 1001e5a4     qt-mt323:qt-mt323.dll
 0002:000005a8       __imp_?okRename@QListViewItem@@MAEXH@Z 1001e5a8     qt-mt323:qt-mt323.dll
 0002:000005ac       __imp_?paintBranches@QListViewItem@@UAEXPAVQPainter@@ABVQColorGroup@@HHH@Z 1001e5ac     qt-mt323:qt-mt323.dll
 0002:000005b0       __imp_?paintCell@QListViewItem@@UAEXPAVQPainter@@ABVQColorGroup@@HHH@Z 1001e5b0     qt-mt323:qt-mt323.dll
 0002:000005b4       __imp_?paintEmptyArea@QListView@@MAEXPAVQPainter@@ABVQRect@@@Z 1001e5b4     qt-mt323:qt-mt323.dll
 0002:000005b8       __imp_?paintEvent@QFrame@@MAEXPAVQPaintEvent@@@Z 1001e5b8     qt-mt323:qt-mt323.dll
 0002:000005bc       __imp_?paintEvent@QPopupMenu@@MAEXPAVQPaintEvent@@@Z 1001e5bc     qt-mt323:qt-mt323.dll
 0002:000005c0       __imp_?paintEvent@QWidget@@MAEXPAVQPaintEvent@@@Z 1001e5c0     qt-mt323:qt-mt323.dll
 0002:000005c4       __imp_?paintFocus@QListViewItem@@UAEXPAVQPainter@@ABVQColorGroup@@ABVQRect@@@Z 1001e5c4     qt-mt323:qt-mt323.dll
 0002:000005c8       __imp_?paletteChange@QWidget@@MAEXABVQPalette@@@Z 1001e5c8     qt-mt323:qt-mt323.dll
 0002:000005cc       __imp_?pixmap@QListViewItem@@UBEPBVQPixmap@@H@Z 1001e5cc     qt-mt323:qt-mt323.dll
 0002:000005d0       __imp_?polish@QWidget@@UAEXXZ 1001e5d0     qt-mt323:qt-mt323.dll
 0002:000005d4       __imp_?property@QObject@@UBE?AVQVariant@@PBD@Z 1001e5d4     qt-mt323:qt-mt323.dll
 0002:000005d8       __imp_?qt_cast@QAction@@UAEPAXPBD@Z 1001e5d8     qt-mt323:qt-mt323.dll
 0002:000005dc       __imp_?qt_cast@QBoxLayout@@UAEPAXPBD@Z 1001e5dc     qt-mt323:qt-mt323.dll
 0002:000005e0       __imp_?qt_cast@QDockWindow@@UAEPAXPBD@Z 1001e5e0     qt-mt323:qt-mt323.dll
 0002:000005e4       __imp_?qt_cast@QGuardedPtrPrivate@@UAEPAXPBD@Z 1001e5e4     qt-mt323:qt-mt323.dll
 0002:000005e8       __imp_?qt_cast@QListView@@UAEPAXPBD@Z 1001e5e8     qt-mt323:qt-mt323.dll
 0002:000005ec       __imp_?qt_cast@QPopupMenu@@UAEPAXPBD@Z 1001e5ec     qt-mt323:qt-mt323.dll
 0002:000005f0       __imp_?qt_cast@QTabWidget@@UAEPAXPBD@Z 1001e5f0     qt-mt323:qt-mt323.dll
 0002:000005f4       __imp_?qt_cast@QToolBar@@UAEPAXPBD@Z 1001e5f4     qt-mt323:qt-mt323.dll
 0002:000005f8       __imp_?qt_cast@QWidget@@UAEPAXPBD@Z 1001e5f8     qt-mt323:qt-mt323.dll
 0002:000005fc       __imp_?qt_emit@QAction@@UAE_NHPAUQUObject@@@Z 1001e5fc     qt-mt323:qt-mt323.dll
 0002:00000600       __imp_?qt_emit@QBoxLayout@@UAE_NHPAUQUObject@@@Z 1001e600     qt-mt323:qt-mt323.dll
 0002:00000604       __imp_?qt_emit@QDockWindow@@UAE_NHPAUQUObject@@@Z 1001e604     qt-mt323:qt-mt323.dll
 0002:00000608       __imp_?qt_emit@QGuardedPtrPrivate@@UAE_NHPAUQUObject@@@Z 1001e608     qt-mt323:qt-mt323.dll
 0002:0000060c       __imp_?qt_emit@QListView@@UAE_NHPAUQUObject@@@Z 1001e60c     qt-mt323:qt-mt323.dll
 0002:00000610       __imp_?qt_emit@QPopupMenu@@UAE_NHPAUQUObject@@@Z 1001e610     qt-mt323:qt-mt323.dll
 0002:00000614       __imp_?qt_emit@QTabWidget@@UAE_NHPAUQUObject@@@Z 1001e614     qt-mt323:qt-mt323.dll
 0002:00000618       __imp_?qt_emit@QToolBar@@UAE_NHPAUQUObject@@@Z 1001e618     qt-mt323:qt-mt323.dll
 0002:0000061c       __imp_?qt_emit@QWidget@@UAE_NHPAUQUObject@@@Z 1001e61c     qt-mt323:qt-mt323.dll
 0002:00000620       __imp_?qt_invoke@QAction@@UAE_NHPAUQUObject@@@Z 1001e620     qt-mt323:qt-mt323.dll
 0002:00000624       __imp_?qt_invoke@QBoxLayout@@UAE_NHPAUQUObject@@@Z 1001e624     qt-mt323:qt-mt323.dll
 0002:00000628       __imp_?qt_invoke@QDockWindow@@UAE_NHPAUQUObject@@@Z 1001e628     qt-mt323:qt-mt323.dll
 0002:0000062c       __imp_?qt_invoke@QGuardedPtrPrivate@@UAE_NHPAUQUObject@@@Z 1001e62c     qt-mt323:qt-mt323.dll
 0002:00000630       __imp_?qt_invoke@QListView@@UAE_NHPAUQUObject@@@Z 1001e630     qt-mt323:qt-mt323.dll
 0002:00000634       __imp_?qt_invoke@QPopupMenu@@UAE_NHPAUQUObject@@@Z 1001e634     qt-mt323:qt-mt323.dll
 0002:00000638       __imp_?qt_invoke@QTabWidget@@UAE_NHPAUQUObject@@@Z 1001e638     qt-mt323:qt-mt323.dll
 0002:0000063c       __imp_?qt_invoke@QToolBar@@UAE_NHPAUQUObject@@@Z 1001e63c     qt-mt323:qt-mt323.dll
 0002:00000640       __imp_?qt_invoke@QWidget@@UAE_NHPAUQUObject@@@Z 1001e640     qt-mt323:qt-mt323.dll
 0002:00000644       __imp_?qt_property@QAction@@UAE_NHHPAVQVariant@@@Z 1001e644     qt-mt323:qt-mt323.dll
 0002:00000648       __imp_?qt_property@QBoxLayout@@UAE_NHHPAVQVariant@@@Z 1001e648     qt-mt323:qt-mt323.dll
 0002:0000064c       __imp_?qt_property@QDockWindow@@UAE_NHHPAVQVariant@@@Z 1001e64c     qt-mt323:qt-mt323.dll
 0002:00000650       __imp_?qt_property@QGuardedPtrPrivate@@UAE_NHHPAVQVariant@@@Z 1001e650     qt-mt323:qt-mt323.dll
 0002:00000654       __imp_?qt_property@QListView@@UAE_NHHPAVQVariant@@@Z 1001e654     qt-mt323:qt-mt323.dll
 0002:00000658       __imp_?qt_property@QPopupMenu@@UAE_NHHPAVQVariant@@@Z 1001e658     qt-mt323:qt-mt323.dll
 0002:0000065c       __imp_?qt_property@QTabWidget@@UAE_NHHPAVQVariant@@@Z 1001e65c     qt-mt323:qt-mt323.dll
 0002:00000660       __imp_?qt_property@QToolBar@@UAE_NHHPAVQVariant@@@Z 1001e660     qt-mt323:qt-mt323.dll
 0002:00000664       __imp_?qt_property@QWidget@@UAE_NHHPAVQVariant@@@Z 1001e664     qt-mt323:qt-mt323.dll
 0002:00000668       __imp_?read@QGList@@MAEAAVQDataStream@@AAV2@AAPAX@Z 1001e668     qt-mt323:qt-mt323.dll
 0002:0000066c       __imp_?removeChild@QObject@@UAEXPAV1@@Z 1001e66c     qt-mt323:qt-mt323.dll
 0002:00000670       __imp_?removeChild@QScrollView@@UAEXPAVQObject@@@Z 1001e670     qt-mt323:qt-mt323.dll
 0002:00000674       __imp_?removeColumn@QListView@@UAEXH@Z 1001e674     qt-mt323:qt-mt323.dll
 0002:00000678       __imp_?removeFrom@QAction@@UAE_NPAVQWidget@@@Z 1001e678     qt-mt323:qt-mt323.dll
 0002:0000067c       __imp_?removeItem@QListView@@UAEXPAVQListViewItem@@@Z 1001e67c     qt-mt323:qt-mt323.dll
 0002:00000680       __imp_?removeItem@QListViewItem@@UAEXPAV1@@Z 1001e680     qt-mt323:qt-mt323.dll
 0002:00000684       __imp_?removePage@QTabWidget@@UAEXPAVQWidget@@@Z 1001e684     qt-mt323:qt-mt323.dll
 0002:00000688       __imp_?reparent@QWidget@@UAEXPAV1@IABVQPoint@@_N@Z 1001e688     qt-mt323:qt-mt323.dll
 0002:0000068c       __imp_?resize@QScrollView@@UAEXHH@Z 1001e68c     qt-mt323:qt-mt323.dll
 0002:00000690       __imp_?resize@QWidget@@UAEXHH@Z 1001e690     qt-mt323:qt-mt323.dll
 0002:00000694       __imp_?resizeContents@QScrollView@@UAEXHH@Z 1001e694     qt-mt323:qt-mt323.dll
 0002:00000698       __imp_?resizeEvent@QDockWindow@@MAEXPAVQResizeEvent@@@Z 1001e698     qt-mt323:qt-mt323.dll
 0002:0000069c       __imp_?resizeEvent@QFrame@@MAEXPAVQResizeEvent@@@Z 1001e69c     qt-mt323:qt-mt323.dll
 0002:000006a0       __imp_?resizeEvent@QListView@@MAEXPAVQResizeEvent@@@Z 1001e6a0     qt-mt323:qt-mt323.dll
 0002:000006a4       __imp_?resizeEvent@QTabWidget@@MAEXPAVQResizeEvent@@@Z 1001e6a4     qt-mt323:qt-mt323.dll
 0002:000006a8       __imp_?resizeEvent@QToolBar@@MAEXPAVQResizeEvent@@@Z 1001e6a8     qt-mt323:qt-mt323.dll
 0002:000006ac       __imp_?resizeEvent@QWidget@@MAEXPAVQResizeEvent@@@Z 1001e6ac     qt-mt323:qt-mt323.dll
 0002:000006b0       __imp_?resolution@QPaintDevice@@UBEHXZ 1001e6b0     qt-mt323:qt-mt323.dll
 0002:000006b4       __imp_?rtti@QListViewItem@@UBEHXZ 1001e6b4     qt-mt323:qt-mt323.dll
 0002:000006b8       __imp_?selectAll@QListView@@UAEX_N@Z 1001e6b8     qt-mt323:qt-mt323.dll
 0002:000006bc       __imp_?setAccel@QAction@@UAEXABVQKeySequence@@@Z 1001e6bc     qt-mt323:qt-mt323.dll
 0002:000006c0       __imp_?setAcceptDrops@QWidget@@UAEX_N@Z 1001e6c0     qt-mt323:qt-mt323.dll
 0002:000006c4       __imp_?setActiveItem@QPopupMenu@@UAEXH@Z 1001e6c4     qt-mt323:qt-mt323.dll
 0002:000006c8       __imp_?setActiveWindow@QWidget@@UAEXXZ 1001e6c8     qt-mt323:qt-mt323.dll
 0002:000006cc       __imp_?setAlignment@QLayoutItem@@UAEXH@Z 1001e6cc     qt-mt323:qt-mt323.dll
 0002:000006d0       __imp_?setAllColumnsShowFocus@QListView@@UAEX_N@Z 1001e6d0     qt-mt323:qt-mt323.dll
 0002:000006d4       __imp_?setAutoAdd@QLayout@@UAEX_N@Z 1001e6d4     qt-mt323:qt-mt323.dll
 0002:000006d8       __imp_?setAutoMask@QWidget@@UAEX_N@Z 1001e6d8     qt-mt323:qt-mt323.dll
 0002:000006dc       __imp_?setBackgroundColor@QWidget@@UAEXABVQColor@@@Z 1001e6dc     qt-mt323:qt-mt323.dll
 0002:000006e0       __imp_?setBackgroundMode@QWidget@@UAEXW4BackgroundMode@Qt@@@Z 1001e6e0     qt-mt323:qt-mt323.dll
 0002:000006e4       __imp_?setBackgroundOrigin@QWidget@@UAEXW4BackgroundOrigin@1@@Z 1001e6e4     qt-mt323:qt-mt323.dll
 0002:000006e8       __imp_?setBackgroundPixmap@QWidget@@UAEXABVQPixmap@@@Z 1001e6e8     qt-mt323:qt-mt323.dll
 0002:000006ec       __imp_?setCaption@QDockWindow@@UAEXABVQString@@@Z 1001e6ec     qt-mt323:qt-mt323.dll
 0002:000006f0       __imp_?setCaption@QWidget@@UAEXABVQString@@@Z 1001e6f0     qt-mt323:qt-mt323.dll
 0002:000006f4       __imp_?setCheckable@QPopupMenu@@UAEX_N@Z 1001e6f4     qt-mt323:qt-mt323.dll
 0002:000006f8       __imp_?setCloseMode@QDockWindow@@UAEXH@Z 1001e6f8     qt-mt323:qt-mt323.dll
 0002:000006fc       __imp_?setColumnAlignment@QListView@@UAEXHH@Z 1001e6fc     qt-mt323:qt-mt323.dll
 0002:00000700       __imp_?setColumnText@QListView@@UAEXHABVQIconSet@@ABVQString@@@Z 1001e700     qt-mt323:qt-mt323.dll
 0002:00000704       __imp_?setColumnText@QListView@@UAEXHABVQString@@@Z 1001e704     qt-mt323:qt-mt323.dll
 0002:00000708       __imp_?setColumnWidth@QListView@@UAEXHH@Z 1001e708     qt-mt323:qt-mt323.dll
 0002:0000070c       __imp_?setColumnWidthMode@QListView@@UAEXHW4WidthMode@1@@Z 1001e70c     qt-mt323:qt-mt323.dll
 0002:00000710       __imp_?setContentsPos@QListView@@UAEXHH@Z 1001e710     qt-mt323:qt-mt323.dll
 0002:00000714       __imp_?setCornerWidget@QScrollView@@UAEXPAVQWidget@@@Z 1001e714     qt-mt323:qt-mt323.dll
 0002:00000718       __imp_?setCurrentItem@QListView@@UAEXPAVQListViewItem@@@Z 1001e718     qt-mt323:qt-mt323.dll
 0002:0000071c       __imp_?setCursor@QWidget@@UAEXABVQCursor@@@Z 1001e71c     qt-mt323:qt-mt323.dll
 0002:00000720       __imp_?setDefaultRenameAction@QListView@@UAEXW4RenameAction@1@@Z 1001e720     qt-mt323:qt-mt323.dll
 0002:00000724       __imp_?setDragAutoScroll@QScrollView@@UAEX_N@Z 1001e724     qt-mt323:qt-mt323.dll
 0002:00000728       __imp_?setDragEnabled@QListViewItem@@UAEX_N@Z 1001e728     qt-mt323:qt-mt323.dll
 0002:0000072c       __imp_?setDropEnabled@QListViewItem@@UAEX_N@Z 1001e72c     qt-mt323:qt-mt323.dll
 0002:00000730       __imp_?setEnabled@QAction@@UAEX_N@Z 1001e730     qt-mt323:qt-mt323.dll
 0002:00000734       __imp_?setEnabled@QListViewItem@@UAEX_N@Z 1001e734     qt-mt323:qt-mt323.dll
 0002:00000738       __imp_?setEnabled@QScrollView@@UAEX_N@Z 1001e738     qt-mt323:qt-mt323.dll
 0002:0000073c       __imp_?setEnabled@QWidget@@UAEX_N@Z 1001e73c     qt-mt323:qt-mt323.dll
 0002:00000740       __imp_?setEraseColor@QWidget@@UAEXABVQColor@@@Z 1001e740     qt-mt323:qt-mt323.dll
 0002:00000744       __imp_?setErasePixmap@QWidget@@UAEXABVQPixmap@@@Z 1001e744     qt-mt323:qt-mt323.dll
 0002:00000748       __imp_?setExpandable@QListViewItem@@UAEX_N@Z 1001e748     qt-mt323:qt-mt323.dll
 0002:0000074c       __imp_?setFirstItemActive@QPopupMenu@@EAEXXZ 1001e74c     qt-mt323:qt-mt323.dll
 0002:00000750       __imp_?setFixedExtentHeight@QDockWindow@@UAEXH@Z 1001e750     qt-mt323:qt-mt323.dll
 0002:00000754       __imp_?setFixedExtentWidth@QDockWindow@@UAEXH@Z 1001e754     qt-mt323:qt-mt323.dll
 0002:00000758       __imp_?setFocus@QWidget@@UAEXXZ 1001e758     qt-mt323:qt-mt323.dll
 0002:0000075c       __imp_?setFocusPolicy@QWidget@@UAEXW4FocusPolicy@1@@Z 1001e75c     qt-mt323:qt-mt323.dll
 0002:00000760       __imp_?setFocusProxy@QWidget@@UAEXPAV1@@Z 1001e760     qt-mt323:qt-mt323.dll
 0002:00000764       __imp_?setFont@QListView@@UAEXABVQFont@@@Z 1001e764     qt-mt323:qt-mt323.dll
 0002:00000768       __imp_?setFont@QPopupMenu@@UAEXABVQFont@@@Z 1001e768     qt-mt323:qt-mt323.dll
 0002:0000076c       __imp_?setFont@QWidget@@UAEXABVQFont@@@Z 1001e76c     qt-mt323:qt-mt323.dll
 0002:00000770       __imp_?setFrameRect@QFrame@@UAEXABVQRect@@@Z 1001e770     qt-mt323:qt-mt323.dll
 0002:00000774       __imp_?setFrameStyle@QFrame@@UAEXH@Z 1001e774     qt-mt323:qt-mt323.dll
 0002:00000778       __imp_?setGeometry@QBoxLayout@@UAEXABVQRect@@@Z 1001e778     qt-mt323:qt-mt323.dll
 0002:0000077c       __imp_?setGeometry@QWidget@@UAEXABVQRect@@@Z 1001e77c     qt-mt323:qt-mt323.dll
 0002:00000780       __imp_?setGeometry@QWidget@@UAEXHHHH@Z 1001e780     qt-mt323:qt-mt323.dll
 0002:00000784       __imp_?setHBarGeometry@QScrollView@@MAEXAAVQScrollBar@@HHHH@Z 1001e784     qt-mt323:qt-mt323.dll
 0002:00000788       __imp_?setHScrollBarMode@QScrollView@@UAEXW4ScrollBarMode@1@@Z 1001e788     qt-mt323:qt-mt323.dll
 0002:0000078c       __imp_?setHeight@QListViewItem@@MAEXH@Z 1001e78c     qt-mt323:qt-mt323.dll
 0002:00000790       __imp_?setHorizontallyStretchable@QDockWindow@@UAEX_N@Z 1001e790     qt-mt323:qt-mt323.dll
 0002:00000794       __imp_?setIcon@QWidget@@UAEXABVQPixmap@@@Z 1001e794     qt-mt323:qt-mt323.dll
 0002:00000798       __imp_?setIconSet@QAction@@UAEXABVQIconSet@@@Z 1001e798     qt-mt323:qt-mt323.dll
 0002:0000079c       __imp_?setIconText@QWidget@@UAEXABVQString@@@Z 1001e79c     qt-mt323:qt-mt323.dll
 0002:000007a0       __imp_?setId@QMenuData@@UAEXHH@Z 1001e7a0     qt-mt323:qt-mt323.dll
 0002:000007a4       __imp_?setItemMargin@QListView@@UAEXH@Z 1001e7a4     qt-mt323:qt-mt323.dll
 0002:000007a8       __imp_?setKeyCompression@QWidget@@MAEX_N@Z 1001e7a8     qt-mt323:qt-mt323.dll
 0002:000007ac       __imp_?setLabel@QToolBar@@UAEXABVQString@@@Z 1001e7ac     qt-mt323:qt-mt323.dll
 0002:000007b0       __imp_?setLineWidth@QFrame@@UAEXH@Z 1001e7b0     qt-mt323:qt-mt323.dll
 0002:000007b4       __imp_?setMargin@QFrame@@UAEXH@Z 1001e7b4     qt-mt323:qt-mt323.dll
 0002:000007b8       __imp_?setMargin@QLayout@@UAEXH@Z 1001e7b8     qt-mt323:qt-mt323.dll
 0002:000007bc       __imp_?setMargins@QScrollView@@MAEXHHHH@Z 1001e7bc     qt-mt323:qt-mt323.dll
 0002:000007c0       __imp_?setMask@QWidget@@UAEXABVQBitmap@@@Z 1001e7c0     qt-mt323:qt-mt323.dll
 0002:000007c4       __imp_?setMask@QWidget@@UAEXABVQRegion@@@Z 1001e7c4     qt-mt323:qt-mt323.dll
 0002:000007c8       __imp_?setMaximumSize@QWidget@@UAEXHH@Z 1001e7c8     qt-mt323:qt-mt323.dll
 0002:000007cc       __imp_?setMenuBar@QLayout@@UAEXPAVQMenuBar@@@Z 1001e7cc     qt-mt323:qt-mt323.dll
 0002:000007d0       __imp_?setMenuText@QAction@@UAEXABVQString@@@Z 1001e7d0     qt-mt323:qt-mt323.dll
 0002:000007d4       __imp_?setMicroFocusHint@QWidget@@MAEXHHHH_NPAVQFont@@@Z 1001e7d4     qt-mt323:qt-mt323.dll
 0002:000007d8       __imp_?setMidLineWidth@QFrame@@UAEXH@Z 1001e7d8     qt-mt323:qt-mt323.dll
 0002:000007dc       __imp_?setMinimumSize@QToolBar@@UAEXHH@Z 1001e7dc     qt-mt323:qt-mt323.dll
 0002:000007e0       __imp_?setMinimumSize@QWidget@@UAEXHH@Z 1001e7e0     qt-mt323:qt-mt323.dll
 0002:000007e4       __imp_?setMouseTracking@QWidget@@UAEX_N@Z 1001e7e4     qt-mt323:qt-mt323.dll
 0002:000007e8       __imp_?setMovingEnabled@QDockWindow@@UAEX_N@Z 1001e7e8     qt-mt323:qt-mt323.dll
 0002:000007ec       __imp_?setMultiLinesEnabled@QListViewItem@@UAEX_N@Z 1001e7ec     qt-mt323:qt-mt323.dll
 0002:000007f0       __imp_?setMultiSelection@QListView@@UAEX_N@Z 1001e7f0     qt-mt323:qt-mt323.dll
 0002:000007f4       __imp_?setName@QObject@@UAEXPBD@Z 1001e7f4     qt-mt323:qt-mt323.dll
 0002:000007f8       __imp_?setNewLine@QDockWindow@@UAEX_N@Z 1001e7f8     qt-mt323:qt-mt323.dll
 0002:000007fc       __imp_?setOffset@QDockWindow@@UAEXH@Z 1001e7fc     qt-mt323:qt-mt323.dll
 0002:00000800       __imp_?setOn@QAction@@UAEX_N@Z 1001e800     qt-mt323:qt-mt323.dll
 0002:00000804       __imp_?setOpaqueMoving@QDockWindow@@UAEX_N@Z 1001e804     qt-mt323:qt-mt323.dll
 0002:00000808       __imp_?setOpen@QListView@@UAEXPAVQListViewItem@@_N@Z 1001e808     qt-mt323:qt-mt323.dll
 0002:0000080c       __imp_?setOpen@QListViewItem@@UAEX_N@Z 1001e80c     qt-mt323:qt-mt323.dll
 0002:00000810       __imp_?setOrientation@QDockWindow@@UAEXW4Orientation@Qt@@@Z 1001e810     qt-mt323:qt-mt323.dll
 0002:00000814       __imp_?setOrientation@QToolBar@@UAEXW4Orientation@Qt@@@Z 1001e814     qt-mt323:qt-mt323.dll
 0002:00000818       __imp_?setPalette@QListView@@UAEXABVQPalette@@@Z 1001e818     qt-mt323:qt-mt323.dll
 0002:0000081c       __imp_?setPalette@QWidget@@UAEXABVQPalette@@@Z 1001e81c     qt-mt323:qt-mt323.dll
 0002:00000820       __imp_?setPaletteBackgroundColor@QWidget@@UAEXABVQColor@@@Z 1001e820     qt-mt323:qt-mt323.dll
 0002:00000824       __imp_?setPaletteBackgroundPixmap@QWidget@@UAEXABVQPixmap@@@Z 1001e824     qt-mt323:qt-mt323.dll
 0002:00000828       __imp_?setPixmap@QListViewItem@@UAEXHABVQPixmap@@@Z 1001e828     qt-mt323:qt-mt323.dll
 0002:0000082c       __imp_?setProperty@QObject@@UAE_NPBDABVQVariant@@@Z 1001e82c     qt-mt323:qt-mt323.dll
 0002:00000830       __imp_?setRenameEnabled@QListViewItem@@UAEXH_N@Z 1001e830     qt-mt323:qt-mt323.dll
 0002:00000834       __imp_?setResizeEnabled@QDockWindow@@UAEX_N@Z 1001e834     qt-mt323:qt-mt323.dll
 0002:00000838       __imp_?setResizeMode@QListView@@UAEXW4ResizeMode@1@@Z 1001e838     qt-mt323:qt-mt323.dll
 0002:0000083c       __imp_?setResizePolicy@QScrollView@@UAEXW4ResizePolicy@1@@Z 1001e83c     qt-mt323:qt-mt323.dll
 0002:00000840       __imp_?setResolution@QPaintDevice@@UAEXH@Z 1001e840     qt-mt323:qt-mt323.dll
 0002:00000844       __imp_?setRootIsDecorated@QListView@@UAEX_N@Z 1001e844     qt-mt323:qt-mt323.dll
 0002:00000848       __imp_?setSelectable@QListViewItem@@UAEX_N@Z 1001e848     qt-mt323:qt-mt323.dll
 0002:0000084c       __imp_?setSelected@QListView@@UAEXPAVQListViewItem@@_N@Z 1001e84c     qt-mt323:qt-mt323.dll
 0002:00000850       __imp_?setSelected@QListViewItem@@UAEX_N@Z 1001e850     qt-mt323:qt-mt323.dll
 0002:00000854       __imp_?setShowSortIndicator@QListView@@UAEX_N@Z 1001e854     qt-mt323:qt-mt323.dll
 0002:00000858       __imp_?setShowToolTips@QListView@@UAEX_N@Z 1001e858     qt-mt323:qt-mt323.dll
 0002:0000085c       __imp_?setSizeIncrement@QWidget@@UAEXHH@Z 1001e85c     qt-mt323:qt-mt323.dll
 0002:00000860       __imp_?setSizePolicy@QWidget@@UAEXVQSizePolicy@@@Z 1001e860     qt-mt323:qt-mt323.dll
 0002:00000864       __imp_?setSorting@QListView@@UAEXH_N@Z 1001e864     qt-mt323:qt-mt323.dll
 0002:00000868       __imp_?setSpacing@QLayout@@UAEXH@Z 1001e868     qt-mt323:qt-mt323.dll
 0002:0000086c       __imp_?setStatusTip@QAction@@UAEXABVQString@@@Z 1001e86c     qt-mt323:qt-mt323.dll
 0002:00000870       __imp_?setStretchableWidget@QToolBar@@UAEXPAVQWidget@@@Z 1001e870     qt-mt323:qt-mt323.dll
 0002:00000874       __imp_?setText@QAction@@UAEXABVQString@@@Z 1001e874     qt-mt323:qt-mt323.dll
 0002:00000878       __imp_?setText@QListViewItem@@UAEXHABVQString@@@Z 1001e878     qt-mt323:qt-mt323.dll
 0002:0000087c       __imp_?setToggleAction@QAction@@UAEX_N@Z 1001e87c     qt-mt323:qt-mt323.dll
 0002:00000880       __imp_?setToolTip@QAction@@UAEXABVQString@@@Z 1001e880     qt-mt323:qt-mt323.dll
 0002:00000884       __imp_?setTreeStepSize@QListView@@UAEXH@Z 1001e884     qt-mt323:qt-mt323.dll
 0002:00000888       __imp_?setUpdatesEnabled@QWidget@@UAEX_N@Z 1001e888     qt-mt323:qt-mt323.dll
 0002:0000088c       __imp_?setVBarGeometry@QScrollView@@MAEXAAVQScrollBar@@HHHH@Z 1001e88c     qt-mt323:qt-mt323.dll
 0002:00000890       __imp_?setVScrollBarMode@QScrollView@@UAEXW4ScrollBarMode@1@@Z 1001e890     qt-mt323:qt-mt323.dll
 0002:00000894       __imp_?setVerticallyStretchable@QDockWindow@@UAEX_N@Z 1001e894     qt-mt323:qt-mt323.dll
 0002:00000898       __imp_?setWFlags@QWidget@@MAEXI@Z 1001e898     qt-mt323:qt-mt323.dll
 0002:0000089c       __imp_?setWState@QWidget@@MAEXI@Z 1001e89c     qt-mt323:qt-mt323.dll
 0002:000008a0       __imp_?setWhatsThis@QAction@@UAEXABVQString@@@Z 1001e8a0     qt-mt323:qt-mt323.dll
 0002:000008a4       __imp_?setWidget@QDockWindow@@UAEXPAVQWidget@@@Z 1001e8a4     qt-mt323:qt-mt323.dll
 0002:000008a8       __imp_?setup@QListViewItem@@UAEXXZ 1001e8a8     qt-mt323:qt-mt323.dll
 0002:000008ac       __imp_?show@QListView@@UAEXXZ 1001e8ac     qt-mt323:qt-mt323.dll
 0002:000008b0       __imp_?show@QPopupMenu@@UAEXXZ 1001e8b0     qt-mt323:qt-mt323.dll
 0002:000008b4       __imp_?show@QToolBar@@UAEXXZ 1001e8b4     qt-mt323:qt-mt323.dll
 0002:000008b8       __imp_?show@QWidget@@UAEXXZ 1001e8b8     qt-mt323:qt-mt323.dll
 0002:000008bc       __imp_?showEvent@QDockWindow@@MAEXPAVQShowEvent@@@Z 1001e8bc     qt-mt323:qt-mt323.dll
 0002:000008c0       __imp_?showEvent@QListView@@MAEXPAVQShowEvent@@@Z 1001e8c0     qt-mt323:qt-mt323.dll
 0002:000008c4       __imp_?showEvent@QTabWidget@@MAEXPAVQShowEvent@@@Z 1001e8c4     qt-mt323:qt-mt323.dll
 0002:000008c8       __imp_?showEvent@QWidget@@MAEXPAVQShowEvent@@@Z 1001e8c8     qt-mt323:qt-mt323.dll
 0002:000008cc       __imp_?showMaximized@QWidget@@UAEXXZ 1001e8cc     qt-mt323:qt-mt323.dll
 0002:000008d0       __imp_?showMinimized@QWidget@@UAEXXZ 1001e8d0     qt-mt323:qt-mt323.dll
 0002:000008d4       __imp_?showNormal@QWidget@@UAEXXZ 1001e8d4     qt-mt323:qt-mt323.dll
 0002:000008d8       __imp_?showPage@QTabWidget@@UAEXPAVQWidget@@@Z 1001e8d8     qt-mt323:qt-mt323.dll
 0002:000008dc       __imp_?sizeHint@QBoxLayout@@UBE?AVQSize@@XZ 1001e8dc     qt-mt323:qt-mt323.dll
 0002:000008e0       __imp_?sizeHint@QDockWindow@@UBE?AVQSize@@XZ 1001e8e0     qt-mt323:qt-mt323.dll
 0002:000008e4       __imp_?sizeHint@QHBox@@UBE?AVQSize@@XZ 1001e8e4     qt-mt323:qt-mt323.dll
 0002:000008e8       __imp_?sizeHint@QListView@@UBE?AVQSize@@XZ 1001e8e8     qt-mt323:qt-mt323.dll
 0002:000008ec       __imp_?sizeHint@QPopupMenu@@UBE?AVQSize@@XZ 1001e8ec     qt-mt323:qt-mt323.dll
 0002:000008f0       __imp_?sizeHint@QTabWidget@@UBE?AVQSize@@XZ 1001e8f0     qt-mt323:qt-mt323.dll
 0002:000008f4       __imp_?sizeHint@QWidget@@UBE?AVQSize@@XZ 1001e8f4     qt-mt323:qt-mt323.dll
 0002:000008f8       __imp_?sizePolicy@QWidget@@UBE?AVQSizePolicy@@XZ 1001e8f8     qt-mt323:qt-mt323.dll
 0002:000008fc       __imp_?sort@QListView@@UAEXXZ 1001e8fc     qt-mt323:qt-mt323.dll
 0002:00000900       __imp_?sort@QListViewItem@@UAEXXZ 1001e900     qt-mt323:qt-mt323.dll
 0002:00000904       __imp_?sortChildItems@QListViewItem@@UAEXH_N@Z 1001e904     qt-mt323:qt-mt323.dll
 0002:00000908       __imp_?spacerItem@QLayoutItem@@UAEPAVQSpacerItem@@XZ 1001e908     qt-mt323:qt-mt323.dll
 0002:0000090c       __imp_?startDrag@QListView@@MAEXXZ 1001e90c     qt-mt323:qt-mt323.dll
 0002:00000910       __imp_?startRename@QListViewItem@@UAEXH@Z 1001e910     qt-mt323:qt-mt323.dll
 0002:00000914       __imp_?styleChange@QFrame@@MAEXAAVQStyle@@@Z 1001e914     qt-mt323:qt-mt323.dll
 0002:00000918       __imp_?styleChange@QListView@@MAEXAAVQStyle@@@Z 1001e918     qt-mt323:qt-mt323.dll
 0002:0000091c       __imp_?styleChange@QPopupMenu@@MAEXAAVQStyle@@@Z 1001e91c     qt-mt323:qt-mt323.dll
 0002:00000920       __imp_?styleChange@QTabWidget@@MAEXAAVQStyle@@@Z 1001e920     qt-mt323:qt-mt323.dll
 0002:00000924       __imp_?styleChange@QToolBar@@MAEXAAVQStyle@@@Z 1001e924     qt-mt323:qt-mt323.dll
 0002:00000928       __imp_?styleChange@QWidget@@MAEXAAVQStyle@@@Z 1001e928     qt-mt323:qt-mt323.dll
 0002:0000092c       __imp_?tabletEvent@QWidget@@MAEXPAVQTabletEvent@@@Z 1001e92c     qt-mt323:qt-mt323.dll
 0002:00000930       __imp_?takeItem@QListView@@UAEXPAVQListViewItem@@@Z 1001e930     qt-mt323:qt-mt323.dll
 0002:00000934       __imp_?takeItem@QListViewItem@@UAEXPAV1@@Z 1001e934     qt-mt323:qt-mt323.dll
 0002:00000938       __imp_?text@QListViewItem@@UBE?AVQString@@H@Z 1001e938     qt-mt323:qt-mt323.dll
 0002:0000093c       __imp_?timerEvent@QObject@@MAEXPAVQTimerEvent@@@Z 1001e93c     qt-mt323:qt-mt323.dll
 0002:00000940       __imp_?timerEvent@QPopupMenu@@MAEXPAVQTimerEvent@@@Z 1001e940     qt-mt323:qt-mt323.dll
 0002:00000944       __imp_?undock@QDockWindow@@UAEXPAVQWidget@@@Z 1001e944     qt-mt323:qt-mt323.dll
 0002:00000948       __imp_?undock@QDockWindow@@UAEXXZ 1001e948     qt-mt323:qt-mt323.dll
 0002:0000094c       __imp_?unsetCursor@QWidget@@UAEXXZ 1001e94c     qt-mt323:qt-mt323.dll
 0002:00000950       __imp_?updateItem@QPopupMenu@@UAEXH@Z 1001e950     qt-mt323:qt-mt323.dll
 0002:00000954       __imp_?updateMask@QTabWidget@@MAEXXZ 1001e954     qt-mt323:qt-mt323.dll
 0002:00000958       __imp_?updateMask@QWidget@@MAEXXZ 1001e958     qt-mt323:qt-mt323.dll
 0002:0000095c       __imp_?viewportContextMenuEvent@QScrollView@@MAEXPAVQContextMenuEvent@@@Z 1001e95c     qt-mt323:qt-mt323.dll
 0002:00000960       __imp_?viewportDragEnterEvent@QScrollView@@MAEXPAVQDragEnterEvent@@@Z 1001e960     qt-mt323:qt-mt323.dll
 0002:00000964       __imp_?viewportDragLeaveEvent@QScrollView@@MAEXPAVQDragLeaveEvent@@@Z 1001e964     qt-mt323:qt-mt323.dll
 0002:00000968       __imp_?viewportDragMoveEvent@QScrollView@@MAEXPAVQDragMoveEvent@@@Z 1001e968     qt-mt323:qt-mt323.dll
 0002:0000096c       __imp_?viewportDropEvent@QScrollView@@MAEXPAVQDropEvent@@@Z 1001e96c     qt-mt323:qt-mt323.dll
 0002:00000970       __imp_?viewportMouseDoubleClickEvent@QScrollView@@MAEXPAVQMouseEvent@@@Z 1001e970     qt-mt323:qt-mt323.dll
 0002:00000974       __imp_?viewportMouseMoveEvent@QScrollView@@MAEXPAVQMouseEvent@@@Z 1001e974     qt-mt323:qt-mt323.dll
 0002:00000978       __imp_?viewportMousePressEvent@QScrollView@@MAEXPAVQMouseEvent@@@Z 1001e978     qt-mt323:qt-mt323.dll
 0002:0000097c       __imp_?viewportMouseReleaseEvent@QScrollView@@MAEXPAVQMouseEvent@@@Z 1001e97c     qt-mt323:qt-mt323.dll
 0002:00000980       __imp_?viewportPaintEvent@QScrollView@@MAEXPAVQPaintEvent@@@Z 1001e980     qt-mt323:qt-mt323.dll
 0002:00000984       __imp_?viewportResizeEvent@QListView@@MAEXPAVQResizeEvent@@@Z 1001e984     qt-mt323:qt-mt323.dll
 0002:00000988       __imp_?viewportWheelEvent@QScrollView@@MAEXPAVQWheelEvent@@@Z 1001e988     qt-mt323:qt-mt323.dll
 0002:0000098c       __imp_?wheelEvent@QScrollView@@MAEXPAVQWheelEvent@@@Z 1001e98c     qt-mt323:qt-mt323.dll
 0002:00000990       __imp_?wheelEvent@QWidget@@MAEXPAVQWheelEvent@@@Z 1001e990     qt-mt323:qt-mt323.dll
 0002:00000994       __imp_?widget@QLayoutItem@@UAEPAVQWidget@@XZ 1001e994     qt-mt323:qt-mt323.dll
 0002:00000998       __imp_?width@QListViewItem@@UBEHABVQFontMetrics@@PBVQListView@@H@Z 1001e998     qt-mt323:qt-mt323.dll
 0002:0000099c       __imp_?winEvent@QWidget@@MAE_NPAUtagMSG@@@Z 1001e99c     qt-mt323:qt-mt323.dll
 0002:000009a0       __imp_?windowActivationChange@QListView@@MAEX_N@Z 1001e9a0     qt-mt323:qt-mt323.dll
 0002:000009a4       __imp_?windowActivationChange@QWidget@@MAEX_N@Z 1001e9a4     qt-mt323:qt-mt323.dll
 0002:000009a8       __imp_?write@QGList@@MBEAAVQDataStream@@AAV2@PAX@Z 1001e9a8     qt-mt323:qt-mt323.dll
 0002:000009ac       __imp_?null@QString@@2V1@A 1001e9ac     qt-mt323:qt-mt323.dll
 0002:000009b0       __imp_?shared_null@QString@@0PAUQStringData@@A 1001e9b0     qt-mt323:qt-mt323.dll
 0002:000009b4       __imp_??_7?$QPtrList@VQDockWindow@@@@6B@ 1001e9b4     qt-mt323:qt-mt323.dll
 0002:000009b8       __imp_?accept@QDialog@@MAEXXZ 1001e9b8     qt-mt323:qt-mt323.dll
 0002:000009bc       __imp_?closeEvent@QDialog@@MAEXPAVQCloseEvent@@@Z 1001e9bc     qt-mt323:qt-mt323.dll
 0002:000009c0       __imp_?contextMenuEvent@QDialog@@MAEXPAVQContextMenuEvent@@@Z 1001e9c0     qt-mt323:qt-mt323.dll
 0002:000009c4       __imp_?done@QDialog@@MAEXH@Z 1001e9c4     qt-mt323:qt-mt323.dll
 0002:000009c8       __imp_?eventFilter@QDialog@@MAE_NPAVQObject@@PAVQEvent@@@Z 1001e9c8     qt-mt323:qt-mt323.dll
 0002:000009cc       __imp_?hide@QDialog@@UAEXXZ 1001e9cc     qt-mt323:qt-mt323.dll
 0002:000009d0       __imp_?keyPressEvent@QDialog@@MAEXPAVQKeyEvent@@@Z 1001e9d0     qt-mt323:qt-mt323.dll
 0002:000009d4       __imp_?minimumSizeHint@QDialog@@UBE?AVQSize@@XZ 1001e9d4     qt-mt323:qt-mt323.dll
 0002:000009d8       __imp_?move@QDialog@@UAEXHH@Z 1001e9d8     qt-mt323:qt-mt323.dll
 0002:000009dc       __imp_?reject@QDialog@@MAEXXZ 1001e9dc     qt-mt323:qt-mt323.dll
 0002:000009e0       __imp_?resize@QDialog@@UAEXHH@Z 1001e9e0     qt-mt323:qt-mt323.dll
 0002:000009e4       __imp_?resizeEvent@QDialog@@MAEXPAVQResizeEvent@@@Z 1001e9e4     qt-mt323:qt-mt323.dll
 0002:000009e8       __imp_?setGeometry@QDialog@@UAEXABVQRect@@@Z 1001e9e8     qt-mt323:qt-mt323.dll
 0002:000009ec       __imp_?setGeometry@QDialog@@UAEXHHHH@Z 1001e9ec     qt-mt323:qt-mt323.dll
 0002:000009f0       __imp_?show@QDialog@@UAEXXZ 1001e9f0     qt-mt323:qt-mt323.dll
 0002:000009f4       __imp_?sizeHint@QDialog@@UBE?AVQSize@@XZ 1001e9f4     qt-mt323:qt-mt323.dll
 0002:000009f8       __imp_?truncate@QString@@QAEXI@Z 1001e9f8     qt-mt323:qt-mt323.dll
 0002:000009fc       __imp_?section@QString@@QBE?AV1@DHHH@Z 1001e9fc     qt-mt323:qt-mt323.dll
 0002:00000a00       __imp_??9@YA_NABVQString@@PBD@Z 1001ea00     qt-mt323:qt-mt323.dll
 0002:00000a04       __imp_??0?$QMap@VQString@@H@@QAE@XZ 1001ea04     qt-mt323:qt-mt323.dll
 0002:00000a08       __imp_?begin@?$QMap@VQString@@H@@QBE?AV?$QMapConstIterator@VQString@@H@@XZ 1001ea08     qt-mt323:qt-mt323.dll
 0002:00000a0c       __imp_?end@?$QMap@VQString@@H@@QBE?AV?$QMapConstIterator@VQString@@H@@XZ 1001ea0c     qt-mt323:qt-mt323.dll
 0002:00000a10       __imp_??A?$QMap@VQString@@H@@QAEAAHABVQString@@@Z 1001ea10     qt-mt323:qt-mt323.dll
 0002:00000a14       __imp_??1QTextStream@@UAE@XZ 1001ea14     qt-mt323:qt-mt323.dll
 0002:00000a18       __imp_??4QDomNode@@QAEAAV0@ABV0@@Z 1001ea18     qt-mt323:qt-mt323.dll
 0002:00000a1c       __imp_?firstChild@QDomNode@@UBE?AV1@XZ 1001ea1c     qt-mt323:qt-mt323.dll
 0002:00000a20       __imp_?nextSibling@QDomNode@@UBE?AV1@XZ 1001ea20     qt-mt323:qt-mt323.dll
 0002:00000a24       __imp_?isNull@QDomNode@@QBE_NXZ 1001ea24     qt-mt323:qt-mt323.dll
 0002:00000a28       __imp_?toElement@QDomNode@@QAE?AVQDomElement@@XZ 1001ea28     qt-mt323:qt-mt323.dll
 0002:00000a2c       __imp_?setContent@QDomDocument@@QAE_NPAVQIODevice@@PAVQString@@PAH2@Z 1001ea2c     qt-mt323:qt-mt323.dll
 0002:00000a30       __imp_?attribute@QDomElement@@QBE?AVQString@@ABV2@0@Z 1001ea30     qt-mt323:qt-mt323.dll
 0002:00000a34       __imp_?tagName@QDomElement@@QBE?AVQString@@XZ 1001ea34     qt-mt323:qt-mt323.dll
 0002:00000a38       __imp_??0QGDict@@IAE@IW4KeyType@0@_N1@Z 1001ea38     qt-mt323:qt-mt323.dll
 0002:00000a3c       __imp_??1QGDict@@MAE@XZ    1001ea3c     qt-mt323:qt-mt323.dll
 0002:00000a40       __imp_?clear@QGDict@@MAEXXZ 1001ea40     qt-mt323:qt-mt323.dll
 0002:00000a44       __imp_?read@QGDict@@MAEAAVQDataStream@@AAV2@AAPAX@Z 1001ea44     qt-mt323:qt-mt323.dll
 0002:00000a48       __imp_?write@QGDict@@MBEAAVQDataStream@@AAV2@PAX@Z 1001ea48     qt-mt323:qt-mt323.dll
 0002:00000a4c       __imp_?sort@QStringList@@QAEXXZ 1001ea4c     qt-mt323:qt-mt323.dll
 0002:00000a50       __imp_??0QColor@@QAE@PBD@Z 1001ea50     qt-mt323:qt-mt323.dll
 0002:00000a54       __imp_?setPaletteForegroundColor@QWidget@@QAEXABVQColor@@@Z 1001ea54     qt-mt323:qt-mt323.dll
 0002:00000a58       __imp_?itemAbove@QListViewItem@@QAEPAV1@XZ 1001ea58     qt-mt323:qt-mt323.dll
 0002:00000a5c       __imp_?itemBelow@QListViewItem@@QAEPAV1@XZ 1001ea5c     qt-mt323:qt-mt323.dll
 0002:00000a60       __imp_?isSelectable@QListViewItem@@QBE_NXZ 1001ea60     qt-mt323:qt-mt323.dll
 0002:00000a64       __imp_?moveItem@QListViewItem@@QAEXPAV1@@Z 1001ea64     qt-mt323:qt-mt323.dll
 0002:00000a68       __imp_?header@QListView@@QBEPAVQHeader@@XZ 1001ea68     qt-mt323:qt-mt323.dll
 0002:00000a6c       __imp_?ensureItemVisible@QListView@@QAEXPBVQListViewItem@@@Z 1001ea6c     qt-mt323:qt-mt323.dll
 0002:00000a70       __imp_?setSelectionMode@QListView@@QAEXW4SelectionMode@1@@Z 1001ea70     qt-mt323:qt-mt323.dll
 0002:00000a74       __imp_?lastItem@QListView@@QBEPAVQListViewItem@@XZ 1001ea74     qt-mt323:qt-mt323.dll
 0002:00000a78       __imp_?sortColumn@QListView@@QBEHXZ 1001ea78     qt-mt323:qt-mt323.dll
 0002:00000a7c       __imp_?setSortColumn@QListView@@QAEXH@Z 1001ea7c     qt-mt323:qt-mt323.dll
 0002:00000a80       __imp_?sortOrder@QListView@@QBE?AW4SortOrder@Qt@@XZ 1001ea80     qt-mt323:qt-mt323.dll
 0002:00000a84       __imp_?setSortOrder@QListView@@QAEXW4SortOrder@Qt@@@Z 1001ea84     qt-mt323:qt-mt323.dll
 0002:00000a88       __imp_?setIconSet@QPushButton@@QAEXABVQIconSet@@@Z 1001ea88     qt-mt323:qt-mt323.dll
 0002:00000a8c       __imp_?text@QClipboard@@QBE?AVQString@@XZ 1001ea8c     qt-mt323:qt-mt323.dll
 0002:00000a90       __imp_?setText@QClipboard@@QAEXABVQString@@@Z 1001ea90     qt-mt323:qt-mt323.dll
 0002:00000a94       __imp_?clipboard@QApplication@@SAPAVQClipboard@@XZ 1001ea94     qt-mt323:qt-mt323.dll
 0002:00000a98       __imp_?setMaxValue@QSpinBox@@QAEXH@Z 1001ea98     qt-mt323:qt-mt323.dll
 0002:00000a9c       __imp_?value@QSpinBox@@QBEHXZ 1001ea9c     qt-mt323:qt-mt323.dll
 0002:00000aa0       __imp_?selectedId@QButtonGroup@@QBEHXZ 1001eaa0     qt-mt323:qt-mt323.dll
 0002:00000aa4       __imp_?insertStringList@QComboBox@@QAEXABVQStringList@@H@Z 1001eaa4     qt-mt323:qt-mt323.dll
 0002:00000aa8       __imp_?currentText@QComboBox@@QBE?AVQString@@XZ 1001eaa8     qt-mt323:qt-mt323.dll
 0002:00000aac       __imp_??0QDialog@@QAE@PAVQWidget@@PBD_NI@Z 1001eaac     qt-mt323:qt-mt323.dll
 0002:00000ab0       __imp_??1QDialog@@UAE@XZ   1001eab0     qt-mt323:qt-mt323.dll
 0002:00000ab4       __imp_?resize@QDialog@@QAEXABVQSize@@@Z 1001eab4     qt-mt323:qt-mt323.dll
 0002:00000ab8       __imp_?setSizeGripEnabled@QDialog@@QAEX_N@Z 1001eab8     qt-mt323:qt-mt323.dll
 0002:00000abc       __imp_??0QKeySequence@@QAE@ABVQString@@@Z 1001eabc     qt-mt323:qt-mt323.dll
 0002:00000ac0       __imp_??1QKeySequence@@QAE@XZ 1001eac0     qt-mt323:qt-mt323.dll
 0002:00000ac4       __imp_??0QPushButton@@QAE@PAVQWidget@@PBD@Z 1001eac4     qt-mt323:qt-mt323.dll
 0002:00000ac8       __imp_??1QPushButton@@UAE@XZ 1001eac8     qt-mt323:qt-mt323.dll
 0002:00000acc       __imp_?setFrameShape@QFrame@@QAEXW4Shape@1@@Z 1001eacc     qt-mt323:qt-mt323.dll
 0002:00000ad0       __imp_?setFrameShadow@QFrame@@QAEXW4Shadow@1@@Z 1001ead0     qt-mt323:qt-mt323.dll
 0002:00000ad4       __imp_??0QLabel@@QAE@PAVQWidget@@PBDI@Z 1001ead4     qt-mt323:qt-mt323.dll
 0002:00000ad8       __imp_??1QLabel@@UAE@XZ    1001ead8     qt-mt323:qt-mt323.dll
 0002:00000adc       __imp_??0QComboBox@@QAE@_NPAVQWidget@@PBD@Z 1001eadc     qt-mt323:qt-mt323.dll
 0002:00000ae0       __imp_??1QComboBox@@UAE@XZ 1001eae0     qt-mt323:qt-mt323.dll
 0002:00000ae4       __imp_?changeTab@QTabWidget@@QAEXPAVQWidget@@ABVQString@@@Z 1001eae4     qt-mt323:qt-mt323.dll
 0002:00000ae8       __imp_??0QLineEdit@@QAE@PAVQWidget@@PBD@Z 1001eae8     qt-mt323:qt-mt323.dll
 0002:00000aec       __imp_??1QLineEdit@@UAE@XZ 1001eaec     qt-mt323:qt-mt323.dll
 0002:00000af0       __imp_??0QSpinBox@@QAE@PAVQWidget@@PBD@Z 1001eaf0     qt-mt323:qt-mt323.dll
 0002:00000af4       __imp_??1QSpinBox@@UAE@XZ  1001eaf4     qt-mt323:qt-mt323.dll
 0002:00000af8       __imp_?setMinValue@QSpinBox@@QAEXH@Z 1001eaf8     qt-mt323:qt-mt323.dll
 0002:00000afc       __imp_??0QTable@@QAE@PAVQWidget@@PBD@Z 1001eafc     qt-mt323:qt-mt323.dll
 0002:00000b00       __imp_??1QTable@@UAE@XZ    1001eb00     qt-mt323:qt-mt323.dll
 0002:00000b04       __imp_?horizontalHeader@QTable@@QBEPAVQHeader@@XZ 1001eb04     qt-mt323:qt-mt323.dll
 0002:00000b08       __imp_??1QLayoutItem@@UAE@XZ 1001eb08     qt-mt323:qt-mt323.dll
 0002:00000b0c       __imp_??0QSpacerItem@@QAE@HHW4SizeType@QSizePolicy@@0@Z 1001eb0c     qt-mt323:qt-mt323.dll
 0002:00000b10       __imp_??0QGridLayout@@QAE@PAVQWidget@@HHHHPBD@Z 1001eb10     qt-mt323:qt-mt323.dll
 0002:00000b14       __imp_??1QGridLayout@@UAE@XZ 1001eb14     qt-mt323:qt-mt323.dll
 0002:00000b18       __imp_?addWidget@QGridLayout@@QAEXPAVQWidget@@HHH@Z 1001eb18     qt-mt323:qt-mt323.dll
 0002:00000b1c       __imp_?addLayout@QGridLayout@@QAEXPAVQLayout@@HH@Z 1001eb1c     qt-mt323:qt-mt323.dll
 0002:00000b20       __imp_?addWidget@QBoxLayout@@QAEXPAVQWidget@@HH@Z 1001eb20     qt-mt323:qt-mt323.dll
 0002:00000b24       __imp_?addLayout@QBoxLayout@@QAEXPAVQLayout@@H@Z 1001eb24     qt-mt323:qt-mt323.dll
 0002:00000b28       __imp_??0QHBoxLayout@@QAE@PAVQWidget@@HHPBD@Z 1001eb28     qt-mt323:qt-mt323.dll
 0002:00000b2c       __imp_??1QHBoxLayout@@UAE@XZ 1001eb2c     qt-mt323:qt-mt323.dll
 0002:00000b30       __imp_??0QVBoxLayout@@QAE@PAVQWidget@@HHPBD@Z 1001eb30     qt-mt323:qt-mt323.dll
 0002:00000b34       __imp_??1QVBoxLayout@@UAE@XZ 1001eb34     qt-mt323:qt-mt323.dll
 0002:00000b38       __imp_?activateNextCell@QTable@@MAEXXZ 1001eb38     qt-mt323:qt-mt323.dll
 0002:00000b3c       __imp_?addItem@QGridLayout@@UAEXPAVQLayoutItem@@@Z 1001eb3c     qt-mt323:qt-mt323.dll
 0002:00000b40       __imp_?addSelection@QTable@@UAEHABVQTableSelection@@@Z 1001eb40     qt-mt323:qt-mt323.dll
 0002:00000b44       __imp_?adjustColumn@QTable@@UAEXH@Z 1001eb44     qt-mt323:qt-mt323.dll
 0002:00000b48       __imp_?adjustRow@QTable@@UAEXH@Z 1001eb48     qt-mt323:qt-mt323.dll
 0002:00000b4c       __imp_?beginEdit@QTable@@MAEPAVQWidget@@HH_N@Z 1001eb4c     qt-mt323:qt-mt323.dll
 0002:00000b50       __imp_?cellGeometry@QTable@@UBE?AVQRect@@HH@Z 1001eb50     qt-mt323:qt-mt323.dll
 0002:00000b54       __imp_?cellRect@QTable@@UBE?AVQRect@@HH@Z 1001eb54     qt-mt323:qt-mt323.dll
 0002:00000b58       __imp_?cellWidget@QTable@@UBEPAVQWidget@@HH@Z 1001eb58     qt-mt323:qt-mt323.dll
 0002:00000b5c       __imp_?className@QComboBox@@UBEPBDXZ 1001eb5c     qt-mt323:qt-mt323.dll
 0002:00000b60       __imp_?className@QGridLayout@@UBEPBDXZ 1001eb60     qt-mt323:qt-mt323.dll
 0002:00000b64       __imp_?className@QHBoxLayout@@UBEPBDXZ 1001eb64     qt-mt323:qt-mt323.dll
 0002:00000b68       __imp_?className@QLabel@@UBEPBDXZ 1001eb68     qt-mt323:qt-mt323.dll
 0002:00000b6c       __imp_?className@QLineEdit@@UBEPBDXZ 1001eb6c     qt-mt323:qt-mt323.dll
 0002:00000b70       __imp_?className@QPushButton@@UBEPBDXZ 1001eb70     qt-mt323:qt-mt323.dll
 0002:00000b74       __imp_?className@QSpinBox@@UBEPBDXZ 1001eb74     qt-mt323:qt-mt323.dll
 0002:00000b78       __imp_?className@QTable@@UBEPBDXZ 1001eb78     qt-mt323:qt-mt323.dll
 0002:00000b7c       __imp_?className@QVBoxLayout@@UBEPBDXZ 1001eb7c     qt-mt323:qt-mt323.dll
 0002:00000b80       __imp_?cleanText@QSpinBox@@UBE?AVQString@@XZ 1001eb80     qt-mt323:qt-mt323.dll
 0002:00000b84       __imp_?clear@QLineEdit@@UAEXXZ 1001eb84     qt-mt323:qt-mt323.dll
 0002:00000b88       __imp_?clearCell@QTable@@UAEXHH@Z 1001eb88     qt-mt323:qt-mt323.dll
 0002:00000b8c       __imp_?clearCellWidget@QTable@@UAEXHH@Z 1001eb8c     qt-mt323:qt-mt323.dll
 0002:00000b90       __imp_?clearValidator@QLineEdit@@UAEXXZ 1001eb90     qt-mt323:qt-mt323.dll
 0002:00000b94       __imp_?columnAt@QTable@@UBEHH@Z 1001eb94     qt-mt323:qt-mt323.dll
 0002:00000b98       __imp_?columnClicked@QTable@@MAEXH@Z 1001eb98     qt-mt323:qt-mt323.dll
 0002:00000b9c       __imp_?columnIndexChanged@QTable@@MAEXHHH@Z 1001eb9c     qt-mt323:qt-mt323.dll
 0002:00000ba0       __imp_?columnPos@QTable@@UBEHH@Z 1001eba0     qt-mt323:qt-mt323.dll
 0002:00000ba4       __imp_?columnWidth@QTable@@UBEHH@Z 1001eba4     qt-mt323:qt-mt323.dll
 0002:00000ba8       __imp_?columnWidthChanged@QTable@@MAEXH@Z 1001eba8     qt-mt323:qt-mt323.dll
 0002:00000bac       __imp_?contentsContextMenuEvent@QTable@@MAEXPAVQContextMenuEvent@@@Z 1001ebac     qt-mt323:qt-mt323.dll
 0002:00000bb0       __imp_?contentsDragEnterEvent@QTable@@MAEXPAVQDragEnterEvent@@@Z 1001ebb0     qt-mt323:qt-mt323.dll
 0002:00000bb4       __imp_?contentsDragLeaveEvent@QTable@@MAEXPAVQDragLeaveEvent@@@Z 1001ebb4     qt-mt323:qt-mt323.dll
 0002:00000bb8       __imp_?contentsDragMoveEvent@QTable@@MAEXPAVQDragMoveEvent@@@Z 1001ebb8     qt-mt323:qt-mt323.dll
 0002:00000bbc       __imp_?contentsDropEvent@QTable@@MAEXPAVQDropEvent@@@Z 1001ebbc     qt-mt323:qt-mt323.dll
 0002:00000bc0       __imp_?contentsMouseDoubleClickEvent@QTable@@MAEXPAVQMouseEvent@@@Z 1001ebc0     qt-mt323:qt-mt323.dll
 0002:00000bc4       __imp_?contentsMouseMoveEvent@QTable@@MAEXPAVQMouseEvent@@@Z 1001ebc4     qt-mt323:qt-mt323.dll
 0002:00000bc8       __imp_?contentsMousePressEvent@QTable@@MAEXPAVQMouseEvent@@@Z 1001ebc8     qt-mt323:qt-mt323.dll
 0002:00000bcc       __imp_?contentsMouseReleaseEvent@QTable@@MAEXPAVQMouseEvent@@@Z 1001ebcc     qt-mt323:qt-mt323.dll
 0002:00000bd0       __imp_?contextMenuEvent@QLineEdit@@MAEXPAVQContextMenuEvent@@@Z 1001ebd0     qt-mt323:qt-mt323.dll
 0002:00000bd4       __imp_?copy@QLineEdit@@UBEXXZ 1001ebd4     qt-mt323:qt-mt323.dll
 0002:00000bd8       __imp_?createEditor@QTable@@MBEPAVQWidget@@HH_N@Z 1001ebd8     qt-mt323:qt-mt323.dll
 0002:00000bdc       __imp_?createPopupMenu@QLineEdit@@MAEPAVQPopupMenu@@XZ 1001ebdc     qt-mt323:qt-mt323.dll
 0002:00000be0       __imp_?currentSelection@QTable@@UBEHXZ 1001ebe0     qt-mt323:qt-mt323.dll
 0002:00000be4       __imp_?cut@QLineEdit@@UAEXXZ 1001ebe4     qt-mt323:qt-mt323.dll
 0002:00000be8       __imp_?deselect@QLineEdit@@UAEXXZ 1001ebe8     qt-mt323:qt-mt323.dll
 0002:00000bec       __imp_?dragEnterEvent@QLineEdit@@MAEXPAVQDragEnterEvent@@@Z 1001ebec     qt-mt323:qt-mt323.dll
 0002:00000bf0       __imp_?dragLeaveEvent@QLineEdit@@MAEXPAVQDragLeaveEvent@@@Z 1001ebf0     qt-mt323:qt-mt323.dll
 0002:00000bf4       __imp_?dragMoveEvent@QLineEdit@@MAEXPAVQDragMoveEvent@@@Z 1001ebf4     qt-mt323:qt-mt323.dll
 0002:00000bf8       __imp_?dragObject@QTable@@MAEPAVQDragObject@@XZ 1001ebf8     qt-mt323:qt-mt323.dll
 0002:00000bfc       __imp_?drawButton@QPushButton@@MAEXPAVQPainter@@@Z 1001ebfc     qt-mt323:qt-mt323.dll
 0002:00000c00       __imp_?drawButtonLabel@QPushButton@@MAEXPAVQPainter@@@Z 1001ec00     qt-mt323:qt-mt323.dll
 0002:00000c04       __imp_?drawContents@QLabel@@MAEXPAVQPainter@@@Z 1001ec04     qt-mt323:qt-mt323.dll
 0002:00000c08       __imp_?drawContents@QLineEdit@@MAEXPAVQPainter@@@Z 1001ec08     qt-mt323:qt-mt323.dll
 0002:00000c0c       __imp_?drawContents@QTable@@EAEXPAVQPainter@@@Z 1001ec0c     qt-mt323:qt-mt323.dll
 0002:00000c10       __imp_?drawContents@QTable@@MAEXPAVQPainter@@HHHH@Z 1001ec10     qt-mt323:qt-mt323.dll
 0002:00000c14       __imp_?drawContentsOffset@QScrollView@@MAEXPAVQPainter@@HHHHHH@Z 1001ec14     qt-mt323:qt-mt323.dll
 0002:00000c18       __imp_?dropEvent@QLineEdit@@MAEXPAVQDropEvent@@@Z 1001ec18     qt-mt323:qt-mt323.dll
 0002:00000c1c       __imp_?editCell@QTable@@UAEXHH_N@Z 1001ec1c     qt-mt323:qt-mt323.dll
 0002:00000c20       __imp_?enabledChange@QButton@@MAEX_N@Z 1001ec20     qt-mt323:qt-mt323.dll
 0002:00000c24       __imp_?endEdit@QTable@@MAEXHH_N0@Z 1001ec24     qt-mt323:qt-mt323.dll
 0002:00000c28       __imp_?event@QLineEdit@@MAE_NPAVQEvent@@@Z 1001ec28     qt-mt323:qt-mt323.dll
 0002:00000c2c       __imp_?eventFilter@QComboBox@@UAE_NPAVQObject@@PAVQEvent@@@Z 1001ec2c     qt-mt323:qt-mt323.dll
 0002:00000c30       __imp_?eventFilter@QSpinBox@@MAE_NPAVQObject@@PAVQEvent@@@Z 1001ec30     qt-mt323:qt-mt323.dll
 0002:00000c34       __imp_?eventFilter@QTable@@UAE_NPAVQObject@@PAVQEvent@@@Z 1001ec34     qt-mt323:qt-mt323.dll
 0002:00000c38       __imp_?expanding@QGridLayout@@UBE?AW4ExpandData@QSizePolicy@@XZ 1001ec38     qt-mt323:qt-mt323.dll
 0002:00000c3c       __imp_?expanding@QSpacerItem@@UBE?AW4ExpandData@QSizePolicy@@XZ 1001ec3c     qt-mt323:qt-mt323.dll
 0002:00000c40       __imp_?focusInEvent@QComboBox@@MAEXPAVQFocusEvent@@@Z 1001ec40     qt-mt323:qt-mt323.dll
 0002:00000c44       __imp_?focusInEvent@QLineEdit@@MAEXPAVQFocusEvent@@@Z 1001ec44     qt-mt323:qt-mt323.dll
 0002:00000c48       __imp_?focusInEvent@QPushButton@@MAEXPAVQFocusEvent@@@Z 1001ec48     qt-mt323:qt-mt323.dll
 0002:00000c4c       __imp_?focusInEvent@QTable@@MAEXPAVQFocusEvent@@@Z 1001ec4c     qt-mt323:qt-mt323.dll
 0002:00000c50       __imp_?focusOutEvent@QComboBox@@MAEXPAVQFocusEvent@@@Z 1001ec50     qt-mt323:qt-mt323.dll
 0002:00000c54       __imp_?focusOutEvent@QLineEdit@@MAEXPAVQFocusEvent@@@Z 1001ec54     qt-mt323:qt-mt323.dll
 0002:00000c58       __imp_?focusOutEvent@QPushButton@@MAEXPAVQFocusEvent@@@Z 1001ec58     qt-mt323:qt-mt323.dll
 0002:00000c5c       __imp_?focusOutEvent@QTable@@MAEXPAVQFocusEvent@@@Z 1001ec5c     qt-mt323:qt-mt323.dll
 0002:00000c60       __imp_?fontChange@QLabel@@MAEXABVQFont@@@Z 1001ec60     qt-mt323:qt-mt323.dll
 0002:00000c64       __imp_?geometry@QSpacerItem@@UBE?AVQRect@@XZ 1001ec64     qt-mt323:qt-mt323.dll
 0002:00000c68       __imp_?hasHeightForWidth@QGridLayout@@UBE_NXZ 1001ec68     qt-mt323:qt-mt323.dll
 0002:00000c6c       __imp_?hasHeightForWidth@QLayoutItem@@UBE_NXZ 1001ec6c     qt-mt323:qt-mt323.dll
 0002:00000c70       __imp_?heightForWidth@QGridLayout@@UBEHH@Z 1001ec70     qt-mt323:qt-mt323.dll
 0002:00000c74       __imp_?heightForWidth@QLabel@@UBEHH@Z 1001ec74     qt-mt323:qt-mt323.dll
 0002:00000c78       __imp_?heightForWidth@QLayoutItem@@UBEHH@Z 1001ec78     qt-mt323:qt-mt323.dll
 0002:00000c7c       __imp_?hideColumn@QTable@@UAEXH@Z 1001ec7c     qt-mt323:qt-mt323.dll
 0002:00000c80       __imp_?hideRow@QTable@@UAEXH@Z 1001ec80     qt-mt323:qt-mt323.dll
 0002:00000c84       __imp_?hitButton@QButton@@MBE_NABVQPoint@@@Z 1001ec84     qt-mt323:qt-mt323.dll
 0002:00000c88       __imp_?imComposeEvent@QLineEdit@@MAEXPAVQIMEvent@@@Z 1001ec88     qt-mt323:qt-mt323.dll
 0002:00000c8c       __imp_?imEndEvent@QLineEdit@@MAEXPAVQIMEvent@@@Z 1001ec8c     qt-mt323:qt-mt323.dll
 0002:00000c90       __imp_?imStartEvent@QLineEdit@@MAEXPAVQIMEvent@@@Z 1001ec90     qt-mt323:qt-mt323.dll
 0002:00000c94       __imp_?insert@QLineEdit@@UAEXABVQString@@@Z 1001ec94     qt-mt323:qt-mt323.dll
 0002:00000c98       __imp_?insertColumns@QTable@@UAEXHH@Z 1001ec98     qt-mt323:qt-mt323.dll
 0002:00000c9c       __imp_?insertRows@QTable@@UAEXHH@Z 1001ec9c     qt-mt323:qt-mt323.dll
 0002:00000ca0       __imp_?insertWidget@QTable@@MAEXHHPAVQWidget@@@Z 1001eca0     qt-mt323:qt-mt323.dll
 0002:00000ca4       __imp_?interpretText@QSpinBox@@MAEXXZ 1001eca4     qt-mt323:qt-mt323.dll
 0002:00000ca8       __imp_?invalidate@QGridLayout@@UAEXXZ 1001eca8     qt-mt323:qt-mt323.dll
 0002:00000cac       __imp_?invalidate@QLayoutItem@@UAEXXZ 1001ecac     qt-mt323:qt-mt323.dll
 0002:00000cb0       __imp_?isEmpty@QSpacerItem@@UBE_NXZ 1001ecb0     qt-mt323:qt-mt323.dll
 0002:00000cb4       __imp_?item@QTable@@UBEPAVQTableItem@@HH@Z 1001ecb4     qt-mt323:qt-mt323.dll
 0002:00000cb8       __imp_?iterator@QGridLayout@@UAE?AVQLayoutIterator@@XZ 1001ecb8     qt-mt323:qt-mt323.dll
 0002:00000cbc       __imp_?iterator@QLayoutItem@@UAE?AVQLayoutIterator@@XZ 1001ecbc     qt-mt323:qt-mt323.dll
 0002:00000cc0       __imp_?keyPressEvent@QButton@@MAEXPAVQKeyEvent@@@Z 1001ecc0     qt-mt323:qt-mt323.dll
 0002:00000cc4       __imp_?keyPressEvent@QComboBox@@MAEXPAVQKeyEvent@@@Z 1001ecc4     qt-mt323:qt-mt323.dll
 0002:00000cc8       __imp_?keyPressEvent@QLineEdit@@MAEXPAVQKeyEvent@@@Z 1001ecc8     qt-mt323:qt-mt323.dll
 0002:00000ccc       __imp_?keyPressEvent@QTable@@MAEXPAVQKeyEvent@@@Z 1001eccc     qt-mt323:qt-mt323.dll
 0002:00000cd0       __imp_?keyReleaseEvent@QButton@@MAEXPAVQKeyEvent@@@Z 1001ecd0     qt-mt323:qt-mt323.dll
 0002:00000cd4       __imp_?layout@QLayoutItem@@UAEPAVQLayout@@XZ 1001ecd4     qt-mt323:qt-mt323.dll
 0002:00000cd8       __imp_?leaveEvent@QSpinBox@@MAEXPAVQEvent@@@Z 1001ecd8     qt-mt323:qt-mt323.dll
 0002:00000cdc       __imp_?mapTextToValue@QSpinBox@@MAEHPA_N@Z 1001ecdc     qt-mt323:qt-mt323.dll
 0002:00000ce0       __imp_?mapValueToText@QSpinBox@@MAE?AVQString@@H@Z 1001ece0     qt-mt323:qt-mt323.dll
 0002:00000ce4       __imp_?maximumSize@QGridLayout@@UBE?AVQSize@@XZ 1001ece4     qt-mt323:qt-mt323.dll
 0002:00000ce8       __imp_?maximumSize@QSpacerItem@@UBE?AVQSize@@XZ 1001ece8     qt-mt323:qt-mt323.dll
 0002:00000cec       __imp_?metaObject@QComboBox@@UBEPAVQMetaObject@@XZ 1001ecec     qt-mt323:qt-mt323.dll
 0002:00000cf0       __imp_?metaObject@QGridLayout@@UBEPAVQMetaObject@@XZ 1001ecf0     qt-mt323:qt-mt323.dll
 0002:00000cf4       __imp_?metaObject@QHBoxLayout@@UBEPAVQMetaObject@@XZ 1001ecf4     qt-mt323:qt-mt323.dll
 0002:00000cf8       __imp_?metaObject@QLabel@@UBEPAVQMetaObject@@XZ 1001ecf8     qt-mt323:qt-mt323.dll
 0002:00000cfc       __imp_?metaObject@QLineEdit@@UBEPAVQMetaObject@@XZ 1001ecfc     qt-mt323:qt-mt323.dll
 0002:00000d00       __imp_?metaObject@QPushButton@@UBEPAVQMetaObject@@XZ 1001ed00     qt-mt323:qt-mt323.dll
 0002:00000d04       __imp_?metaObject@QSpinBox@@UBEPAVQMetaObject@@XZ 1001ed04     qt-mt323:qt-mt323.dll
 0002:00000d08       __imp_?metaObject@QTable@@UBEPAVQMetaObject@@XZ 1001ed08     qt-mt323:qt-mt323.dll
 0002:00000d0c       __imp_?metaObject@QVBoxLayout@@UBEPAVQMetaObject@@XZ 1001ed0c     qt-mt323:qt-mt323.dll
 0002:00000d10       __imp_?minimumSize@QGridLayout@@UBE?AVQSize@@XZ 1001ed10     qt-mt323:qt-mt323.dll
 0002:00000d14       __imp_?minimumSize@QSpacerItem@@UBE?AVQSize@@XZ 1001ed14     qt-mt323:qt-mt323.dll
 0002:00000d18       __imp_?minimumSizeHint@QLabel@@UBE?AVQSize@@XZ 1001ed18     qt-mt323:qt-mt323.dll
 0002:00000d1c       __imp_?minimumSizeHint@QLineEdit@@UBE?AVQSize@@XZ 1001ed1c     qt-mt323:qt-mt323.dll
 0002:00000d20       __imp_?minimumSizeHint@QScrollView@@UBE?AVQSize@@XZ 1001ed20     qt-mt323:qt-mt323.dll
 0002:00000d24       __imp_?minimumSizeHint@QSpinBox@@UBE?AVQSize@@XZ 1001ed24     qt-mt323:qt-mt323.dll
 0002:00000d28       __imp_?mouseDoubleClickEvent@QComboBox@@MAEXPAVQMouseEvent@@@Z 1001ed28     qt-mt323:qt-mt323.dll
 0002:00000d2c       __imp_?mouseDoubleClickEvent@QLineEdit@@MAEXPAVQMouseEvent@@@Z 1001ed2c     qt-mt323:qt-mt323.dll
 0002:00000d30       __imp_?mouseMoveEvent@QButton@@MAEXPAVQMouseEvent@@@Z 1001ed30     qt-mt323:qt-mt323.dll
 0002:00000d34       __imp_?mouseMoveEvent@QComboBox@@MAEXPAVQMouseEvent@@@Z 1001ed34     qt-mt323:qt-mt323.dll
 0002:00000d38       __imp_?mouseMoveEvent@QLineEdit@@MAEXPAVQMouseEvent@@@Z 1001ed38     qt-mt323:qt-mt323.dll
 0002:00000d3c       __imp_?mousePressEvent@QButton@@MAEXPAVQMouseEvent@@@Z 1001ed3c     qt-mt323:qt-mt323.dll
 0002:00000d40       __imp_?mousePressEvent@QComboBox@@MAEXPAVQMouseEvent@@@Z 1001ed40     qt-mt323:qt-mt323.dll
 0002:00000d44       __imp_?mousePressEvent@QLineEdit@@MAEXPAVQMouseEvent@@@Z 1001ed44     qt-mt323:qt-mt323.dll
 0002:00000d48       __imp_?mouseReleaseEvent@QButton@@MAEXPAVQMouseEvent@@@Z 1001ed48     qt-mt323:qt-mt323.dll
 0002:00000d4c       __imp_?mouseReleaseEvent@QComboBox@@MAEXPAVQMouseEvent@@@Z 1001ed4c     qt-mt323:qt-mt323.dll
 0002:00000d50       __imp_?mouseReleaseEvent@QLineEdit@@MAEXPAVQMouseEvent@@@Z 1001ed50     qt-mt323:qt-mt323.dll
 0002:00000d54       __imp_?move@QPushButton@@UAEXHH@Z 1001ed54     qt-mt323:qt-mt323.dll
 0002:00000d58       __imp_?numCols@QTable@@UBEHXZ 1001ed58     qt-mt323:qt-mt323.dll
 0002:00000d5c       __imp_?numRows@QTable@@UBEHXZ 1001ed5c     qt-mt323:qt-mt323.dll
 0002:00000d60       __imp_?paintCell@QTable@@UAEXPAVQPainter@@HHABVQRect@@_N@Z 1001ed60     qt-mt323:qt-mt323.dll
 0002:00000d64       __imp_?paintCell@QTable@@UAEXPAVQPainter@@HHABVQRect@@_NABVQColorGroup@@@Z 1001ed64     qt-mt323:qt-mt323.dll
 0002:00000d68       __imp_?paintEmptyArea@QTable@@MAEXPAVQPainter@@HHHH@Z 1001ed68     qt-mt323:qt-mt323.dll
 0002:00000d6c       __imp_?paintEvent@QButton@@MAEXPAVQPaintEvent@@@Z 1001ed6c     qt-mt323:qt-mt323.dll
 0002:00000d70       __imp_?paintEvent@QComboBox@@MAEXPAVQPaintEvent@@@Z 1001ed70     qt-mt323:qt-mt323.dll
 0002:00000d74       __imp_?paintEvent@QTable@@MAEXPAVQPaintEvent@@@Z 1001ed74     qt-mt323:qt-mt323.dll
 0002:00000d78       __imp_?paintFocus@QTable@@UAEXPAVQPainter@@ABVQRect@@@Z 1001ed78     qt-mt323:qt-mt323.dll
 0002:00000d7c       __imp_?paste@QLineEdit@@UAEXXZ 1001ed7c     qt-mt323:qt-mt323.dll
 0002:00000d80       __imp_?pixmap@QTable@@UBE?AVQPixmap@@HH@Z 1001ed80     qt-mt323:qt-mt323.dll
 0002:00000d84       __imp_?popup@QComboBox@@UAEXXZ 1001ed84     qt-mt323:qt-mt323.dll
 0002:00000d88       __imp_?prefix@QSpinBox@@UBE?AVQString@@XZ 1001ed88     qt-mt323:qt-mt323.dll
 0002:00000d8c       __imp_?qt_cast@QComboBox@@UAEPAXPBD@Z 1001ed8c     qt-mt323:qt-mt323.dll
 0002:00000d90       __imp_?qt_cast@QGridLayout@@UAEPAXPBD@Z 1001ed90     qt-mt323:qt-mt323.dll
 0002:00000d94       __imp_?qt_cast@QHBoxLayout@@UAEPAXPBD@Z 1001ed94     qt-mt323:qt-mt323.dll
 0002:00000d98       __imp_?qt_cast@QLabel@@UAEPAXPBD@Z 1001ed98     qt-mt323:qt-mt323.dll
 0002:00000d9c       __imp_?qt_cast@QLineEdit@@UAEPAXPBD@Z 1001ed9c     qt-mt323:qt-mt323.dll
 0002:00000da0       __imp_?qt_cast@QPushButton@@UAEPAXPBD@Z 1001eda0     qt-mt323:qt-mt323.dll
 0002:00000da4       __imp_?qt_cast@QSpinBox@@UAEPAXPBD@Z 1001eda4     qt-mt323:qt-mt323.dll
 0002:00000da8       __imp_?qt_cast@QTable@@UAEPAXPBD@Z 1001eda8     qt-mt323:qt-mt323.dll
 0002:00000dac       __imp_?qt_cast@QVBoxLayout@@UAEPAXPBD@Z 1001edac     qt-mt323:qt-mt323.dll
 0002:00000db0       __imp_?qt_emit@QComboBox@@UAE_NHPAUQUObject@@@Z 1001edb0     qt-mt323:qt-mt323.dll
 0002:00000db4       __imp_?qt_emit@QGridLayout@@UAE_NHPAUQUObject@@@Z 1001edb4     qt-mt323:qt-mt323.dll
 0002:00000db8       __imp_?qt_emit@QHBoxLayout@@UAE_NHPAUQUObject@@@Z 1001edb8     qt-mt323:qt-mt323.dll
 0002:00000dbc       __imp_?qt_emit@QLabel@@UAE_NHPAUQUObject@@@Z 1001edbc     qt-mt323:qt-mt323.dll
 0002:00000dc0       __imp_?qt_emit@QLineEdit@@UAE_NHPAUQUObject@@@Z 1001edc0     qt-mt323:qt-mt323.dll
 0002:00000dc4       __imp_?qt_emit@QPushButton@@UAE_NHPAUQUObject@@@Z 1001edc4     qt-mt323:qt-mt323.dll
 0002:00000dc8       __imp_?qt_emit@QSpinBox@@UAE_NHPAUQUObject@@@Z 1001edc8     qt-mt323:qt-mt323.dll
 0002:00000dcc       __imp_?qt_emit@QTable@@UAE_NHPAUQUObject@@@Z 1001edcc     qt-mt323:qt-mt323.dll
 0002:00000dd0       __imp_?qt_emit@QVBoxLayout@@UAE_NHPAUQUObject@@@Z 1001edd0     qt-mt323:qt-mt323.dll
 0002:00000dd4       __imp_?qt_invoke@QComboBox@@UAE_NHPAUQUObject@@@Z 1001edd4     qt-mt323:qt-mt323.dll
 0002:00000dd8       __imp_?qt_invoke@QGridLayout@@UAE_NHPAUQUObject@@@Z 1001edd8     qt-mt323:qt-mt323.dll
 0002:00000ddc       __imp_?qt_invoke@QHBoxLayout@@UAE_NHPAUQUObject@@@Z 1001eddc     qt-mt323:qt-mt323.dll
 0002:00000de0       __imp_?qt_invoke@QLabel@@UAE_NHPAUQUObject@@@Z 1001ede0     qt-mt323:qt-mt323.dll
 0002:00000de4       __imp_?qt_invoke@QLineEdit@@UAE_NHPAUQUObject@@@Z 1001ede4     qt-mt323:qt-mt323.dll
 0002:00000de8       __imp_?qt_invoke@QPushButton@@UAE_NHPAUQUObject@@@Z 1001ede8     qt-mt323:qt-mt323.dll
 0002:00000dec       __imp_?qt_invoke@QSpinBox@@UAE_NHPAUQUObject@@@Z 1001edec     qt-mt323:qt-mt323.dll
 0002:00000df0       __imp_?qt_invoke@QTable@@UAE_NHPAUQUObject@@@Z 1001edf0     qt-mt323:qt-mt323.dll
 0002:00000df4       __imp_?qt_invoke@QVBoxLayout@@UAE_NHPAUQUObject@@@Z 1001edf4     qt-mt323:qt-mt323.dll
 0002:00000df8       __imp_?qt_property@QComboBox@@UAE_NHHPAVQVariant@@@Z 1001edf8     qt-mt323:qt-mt323.dll
 0002:00000dfc       __imp_?qt_property@QGridLayout@@UAE_NHHPAVQVariant@@@Z 1001edfc     qt-mt323:qt-mt323.dll
 0002:00000e00       __imp_?qt_property@QHBoxLayout@@UAE_NHHPAVQVariant@@@Z 1001ee00     qt-mt323:qt-mt323.dll
 0002:00000e04       __imp_?qt_property@QLabel@@UAE_NHHPAVQVariant@@@Z 1001ee04     qt-mt323:qt-mt323.dll
 0002:00000e08       __imp_?qt_property@QLineEdit@@UAE_NHHPAVQVariant@@@Z 1001ee08     qt-mt323:qt-mt323.dll
 0002:00000e0c       __imp_?qt_property@QPushButton@@UAE_NHHPAVQVariant@@@Z 1001ee0c     qt-mt323:qt-mt323.dll
 0002:00000e10       __imp_?qt_property@QSpinBox@@UAE_NHHPAVQVariant@@@Z 1001ee10     qt-mt323:qt-mt323.dll
 0002:00000e14       __imp_?qt_property@QTable@@UAE_NHHPAVQVariant@@@Z 1001ee14     qt-mt323:qt-mt323.dll
 0002:00000e18       __imp_?qt_property@QVBoxLayout@@UAE_NHHPAVQVariant@@@Z 1001ee18     qt-mt323:qt-mt323.dll
 0002:00000e1c       __imp_?rangeChange@QSpinBox@@MAEXXZ 1001ee1c     qt-mt323:qt-mt323.dll
 0002:00000e20       __imp_?redo@QLineEdit@@UAEXXZ 1001ee20     qt-mt323:qt-mt323.dll
 0002:00000e24       __imp_?removeColumn@QTable@@UAEXH@Z 1001ee24     qt-mt323:qt-mt323.dll
 0002:00000e28       __imp_?removeColumns@QTable@@UAEXABV?$QMemArray@H@@@Z 1001ee28     qt-mt323:qt-mt323.dll
 0002:00000e2c       __imp_?removeRow@QTable@@UAEXH@Z 1001ee2c     qt-mt323:qt-mt323.dll
 0002:00000e30       __imp_?removeRows@QTable@@UAEXABV?$QMemArray@H@@@Z 1001ee30     qt-mt323:qt-mt323.dll
 0002:00000e34       __imp_?removeSelection@QTable@@UAEXABVQTableSelection@@@Z 1001ee34     qt-mt323:qt-mt323.dll
 0002:00000e38       __imp_?removeSelection@QTable@@UAEXH@Z 1001ee38     qt-mt323:qt-mt323.dll
 0002:00000e3c       __imp_?resize@QPushButton@@UAEXHH@Z 1001ee3c     qt-mt323:qt-mt323.dll
 0002:00000e40       __imp_?resizeData@QTable@@MAEXH@Z 1001ee40     qt-mt323:qt-mt323.dll
 0002:00000e44       __imp_?resizeEvent@QComboBox@@MAEXPAVQResizeEvent@@@Z 1001ee44     qt-mt323:qt-mt323.dll
 0002:00000e48       __imp_?resizeEvent@QLabel@@MAEXPAVQResizeEvent@@@Z 1001ee48     qt-mt323:qt-mt323.dll
 0002:00000e4c       __imp_?resizeEvent@QLineEdit@@MAEXPAVQResizeEvent@@@Z 1001ee4c     qt-mt323:qt-mt323.dll
 0002:00000e50       __imp_?resizeEvent@QPushButton@@MAEXPAVQResizeEvent@@@Z 1001ee50     qt-mt323:qt-mt323.dll
 0002:00000e54       __imp_?resizeEvent@QScrollView@@MAEXPAVQResizeEvent@@@Z 1001ee54     qt-mt323:qt-mt323.dll
 0002:00000e58       __imp_?resizeEvent@QSpinBox@@MAEXPAVQResizeEvent@@@Z 1001ee58     qt-mt323:qt-mt323.dll
 0002:00000e5c       __imp_?rowAt@QTable@@UBEHH@Z 1001ee5c     qt-mt323:qt-mt323.dll
 0002:00000e60       __imp_?rowHeight@QTable@@UBEHH@Z 1001ee60     qt-mt323:qt-mt323.dll
 0002:00000e64       __imp_?rowHeightChanged@QTable@@MAEXH@Z 1001ee64     qt-mt323:qt-mt323.dll
 0002:00000e68       __imp_?rowIndexChanged@QTable@@MAEXHHH@Z 1001ee68     qt-mt323:qt-mt323.dll
 0002:00000e6c       __imp_?rowPos@QTable@@UBEHH@Z 1001ee6c     qt-mt323:qt-mt323.dll
 0002:00000e70       __imp_?selectAll@QLineEdit@@UAEXXZ 1001ee70     qt-mt323:qt-mt323.dll
 0002:00000e74       __imp_?selectAll@QSpinBox@@UAEXXZ 1001ee74     qt-mt323:qt-mt323.dll
 0002:00000e78       __imp_?setAccel@QButton@@UAEXABVQKeySequence@@@Z 1001ee78     qt-mt323:qt-mt323.dll
 0002:00000e7c       __imp_?setAlignment@QLabel@@UAEXH@Z 1001ee7c     qt-mt323:qt-mt323.dll
 0002:00000e80       __imp_?setAlignment@QLineEdit@@UAEXH@Z 1001ee80     qt-mt323:qt-mt323.dll
 0002:00000e84       __imp_?setAutoCompletion@QComboBox@@UAEX_N@Z 1001ee84     qt-mt323:qt-mt323.dll
 0002:00000e88       __imp_?setAutoDefault@QPushButton@@UAEX_N@Z 1001ee88     qt-mt323:qt-mt323.dll
 0002:00000e8c       __imp_?setAutoRepeat@QButton@@UAEX_N@Z 1001ee8c     qt-mt323:qt-mt323.dll
 0002:00000e90       __imp_?setAutoResize@QComboBox@@UAEX_N@Z 1001ee90     qt-mt323:qt-mt323.dll
 0002:00000e94       __imp_?setAutoResize@QLabel@@UAEX_N@Z 1001ee94     qt-mt323:qt-mt323.dll
 0002:00000e98       __imp_?setBuddy@QLabel@@UAEXPAVQWidget@@@Z 1001ee98     qt-mt323:qt-mt323.dll
 0002:00000e9c       __imp_?setButtonSymbols@QSpinBox@@UAEXW4ButtonSymbols@1@@Z 1001ee9c     qt-mt323:qt-mt323.dll
 0002:00000ea0       __imp_?setCellContentFromEditor@QTable@@MAEXHH@Z 1001eea0     qt-mt323:qt-mt323.dll
 0002:00000ea4       __imp_?setCellWidget@QTable@@UAEXHHPAVQWidget@@@Z 1001eea4     qt-mt323:qt-mt323.dll
 0002:00000ea8       __imp_?setColStretch@QGridLayout@@UAEXHH@Z 1001eea8     qt-mt323:qt-mt323.dll
 0002:00000eac       __imp_?setColumnMovingEnabled@QTable@@UAEX_N@Z 1001eeac     qt-mt323:qt-mt323.dll
 0002:00000eb0       __imp_?setColumnReadOnly@QTable@@UAEXH_N@Z 1001eeb0     qt-mt323:qt-mt323.dll
 0002:00000eb4       __imp_?setColumnStretchable@QTable@@UAEXH_N@Z 1001eeb4     qt-mt323:qt-mt323.dll
 0002:00000eb8       __imp_?setColumnWidth@QTable@@UAEXHH@Z 1001eeb8     qt-mt323:qt-mt323.dll
 0002:00000ebc       __imp_?setContentsPos@QScrollView@@UAEXHH@Z 1001eebc     qt-mt323:qt-mt323.dll
 0002:00000ec0       __imp_?setCurrentCell@QTable@@UAEXHH@Z 1001eec0     qt-mt323:qt-mt323.dll
 0002:00000ec4       __imp_?setCurrentItem@QComboBox@@UAEXH@Z 1001eec4     qt-mt323:qt-mt323.dll
 0002:00000ec8       __imp_?setCurrentText@QComboBox@@UAEXABVQString@@@Z 1001eec8     qt-mt323:qt-mt323.dll
 0002:00000ecc       __imp_?setCursorPosition@QLineEdit@@UAEXH@Z 1001eecc     qt-mt323:qt-mt323.dll
 0002:00000ed0       __imp_?setDefault@QPushButton@@UAEX_N@Z 1001eed0     qt-mt323:qt-mt323.dll
 0002:00000ed4       __imp_?setDown@QButton@@UAEX_N@Z 1001eed4     qt-mt323:qt-mt323.dll
 0002:00000ed8       __imp_?setDragEnabled@QLineEdit@@UAEX_N@Z 1001eed8     qt-mt323:qt-mt323.dll
 0002:00000edc       __imp_?setDragEnabled@QTable@@UAEX_N@Z 1001eedc     qt-mt323:qt-mt323.dll
 0002:00000ee0       __imp_?setEchoMode@QLineEdit@@UAEXW4EchoMode@1@@Z 1001eee0     qt-mt323:qt-mt323.dll
 0002:00000ee4       __imp_?setEditText@QComboBox@@UAEXABVQString@@@Z 1001eee4     qt-mt323:qt-mt323.dll
 0002:00000ee8       __imp_?setEnabled@QComboBox@@UAEX_N@Z 1001eee8     qt-mt323:qt-mt323.dll
 0002:00000eec       __imp_?setEnabled@QSpinBox@@UAEX_N@Z 1001eeec     qt-mt323:qt-mt323.dll
 0002:00000ef0       __imp_?setEnabled@QTable@@UAEX_N@Z 1001eef0     qt-mt323:qt-mt323.dll
 0002:00000ef4       __imp_?setFocusStyle@QTable@@UAEXW4FocusStyle@1@@Z 1001eef4     qt-mt323:qt-mt323.dll
 0002:00000ef8       __imp_?setFont@QComboBox@@UAEXABVQFont@@@Z 1001eef8     qt-mt323:qt-mt323.dll
 0002:00000efc       __imp_?setFont@QLabel@@UAEXABVQFont@@@Z 1001eefc     qt-mt323:qt-mt323.dll
 0002:00000f00       __imp_?setFont@QLineEdit@@UAEXABVQFont@@@Z 1001ef00     qt-mt323:qt-mt323.dll
 0002:00000f04       __imp_?setFrame@QLineEdit@@UAEX_N@Z 1001ef04     qt-mt323:qt-mt323.dll
 0002:00000f08       __imp_?setGeometry@QGridLayout@@UAEXABVQRect@@@Z 1001ef08     qt-mt323:qt-mt323.dll
 0002:00000f0c       __imp_?setGeometry@QPushButton@@UAEXABVQRect@@@Z 1001ef0c     qt-mt323:qt-mt323.dll
 0002:00000f10       __imp_?setGeometry@QPushButton@@UAEXHHHH@Z 1001ef10     qt-mt323:qt-mt323.dll
 0002:00000f14       __imp_?setGeometry@QSpacerItem@@UAEXABVQRect@@@Z 1001ef14     qt-mt323:qt-mt323.dll
 0002:00000f18       __imp_?setGroup@QButton@@EAEXPAVQButtonGroup@@@Z 1001ef18     qt-mt323:qt-mt323.dll
 0002:00000f1c       __imp_?setInsertionPolicy@QComboBox@@UAEXW4Policy@1@@Z 1001ef1c     qt-mt323:qt-mt323.dll
 0002:00000f20       __imp_?setIsMenuButton@QPushButton@@UAEX_N@Z 1001ef20     qt-mt323:qt-mt323.dll
 0002:00000f24       __imp_?setItem@QTable@@UAEXHHPAVQTableItem@@@Z 1001ef24     qt-mt323:qt-mt323.dll
 0002:00000f28       __imp_?setLeftMargin@QTable@@UAEXH@Z 1001ef28     qt-mt323:qt-mt323.dll
 0002:00000f2c       __imp_?setLineEdit@QComboBox@@UAEXPAVQLineEdit@@@Z 1001ef2c     qt-mt323:qt-mt323.dll
 0002:00000f30       __imp_?setListBox@QComboBox@@UAEXPAVQListBox@@@Z 1001ef30     qt-mt323:qt-mt323.dll
 0002:00000f34       __imp_?setMaxCount@QComboBox@@UAEXH@Z 1001ef34     qt-mt323:qt-mt323.dll
 0002:00000f38       __imp_?setMaxLength@QLineEdit@@UAEXH@Z 1001ef38     qt-mt323:qt-mt323.dll
 0002:00000f3c       __imp_?setMovie@QLabel@@UAEXABVQMovie@@@Z 1001ef3c     qt-mt323:qt-mt323.dll
 0002:00000f40       __imp_?setNum@QLabel@@UAEXH@Z 1001ef40     qt-mt323:qt-mt323.dll
 0002:00000f44       __imp_?setNum@QLabel@@UAEXN@Z 1001ef44     qt-mt323:qt-mt323.dll
 0002:00000f48       __imp_?setNumCols@QTable@@UAEXH@Z 1001ef48     qt-mt323:qt-mt323.dll
 0002:00000f4c       __imp_?setNumRows@QTable@@UAEXH@Z 1001ef4c     qt-mt323:qt-mt323.dll
 0002:00000f50       __imp_?setOn@QPushButton@@UAEX_N@Z 1001ef50     qt-mt323:qt-mt323.dll
 0002:00000f54       __imp_?setPalette@QComboBox@@UAEXABVQPalette@@@Z 1001ef54     qt-mt323:qt-mt323.dll
 0002:00000f58       __imp_?setPalette@QLineEdit@@UAEXABVQPalette@@@Z 1001ef58     qt-mt323:qt-mt323.dll
 0002:00000f5c       __imp_?setPicture@QLabel@@UAEXABVQPicture@@@Z 1001ef5c     qt-mt323:qt-mt323.dll
 0002:00000f60       __imp_?setPixmap@QButton@@UAEXABVQPixmap@@@Z 1001ef60     qt-mt323:qt-mt323.dll
 0002:00000f64       __imp_?setPixmap@QLabel@@UAEXABVQPixmap@@@Z 1001ef64     qt-mt323:qt-mt323.dll
 0002:00000f68       __imp_?setPixmap@QTable@@UAEXHHABVQPixmap@@@Z 1001ef68     qt-mt323:qt-mt323.dll
 0002:00000f6c       __imp_?setPrefix@QSpinBox@@UAEXABVQString@@@Z 1001ef6c     qt-mt323:qt-mt323.dll
 0002:00000f70       __imp_?setReadOnly@QLineEdit@@UAEX_N@Z 1001ef70     qt-mt323:qt-mt323.dll
 0002:00000f74       __imp_?setReadOnly@QTable@@UAEX_N@Z 1001ef74     qt-mt323:qt-mt323.dll
 0002:00000f78       __imp_?setRowHeight@QTable@@UAEXHH@Z 1001ef78     qt-mt323:qt-mt323.dll
 0002:00000f7c       __imp_?setRowMovingEnabled@QTable@@UAEX_N@Z 1001ef7c     qt-mt323:qt-mt323.dll
 0002:00000f80       __imp_?setRowReadOnly@QTable@@UAEXH_N@Z 1001ef80     qt-mt323:qt-mt323.dll
 0002:00000f84       __imp_?setRowStretch@QGridLayout@@UAEXHH@Z 1001ef84     qt-mt323:qt-mt323.dll
 0002:00000f88       __imp_?setRowStretchable@QTable@@UAEXH_N@Z 1001ef88     qt-mt323:qt-mt323.dll
 0002:00000f8c       __imp_?setSelection@QLineEdit@@UAEXHH@Z 1001ef8c     qt-mt323:qt-mt323.dll
 0002:00000f90       __imp_?setSelectionMode@QTable@@UAEXW4SelectionMode@1@@Z 1001ef90     qt-mt323:qt-mt323.dll
 0002:00000f94       __imp_?setShowGrid@QTable@@UAEX_N@Z 1001ef94     qt-mt323:qt-mt323.dll
 0002:00000f98       __imp_?setSizeLimit@QComboBox@@UAEXH@Z 1001ef98     qt-mt323:qt-mt323.dll
 0002:00000f9c       __imp_?setSorting@QTable@@UAEX_N@Z 1001ef9c     qt-mt323:qt-mt323.dll
 0002:00000fa0       __imp_?setSpecialValueText@QSpinBox@@UAEXABVQString@@@Z 1001efa0     qt-mt323:qt-mt323.dll
 0002:00000fa4       __imp_?setState@QButton@@MAEXW4ToggleState@1@@Z 1001efa4     qt-mt323:qt-mt323.dll
 0002:00000fa8       __imp_?setSuffix@QSpinBox@@UAEXABVQString@@@Z 1001efa8     qt-mt323:qt-mt323.dll
 0002:00000fac       __imp_?setText@QButton@@UAEXABVQString@@@Z 1001efac     qt-mt323:qt-mt323.dll
 0002:00000fb0       __imp_?setText@QLabel@@UAEXABVQString@@@Z 1001efb0     qt-mt323:qt-mt323.dll
 0002:00000fb4       __imp_?setText@QLineEdit@@UAEXABVQString@@@Z 1001efb4     qt-mt323:qt-mt323.dll
 0002:00000fb8       __imp_?setText@QTable@@UAEXHHABVQString@@@Z 1001efb8     qt-mt323:qt-mt323.dll
 0002:00000fbc       __imp_?setToggleType@QButton@@MAEXW4ToggleType@1@@Z 1001efbc     qt-mt323:qt-mt323.dll
 0002:00000fc0       __imp_?setTopMargin@QTable@@UAEXH@Z 1001efc0     qt-mt323:qt-mt323.dll
 0002:00000fc4       __imp_?setValidator@QComboBox@@UAEXPBVQValidator@@@Z 1001efc4     qt-mt323:qt-mt323.dll
 0002:00000fc8       __imp_?setValidator@QLineEdit@@UAEXPBVQValidator@@@Z 1001efc8     qt-mt323:qt-mt323.dll
 0002:00000fcc       __imp_?setValidator@QSpinBox@@UAEXPBVQValidator@@@Z 1001efcc     qt-mt323:qt-mt323.dll
 0002:00000fd0       __imp_?setValue@QSpinBox@@UAEXH@Z 1001efd0     qt-mt323:qt-mt323.dll
 0002:00000fd4       __imp_?setWrapping@QSpinBox@@UAEX_N@Z 1001efd4     qt-mt323:qt-mt323.dll
 0002:00000fd8       __imp_?show@QScrollView@@UAEXXZ 1001efd8     qt-mt323:qt-mt323.dll
 0002:00000fdc       __imp_?showColumn@QTable@@UAEXH@Z 1001efdc     qt-mt323:qt-mt323.dll
 0002:00000fe0       __imp_?showEvent@QTable@@MAEXPAVQShowEvent@@@Z 1001efe0     qt-mt323:qt-mt323.dll
 0002:00000fe4       __imp_?showRow@QTable@@UAEXH@Z 1001efe4     qt-mt323:qt-mt323.dll
 0002:00000fe8       __imp_?sizeHint@QComboBox@@UBE?AVQSize@@XZ 1001efe8     qt-mt323:qt-mt323.dll
 0002:00000fec       __imp_?sizeHint@QGridLayout@@UBE?AVQSize@@XZ 1001efec     qt-mt323:qt-mt323.dll
 0002:00000ff0       __imp_?sizeHint@QLabel@@UBE?AVQSize@@XZ 1001eff0     qt-mt323:qt-mt323.dll
 0002:00000ff4       __imp_?sizeHint@QLineEdit@@UBE?AVQSize@@XZ 1001eff4     qt-mt323:qt-mt323.dll
 0002:00000ff8       __imp_?sizeHint@QPushButton@@UBE?AVQSize@@XZ 1001eff8     qt-mt323:qt-mt323.dll
 0002:00000ffc       __imp_?sizeHint@QSpacerItem@@UBE?AVQSize@@XZ 1001effc     qt-mt323:qt-mt323.dll
 0002:00001000       __imp_?sizeHint@QSpinBox@@UBE?AVQSize@@XZ 1001f000     qt-mt323:qt-mt323.dll
 0002:00001004       __imp_?sizeHint@QTable@@UBE?AVQSize@@XZ 1001f004     qt-mt323:qt-mt323.dll
 0002:00001008       __imp_?sortColumn@QTable@@UAEXH_N0@Z 1001f008     qt-mt323:qt-mt323.dll
 0002:0000100c       __imp_?spacerItem@QSpacerItem@@UAEPAV1@XZ 1001f00c     qt-mt323:qt-mt323.dll
 0002:00001010       __imp_?startDrag@QTable@@MAEXXZ 1001f010     qt-mt323:qt-mt323.dll
 0002:00001014       __imp_?stepChange@QRangeControl@@MAEXXZ 1001f014     qt-mt323:qt-mt323.dll
 0002:00001018       __imp_?stepDown@QSpinBox@@UAEXXZ 1001f018     qt-mt323:qt-mt323.dll
 0002:0000101c       __imp_?stepUp@QSpinBox@@UAEXXZ 1001f01c     qt-mt323:qt-mt323.dll
 0002:00001020       __imp_?styleChange@QComboBox@@MAEXAAVQStyle@@@Z 1001f020     qt-mt323:qt-mt323.dll
 0002:00001024       __imp_?styleChange@QScrollView@@UAEXAAVQStyle@@@Z 1001f024     qt-mt323:qt-mt323.dll
 0002:00001028       __imp_?styleChange@QSpinBox@@MAEXAAVQStyle@@@Z 1001f028     qt-mt323:qt-mt323.dll
 0002:0000102c       __imp_?suffix@QSpinBox@@UBE?AVQString@@XZ 1001f02c     qt-mt323:qt-mt323.dll
 0002:00001030       __imp_?swapCells@QTable@@UAEXHHHH@Z 1001f030     qt-mt323:qt-mt323.dll
 0002:00001034       __imp_?swapColumns@QTable@@UAEXHH_N@Z 1001f034     qt-mt323:qt-mt323.dll
 0002:00001038       __imp_?swapRows@QTable@@UAEXHH_N@Z 1001f038     qt-mt323:qt-mt323.dll
 0002:0000103c       __imp_?takeItem@QTable@@UAEXPAVQTableItem@@@Z 1001f03c     qt-mt323:qt-mt323.dll
 0002:00001040       __imp_?text@QTable@@UBE?AVQString@@HH@Z 1001f040     qt-mt323:qt-mt323.dll
 0002:00001044       __imp_?undo@QLineEdit@@UAEXXZ 1001f044     qt-mt323:qt-mt323.dll
 0002:00001048       __imp_?updateDisplay@QSpinBox@@MAEXXZ 1001f048     qt-mt323:qt-mt323.dll
 0002:0000104c       __imp_?updateMask@QComboBox@@MAEXXZ 1001f04c     qt-mt323:qt-mt323.dll
 0002:00001050       __imp_?updateMask@QPushButton@@MAEXXZ 1001f050     qt-mt323:qt-mt323.dll
 0002:00001054       __imp_?valueChange@QSpinBox@@MAEXXZ 1001f054     qt-mt323:qt-mt323.dll
 0002:00001058       __imp_?viewportResizeEvent@QTable@@MAEXPAVQResizeEvent@@@Z 1001f058     qt-mt323:qt-mt323.dll
 0002:0000105c       __imp_?wheelEvent@QComboBox@@MAEXPAVQWheelEvent@@@Z 1001f05c     qt-mt323:qt-mt323.dll
 0002:00001060       __imp_?wheelEvent@QSpinBox@@MAEXPAVQWheelEvent@@@Z 1001f060     qt-mt323:qt-mt323.dll
 0002:00001064       __imp_?windowActivationChange@QLineEdit@@MAEX_N@Z 1001f064     qt-mt323:qt-mt323.dll
 0002:00001068       __imp_?windowActivationChange@QTable@@MAEX_N@Z 1001f068     qt-mt323:qt-mt323.dll
 0002:0000106c       __imp_??4?$QMap@VQString@@H@@QAEAAV0@ABV0@@Z 1001f06c     qt-mt323:qt-mt323.dll
 0002:00001070       __imp_?contains@?$QMap@VQString@@H@@QBE_NABVQString@@@Z 1001f070     qt-mt323:qt-mt323.dll
 0002:00001074       __imp_?insert@?$QMap@VQString@@H@@QAE?AV?$QMapIterator@VQString@@H@@ABVQString@@ABH_N@Z 1001f074     qt-mt323:qt-mt323.dll
 0002:00001078       __imp_?pos@QWidget@@QBE?AVQPoint@@XZ 1001f078     qt-mt323:qt-mt323.dll
 0002:0000107c       __imp_?update@QWidget@@QAEXXZ 1001f07c     qt-mt323:qt-mt323.dll
 0002:00001080       __imp_?isMaximized@QWidget@@QBE_NXZ 1001f080     qt-mt323:qt-mt323.dll
 0002:00001084       __imp_?insertItem@QComboBox@@QAEXABVQString@@H@Z 1001f084     qt-mt323:qt-mt323.dll
 0002:00001088       __imp_?listBox@QComboBox@@QBEPAVQListBox@@XZ 1001f088     qt-mt323:qt-mt323.dll
 0002:0000108c       __imp_?text@QLineEdit@@QBE?AVQString@@XZ 1001f08c     qt-mt323:qt-mt323.dll
 0002:00001090       __imp_??1QTableItem@@UAE@XZ 1001f090     qt-mt323:qt-mt323.dll
 0002:00001094       __imp_??0QCheckTableItem@@QAE@PAVQTable@@ABVQString@@@Z 1001f094     qt-mt323:qt-mt323.dll
 0002:00001098       __imp_?isChecked@QCheckTableItem@@QBE_NXZ 1001f098     qt-mt323:qt-mt323.dll
 0002:0000109c       __imp_?isSelected@QTable@@QBE_NHH@Z 1001f09c     qt-mt323:qt-mt323.dll
 0002:000010a0       __imp_?currentPageIndex@QTabWidget@@QBEHXZ 1001f0a0     qt-mt323:qt-mt323.dll
 0002:000010a4       __imp_?move@QDialog@@QAEXABVQPoint@@@Z 1001f0a4     qt-mt323:qt-mt323.dll
 0002:000010a8       __imp_?getText@QInputDialog@@SA?AVQString@@ABV2@0W4EchoMode@QLineEdit@@0PA_NPAVQWidget@@PBD@Z 1001f0a8     qt-mt323:qt-mt323.dll
 0002:000010ac       __imp_?sort@QListBox@@QAEX_N@Z 1001f0ac     qt-mt323:qt-mt323.dll
 0002:000010b0       __imp_?alignment@QTableItem@@UBEHXZ 1001f0b0     qt-mt323:qt-mt323.dll
 0002:000010b4       __imp_?createEditor@QCheckTableItem@@UBEPAVQWidget@@XZ 1001f0b4     qt-mt323:qt-mt323.dll
 0002:000010b8       __imp_?key@QTableItem@@UBE?AVQString@@XZ 1001f0b8     qt-mt323:qt-mt323.dll
 0002:000010bc       __imp_?paint@QCheckTableItem@@UAEXPAVQPainter@@ABVQColorGroup@@ABVQRect@@_N@Z 1001f0bc     qt-mt323:qt-mt323.dll
 0002:000010c0       __imp_?pixmap@QTableItem@@UBE?AVQPixmap@@XZ 1001f0c0     qt-mt323:qt-mt323.dll
 0002:000010c4       __imp_?rtti@QCheckTableItem@@UBEHXZ 1001f0c4     qt-mt323:qt-mt323.dll
 0002:000010c8       __imp_?setChecked@QCheckTableItem@@UAEX_N@Z 1001f0c8     qt-mt323:qt-mt323.dll
 0002:000010cc       __imp_?setCol@QTableItem@@UAEXH@Z 1001f0cc     qt-mt323:qt-mt323.dll
 0002:000010d0       __imp_?setContentFromEditor@QCheckTableItem@@UAEXPAVQWidget@@@Z 1001f0d0     qt-mt323:qt-mt323.dll
 0002:000010d4       __imp_?setEnabled@QTableItem@@UAEX_N@Z 1001f0d4     qt-mt323:qt-mt323.dll
 0002:000010d8       __imp_?setPixmap@QTableItem@@UAEXABVQPixmap@@@Z 1001f0d8     qt-mt323:qt-mt323.dll
 0002:000010dc       __imp_?setReplaceable@QTableItem@@UAEX_N@Z 1001f0dc     qt-mt323:qt-mt323.dll
 0002:000010e0       __imp_?setRow@QTableItem@@UAEXH@Z 1001f0e0     qt-mt323:qt-mt323.dll
 0002:000010e4       __imp_?setSpan@QTableItem@@UAEXHH@Z 1001f0e4     qt-mt323:qt-mt323.dll
 0002:000010e8       __imp_?setText@QCheckTableItem@@UAEXABVQString@@@Z 1001f0e8     qt-mt323:qt-mt323.dll
 0002:000010ec       __imp_?setWordWrap@QTableItem@@UAEX_N@Z 1001f0ec     qt-mt323:qt-mt323.dll
 0002:000010f0       __imp_?sizeHint@QCheckTableItem@@UBE?AVQSize@@XZ 1001f0f0     qt-mt323:qt-mt323.dll
 0002:000010f4       __imp_?text@QTableItem@@UBE?AVQString@@XZ 1001f0f4     qt-mt323:qt-mt323.dll
 0002:000010f8       __imp_?qstrcmp@@YAHPBD0@Z  1001f0f8     qt-mt323:qt-mt323.dll
 0002:000010fc       __imp_?fromLatin1@QString@@SA?AV1@PBDH@Z 1001f0fc     qt-mt323:qt-mt323.dll
 0002:00001100       __imp_?qt_cast@QDialog@@UAEPAXPBD@Z 1001f100     qt-mt323:qt-mt323.dll
 0002:00001104       __imp_?qt_invoke@QDialog@@UAE_NHPAUQUObject@@@Z 1001f104     qt-mt323:qt-mt323.dll
 0002:00001108       __imp_?qt_emit@QDialog@@UAE_NHPAUQUObject@@@Z 1001f108     qt-mt323:qt-mt323.dll
 0002:0000110c       __imp_?qt_property@QDialog@@UAE_NHHPAVQVariant@@@Z 1001f10c     qt-mt323:qt-mt323.dll
 0002:00001110       __imp_?staticMetaObject@QDialog@@SAPAVQMetaObject@@XZ 1001f110     qt-mt323:qt-mt323.dll
 0002:00001114       __imp_?new_metaobject@QMetaObject@@SAPAV1@PBDPAV1@QBUQMetaData@@H2HQBVQMetaProperty@@HQBUQMetaEnum@@HQBUQClassInfo@@H@Z 1001f114     qt-mt323:qt-mt323.dll
 0002:00001118       __imp_??0QMetaObjectCleanUp@@QAE@PBDP6APAVQMetaObject@@XZ@Z 1001f118     qt-mt323:qt-mt323.dll
 0002:0000111c       __imp_??1QMetaObjectCleanUp@@QAE@XZ 1001f11c     qt-mt323:qt-mt323.dll
 0002:00001120       __imp_?setMetaObject@QMetaObjectCleanUp@@QAEXAAPAVQMetaObject@@@Z 1001f120     qt-mt323:qt-mt323.dll
 0002:00001124       __imp_?translate@QApplication@@QBE?AVQString@@PBD00W4Encoding@1@@Z 1001f124     qt-mt323:qt-mt323.dll
 0002:00001128       __imp_?qApp@@3PAVQApplication@@A 1001f128     qt-mt323:qt-mt323.dll
 0002:0000112c       __imp_?static_QUType_ptr@@3UQUType_ptr@@A 1001f12c     qt-mt323:qt-mt323.dll
 0002:00001130       __imp_?static_QUType_int@@3UQUType_int@@A 1001f130     qt-mt323:qt-mt323.dll
 0002:00001134       __imp_?static_QUType_QString@@3UQUType_QString@@A 1001f134     qt-mt323:qt-mt323.dll
 0002:00001138       __imp_??6?$QValueList@VQString@@@@QAEAAV0@ABVQString@@@Z 1001f138     qt-mt323:qt-mt323.dll
 0002:0000113c       __imp_??0QColorGroup@@QAE@ABV0@@Z 1001f13c     qt-mt323:qt-mt323.dll
 0002:00001140       __imp_??1QColorGroup@@QAE@XZ 1001f140     qt-mt323:qt-mt323.dll
 0002:00001144       __imp_?setColor@QColorGroup@@QAEXW4ColorRole@1@ABVQColor@@@Z 1001f144     qt-mt323:qt-mt323.dll
 0002:00001148       __imp_??1QButton@@UAE@XZ   1001f148     qt-mt323:qt-mt323.dll
 0002:0000114c       __imp_??0QGroupBox@@QAE@PAVQWidget@@PBD@Z 1001f14c     qt-mt323:qt-mt323.dll
 0002:00001150       __imp_??1QGroupBox@@UAE@XZ 1001f150     qt-mt323:qt-mt323.dll
 0002:00001154       __imp_??0QButtonGroup@@QAE@PAVQWidget@@PBD@Z 1001f154     qt-mt323:qt-mt323.dll
 0002:00001158       __imp_??1QButtonGroup@@UAE@XZ 1001f158     qt-mt323:qt-mt323.dll
 0002:0000115c       __imp_??0QRadioButton@@QAE@PAVQWidget@@PBD@Z 1001f15c     qt-mt323:qt-mt323.dll
 0002:00001160       __imp_?setDuplicatesEnabled@QComboBox@@QAEX_N@Z 1001f160     qt-mt323:qt-mt323.dll
 0002:00001164       __imp_?setResizeMode@QLayout@@QAEXW4ResizeMode@1@@Z 1001f164     qt-mt323:qt-mt323.dll
 0002:00001168       __imp_??0QGridLayout@@QAE@PAVQLayout@@HHHPBD@Z 1001f168     qt-mt323:qt-mt323.dll
 0002:0000116c       __imp_?childEvent@QGroupBox@@MAEXPAVQChildEvent@@@Z 1001f16c     qt-mt323:qt-mt323.dll
 0002:00001170       __imp_?className@QButtonGroup@@UBEPBDXZ 1001f170     qt-mt323:qt-mt323.dll
 0002:00001174       __imp_?className@QGroupBox@@UBEPBDXZ 1001f174     qt-mt323:qt-mt323.dll
 0002:00001178       __imp_?className@QRadioButton@@UBEPBDXZ 1001f178     qt-mt323:qt-mt323.dll
 0002:0000117c       __imp_?drawButton@QRadioButton@@MAEXPAVQPainter@@@Z 1001f17c     qt-mt323:qt-mt323.dll
 0002:00001180       __imp_?drawButtonLabel@QRadioButton@@MAEXPAVQPainter@@@Z 1001f180     qt-mt323:qt-mt323.dll
 0002:00001184       __imp_?event@QButtonGroup@@MAE_NPAVQEvent@@@Z 1001f184     qt-mt323:qt-mt323.dll
 0002:00001188       __imp_?event@QGroupBox@@MAE_NPAVQEvent@@@Z 1001f188     qt-mt323:qt-mt323.dll
 0002:0000118c       __imp_?focusInEvent@QButton@@MAEXPAVQFocusEvent@@@Z 1001f18c     qt-mt323:qt-mt323.dll
 0002:00001190       __imp_?focusInEvent@QGroupBox@@MAEXPAVQFocusEvent@@@Z 1001f190     qt-mt323:qt-mt323.dll
 0002:00001194       __imp_?focusOutEvent@QButton@@MAEXPAVQFocusEvent@@@Z 1001f194     qt-mt323:qt-mt323.dll
 0002:00001198       __imp_?fontChange@QGroupBox@@MAEXABVQFont@@@Z 1001f198     qt-mt323:qt-mt323.dll
 0002:0000119c       __imp_?hitButton@QRadioButton@@MBE_NABVQPoint@@@Z 1001f19c     qt-mt323:qt-mt323.dll
 0002:000011a0       __imp_?metaObject@QButtonGroup@@UBEPAVQMetaObject@@XZ 1001f1a0     qt-mt323:qt-mt323.dll
 0002:000011a4       __imp_?metaObject@QGroupBox@@UBEPAVQMetaObject@@XZ 1001f1a4     qt-mt323:qt-mt323.dll
 0002:000011a8       __imp_?metaObject@QRadioButton@@UBEPAVQMetaObject@@XZ 1001f1a8     qt-mt323:qt-mt323.dll
 0002:000011ac       __imp_?moveFocus@QButtonGroup@@UAEXH@Z 1001f1ac     qt-mt323:qt-mt323.dll
 0002:000011b0       __imp_?paintEvent@QGroupBox@@MAEXPAVQPaintEvent@@@Z 1001f1b0     qt-mt323:qt-mt323.dll
 0002:000011b4       __imp_?qt_cast@QButtonGroup@@UAEPAXPBD@Z 1001f1b4     qt-mt323:qt-mt323.dll
 0002:000011b8       __imp_?qt_cast@QGroupBox@@UAEPAXPBD@Z 1001f1b8     qt-mt323:qt-mt323.dll
 0002:000011bc       __imp_?qt_cast@QRadioButton@@UAEPAXPBD@Z 1001f1bc     qt-mt323:qt-mt323.dll
 0002:000011c0       __imp_?qt_emit@QButtonGroup@@UAE_NHPAUQUObject@@@Z 1001f1c0     qt-mt323:qt-mt323.dll
 0002:000011c4       __imp_?qt_emit@QGroupBox@@UAE_NHPAUQUObject@@@Z 1001f1c4     qt-mt323:qt-mt323.dll
 0002:000011c8       __imp_?qt_emit@QRadioButton@@UAE_NHPAUQUObject@@@Z 1001f1c8     qt-mt323:qt-mt323.dll
 0002:000011cc       __imp_?qt_invoke@QButtonGroup@@UAE_NHPAUQUObject@@@Z 1001f1cc     qt-mt323:qt-mt323.dll
 0002:000011d0       __imp_?qt_invoke@QGroupBox@@UAE_NHPAUQUObject@@@Z 1001f1d0     qt-mt323:qt-mt323.dll
 0002:000011d4       __imp_?qt_invoke@QRadioButton@@UAE_NHPAUQUObject@@@Z 1001f1d4     qt-mt323:qt-mt323.dll
 0002:000011d8       __imp_?qt_property@QButtonGroup@@UAE_NHHPAVQVariant@@@Z 1001f1d8     qt-mt323:qt-mt323.dll
 0002:000011dc       __imp_?qt_property@QGroupBox@@UAE_NHHPAVQVariant@@@Z 1001f1dc     qt-mt323:qt-mt323.dll
 0002:000011e0       __imp_?qt_property@QRadioButton@@UAE_NHHPAVQVariant@@@Z 1001f1e0     qt-mt323:qt-mt323.dll
 0002:000011e4       __imp_?resizeEvent@QGroupBox@@MAEXPAVQResizeEvent@@@Z 1001f1e4     qt-mt323:qt-mt323.dll
 0002:000011e8       __imp_?resizeEvent@QRadioButton@@MAEXPAVQResizeEvent@@@Z 1001f1e8     qt-mt323:qt-mt323.dll
 0002:000011ec       __imp_?setAlignment@QGroupBox@@UAEXH@Z 1001f1ec     qt-mt323:qt-mt323.dll
 0002:000011f0       __imp_?setButton@QButtonGroup@@UAEXH@Z 1001f1f0     qt-mt323:qt-mt323.dll
 0002:000011f4       __imp_?setChecked@QRadioButton@@UAEX_N@Z 1001f1f4     qt-mt323:qt-mt323.dll
 0002:000011f8       __imp_?setColumnLayout@QGroupBox@@UAEXHW4Orientation@Qt@@@Z 1001f1f8     qt-mt323:qt-mt323.dll
 0002:000011fc       __imp_?setEnabled@QGroupBox@@UAEX_N@Z 1001f1fc     qt-mt323:qt-mt323.dll
 0002:00001200       __imp_?setExclusive@QButtonGroup@@UAEX_N@Z 1001f200     qt-mt323:qt-mt323.dll
 0002:00001204       __imp_?setRadioButtonExclusive@QButtonGroup@@UAEX_N@Z 1001f204     qt-mt323:qt-mt323.dll
 0002:00001208       __imp_?setTitle@QGroupBox@@UAEXABVQString@@@Z 1001f208     qt-mt323:qt-mt323.dll
 0002:0000120c       __imp_?sizeHint@QGroupBox@@UBE?AVQSize@@XZ 1001f20c     qt-mt323:qt-mt323.dll
 0002:00001210       __imp_?sizeHint@QRadioButton@@UBE?AVQSize@@XZ 1001f210     qt-mt323:qt-mt323.dll
 0002:00001214       __imp_?updateMask@QRadioButton@@MAEXXZ 1001f214     qt-mt323:qt-mt323.dll
 0002:00001218       __imp_?setMinimumSize@QWidget@@QAEXABVQSize@@@Z 1001f218     qt-mt323:qt-mt323.dll
 0002:0000121c       __imp_?resize@QWidget@@QAEXABVQSize@@@Z 1001f21c     qt-mt323:qt-mt323.dll
 0002:00001220       __imp_?addMultiCell@QGridLayout@@QAEXPAVQLayoutItem@@HHHHH@Z 1001f220     qt-mt323:qt-mt323.dll
 0002:00001224       __imp_?add@QToolTip@@SAXPAVQWidget@@ABVQString@@@Z 1001f224     qt-mt323:qt-mt323.dll
 0002:00001228       __imp_?add@QWhatsThis@@SAXPAVQWidget@@ABVQString@@@Z 1001f228     qt-mt323:qt-mt323.dll
 0002:0000122c       __imp_?receivers@QObject@@IBEPAVQConnectionList@@H@Z 1001f22c     qt-mt323:qt-mt323.dll
 0002:00001230       __imp_?activate_signal@QObject@@IAEXPAVQConnectionList@@PAUQUObject@@@Z 1001f230     qt-mt323:qt-mt323.dll
 0002:00001234       __imp_?staticMetaObject@QWidget@@SAPAVQMetaObject@@XZ 1001f234     qt-mt323:qt-mt323.dll
 0002:00001238       __imp_??0QUObject@@QAE@XZ  1001f238     qt-mt323:qt-mt323.dll
 0002:0000123c       __imp_??1QUObject@@QAE@XZ  1001f23c     qt-mt323:qt-mt323.dll
 0002:00001240       __imp_?set@QUType_bool@@QAEXPAUQUObject@@_N@Z 1001f240     qt-mt323:qt-mt323.dll
 0002:00001244       __imp_?set@QUType_QString@@QAEXPAUQUObject@@ABVQString@@@Z 1001f244     qt-mt323:qt-mt323.dll
 0002:00001248       __imp_?static_QUType_bool@@3UQUType_bool@@A 1001f248     qt-mt323:qt-mt323.dll
 0002:0000124c       __imp_?static_QUType_varptr@@3UQUType_varptr@@A 1001f24c     qt-mt323:qt-mt323.dll
 0002:00001250       __imp_?activate_signal@QObject@@IAEXH@Z 1001f250     qt-mt323:qt-mt323.dll
 0002:00001254       __imp_??0QTextStream@@QAE@PAVQIODevice@@@Z 1001f254     qt-mt323:qt-mt323.dll
 0002:00001258       __imp_?setCodec@QTextStream@@QAEXPAVQTextCodec@@@Z 1001f258     qt-mt323:qt-mt323.dll
 0002:0000125c       __imp_?reset@QIODevice@@QAE_NXZ 1001f25c     qt-mt323:qt-mt323.dll
 0002:00001260       __imp_??H@YA?BVQString@@ABV0@D@Z 1001f260     qt-mt323:qt-mt323.dll
 0002:00001264       __imp_??H@YA?BVQString@@PBDABV0@@Z 1001f264     qt-mt323:qt-mt323.dll
 0002:00001268       __imp_??H@YA?BVQString@@ABV0@PBD@Z 1001f268     qt-mt323:qt-mt323.dll
 0002:0000126c       __imp_??H@YA?BVQString@@ABV0@0@Z 1001f26c     qt-mt323:qt-mt323.dll
 0002:00001270       __imp_??8@YA_NABVQString@@PBD@Z 1001f270     qt-mt323:qt-mt323.dll
 0002:00001274       __imp_??8@YA_NABVQString@@0@Z 1001f274     qt-mt323:qt-mt323.dll
 0002:00001278       __imp_??M@YA_NABVQString@@0@Z 1001f278     qt-mt323:qt-mt323.dll
 0002:0000127c       __imp_??9@YA_NABVQString@@0@Z 1001f27c     qt-mt323:qt-mt323.dll
 0002:00001280       __imp_?setLength@QString@@QAEXI@Z 1001f280     qt-mt323:qt-mt323.dll
 0002:00001284       __imp_?endsWith@QString@@QBE_NABV1@@Z 1001f284     qt-mt323:qt-mt323.dll
 0002:00001288       __imp_?startsWith@QString@@QBE_NABV1@_N@Z 1001f288     qt-mt323:qt-mt323.dll
 0002:0000128c       __imp_?startsWith@QString@@QBE_NABV1@@Z 1001f28c     qt-mt323:qt-mt323.dll
 0002:00001290       __imp_?latin1@QString@@QBEPBDXZ 1001f290     qt-mt323:qt-mt323.dll
 0002:00001294       __imp_?fromAscii@QString@@SA?AV1@PBDH@Z 1001f294     qt-mt323:qt-mt323.dll
 0002:00001298       __imp_?ascii@QString@@QBEPBDXZ 1001f298     qt-mt323:qt-mt323.dll
 0002:0000129c       __imp_??YQString@@QAEAAV0@D@Z 1001f29c     qt-mt323:qt-mt323.dll
 0002:000012a0       __imp_??YQString@@QAEAAV0@PBD@Z 1001f2a0     qt-mt323:qt-mt323.dll
 0002:000012a4       __imp_??YQString@@QAEAAV0@ABV0@@Z 1001f2a4     qt-mt323:qt-mt323.dll
 0002:000012a8       __imp_?number@QString@@SA?AV1@HH@Z 1001f2a8     qt-mt323:qt-mt323.dll
 0002:000012ac       __imp_?toInt@QString@@QBEHPA_NH@Z 1001f2ac     qt-mt323:qt-mt323.dll
 0002:000012b0       __imp_?replace@QString@@QAEAAV1@ABV1@0@Z 1001f2b0     qt-mt323:qt-mt323.dll
 0002:000012b4       __imp_?remove@QString@@QAEAAV1@ABV1@_N@Z 1001f2b4     qt-mt323:qt-mt323.dll
 0002:000012b8       __imp_?remove@QString@@QAEAAV1@ABV1@@Z 1001f2b8     qt-mt323:qt-mt323.dll
 0002:000012bc       __imp_?remove@QString@@QAEAAV1@II@Z 1001f2bc     qt-mt323:qt-mt323.dll
 0002:000012c0       __imp_?insert@QString@@QAEAAV1@IABV1@@Z 1001f2c0     qt-mt323:qt-mt323.dll
 0002:000012c4       __imp_?stripWhiteSpace@QString@@QBE?AV1@XZ 1001f2c4     qt-mt323:qt-mt323.dll
 0002:000012c8       __imp_?rightJustify@QString@@QBE?AV1@IVQChar@@_N@Z 1001f2c8     qt-mt323:qt-mt323.dll
 0002:000012cc       __imp_?right@QString@@QBE?AV1@I@Z 1001f2cc     qt-mt323:qt-mt323.dll
 0002:000012d0       __imp_?section@QString@@QBE?AV1@PBDHHH@Z 1001f2d0     qt-mt323:qt-mt323.dll
 0002:000012d4       __imp_?contains@QString@@QBEHABVQRegExp@@@Z 1001f2d4     qt-mt323:qt-mt323.dll
 0002:000012d8       __imp_?contains@QString@@QBEHABV1@_N@Z 1001f2d8     qt-mt323:qt-mt323.dll
 0002:000012dc       __imp_?contains@QString@@QBEHPBD_N@Z 1001f2dc     qt-mt323:qt-mt323.dll
 0002:000012e0       __imp_?find@QString@@QBEHABV1@H_N@Z 1001f2e0     qt-mt323:qt-mt323.dll
 0002:000012e4       __imp_?sprintf@QString@@QAAAAV1@PBDZZ 1001f2e4     qt-mt323:qt-mt323.dll
 0002:000012e8       __imp_?arg@QString@@QBE?AV1@ABV1@H@Z 1001f2e8     qt-mt323:qt-mt323.dll
 0002:000012ec       __imp_?arg@QString@@QBE?AV1@HHH@Z 1001f2ec     qt-mt323:qt-mt323.dll
 0002:000012f0       __imp_??4QString@@QAEAAV0@PBD@Z 1001f2f0     qt-mt323:qt-mt323.dll
 0002:000012f4       __imp_??4QString@@QAEAAV0@ABV0@@Z 1001f2f4     qt-mt323:qt-mt323.dll
 0002:000012f8       __imp_??1QString@@QAE@XZ   1001f2f8     qt-mt323:qt-mt323.dll
 0002:000012fc       __imp_??0QString@@QAE@PBD@Z 1001f2fc     qt-mt323:qt-mt323.dll
 0002:00001300       __imp_??0QString@@QAE@ABV0@@Z 1001f300     qt-mt323:qt-mt323.dll
 0002:00001304       __imp_??0QString@@QAE@XZ   1001f304     qt-mt323:qt-mt323.dll
 0002:00001308       __imp_?deleteSelf@QStringData@@QAEXXZ 1001f308     qt-mt323:qt-mt323.dll
 0002:0000130c       __imp_??1QCString@@UAE@XZ  1001f30c     qt-mt323:qt-mt323.dll
 0002:00001310       __imp_?next@QGList@@IAEPAXXZ 1001f310     qt-mt323:qt-mt323.dll
 0002:00001314       __imp_?split@QStringList@@SA?AV1@ABVQChar@@ABVQString@@_N@Z 1001f314     qt-mt323:qt-mt323.dll
 0002:00001318       __imp_??0QSettings@@QAE@W4Format@0@@Z 1001f318     qt-mt323:qt-mt323.dll
 0002:0000131c       __imp_??1QSettings@@QAE@XZ 1001f31c     qt-mt323:qt-mt323.dll
 0002:00001320       __imp_?writeEntry@QSettings@@QAE_NABVQString@@0@Z 1001f320     qt-mt323:qt-mt323.dll
 0002:00001324       __imp_?readEntry@QSettings@@QAE?AVQString@@ABV2@0PA_N@Z 1001f324     qt-mt323:qt-mt323.dll
 0002:00001328       __imp_?columnWidth@QListView@@QBEHH@Z 1001f328     qt-mt323:qt-mt323.dll
 0002:0000132c       __imp_?columns@QListView@@QBEHXZ 1001f32c     qt-mt323:qt-mt323.dll
 0002:00001330       __imp_?lower@QString@@QBE?AV1@XZ 1001f330     qt-mt323:qt-mt323.dll
 0002:00001334       __imp_?makeSharedNull@QString@@CAPAUQStringData@@XZ 1001f334     qt-mt323:qt-mt323.dll
 0002:00001338       __imp_?first@QGList@@IAEPAXXZ 1001f338     qt-mt323:qt-mt323.dll
 0002:0000133c       __imp_?clear@QGList@@MAEXXZ 1001f33c     qt-mt323:qt-mt323.dll
 0002:00001340       __imp_?remove@QGList@@IAE_NPAX@Z 1001f340     qt-mt323:qt-mt323.dll
 0002:00001344       __imp_?append@QGList@@IAEXPAX@Z 1001f344     qt-mt323:qt-mt323.dll
 0002:00001348       __imp_??1QGList@@MAE@XZ    1001f348     qt-mt323:qt-mt323.dll
 0002:0000134c       __imp_??0QGList@@IAE@XZ    1001f34c     qt-mt323:qt-mt323.dll
 0002:00001350       __imp_?qDebug@@YAXPBDZZ    1001f350     qt-mt323:qt-mt323.dll
 0002:00001354       __imp_?clear@?$QMap@VQString@@H@@QAEXXZ 1001f354     qt-mt323:qt-mt323.dll
 0002:00001358       \177qt-mt323_NULL_THUNK_DATA 1001f358     qt-mt323:qt-mt323.dll
 0002:0000135c       ___xc_a                    1001f35c     MSVCRT:cinitexe.obj
 0002:00001384       ___xc_z                    1001f384     MSVCRT:cinitexe.obj
 0002:00001388       ___xi_a                    1001f388     MSVCRT:cinitexe.obj
 0002:00001394       ___xi_z                    1001f394     MSVCRT:cinitexe.obj
 0002:0000139c       ??_SQWidget@@6BQObject@@@  1001f39c     alm_bncs_output.obj
 0002:00001550       ??_SQWidget@@6BQPaintDevice@@@ 1001f550     alm_bncs_output.obj
 0002:00001570       ??_C@_02GIPFHKNO@OK?$AA@   1001f570     alm_bncs_output.obj
 0002:0000157c       ??_SQAction@@6B@           1001f57c     alm_bncs_output.obj
 0002:0000160c       ??_SQDockWindow@@6BQObject@@@ 1001f60c     alm_bncs_output.obj
 0002:0000181c       ??_SQDockWindow@@6BQPaintDevice@@@ 1001f81c     alm_bncs_output.obj
 0002:00001844       ??_SQToolBar@@6BQObject@@@ 1001f844     alm_bncs_output.obj
 0002:00001a60       ??_SQToolBar@@6BQPaintDevice@@@ 1001fa60     alm_bncs_output.obj
 0002:00001a84       ??_SQListViewItem@@6B@     1001fa84     alm_bncs_output.obj
 0002:00001b24       ??_SQListView@@6BQObject@@@ 1001fb24     alm_bncs_output.obj
 0002:00001e08       ??_SQListView@@6BQPaintDevice@@@ 1001fe08     alm_bncs_output.obj
 0002:00001e2c       ??_SQTabWidget@@6BQObject@@@ 1001fe2c     alm_bncs_output.obj
 0002:00002000       ??_SQTabWidget@@6BQPaintDevice@@@ 10020000     alm_bncs_output.obj
 0002:00002024       ??_SQBoxLayout@@6BQObject@@@ 10020024     alm_bncs_output.obj
 0002:0000208c       ??_SQBoxLayout@@6BQLayoutItem@@@ 1002008c     alm_bncs_output.obj
 0002:000020d4       ??_SCAlm_sys_select@@6BQObject@@@ 100200d4     alm_bncs_output.obj
 0002:000022a8       ??_SCAlm_sys_select@@6BQPaintDevice@@@ 100202a8     alm_bncs_output.obj
 0002:000022cc       ??_SQGuardedPtrPrivate@@6B@ 100202cc     alm_bncs_output.obj
 0002:00002320       ??_7QDockWindowList@@6B@   10020320     alm_bncs_output.obj
 0002:00002344       ??_SQPopupMenu@@6BQObject@@@ 10020344     alm_bncs_output.obj
 0002:00002524       ??_SQPopupMenu@@6BQPaintDevice@@@ 10020524     alm_bncs_output.obj
 0002:00002548       ??_SQPopupMenu@@6B@        10020548     alm_bncs_output.obj
 0002:0000256c       ??_7?$QPtrList@VQPopupMenu@@@@6B@ 1002056c     alm_bncs_output.obj
 0002:00002590       ??_7QPopupMenuList@@6B@    10020590     alm_bncs_output.obj
 0002:000025b4       ??_7config_plugin_base@@6BQObject@@@ 100205b4     alm_bncs_output.obj
 0002:0000278c       ??_7config_plugin_base@@6BQPaintDevice@@@ 1002078c     alm_bncs_output.obj
 0002:000027b0       ??_C@_0EB@GNDACMDJ@?$CC?5?9?5the?5author?5should?5have?5defin@ 100207b0     alm_bncs_output.obj
 0002:000027f4       ??_C@_0CH@BDPDPLDP@This?5is?5the?5default?5?$CCAbout?$CC?5text@ 100207f4     alm_bncs_output.obj
 0002:00002820       ??_7IDomDoc@@6B@           10020820     alm_bncs_output.obj
 0002:00002830       ??_7devTemplate@@6B@       10020830     alm_bncs_output.obj
 0002:00002838       ??_7IGetDocuments@@6B@     10020838     alm_bncs_output.obj
 0002:00002854       ??_7ISendCommand@@6B@      10020854     alm_bncs_output.obj
 0002:0000285c       ??_7FileLoad_BncsSystem@alm_bncs_output@@6B@ 1002085c     alm_bncs_output.obj
 0002:0000286c       ??_7?$QPtrList@VcOutputFile@@@@6B@ 1002086c     alm_bncs_output.obj
 0002:00002890       ??_7alm_bncs_output@@6BQObject@@@ 10020890     alm_bncs_output.obj
 0002:00002a68       ??_7alm_bncs_output@@6BQPaintDevice@@@ 10020a68     alm_bncs_output.obj
 0002:00002a8c       ??_7alm_bncs_output@@6BIDomDoc@@@ 10020a8c     alm_bncs_output.obj
 0002:00002a9c       ??_7alm_bncs_output@@6BIGetDocuments@@@ 10020a9c     alm_bncs_output.obj
 0002:00002ab8       ??_7alm_bncs_output@@6BISendCommand@@@ 10020ab8     alm_bncs_output.obj
 0002:00002abc       ??_C@_0N@BCBHFELI@windows?91252?$AA@ 10020abc     alm_bncs_output.obj
 0002:00002acc       ??_C@_08DFEIFMHK@?1browser?$AA@ 10020acc     alm_bncs_output.obj
 0002:00002ad8       ??_C@_0BG@LMBECLGB@Alarm?5Outputs?5modules?$AA@ 10020ad8     alm_bncs_output.obj
 0002:00002af0       ??_C@_04FABLJDN@Name?$AA@  10020af0     alm_bncs_output.obj
 0002:00002af8       ??_C@_0M@KOGPIGII@Config?5File?$AA@ 10020af8     alm_bncs_output.obj
 0002:00002b04       ??_C@_08KJDMPFAO@FileList?$AA@ 10020b04     alm_bncs_output.obj
 0002:00002b10       ??_C@_0CB@MDFLINCH@Home?1Alarms?1Outputs?1Bncs?5Output?1@ 10020b10     alm_bncs_output.obj
 0002:00002b34       ??_C@_0N@OLPKPMKN@?$CGBNCS?5Output?$AA@ 10020b34     alm_bncs_output.obj
 0002:00002b44       ??_C@_0N@GMGPPGEF@?1BNCS?5Output?$AA@ 10020b44     alm_bncs_output.obj
 0002:00002b54       ??_C@_03CLCAEGCJ@new?$AA@  10020b54     alm_bncs_output.obj
 0002:00002b58       ??_C@_0BB@PEPEPDAB@?$CGNew?5BNCS?5Output?$AA@ 10020b58     alm_bncs_output.obj
 0002:00002b6c       ??_C@_07EJAINBEK@filenew?$AA@ 10020b6c     alm_bncs_output.obj
 0002:00002b74       ??_C@_0BH@FCFHLCMF@New?5BNCS?5Output?5Module?$AA@ 10020b74     alm_bncs_output.obj
 0002:00002b8c       ??_C@_0P@CBINDBNH@1menuNewFile?$CI?$CJ?$AA@ 10020b8c     alm_bncs_output.obj
 0002:00002b9c       ??_C@_0N@KCMOKDBB@2activated?$CI?$CJ?$AA@ 10020b9c     alm_bncs_output.obj
 0002:00002bac       ??_C@_06FOBLBEIN@delete?$AA@ 10020bac     alm_bncs_output.obj
 0002:00002bb4       ??_C@_0BL@IHABNMMP@?$CGDelete?5BNCS?5Output?5Module?$AA@ 10020bb4     alm_bncs_output.obj
 0002:00002bd0       ??_C@_0L@BPDPNFLB@filedelete?$AA@ 10020bd0     alm_bncs_output.obj
 0002:00002bdc       ??_C@_0BK@DCCHDLCD@Delete?5BNCS?5Output?5Module?$AA@ 10020bdc     alm_bncs_output.obj
 0002:00002bf8       ??_C@_0BC@FIBCFKLP@1menuDeleteFile?$CI?$CJ?$AA@ 10020bf8     alm_bncs_output.obj
 0002:00002c0c       ??_C@_09KHIKJOBP@duplicate?$AA@ 10020c0c     alm_bncs_output.obj
 0002:00002c18       ??_C@_0BO@DNEKFBDO@?$CGDuplicate?5BNCS?5Output?5Module?$AA@ 10020c18     alm_bncs_output.obj
 0002:00002c38       ??_C@_0BN@FOIAJIJJ@Duplicate?5BNCS?5Output?5Module?$AA@ 10020c38     alm_bncs_output.obj
 0002:00002c58       ??_C@_0BF@LDLOGHID@1menuDuplicateFile?$CI?$CJ?$AA@ 10020c58     alm_bncs_output.obj
 0002:00002c70       ??_C@_06LMEAOBLB@rename?$AA@ 10020c70     alm_bncs_output.obj
 0002:00002c78       ??_C@_0BL@MMHGDPBL@?$CGRename?5BNCS?5Output?5Module?$AA@ 10020c78     alm_bncs_output.obj
 0002:00002c94       ??_C@_0BK@HJFANIPH@Rename?5BNCS?5Output?5Module?$AA@ 10020c94     alm_bncs_output.obj
 0002:00002cb0       ??_C@_0O@DALNGBDG@1menuRename?$CI?$CJ?$AA@ 10020cb0     alm_bncs_output.obj
 0002:00002cc0       ??_C@_0DL@BGNECHKO@1fileListContextMenu?$CIQListViewIt@ 10020cc0     alm_bncs_output.obj
 0002:00002cfc       ??_C@_0DL@JIJPNNOD@2contextMenuRequested?$CIQListViewI@ 10020cfc     alm_bncs_output.obj
 0002:00002d38       ??_C@_0BN@PALMGDOM@1selectFile?$CIQListViewItem?5?$CK?$CJ?$AA@ 10020d38     alm_bncs_output.obj
 0002:00002d58       ??_C@_0CC@LCOLGNI@2selectionChanged?$CIQListViewItem?$CK@ 10020d58     alm_bncs_output.obj
 0002:00002d7c       ??_C@_0DE@NNBCFON@1renameModule?$CIQListViewItem?$CK?0?5in@ 10020d7c     alm_bncs_output.obj
 0002:00002db0       ??_C@_0DD@FNLKOMHF@2itemRenamed?$CIQListViewItem?$CK?0?5int@ 10020db0     alm_bncs_output.obj
 0002:00002de4       ??_C@_0BP@KFJPMMLE@1selectSystem?$CIconst?5QString?5?$CG?$CJ?$AA@ 10020de4     alm_bncs_output.obj
 0002:00002e04       ??_C@_0BN@DDAIKEMB@2sysChanged?$CIconst?5QString?5?$CG?$CJ?$AA@ 10020e04     alm_bncs_output.obj
 0002:00002e24       ??_C@_0N@LMCHKLFE@1markDirty?$CI?$CJ?$AA@ 10020e24     alm_bncs_output.obj
 0002:00002e34       ??_C@_0BA@LHBDKNBL@2itemsChanged?$CI?$CJ?$AA@ 10020e34     alm_bncs_output.obj
 0002:00002e44       ??_C@_0P@JECNNCNO@1EditProcess?$CI?$CJ?$AA@ 10020e44     alm_bncs_output.obj
 0002:00002e54       ??_C@_0L@OELOHDKG@2clicked?$CI?$CJ?$AA@ 10020e54     alm_bncs_output.obj
 0002:00002e60       ??_C@_0BC@IMBGNLLE@1manageTemplate?$CI?$CJ?$AA@ 10020e60     alm_bncs_output.obj
 0002:00002e74       ??_C@_0CF@OJDACOJP@closeEvent?4?5command?$DNunlock?5file?$DN@ 10020e74     alm_bncs_output.obj
 0002:00002e9c       ??_C@_06BNCCALCL@unlock?$AA@ 10020e9c     alm_bncs_output.obj
 0002:00002ea4       ??_C@_0BH@FJKOLNHB@config?1devicetypes?4xml?$AA@ 10020ea4     alm_bncs_output.obj
 0002:00002ebc       ??_C@_0BF@NLODMMOO@config?1instances?4xml?$AA@ 10020ebc     alm_bncs_output.obj
 0002:00002ed4       ??_C@_08HNIAHLMM@download?$AA@ 10020ed4     alm_bncs_output.obj
 0002:00002ee0       ??_C@_04MKMCLCOO@lock?$AA@ 10020ee0     alm_bncs_output.obj
 0002:00002ee8       ??_C@_06KAOCKAGB@upload?$AA@ 10020ee8     alm_bncs_output.obj
 0002:00002ef0       ??_C@_03DAPAKLGM@dir?$AA@  10020ef0     alm_bncs_output.obj
 0002:00002ef4       ??_C@_0CF@OBKGBDGC@reply?4?5operation?$DNdir?4?5ok?0?5error?$DN@ 10020ef4     alm_bncs_output.obj
 0002:00002f1c       ??_C@_0CH@NOONMDDD@reply?4?5operation?$DNdir?4?5else?0?5erro@ 10020f1c     alm_bncs_output.obj
 0002:00002f44       ??_C@_0CD@BDMEEGML@navigate?5to?5?8?$CFs?8?5with?5context?5?8?$CF@ 10020f44     alm_bncs_output.obj
 0002:00002f68       ??_C@_01ICJEACDI@?$DL?$AA@ 10020f68     alm_bncs_output.obj
 0002:00002f6c       ??_C@_08JBEPPOLH@?1outputs?$AA@ 10020f6c     alm_bncs_output.obj
 0002:00002f78       ??_C@_01KMDKNFGN@?1?$AA@   10020f78     alm_bncs_output.obj
 0002:00002f7c       ??_C@_0O@MIFBLPDN@config?1alarms?$AA@ 10020f7c     alm_bncs_output.obj
 0002:00002f8c       ??_C@_02PEIOPPKO@?2S?$AA@  10020f8c     alm_bncs_output.obj
 0002:00002f90       ??_C@_0BC@PDAHGCDI@Process?5not?5found?$AA@ 10020f90     alm_bncs_output.obj
 0002:00002fa4       ??_C@_03NLJIHOMM@?5?9?5?$AA@ 10020fa4     alm_bncs_output.obj
 0002:00002fa8       ??_C@_09OLBIFBJN@Process?3?5?$AA@ 10020fa8     alm_bncs_output.obj
 0002:00002fb4       ??_C@_07MNGBFJEN@Process?$AA@ 10020fb4     alm_bncs_output.obj
 0002:00002fbc       ??_C@_0P@DBCHBMCI@File?5not?5found?$AA@ 10020fbc     alm_bncs_output.obj
 0002:00002fcc       ??_C@_06IGPBOHMJ@File?3?5?$AA@ 10020fcc     alm_bncs_output.obj
 0002:00002fd4       ??_C@_04PBAHLACE@File?$AA@ 10020fd4     alm_bncs_output.obj
 0002:00002fdc       ??_C@_0CA@OFNGENAG@activate?4?5command?$DNdir?5file?$DN?8?$CFs?8?$AA@ 10020fdc     alm_bncs_output.obj
 0002:00002ffc       ??_C@_0CJ@JBMAFIGN@activate?4?5command?$DNcheckoutFile?5f@ 10020ffc     alm_bncs_output.obj
 0002:00003028       ??_C@_0N@EHHLDFOB@checkoutFile?$AA@ 10021028     alm_bncs_output.obj
 0002:00003038       ??_C@_0BD@CODAMBFP@config?1devicetypes?$AA@ 10021038     alm_bncs_output.obj
 0002:0000304c       ??_C@_0CM@PCJGDMCM@activate?4?5command?$DNsyncDirDownloa@ 1002104c     alm_bncs_output.obj
 0002:00003078       ??_C@_0BA@GNHMHBBC@syncDirDownload?$AA@ 10021078     alm_bncs_output.obj
 0002:00003088       ??_C@_0CH@DAMAJOPA@apply?4?5command?$DNsyncDirUpload?5fil@ 10021088     alm_bncs_output.obj
 0002:000030b0       ??_C@_0O@JFGJGFB@syncDirUpload?$AA@ 100210b0     alm_bncs_output.obj
 0002:000030c0       ??_C@_0CE@KLBKCIPA@apply?4?5command?$DNuploadFile?5file?$DN?8@ 100210c0     alm_bncs_output.obj
 0002:000030e4       ??_C@_0L@CIKGEHEG@uploadFile?$AA@ 100210e4     alm_bncs_output.obj
 0002:000030f0       ??_C@_0BC@CGAJBIJG@File?5not?5valid?5?9?5?$AA@ 100210f0     alm_bncs_output.obj
 0002:00003104       ??_C@_01OHGJGJJP@?$FL?$AA@ 10021104     alm_bncs_output.obj
 0002:00003108       ??_C@_01LBDDMOBJ@?$FN?$AA@ 10021108     alm_bncs_output.obj
 0002:0000310a       ??_C@_00CNPNBAHC@?$AA@     1002110a     alm_bncs_output.obj
 0002:0000310c       ??_C@_05MBDCODDP@Group?$AA@ 1002110c     alm_bncs_output.obj
 0002:00003114       ??_C@_01NEMOKFLO@?$DN?$AA@ 10021114     alm_bncs_output.obj
 0002:00003118       ??_C@_0BM@ONJJDKHD@Load?5processes?5took?5?$CFd?5?$CI?$CFd?$CJ?$AA@ 10021118     alm_bncs_output.obj
 0002:00003134       ??_C@_09EHIIFBLM@?1outputs?1?$AA@ 10021134     alm_bncs_output.obj
 0002:00003140       ??_C@_01GEODFPGF@?8?$AA@   10021140     alm_bncs_output.obj
 0002:00003144       ??_C@_05CFIFMHLA@?8?5?9?5?8?$AA@ 10021144     alm_bncs_output.obj
 0002:0000314c       ??_C@_0BM@GKHBNOHF@newFile?4?5Failed?5to?5remove?5?8?$AA@ 1002114c     alm_bncs_output.obj
 0002:00003168       ??_C@_04GAOAGNCM@?4xml?$AA@ 10021168     alm_bncs_output.obj
 0002:00003170       ??_C@_01IDAFKMJL@_?$AA@    10021170     alm_bncs_output.obj
 0002:00003174       ??_C@_0BE@OJOGEEMJ@config?1devicetypes?1?$AA@ 10021174     alm_bncs_output.obj
 0002:00003188       ??_C@_0O@DHFAHCBE@No?5file?5found?$AA@ 10021188     alm_bncs_output.obj
 0002:00003198       ??_C@_0M@HMDKFLHF@BNCS_CONFIG?$AA@ 10021198     alm_bncs_output.obj
 0002:000031a4       ??_C@_06JIODDOFH@System?$AA@ 100211a4     alm_bncs_output.obj
 0002:000031ac       ??_C@_09GIMPJFPI@Templates?$AA@ 100211ac     alm_bncs_output.obj
 0002:000031b8       ??_C@_09FGLEONFO@Instances?$AA@ 100211b8     alm_bncs_output.obj
 0002:000031c4       ??_C@_06BNFOCFOC@Driver?$AA@ 100211c4     alm_bncs_output.obj
 0002:000031cc       ??_C@_05OEOKGKGJ@?$DM?1h1?$DO?$AA@ 100211cc     alm_bncs_output.obj
 0002:000031d4       ??_C@_0BK@FOHJCMCF@?$DMh1?$DOAlarms?5BNCS?5Output?5?9?5?$AA@ 100211d4     alm_bncs_output.obj
 0002:000031f0       ??_C@_06NHPJKFDC@Module?$AA@ 100211f0     alm_bncs_output.obj
 0002:000031f8       ??_C@_02BIKLEMDE@db?$AA@   100211f8     alm_bncs_output.obj
 0002:000031fc       ??_C@_0BH@MFOOPBMJ@Load?5File?5took?5?$CFd?5?$CI?$CFd?$CJ?$AA@ 100211fc     alm_bncs_output.obj
 0002:00003214       ??_C@_04MEMAJGDJ@name?$AA@ 10021214     alm_bncs_output.obj
 0002:0000321c       ??_C@_0BF@HMOKLADJ@?1config?1devicetypes?1?$AA@ 1002121c     alm_bncs_output.obj
 0002:00003234       ??_C@_01IHBHIGKO@?0?$AA@   10021234     alm_bncs_output.obj
 0002:00003238       ??_C@_0CE@LBNHEBHP@alm_bncs_output?3?3saveFile?4?5no?5fi@ 10021238     alm_bncs_output.obj
 0002:0000325c       ??_C@_0CJ@GHPGJALJ@alm_bncs_output?3?3saveFile?4?5no?5fi@ 1002125c     alm_bncs_output.obj
 0002:00003288       ??_C@_0BL@MKFNCHPB@alm_bncs_output?3?3saveFile?5?$AA@ 10021288     alm_bncs_output.obj
 0002:000032a4       ??_C@_0DI@ILJLHKNF@alm_bncs_output?3?3saveFile?5?9?5Fail@ 100212a4     alm_bncs_output.obj
 0002:000032dc       ??_C@_08IJKOBABM@?$FLSystem?$FN?$AA@ 100212dc     alm_bncs_output.obj
 0002:000032e8       ??_C@_01EEMJAFIK@?6?$AA@   100212e8     alm_bncs_output.obj
 0002:000032ec       ??_C@_05DCIFAFBG@Name?$DN?$AA@ 100212ec     alm_bncs_output.obj
 0002:000032f4       ??_C@_0M@KFAEAMKK@ConfigTool?$DN?$AA@ 100212f4     alm_bncs_output.obj
 0002:00003300       ??_C@_0BD@ECBGAABG@Module?$DNalm_bncs_op?$AA@ 10021300     alm_bncs_output.obj
 0002:00003314       ??_C@_0L@OAOLEFHA@AlmSystem?$DN?$AA@ 10021314     alm_bncs_output.obj
 0002:00003320       ??_C@_0O@JJPKFDME@?$FLBNCS_CONFIG?$FN?$AA@ 10021320     alm_bncs_output.obj
 0002:00003330       ??_C@_07CEPBJFMP@Driver?$DN?$AA@ 10021330     alm_bncs_output.obj
 0002:00003338       ??_C@_0M@OBKABPCD@?$FLTemplates?$FN?$AA@ 10021338     alm_bncs_output.obj
 0002:00003344       ??_C@_0M@NOCLGCIG@?$FLInstances?$FN?$AA@ 10021344     alm_bncs_output.obj
 0002:00003350       ??_C@_09EDMCHOAK@?$FLProcess?$FN?$AA@ 10021350     alm_bncs_output.obj
 0002:0000335c       ??_C@_0BH@BACOLKKM@Failed?5to?5open?5file?5?9?5?$AA@ 1002135c     alm_bncs_output.obj
 0002:00003374       ??_C@_0N@NCGBJIIG@Alarm?5output?$AA@ 10021374     alm_bncs_output.obj
 0002:00003384       ??_C@_0BJ@JFKPNGEC@New?5name?5already?5exists?4?$AA@ 10021384     alm_bncs_output.obj
 0002:000033a0       ??_C@_0BE@LHJFFFK@cBNCS?5Output?5Editor?$AA@ 100213a0     alm_bncs_output.obj
 0002:000033b4       ??_C@_0BH@LOOPHGAH@Home?1Alarms?1Processes?0?$AA@ 100213b4     alm_bncs_output.obj
 0002:000033cc       ??_C@_0CI@HFECGJBN@EditProcess?4?5command?$DNnavigate?5fi@ 100213cc     alm_bncs_output.obj
 0002:000033f4       ??_C@_08NCKPMOJE@navigate?$AA@ 100213f4     alm_bncs_output.obj
 0002:00003400       ??_C@_0DK@BDJFPJFJ@alm_bncs_output?3?3menuDuplicateFi@ 10021400     alm_bncs_output.obj
 0002:0000343c       ??_C@_0CF@BJEPEFIO@alm_bncs_output?3?3menuDuplicateFi@ 1002143c     alm_bncs_output.obj
 0002:00003464       ??_C@_0BB@FNGGGEL@?8?0?5module?5name?5?8?$AA@ 10021464     alm_bncs_output.obj
 0002:00003478       ??_C@_0P@DIBEAHNC@?8?0?5full?5name?5?8?$AA@ 10021478     alm_bncs_output.obj
 0002:00003488       ??_C@_0CL@DBNNALIB@alm_bncs_output?3?3menuDuplicateFi@ 10021488     alm_bncs_output.obj
 0002:000034b4       ??_C@_0DD@KKAPHFNA@alm_bncs_output?3?3menuDuplicateFi@ 100214b4     alm_bncs_output.obj
 0002:000034e8       ??_C@_0CN@PIIDDPG@alm_bncs_output?3?3menuDuplicateFi@ 100214e8     alm_bncs_output.obj
 0002:00003518       ??_C@_0BP@FNILKJIN@deleteFile?4?5Failed?5to?5remove?5?8?$AA@ 10021518     alm_bncs_output.obj
 0002:00003538       ??_C@_0CE@POGKJFEJ@Failed?5to?5remove?5the?5file?5from?5l@ 10021538     alm_bncs_output.obj
 0002:0000355c       ??_C@_0CC@CDAKKADF@alm_bncs_output?3?3updateFileList?$CI@ 1002155c     alm_bncs_output.obj
 0002:00003580       ??_C@_0BD@BOKADGCH@?$FOal_out_?2d?$HL4?$HN?4cfg$?$AA@ 10021580     alm_bncs_output.obj
 0002:00003594       ??_C@_0L@FGNBINDG@ConfigTool?$AA@ 10021594     alm_bncs_output.obj
 0002:000035a0       ??_C@_07BOAKCNCF@al_out_?$AA@ 100215a0     alm_bncs_output.obj
 0002:000035a8       ??_C@_04OCCELDNI@?$CF04d?$AA@ 100215a8     alm_bncs_output.obj
 0002:000035b0       ??_C@_04IFJILJI@?4cfg?$AA@ 100215b0     alm_bncs_output.obj
 0002:000035b8       ??_C@_0O@GMPFIJO@Copy?5?$CF1?5of?5?$CF2?$AA@ 100215b8     alm_bncs_output.obj
 0002:000035c8       ??_C@_0BO@KHKJPMKP@config?1system?1bncs_system?4ini?$AA@ 100215c8     alm_bncs_output.obj
 0002:000035e8       ??_C@_0BJ@PCAHEBMF@markDirty?4?5command?$DNdirty?$AA@ 100215e8     alm_bncs_output.obj
 0002:00003604       ??_C@_05CFEJGMAI@dirty?$AA@ 10021604     alm_bncs_output.obj
 0002:0000360c       ??_C@_0CP@FGJOKIPK@?$DMnobr?$DO?$DMh3?$DOAlarm?5System?5BNCS?5Outp@ 1002160c     alm_bncs_output.obj
 0002:0000363c       ??_C@_0BO@DBHAAIPO@?$DMp?$DOWritten?5by?5Mark?5Baldry?$DM?1p?$DO?$AA@ 1002163c     alm_bncs_output.obj
 0002:0000365c       ??_C@_0BL@EAFPCCN@?$DMp?$DOAlso?3?5Richard?5Kerry?$DM?1p?$DO?$AA@ 1002165c     alm_bncs_output.obj
 0002:00003678       ??_C@_0BB@MKCFKDOD@?8?0?5sFileName?5?$DN?5?8?$AA@ 10021678     alm_bncs_output.obj
 0002:0000368c       ??_C@_0DD@BOCIPJDC@alm_bncs_output?3?3writeDevDescFil@ 1002168c     alm_bncs_output.obj
 0002:000036c0       ??_C@_0CE@FBANFAMH@We?5have?5not?5got?5the?5lock?5on?5file@ 100216c0     alm_bncs_output.obj
 0002:000036e4       ??_C@_0BD@HLAANKPB@Alarms?5BNCS?5Output?$AA@ 100216e4     alm_bncs_output.obj
 0002:000036f8       ??_C@_0EH@NAILNNNP@alm_bncs_output?3?3writeDevDescFil@ 100216f8     alm_bncs_output.obj
 0002:00003740       ??_C@_0CF@LPOLIE@writeDevDescFile?4?5Failed?5to?5remo@ 10021740     alm_bncs_output.obj
 0002:00003768       ??_C@_0DL@HDOJJJBH@alm_bncs_output?3?3writeDevDescFil@ 10021768     alm_bncs_output.obj
 0002:000037a4       ??_C@_0BH@HMDOIPGJ@?$DM?$DPxml?5version?$DN?$CC1?40?$CC?$DP?$DO?6?$AA@ 100217a4     alm_bncs_output.obj
 0002:000037bc       ??_C@_0DP@FOLFKOPD@?$DM?$CBDOCTYPE?5device_description?5SYS@ 100217bc     alm_bncs_output.obj
 0002:000037fc       ??_C@_03JKGHEG@?$CC?$DO?6?$AA@ 100217fc     alm_bncs_output.obj
 0002:00003800       ??_C@_0BL@IINFBLL@?$DMdevice_description?5name?$DN?$CC?$AA@ 10021800     alm_bncs_output.obj
 0002:0000381c       ??_C@_01BJJEKLCA@?$CC?$AA@ 1002181c     alm_bncs_output.obj
 0002:00003820       ??_C@_06JMOJEPOI@name?$DN?$CC?$AA@ 10021820     alm_bncs_output.obj
 0002:00003828       ??_C@_06LEBLMCKC@slot?$DN?$CC?$AA@ 10021828     alm_bncs_output.obj
 0002:00003830       ??_C@_0EK@CJCAPJNB@class?$DN?$CCenum?$CC?5style?$DN?$CCpopup_list?$CC?5@ 10021830     alm_bncs_output.obj
 0002:00003880       ??_C@_0EO@OMJBFCEK@?$CC?5class?$DN?$CCenum?$CC?5style?$DN?$CCpopup_list@ 10021880     alm_bncs_output.obj
 0002:000038d0       ??_C@_08JKAPMBAB@?$CC?5slot?$DN?$CC?$AA@ 100218d0     alm_bncs_output.obj
 0002:000038dc       ??_C@_0P@OEDFINLN@?7?$DMparam?5name?$DN?$CC?$AA@ 100218dc     alm_bncs_output.obj
 0002:000038ec       ??_C@_0L@LOMNHEGK@?7?$DM?1param?$DO?6?$AA@ 100218ec     alm_bncs_output.obj
 0002:000038f8       ??_C@_0BG@DOMCDJB@?$DM?1device_description?$DO?$AA@ 100218f8     alm_bncs_output.obj
 0002:00003910       ??_C@_0CO@GPOENMDC@?8?4?5got?5Dev?5Types?5Xml?5?$CFd?0?5got?5Ins@ 10021910     alm_bncs_output.obj
 0002:00003940       ??_C@_06OCLKHHHK@?8?5to?5?8?$AA@ 10021940     alm_bncs_output.obj
 0002:00003948       ??_C@_0CB@NGMLMDFM@alm_bncs_output?3?3changeDevType?5?8@ 10021948     alm_bncs_output.obj
 0002:0000396c       ??_C@_0DC@HJLKDFBJ@alm_bncs_output?3?3deleteAndLockDe@ 1002196c     alm_bncs_output.obj
 0002:000039a0       ??_C@_0DM@BPJJHMDK@alm_bncs_output?3?3deleteAndLockDe@ 100219a0     alm_bncs_output.obj
 0002:000039dc       ??_C@_0DB@MDIHAIGC@alm_bncs_output?3?3deleteAndLockDe@ 100219dc     alm_bncs_output.obj
 0002:00003a10       ??_C@_0DL@OGPFOBLI@alm_bncs_output?3?3deleteAndLockDe@ 10021a10     alm_bncs_output.obj
 0002:00003a4c       ??_C@_0BH@OHLJKBI@lockDevDesc?4?5file?$DN?8?$CFs?8?$AA@ 10021a4c     alm_bncs_output.obj
 0002:00003a64       ??_C@_0CH@KDMPNBJF@lockDevDesc?4?5already?5locked?4?5fil@ 10021a64     alm_bncs_output.obj
 0002:00003a8c       ??_C@_0CE@GIKDOBGP@lockDevDesc?4?5command?$DNlock?5file?$DN?8@ 10021a8c     alm_bncs_output.obj
 0002:00003ab0       ??_C@_0N@LEBPCLIG@proc_def?4cfg?$AA@ 10021ab0     alm_bncs_output.obj
 0002:00003ac0       ??_C@_0CN@OGGGLPMC@selectSystem?4?5command?$DNdownloadFi@ 10021ac0     alm_bncs_output.obj
 0002:00003af0       ??_C@_0N@LJNCPLAD@downloadFile?$AA@ 10021af0     alm_bncs_output.obj
 0002:00003b00       ??_C@_0CM@MCPBNPJL@selectSystem?4?5command?$DNcheckoutDi@ 10021b00     alm_bncs_output.obj
 0002:00003b2c       ??_C@_0M@IKGKPMGN@checkoutDir?$AA@ 10021b2c     alm_bncs_output.obj
 0002:00003b38       ??_C@_0CO@JJIHFGPF@manage?5templates?4?5checkout?5Dev?5D@ 10021b38     alm_bncs_output.obj
 0002:00003b68       ??_C@_0CL@GMMPLDFO@alm_bncs_output?3?3manageTemplate?$CI@ 10021b68     alm_bncs_output.obj
 0002:00003b94       ??_C@_0DE@NNMOIJHL@manage?5templates?4?5unable?5to?5load@ 10021b94     alm_bncs_output.obj
 0002:00003bc8       ??_C@_0DP@BFAMPNHO@The?5following?5processes?5are?5defi@ 10021bc8     alm_bncs_output.obj
 0002:00003c08       ??_C@_02NMOLBIHC@?6?7?$AA@ 10021c08     alm_bncs_output.obj
 0002:00003c0c       ??_C@_02PHMGELLB@?6?6?$AA@ 10021c0c     alm_bncs_output.obj
 0002:00003c10       ??_C@_0CJ@JBGHJOJD@The?5following?5processes?5do?5not?5e@ 10021c10     alm_bncs_output.obj
 0002:00003c3c       ??_C@_0BI@EJMHEFII@Applying?5template?5error?$AA@ 10021c3c     alm_bncs_output.obj
 0002:00003c54       ??_C@_0O@NNPBEDNJ@instances?4dtd?$AA@ 10021c54     alm_bncs_output.obj
 0002:00003c64       ??_C@_09BJOJOOIO@instances?$AA@ 10021c64     alm_bncs_output.obj
 0002:00003c70       ??_C@_08EMNENPBA@instance?$AA@ 10021c70     alm_bncs_output.obj
 0002:00003c7c       ??_C@_02EGCJHIOB@id?$AA@   10021c7c     alm_bncs_output.obj
 0002:00003c80       ??_C@_04GPMDFGEJ@type?$AA@ 10021c80     alm_bncs_output.obj
 0002:00003c88       ??_C@_02KAJCLHKP@no?$AA@   10021c88     alm_bncs_output.obj
 0002:00003c8c       ??_C@_09EIHFMDLJ@composite?$AA@ 10021c8c     alm_bncs_output.obj
 0002:00003c98       ??_C@_09PPOABKOI@?0offset?$DN0?$AA@ 10021c98     alm_bncs_output.obj
 0002:00003ca4       ??_C@_07FDMMAPON@device?$DN?$AA@ 10021ca4     alm_bncs_output.obj
 0002:00003cac       ??_C@_03GCDGINBO@ref?$AA@  10021cac     alm_bncs_output.obj
 0002:00003cb0       ??_C@_08MJKJKIHF@?0offset?$DN?$AA@ 10021cb0     alm_bncs_output.obj
 0002:00003cbc       ??_C@_0CA@BMAJJLKN@alm_bncs_output?3?3writeInstances?$AA@ 10021cbc     alm_bncs_output.obj
 0002:00003ce0       ??_C@_0FB@OMFELICM@alm_bncs_output?3?3writeInstances?5@ 10021ce0     alm_bncs_output.obj
 0002:00003d38       ??_C@_0ED@PBMHKLPF@alm_bncs_output?3?3writeInstances?5@ 10021d38     alm_bncs_output.obj
 0002:00003d7c       ??_C@_0O@NFBOGKON@?8?4?5hanging?5?$CFd?$AA@ 10021d7c     alm_bncs_output.obj
 0002:00003d8c       ??_C@_0CN@MICFBJGO@alm_bncs_output?3?3writeInstances?5@ 10021d8c     alm_bncs_output.obj
 0002:00003dbc       ??_C@_02HCGKDMEN@?1?$DO?$AA@ 10021dbc     alm_bncs_output.obj
 0002:00003dc0       ??_C@_0BK@CPPOHGKK@?8?5removed?4?5add?5new?5base?5?8?$AA@ 10021dc0     alm_bncs_output.obj
 0002:00003ddc       ??_C@_0CN@DLHIKJDF@alm_bncs_output?3?3writeInstances?5@ 10021ddc     alm_bncs_output.obj
 0002:00003e0c       ??_C@_0O@OGEMLAAM@?0offset?$DN0?$CC?1?$DO?6?$AA@ 10021e0c     alm_bncs_output.obj
 0002:00003e1c       ??_C@_0BO@OGAMGDDA@?$CC?5composite?$DN?$CCno?$CC?5ref?$DN?$CCdevice?$DN?$AA@ 10021e1c     alm_bncs_output.obj
 0002:00003e3c       ??_C@_08GKGFMAO@?$CC?5type?$DN?$CC?$AA@ 10021e3c     alm_bncs_output.obj
 0002:00003e48       ??_C@_0BA@NHJNHGM@?7?$DMinstance?5id?$DN?$CC?$AA@ 10021e48     alm_bncs_output.obj
 0002:00003e58       ??_C@_0CG@GHOGFNMD@?8?5removed?4?5insert?5modified?5insta@ 10021e58     alm_bncs_output.obj
 0002:00003e80       ??_C@_0N@NIEJLLIH@?$DM?1instances?$DO?$AA@ 10021e80     alm_bncs_output.obj
 0002:00003e90       ??_C@_0CD@GDNAJKNJ@?8?5removed?4?5end?5tag?4?5add?5new?5base@ 10021e90     alm_bncs_output.obj
 0002:00003eb4       ??_C@_0CP@HACPPMNH@?8?5removed?4?5end?5tag?4?5insert?5modif@ 10021eb4     alm_bncs_output.obj
 0002:00003ee4       ??_C@_0DE@NDLLJDHH@alm_bncs_output?3?3writeInstances?5@ 10021ee4     alm_bncs_output.obj
 0002:00003f18       ??_C@_0DJ@COEGFHBN@alm_bncs_output?3?3writeInstances?5@ 10021f18     alm_bncs_output.obj
 0002:00003f54       ??_C@_0BD@EOMHPFKD@?8?0?5sInsertDevice?5?8?$AA@ 10021f54     alm_bncs_output.obj
 0002:00003f68       ??_C@_0BB@ILPDDKOI@?8?0?5sInsertBase?5?8?$AA@ 10021f68     alm_bncs_output.obj
 0002:00003f7c       ??_C@_0DD@DMPBAEEP@alm_bncs_output?3?3insertModifiedI@ 10021f7c     alm_bncs_output.obj
 0002:00003fb0       ??_C@_09POPCHIL@?8?0?5type?5?8?$AA@ 10021fb0     alm_bncs_output.obj
 0002:00003fbc       ??_C@_0DK@MMAJHCCG@alm_bncs_output?3?3insertModifiedI@ 10021fbc     alm_bncs_output.obj
 0002:00003ff8       ??_C@_04KOJHOLPO@?$CC?1?$DO?6?$AA@ 10021ff8     alm_bncs_output.obj
 0002:00004000       ??_C@_02ILLPBGAO@?$DN?$CC?$AA@ 10022000     alm_bncs_output.obj
 0002:00004004       ??_C@_01CLKCMJKC@?5?$AA@   10022004     alm_bncs_output.obj
 0002:00004008       ??_C@_0BA@KJBPGAMK@devicetypes?4dtd?$AA@ 10022008     alm_bncs_output.obj
 0002:00004018       ??_C@_0M@EHMABMKM@devicetypes?$AA@ 10022018     alm_bncs_output.obj
 0002:00004024       ??_C@_06BBBNOMFN@alarms?$AA@ 10022024     alm_bncs_output.obj
 0002:0000402c       ??_C@_06NBOBHOCP@family?$AA@ 1002202c     alm_bncs_output.obj
 0002:00004034       ??_C@_0CG@NGPKNPDG@alm_bncs_output?3?3writeDeviceType@ 10022034     alm_bncs_output.obj
 0002:00004060       ??_C@_0FJ@LECIKHEI@alm_bncs_output?3?3writeDeviceType@ 10022060     alm_bncs_output.obj
 0002:000040c0       ??_C@_0EL@BCIDCDAP@alm_bncs_output?3?3writeDeviceType@ 100220c0     alm_bncs_output.obj
 0002:0000410c       ??_C@_0BP@BELJKNIO@family?$DN?$CCalarms?$CC?5composite?$DN?$CCno?$CC?$AA@ 1002210c     alm_bncs_output.obj
 0002:0000412c       ??_C@_02KOPDJAMB@?$CC?5?$AA@ 1002212c     alm_bncs_output.obj
 0002:00004130       ??_C@_0M@EBEEDINJ@?7?$DMtype?5id?$DN?$CC?$AA@ 10022130     alm_bncs_output.obj
 0002:0000413c       ??_C@_0P@ENJEBNMA@?8?0?5templates?5?8?$AA@ 1002213c     alm_bncs_output.obj
 0002:0000414c       ??_C@_0CP@MMGJKLKH@alm_bncs_output?3?3writeDeviceType@ 1002214c     alm_bncs_output.obj
 0002:0000417c       ??_C@_0DF@CLIKBDPP@alm_bncs_output?3?3writeDeviceType@ 1002217c     alm_bncs_output.obj
 0002:000041b8       ??_C@_0EF@DAJBKPLM@alm_bncs_output?3?3writeDeviceType@ 100221b8     alm_bncs_output.obj
 0002:00004200       ??_C@_0ED@BLPOFGAA@alm_bncs_output?3?3writeDeviceType@ 10022200     alm_bncs_output.obj
 0002:00004244       ??_C@_0P@FEOHLFNM@?$DM?1devicetypes?$DO?$AA@ 10022244     alm_bncs_output.obj
 0002:00004258       ??_C@_0FB@EMHJFMIK@alm_bncs_output?3?3writeDeviceType@ 10022258     alm_bncs_output.obj
 0002:000042ac       ??_C@_08KNIPCEPG@?8?5line?5?8?$AA@ 100222ac     alm_bncs_output.obj
 0002:000042b8       ??_C@_0DG@BNMGFEEN@alm_bncs_output?3?3writeDeviceType@ 100222b8     alm_bncs_output.obj
 0002:000042f0       ??_C@_0EC@CHLHNDPA@alm_bncs_output?3?3writeDeviceType@ 100222f0     alm_bncs_output.obj
 0002:00004334       ??_C@_0DK@JGPNNMCC@alm_bncs_output?3?3writeDeviceType@ 10022334     alm_bncs_output.obj
 0002:00004370       ??_C@_0DP@OENLBFPP@alm_bncs_output?3?3writeDeviceType@ 10022370     alm_bncs_output.obj
 0002:000043b0       ??_C@_08OJEOLAAJ@?8?0?5new?5?8?$AA@ 100223b0     alm_bncs_output.obj
 0002:000043bc       ??_C@_0DC@GDHOAEPA@alm_bncs_output?3?3changeDevTypeDe@ 100223bc     alm_bncs_output.obj
 0002:000043f0       ??_C@_0FN@BDBADJJD@alm_bncs_output?3?3changeDevTypeDe@ 100223f0     alm_bncs_output.obj
 0002:00004450       ??_C@_0FA@IHIHNKLJ@alm_bncs_output?3?3changeDevTypeDe@ 10022450     alm_bncs_output.obj
 0002:000044a0       ??_C@_0DJ@GEBAAEEA@alm_bncs_output?3?3changeDevTypeDe@ 100224a0     alm_bncs_output.obj
 0002:000044dc       ??_C@_0DC@ENIIKGCI@alm_bncs_output?3?3changeDevTypeDe@ 100224dc     alm_bncs_output.obj
 0002:00004510       ??_C@_03PCPALPJL@?1?$DO?6?$AA@ 10022510     alm_bncs_output.obj
 0002:00004518       ??_C@_0EA@FBDMIHIM@alm_bncs_output?3?3changeDevTypeDe@ 10022518     alm_bncs_output.obj
 0002:00004558       ??_C@_0DO@FHFOGCEI@alm_bncs_output?3?3changeDevTypeDe@ 10022558     alm_bncs_output.obj
 0002:00004598       ??_C@_0DK@CPHFNOJO@alm_bncs_output?3?3changeDevTypeDe@ 10022598     alm_bncs_output.obj
 0002:000045d4       ??_C@_0DP@JPFECPFC@alm_bncs_output?3?3changeDevTypeDe@ 100225d4     alm_bncs_output.obj
 0002:00004618       ??_C@_0FA@FAPFAJHA@alm_bncs_output?3?3changeDevTypeDe@ 10022618     alm_bncs_output.obj
 0002:00004668       ??_C@_0FJ@KNKEJAHJ@alm_bncs_output?3?3changeDevTypeIn@ 10022668     alm_bncs_output.obj
 0002:000046c8       ??_C@_0EP@DMOMHNEH@alm_bncs_output?3?3changeDevTypeIn@ 100226c8     alm_bncs_output.obj
 0002:00004718       ??_C@_0DH@KMBCGPMM@alm_bncs_output?3?3changeDevTypeIn@ 10022718     alm_bncs_output.obj
 0002:00004750       ??_C@_06CILCFPKN@type?$DN?$CC?$AA@ 10022750     alm_bncs_output.obj
 0002:00004758       ??_C@_0N@NKKILLAH@ref?$DN?$CCdevice?$DN?$AA@ 10022758     alm_bncs_output.obj
 0002:00004768       ??_C@_0N@MPDJOEFB@?0offset?$DN0?$CC?1?$DO?$AA@ 10022768     alm_bncs_output.obj
 0002:00004778       ??_C@_0GM@MEBCCBKB@alm_bncs_output?3?3changeDevTypeIn@ 10022778     alm_bncs_output.obj
 0002:000047e4       ??_C@_04JCLKENGJ@id?$DN?$CC?$AA@ 100227e4     alm_bncs_output.obj
 0002:000047f0       ??_C@_0GP@GPDIBFJN@alm_bncs_output?3?3changeDevTypeIn@ 100227f0     alm_bncs_output.obj
 0002:00004860       ??_C@_0DC@FCBLHBOD@alm_bncs_output?3?3changeDevTypeIn@ 10022860     alm_bncs_output.obj
 0002:00004894       ??_C@_0DA@JEGAJKHO@alm_bncs_output?3?3changeDevTypeIn@ 10022894     alm_bncs_output.obj
 0002:000048c4       ??_C@_0DM@NGFHOGJE@alm_bncs_output?3?3changeDevTypeIn@ 100228c4     alm_bncs_output.obj
 0002:00004900       ??_C@_0FD@CKCIOBLM@alm_bncs_output?3?3changeDevTypeIn@ 10022900     alm_bncs_output.obj
 0002:00004954       ??_C@_02KIDIFCCK@?8?5?$AA@ 10022954     alm_bncs_output.obj
 0002:00004958       ??_C@_0BL@LJGEJILJ@version?5?$DN?5?81?40?8?5encoding?$DN?8?$AA@ 10022958     alm_bncs_output.obj
 0002:00004974       ??_C@_03PJHHNEEI@xml?$AA@  10022974     alm_bncs_output.obj
 0002:00004978       ??_C@_08FKACIMPB@?1config?1?$AA@ 10022978     alm_bncs_output.obj
 0002:00004984       ??_C@_0CA@FKIPKAAN@replyDownload?4?5Fail?4?5error?5?8?$CFs?8?$AA@ 10022984     alm_bncs_output.obj
 0002:000049a4       ??_C@_0CK@DJMIMKJE@?6New?5file?5may?5be?5generated?5autom@ 100229a4     alm_bncs_output.obj
 0002:000049d0       ??_C@_07MPPKIBJA@Error?3?6?$AA@ 100229d0     alm_bncs_output.obj
 0002:000049d8       ??_C@_05NAOIJFC@Error?$AA@ 100229d8     alm_bncs_output.obj
 0002:000049e0       ??_C@_0BN@JJMCBDNN@BNCS?5Output?3Unknown?5response?$AA@ 100229e0     alm_bncs_output.obj
 0002:00004a00       ??_C@_0CB@MCNKMHPJ@replyDownload?4?5Ok?1r?9o?4?5?8?$CFs?8?5?8?$CFs?8@ 10022a00     alm_bncs_output.obj
 0002:00004a24       ??_C@_0M@FNMDGLGJ@Got?5file?5?9?5?$AA@ 10022a24     alm_bncs_output.obj
 0002:00004a30       ??_C@_0L@GBLJJCHL@File?5is?5?$CFs?$AA@ 10022a30     alm_bncs_output.obj
 0002:00004a3c       ??_C@_0BP@HPEFIJDM@replyDownload?4?5Done?4?5?8?$CFs?8?5?8?$CFs?8?$AA@ 10022a3c     alm_bncs_output.obj
 0002:00004a5c       ??_C@_03GJCOJFLC@?4?6?6?$AA@ 10022a5c     alm_bncs_output.obj
 0002:00004a60       ??_C@_0BM@CGOIHJMM@Could?5not?5Create?5directory?6?$AA@ 10022a60     alm_bncs_output.obj
 0002:00004a7c       ??_C@_0BB@IMCDCEGC@Alarms?1Processes?$AA@ 10022a7c     alm_bncs_output.obj
 0002:00004a90       ??_C@_0CA@NJNGGAOK@doDone?3no?5handler?5for?5file?5?8?$CFs?8?$AA@ 10022a90     alm_bncs_output.obj
 0002:00004ab0       ??_C@_0BG@DALBJPIB@replyLock?4?5Fail?4?5?8?$CFs?8?$AA@ 10022ab0     alm_bncs_output.obj
 0002:00004ac8       ??_C@_0CC@OAGIAEAC@?6File?5will?5be?5available?5read?5onl@ 10022ac8     alm_bncs_output.obj
 0002:00004aec       ??_C@_06JGFHLLHI@Lock?3?5?$AA@ 10022aec     alm_bncs_output.obj
 0002:00004af4       ??_C@_04LADJNOK@Lock?$AA@  10022af4     alm_bncs_output.obj
 0002:00004afc       ??_C@_0BJ@GMKILPME@replyLock?4?5Else?5?$CFd?4?5?8?$CFs?8?$AA@ 10022afc     alm_bncs_output.obj
 0002:00004b18       ??_C@_0BD@OKIEINHG@got?5new?5lock?5on?5?9?5?$AA@ 10022b18     alm_bncs_output.obj
 0002:00004b2c       ??_C@_0BE@CKAOIKJF@replyUpload?4?5Done?4?5?$AA@ 10022b2c     alm_bncs_output.obj
 0002:00004b40       ??_C@_0BL@JPFFJHGP@replyUpload?4?5command?$DNclean?$AA@ 10022b40     alm_bncs_output.obj
 0002:00004b5c       ??_C@_05CCAMFJOL@clean?$AA@ 10022b5c     alm_bncs_output.obj
 0002:00004b64       ??_C@_0CO@BCOKJKIG@alm_bncs_output?3?3saveTemplates?4?5@ 10022b64     alm_bncs_output.obj
 0002:00004b94       ??_C@_0CA@FBNMKKKC@alm_bncs_output?3?3saveTemplates?5?$AA@ 10022b94     alm_bncs_output.obj
 0002:00004bb4       ??_C@_02OLCMCLAM@?0?8?$AA@ 10022bb4     alm_bncs_output.obj
 0002:00004bb8       ??_C@_0DI@OGAIJPFG@alm_bncs_output?3?3saveTemplates?5?9@ 10022bb8     alm_bncs_output.obj
 0002:00004bf0       ??_C@_0BJ@JBOJMBFB@?$CF1?1?$CF2?3Dev?5desc?5file?5?9?5?$CF3?$AA@ 10022bf0     alm_bncs_output.obj
 0002:00004c0c       ??_C@_0BH@DBJAHDGO@0?10?3No?5dev?5desc?5files?4?$AA@ 10022c0c     alm_bncs_output.obj
 0002:00004c24       ??_C@_0BB@MKEIEHFB@Creating?5folder?5?$AA@ 10022c24     alm_bncs_output.obj
 0002:00004c38       ??_C@_0DP@NKDBFOMD@alm_bncs_output?3?3writeDevDescFil@ 10022c38     alm_bncs_output.obj
 0002:00004c7c       ??_7autoNumberDialog@@6BQObject@@@ 10022c7c     autonumberdialogimpl.obj
 0002:00004e40       ??_7autoNumberDialog@@6BQPaintDevice@@@ 10022e40     autonumberdialogimpl.obj
 0002:00004e64       ??_7cOutputFile@@6B@       10022e64     cOutputFile.obj
 0002:00004e6c       ??_7?$QDict@VdevTemplate@@@@6B@ 10022e6c     devTemplate.obj
 0002:00004e8c       ??_7TemplateList@@6B@      10022e8c     devTemplate.obj
 0002:00004ea8       ??_C@_0DG@NFJIOOMA@loadDevDesc?5fail?4?5can?8t?5open?5for@ 10022ea8     devTemplate.obj
 0002:00004ee0       ??_C@_0DA@DIPGKCEB@loadDevDesc?5fail?4?5can?8t?5set?5cont@ 10022ee0     devTemplate.obj
 0002:00004f10       ??_C@_0BD@INOIJGBO@device_description?$AA@ 10022f10     devTemplate.obj
 0002:00004f28       ??_C@_0FO@EIODHCDL@loadDevDesc?5fail?4?5document?5eleme@ 10022f28     devTemplate.obj
 0002:00004f88       ??_C@_0FE@IAFNKMBE@loadDevDesc?5fail?4?5document?5eleme@ 10022f88     devTemplate.obj
 0002:00004fdc       ??_C@_05LJDNNBIK@param?$AA@ 10022fdc     devTemplate.obj
 0002:00004fe4       ??_C@_04POIHOKKJ@slot?$AA@ 10022fe4     devTemplate.obj
 0002:00004fec       ??_C@_03BNGEDOB@?8?5?8?$AA@ 10022fec     devTemplate.obj
 0002:00004ff0       ??_C@_0BK@ONNEFOBL@devTemplate?3?3saveFile?5?9?5?8?$AA@ 10022ff0     devTemplate.obj
 0002:00005010       ??_7dialog@@6BQObject@@@   10023010     dialogimpl.obj
 0002:000051c8       ??_7dialog@@6BQPaintDevice@@@ 100231c8     dialogimpl.obj
 0002:000051e8       ??_C@_08LAIGBKAI@ProcList?$AA@ 100231e8     dialogimpl.obj
 0002:000051f4       ??_C@_03PADCEAKC@Red?$AA@  100231f4     dialogimpl.obj
 0002:000051f8       ??_C@_02HNLLPFKA@up?$AA@   100231f8     dialogimpl.obj
 0002:000051fc       ??_C@_04JMOKAGMG@down?$AA@ 100231fc     dialogimpl.obj
 0002:00005204       ??_C@_0O@KMLAMDNA@1moveProcUp?$CI?$CJ?$AA@ 10023204     dialogimpl.obj
 0002:00005214       ??_C@_0BA@HOOEGNLM@1moveProcDown?$CI?$CJ?$AA@ 10023214     dialogimpl.obj
 0002:00005224       ??_C@_0N@FHKHPEBN@1reSort?$CIint?$CJ?$AA@ 10023224     dialogimpl.obj
 0002:00005234       ??_C@_0O@GBIKBCJG@2clicked?$CIint?$CJ?$AA@ 10023234     dialogimpl.obj
 0002:00005244       ??_C@_0DD@PEPJEGHO@1slotChange?$CIQListViewItem?5?$CK?0?5int@ 10023244     dialogimpl.obj
 0002:00005278       ??_C@_0DE@IGFEKAPA@2itemRenamed?$CIQListViewItem?5?$CK?0int@ 10023278     dialogimpl.obj
 0002:000052ac       ??_C@_0CE@FPOPOGMP@1itemDoubleClicked?$CIQListViewItem@ 100232ac     dialogimpl.obj
 0002:000052d0       ??_C@_0CB@GDMHAGOL@2doubleClicked?5?$CIQListViewItem?5?$CK?$CJ@ 100232d0     dialogimpl.obj
 0002:000052f4       ??_C@_0BN@MMHKMIN@1selectProc?$CIQListViewItem?5?$CK?$CJ?$AA@ 100232f4     dialogimpl.obj
 0002:00005314       ??_C@_0CC@CCEKIDAP@2currentChanged?5?$CIQListViewItem?5?$CK@ 10023314     dialogimpl.obj
 0002:00005338       ??_C@_0BD@PBLBIMCO@1changeSelection?$CI?$CJ?$AA@ 10023338     dialogimpl.obj
 0002:0000534c       ??_C@_0BF@DCJGEHLJ@2selectionChanged?5?$CI?$CJ?$AA@ 1002334c     dialogimpl.obj
 0002:00005364       ??_C@_0O@KGEHHEMF@1autoNumber?$CI?$CJ?$AA@ 10023364     dialogimpl.obj
 0002:00005374       ??_C@_0M@CPPMHGBO@1copyData?$CI?$CJ?$AA@ 10023374     dialogimpl.obj
 0002:00005380       ??_C@_0N@DJHCJEAJ@1pasteData?$CI?$CJ?$AA@ 10023380     dialogimpl.obj
 0002:00005390       ??_C@_0O@CONCKEHB@1clearSlots?$CI?$CJ?$AA@ 10023390     dialogimpl.obj
 0002:000053a0       ??_C@_05NDLFFNHM@paste?$AA@ 100233a0     dialogimpl.obj
 0002:000053a8       ??_C@_06FENKCKDB@?$CGPaste?$AA@ 100233a8     dialogimpl.obj
 0002:000053b0       ??_C@_05NEBJFIEK@Paste?$AA@ 100233b0     dialogimpl.obj
 0002:000053b8       ??_C@_04COAGEIMF@copy?$AA@ 100233b8     dialogimpl.obj
 0002:000053c0       ??_C@_05EJNCNHFE@?$CGCopy?$AA@ 100233c0     dialogimpl.obj
 0002:000053c8       ??_C@_04OPMHGHMB@Copy?$AA@ 100233c8     dialogimpl.obj
 0002:000053d0       ??_C@_0BO@FHLKKLPM@1itemChanged?$CIconst?5QString?5?$CG?$CJ?$AA@ 100233d0     dialogimpl.obj
 0002:000053f0       ??_C@_0BO@GCMLDCHC@2valueChanged?$CIconst?5QString?$CG?$CJ?$AA@ 100233f0     dialogimpl.obj
 0002:00005410       ??_C@_0BH@HOHNNCNI@1clipboardDataChange?$CI?$CJ?$AA@ 10023410     dialogimpl.obj
 0002:00005428       ??_C@_0P@GLIODLHI@2dataChanged?$CI?$CJ?$AA@ 10023428     dialogimpl.obj
 0002:00005438       ??_C@_01GBGANLPD@0?$AA@    10023438     dialogimpl.obj
 0002:0000543c       ??_C@_0CL@ECKAIIK@Valid?5entries?5are?5numbers?5betwee@ 1002343c     dialogimpl.obj
 0002:00005468       ??_C@_0BK@DIELLHKN@BNCS?5Output?5Configuration?$AA@ 10023468     dialogimpl.obj
 0002:00005484       ??_C@_01GPOEFGEJ@?7?$AA@   10023484     dialogimpl.obj
 0002:00005488       ??_C@_07JLEKEEPN@?$CGCancel?$AA@ 10023488     dialogimpl.obj
 0002:00005490       ??_C@_05GEGFPEDH@?$CGSkip?$AA@ 10023490     dialogimpl.obj
 0002:00005498       ??_C@_0P@NBCLPJFJ@?$CGIgnore?5Groups?$AA@ 10023498     dialogimpl.obj
 0002:000054a8       ??_C@_0BI@PGBDCOHI@?5is?5not?5a?5member?6group?5?$AA@ 100234a8     dialogimpl.obj
 0002:000054c0       ??_C@_08JNCEHING@Process?5?$AA@ 100234c0     dialogimpl.obj
 0002:000054cc       ??_C@_0M@IMMAOIGI@BNCS?5Output?$AA@ 100234cc     dialogimpl.obj
 0002:000054d8       ??_C@_0BH@LNFBOAFN@?6There?5are?5duplicates?4?$AA@ 100234d8     dialogimpl.obj
 0002:000054f0       ??_C@_0CK@OKFNLNGP@?$DMp?$DOThere?5are?5entries?5out?5of?5rang@ 100234f0     dialogimpl.obj
 0002:0000551c       ??_C@_0BB@LKLALJMG@?$DMh1?$DOWarning?$DM?1h1?$DO?$AA@ 1002351c     dialogimpl.obj
 0002:00005530       ??_C@_0BF@NNDHAIMI@Clear?5Selected?5Slots?$AA@ 10023530     dialogimpl.obj
 0002:00005548       ??_C@_0BA@OHGOBHDJ@Clear?5All?5Slots?$AA@ 10023548     dialogimpl.obj
 0002:00005558       ??_C@_0NF@BIDMPGOE@Do?5you?5want?5to?5delete?5the?5slot?5a@ 10023558     dialogimpl.obj
 0002:00005630       ??_C@_0BH@DHBBLIIC@?$CGNon?5template?5assigned?$AA@ 10023630     dialogimpl.obj
 0002:00005648       ??_C@_04NMHBPLPB@?$CGAll?$AA@ 10023648     dialogimpl.obj
 0002:00005650       ??_C@_0BE@MONDOIGF@Alarms?5BNCS?5Outputs?$AA@ 10023650     dialogimpl.obj
 0002:00005664       ??_C@_0BD@OLBABOEK@vector?$DMT?$DO?5too?5long?$AA@ 10023664     dialogimpl.obj
 0002:0000567c       ??_7manage_tempBase@@6BQObject@@@ 1002367c     manage_temp.obj
 0002:00005840       ??_7manage_tempBase@@6BQPaintDevice@@@ 10023840     manage_temp.obj
 0002:00005864       ??_SQPushButton@@6BQObject@@@ 10023864     manage_temp.obj
 0002:00005a54       ??_SQPushButton@@6BQPaintDevice@@@ 10023a54     manage_temp.obj
 0002:00005a7c       ??_SQLabel@@6BQObject@@@   10023a7c     manage_temp.obj
 0002:00005c74       ??_SQLabel@@6BQPaintDevice@@@ 10023c74     manage_temp.obj
 0002:00005c9c       ??_SQComboBox@@6BQObject@@@ 10023c9c     manage_temp.obj
 0002:00005e80       ??_SQComboBox@@6BQPaintDevice@@@ 10023e80     manage_temp.obj
 0002:00005ea4       ??_SQLineEdit@@6BQObject@@@ 10023ea4     manage_temp.obj
 0002:000060cc       ??_SQLineEdit@@6BQPaintDevice@@@ 100240cc     manage_temp.obj
 0002:000060f4       ??_SQSpinBox@@6BQObject@@@ 100240f4     manage_temp.obj
 0002:000062ec       ??_SQSpinBox@@6BQPaintDevice@@@ 100242ec     manage_temp.obj
 0002:00006310       ??_SQSpinBox@@6B@          10024310     manage_temp.obj
 0002:00006324       ??_SQTable@@6BQObject@@@   10024324     manage_temp.obj
 0002:000066c4       ??_SQTable@@6BQPaintDevice@@@ 100246c4     manage_temp.obj
 0002:000066ec       ??_SQSpacerItem@@6B@       100246ec     manage_temp.obj
 0002:00006734       ??_SQGridLayout@@6BQObject@@@ 10024734     manage_temp.obj
 0002:000067a4       ??_SQGridLayout@@6BQLayoutItem@@@ 100247a4     manage_temp.obj
 0002:000067ec       ??_SQHBoxLayout@@6BQObject@@@ 100247ec     manage_temp.obj
 0002:00006854       ??_SQHBoxLayout@@6BQLayoutItem@@@ 10024854     manage_temp.obj
 0002:0000689c       ??_SQVBoxLayout@@6BQObject@@@ 1002489c     manage_temp.obj
 0002:00006904       ??_SQVBoxLayout@@6BQLayoutItem@@@ 10024904     manage_temp.obj
 0002:00006944       ??_C@_0BA@ECGMJAHD@manage_tempBase?$AA@ 10024944     manage_temp.obj
 0002:00006954       ??_C@_0BG@JALDPJDK@manage_tempBaseLayout?$AA@ 10024954     manage_temp.obj
 0002:0000696c       ??_C@_07KKDPDMDC@layout5?$AA@ 1002496c     manage_temp.obj
 0002:00006974       ??_C@_0L@KGLFILOJ@textLabel1?$AA@ 10024974     manage_temp.obj
 0002:00006980       ??_C@_0P@JLAGMAGF@comboTemplates?$AA@ 10024980     manage_temp.obj
 0002:00006990       ??_C@_09MJGHBDFL@buttonNew?$AA@ 10024990     manage_temp.obj
 0002:0000699c       ??_C@_07IBBCGPPB@layout6?$AA@ 1002499c     manage_temp.obj
 0002:000069a4       ??_C@_08DKBDHOFF@buttonOk?$AA@ 100249a4     manage_temp.obj
 0002:000069b0       ??_C@_0N@OLKBNHFJ@buttonCancel?$AA@ 100249b0     manage_temp.obj
 0002:000069c0       ??_C@_09DMIEKCOP@tabWidget?$AA@ 100249c0     manage_temp.obj
 0002:000069cc       ??_C@_03CEDILPBK@tab?$AA@  100249cc     manage_temp.obj
 0002:000069d0       ??_C@_09PEOMDABK@tabLayout?$AA@ 100249d0     manage_temp.obj
 0002:000069dc       ??_C@_07LDCEANHD@layout4?$AA@ 100249dc     manage_temp.obj
 0002:000069e4       ??_C@_0N@HPEGIJEE@textLabel1_2?$AA@ 100249e4     manage_temp.obj
 0002:000069f4       ??_C@_0L@DPGNGODI@editPrefix?$AA@ 100249f4     manage_temp.obj
 0002:00006a00       ??_C@_07OFHOKKPF@layout2?$AA@ 10024a00     manage_temp.obj
 0002:00006a08       ??_C@_0BB@PGPKDOIH@textLabel1_2_2_2?$AA@ 10024a08     manage_temp.obj
 0002:00006a1c       ??_C@_08LPMMDAGJ@spinBase?$AA@ 10024a1c     manage_temp.obj
 0002:00006a28       ??_C@_07MOFDPJDG@layout1?$AA@ 10024a28     manage_temp.obj
 0002:00006a30       ??_C@_0P@IKOBPDDP@textLabel1_2_2?$AA@ 10024a30     manage_temp.obj
 0002:00006a40       ??_C@_0L@DGAJKLHO@spinOffset?$AA@ 10024a40     manage_temp.obj
 0002:00006a4c       ??_C@_09PPOBMLDK@listSlots?$AA@ 10024a4c     manage_temp.obj
 0002:00006a58       ??_C@_09HPDNJEFH@Parameter?$AA@ 10024a58     manage_temp.obj
 0002:00006a64       ??_C@_04DPEGMFKN@Slot?$AA@ 10024a64     manage_temp.obj
 0002:00006a6c       ??_C@_09FAEDEDKO@layoutNew?$AA@ 10024a6c     manage_temp.obj
 0002:00006a78       ??_C@_0BG@MDOIBKIO@buttonAutoNumberSlots?$AA@ 10024a78     manage_temp.obj
 0002:00006a90       ??_C@_0BB@LELBEHEN@buttonClearSlots?$AA@ 10024a90     manage_temp.obj
 0002:00006aa4       ??_C@_05GBGDENAC@tab_2?$AA@ 10024aa4     manage_temp.obj
 0002:00006aac       ??_C@_0M@BMGEADGH@tabLayout_2?$AA@ 10024aac     manage_temp.obj
 0002:00006ab8       ??_C@_0O@HAFIDGAD@tableInstance?$AA@ 10024ab8     manage_temp.obj
 0002:00006ac8       ??_C@_08MOCFFNLD@Instance?$AA@ 10024ac8     manage_temp.obj
 0002:00006ad4       ??_C@_07DOAOMMKG@Enabled?$AA@ 10024ad4     manage_temp.obj
 0002:00006adc       ??_C@_08HEFODFJH@layout14?$AA@ 10024adc     manage_temp.obj
 0002:00006ae8       ??_C@_0BA@HKJGCBDI@buttonSelectAll?$AA@ 10024ae8     manage_temp.obj
 0002:00006af8       ??_C@_0BC@JJOPLCFG@buttonUnselectAll?$AA@ 10024af8     manage_temp.obj
 0002:00006b0c       ??_C@_0BF@BFJDBMCJ@buttonSelectSelected?$AA@ 10024b0c     manage_temp.obj
 0002:00006b24       ??_C@_0BH@LCBHGILP@buttonUnselectSelected?$AA@ 10024b24     manage_temp.obj
 0002:00006b3c       ??_C@_09DMINLBG@1accept?$CI?$CJ?$AA@ 10024b3c     manage_temp.obj
 0002:00006b48       ??_C@_09OCDCAEKE@1reject?$CI?$CJ?$AA@ 10024b48     manage_temp.obj
 0002:00006b54       ??_C@_0BB@GBAJKNMD@Manage?5Templates?$AA@ 10024b54     manage_temp.obj
 0002:00006b68       ??_C@_08NLCKCAFE@Template?$AA@ 10024b68     manage_temp.obj
 0002:00006b74       ??_C@_03ILBCOJBH@New?$AA@  10024b74     manage_temp.obj
 0002:00006b78       ??_C@_03DDKJIMDC@?$CGOK?$AA@ 10024b78     manage_temp.obj
 0002:00006b7c       ??_C@_05HBFPNANJ@Alt?$CLO?$AA@ 10024b7c     manage_temp.obj
 0002:00006b84       ??_C@_0BE@MBBKLJIA@Prefix?5for?5Template?$AA@ 10024b84     manage_temp.obj
 0002:00006b98       ??_C@_09DHEEOILL@Base?5Slot?$AA@ 10024b98     manage_temp.obj
 0002:00006ba4       ??_C@_06GEMKPBPA@Offset?$AA@ 10024ba4     manage_temp.obj
 0002:00006bac       ??_C@_0M@MJNEDJOC@Auto?5Number?$AA@ 10024bac     manage_temp.obj
 0002:00006bb8       ??_C@_0M@CGHAEADE@Clear?5Slots?$AA@ 10024bb8     manage_temp.obj
 0002:00006bc4       ??_C@_0O@PIILMNHI@Configuration?$AA@ 10024bc4     manage_temp.obj
 0002:00006bd4       ??_C@_0L@CALHPJHB@Select?5All?$AA@ 10024bd4     manage_temp.obj
 0002:00006be0       ??_C@_0N@BHBOLKLM@Unselect?5All?$AA@ 10024be0     manage_temp.obj
 0002:00006bf0       ??_C@_0BA@NKELCOGO@Select?5Selected?$AA@ 10024bf0     manage_temp.obj
 0002:00006c00       ??_C@_0BC@EMBDDAM@Unselect?5Selected?$AA@ 10024c00     manage_temp.obj
 0002:00006c1c       ??_SQCheckTableItem@@6B@   10024c1c     manage_tempimpl.obj
 0002:00006c6c       ??_7manage_temp@@6BQObject@@@ 10024c6c     manage_tempimpl.obj
 0002:00006e30       ??_7manage_temp@@6BQPaintDevice@@@ 10024e30     manage_tempimpl.obj
 0002:00006e50       ??_C@_07EHMCOPMF@PosSize?$AA@ 10024e50     manage_tempimpl.obj
 0002:00006e58       ??_C@_0DB@EMEFP@Home?1Alarms?1Outputs?1Bncs?5Output?1@ 10024e58     manage_tempimpl.obj
 0002:00006e8c       ??_C@_09LALMMIOK@ListSlots?$AA@ 10024e8c     manage_tempimpl.obj
 0002:00006e98       ??_C@_0O@LNDMEONL@TableInstance?$AA@ 10024e98     manage_tempimpl.obj
 0002:00006ea8       ??_C@_0DE@GMIMNEPP@2itemRenamed?$CIQListViewItem?5?$CK?0?5in@ 10024ea8     manage_tempimpl.obj
 0002:00006edc       ??_C@_0CB@PDIPNFDF@1selectTemplate?$CIconst?5QString?5?$CG?$CJ@ 10024edc     manage_tempimpl.obj
 0002:00006f00       ??_C@_0BL@PBFONBLG@2activated?$CIconst?5QString?$CG?$CJ?$AA@ 10024f00     manage_tempimpl.obj
 0002:00006f1c       ??_C@_0BP@EHIPOOKP@1changePrefix?$CIconst?5QString?5?$CG?$CJ?$AA@ 10024f1c     manage_tempimpl.obj
 0002:00006f3c       ??_C@_0BN@HELOKIBG@2textChanged?$CIconst?5QString?$CG?$CJ?$AA@ 10024f3c     manage_tempimpl.obj
 0002:00006f5c       ??_C@_0P@FKOBPIKM@1newTemplate?$CI?$CJ?$AA@ 10024f5c     manage_tempimpl.obj
 0002:00006f6c       ??_C@_0BG@NIEHCODN@1selectAllInstances?$CI?$CJ?$AA@ 10024f6c     manage_tempimpl.obj
 0002:00006f84       ??_C@_0BI@PBGGBIPI@1unselectAllInstances?$CI?$CJ?$AA@ 10024f84     manage_tempimpl.obj
 0002:00006f9c       ??_C@_0BL@JEPDDKNC@1selectSelectedInstances?$CI?$CJ?$AA@ 10024f9c     manage_tempimpl.obj
 0002:00006fb8       ??_C@_0BN@BNIPEJDI@1unselectSelectedInstances?$CI?$CJ?$AA@ 10024fb8     manage_tempimpl.obj
 0002:00006fd8       ??_C@_0BF@KEHKIODN@1changeTab?$CIQWidget?$CK?$CJ?$AA@ 10024fd8     manage_tempimpl.obj
 0002:00006ff0       ??_C@_0BK@EHJILHMI@2currentChanged?$CIQWidget?$CK?$CJ?$AA@ 10024ff0     manage_tempimpl.obj
 0002:0000700c       ??_C@_0BD@FBELHLBD@1autoNumberSlots?$CI?$CJ?$AA@ 1002500c     manage_tempimpl.obj
 0002:00007020       ??_C@_0DH@BLOCANNO@manage_temp?3?3selectTemplate?5?9?5ca@ 10025020     manage_tempimpl.obj
 0002:00007058       ??_C@_0EM@BODNBDBD@manage_temp?3?3selectTemplate?5?9?5di@ 10025058     manage_tempimpl.obj
 0002:000070a4       ??_C@_0CG@FJBOBHMI@currentTemplate?5?9?5no?5current?5tem@ 100250a4     manage_tempimpl.obj
 0002:000070cc       ??_C@_0CD@OBIHLPGN@currentTemplate?5?9?5no?5instances?5s@ 100250cc     manage_tempimpl.obj
 0002:000070f0       ??_C@_08KLEPBNHL@Selected?$AA@ 100250f0     manage_tempimpl.obj
 0002:000070fc       ??_C@_0BI@PCEJKEHM@Enter?5new?5template?5name?$AA@ 100250fc     manage_tempimpl.obj
 0002:00007114       ??_C@_0N@FNIJLANL@New?5Template?$AA@ 10025114     manage_tempimpl.obj
 0002:00007124       ??_C@_0BC@DGKPKLHE@?8?5already?5exists?4?$AA@ 10025124     manage_tempimpl.obj
 0002:00007138       ??_C@_0BF@PNIBPIJJ@The?5specified?5name?5?8?$AA@ 10025138     manage_tempimpl.obj
 0002:00007150       ??_C@_0BE@IBMFEFFD@New?5Template?5Failed?$AA@ 10025150     manage_tempimpl.obj
 0002:00007164       ??_C@_0CG@PKIFDLEK@Please?5select?5rows?5for?5auto?5numb@ 10025164     manage_tempimpl.obj
 0002:0000718c       ??_C@_0BD@BMBHMFKK@No?5row?5is?5selected?$AA@ 1002518c     manage_tempimpl.obj
 0002:000071a0       ??_C@_0BM@LALOLANA@Please?5select?5rows?5to?5clear?$AA@ 100251a0     manage_tempimpl.obj
 0002:000071c8       ??_C@_0P@DMEOIADN@languageChange?$AA@ 100251c8     moc_manage_temp.obj
 0002:000071e4       ??_C@_0BB@PFEIHPGD@languageChange?$CI?$CJ?$AA@ 100251e4     moc_manage_temp.obj
 0002:000071f8       ??_C@_0M@LGFJKMND@manage_temp?$AA@ 100251f8     moc_manage_tempimpl.obj
 0002:00007210       ??_C@_05JLNEMJLN@dummy?$AA@ 10025210     moc_manage_tempimpl.obj
 0002:00007224       ??_C@_0BD@KFHHNDDN@selectAllInstances?$AA@ 10025224     moc_manage_tempimpl.obj
 0002:00007244       ??_C@_0BF@KNGJJJED@unselectAllInstances?$AA@ 10025244     moc_manage_tempimpl.obj
 0002:00007268       ??_C@_0BI@OBIGJEML@selectSelectedInstances?$AA@ 10025268     moc_manage_tempimpl.obj
 0002:0000728c       ??_C@_0BK@INKMHGEO@unselectSelectedInstances?$AA@ 1002528c     moc_manage_tempimpl.obj
 0002:000072b4       ??_C@_0M@LCIDOJBI@newTemplate?$AA@ 100252b4     moc_manage_tempimpl.obj
 0002:000072c0       ??_C@_07FNEPBGL@QWidget?$AA@ 100252c0     moc_manage_tempimpl.obj
 0002:000072d4       ??_C@_09BIEEGLMD@changeTab?$AA@ 100252d4     moc_manage_tempimpl.obj
 0002:000072ec       ??_C@_0BE@JJCLGC@saveCurrentTemplate?$AA@ 100252ec     moc_manage_tempimpl.obj
 0002:00007300       ??_C@_0O@LAFKAPIP@QListViewItem?$AA@ 10025300     moc_manage_tempimpl.obj
 0002:0000731c       ??_C@_0BC@MMJHIHLO@itemDoubleClicked?$AA@ 1002531c     moc_manage_tempimpl.obj
 0002:0000733c       ??_C@_0L@CIFODBFJ@slotChange?$AA@ 1002533c     moc_manage_tempimpl.obj
 0002:00007348       ??_C@_07DCECKACL@sPrefix?$AA@ 10025348     moc_manage_tempimpl.obj
 0002:0000735c       ??_C@_0N@BJNBDMFM@changePrefix?$AA@ 1002535c     moc_manage_tempimpl.obj
 0002:0000736c       ??_C@_09MDNHGCBH@sTemplate?$AA@ 1002536c     moc_manage_tempimpl.obj
 0002:00007384       ??_C@_0P@OHIDMLOK@selectTemplate?$AA@ 10025384     moc_manage_tempimpl.obj
 0002:000073a0       ??_C@_0BA@GKNGMBDH@autoNumberSlots?$AA@ 100253a0     moc_manage_tempimpl.obj
 0002:000073bc       ??_C@_0L@FKABCOB@clearSlots?$AA@ 100253bc     moc_manage_tempimpl.obj
 0002:000073c8       ??_C@_0P@JKIOBDBA@pDictTemplates?$AA@ 100253c8     moc_manage_tempimpl.obj
 0002:000073d8       ??_C@_0BD@NLDKFICJ@TemplateList?$CKconst?$AA@ 100253d8     moc_manage_tempimpl.obj
 0002:000073f8       ??_C@_0N@JLLFNGD@getTemplates?$AA@ 100253f8     moc_manage_tempimpl.obj
 0002:000074bc       ??_C@_07MBMLLJIG@dummy?$CI?$CJ?$AA@ 100254bc     moc_manage_tempimpl.obj
 0002:000074c4       ??_C@_0BF@HCKOGBE@selectAllInstances?$CI?$CJ?$AA@ 100254c4     moc_manage_tempimpl.obj
 0002:000074dc       ??_C@_0BH@CAJPBCPM@unselectAllInstances?$CI?$CJ?$AA@ 100254dc     moc_manage_tempimpl.obj
 0002:000074f4       ??_C@_0BK@KNHEDAON@selectSelectedInstances?$CI?$CJ?$AA@ 100254f4     moc_manage_tempimpl.obj
 0002:00007510       ??_C@_0BM@KFIELDJN@unselectSelectedInstances?$CI?$CJ?$AA@ 10025510     moc_manage_tempimpl.obj
 0002:0000752c       ??_C@_0O@CJNFPILF@newTemplate?$CI?$CJ?$AA@ 1002552c     moc_manage_tempimpl.obj
 0002:0000753c       ??_C@_0BE@KJFNGEJB@changeTab?$CIQWidget?$CK?$CJ?$AA@ 1002553c     moc_manage_tempimpl.obj
 0002:00007550       ??_C@_0BG@IJGPHIEP@saveCurrentTemplate?$CI?$CJ?$AA@ 10025550     moc_manage_tempimpl.obj
 0002:00007568       ??_C@_0CC@NJHPGJEI@itemDoubleClicked?$CIQListViewItem?$CK@ 10025568     moc_manage_tempimpl.obj
 0002:0000758c       ??_C@_0CO@BMLEEMKN@slotChange?$CIQListViewItem?$CK?0int?0co@ 1002558c     moc_manage_tempimpl.obj
 0002:000075bc       ??_C@_0BN@FKICHEGC@changePrefix?$CIconst?5QString?$CG?$CJ?$AA@ 100255bc     moc_manage_tempimpl.obj
 0002:000075dc       ??_C@_0BP@FBDBMKIP@selectTemplate?$CIconst?5QString?$CG?$CJ?$AA@ 100255dc     moc_manage_tempimpl.obj
 0002:000075fc       ??_C@_0BC@OHMLAHH@autoNumberSlots?$CI?$CJ?$AA@ 100255fc     moc_manage_tempimpl.obj
 0002:00007610       ??_C@_0N@MGMEDOPG@clearSlots?$CI?$CJ?$AA@ 10025610     moc_manage_tempimpl.obj
 0002:00007620       ??_C@_0CB@OMBMHKND@getTemplates?$CITemplateList?$CKconst?$CJ@ 10025620     moc_manage_tempimpl.obj
 0002:00007644       ??_C@_0CD@BFGBAEB@?5?5?5?514?5?5?5?514?5?5?5?5?5?5?5?54?5?5?5?5?5?5?5?5?5?5?5@ 10025644     plugindesc.obj
 0002:00007668       ??_C@_0M@EKMPMHDK@?4?5c?5?$CD040404?$AA@ 10025668     plugindesc.obj
 0002:00007674       ??_C@_0M@NBLJLJNN@?$CD?5c?5?$CD808304?$AA@ 10025674     plugindesc.obj
 0002:00007680       ??_C@_0M@EAFJJBBG@a?5c?5?$CDbfc2bf?$AA@ 10025680     plugindesc.obj
 0002:0000768c       ??_C@_08PBKCALNO@b?5c?5None?$AA@ 1002568c     plugindesc.obj
 0002:00007698       ??_C@_0P@HFKAALMG@?4?4?4?4?4?4?4?4?4?4?4?4?4?4?$AA@ 10025698     plugindesc.obj
 0002:000076a8       ??_C@_0P@LGBCEGMD@?4?$CD?4aaaaaaaa?4a?4?$AA@ 100256a8     plugindesc.obj
 0002:000076b8       ??_C@_0P@MNNEIMDO@?4?$CD?4aaaaaaaa?4?4?4?$AA@ 100256b8     plugindesc.obj
 0002:000076c8       ??_C@_0P@MFAMBPGN@?4?$CD?4aaaaaaaa?4?$CD?4?$AA@ 100256c8     plugindesc.obj
 0002:000076d8       ??_C@_0P@HPMEFAGN@?4?$CD?$CD?4?4?4?4?4?4?4?4?$CD?$CD?4?$AA@ 100256d8     plugindesc.obj
 0002:000076e8       ??_C@_0P@JAJCNDBN@?4?$CD?$CD?$CD?$CD?$CD?$CD?$CD?$CD?$CD?$CD?$CD?$CD?4?$AA@ 100256e8     plugindesc.obj
 0002:000076f8       ??_C@_0P@INKOIILA@?4?$CD?$CD?4?4?4?4?4?4?4?4?4?$CD?4?$AA@ 100256f8     plugindesc.obj
 0002:00007708       ??_C@_0P@KJADPPJB@?4?$CD?$CD?4?4?4?4?4?4aa?4?$CD?4?$AA@ 10025708     plugindesc.obj
 0002:00007718       ??_C@_0P@PKKONJFP@b?4?4?4?4?4?4?4?4?4?4?4?4?4?$AA@ 10025718     plugindesc.obj
 0002:0000772c       ??_7config_plugin_desc_base@@6B@ 1002572c     plugindesc.obj
 0002:00007740       ??_7plugindesc@@6B@        10025740     plugindesc.obj
 0002:00007750       ??_C@_0CA@PMNCLLKE@Home?1Alarms?1Outputs?1Bncs?5Output?$AA@ 10025750     plugindesc.obj
 0002:00007774       ??_7processItem@@6B@       10025774     processItem.obj
 0002:0000780c       ??_C@_07GFDMEDFB@darkRed?$AA@ 1002580c     processItem.obj
 0002:00007814       ??_C@_06ENJNJKEL@yellow?$AA@ 10025814     processItem.obj
 0002:0000781c       ??_C@_03FAAAOPJM@red?$AA@  1002581c     processItem.obj
 0002:00007824       ??_7autoNumberDialogBase@@6BQObject@@@ 10025824     autonumberdialog.obj
 0002:000079e8       ??_7autoNumberDialogBase@@6BQPaintDevice@@@ 100259e8     autonumberdialog.obj
 0002:00007a0c       ??_SQGroupBox@@6BQObject@@@ 10025a0c     autonumberdialog.obj
 0002:00007bec       ??_SQGroupBox@@6BQPaintDevice@@@ 10025bec     autonumberdialog.obj
 0002:00007c14       ??_SQButtonGroup@@6BQObject@@@ 10025c14     autonumberdialog.obj
 0002:00007e04       ??_SQButtonGroup@@6BQPaintDevice@@@ 10025e04     autonumberdialog.obj
 0002:00007e2c       ??_SQRadioButton@@6BQObject@@@ 10025e2c     autonumberdialog.obj
 0002:00008010       ??_SQRadioButton@@6BQPaintDevice@@@ 10026010     autonumberdialog.obj
 0002:00008030       ??_C@_0BF@JHIFNHKG@autoNumberDialogBase?$AA@ 10026030     autonumberdialog.obj
 0002:00008048       ??_C@_0BL@BIKGAJJG@autoNumberDialogBaseLayout?$AA@ 10026048     autonumberdialog.obj
 0002:00008064       ??_C@_0M@OCBOJOPI@selectGroup?$AA@ 10026064     autonumberdialog.obj
 0002:00008070       ??_C@_08DLKPFPGI@radioAll?$AA@ 10026070     autonumberdialog.obj
 0002:0000807c       ??_C@_0O@GELIKEBG@radioSelected?$AA@ 1002607c     autonumberdialog.obj
 0002:0000808c       ??_C@_0L@LALBKBIN@comboGroup?$AA@ 1002608c     autonumberdialog.obj
 0002:00008098       ??_C@_0L@DAMJCADI@radioGroup?$AA@ 10026098     autonumberdialog.obj
 0002:000080a4       ??_C@_09LLEGKCGM@groupBox2?$AA@ 100260a4     autonumberdialog.obj
 0002:000080b0       ??_C@_0BC@DLEJKFKG@1setEnabled?$CIbool?$CJ?$AA@ 100260b0     autonumberdialog.obj
 0002:000080c4       ??_C@_0P@POCECEMJ@2toggled?$CIbool?$CJ?$AA@ 100260c4     autonumberdialog.obj
 0002:000080d4       ??_C@_0BG@HJJECPBH@Auto?9Number?5Selection?$AA@ 100260d4     autonumberdialog.obj
 0002:000080ec       ??_C@_0P@HINHMFAJ@Select?5Process?$AA@ 100260ec     autonumberdialog.obj
 0002:000080fc       ??_C@_03HFJGAJFE@All?$AA@  100260fc     autonumberdialog.obj
 0002:00008100       ??_C@_0N@JEHMJEOF@Select?5Group?$AA@ 10026100     autonumberdialog.obj
 0002:00008110       ??_C@_09IEAFEACD@Numbering?$AA@ 10026110     autonumberdialog.obj
 0002:0000811c       ??_C@_04NGEJNKEG@Base?$AA@ 1002611c     autonumberdialog.obj
 0002:00008124       ??_C@_0CC@MEDMAJJI@Group?5Offset?5?9?5sort?5by?5group?5onl@ 10026124     autonumberdialog.obj
 0002:00008148       ??_C@_05NNOKJPNF@Alt?$CLC?$AA@ 10026148     autonumberdialog.obj
 0002:00008154       ??_7dialogBase@@6BQObject@@@ 10026154     dialog.obj
 0002:0000830c       ??_7dialogBase@@6BQPaintDevice@@@ 1002630c     dialog.obj
 0002:0000832c       ??_C@_0L@BCEAHFEK@dialogBase?$AA@ 1002632c     dialog.obj
 0002:00008338       ??_C@_0BB@NFKKNJMG@dialogBaseLayout?$AA@ 10026338     dialog.obj
 0002:0000834c       ??_C@_08JLKJJNLG@topLabel?$AA@ 1002634c     dialog.obj
 0002:00008358       ??_C@_08BADCPAJD@layout10?$AA@ 10026358     dialog.obj
 0002:00008364       ??_C@_08DCHHJIKL@procList?$AA@ 10026364     dialog.obj
 0002:00008370       ??_C@_08BNEIIGAN@Dev?5Type?$AA@ 10026370     dialog.obj
 0002:0000837c       ??_C@_0BA@NDAKFEOI@Infodriver?5Slot?$AA@ 1002637c     dialog.obj
 0002:0000838c       ??_C@_07GIKHDDO@layout9?$AA@ 1002638c     dialog.obj
 0002:00008394       ??_C@_08DLBPKDFA@layout13?$AA@ 10026394     dialog.obj
 0002:000083a0       ??_C@_0BB@EFDKKACJ@infodriverNumber?$AA@ 100263a0     dialog.obj
 0002:000083b4       ??_C@_0M@PJOMGFDC@statusLabel?$AA@ 100263b4     dialog.obj
 0002:000083c0       ??_C@_07JIAJFOLA@layout7?$AA@ 100263c0     dialog.obj
 0002:000083c8       ??_C@_08NHBDLPIJ@upButton?$AA@ 100263c8     dialog.obj
 0002:000083d4       ??_C@_0L@NNLLKLBD@downButton?$AA@ 100263d4     dialog.obj
 0002:000083e0       ??_C@_07BPJBECHP@layout8?$AA@ 100263e0     dialog.obj
 0002:000083e8       ??_C@_09OCIGHHLO@layout7_2?$AA@ 100263e8     dialog.obj
 0002:000083f4       ??_C@_07GAFHPDDI@manTemp?$AA@ 100263f4     dialog.obj
 0002:000083fc       ??_C@_07EKLPEACL@autoNum?$AA@ 100263fc     dialog.obj
 0002:00008404       ??_C@_0BB@FEBJJEPJ@clearSlotsButton?$AA@ 10026404     dialog.obj
 0002:00008418       ??_C@_09CIDKMNDE@navToProc?$AA@ 10026418     dialog.obj
 0002:00008424       ??_C@_06IOAEHBNO@dialog?$AA@ 10026424     dialog.obj
 0002:0000842c       ??_C@_0BL@PFIBKMLM@?$DMh1?$DOAlarm?5BNCS?5Output?$DM?1h1?$DO?$AA@ 1002642c     dialog.obj
 0002:00008448       ??_C@_0BH@NGLJDKBH@Selected?5Output?5Module?$AA@ 10026448     dialog.obj
 0002:00008460       ??_C@_0N@OAECLGMI@Process?5List?$AA@ 10026460     dialog.obj
 0002:00008470       ??_C@_0BGM@NLPNFPNH@?$DMh3?$DOProcess?5List?$DM?1h3?$DO?6This?5displ@ 10026470     dialog.obj
 0002:000085dc       ??_C@_0BC@IENGNIMC@Infodriver?5Number?$AA@ 100265dc     dialog.obj
 0002:000085f0       ??_C@_0BC@ELGLOBFO@Infodriver?5number?$AA@ 100265f0     dialog.obj
 0002:00008608       ??_C@_0GE@GNDPFJEM@This?5is?5the?5infodriver?5device?5nu@ 10026608     dialog.obj
 0002:0000866c       ??_C@_06PGDKHFME@Status?$AA@ 1002666c     dialog.obj
 0002:00008674       ??_C@_07DMGIOHNE@Move?5Up?$AA@ 10026674     dialog.obj
 0002:0000867c       ??_C@_0BC@BOLNCOLB@Manually?5re?9order?$AA@ 1002667c     dialog.obj
 0002:00008690       ??_C@_0EE@CLMPNPHE@Move?5the?5current?5process?5up?1down@ 10026690     dialog.obj
 0002:000086d4       ??_C@_09CEAAIKKP@Move?5Down?$AA@ 100266d4     dialog.obj
 0002:000086e0       ??_C@_0CB@PNIKNLBA@Auto?5number?5the?5infodriver?5slots@ 100266e0     dialog.obj
 0002:00008708       ??_C@_0NL@IFOLNNMA@Allows?5rapid?5numbering?5of?5the?5in@ 10026708     dialog.obj
 0002:000087e4       ??_C@_0BA@CMLLBBFE@Clear?5the?5slots?$AA@ 100267e4     dialog.obj
 0002:000087f8       ??_C@_0FF@IBGBGPHA@Clears?5either?5the?5selected?5slots@ 100267f8     dialog.obj
 0002:00008850       ??_C@_0BC@NOIFPMEL@Copy?5to?5Clipboard?$AA@ 10026850     dialog.obj
 0002:00008868       ??_C@_0FG@OPDLLDBN@Copy?5the?5selection?5to?5the?5clipbo@ 10026868     dialog.obj
 0002:000088c0       ??_C@_0BF@NHKAGICB@Paste?5from?5Clipboard?$AA@ 100268c0     dialog.obj
 0002:000088d8       ??_C@_0BF@JIPNGLPB@Paste?5from?5clipboard?$AA@ 100268d8     dialog.obj
 0002:000088f0       ??_C@_0EB@DPGIDEKC@Paste?5the?5clipboard?0?5from?5extern@ 100268f0     dialog.obj
 0002:00008934       ??_C@_0N@HKALLKJF@Edit?5Process?$AA@ 10026934     dialog.obj
 0002:00008944       ??_C@_0BJ@KFCMIOCB@Edit?5the?5current?5process?$AA@ 10026944     dialog.obj
 0002:00008960       ??_C@_0DH@MEBFNGED@Go?5to?5the?5process?5editor?5and?5edi@ 10026960     dialog.obj
 0002:00008998       ??_C@_0BA@HHFNOHIJ@alm_bncs_output?$AA@ 10026998     moc_alm_bncs_output.obj
 0002:000089c0       ??_C@_0P@FPPPOCFM@applyTemplates?$AA@ 100269c0     moc_alm_bncs_output.obj
 0002:000089dc       ??_C@_0P@EMNBNEKL@manageTemplate?$AA@ 100269dc     moc_alm_bncs_output.obj
 0002:000089f8       ??_C@_05BEELFHJC@about?$AA@ 100269f8     moc_alm_bncs_output.obj
 0002:00008a0c       ??_C@_07OECBGGNC@isDirty?$AA@ 10026a0c     moc_alm_bncs_output.obj
 0002:00008a20       ??_C@_05KAEIDCAL@apply?$AA@ 10026a20     moc_alm_bncs_output.obj
 0002:00008a34       ??_C@_09HIGIDEDO@markDirty?$AA@ 10026a34     moc_alm_bncs_output.obj
 0002:00008a4c       ??_C@_0P@CNFJKBJI@menuDeleteFile?$AA@ 10026a4c     moc_alm_bncs_output.obj
 0002:00008a68       ??_C@_0BC@HKAEEBBP@menuDuplicateFile?$AA@ 10026a68     moc_alm_bncs_output.obj
 0002:00008a88       ??_C@_0L@FJIJGHHG@menuRename?$AA@ 10026a88     moc_alm_bncs_output.obj
 0002:00008aa0       ??_C@_0M@FNCKOKHH@menuNewFile?$AA@ 10026aa0     moc_alm_bncs_output.obj
 0002:00008ab8       ??_C@_0M@BLOGNIHC@EditProcess?$AA@ 10026ab8     moc_alm_bncs_output.obj
 0002:00008ac4       ??_C@_04NHONDGDE@item?$AA@ 10026ac4     moc_alm_bncs_output.obj
 0002:00008acc       ??_C@_03HNOLNALI@col?$AA@  10026acc     moc_alm_bncs_output.obj
 0002:00008ad0       ??_C@_04CIMGMMMG@text?$AA@ 10026ad0     moc_alm_bncs_output.obj
 0002:00008ae4       ??_C@_0N@CGBIPEEF@renameModule?$AA@ 10026ae4     moc_alm_bncs_output.obj
 0002:00008b00       ??_C@_0L@EBNMIND@selectFile?$AA@ 10026b00     moc_alm_bncs_output.obj
 0002:00008b0c       ??_C@_03PCBNCGFH@pos?$AA@  10026b0c     moc_alm_bncs_output.obj
 0002:00008b10       ??_C@_01CAKFMAIO@?$AO?$AA@ 10026b10     moc_alm_bncs_output.obj
 0002:00008b20       ??_C@_0BE@EOPNNNEB@fileListContextMenu?$AA@ 10026b20     moc_alm_bncs_output.obj
 0002:00008b40       ??_C@_06HDBGBMEK@dummy1?$AA@ 10026b40     moc_alm_bncs_output.obj
 0002:00008b48       ??_C@_07ECHCKIDD@sSystem?$AA@ 10026b48     moc_alm_bncs_output.obj
 0002:00008b5c       ??_C@_0N@JNMAEFDJ@selectSystem?$AA@ 10026b5c     moc_alm_bncs_output.obj
 0002:00008c3c       ??_C@_0BB@CKBCEGEA@applyTemplates?$CI?$CJ?$AA@ 10026c3c     moc_alm_bncs_output.obj
 0002:00008c50       ??_C@_0BB@LOFFLHIN@manageTemplate?$CI?$CJ?$AA@ 10026c50     moc_alm_bncs_output.obj
 0002:00008c64       ??_C@_07MEGALADH@about?$CI?$CJ?$AA@ 10026c64     moc_alm_bncs_output.obj
 0002:00008c6c       ??_C@_09GFMHAPGC@isDirty?$CI?$CJ?$AA@ 10026c6c     moc_alm_bncs_output.obj
 0002:00008c78       ??_C@_07FJDLKALA@apply?$CI?$CJ?$AA@ 10026c78     moc_alm_bncs_output.obj
 0002:00008c80       ??_C@_0M@BCGJBPBD@markDirty?$CI?$CJ?$AA@ 10026c80     moc_alm_bncs_output.obj
 0002:00008c8c       ??_C@_0BB@GKFBDGIG@menuDeleteFile?$CI?$CJ?$AA@ 10026c8c     moc_alm_bncs_output.obj
 0002:00008ca0       ??_C@_0BE@LOJJINCP@menuDuplicateFile?$CI?$CJ?$AA@ 10026ca0     moc_alm_bncs_output.obj
 0002:00008cb4       ??_C@_0N@NIKLPLLB@menuRename?$CI?$CJ?$AA@ 10026cb4     moc_alm_bncs_output.obj
 0002:00008cc4       ??_C@_0O@FCLJDBMO@menuNewFile?$CI?$CJ?$AA@ 10026cc4     moc_alm_bncs_output.obj
 0002:00008cd4       ??_C@_0O@OHBJNCMH@EditProcess?$CI?$CJ?$AA@ 10026cd4     moc_alm_bncs_output.obj
 0002:00008ce4       ??_C@_0DA@KLJABHB@renameModule?$CIQListViewItem?$CK?0int?0@ 10026ce4     moc_alm_bncs_output.obj
 0002:00008d14       ??_C@_0BL@GBKHEMNO@selectFile?$CIQListViewItem?$CK?$CJ?$AA@ 10026d14     moc_alm_bncs_output.obj
 0002:00008d30       ??_C@_0DG@IBBHMLFJ@fileListContextMenu?$CIQListViewIte@ 10026d30     moc_alm_bncs_output.obj
 0002:00008d68       ??_C@_08GMIPAAGF@dummy1?$CI?$CJ?$AA@ 10026d68     moc_alm_bncs_output.obj
 0002:00008d74       ??_C@_0BN@PCNKHLKL@selectSystem?$CIconst?5QString?$CG?$CJ?$AA@ 10026d74     moc_alm_bncs_output.obj
 0002:00008da0       ??_C@_07KMMNMMFF@command?$AA@ 10026da0     moc_alm_bncs_output.obj
 0002:00008db4       ??_C@_0BJ@FEFNJDLM@command?$CIQString?0QString?$CJ?$AA@ 10026db4     moc_alm_bncs_output.obj
 0002:00008dd0       ??_C@_07JNGGNNFK@IDomDoc?$AA@ 10026dd0     moc_alm_bncs_output.obj
 0002:00008dd8       ??_C@_0O@GCELBMFI@IGetDocuments?$AA@ 10026dd8     moc_alm_bncs_output.obj
 0002:00008de8       ??_C@_0N@KBDCPKEG@ISendCommand?$AA@ 10026de8     moc_alm_bncs_output.obj
 0002:00008e10       ??_C@_0BB@FPHOCGFI@autoNumberDialog?$AA@ 10026e10     moc_autonumberdialogimpl.obj
 0002:00008e54       ??_C@_0O@HJGKCBPC@clearAllSlots?$AA@ 10026e54     moc_dialogimpl.obj
 0002:00008e7c       ??_C@_0BF@HDAPLING@clearSelectableSlots?$AA@ 10026e7c     moc_dialogimpl.obj
 0002:00008ea0       ??_C@_0BD@HONAMNHE@clearSelectedSlots?$AA@ 10026ea0     moc_dialogimpl.obj
 0002:00008eb4       ??_C@_04KOJNECLL@iCol?$AA@ 10026eb4     moc_dialogimpl.obj
 0002:00008ec8       ??_C@_06EBINCNOI@reSort?$AA@ 10026ec8     moc_dialogimpl.obj
 0002:00008edc       ??_C@_0BA@HAAAGFKH@changeSelection?$AA@ 10026edc     moc_dialogimpl.obj
 0002:00008ef8       ??_C@_0L@CGOALGPA@moveProcUp?$AA@ 10026ef8     moc_dialogimpl.obj
 0002:00008f10       ??_C@_0N@MJIEBAOD@moveProcDown?$AA@ 10026f10     moc_dialogimpl.obj
 0002:00008f2c       ??_C@_0M@PGFFFNDC@itemChanged?$AA@ 10026f2c     moc_dialogimpl.obj
 0002:00008f38       ??_C@_06ICGJLFIM@string?$AA@ 10026f38     moc_dialogimpl.obj
 0002:00008f58       ??_C@_0L@FNIFGFGE@autoNumber?$AA@ 10026f58     moc_dialogimpl.obj
 0002:00008f70       ??_C@_0BE@JKIANKML@clipboardDataChange?$AA@ 10026f70     moc_dialogimpl.obj
 0002:00008f90       ??_C@_09MCBCIPNB@pasteData?$AA@ 10026f90     moc_dialogimpl.obj
 0002:00008fa8       ??_C@_08LEGBJMIA@copyData?$AA@ 10026fa8     moc_dialogimpl.obj
 0002:00008fc0       ??_C@_0L@DILJGDLA@selectProc?$AA@ 10026fc0     moc_dialogimpl.obj
 0002:00008ff0       ??_C@_0BD@NFGPONGO@checkForDuplicates?$AA@ 10026ff0     moc_dialogimpl.obj
 0002:000090ec       ??_C@_0BA@BIPLGCLI@clearAllSlots?$CI?$CJ?$AA@ 100270ec     moc_dialogimpl.obj
 0002:000090fc       ??_C@_0BH@GAMAKCJL@clearSelectableSlots?$CI?$CJ?$AA@ 100270fc     moc_dialogimpl.obj
 0002:00009114       ??_C@_0BF@NMJOPEJM@clearSelectedSlots?$CI?$CJ?$AA@ 10027114     moc_dialogimpl.obj
 0002:0000912c       ??_C@_0M@PJOJEAFK@reSort?$CIint?$CJ?$AA@ 1002712c     moc_dialogimpl.obj
 0002:00009138       ??_C@_0BC@KOIGEHEK@changeSelection?$CI?$CJ?$AA@ 10027138     moc_dialogimpl.obj
 0002:0000914c       ??_C@_0N@EEKGFJFH@moveProcUp?$CI?$CJ?$AA@ 1002714c     moc_dialogimpl.obj
 0002:0000915c       ??_C@_0P@BKPMPBHM@moveProcDown?$CI?$CJ?$AA@ 1002715c     moc_dialogimpl.obj
 0002:0000916c       ??_C@_0O@IKLCAHNO@itemChanged?$CI?$CJ?$AA@ 1002716c     moc_dialogimpl.obj
 0002:0000917c       ??_C@_0BM@KLLCNLMA@itemChanged?$CIconst?5QString?$CG?$CJ?$AA@ 1002717c     moc_dialogimpl.obj
 0002:00009198       ??_C@_0N@EOFBOOEC@autoNumber?$CI?$CJ?$AA@ 10027198     moc_dialogimpl.obj
 0002:000091a8       ??_C@_0BG@DMBACHHM@clipboardDataChange?$CI?$CJ?$AA@ 100271a8     moc_dialogimpl.obj
 0002:000091c0       ??_C@_0M@JHDMCAEO@pasteData?$CI?$CJ?$AA@ 100271c0     moc_dialogimpl.obj
 0002:000091cc       ??_C@_0L@LACCHLPG@copyData?$CI?$CJ?$AA@ 100271cc     moc_dialogimpl.obj
 0002:000091d8       ??_C@_0BL@KDOAFBIF@selectProc?$CIQListViewItem?$CK?$CJ?$AA@ 100271d8     moc_dialogimpl.obj
 0002:000091f4       ??_C@_0BF@FHNNIFDA@checkForDuplicates?$CI?$CJ?$AA@ 100271f4     moc_dialogimpl.obj
 0002:00009218       ??_C@_0N@IBIICDGH@itemsChanged?$AA@ 10027218     moc_dialogimpl.obj
 0002:00009234       ??_C@_0P@PKMDIFCJ@itemsChanged?$CI?$CJ?$AA@ 10027234     moc_dialogimpl.obj
 0002:00009244       ??_C@_0BI@GGLIKMPP@CC_ConfigEdit?1Controls?1?$AA@ 10027244     cfg_widgets001:cfg_Settings.obj
 0002:0000925c       ??_C@_02PIGFKFFE@?$CF1?$AA@ 1002725c     cfg_widgets001:cfg_Settings.obj
 0002:00009260       ??_C@_03MMIELDNM@?0?$CF1?$AA@ 10027260     cfg_widgets001:cfg_Settings.obj
 0002:00009264       ??_C@_0P@JHCMIKMI@?$CF1?0?$CF2?0?$CF3?0?$CF4?0?$CF5?$AA@ 10027264     cfg_widgets001:cfg_Settings.obj
 0002:00009274       ??_C@_04LOAJBDKD@true?$AA@ 10027274     cfg_widgets001:cfg_Settings.obj
 0002:0000927c       ??_C@_05LAPONLG@false?$AA@ 1002727c     cfg_widgets001:cfg_Settings.obj
 0002:00009288       ??_7Document@@6B@          10027288     config_alarm_utilities:Document.obj
 0002:00009290       ??_7Document_BncsSystem@@6B@ 10027290     config_alarm_utilities:Document.obj
 0002:00009294       ??_C@_0BH@EEDFIBDB@system?1bncs_system?4ini?$AA@ 10027294     config_alarm_utilities:Document.obj
 0002:000092ac       ??_C@_02PGHGPEOM@?91?$AA@  100272ac     config_alarm_utilities:Document.obj
 0002:000092b0       ??_C@_0BD@FPEGEEKL@DeviceInfodriverId?$AA@ 100272b0     config_alarm_utilities:Document.obj
 0002:000092c4       ??_C@_0CA@EAAGFFNA@Failed?5to?5read?5Device?5Status?5ID?$AA@ 100272c4     config_alarm_utilities:Document.obj
 0002:000092e8       ??_7FileLoad@@6B@          100272e8     config_alarm_utilities:Loaders.obj
 0002:000092f8       ??_7?$QPtrList@VFileLoad@@@@6B@ 100272f8     config_alarm_utilities:Loaders.obj
 0002:0000931c       ??_7?$QPtrList@VDirLoad@@@@6B@ 1002731c     config_alarm_utilities:Loaders.obj
 0002:00009340       ??_7Loaders@@6B@           10027340     config_alarm_utilities:Loaders.obj
 0002:00009348       ??_7type_info@@6B@         10027348     MSVCRT:ti_inst.obj
 0002:0000934c       __pDefaultRawDllMain       1002734c     MSVCRT:crtdll.obj
 0002:0000934c       __pRawDllMain              1002734c     MSVCRT:crtdll.obj
 0002:00009358       __load_config_used         10027358     MSVCRT:loadcfg.obj
 0002:000093a0       ??_R1A@?0A@EA@QGList@@8    100273a0     alm_bncs_output.obj
 0002:000093bc       ??_R3QGList@@8             100273bc     alm_bncs_output.obj
 0002:000093cc       ??_R2QGList@@8             100273cc     alm_bncs_output.obj
 0002:000093d8       ??_R1A@?0A@EA@QPtrCollection@@8 100273d8     alm_bncs_output.obj
 0002:000093f4       ??_R3QPtrCollection@@8     100273f4     alm_bncs_output.obj
 0002:00009404       ??_R2QPtrCollection@@8     10027404     alm_bncs_output.obj
 0002:0000940c       ??_R4QWidget@@6BQObject@@@ 1002740c     alm_bncs_output.obj
 0002:00009420       ??_R3QWidget@@8            10027420     alm_bncs_output.obj
 0002:00009430       ??_R2QWidget@@8            10027430     alm_bncs_output.obj
 0002:00009444       ??_R1A@?0A@EA@QWidget@@8   10027444     alm_bncs_output.obj
 0002:00009460       ??_R1A@?0A@EA@QObject@@8   10027460     alm_bncs_output.obj
 0002:0000947c       ??_R3QObject@@8            1002747c     alm_bncs_output.obj
 0002:0000948c       ??_R2QObject@@8            1002748c     alm_bncs_output.obj
 0002:00009498       ??_R13?0A@EA@Qt@@8         10027498     alm_bncs_output.obj
 0002:000094b4       ??_R3Qt@@8                 100274b4     alm_bncs_output.obj
 0002:000094c4       ??_R2Qt@@8                 100274c4     alm_bncs_output.obj
 0002:000094cc       ??_R1A@?0A@EA@Qt@@8        100274cc     alm_bncs_output.obj
 0002:000094e8       ??_R1CI@?0A@EA@QPaintDevice@@8 100274e8     alm_bncs_output.obj
 0002:00009504       ??_R3QPaintDevice@@8       10027504     alm_bncs_output.obj
 0002:00009514       ??_R2QPaintDevice@@8       10027514     alm_bncs_output.obj
 0002:0000951c       ??_R1A@?0A@EA@QPaintDevice@@8 1002751c     alm_bncs_output.obj
 0002:00009538       ??_R4QWidget@@6BQPaintDevice@@@ 10027538     alm_bncs_output.obj
 0002:0000954c       ??_R3QShared@@8            1002754c     alm_bncs_output.obj
 0002:0000955c       ??_R2QShared@@8            1002755c     alm_bncs_output.obj
 0002:00009564       ??_R1A@?0A@EA@QShared@@8   10027564     alm_bncs_output.obj
 0002:00009580       ??_R4QPopupMenu@@6BQObject@@@ 10027580     alm_bncs_output.obj
 0002:00009594       ??_R3QPopupMenu@@8         10027594     alm_bncs_output.obj
 0002:000095a4       ??_R2QPopupMenu@@8         100275a4     alm_bncs_output.obj
 0002:000095c4       ??_R1A@?0A@EA@QPopupMenu@@8 100275c4     alm_bncs_output.obj
 0002:000095e0       ??_R1A@?0A@EA@QFrame@@8    100275e0     alm_bncs_output.obj
 0002:000095fc       ??_R3QFrame@@8             100275fc     alm_bncs_output.obj
 0002:0000960c       ??_R2QFrame@@8             1002760c     alm_bncs_output.obj
 0002:00009624       ??_R1IM@?0A@EA@QMenuData@@8 10027624     alm_bncs_output.obj
 0002:00009640       ??_R3QMenuData@@8          10027640     alm_bncs_output.obj
 0002:00009650       ??_R2QMenuData@@8          10027650     alm_bncs_output.obj
 0002:00009658       ??_R1A@?0A@EA@QMenuData@@8 10027658     alm_bncs_output.obj
 0002:00009674       ??_R4QPopupMenu@@6BQPaintDevice@@@ 10027674     alm_bncs_output.obj
 0002:00009688       ??_R4QPopupMenu@@6B@       10027688     alm_bncs_output.obj
 0002:0000969c       ??_R4QAction@@6B@          1002769c     alm_bncs_output.obj
 0002:000096b0       ??_R3QAction@@8            100276b0     alm_bncs_output.obj
 0002:000096c0       ??_R2QAction@@8            100276c0     alm_bncs_output.obj
 0002:000096d0       ??_R1A@?0A@EA@QAction@@8   100276d0     alm_bncs_output.obj
 0002:000096ec       ??_R4QBoxLayout@@6BQObject@@@ 100276ec     alm_bncs_output.obj
 0002:00009700       ??_R3QBoxLayout@@8         10027700     alm_bncs_output.obj
 0002:00009710       ??_R2QBoxLayout@@8         10027710     alm_bncs_output.obj
 0002:00009728       ??_R1A@?0A@EA@QBoxLayout@@8 10027728     alm_bncs_output.obj
 0002:00009744       ??_R1A@?0A@EA@QLayout@@8   10027744     alm_bncs_output.obj
 0002:00009760       ??_R3QLayout@@8            10027760     alm_bncs_output.obj
 0002:00009770       ??_R2QLayout@@8            10027770     alm_bncs_output.obj
 0002:00009784       ??_R1CI@?0A@EA@QLayoutItem@@8 10027784     alm_bncs_output.obj
 0002:000097a0       ??_R3QLayoutItem@@8        100277a0     alm_bncs_output.obj
 0002:000097b0       ??_R2QLayoutItem@@8        100277b0     alm_bncs_output.obj
 0002:000097b8       ??_R1A@?0A@EA@QLayoutItem@@8 100277b8     alm_bncs_output.obj
 0002:000097d4       ??_R4QBoxLayout@@6BQLayoutItem@@@ 100277d4     alm_bncs_output.obj
 0002:000097e8       ??_R4QToolBar@@6BQObject@@@ 100277e8     alm_bncs_output.obj
 0002:000097fc       ??_R3QToolBar@@8           100277fc     alm_bncs_output.obj
 0002:0000980c       ??_R2QToolBar@@8           1002780c     alm_bncs_output.obj
 0002:0000982c       ??_R1A@?0A@EA@QToolBar@@8  1002782c     alm_bncs_output.obj
 0002:00009848       ??_R1A@?0A@EA@QDockWindow@@8 10027848     alm_bncs_output.obj
 0002:00009864       ??_R3QDockWindow@@8        10027864     alm_bncs_output.obj
 0002:00009874       ??_R2QDockWindow@@8        10027874     alm_bncs_output.obj
 0002:00009890       ??_R4QToolBar@@6BQPaintDevice@@@ 10027890     alm_bncs_output.obj
 0002:000098a4       ??_R4QDockWindow@@6BQObject@@@ 100278a4     alm_bncs_output.obj
 0002:000098b8       ??_R4QDockWindow@@6BQPaintDevice@@@ 100278b8     alm_bncs_output.obj
 0002:000098cc       ??_R4QListView@@6BQObject@@@ 100278cc     alm_bncs_output.obj
 0002:000098e0       ??_R3QListView@@8          100278e0     alm_bncs_output.obj
 0002:000098f0       ??_R2QListView@@8          100278f0     alm_bncs_output.obj
 0002:00009910       ??_R1A@?0A@EA@QListView@@8 10027910     alm_bncs_output.obj
 0002:0000992c       ??_R1A@?0A@EA@QScrollView@@8 1002792c     alm_bncs_output.obj
 0002:00009948       ??_R3QScrollView@@8        10027948     alm_bncs_output.obj
 0002:00009958       ??_R2QScrollView@@8        10027958     alm_bncs_output.obj
 0002:00009974       ??_R4QListView@@6BQPaintDevice@@@ 10027974     alm_bncs_output.obj
 0002:00009988       ??_R4QListViewItem@@6B@    10027988     alm_bncs_output.obj
 0002:0000999c       ??_R3QListViewItem@@8      1002799c     alm_bncs_output.obj
 0002:000099ac       ??_R2QListViewItem@@8      100279ac     alm_bncs_output.obj
 0002:000099b8       ??_R1A@?0A@EA@QListViewItem@@8 100279b8     alm_bncs_output.obj
 0002:000099d4       ??_R4QTabWidget@@6BQObject@@@ 100279d4     alm_bncs_output.obj
 0002:000099e8       ??_R3QTabWidget@@8         100279e8     alm_bncs_output.obj
 0002:000099f8       ??_R2QTabWidget@@8         100279f8     alm_bncs_output.obj
 0002:00009a10       ??_R1A@?0A@EA@QTabWidget@@8 10027a10     alm_bncs_output.obj
 0002:00009a2c       ??_R4QTabWidget@@6BQPaintDevice@@@ 10027a2c     alm_bncs_output.obj
 0002:00009a40       ??_R4CAlm_sys_select@@6BQObject@@@ 10027a40     alm_bncs_output.obj
 0002:00009a54       ??_R3CAlm_sys_select@@8    10027a54     alm_bncs_output.obj
 0002:00009a64       ??_R2CAlm_sys_select@@8    10027a64     alm_bncs_output.obj
 0002:00009a88       ??_R1A@?0A@EA@CAlm_sys_select@@8 10027a88     alm_bncs_output.obj
 0002:00009aa4       ??_R1A@?0A@EA@QVBox@@8     10027aa4     alm_bncs_output.obj
 0002:00009ac0       ??_R3QVBox@@8              10027ac0     alm_bncs_output.obj
 0002:00009ad0       ??_R2QVBox@@8              10027ad0     alm_bncs_output.obj
 0002:00009af0       ??_R1A@?0A@EA@QHBox@@8     10027af0     alm_bncs_output.obj
 0002:00009b0c       ??_R3QHBox@@8              10027b0c     alm_bncs_output.obj
 0002:00009b1c       ??_R2QHBox@@8              10027b1c     alm_bncs_output.obj
 0002:00009b38       ??_R4CAlm_sys_select@@6BQPaintDevice@@@ 10027b38     alm_bncs_output.obj
 0002:00009b4c       ??_R4QGuardedPtrPrivate@@6B@ 10027b4c     alm_bncs_output.obj
 0002:00009b60       ??_R3QGuardedPtrPrivate@@8 10027b60     alm_bncs_output.obj
 0002:00009b70       ??_R2QGuardedPtrPrivate@@8 10027b70     alm_bncs_output.obj
 0002:00009b84       ??_R1A@?0A@EA@QGuardedPtrPrivate@@8 10027b84     alm_bncs_output.obj
 0002:00009ba0       ??_R1CI@?0A@EA@QShared@@8  10027ba0     alm_bncs_output.obj
 0002:00009bbc       ??_R4QDockWindowList@@6B@  10027bbc     alm_bncs_output.obj
 0002:00009bd0       ??_R3QDockWindowList@@8    10027bd0     alm_bncs_output.obj
 0002:00009be0       ??_R2QDockWindowList@@8    10027be0     alm_bncs_output.obj
 0002:00009bf4       ??_R1A@?0A@EA@QDockWindowList@@8 10027bf4     alm_bncs_output.obj
 0002:00009c10       ??_R1A@?0A@EA@?$QPtrList@VQDockWindow@@@@8 10027c10     alm_bncs_output.obj
 0002:00009c2c       ??_R3?$QPtrList@VQDockWindow@@@@8 10027c2c     alm_bncs_output.obj
 0002:00009c3c       ??_R2?$QPtrList@VQDockWindow@@@@8 10027c3c     alm_bncs_output.obj
 0002:00009c4c       ??_R4QPopupMenuList@@6B@   10027c4c     alm_bncs_output.obj
 0002:00009c60       ??_R3QPopupMenuList@@8     10027c60     alm_bncs_output.obj
 0002:00009c70       ??_R2QPopupMenuList@@8     10027c70     alm_bncs_output.obj
 0002:00009c84       ??_R1A@?0A@EA@QPopupMenuList@@8 10027c84     alm_bncs_output.obj
 0002:00009ca0       ??_R1A@?0A@EA@?$QPtrList@VQPopupMenu@@@@8 10027ca0     alm_bncs_output.obj
 0002:00009cbc       ??_R3?$QPtrList@VQPopupMenu@@@@8 10027cbc     alm_bncs_output.obj
 0002:00009ccc       ??_R2?$QPtrList@VQPopupMenu@@@@8 10027ccc     alm_bncs_output.obj
 0002:00009cdc       ??_R4?$QPtrList@VQPopupMenu@@@@6B@ 10027cdc     alm_bncs_output.obj
 0002:00009cf0       ??_R4config_plugin_base@@6BQObject@@@ 10027cf0     alm_bncs_output.obj
 0002:00009d04       ??_R3config_plugin_base@@8 10027d04     alm_bncs_output.obj
 0002:00009d14       ??_R2config_plugin_base@@8 10027d14     alm_bncs_output.obj
 0002:00009d2c       ??_R1A@?0A@EA@config_plugin_base@@8 10027d2c     alm_bncs_output.obj
 0002:00009d48       ??_R4config_plugin_base@@6BQPaintDevice@@@ 10027d48     alm_bncs_output.obj
 0002:00009d5c       ??_R4IGetDocuments@@6B@    10027d5c     alm_bncs_output.obj
 0002:00009d70       ??_R3IGetDocuments@@8      10027d70     alm_bncs_output.obj
 0002:00009d80       ??_R2IGetDocuments@@8      10027d80     alm_bncs_output.obj
 0002:00009d88       ??_R1A@?0A@EA@IGetDocuments@@8 10027d88     alm_bncs_output.obj
 0002:00009da4       ??_R4IDomDoc@@6B@          10027da4     alm_bncs_output.obj
 0002:00009db8       ??_R3IDomDoc@@8            10027db8     alm_bncs_output.obj
 0002:00009dc8       ??_R2IDomDoc@@8            10027dc8     alm_bncs_output.obj
 0002:00009dd0       ??_R1A@?0A@EA@IDomDoc@@8   10027dd0     alm_bncs_output.obj
 0002:00009dec       ??_R4devTemplate@@6B@      10027dec     alm_bncs_output.obj
 0002:00009e00       ??_R3devTemplate@@8        10027e00     alm_bncs_output.obj
 0002:00009e10       ??_R2devTemplate@@8        10027e10     alm_bncs_output.obj
 0002:00009e18       ??_R1A@?0A@EA@devTemplate@@8 10027e18     alm_bncs_output.obj
 0002:00009e34       ??_R4ISendCommand@@6B@     10027e34     alm_bncs_output.obj
 0002:00009e48       ??_R3ISendCommand@@8       10027e48     alm_bncs_output.obj
 0002:00009e58       ??_R2ISendCommand@@8       10027e58     alm_bncs_output.obj
 0002:00009e60       ??_R1A@?0A@EA@ISendCommand@@8 10027e60     alm_bncs_output.obj
 0002:00009e7c       ??_R4alm_bncs_output@@6BQObject@@@ 10027e7c     alm_bncs_output.obj
 0002:00009e90       ??_R3alm_bncs_output@@8    10027e90     alm_bncs_output.obj
 0002:00009ea0       ??_R2alm_bncs_output@@8    10027ea0     alm_bncs_output.obj
 0002:00009ec8       ??_R1A@?0A@EA@alm_bncs_output@@8 10027ec8     alm_bncs_output.obj
 0002:00009ee4       ??_R1HI@?0A@EA@IDomDoc@@8  10027ee4     alm_bncs_output.obj
 0002:00009f00       ??_R1HM@?0A@EA@IGetDocuments@@8 10027f00     alm_bncs_output.obj
 0002:00009f1c       ??_R1IA@?0A@EA@ISendCommand@@8 10027f1c     alm_bncs_output.obj
 0002:00009f38       ??_R4alm_bncs_output@@6BQPaintDevice@@@ 10027f38     alm_bncs_output.obj
 0002:00009f4c       ??_R4alm_bncs_output@@6BIDomDoc@@@ 10027f4c     alm_bncs_output.obj
 0002:00009f60       ??_R4alm_bncs_output@@6BIGetDocuments@@@ 10027f60     alm_bncs_output.obj
 0002:00009f74       ??_R4alm_bncs_output@@6BISendCommand@@@ 10027f74     alm_bncs_output.obj
 0002:00009f88       ??_R4FileLoad_BncsSystem@alm_bncs_output@@6B@ 10027f88     alm_bncs_output.obj
 0002:00009f9c       ??_R3FileLoad_BncsSystem@alm_bncs_output@@8 10027f9c     alm_bncs_output.obj
 0002:00009fac       ??_R2FileLoad_BncsSystem@alm_bncs_output@@8 10027fac     alm_bncs_output.obj
 0002:00009fb8       ??_R1A@?0A@EA@FileLoad_BncsSystem@alm_bncs_output@@8 10027fb8     alm_bncs_output.obj
 0002:00009fd4       ??_R1A@?0A@EA@FileLoad@@8  10027fd4     alm_bncs_output.obj
 0002:00009ff0       ??_R3FileLoad@@8           10027ff0     alm_bncs_output.obj
 0002:0000a000       ??_R2FileLoad@@8           10028000     alm_bncs_output.obj
 0002:0000a008       ??_R4?$QPtrList@VcOutputFile@@@@6B@ 10028008     alm_bncs_output.obj
 0002:0000a01c       ??_R3?$QPtrList@VcOutputFile@@@@8 1002801c     alm_bncs_output.obj
 0002:0000a02c       ??_R2?$QPtrList@VcOutputFile@@@@8 1002802c     alm_bncs_output.obj
 0002:0000a03c       ??_R1A@?0A@EA@?$QPtrList@VcOutputFile@@@@8 1002803c     alm_bncs_output.obj
 0002:0000a058       ??_R4autoNumberDialog@@6BQObject@@@ 10028058     autonumberdialogimpl.obj
 0002:0000a06c       ??_R3autoNumberDialog@@8   1002806c     autonumberdialogimpl.obj
 0002:0000a07c       ??_R2autoNumberDialog@@8   1002807c     autonumberdialogimpl.obj
 0002:0000a09c       ??_R1A@?0A@EA@autoNumberDialog@@8 1002809c     autonumberdialogimpl.obj
 0002:0000a0b8       ??_R1A@?0A@EA@autoNumberDialogBase@@8 100280b8     autonumberdialogimpl.obj
 0002:0000a0d4       ??_R3autoNumberDialogBase@@8 100280d4     autonumberdialogimpl.obj
 0002:0000a0e4       ??_R2autoNumberDialogBase@@8 100280e4     autonumberdialogimpl.obj
 0002:0000a100       ??_R1A@?0A@EA@QDialog@@8   10028100     autonumberdialogimpl.obj
 0002:0000a11c       ??_R3QDialog@@8            1002811c     autonumberdialogimpl.obj
 0002:0000a12c       ??_R2QDialog@@8            1002812c     autonumberdialogimpl.obj
 0002:0000a144       ??_R4autoNumberDialog@@6BQPaintDevice@@@ 10028144     autonumberdialogimpl.obj
 0002:0000a158       ??_R4cOutputFile@@6B@      10028158     cOutputFile.obj
 0002:0000a16c       ??_R3cOutputFile@@8        1002816c     cOutputFile.obj
 0002:0000a17c       ??_R2cOutputFile@@8        1002817c     cOutputFile.obj
 0002:0000a184       ??_R1A@?0A@EA@cOutputFile@@8 10028184     cOutputFile.obj
 0002:0000a1a0       ??_R1A@?0A@EA@QGDict@@8    100281a0     devTemplate.obj
 0002:0000a1bc       ??_R3QGDict@@8             100281bc     devTemplate.obj
 0002:0000a1cc       ??_R2QGDict@@8             100281cc     devTemplate.obj
 0002:0000a1d8       ??_R4TemplateList@@6B@     100281d8     devTemplate.obj
 0002:0000a1ec       ??_R3TemplateList@@8       100281ec     devTemplate.obj
 0002:0000a1fc       ??_R2TemplateList@@8       100281fc     devTemplate.obj
 0002:0000a210       ??_R1A@?0A@EA@TemplateList@@8 10028210     devTemplate.obj
 0002:0000a22c       ??_R1A@?0A@EA@?$QDict@VdevTemplate@@@@8 1002822c     devTemplate.obj
 0002:0000a248       ??_R3?$QDict@VdevTemplate@@@@8 10028248     devTemplate.obj
 0002:0000a258       ??_R2?$QDict@VdevTemplate@@@@8 10028258     devTemplate.obj
 0002:0000a268       ??_R4?$QDict@VdevTemplate@@@@6B@ 10028268     devTemplate.obj
 0002:0000a27c       ??_R4dialog@@6BQObject@@@  1002827c     dialogimpl.obj
 0002:0000a290       ??_R3dialog@@8             10028290     dialogimpl.obj
 0002:0000a2a0       ??_R2dialog@@8             100282a0     dialogimpl.obj
 0002:0000a2bc       ??_R1A@?0A@EA@dialog@@8    100282bc     dialogimpl.obj
 0002:0000a2d8       ??_R1A@?0A@EA@dialogBase@@8 100282d8     dialogimpl.obj
 0002:0000a2f4       ??_R3dialogBase@@8         100282f4     dialogimpl.obj
 0002:0000a304       ??_R2dialogBase@@8         10028304     dialogimpl.obj
 0002:0000a31c       ??_R4dialog@@6BQPaintDevice@@@ 1002831c     dialogimpl.obj
 0002:0000a330       ??_R4QPushButton@@6BQObject@@@ 10028330     manage_temp.obj
 0002:0000a344       ??_R3QPushButton@@8        10028344     manage_temp.obj
 0002:0000a354       ??_R2QPushButton@@8        10028354     manage_temp.obj
 0002:0000a370       ??_R1A@?0A@EA@QPushButton@@8 10028370     manage_temp.obj
 0002:0000a38c       ??_R1A@?0A@EA@QButton@@8   1002838c     manage_temp.obj
 0002:0000a3a8       ??_R3QButton@@8            100283a8     manage_temp.obj
 0002:0000a3b8       ??_R2QButton@@8            100283b8     manage_temp.obj
 0002:0000a3d0       ??_R4QPushButton@@6BQPaintDevice@@@ 100283d0     manage_temp.obj
 0002:0000a3e4       ??_R4QVBoxLayout@@6BQObject@@@ 100283e4     manage_temp.obj
 0002:0000a3f8       ??_R3QVBoxLayout@@8        100283f8     manage_temp.obj
 0002:0000a408       ??_R2QVBoxLayout@@8        10028408     manage_temp.obj
 0002:0000a424       ??_R1A@?0A@EA@QVBoxLayout@@8 10028424     manage_temp.obj
 0002:0000a440       ??_R4QVBoxLayout@@6BQLayoutItem@@@ 10028440     manage_temp.obj
 0002:0000a454       ??_R4QHBoxLayout@@6BQObject@@@ 10028454     manage_temp.obj
 0002:0000a468       ??_R3QHBoxLayout@@8        10028468     manage_temp.obj
 0002:0000a478       ??_R2QHBoxLayout@@8        10028478     manage_temp.obj
 0002:0000a494       ??_R1A@?0A@EA@QHBoxLayout@@8 10028494     manage_temp.obj
 0002:0000a4b0       ??_R4QHBoxLayout@@6BQLayoutItem@@@ 100284b0     manage_temp.obj
 0002:0000a4c4       ??_R4QGridLayout@@6BQObject@@@ 100284c4     manage_temp.obj
 0002:0000a4d8       ??_R3QGridLayout@@8        100284d8     manage_temp.obj
 0002:0000a4e8       ??_R2QGridLayout@@8        100284e8     manage_temp.obj
 0002:0000a500       ??_R1A@?0A@EA@QGridLayout@@8 10028500     manage_temp.obj
 0002:0000a51c       ??_R4QGridLayout@@6BQLayoutItem@@@ 1002851c     manage_temp.obj
 0002:0000a530       ??_R4QLabel@@6BQObject@@@  10028530     manage_temp.obj
 0002:0000a544       ??_R3QLabel@@8             10028544     manage_temp.obj
 0002:0000a554       ??_R2QLabel@@8             10028554     manage_temp.obj
 0002:0000a570       ??_R1A@?0A@EA@QLabel@@8    10028570     manage_temp.obj
 0002:0000a58c       ??_R4QLabel@@6BQPaintDevice@@@ 1002858c     manage_temp.obj
 0002:0000a5a0       ??_R4QComboBox@@6BQObject@@@ 100285a0     manage_temp.obj
 0002:0000a5b4       ??_R3QComboBox@@8          100285b4     manage_temp.obj
 0002:0000a5c4       ??_R2QComboBox@@8          100285c4     manage_temp.obj
 0002:0000a5dc       ??_R1A@?0A@EA@QComboBox@@8 100285dc     manage_temp.obj
 0002:0000a5f8       ??_R4QComboBox@@6BQPaintDevice@@@ 100285f8     manage_temp.obj
 0002:0000a60c       ??_R4QLineEdit@@6BQObject@@@ 1002860c     manage_temp.obj
 0002:0000a620       ??_R3QLineEdit@@8          10028620     manage_temp.obj
 0002:0000a630       ??_R2QLineEdit@@8          10028630     manage_temp.obj
 0002:0000a64c       ??_R1A@?0A@EA@QLineEdit@@8 1002864c     manage_temp.obj
 0002:0000a668       ??_R4QLineEdit@@6BQPaintDevice@@@ 10028668     manage_temp.obj
 0002:0000a67c       ??_R4QSpinBox@@6BQObject@@@ 1002867c     manage_temp.obj
 0002:0000a690       ??_R3QSpinBox@@8           10028690     manage_temp.obj
 0002:0000a6a0       ??_R2QSpinBox@@8           100286a0     manage_temp.obj
 0002:0000a6bc       ??_R1A@?0A@EA@QSpinBox@@8  100286bc     manage_temp.obj
 0002:0000a6d8       ??_R1GM@?0A@EA@QRangeControl@@8 100286d8     manage_temp.obj
 0002:0000a6f4       ??_R3QRangeControl@@8      100286f4     manage_temp.obj
 0002:0000a704       ??_R2QRangeControl@@8      10028704     manage_temp.obj
 0002:0000a70c       ??_R1A@?0A@EA@QRangeControl@@8 1002870c     manage_temp.obj
 0002:0000a728       ??_R4QSpinBox@@6BQPaintDevice@@@ 10028728     manage_temp.obj
 0002:0000a73c       ??_R4QSpinBox@@6B@         1002873c     manage_temp.obj
 0002:0000a750       ??_R4QTable@@6BQObject@@@  10028750     manage_temp.obj
 0002:0000a764       ??_R3QTable@@8             10028764     manage_temp.obj
 0002:0000a774       ??_R2QTable@@8             10028774     manage_temp.obj
 0002:0000a794       ??_R1A@?0A@EA@QTable@@8    10028794     manage_temp.obj
 0002:0000a7b0       ??_R4QTable@@6BQPaintDevice@@@ 100287b0     manage_temp.obj
 0002:0000a7c4       ??_R4manage_tempBase@@6BQObject@@@ 100287c4     manage_temp.obj
 0002:0000a7d8       ??_R3manage_tempBase@@8    100287d8     manage_temp.obj
 0002:0000a7e8       ??_R2manage_tempBase@@8    100287e8     manage_temp.obj
 0002:0000a804       ??_R1A@?0A@EA@manage_tempBase@@8 10028804     manage_temp.obj
 0002:0000a820       ??_R4manage_tempBase@@6BQPaintDevice@@@ 10028820     manage_temp.obj
 0002:0000a834       ??_R4QSpacerItem@@6B@      10028834     manage_temp.obj
 0002:0000a848       ??_R3QSpacerItem@@8        10028848     manage_temp.obj
 0002:0000a858       ??_R2QSpacerItem@@8        10028858     manage_temp.obj
 0002:0000a864       ??_R1A@?0A@EA@QSpacerItem@@8 10028864     manage_temp.obj
 0002:0000a880       ??_R4QCheckTableItem@@6B@  10028880     manage_tempimpl.obj
 0002:0000a894       ??_R3QCheckTableItem@@8    10028894     manage_tempimpl.obj
 0002:0000a8a4       ??_R2QCheckTableItem@@8    100288a4     manage_tempimpl.obj
 0002:0000a8b4       ??_R1A@?0A@EA@QCheckTableItem@@8 100288b4     manage_tempimpl.obj
 0002:0000a8d0       ??_R1A@?0A@EA@QTableItem@@8 100288d0     manage_tempimpl.obj
 0002:0000a8ec       ??_R3QTableItem@@8         100288ec     manage_tempimpl.obj
 0002:0000a8fc       ??_R2QTableItem@@8         100288fc     manage_tempimpl.obj
 0002:0000a908       ??_R4manage_temp@@6BQObject@@@ 10028908     manage_tempimpl.obj
 0002:0000a91c       ??_R3manage_temp@@8        1002891c     manage_tempimpl.obj
 0002:0000a92c       ??_R2manage_temp@@8        1002892c     manage_tempimpl.obj
 0002:0000a94c       ??_R1A@?0A@EA@manage_temp@@8 1002894c     manage_tempimpl.obj
 0002:0000a968       ??_R4manage_temp@@6BQPaintDevice@@@ 10028968     manage_tempimpl.obj
 0002:0000a97c       ??_R4config_plugin_desc_base@@6B@ 1002897c     plugindesc.obj
 0002:0000a990       ??_R3config_plugin_desc_base@@8 10028990     plugindesc.obj
 0002:0000a9a0       ??_R2config_plugin_desc_base@@8 100289a0     plugindesc.obj
 0002:0000a9a8       ??_R1A@?0A@EA@config_plugin_desc_base@@8 100289a8     plugindesc.obj
 0002:0000a9c4       ??_R4plugindesc@@6B@       100289c4     plugindesc.obj
 0002:0000a9d8       ??_R3plugindesc@@8         100289d8     plugindesc.obj
 0002:0000a9e8       ??_R2plugindesc@@8         100289e8     plugindesc.obj
 0002:0000a9f4       ??_R1A@?0A@EA@plugindesc@@8 100289f4     plugindesc.obj
 0002:0000aa10       ??_R4processItem@@6B@      10028a10     processItem.obj
 0002:0000aa24       ??_R3processItem@@8        10028a24     processItem.obj
 0002:0000aa34       ??_R2processItem@@8        10028a34     processItem.obj
 0002:0000aa44       ??_R1A@?0A@EA@processItem@@8 10028a44     processItem.obj
 0002:0000aa60       ??_R4QButtonGroup@@6BQObject@@@ 10028a60     autonumberdialog.obj
 0002:0000aa74       ??_R3QButtonGroup@@8       10028a74     autonumberdialog.obj
 0002:0000aa84       ??_R2QButtonGroup@@8       10028a84     autonumberdialog.obj
 0002:0000aaa4       ??_R1A@?0A@EA@QButtonGroup@@8 10028aa4     autonumberdialog.obj
 0002:0000aac0       ??_R1A@?0A@EA@QGroupBox@@8 10028ac0     autonumberdialog.obj
 0002:0000aadc       ??_R3QGroupBox@@8          10028adc     autonumberdialog.obj
 0002:0000aaec       ??_R2QGroupBox@@8          10028aec     autonumberdialog.obj
 0002:0000ab08       ??_R4QButtonGroup@@6BQPaintDevice@@@ 10028b08     autonumberdialog.obj
 0002:0000ab1c       ??_R4QRadioButton@@6BQObject@@@ 10028b1c     autonumberdialog.obj
 0002:0000ab30       ??_R3QRadioButton@@8       10028b30     autonumberdialog.obj
 0002:0000ab40       ??_R2QRadioButton@@8       10028b40     autonumberdialog.obj
 0002:0000ab5c       ??_R1A@?0A@EA@QRadioButton@@8 10028b5c     autonumberdialog.obj
 0002:0000ab78       ??_R4QRadioButton@@6BQPaintDevice@@@ 10028b78     autonumberdialog.obj
 0002:0000ab8c       ??_R4QGroupBox@@6BQObject@@@ 10028b8c     autonumberdialog.obj
 0002:0000aba0       ??_R4QGroupBox@@6BQPaintDevice@@@ 10028ba0     autonumberdialog.obj
 0002:0000abb4       ??_R4autoNumberDialogBase@@6BQObject@@@ 10028bb4     autonumberdialog.obj
 0002:0000abc8       ??_R4autoNumberDialogBase@@6BQPaintDevice@@@ 10028bc8     autonumberdialog.obj
 0002:0000abdc       ??_R4dialogBase@@6BQObject@@@ 10028bdc     dialog.obj
 0002:0000abf0       ??_R4dialogBase@@6BQPaintDevice@@@ 10028bf0     dialog.obj
 0002:0000ac04       ??_R4Document@@6B@         10028c04     config_alarm_utilities:Document.obj
 0002:0000ac18       ??_R3Document@@8           10028c18     config_alarm_utilities:Document.obj
 0002:0000ac28       ??_R2Document@@8           10028c28     config_alarm_utilities:Document.obj
 0002:0000ac30       ??_R1A@?0A@EA@Document@@8  10028c30     config_alarm_utilities:Document.obj
 0002:0000ac4c       ??_R4Document_BncsSystem@@6B@ 10028c4c     config_alarm_utilities:Document.obj
 0002:0000ac60       ??_R3Document_BncsSystem@@8 10028c60     config_alarm_utilities:Document.obj
 0002:0000ac70       ??_R2Document_BncsSystem@@8 10028c70     config_alarm_utilities:Document.obj
 0002:0000ac7c       ??_R1A@?0A@EA@Document_BncsSystem@@8 10028c7c     config_alarm_utilities:Document.obj
 0002:0000ac98       ??_R1A@?0A@EN@Document@@8  10028c98     config_alarm_utilities:Document.obj
 0002:0000acb4       ??_R4FileLoad@@6B@         10028cb4     config_alarm_utilities:Loaders.obj
 0002:0000acc8       ??_R4Loaders@@6B@          10028cc8     config_alarm_utilities:Loaders.obj
 0002:0000acdc       ??_R3Loaders@@8            10028cdc     config_alarm_utilities:Loaders.obj
 0002:0000acec       ??_R2Loaders@@8            10028cec     config_alarm_utilities:Loaders.obj
 0002:0000acf4       ??_R1A@?0A@EA@Loaders@@8   10028cf4     config_alarm_utilities:Loaders.obj
 0002:0000ad10       ??_R4?$QPtrList@VFileLoad@@@@6B@ 10028d10     config_alarm_utilities:Loaders.obj
 0002:0000ad24       ??_R3?$QPtrList@VFileLoad@@@@8 10028d24     config_alarm_utilities:Loaders.obj
 0002:0000ad34       ??_R2?$QPtrList@VFileLoad@@@@8 10028d34     config_alarm_utilities:Loaders.obj
 0002:0000ad44       ??_R1A@?0A@EA@?$QPtrList@VFileLoad@@@@8 10028d44     config_alarm_utilities:Loaders.obj
 0002:0000ad60       ??_R4?$QPtrList@VDirLoad@@@@6B@ 10028d60     config_alarm_utilities:Loaders.obj
 0002:0000ad74       ??_R3?$QPtrList@VDirLoad@@@@8 10028d74     config_alarm_utilities:Loaders.obj
 0002:0000ad84       ??_R2?$QPtrList@VDirLoad@@@@8 10028d84     config_alarm_utilities:Loaders.obj
 0002:0000ad94       ??_R1A@?0A@EA@?$QPtrList@VDirLoad@@@@8 10028d94     config_alarm_utilities:Loaders.obj
 0002:0000adb0       ??_R4type_info@@6B@        10028db0     MSVCRT:ti_inst.obj
 0002:0000adc4       ??_R3type_info@@8          10028dc4     MSVCRT:ti_inst.obj
 0002:0000add4       ??_R2type_info@@8          10028dd4     MSVCRT:ti_inst.obj
 0002:0000addc       ??_R1A@?0A@EA@type_info@@8 10028ddc     MSVCRT:ti_inst.obj
 0002:0000adf8       ___rtc_iaa                 10028df8     MSVCRT:initsect.obj
 0002:0000adfc       ___rtc_izz                 10028dfc     MSVCRT:initsect.obj
 0002:0000ae00       ___rtc_taa                 10028e00     MSVCRT:initsect.obj
 0002:0000ae04       ___rtc_tzz                 10028e04     MSVCRT:initsect.obj
 0002:0000f02c       __IMPORT_DESCRIPTOR_config_icons 1002d02c     config_icons:config_icons.dll
 0002:0000f040       __IMPORT_DESCRIPTOR_qt-mt323 1002d040     qt-mt323:qt-mt323.dll
 0002:0000f054       __IMPORT_DESCRIPTOR_alm_sys_select 1002d054     alm_sys_select:alm_sys_select.dll
 0002:0000f068       __IMPORT_DESCRIPTOR_KERNEL32 1002d068     kernel32:KERNEL32.dll
 0002:0000f07c       __IMPORT_DESCRIPTOR_MSVCR120 1002d07c     MSVCRT:MSVCR120.dll
 0002:0000f090       __IMPORT_DESCRIPTOR_MSVCP120 1002d090     msvcprt:MSVCP120.dll
 0002:0000f0a4       __NULL_IMPORT_DESCRIPTOR   1002d0a4     config_icons:config_icons.dll
 0003:00000160       ___security_cookie         1003b160     MSVCRT:gs_cookie.obj
 0003:00000164       ___security_cookie_complement 1003b164     MSVCRT:gs_cookie.obj
 0003:00000170       ___native_dllmain_reason   1003b170     MSVCRT:natstart.obj
 0003:00000174       ??_R0?AVQGList@@@8         1003b174     alm_bncs_output.obj
 0003:0000018c       ??_R0?AVQPtrCollection@@@8 1003b18c     alm_bncs_output.obj
 0003:000001ac       ??_R0?AVQWidget@@@8        1003b1ac     alm_bncs_output.obj
 0003:000001c4       ??_R0?AVQObject@@@8        1003b1c4     alm_bncs_output.obj
 0003:000001dc       ??_R0?AVQt@@@8             1003b1dc     alm_bncs_output.obj
 0003:000001f0       ??_R0?AVQPaintDevice@@@8   1003b1f0     alm_bncs_output.obj
 0003:0000020c       ??_R0?AUQShared@@@8        1003b20c     alm_bncs_output.obj
 0003:00000224       ??_R0?AVQPopupMenu@@@8     1003b224     alm_bncs_output.obj
 0003:00000240       ??_R0?AVQFrame@@@8         1003b240     alm_bncs_output.obj
 0003:00000258       ??_R0?AVQMenuData@@@8      1003b258     alm_bncs_output.obj
 0003:00000270       ??_R0?AVQAction@@@8        1003b270     alm_bncs_output.obj
 0003:00000288       ??_R0?AVQBoxLayout@@@8     1003b288     alm_bncs_output.obj
 0003:000002a4       ??_R0?AVQLayout@@@8        1003b2a4     alm_bncs_output.obj
 0003:000002bc       ??_R0?AVQLayoutItem@@@8    1003b2bc     alm_bncs_output.obj
 0003:000002d8       ??_R0?AVQToolBar@@@8       1003b2d8     alm_bncs_output.obj
 0003:000002f0       ??_R0?AVQDockWindow@@@8    1003b2f0     alm_bncs_output.obj
 0003:0000030c       ??_R0?AVQListView@@@8      1003b30c     alm_bncs_output.obj
 0003:00000324       ??_R0?AVQScrollView@@@8    1003b324     alm_bncs_output.obj
 0003:00000340       ??_R0?AVQListViewItem@@@8  1003b340     alm_bncs_output.obj
 0003:0000035c       ??_R0?AVQTabWidget@@@8     1003b35c     alm_bncs_output.obj
 0003:00000378       ??_R0?AVCAlm_sys_select@@@8 1003b378     alm_bncs_output.obj
 0003:00000398       ??_R0?AVQVBox@@@8          1003b398     alm_bncs_output.obj
 0003:000003ac       ??_R0?AVQHBox@@@8          1003b3ac     alm_bncs_output.obj
 0003:000003c0       ??_R0?AVQGuardedPtrPrivate@@@8 1003b3c0     alm_bncs_output.obj
 0003:000003e4       ??_R0?AVQDockWindowList@@@8 1003b3e4     alm_bncs_output.obj
 0003:00000404       ??_R0?AV?$QPtrList@VQDockWindow@@@@@8 1003b404     alm_bncs_output.obj
 0003:0000042c       ??_R0?AVQPopupMenuList@@@8 1003b42c     alm_bncs_output.obj
 0003:0000044c       ??_R0?AV?$QPtrList@VQPopupMenu@@@@@8 1003b44c     alm_bncs_output.obj
 0003:00000474       ??_R0?AVconfig_plugin_base@@@8 1003b474     alm_bncs_output.obj
 0003:00000498       ??_R0?AVIGetDocuments@@@8  1003b498     alm_bncs_output.obj
 0003:000004b4       ??_R0?AVIDomDoc@@@8        1003b4b4     alm_bncs_output.obj
 0003:000004cc       ??_R0?AVdevTemplate@@@8    1003b4cc     alm_bncs_output.obj
 0003:000004e8       ??_R0?AVISendCommand@@@8   1003b4e8     alm_bncs_output.obj
 0003:00000504       ??_R0?AValm_bncs_output@@@8 1003b504     alm_bncs_output.obj
 0003:00000524       ??_R0?AVFileLoad_BncsSystem@alm_bncs_output@@@8 1003b524     alm_bncs_output.obj
 0003:00000558       ??_R0?AVFileLoad@@@8       1003b558     alm_bncs_output.obj
 0003:00000570       ??_R0?AV?$QPtrList@VcOutputFile@@@@@8 1003b570     alm_bncs_output.obj
 0003:00000598       ??_R0?AVautoNumberDialog@@@8 1003b598     autonumberdialogimpl.obj
 0003:000005b8       ??_R0?AVautoNumberDialogBase@@@8 1003b5b8     autonumberdialogimpl.obj
 0003:000005dc       ??_R0?AVQDialog@@@8        1003b5dc     autonumberdialogimpl.obj
 0003:000005f4       ??_R0?AVcOutputFile@@@8    1003b5f4     cOutputFile.obj
 0003:00000610       ??_R0?AVQGDict@@@8         1003b610     devTemplate.obj
 0003:00000628       ??_R0?AVTemplateList@@@8   1003b628     devTemplate.obj
 0003:00000644       ??_R0?AV?$QDict@VdevTemplate@@@@@8 1003b644     devTemplate.obj
 0003:0000066c       ??_R0?AVdialog@@@8         1003b66c     dialogimpl.obj
 0003:00000684       ??_R0?AVdialogBase@@@8     1003b684     dialogimpl.obj
 0003:000006a0       ??_R0?AVQPushButton@@@8    1003b6a0     manage_temp.obj
 0003:000006bc       ??_R0?AVQButton@@@8        1003b6bc     manage_temp.obj
 0003:000006d4       ??_R0?AVQVBoxLayout@@@8    1003b6d4     manage_temp.obj
 0003:000006f0       ??_R0?AVQHBoxLayout@@@8    1003b6f0     manage_temp.obj
 0003:0000070c       ??_R0?AVQGridLayout@@@8    1003b70c     manage_temp.obj
 0003:00000728       ??_R0?AVQLabel@@@8         1003b728     manage_temp.obj
 0003:00000740       ??_R0?AVQComboBox@@@8      1003b740     manage_temp.obj
 0003:00000758       ??_R0?AVQLineEdit@@@8      1003b758     manage_temp.obj
 0003:00000770       ??_R0?AVQSpinBox@@@8       1003b770     manage_temp.obj
 0003:00000788       ??_R0?AVQRangeControl@@@8  1003b788     manage_temp.obj
 0003:000007a4       ??_R0?AVQTable@@@8         1003b7a4     manage_temp.obj
 0003:000007bc       ??_R0?AVmanage_tempBase@@@8 1003b7bc     manage_temp.obj
 0003:000007dc       ??_R0?AVQSpacerItem@@@8    1003b7dc     manage_temp.obj
 0003:000007f8       ??_R0?AVQCheckTableItem@@@8 1003b7f8     manage_tempimpl.obj
 0003:00000818       ??_R0?AVQTableItem@@@8     1003b818     manage_tempimpl.obj
 0003:00000834       ??_R0?AVmanage_temp@@@8    1003b834     manage_tempimpl.obj
 0003:00000850       ??_R0?AVconfig_plugin_desc_base@@@8 1003b850     plugindesc.obj
 0003:00000878       ??_R0?AVplugindesc@@@8     1003b878     plugindesc.obj
 0003:00000894       ??_R0?AVprocessItem@@@8    1003b894     processItem.obj
 0003:000008b0       ??_R0?AVQButtonGroup@@@8   1003b8b0     autonumberdialog.obj
 0003:000008cc       ??_R0?AVQGroupBox@@@8      1003b8cc     autonumberdialog.obj
 0003:000008e4       ??_R0?AVQRadioButton@@@8   1003b8e4     autonumberdialog.obj
 0003:00000900       ??_R0?AVDocument@@@8       1003b900     config_alarm_utilities:Document.obj
 0003:00000918       ??_R0?AVDocument_BncsSystem@@@8 1003b918     config_alarm_utilities:Document.obj
 0003:0000093c       ??_R0?AVLoaders@@@8        1003b93c     config_alarm_utilities:Loaders.obj
 0003:00000954       ??_R0?AV?$QPtrList@VFileLoad@@@@@8 1003b954     config_alarm_utilities:Loaders.obj
 0003:0000097c       ??_R0?AV?$QPtrList@VDirLoad@@@@@8 1003b97c     config_alarm_utilities:Loaders.obj
 0003:000009a0       ??_R0?AVtype_info@@@8      1003b9a0     MSVCRT:ti_inst.obj
 0003:000009b8       ?sm_sDomEncoding@alm_bncs_output@@0VQString@@B 1003b9b8     alm_bncs_output.obj
 0003:000009c4       ?metaObj@manage_tempBase@@0PAVQMetaObject@@A 1003b9c4     moc_manage_temp.obj
 0003:000009cc       ?metaObj@manage_temp@@0PAVQMetaObject@@A 1003b9cc     moc_manage_tempimpl.obj
 0003:00000a28       ?metaObj@alm_bncs_output@@0PAVQMetaObject@@A 1003ba28     moc_alm_bncs_output.obj
 0003:00000a84       ?metaObj@autoNumberDialogBase@@0PAVQMetaObject@@A 1003ba84     moc_autonumberdialog.obj
 0003:00000a8c       ?metaObj@autoNumberDialog@@0PAVQMetaObject@@A 1003ba8c     moc_autonumberdialogimpl.obj
 0003:00000a94       ?metaObj@dialogBase@@0PAVQMetaObject@@A 1003ba94     moc_dialog.obj
 0003:00000a9c       ?metaObj@dialog@@0PAVQMetaObject@@A 1003ba9c     moc_dialogimpl.obj
 0003:00000ac8       ?sm_sSystemFolder@Document@@1VQString@@A 1003bac8     config_alarm_utilities:Document.obj
 0003:00000df0       ?__type_info_root_node@@3U__type_info_node@@A 1003bdf0     MSVCRT:tncleanup.obj
 0003:00000df8       ___native_startup_lock     1003bdf8     <common>
 0003:00000dfc       ___native_startup_state    1003bdfc     <common>
 0003:00000e00       ___dyn_tls_init_callback   1003be00     <common>
 0003:00000e04       ___onexitend               1003be04     <common>
 0003:00000e08       ___onexitbegin             1003be08     <common>

 entry point at        0001:000176b2

 Static symbols

 0001:00000000       ??__E?sm_sDomEncoding@alm_bncs_output@@0VQString@@B@@YAXXZ 10001000 f   alm_bncs_output.obj
 0001:0000001c       ??__EcleanUp_manage_tempBase@@YAXXZ 1000101c f   moc_manage_temp.obj
 0001:0000003d       ??__EcleanUp_manage_temp@@YAXXZ 1000103d f   moc_manage_tempimpl.obj
 0001:0000005e       ??__EcleanUp_alm_bncs_output@@YAXXZ 1000105e f   moc_alm_bncs_output.obj
 0001:0000007f       ??__EcleanUp_autoNumberDialogBase@@YAXXZ 1000107f f   moc_autonumberdialog.obj
 0001:000000a0       ??__EcleanUp_autoNumberDialog@@YAXXZ 100010a0 f   moc_autonumberdialogimpl.obj
 0001:000000c1       ??__EcleanUp_dialogBase@@YAXXZ 100010c1 f   moc_dialog.obj
 0001:000000e2       ??__EcleanUp_dialog@@YAXXZ 100010e2 f   moc_dialogimpl.obj
 0001:00000110       ??__E?sm_sSystemFolder@Document@@1VQString@@A@@YAXXZ 10001110 f   config_alarm_utilities:Document.obj
 0001:000120c9       $LN42                      100130c9     moc_manage_tempimpl.obj
 0001:000145d5       $LN53                      100155d5     moc_alm_bncs_output.obj
 0001:00014c7b       $LN51                      10015c7b     moc_dialogimpl.obj
 0001:0001746f       _pre_c_init                1001846f f   MSVCRT:crtdll.obj
 0001:000176d5       ___DllMainCRTStartup       100186d5 f   MSVCRT:crtdll.obj
 0001:00017820       $$000000                   10018820     MSVCRT:sehprolg4.obj
 0001:00017c70       __unwindfunclet$??0?$QMapNode@VQString@@W4ESection@@@@QAE@ABU0@@Z$0 10018c70 f   alm_bncs_output.obj
 0001:00017c70       __unwindfunclet$??0?$QMapNode@VQString@@W4ESection@@@@QAE@ABVQString@@@Z$0 10018c70 f   alm_bncs_output.obj
 0001:00017c7c       __ehhandler$??0?$QMapNode@VQString@@W4ESection@@@@QAE@ABVQString@@@Z 10018c7c f   alm_bncs_output.obj
 0001:00017c7c       __ehhandler$??0?$QMapNode@VQString@@W4ESection@@@@QAE@ABU0@@Z 10018c7c f   alm_bncs_output.obj
 0001:00017c97       __unwindfunclet$?insert@?$QMapPrivate@VQString@@W4ESection@@@@QAE?AV?$QMapIterator@VQString@@W4ESection@@@@PAUQMapNodeBase@@0ABVQString@@@Z$0 10018c97 f   alm_bncs_output.obj
 0001:00017c97       __unwindfunclet$??0?$QMapPrivate@VQString@@W4ESection@@@@QAE@XZ$0 10018c97 f   alm_bncs_output.obj
 0001:00017c97       __unwindfunclet$??0?$QMap@VQString@@W4ESection@@@@QAE@XZ$0 10018c97 f   alm_bncs_output.obj
 0001:00017c97       __unwindfunclet$?detachInternal@?$QMap@VQString@@W4ESection@@@@AAEXXZ$0 10018c97 f   alm_bncs_output.obj
 0001:00017c97       __unwindfunclet$??4?$QGuardedPtr@VQPopupMenu@@@@QAEAAV0@PAVQPopupMenu@@@Z$0 10018c97 f   alm_bncs_output.obj
 0001:00017c97       __unwindfunclet$?create@plugindesc@@UAEPAVconfig_plugin_base@@ABVQString@@00@Z$0 10018c97 f   alm_bncs_output.obj
 0001:00017c97       __unwindfunclet$??0?$QGuardedPtr@VQPopupMenu@@@@QAE@XZ$0 10018c97 f   alm_bncs_output.obj
 0001:00017c97       __unwindfunclet$??0?$QGuardedPtr@VQDockWindow@@@@QAE@XZ$0 10018c97 f   alm_bncs_output.obj
 0001:00017c97       __unwindfunclet$??4?$QGuardedPtr@VQDockWindow@@@@QAEAAV0@PAVQDockWindow@@@Z$0 10018c97 f   alm_bncs_output.obj
 0001:00017ca1       __ehhandler$??4?$QGuardedPtr@VQDockWindow@@@@QAEAAV0@PAVQDockWindow@@@Z 10018ca1 f   alm_bncs_output.obj
 0001:00017ca1       __ehhandler$??0?$QGuardedPtr@VQPopupMenu@@@@QAE@XZ 10018ca1 f   alm_bncs_output.obj
 0001:00017ca1       __ehhandler$?create@plugindesc@@UAEPAVconfig_plugin_base@@ABVQString@@00@Z 10018ca1 f   alm_bncs_output.obj
 0001:00017ca1       __ehhandler$??4?$QGuardedPtr@VQPopupMenu@@@@QAEAAV0@PAVQPopupMenu@@@Z 10018ca1 f   alm_bncs_output.obj
 0001:00017ca1       __ehhandler$??0?$QGuardedPtr@VQDockWindow@@@@QAE@XZ 10018ca1 f   alm_bncs_output.obj
 0001:00017ca1       __ehhandler$?insert@?$QMapPrivate@VQString@@W4ESection@@@@QAE?AV?$QMapIterator@VQString@@W4ESection@@@@PAUQMapNodeBase@@0ABVQString@@@Z 10018ca1 f   alm_bncs_output.obj
 0001:00017ca1       __ehhandler$??0?$QMapPrivate@VQString@@W4ESection@@@@QAE@XZ 10018ca1 f   alm_bncs_output.obj
 0001:00017ca1       __ehhandler$?detachInternal@?$QMap@VQString@@W4ESection@@@@AAEXXZ 10018ca1 f   alm_bncs_output.obj
 0001:00017ca1       __ehhandler$??0?$QMap@VQString@@W4ESection@@@@QAE@XZ 10018ca1 f   alm_bncs_output.obj
 0001:00017cbc       __unwindfunclet$??0FileLoad_BncsSystem@alm_bncs_output@@QAE@PAV1@@Z$0 10018cbc f   alm_bncs_output.obj
 0001:00017cc5       __unwindfunclet$??0FileLoad_BncsSystem@alm_bncs_output@@QAE@PAV1@@Z$1 10018cc5 f   alm_bncs_output.obj
 0001:00017ccd       __unwindfunclet$??0FileLoad_BncsSystem@alm_bncs_output@@QAE@PAV1@@Z$2 10018ccd f   alm_bncs_output.obj
 0001:00017cd7       __ehhandler$??0FileLoad_BncsSystem@alm_bncs_output@@QAE@PAV1@@Z 10018cd7 f   alm_bncs_output.obj
 0001:00017cf2       __unwindfunclet$??0alm_bncs_output@@QAE@ABVQString@@00@Z$0 10018cf2 f   alm_bncs_output.obj
 0001:00017cfa       __unwindfunclet$??0alm_bncs_output@@QAE@ABVQString@@00@Z$1 10018cfa f   alm_bncs_output.obj
 0001:00017d05       __unwindfunclet$??0alm_bncs_output@@QAE@ABVQString@@00@Z$2 10018d05 f   alm_bncs_output.obj
 0001:00017d14       __unwindfunclet$??0alm_bncs_output@@QAE@ABVQString@@00@Z$3 10018d14 f   alm_bncs_output.obj
 0001:00017d23       __unwindfunclet$??0alm_bncs_output@@QAE@ABVQString@@00@Z$4 10018d23 f   alm_bncs_output.obj
 0001:00017d32       __unwindfunclet$??0alm_bncs_output@@QAE@ABVQString@@00@Z$5 10018d32 f   alm_bncs_output.obj
 0001:00017d41       __unwindfunclet$??0alm_bncs_output@@QAE@ABVQString@@00@Z$6 10018d41 f   alm_bncs_output.obj
 0001:00017d50       __unwindfunclet$??0alm_bncs_output@@QAE@ABVQString@@00@Z$7 10018d50 f   alm_bncs_output.obj
 0001:00017d5f       __unwindfunclet$??0alm_bncs_output@@QAE@ABVQString@@00@Z$8 10018d5f f   alm_bncs_output.obj
 0001:00017d6e       __unwindfunclet$??0alm_bncs_output@@QAE@ABVQString@@00@Z$9 10018d6e f   alm_bncs_output.obj
 0001:00017d7c       __unwindfunclet$??0alm_bncs_output@@QAE@ABVQString@@00@Z$10 10018d7c f   alm_bncs_output.obj
 0001:00017d8a       __unwindfunclet$??0alm_bncs_output@@QAE@ABVQString@@00@Z$11 10018d8a f   alm_bncs_output.obj
 0001:00017d98       __unwindfunclet$??0alm_bncs_output@@QAE@ABVQString@@00@Z$12 10018d98 f   alm_bncs_output.obj
 0001:00017da6       __unwindfunclet$??0alm_bncs_output@@QAE@ABVQString@@00@Z$13 10018da6 f   alm_bncs_output.obj
 0001:00017db4       __unwindfunclet$??0alm_bncs_output@@QAE@ABVQString@@00@Z$14 10018db4 f   alm_bncs_output.obj
 0001:00017dbe       __unwindfunclet$??0alm_bncs_output@@QAE@ABVQString@@00@Z$15 10018dbe f   alm_bncs_output.obj
 0001:00017dc8       __unwindfunclet$??0alm_bncs_output@@QAE@ABVQString@@00@Z$16 10018dc8 f   alm_bncs_output.obj
 0001:00017dd2       __unwindfunclet$??0alm_bncs_output@@QAE@ABVQString@@00@Z$17 10018dd2 f   alm_bncs_output.obj
 0001:00017ddb       __unwindfunclet$??0alm_bncs_output@@QAE@ABVQString@@00@Z$18 10018ddb f   alm_bncs_output.obj
 0001:00017de5       __unwindfunclet$??0alm_bncs_output@@QAE@ABVQString@@00@Z$19 10018de5 f   alm_bncs_output.obj
 0001:00017def       __unwindfunclet$??0alm_bncs_output@@QAE@ABVQString@@00@Z$20 10018def f   alm_bncs_output.obj
 0001:00017df8       __unwindfunclet$??0alm_bncs_output@@QAE@ABVQString@@00@Z$21 10018df8 f   alm_bncs_output.obj
 0001:00017e02       __unwindfunclet$??0alm_bncs_output@@QAE@ABVQString@@00@Z$22 10018e02 f   alm_bncs_output.obj
 0001:00017e0c       __unwindfunclet$??0alm_bncs_output@@QAE@ABVQString@@00@Z$23 10018e0c f   alm_bncs_output.obj
 0001:00017e16       __unwindfunclet$??0alm_bncs_output@@QAE@ABVQString@@00@Z$24 10018e16 f   alm_bncs_output.obj
 0001:00017e1f       __unwindfunclet$??0alm_bncs_output@@QAE@ABVQString@@00@Z$25 10018e1f f   alm_bncs_output.obj
 0001:00017e28       __unwindfunclet$??0alm_bncs_output@@QAE@ABVQString@@00@Z$26 10018e28 f   alm_bncs_output.obj
 0001:00017e31       __unwindfunclet$??0alm_bncs_output@@QAE@ABVQString@@00@Z$27 10018e31 f   alm_bncs_output.obj
 0001:00017e3a       __unwindfunclet$??0alm_bncs_output@@QAE@ABVQString@@00@Z$28 10018e3a f   alm_bncs_output.obj
 0001:00017e44       __unwindfunclet$??0alm_bncs_output@@QAE@ABVQString@@00@Z$29 10018e44 f   alm_bncs_output.obj
 0001:00017e4e       __unwindfunclet$??0alm_bncs_output@@QAE@ABVQString@@00@Z$30 10018e4e f   alm_bncs_output.obj
 0001:00017e57       __unwindfunclet$??0alm_bncs_output@@QAE@ABVQString@@00@Z$31 10018e57 f   alm_bncs_output.obj
 0001:00017e61       __unwindfunclet$??0alm_bncs_output@@QAE@ABVQString@@00@Z$32 10018e61 f   alm_bncs_output.obj
 0001:00017e7b       __unwindfunclet$??0alm_bncs_output@@QAE@ABVQString@@00@Z$33 10018e7b f   alm_bncs_output.obj
 0001:00017e95       __unwindfunclet$??0alm_bncs_output@@QAE@ABVQString@@00@Z$34 10018e95 f   alm_bncs_output.obj
 0001:00017eaf       __unwindfunclet$??0alm_bncs_output@@QAE@ABVQString@@00@Z$35 10018eaf f   alm_bncs_output.obj
 0001:00017ec9       __unwindfunclet$??0alm_bncs_output@@QAE@ABVQString@@00@Z$37 10018ec9 f   alm_bncs_output.obj
 0001:00017ed3       __unwindfunclet$??0alm_bncs_output@@QAE@ABVQString@@00@Z$38 10018ed3 f   alm_bncs_output.obj
 0001:00017eed       __unwindfunclet$??0alm_bncs_output@@QAE@ABVQString@@00@Z$39 10018eed f   alm_bncs_output.obj
 0001:00017f07       __unwindfunclet$??0alm_bncs_output@@QAE@ABVQString@@00@Z$40 10018f07 f   alm_bncs_output.obj
 0001:00017f21       __unwindfunclet$??0alm_bncs_output@@QAE@ABVQString@@00@Z$41 10018f21 f   alm_bncs_output.obj
 0001:00017f40       __unwindfunclet$??0alm_bncs_output@@QAE@ABVQString@@00@Z$43 10018f40 f   alm_bncs_output.obj
 0001:00017f4a       __unwindfunclet$??0alm_bncs_output@@QAE@ABVQString@@00@Z$44 10018f4a f   alm_bncs_output.obj
 0001:00017f69       __unwindfunclet$??0alm_bncs_output@@QAE@ABVQString@@00@Z$45 10018f69 f   alm_bncs_output.obj
 0001:00017f88       __unwindfunclet$??0alm_bncs_output@@QAE@ABVQString@@00@Z$46 10018f88 f   alm_bncs_output.obj
 0001:00017fa7       __unwindfunclet$??0alm_bncs_output@@QAE@ABVQString@@00@Z$47 10018fa7 f   alm_bncs_output.obj
 0001:00017fc6       __unwindfunclet$??0alm_bncs_output@@QAE@ABVQString@@00@Z$49 10018fc6 f   alm_bncs_output.obj
 0001:00017fd0       __unwindfunclet$??0alm_bncs_output@@QAE@ABVQString@@00@Z$50 10018fd0 f   alm_bncs_output.obj
 0001:00017fef       __unwindfunclet$??0alm_bncs_output@@QAE@ABVQString@@00@Z$51 10018fef f   alm_bncs_output.obj
 0001:0001800e       __unwindfunclet$??0alm_bncs_output@@QAE@ABVQString@@00@Z$52 1001900e f   alm_bncs_output.obj
 0001:0001802d       __unwindfunclet$??0alm_bncs_output@@QAE@ABVQString@@00@Z$53 1001902d f   alm_bncs_output.obj
 0001:0001804c       __ehhandler$??0alm_bncs_output@@QAE@ABVQString@@00@Z 1001904c f   alm_bncs_output.obj
 0001:00018067       __unwindfunclet$??0config_plugin_base@@QAE@ABVQString@@00@Z$0 10019067 f   alm_bncs_output.obj
 0001:00018070       __unwindfunclet$??0config_plugin_base@@QAE@ABVQString@@00@Z$1 10019070 f   alm_bncs_output.obj
 0001:0001807c       __unwindfunclet$??0config_plugin_base@@QAE@ABVQString@@00@Z$2 1001907c f   alm_bncs_output.obj
 0001:00018088       __unwindfunclet$??0config_plugin_base@@QAE@ABVQString@@00@Z$3 10019088 f   alm_bncs_output.obj
 0001:00018094       __ehhandler$??0config_plugin_base@@QAE@ABVQString@@00@Z 10019094 f   alm_bncs_output.obj
 0001:000180af       __unwindfunclet$??1?$QPtrList@VcOutputFile@@@@UAE@XZ$0 100190af f   alm_bncs_output.obj
 0001:000180af       __unwindfunclet$??1?$QPtrList@VQPopupMenu@@@@UAE@XZ$0 100190af f   alm_bncs_output.obj
 0001:000180b8       __ehhandler$??1?$QPtrList@VcOutputFile@@@@UAE@XZ 100190b8 f   alm_bncs_output.obj
 0001:000180b8       __ehhandler$??1?$QPtrList@VQPopupMenu@@@@UAE@XZ 100190b8 f   alm_bncs_output.obj
 0001:000180d3       __unwindfunclet$??1FileLoad_BncsSystem@alm_bncs_output@@UAE@XZ$0 100190d3 f   alm_bncs_output.obj
 0001:000180db       __ehhandler$??1FileLoad_BncsSystem@alm_bncs_output@@UAE@XZ 100190db f   alm_bncs_output.obj
 0001:000180f6       __unwindfunclet$??1QDockWindowList@@UAE@XZ$0 100190f6 f   alm_bncs_output.obj
 0001:000180ff       __unwindfunclet$??1QDockWindowList@@UAE@XZ$1 100190ff f   alm_bncs_output.obj
 0001:00018108       __ehhandler$??1QDockWindowList@@UAE@XZ 10019108 f   alm_bncs_output.obj
 0001:00018123       __unwindfunclet$??1QPopupMenuList@@UAE@XZ$0 10019123 f   alm_bncs_output.obj
 0001:0001812b       __ehhandler$??1QPopupMenuList@@UAE@XZ 1001912b f   alm_bncs_output.obj
 0001:00018146       __unwindfunclet$??1alm_bncs_output@@UAE@XZ$0 10019146 f   alm_bncs_output.obj
 0001:0001814e       __unwindfunclet$??1alm_bncs_output@@UAE@XZ$1 1001914e f   alm_bncs_output.obj
 0001:00018159       __unwindfunclet$??1alm_bncs_output@@UAE@XZ$2 10019159 f   alm_bncs_output.obj
 0001:00018168       __unwindfunclet$??1alm_bncs_output@@UAE@XZ$3 10019168 f   alm_bncs_output.obj
 0001:00018177       __unwindfunclet$??1alm_bncs_output@@UAE@XZ$4 10019177 f   alm_bncs_output.obj
 0001:00018186       __unwindfunclet$??1alm_bncs_output@@UAE@XZ$5 10019186 f   alm_bncs_output.obj
 0001:00018195       __unwindfunclet$??1alm_bncs_output@@UAE@XZ$6 10019195 f   alm_bncs_output.obj
 0001:000181a4       __unwindfunclet$??1alm_bncs_output@@UAE@XZ$7 100191a4 f   alm_bncs_output.obj
 0001:000181b3       __unwindfunclet$??1alm_bncs_output@@UAE@XZ$8 100191b3 f   alm_bncs_output.obj
 0001:000181c2       __unwindfunclet$??1alm_bncs_output@@UAE@XZ$9 100191c2 f   alm_bncs_output.obj
 0001:000181d0       __unwindfunclet$??1alm_bncs_output@@UAE@XZ$10 100191d0 f   alm_bncs_output.obj
 0001:000181de       __unwindfunclet$??1alm_bncs_output@@UAE@XZ$11 100191de f   alm_bncs_output.obj
 0001:000181ec       __unwindfunclet$??1alm_bncs_output@@UAE@XZ$12 100191ec f   alm_bncs_output.obj
 0001:000181fa       __unwindfunclet$??1alm_bncs_output@@UAE@XZ$13 100191fa f   alm_bncs_output.obj
 0001:00018208       __unwindfunclet$??1alm_bncs_output@@UAE@XZ$14 10019208 f   alm_bncs_output.obj
 0001:00018211       __unwindfunclet$??1alm_bncs_output@@UAE@XZ$15 10019211 f   alm_bncs_output.obj
 0001:0001821a       __ehhandler$??1alm_bncs_output@@UAE@XZ 1001921a f   alm_bncs_output.obj
 0001:00018235       __unwindfunclet$??1config_plugin_base@@UAE@XZ$0 10019235 f   alm_bncs_output.obj
 0001:0001823e       __unwindfunclet$??1config_plugin_base@@UAE@XZ$1 1001923e f   alm_bncs_output.obj
 0001:0001824a       __unwindfunclet$??1config_plugin_base@@UAE@XZ$2 1001924a f   alm_bncs_output.obj
 0001:00018256       __ehhandler$??1config_plugin_base@@UAE@XZ 10019256 f   alm_bncs_output.obj
 0001:00018271       __unwindfunclet$?EditProcess@alm_bncs_output@@QAEXXZ$0 10019271 f   alm_bncs_output.obj
 0001:0001827a       __unwindfunclet$?EditProcess@alm_bncs_output@@QAEXXZ$1 1001927a f   alm_bncs_output.obj
 0001:00018283       __unwindfunclet$?EditProcess@alm_bncs_output@@QAEXXZ$2 10019283 f   alm_bncs_output.obj
 0001:0001828c       __unwindfunclet$?EditProcess@alm_bncs_output@@QAEXXZ$3 1001928c f   alm_bncs_output.obj
 0001:00018295       __ehhandler$?EditProcess@alm_bncs_output@@QAEXXZ 10019295 f   alm_bncs_output.obj
 0001:000182b0       __unwindfunclet$?about@alm_bncs_output@@UAE?AVQString@@XZ$0 100192b0 f   alm_bncs_output.obj
 0001:000182ca       __ehhandler$?about@alm_bncs_output@@UAE?AVQString@@XZ 100192ca f   alm_bncs_output.obj
 0001:000182e5       __unwindfunclet$?about@config_plugin_base@@UAE?AVQString@@XZ$0 100192e5 f   alm_bncs_output.obj
 0001:000182ee       __unwindfunclet$?about@config_plugin_base@@UAE?AVQString@@XZ$1 100192ee f   alm_bncs_output.obj
 0001:00018308       __ehhandler$?about@config_plugin_base@@UAE?AVQString@@XZ 10019308 f   alm_bncs_output.obj
 0001:00018323       __unwindfunclet$?activate@alm_bncs_output@@UAEX_N@Z$0 10019323 f   alm_bncs_output.obj
 0001:0001832c       __unwindfunclet$?activate@alm_bncs_output@@UAEX_N@Z$3 1001932c f   alm_bncs_output.obj
 0001:00018335       __unwindfunclet$?activate@alm_bncs_output@@UAEX_N@Z$4 10019335 f   alm_bncs_output.obj
 0001:0001833f       __unwindfunclet$?activate@alm_bncs_output@@UAEX_N@Z$5 1001933f f   alm_bncs_output.obj
 0001:00018348       __unwindfunclet$?activate@alm_bncs_output@@UAEX_N@Z$7 10019348 f   alm_bncs_output.obj
 0001:00018351       __unwindfunclet$?activate@alm_bncs_output@@UAEX_N@Z$9 10019351 f   alm_bncs_output.obj
 0001:0001835a       __ehhandler$?activate@alm_bncs_output@@UAEX_N@Z 1001935a f   alm_bncs_output.obj
 0001:00018375       __unwindfunclet$?allocateCfgFileName@alm_bncs_output@@AAEXAAVQString@@0@Z$0 10019375 f   alm_bncs_output.obj
 0001:0001837e       __unwindfunclet$?allocateCfgFileName@alm_bncs_output@@AAEXAAVQString@@0@Z$1 1001937e f   alm_bncs_output.obj
 0001:00018387       __unwindfunclet$?allocateCfgFileName@alm_bncs_output@@AAEXAAVQString@@0@Z$2 10019387 f   alm_bncs_output.obj
 0001:00018390       __unwindfunclet$?allocateCfgFileName@alm_bncs_output@@AAEXAAVQString@@0@Z$3 10019390 f   alm_bncs_output.obj
 0001:00018399       __unwindfunclet$?allocateCfgFileName@alm_bncs_output@@AAEXAAVQString@@0@Z$4 10019399 f   alm_bncs_output.obj
 0001:000183a2       __unwindfunclet$?allocateCfgFileName@alm_bncs_output@@AAEXAAVQString@@0@Z$5 100193a2 f   alm_bncs_output.obj
 0001:000183ab       __unwindfunclet$?allocateCfgFileName@alm_bncs_output@@AAEXAAVQString@@0@Z$6 100193ab f   alm_bncs_output.obj
 0001:000183b4       __ehhandler$?allocateCfgFileName@alm_bncs_output@@AAEXAAVQString@@0@Z 100193b4 f   alm_bncs_output.obj
 0001:000183cf       __unwindfunclet$?allocateModuleName@alm_bncs_output@@AAEXAAVQString@@@Z$0 100193cf f   alm_bncs_output.obj
 0001:000183d8       __unwindfunclet$?allocateModuleName@alm_bncs_output@@AAEXAAVQString@@@Z$1 100193d8 f   alm_bncs_output.obj
 0001:000183e1       __ehhandler$?allocateModuleName@alm_bncs_output@@AAEXAAVQString@@@Z 100193e1 f   alm_bncs_output.obj
 0001:000183fc       __unwindfunclet$?apply@alm_bncs_output@@UAEXXZ$0 100193fc f   alm_bncs_output.obj
 0001:00018405       __unwindfunclet$?apply@alm_bncs_output@@UAEXXZ$2 10019405 f   alm_bncs_output.obj
 0001:0001840e       __unwindfunclet$?apply@alm_bncs_output@@UAEXXZ$4 1001940e f   alm_bncs_output.obj
 0001:00018417       __unwindfunclet$?apply@alm_bncs_output@@UAEXXZ$6 10019417 f   alm_bncs_output.obj
 0001:00018420       __ehhandler$?apply@alm_bncs_output@@UAEXXZ 10019420 f   alm_bncs_output.obj
 0001:0001843b       __unwindfunclet$?applyTemplates@alm_bncs_output@@QAEXXZ$1 1001943b f   alm_bncs_output.obj
 0001:00018444       __unwindfunclet$?applyTemplates@alm_bncs_output@@QAEXXZ$2 10019444 f   alm_bncs_output.obj
 0001:0001844d       __unwindfunclet$?applyTemplates@alm_bncs_output@@QAEXXZ$3 1001944d f   alm_bncs_output.obj
 0001:00018456       __unwindfunclet$?applyTemplates@alm_bncs_output@@QAEXXZ$4 10019456 f   alm_bncs_output.obj
 0001:0001845f       __unwindfunclet$?applyTemplates@alm_bncs_output@@QAEXXZ$5 1001945f f   alm_bncs_output.obj
 0001:00018468       __unwindfunclet$?applyTemplates@alm_bncs_output@@QAEXXZ$6 10019468 f   alm_bncs_output.obj
 0001:00018470       __unwindfunclet$?applyTemplates@alm_bncs_output@@QAEXXZ$7 10019470 f   alm_bncs_output.obj
 0001:00018479       __unwindfunclet$?applyTemplates@alm_bncs_output@@QAEXXZ$8 10019479 f   alm_bncs_output.obj
 0001:00018482       __unwindfunclet$?applyTemplates@alm_bncs_output@@QAEXXZ$10 10019482 f   alm_bncs_output.obj
 0001:0001848b       __unwindfunclet$?applyTemplates@alm_bncs_output@@QAEXXZ$11 1001948b f   alm_bncs_output.obj
 0001:00018494       __unwindfunclet$?applyTemplates@alm_bncs_output@@QAEXXZ$12 10019494 f   alm_bncs_output.obj
 0001:0001849d       __unwindfunclet$?applyTemplates@alm_bncs_output@@QAEXXZ$13 1001949d f   alm_bncs_output.obj
 0001:000184a6       __unwindfunclet$?applyTemplates@alm_bncs_output@@QAEXXZ$14 100194a6 f   alm_bncs_output.obj
 0001:000184af       __unwindfunclet$?applyTemplates@alm_bncs_output@@QAEXXZ$15 100194af f   alm_bncs_output.obj
 0001:000184b8       __unwindfunclet$?applyTemplates@alm_bncs_output@@QAEXXZ$16 100194b8 f   alm_bncs_output.obj
 0001:000184c1       __unwindfunclet$?applyTemplates@alm_bncs_output@@QAEXXZ$17 100194c1 f   alm_bncs_output.obj
 0001:000184ca       __ehhandler$?applyTemplates@alm_bncs_output@@QAEXXZ 100194ca f   alm_bncs_output.obj
 0001:000184e5       __unwindfunclet$?changeDevType@alm_bncs_output@@AAEXABVQString@@0@Z$0 100194e5 f   alm_bncs_output.obj
 0001:000184ee       __unwindfunclet$?changeDevType@alm_bncs_output@@AAEXABVQString@@0@Z$1 100194ee f   alm_bncs_output.obj
 0001:000184f7       __unwindfunclet$?changeDevType@alm_bncs_output@@AAEXABVQString@@0@Z$2 100194f7 f   alm_bncs_output.obj
 0001:00018500       __unwindfunclet$?changeDevType@alm_bncs_output@@AAEXABVQString@@0@Z$3 10019500 f   alm_bncs_output.obj
 0001:00018509       __ehhandler$?changeDevType@alm_bncs_output@@AAEXABVQString@@0@Z 10019509 f   alm_bncs_output.obj
 0001:00018524       __unwindfunclet$?changeDevTypeDevicetypes@alm_bncs_output@@AAEXABVQString@@0@Z$0 10019524 f   alm_bncs_output.obj
 0001:0001852d       __unwindfunclet$?changeDevTypeDevicetypes@alm_bncs_output@@AAEXABVQString@@0@Z$1 1001952d f   alm_bncs_output.obj
 0001:00018536       __unwindfunclet$?changeDevTypeDevicetypes@alm_bncs_output@@AAEXABVQString@@0@Z$2 10019536 f   alm_bncs_output.obj
 0001:0001853f       __unwindfunclet$?changeDevTypeDevicetypes@alm_bncs_output@@AAEXABVQString@@0@Z$3 1001953f f   alm_bncs_output.obj
 0001:00018548       __unwindfunclet$?changeDevTypeDevicetypes@alm_bncs_output@@AAEXABVQString@@0@Z$4 10019548 f   alm_bncs_output.obj
 0001:00018551       __unwindfunclet$?changeDevTypeDevicetypes@alm_bncs_output@@AAEXABVQString@@0@Z$5 10019551 f   alm_bncs_output.obj
 0001:0001855a       __unwindfunclet$?changeDevTypeDevicetypes@alm_bncs_output@@AAEXABVQString@@0@Z$6 1001955a f   alm_bncs_output.obj
 0001:00018566       __unwindfunclet$?changeDevTypeDevicetypes@alm_bncs_output@@AAEXABVQString@@0@Z$7 10019566 f   alm_bncs_output.obj
 0001:0001856f       __unwindfunclet$?changeDevTypeDevicetypes@alm_bncs_output@@AAEXABVQString@@0@Z$8 1001956f f   alm_bncs_output.obj
 0001:00018578       __unwindfunclet$?changeDevTypeDevicetypes@alm_bncs_output@@AAEXABVQString@@0@Z$9 10019578 f   alm_bncs_output.obj
 0001:00018581       __unwindfunclet$?changeDevTypeDevicetypes@alm_bncs_output@@AAEXABVQString@@0@Z$10 10019581 f   alm_bncs_output.obj
 0001:0001858a       __unwindfunclet$?changeDevTypeDevicetypes@alm_bncs_output@@AAEXABVQString@@0@Z$11 1001958a f   alm_bncs_output.obj
 0001:00018593       __unwindfunclet$?changeDevTypeDevicetypes@alm_bncs_output@@AAEXABVQString@@0@Z$12 10019593 f   alm_bncs_output.obj
 0001:0001859c       __unwindfunclet$?changeDevTypeDevicetypes@alm_bncs_output@@AAEXABVQString@@0@Z$13 1001959c f   alm_bncs_output.obj
 0001:000185a4       __unwindfunclet$?changeDevTypeDevicetypes@alm_bncs_output@@AAEXABVQString@@0@Z$14 100195a4 f   alm_bncs_output.obj
 0001:000185ad       __unwindfunclet$?changeDevTypeDevicetypes@alm_bncs_output@@AAEXABVQString@@0@Z$15 100195ad f   alm_bncs_output.obj
 0001:000185b6       __unwindfunclet$?changeDevTypeDevicetypes@alm_bncs_output@@AAEXABVQString@@0@Z$16 100195b6 f   alm_bncs_output.obj
 0001:000185bf       __unwindfunclet$?changeDevTypeDevicetypes@alm_bncs_output@@AAEXABVQString@@0@Z$17 100195bf f   alm_bncs_output.obj
 0001:000185c8       __unwindfunclet$?changeDevTypeDevicetypes@alm_bncs_output@@AAEXABVQString@@0@Z$18 100195c8 f   alm_bncs_output.obj
 0001:000185d4       __unwindfunclet$?changeDevTypeDevicetypes@alm_bncs_output@@AAEXABVQString@@0@Z$19 100195d4 f   alm_bncs_output.obj
 0001:000185dd       __unwindfunclet$?changeDevTypeDevicetypes@alm_bncs_output@@AAEXABVQString@@0@Z$20 100195dd f   alm_bncs_output.obj
 0001:000185e6       __unwindfunclet$?changeDevTypeDevicetypes@alm_bncs_output@@AAEXABVQString@@0@Z$21 100195e6 f   alm_bncs_output.obj
 0001:000185ef       __unwindfunclet$?changeDevTypeDevicetypes@alm_bncs_output@@AAEXABVQString@@0@Z$22 100195ef f   alm_bncs_output.obj
 0001:000185f8       __unwindfunclet$?changeDevTypeDevicetypes@alm_bncs_output@@AAEXABVQString@@0@Z$23 100195f8 f   alm_bncs_output.obj
 0001:00018601       __unwindfunclet$?changeDevTypeDevicetypes@alm_bncs_output@@AAEXABVQString@@0@Z$24 10019601 f   alm_bncs_output.obj
 0001:0001860a       __unwindfunclet$?changeDevTypeDevicetypes@alm_bncs_output@@AAEXABVQString@@0@Z$25 1001960a f   alm_bncs_output.obj
 0001:00018613       __unwindfunclet$?changeDevTypeDevicetypes@alm_bncs_output@@AAEXABVQString@@0@Z$26 10019613 f   alm_bncs_output.obj
 0001:0001861c       __unwindfunclet$?changeDevTypeDevicetypes@alm_bncs_output@@AAEXABVQString@@0@Z$27 1001961c f   alm_bncs_output.obj
 0001:00018625       __unwindfunclet$?changeDevTypeDevicetypes@alm_bncs_output@@AAEXABVQString@@0@Z$28 10019625 f   alm_bncs_output.obj
 0001:0001862e       __unwindfunclet$?changeDevTypeDevicetypes@alm_bncs_output@@AAEXABVQString@@0@Z$29 1001962e f   alm_bncs_output.obj
 0001:00018637       __unwindfunclet$?changeDevTypeDevicetypes@alm_bncs_output@@AAEXABVQString@@0@Z$30 10019637 f   alm_bncs_output.obj
 0001:00018640       __unwindfunclet$?changeDevTypeDevicetypes@alm_bncs_output@@AAEXABVQString@@0@Z$31 10019640 f   alm_bncs_output.obj
 0001:00018649       __unwindfunclet$?changeDevTypeDevicetypes@alm_bncs_output@@AAEXABVQString@@0@Z$32 10019649 f   alm_bncs_output.obj
 0001:00018652       __unwindfunclet$?changeDevTypeDevicetypes@alm_bncs_output@@AAEXABVQString@@0@Z$33 10019652 f   alm_bncs_output.obj
 0001:0001865b       __unwindfunclet$?changeDevTypeDevicetypes@alm_bncs_output@@AAEXABVQString@@0@Z$34 1001965b f   alm_bncs_output.obj
 0001:00018664       __unwindfunclet$?changeDevTypeDevicetypes@alm_bncs_output@@AAEXABVQString@@0@Z$35 10019664 f   alm_bncs_output.obj
 0001:0001866d       __unwindfunclet$?changeDevTypeDevicetypes@alm_bncs_output@@AAEXABVQString@@0@Z$36 1001966d f   alm_bncs_output.obj
 0001:00018676       __unwindfunclet$?changeDevTypeDevicetypes@alm_bncs_output@@AAEXABVQString@@0@Z$37 10019676 f   alm_bncs_output.obj
 0001:0001867f       __unwindfunclet$?changeDevTypeDevicetypes@alm_bncs_output@@AAEXABVQString@@0@Z$38 1001967f f   alm_bncs_output.obj
 0001:00018688       __unwindfunclet$?changeDevTypeDevicetypes@alm_bncs_output@@AAEXABVQString@@0@Z$39 10019688 f   alm_bncs_output.obj
 0001:00018691       __unwindfunclet$?changeDevTypeDevicetypes@alm_bncs_output@@AAEXABVQString@@0@Z$40 10019691 f   alm_bncs_output.obj
 0001:0001869a       __ehhandler$?changeDevTypeDevicetypes@alm_bncs_output@@AAEXABVQString@@0@Z 1001969a f   alm_bncs_output.obj
 0001:000186b8       __unwindfunclet$?changeDevTypeInstances@alm_bncs_output@@AAEXABVQString@@0@Z$0 100196b8 f   alm_bncs_output.obj
 0001:000186c4       __unwindfunclet$?changeDevTypeInstances@alm_bncs_output@@AAEXABVQString@@0@Z$1 100196c4 f   alm_bncs_output.obj
 0001:000186cd       __unwindfunclet$?changeDevTypeInstances@alm_bncs_output@@AAEXABVQString@@0@Z$2 100196cd f   alm_bncs_output.obj
 0001:000186d9       __unwindfunclet$?changeDevTypeInstances@alm_bncs_output@@AAEXABVQString@@0@Z$3 100196d9 f   alm_bncs_output.obj
 0001:000186e2       __unwindfunclet$?changeDevTypeInstances@alm_bncs_output@@AAEXABVQString@@0@Z$4 100196e2 f   alm_bncs_output.obj
 0001:000186eb       __unwindfunclet$?changeDevTypeInstances@alm_bncs_output@@AAEXABVQString@@0@Z$5 100196eb f   alm_bncs_output.obj
 0001:000186f4       __unwindfunclet$?changeDevTypeInstances@alm_bncs_output@@AAEXABVQString@@0@Z$6 100196f4 f   alm_bncs_output.obj
 0001:000186fd       __unwindfunclet$?changeDevTypeInstances@alm_bncs_output@@AAEXABVQString@@0@Z$7 100196fd f   alm_bncs_output.obj
 0001:00018706       __unwindfunclet$?changeDevTypeInstances@alm_bncs_output@@AAEXABVQString@@0@Z$8 10019706 f   alm_bncs_output.obj
 0001:0001870f       __unwindfunclet$?changeDevTypeInstances@alm_bncs_output@@AAEXABVQString@@0@Z$9 1001970f f   alm_bncs_output.obj
 0001:0001871b       __unwindfunclet$?changeDevTypeInstances@alm_bncs_output@@AAEXABVQString@@0@Z$10 1001971b f   alm_bncs_output.obj
 0001:00018724       __unwindfunclet$?changeDevTypeInstances@alm_bncs_output@@AAEXABVQString@@0@Z$11 10019724 f   alm_bncs_output.obj
 0001:0001872d       __unwindfunclet$?changeDevTypeInstances@alm_bncs_output@@AAEXABVQString@@0@Z$12 1001972d f   alm_bncs_output.obj
 0001:00018736       __unwindfunclet$?changeDevTypeInstances@alm_bncs_output@@AAEXABVQString@@0@Z$13 10019736 f   alm_bncs_output.obj
 0001:0001873f       __unwindfunclet$?changeDevTypeInstances@alm_bncs_output@@AAEXABVQString@@0@Z$14 1001973f f   alm_bncs_output.obj
 0001:00018748       __unwindfunclet$?changeDevTypeInstances@alm_bncs_output@@AAEXABVQString@@0@Z$15 10019748 f   alm_bncs_output.obj
 0001:00018754       __unwindfunclet$?changeDevTypeInstances@alm_bncs_output@@AAEXABVQString@@0@Z$16 10019754 f   alm_bncs_output.obj
 0001:0001875d       __unwindfunclet$?changeDevTypeInstances@alm_bncs_output@@AAEXABVQString@@0@Z$17 1001975d f   alm_bncs_output.obj
 0001:00018769       __unwindfunclet$?changeDevTypeInstances@alm_bncs_output@@AAEXABVQString@@0@Z$18 10019769 f   alm_bncs_output.obj
 0001:00018772       __unwindfunclet$?changeDevTypeInstances@alm_bncs_output@@AAEXABVQString@@0@Z$19 10019772 f   alm_bncs_output.obj
 0001:0001877b       __unwindfunclet$?changeDevTypeInstances@alm_bncs_output@@AAEXABVQString@@0@Z$20 1001977b f   alm_bncs_output.obj
 0001:00018784       __unwindfunclet$?changeDevTypeInstances@alm_bncs_output@@AAEXABVQString@@0@Z$21 10019784 f   alm_bncs_output.obj
 0001:0001878d       __unwindfunclet$?changeDevTypeInstances@alm_bncs_output@@AAEXABVQString@@0@Z$22 1001978d f   alm_bncs_output.obj
 0001:00018796       __unwindfunclet$?changeDevTypeInstances@alm_bncs_output@@AAEXABVQString@@0@Z$23 10019796 f   alm_bncs_output.obj
 0001:0001879f       __unwindfunclet$?changeDevTypeInstances@alm_bncs_output@@AAEXABVQString@@0@Z$24 1001979f f   alm_bncs_output.obj
 0001:000187a8       __unwindfunclet$?changeDevTypeInstances@alm_bncs_output@@AAEXABVQString@@0@Z$25 100197a8 f   alm_bncs_output.obj
 0001:000187b1       __unwindfunclet$?changeDevTypeInstances@alm_bncs_output@@AAEXABVQString@@0@Z$26 100197b1 f   alm_bncs_output.obj
 0001:000187ba       __unwindfunclet$?changeDevTypeInstances@alm_bncs_output@@AAEXABVQString@@0@Z$27 100197ba f   alm_bncs_output.obj
 0001:000187c3       __unwindfunclet$?changeDevTypeInstances@alm_bncs_output@@AAEXABVQString@@0@Z$28 100197c3 f   alm_bncs_output.obj
 0001:000187cf       __unwindfunclet$?changeDevTypeInstances@alm_bncs_output@@AAEXABVQString@@0@Z$29 100197cf f   alm_bncs_output.obj
 0001:000187d8       __unwindfunclet$?changeDevTypeInstances@alm_bncs_output@@AAEXABVQString@@0@Z$30 100197d8 f   alm_bncs_output.obj
 0001:000187e1       __unwindfunclet$?changeDevTypeInstances@alm_bncs_output@@AAEXABVQString@@0@Z$31 100197e1 f   alm_bncs_output.obj
 0001:000187ea       __unwindfunclet$?changeDevTypeInstances@alm_bncs_output@@AAEXABVQString@@0@Z$32 100197ea f   alm_bncs_output.obj
 0001:000187f3       __unwindfunclet$?changeDevTypeInstances@alm_bncs_output@@AAEXABVQString@@0@Z$33 100197f3 f   alm_bncs_output.obj
 0001:000187fc       __unwindfunclet$?changeDevTypeInstances@alm_bncs_output@@AAEXABVQString@@0@Z$34 100197fc f   alm_bncs_output.obj
 0001:00018805       __unwindfunclet$?changeDevTypeInstances@alm_bncs_output@@AAEXABVQString@@0@Z$35 10019805 f   alm_bncs_output.obj
 0001:0001880e       __unwindfunclet$?changeDevTypeInstances@alm_bncs_output@@AAEXABVQString@@0@Z$36 1001980e f   alm_bncs_output.obj
 0001:00018817       __unwindfunclet$?changeDevTypeInstances@alm_bncs_output@@AAEXABVQString@@0@Z$37 10019817 f   alm_bncs_output.obj
 0001:00018820       __unwindfunclet$?changeDevTypeInstances@alm_bncs_output@@AAEXABVQString@@0@Z$38 10019820 f   alm_bncs_output.obj
 0001:00018829       __unwindfunclet$?changeDevTypeInstances@alm_bncs_output@@AAEXABVQString@@0@Z$39 10019829 f   alm_bncs_output.obj
 0001:00018832       __unwindfunclet$?changeDevTypeInstances@alm_bncs_output@@AAEXABVQString@@0@Z$40 10019832 f   alm_bncs_output.obj
 0001:0001883b       __unwindfunclet$?changeDevTypeInstances@alm_bncs_output@@AAEXABVQString@@0@Z$41 1001983b f   alm_bncs_output.obj
 0001:00018844       __unwindfunclet$?changeDevTypeInstances@alm_bncs_output@@AAEXABVQString@@0@Z$42 10019844 f   alm_bncs_output.obj
 0001:0001884d       __unwindfunclet$?changeDevTypeInstances@alm_bncs_output@@AAEXABVQString@@0@Z$43 1001984d f   alm_bncs_output.obj
 0001:00018856       __unwindfunclet$?changeDevTypeInstances@alm_bncs_output@@AAEXABVQString@@0@Z$44 10019856 f   alm_bncs_output.obj
 0001:0001885f       __unwindfunclet$?changeDevTypeInstances@alm_bncs_output@@AAEXABVQString@@0@Z$45 1001985f f   alm_bncs_output.obj
 0001:00018868       __unwindfunclet$?changeDevTypeInstances@alm_bncs_output@@AAEXABVQString@@0@Z$46 10019868 f   alm_bncs_output.obj
 0001:00018871       __unwindfunclet$?changeDevTypeInstances@alm_bncs_output@@AAEXABVQString@@0@Z$47 10019871 f   alm_bncs_output.obj
 0001:0001887a       __unwindfunclet$?changeDevTypeInstances@alm_bncs_output@@AAEXABVQString@@0@Z$48 1001987a f   alm_bncs_output.obj
 0001:00018883       __unwindfunclet$?changeDevTypeInstances@alm_bncs_output@@AAEXABVQString@@0@Z$49 10019883 f   alm_bncs_output.obj
 0001:0001888c       __unwindfunclet$?changeDevTypeInstances@alm_bncs_output@@AAEXABVQString@@0@Z$50 1001988c f   alm_bncs_output.obj
 0001:00018895       __ehhandler$?changeDevTypeInstances@alm_bncs_output@@AAEXABVQString@@0@Z 10019895 f   alm_bncs_output.obj
 0001:000188b3       __unwindfunclet$?closeEvent@alm_bncs_output@@UAEXPAVQCloseEvent@@@Z$0 100198b3 f   alm_bncs_output.obj
 0001:000188bc       __unwindfunclet$?closeEvent@alm_bncs_output@@UAEXPAVQCloseEvent@@@Z$2 100198bc f   alm_bncs_output.obj
 0001:000188c5       __unwindfunclet$?closeEvent@alm_bncs_output@@UAEXPAVQCloseEvent@@@Z$4 100198c5 f   alm_bncs_output.obj
 0001:000188ce       __unwindfunclet$?closeEvent@alm_bncs_output@@UAEXPAVQCloseEvent@@@Z$6 100198ce f   alm_bncs_output.obj
 0001:000188d7       __ehhandler$?closeEvent@alm_bncs_output@@UAEXPAVQCloseEvent@@@Z 100198d7 f   alm_bncs_output.obj
 0001:000188f2       __unwindfunclet$??0?$QMapPrivate@VQString@@W4ESection@@@@QAE@PBV0@@Z$0 100198f2 f   alm_bncs_output.obj
 0001:000188f2       __unwindfunclet$?copy@?$QMapPrivate@VQString@@W4ESection@@@@QAEPAU?$QMapNode@VQString@@W4ESection@@@@PAU2@@Z$0 100198f2 f   alm_bncs_output.obj
 0001:000188fc       __ehhandler$?copy@?$QMapPrivate@VQString@@W4ESection@@@@QAEPAU?$QMapNode@VQString@@W4ESection@@@@PAU2@@Z 100198fc f   alm_bncs_output.obj
 0001:000188fc       __ehhandler$??0?$QMapPrivate@VQString@@W4ESection@@@@QAE@PBV0@@Z 100198fc f   alm_bncs_output.obj
 0001:00018917       __unwindfunclet$?createEmptyDomDoc@alm_bncs_output@@EBEXABVQString@@0AAVQDomDocument@@@Z$0 10019917 f   alm_bncs_output.obj
 0001:00018920       __unwindfunclet$?createEmptyDomDoc@alm_bncs_output@@EBEXABVQString@@0AAVQDomDocument@@@Z$1 10019920 f   alm_bncs_output.obj
 0001:00018929       __unwindfunclet$?createEmptyDomDoc@alm_bncs_output@@EBEXABVQString@@0AAVQDomDocument@@@Z$2 10019929 f   alm_bncs_output.obj
 0001:00018932       __unwindfunclet$?createEmptyDomDoc@alm_bncs_output@@EBEXABVQString@@0AAVQDomDocument@@@Z$3 10019932 f   alm_bncs_output.obj
 0001:0001893b       __unwindfunclet$?createEmptyDomDoc@alm_bncs_output@@EBEXABVQString@@0AAVQDomDocument@@@Z$4 1001993b f   alm_bncs_output.obj
 0001:00018944       __unwindfunclet$?createEmptyDomDoc@alm_bncs_output@@EBEXABVQString@@0AAVQDomDocument@@@Z$5 10019944 f   alm_bncs_output.obj
 0001:0001894d       __unwindfunclet$?createEmptyDomDoc@alm_bncs_output@@EBEXABVQString@@0AAVQDomDocument@@@Z$6 1001994d f   alm_bncs_output.obj
 0001:00018956       __unwindfunclet$?createEmptyDomDoc@alm_bncs_output@@EBEXABVQString@@0AAVQDomDocument@@@Z$8 10019956 f   alm_bncs_output.obj
 0001:0001895f       __ehhandler$?createEmptyDomDoc@alm_bncs_output@@EBEXABVQString@@0AAVQDomDocument@@@Z 1001995f f   alm_bncs_output.obj
 0001:0001897a       __unwindfunclet$?deleteAndLockDevDescs@alm_bncs_output@@AAEXABVQString@@0@Z$0 1001997a f   alm_bncs_output.obj
 0001:00018983       __unwindfunclet$?deleteAndLockDevDescs@alm_bncs_output@@AAEXABVQString@@0@Z$1 10019983 f   alm_bncs_output.obj
 0001:0001898c       __unwindfunclet$?deleteAndLockDevDescs@alm_bncs_output@@AAEXABVQString@@0@Z$2 1001998c f   alm_bncs_output.obj
 0001:00018995       __unwindfunclet$?deleteAndLockDevDescs@alm_bncs_output@@AAEXABVQString@@0@Z$3 10019995 f   alm_bncs_output.obj
 0001:0001899e       __unwindfunclet$?deleteAndLockDevDescs@alm_bncs_output@@AAEXABVQString@@0@Z$4 1001999e f   alm_bncs_output.obj
 0001:000189a7       __unwindfunclet$?deleteAndLockDevDescs@alm_bncs_output@@AAEXABVQString@@0@Z$5 100199a7 f   alm_bncs_output.obj
 0001:000189b0       __unwindfunclet$?deleteAndLockDevDescs@alm_bncs_output@@AAEXABVQString@@0@Z$6 100199b0 f   alm_bncs_output.obj
 0001:000189b9       __unwindfunclet$?deleteAndLockDevDescs@alm_bncs_output@@AAEXABVQString@@0@Z$7 100199b9 f   alm_bncs_output.obj
 0001:000189c5       __unwindfunclet$?deleteAndLockDevDescs@alm_bncs_output@@AAEXABVQString@@0@Z$8 100199c5 f   alm_bncs_output.obj
 0001:000189ce       __unwindfunclet$?deleteAndLockDevDescs@alm_bncs_output@@AAEXABVQString@@0@Z$9 100199ce f   alm_bncs_output.obj
 0001:000189d7       __unwindfunclet$?deleteAndLockDevDescs@alm_bncs_output@@AAEXABVQString@@0@Z$10 100199d7 f   alm_bncs_output.obj
 0001:000189e0       __unwindfunclet$?deleteAndLockDevDescs@alm_bncs_output@@AAEXABVQString@@0@Z$11 100199e0 f   alm_bncs_output.obj
 0001:000189e9       __unwindfunclet$?deleteAndLockDevDescs@alm_bncs_output@@AAEXABVQString@@0@Z$12 100199e9 f   alm_bncs_output.obj
 0001:000189f2       __unwindfunclet$?deleteAndLockDevDescs@alm_bncs_output@@AAEXABVQString@@0@Z$13 100199f2 f   alm_bncs_output.obj
 0001:000189fb       __unwindfunclet$?deleteAndLockDevDescs@alm_bncs_output@@AAEXABVQString@@0@Z$14 100199fb f   alm_bncs_output.obj
 0001:00018a04       __unwindfunclet$?deleteAndLockDevDescs@alm_bncs_output@@AAEXABVQString@@0@Z$15 10019a04 f   alm_bncs_output.obj
 0001:00018a0d       __unwindfunclet$?deleteAndLockDevDescs@alm_bncs_output@@AAEXABVQString@@0@Z$16 10019a0d f   alm_bncs_output.obj
 0001:00018a16       __unwindfunclet$?deleteAndLockDevDescs@alm_bncs_output@@AAEXABVQString@@0@Z$17 10019a16 f   alm_bncs_output.obj
 0001:00018a1e       __unwindfunclet$?deleteAndLockDevDescs@alm_bncs_output@@AAEXABVQString@@0@Z$18 10019a1e f   alm_bncs_output.obj
 0001:00018a27       __unwindfunclet$?deleteAndLockDevDescs@alm_bncs_output@@AAEXABVQString@@0@Z$19 10019a27 f   alm_bncs_output.obj
 0001:00018a30       __unwindfunclet$?deleteAndLockDevDescs@alm_bncs_output@@AAEXABVQString@@0@Z$20 10019a30 f   alm_bncs_output.obj
 0001:00018a39       __unwindfunclet$?deleteAndLockDevDescs@alm_bncs_output@@AAEXABVQString@@0@Z$21 10019a39 f   alm_bncs_output.obj
 0001:00018a42       __unwindfunclet$?deleteAndLockDevDescs@alm_bncs_output@@AAEXABVQString@@0@Z$22 10019a42 f   alm_bncs_output.obj
 0001:00018a4b       __unwindfunclet$?deleteAndLockDevDescs@alm_bncs_output@@AAEXABVQString@@0@Z$23 10019a4b f   alm_bncs_output.obj
 0001:00018a54       __unwindfunclet$?deleteAndLockDevDescs@alm_bncs_output@@AAEXABVQString@@0@Z$24 10019a54 f   alm_bncs_output.obj
 0001:00018a5d       __unwindfunclet$?deleteAndLockDevDescs@alm_bncs_output@@AAEXABVQString@@0@Z$25 10019a5d f   alm_bncs_output.obj
 0001:00018a66       __unwindfunclet$?deleteAndLockDevDescs@alm_bncs_output@@AAEXABVQString@@0@Z$26 10019a66 f   alm_bncs_output.obj
 0001:00018a6f       __unwindfunclet$?deleteAndLockDevDescs@alm_bncs_output@@AAEXABVQString@@0@Z$27 10019a6f f   alm_bncs_output.obj
 0001:00018a78       __unwindfunclet$?deleteAndLockDevDescs@alm_bncs_output@@AAEXABVQString@@0@Z$28 10019a78 f   alm_bncs_output.obj
 0001:00018a84       __unwindfunclet$?deleteAndLockDevDescs@alm_bncs_output@@AAEXABVQString@@0@Z$29 10019a84 f   alm_bncs_output.obj
 0001:00018a8d       __unwindfunclet$?deleteAndLockDevDescs@alm_bncs_output@@AAEXABVQString@@0@Z$30 10019a8d f   alm_bncs_output.obj
 0001:00018a96       __unwindfunclet$?deleteAndLockDevDescs@alm_bncs_output@@AAEXABVQString@@0@Z$31 10019a96 f   alm_bncs_output.obj
 0001:00018a9f       __unwindfunclet$?deleteAndLockDevDescs@alm_bncs_output@@AAEXABVQString@@0@Z$32 10019a9f f   alm_bncs_output.obj
 0001:00018aa8       __unwindfunclet$?deleteAndLockDevDescs@alm_bncs_output@@AAEXABVQString@@0@Z$33 10019aa8 f   alm_bncs_output.obj
 0001:00018ab1       __unwindfunclet$?deleteAndLockDevDescs@alm_bncs_output@@AAEXABVQString@@0@Z$34 10019ab1 f   alm_bncs_output.obj
 0001:00018aba       __unwindfunclet$?deleteAndLockDevDescs@alm_bncs_output@@AAEXABVQString@@0@Z$35 10019aba f   alm_bncs_output.obj
 0001:00018ac3       __unwindfunclet$?deleteAndLockDevDescs@alm_bncs_output@@AAEXABVQString@@0@Z$36 10019ac3 f   alm_bncs_output.obj
 0001:00018acc       __ehhandler$?deleteAndLockDevDescs@alm_bncs_output@@AAEXABVQString@@0@Z 10019acc f   alm_bncs_output.obj
 0001:00018aea       __unwindfunclet$?doDone@alm_bncs_output@@AAEXPAVresponse@@@Z$0 10019aea f   alm_bncs_output.obj
 0001:00018af3       __unwindfunclet$?doDone@alm_bncs_output@@AAEXPAVresponse@@@Z$1 10019af3 f   alm_bncs_output.obj
 0001:00018afc       __unwindfunclet$?doDone@alm_bncs_output@@AAEXPAVresponse@@@Z$2 10019afc f   alm_bncs_output.obj
 0001:00018b05       __unwindfunclet$?doDone@alm_bncs_output@@AAEXPAVresponse@@@Z$3 10019b05 f   alm_bncs_output.obj
 0001:00018b0e       __unwindfunclet$?doDone@alm_bncs_output@@AAEXPAVresponse@@@Z$4 10019b0e f   alm_bncs_output.obj
 0001:00018b17       __unwindfunclet$?doDone@alm_bncs_output@@AAEXPAVresponse@@@Z$5 10019b17 f   alm_bncs_output.obj
 0001:00018b20       __unwindfunclet$?doDone@alm_bncs_output@@AAEXPAVresponse@@@Z$6 10019b20 f   alm_bncs_output.obj
 0001:00018b29       __unwindfunclet$?doDone@alm_bncs_output@@AAEXPAVresponse@@@Z$7 10019b29 f   alm_bncs_output.obj
 0001:00018b32       __unwindfunclet$?doDone@alm_bncs_output@@AAEXPAVresponse@@@Z$8 10019b32 f   alm_bncs_output.obj
 0001:00018b3b       __unwindfunclet$?doDone@alm_bncs_output@@AAEXPAVresponse@@@Z$9 10019b3b f   alm_bncs_output.obj
 0001:00018b44       __unwindfunclet$?doDone@alm_bncs_output@@AAEXPAVresponse@@@Z$10 10019b44 f   alm_bncs_output.obj
 0001:00018b4d       __unwindfunclet$?doDone@alm_bncs_output@@AAEXPAVresponse@@@Z$11 10019b4d f   alm_bncs_output.obj
 0001:00018b56       __unwindfunclet$?doDone@alm_bncs_output@@AAEXPAVresponse@@@Z$12 10019b56 f   alm_bncs_output.obj
 0001:00018b5f       __unwindfunclet$?doDone@alm_bncs_output@@AAEXPAVresponse@@@Z$13 10019b5f f   alm_bncs_output.obj
 0001:00018b68       __unwindfunclet$?doDone@alm_bncs_output@@AAEXPAVresponse@@@Z$14 10019b68 f   alm_bncs_output.obj
 0001:00018b71       __unwindfunclet$?doDone@alm_bncs_output@@AAEXPAVresponse@@@Z$15 10019b71 f   alm_bncs_output.obj
 0001:00018b7a       __unwindfunclet$?doDone@alm_bncs_output@@AAEXPAVresponse@@@Z$16 10019b7a f   alm_bncs_output.obj
 0001:00018b83       __unwindfunclet$?doDone@alm_bncs_output@@AAEXPAVresponse@@@Z$17 10019b83 f   alm_bncs_output.obj
 0001:00018b8c       __ehhandler$?doDone@alm_bncs_output@@AAEXPAVresponse@@@Z 10019b8c f   alm_bncs_output.obj
 0001:00018ba7       __unwindfunclet$?doDownloadRead@alm_bncs_output@@AAEXPAVresponse@@@Z$0 10019ba7 f   alm_bncs_output.obj
 0001:00018bb3       __unwindfunclet$?doDownloadRead@alm_bncs_output@@AAEXPAVresponse@@@Z$1 10019bb3 f   alm_bncs_output.obj
 0001:00018bbf       __unwindfunclet$?doDownloadRead@alm_bncs_output@@AAEXPAVresponse@@@Z$2 10019bbf f   alm_bncs_output.obj
 0001:00018bcb       __unwindfunclet$?doDownloadRead@alm_bncs_output@@AAEXPAVresponse@@@Z$3 10019bcb f   alm_bncs_output.obj
 0001:00018bd7       __unwindfunclet$?doDownloadRead@alm_bncs_output@@AAEXPAVresponse@@@Z$4 10019bd7 f   alm_bncs_output.obj
 0001:00018be3       __unwindfunclet$?doDownloadRead@alm_bncs_output@@AAEXPAVresponse@@@Z$5 10019be3 f   alm_bncs_output.obj
 0001:00018bef       __unwindfunclet$?doDownloadRead@alm_bncs_output@@AAEXPAVresponse@@@Z$6 10019bef f   alm_bncs_output.obj
 0001:00018bfb       __unwindfunclet$?doDownloadRead@alm_bncs_output@@AAEXPAVresponse@@@Z$7 10019bfb f   alm_bncs_output.obj
 0001:00018c07       __unwindfunclet$?doDownloadRead@alm_bncs_output@@AAEXPAVresponse@@@Z$8 10019c07 f   alm_bncs_output.obj
 0001:00018c13       __unwindfunclet$?doDownloadRead@alm_bncs_output@@AAEXPAVresponse@@@Z$9 10019c13 f   alm_bncs_output.obj
 0001:00018c1f       __unwindfunclet$?doDownloadRead@alm_bncs_output@@AAEXPAVresponse@@@Z$10 10019c1f f   alm_bncs_output.obj
 0001:00018c2b       __unwindfunclet$?doDownloadRead@alm_bncs_output@@AAEXPAVresponse@@@Z$11 10019c2b f   alm_bncs_output.obj
 0001:00018c37       __unwindfunclet$?doDownloadRead@alm_bncs_output@@AAEXPAVresponse@@@Z$12 10019c37 f   alm_bncs_output.obj
 0001:00018c43       __unwindfunclet$?doDownloadRead@alm_bncs_output@@AAEXPAVresponse@@@Z$13 10019c43 f   alm_bncs_output.obj
 0001:00018c4f       __unwindfunclet$?doDownloadRead@alm_bncs_output@@AAEXPAVresponse@@@Z$14 10019c4f f   alm_bncs_output.obj
 0001:00018c5b       __unwindfunclet$?doDownloadRead@alm_bncs_output@@AAEXPAVresponse@@@Z$15 10019c5b f   alm_bncs_output.obj
 0001:00018c67       __unwindfunclet$?doDownloadRead@alm_bncs_output@@AAEXPAVresponse@@@Z$16 10019c67 f   alm_bncs_output.obj
 0001:00018c74       __unwindfunclet$?doDownloadRead@alm_bncs_output@@AAEXPAVresponse@@@Z$17 10019c74 f   alm_bncs_output.obj
 0001:00018c80       __unwindfunclet$?doDownloadRead@alm_bncs_output@@AAEXPAVresponse@@@Z$18 10019c80 f   alm_bncs_output.obj
 0001:00018c8d       __unwindfunclet$?doDownloadRead@alm_bncs_output@@AAEXPAVresponse@@@Z$19 10019c8d f   alm_bncs_output.obj
 0001:00018c99       __unwindfunclet$?doDownloadRead@alm_bncs_output@@AAEXPAVresponse@@@Z$20 10019c99 f   alm_bncs_output.obj
 0001:00018ca5       __unwindfunclet$?doDownloadRead@alm_bncs_output@@AAEXPAVresponse@@@Z$21 10019ca5 f   alm_bncs_output.obj
 0001:00018cb1       __unwindfunclet$?doDownloadRead@alm_bncs_output@@AAEXPAVresponse@@@Z$22 10019cb1 f   alm_bncs_output.obj
 0001:00018cbd       __unwindfunclet$?doDownloadRead@alm_bncs_output@@AAEXPAVresponse@@@Z$23 10019cbd f   alm_bncs_output.obj
 0001:00018cc9       __unwindfunclet$?doDownloadRead@alm_bncs_output@@AAEXPAVresponse@@@Z$24 10019cc9 f   alm_bncs_output.obj
 0001:00018cd5       __unwindfunclet$?doDownloadRead@alm_bncs_output@@AAEXPAVresponse@@@Z$25 10019cd5 f   alm_bncs_output.obj
 0001:00018ce1       __unwindfunclet$?doDownloadRead@alm_bncs_output@@AAEXPAVresponse@@@Z$27 10019ce1 f   alm_bncs_output.obj
 0001:00018ced       __unwindfunclet$?doDownloadRead@alm_bncs_output@@AAEXPAVresponse@@@Z$28 10019ced f   alm_bncs_output.obj
 0001:00018cf9       __unwindfunclet$?doDownloadRead@alm_bncs_output@@AAEXPAVresponse@@@Z$29 10019cf9 f   alm_bncs_output.obj
 0001:00018d05       __ehhandler$?doDownloadRead@alm_bncs_output@@AAEXPAVresponse@@@Z 10019d05 f   alm_bncs_output.obj
 0001:00018d2d       __unwindfunclet$?enableControls@alm_bncs_output@@AAEXXZ$0 10019d2d f   alm_bncs_output.obj
 0001:00018d36       __unwindfunclet$?enableControls@alm_bncs_output@@AAEXXZ$1 10019d36 f   alm_bncs_output.obj
 0001:00018d3f       __unwindfunclet$?enableControls@alm_bncs_output@@AAEXXZ$2 10019d3f f   alm_bncs_output.obj
 0001:00018d48       __unwindfunclet$?enableControls@alm_bncs_output@@AAEXXZ$3 10019d48 f   alm_bncs_output.obj
 0001:00018d51       __ehhandler$?enableControls@alm_bncs_output@@AAEXXZ 10019d51 f   alm_bncs_output.obj
 0001:00018d6c       __unwindfunclet$?ensureFolderExists@alm_bncs_output@@AAE_NABVQString@@@Z$0 10019d6c f   alm_bncs_output.obj
 0001:00018d75       __unwindfunclet$?ensureFolderExists@alm_bncs_output@@AAE_NABVQString@@@Z$1 10019d75 f   alm_bncs_output.obj
 0001:00018d7e       __unwindfunclet$?ensureFolderExists@alm_bncs_output@@AAE_NABVQString@@@Z$2 10019d7e f   alm_bncs_output.obj
 0001:00018d87       __unwindfunclet$?ensureFolderExists@alm_bncs_output@@AAE_NABVQString@@@Z$3 10019d87 f   alm_bncs_output.obj
 0001:00018d90       __unwindfunclet$?ensureFolderExists@alm_bncs_output@@AAE_NABVQString@@@Z$4 10019d90 f   alm_bncs_output.obj
 0001:00018d99       __unwindfunclet$?ensureFolderExists@alm_bncs_output@@AAE_NABVQString@@@Z$5 10019d99 f   alm_bncs_output.obj
 0001:00018da2       __ehhandler$?ensureFolderExists@alm_bncs_output@@AAE_NABVQString@@@Z 10019da2 f   alm_bncs_output.obj
 0001:00018dbd       __unwindfunclet$?extractParam@alm_bncs_output@@AAE?AVQString@@ABV2@0PA_N@Z$0 10019dbd f   alm_bncs_output.obj
 0001:00018dc6       __unwindfunclet$?extractParam@alm_bncs_output@@AAE?AVQString@@ABV2@0PA_N@Z$2 10019dc6 f   alm_bncs_output.obj
 0001:00018dcf       __unwindfunclet$?extractParam@alm_bncs_output@@AAE?AVQString@@ABV2@0PA_N@Z$3 10019dcf f   alm_bncs_output.obj
 0001:00018dd8       __unwindfunclet$?extractParam@alm_bncs_output@@AAE?AVQString@@ABV2@0PA_N@Z$4 10019dd8 f   alm_bncs_output.obj
 0001:00018de1       __unwindfunclet$?extractParam@alm_bncs_output@@AAE?AVQString@@ABV2@0PA_N@Z$5 10019de1 f   alm_bncs_output.obj
 0001:00018dea       __unwindfunclet$?extractParam@alm_bncs_output@@AAE?AVQString@@ABV2@0PA_N@Z$6 10019dea f   alm_bncs_output.obj
 0001:00018df3       __unwindfunclet$?extractParam@alm_bncs_output@@AAE?AVQString@@ABV2@0PA_N@Z$1 10019df3 f   alm_bncs_output.obj
 0001:00018e0d       __ehhandler$?extractParam@alm_bncs_output@@AAE?AVQString@@ABV2@0PA_N@Z 10019e0d f   alm_bncs_output.obj
 0001:00018e28       __unwindfunclet$?insertModifiedInstances@alm_bncs_output@@AAE?AVQString@@PAV?$QDictIterator@VdevTemplate@@@@ABV2@11@Z$0 10019e28 f   alm_bncs_output.obj
 0001:00018e31       __unwindfunclet$?insertModifiedInstances@alm_bncs_output@@AAE?AVQString@@PAV?$QDictIterator@VdevTemplate@@@@ABV2@11@Z$1 10019e31 f   alm_bncs_output.obj
 0001:00018e3a       __unwindfunclet$?insertModifiedInstances@alm_bncs_output@@AAE?AVQString@@PAV?$QDictIterator@VdevTemplate@@@@ABV2@11@Z$2 10019e3a f   alm_bncs_output.obj
 0001:00018e43       __unwindfunclet$?insertModifiedInstances@alm_bncs_output@@AAE?AVQString@@PAV?$QDictIterator@VdevTemplate@@@@ABV2@11@Z$3 10019e43 f   alm_bncs_output.obj
 0001:00018e4c       __unwindfunclet$?insertModifiedInstances@alm_bncs_output@@AAE?AVQString@@PAV?$QDictIterator@VdevTemplate@@@@ABV2@11@Z$4 10019e4c f   alm_bncs_output.obj
 0001:00018e55       __unwindfunclet$?insertModifiedInstances@alm_bncs_output@@AAE?AVQString@@PAV?$QDictIterator@VdevTemplate@@@@ABV2@11@Z$5 10019e55 f   alm_bncs_output.obj
 0001:00018e5e       __unwindfunclet$?insertModifiedInstances@alm_bncs_output@@AAE?AVQString@@PAV?$QDictIterator@VdevTemplate@@@@ABV2@11@Z$6 10019e5e f   alm_bncs_output.obj
 0001:00018e78       __unwindfunclet$?insertModifiedInstances@alm_bncs_output@@AAE?AVQString@@PAV?$QDictIterator@VdevTemplate@@@@ABV2@11@Z$7 10019e78 f   alm_bncs_output.obj
 0001:00018e81       __unwindfunclet$?insertModifiedInstances@alm_bncs_output@@AAE?AVQString@@PAV?$QDictIterator@VdevTemplate@@@@ABV2@11@Z$8 10019e81 f   alm_bncs_output.obj
 0001:00018e8a       __unwindfunclet$?insertModifiedInstances@alm_bncs_output@@AAE?AVQString@@PAV?$QDictIterator@VdevTemplate@@@@ABV2@11@Z$9 10019e8a f   alm_bncs_output.obj
 0001:00018e93       __unwindfunclet$?insertModifiedInstances@alm_bncs_output@@AAE?AVQString@@PAV?$QDictIterator@VdevTemplate@@@@ABV2@11@Z$10 10019e93 f   alm_bncs_output.obj
 0001:00018e9c       __unwindfunclet$?insertModifiedInstances@alm_bncs_output@@AAE?AVQString@@PAV?$QDictIterator@VdevTemplate@@@@ABV2@11@Z$11 10019e9c f   alm_bncs_output.obj
 0001:00018ea5       __unwindfunclet$?insertModifiedInstances@alm_bncs_output@@AAE?AVQString@@PAV?$QDictIterator@VdevTemplate@@@@ABV2@11@Z$12 10019ea5 f   alm_bncs_output.obj
 0001:00018eae       __unwindfunclet$?insertModifiedInstances@alm_bncs_output@@AAE?AVQString@@PAV?$QDictIterator@VdevTemplate@@@@ABV2@11@Z$13 10019eae f   alm_bncs_output.obj
 0001:00018eb7       __unwindfunclet$?insertModifiedInstances@alm_bncs_output@@AAE?AVQString@@PAV?$QDictIterator@VdevTemplate@@@@ABV2@11@Z$14 10019eb7 f   alm_bncs_output.obj
 0001:00018ec0       __unwindfunclet$?insertModifiedInstances@alm_bncs_output@@AAE?AVQString@@PAV?$QDictIterator@VdevTemplate@@@@ABV2@11@Z$15 10019ec0 f   alm_bncs_output.obj
 0001:00018ec9       __unwindfunclet$?insertModifiedInstances@alm_bncs_output@@AAE?AVQString@@PAV?$QDictIterator@VdevTemplate@@@@ABV2@11@Z$16 10019ec9 f   alm_bncs_output.obj
 0001:00018ed2       __unwindfunclet$?insertModifiedInstances@alm_bncs_output@@AAE?AVQString@@PAV?$QDictIterator@VdevTemplate@@@@ABV2@11@Z$17 10019ed2 f   alm_bncs_output.obj
 0001:00018edb       __unwindfunclet$?insertModifiedInstances@alm_bncs_output@@AAE?AVQString@@PAV?$QDictIterator@VdevTemplate@@@@ABV2@11@Z$18 10019edb f   alm_bncs_output.obj
 0001:00018ee4       __unwindfunclet$?insertModifiedInstances@alm_bncs_output@@AAE?AVQString@@PAV?$QDictIterator@VdevTemplate@@@@ABV2@11@Z$19 10019ee4 f   alm_bncs_output.obj
 0001:00018eed       __unwindfunclet$?insertModifiedInstances@alm_bncs_output@@AAE?AVQString@@PAV?$QDictIterator@VdevTemplate@@@@ABV2@11@Z$20 10019eed f   alm_bncs_output.obj
 0001:00018ef6       __unwindfunclet$?insertModifiedInstances@alm_bncs_output@@AAE?AVQString@@PAV?$QDictIterator@VdevTemplate@@@@ABV2@11@Z$21 10019ef6 f   alm_bncs_output.obj
 0001:00018eff       __unwindfunclet$?insertModifiedInstances@alm_bncs_output@@AAE?AVQString@@PAV?$QDictIterator@VdevTemplate@@@@ABV2@11@Z$22 10019eff f   alm_bncs_output.obj
 0001:00018f08       __unwindfunclet$?insertModifiedInstances@alm_bncs_output@@AAE?AVQString@@PAV?$QDictIterator@VdevTemplate@@@@ABV2@11@Z$23 10019f08 f   alm_bncs_output.obj
 0001:00018f11       __unwindfunclet$?insertModifiedInstances@alm_bncs_output@@AAE?AVQString@@PAV?$QDictIterator@VdevTemplate@@@@ABV2@11@Z$24 10019f11 f   alm_bncs_output.obj
 0001:00018f1a       __ehhandler$?insertModifiedInstances@alm_bncs_output@@AAE?AVQString@@PAV?$QDictIterator@VdevTemplate@@@@ABV2@11@Z 10019f1a f   alm_bncs_output.obj
 0001:00018f35       __unwindfunclet$?loadFile@alm_bncs_output@@AAE_NABVQString@@@Z$0 10019f35 f   alm_bncs_output.obj
 0001:00018f41       __unwindfunclet$?loadFile@alm_bncs_output@@AAE_NABVQString@@@Z$1 10019f41 f   alm_bncs_output.obj
 0001:00018f4a       __unwindfunclet$?loadFile@alm_bncs_output@@AAE_NABVQString@@@Z$2 10019f4a f   alm_bncs_output.obj
 0001:00018f52       __unwindfunclet$?loadFile@alm_bncs_output@@AAE_NABVQString@@@Z$3 10019f52 f   alm_bncs_output.obj
 0001:00018f5b       __unwindfunclet$?loadFile@alm_bncs_output@@AAE_NABVQString@@@Z$4 10019f5b f   alm_bncs_output.obj
 0001:00018f64       __unwindfunclet$?loadFile@alm_bncs_output@@AAE_NABVQString@@@Z$5 10019f64 f   alm_bncs_output.obj
 0001:00018f6d       __unwindfunclet$?loadFile@alm_bncs_output@@AAE_NABVQString@@@Z$6 10019f6d f   alm_bncs_output.obj
 0001:00018f76       __unwindfunclet$?loadFile@alm_bncs_output@@AAE_NABVQString@@@Z$7 10019f76 f   alm_bncs_output.obj
 0001:00018f7f       __unwindfunclet$?loadFile@alm_bncs_output@@AAE_NABVQString@@@Z$8 10019f7f f   alm_bncs_output.obj
 0001:00018f88       __unwindfunclet$?loadFile@alm_bncs_output@@AAE_NABVQString@@@Z$9 10019f88 f   alm_bncs_output.obj
 0001:00018f91       __unwindfunclet$?loadFile@alm_bncs_output@@AAE_NABVQString@@@Z$10 10019f91 f   alm_bncs_output.obj
 0001:00018f9a       __unwindfunclet$?loadFile@alm_bncs_output@@AAE_NABVQString@@@Z$11 10019f9a f   alm_bncs_output.obj
 0001:00018fa6       __unwindfunclet$?loadFile@alm_bncs_output@@AAE_NABVQString@@@Z$12 10019fa6 f   alm_bncs_output.obj
 0001:00018fb2       __unwindfunclet$?loadFile@alm_bncs_output@@AAE_NABVQString@@@Z$13 10019fb2 f   alm_bncs_output.obj
 0001:00018fbb       __unwindfunclet$?loadFile@alm_bncs_output@@AAE_NABVQString@@@Z$14 10019fbb f   alm_bncs_output.obj
 0001:00018fc4       __unwindfunclet$?loadFile@alm_bncs_output@@AAE_NABVQString@@@Z$15 10019fc4 f   alm_bncs_output.obj
 0001:00018fd0       __unwindfunclet$?loadFile@alm_bncs_output@@AAE_NABVQString@@@Z$16 10019fd0 f   alm_bncs_output.obj
 0001:00018fd9       __unwindfunclet$?loadFile@alm_bncs_output@@AAE_NABVQString@@@Z$17 10019fd9 f   alm_bncs_output.obj
 0001:00018ff3       __unwindfunclet$?loadFile@alm_bncs_output@@AAE_NABVQString@@@Z$18 10019ff3 f   alm_bncs_output.obj
 0001:0001900d       __unwindfunclet$?loadFile@alm_bncs_output@@AAE_NABVQString@@@Z$31 1001a00d f   alm_bncs_output.obj
 0001:00019016       __unwindfunclet$?loadFile@alm_bncs_output@@AAE_NABVQString@@@Z$32 1001a016 f   alm_bncs_output.obj
 0001:0001901f       __unwindfunclet$?loadFile@alm_bncs_output@@AAE_NABVQString@@@Z$23 1001a01f f   alm_bncs_output.obj
 0001:00019028       __unwindfunclet$?loadFile@alm_bncs_output@@AAE_NABVQString@@@Z$24 1001a028 f   alm_bncs_output.obj
 0001:00019031       __unwindfunclet$?loadFile@alm_bncs_output@@AAE_NABVQString@@@Z$25 1001a031 f   alm_bncs_output.obj
 0001:0001903a       __unwindfunclet$?loadFile@alm_bncs_output@@AAE_NABVQString@@@Z$26 1001a03a f   alm_bncs_output.obj
 0001:00019043       __unwindfunclet$?loadFile@alm_bncs_output@@AAE_NABVQString@@@Z$27 1001a043 f   alm_bncs_output.obj
 0001:0001904c       __unwindfunclet$?loadFile@alm_bncs_output@@AAE_NABVQString@@@Z$28 1001a04c f   alm_bncs_output.obj
 0001:00019058       __unwindfunclet$?loadFile@alm_bncs_output@@AAE_NABVQString@@@Z$29 1001a058 f   alm_bncs_output.obj
 0001:00019061       __unwindfunclet$?loadFile@alm_bncs_output@@AAE_NABVQString@@@Z$30 1001a061 f   alm_bncs_output.obj
 0001:0001906a       __unwindfunclet$?loadFile@alm_bncs_output@@AAE_NABVQString@@@Z$21 1001a06a f   alm_bncs_output.obj
 0001:00019073       __unwindfunclet$?loadFile@alm_bncs_output@@AAE_NABVQString@@@Z$22 1001a073 f   alm_bncs_output.obj
 0001:0001907c       __unwindfunclet$?loadFile@alm_bncs_output@@AAE_NABVQString@@@Z$19 1001a07c f   alm_bncs_output.obj
 0001:00019085       __unwindfunclet$?loadFile@alm_bncs_output@@AAE_NABVQString@@@Z$20 1001a085 f   alm_bncs_output.obj
 0001:0001908e       __unwindfunclet$?loadFile@alm_bncs_output@@AAE_NABVQString@@@Z$33 1001a08e f   alm_bncs_output.obj
 0001:00019097       __unwindfunclet$?loadFile@alm_bncs_output@@AAE_NABVQString@@@Z$34 1001a097 f   alm_bncs_output.obj
 0001:000190a0       __unwindfunclet$?loadFile@alm_bncs_output@@AAE_NABVQString@@@Z$35 1001a0a0 f   alm_bncs_output.obj
 0001:000190a9       __unwindfunclet$?loadFile@alm_bncs_output@@AAE_NABVQString@@@Z$36 1001a0a9 f   alm_bncs_output.obj
 0001:000190b2       __unwindfunclet$?loadFile@alm_bncs_output@@AAE_NABVQString@@@Z$37 1001a0b2 f   alm_bncs_output.obj
 0001:000190bb       __ehhandler$?loadFile@alm_bncs_output@@AAE_NABVQString@@@Z 1001a0bb f   alm_bncs_output.obj
 0001:000190d9       __unwindfunclet$?loadProcesses@alm_bncs_output@@AAE_NABVQString@@@Z$0 1001a0d9 f   alm_bncs_output.obj
 0001:000190e2       __unwindfunclet$?loadProcesses@alm_bncs_output@@AAE_NABVQString@@@Z$1 1001a0e2 f   alm_bncs_output.obj
 0001:000190eb       __unwindfunclet$?loadProcesses@alm_bncs_output@@AAE_NABVQString@@@Z$2 1001a0eb f   alm_bncs_output.obj
 0001:000190f7       __unwindfunclet$?loadProcesses@alm_bncs_output@@AAE_NABVQString@@@Z$3 1001a0f7 f   alm_bncs_output.obj
 0001:00019103       __unwindfunclet$?loadProcesses@alm_bncs_output@@AAE_NABVQString@@@Z$4 1001a103 f   alm_bncs_output.obj
 0001:0001910c       __unwindfunclet$?loadProcesses@alm_bncs_output@@AAE_NABVQString@@@Z$5 1001a10c f   alm_bncs_output.obj
 0001:00019115       __unwindfunclet$?loadProcesses@alm_bncs_output@@AAE_NABVQString@@@Z$6 1001a115 f   alm_bncs_output.obj
 0001:0001911e       __unwindfunclet$?loadProcesses@alm_bncs_output@@AAE_NABVQString@@@Z$7 1001a11e f   alm_bncs_output.obj
 0001:00019127       __unwindfunclet$?loadProcesses@alm_bncs_output@@AAE_NABVQString@@@Z$8 1001a127 f   alm_bncs_output.obj
 0001:00019130       __unwindfunclet$?loadProcesses@alm_bncs_output@@AAE_NABVQString@@@Z$9 1001a130 f   alm_bncs_output.obj
 0001:0001914a       __unwindfunclet$?loadProcesses@alm_bncs_output@@AAE_NABVQString@@@Z$10 1001a14a f   alm_bncs_output.obj
 0001:00019164       __unwindfunclet$?loadProcesses@alm_bncs_output@@AAE_NABVQString@@@Z$11 1001a164 f   alm_bncs_output.obj
 0001:0001916e       __unwindfunclet$?loadProcesses@alm_bncs_output@@AAE_NABVQString@@@Z$12 1001a16e f   alm_bncs_output.obj
 0001:00019177       __unwindfunclet$?loadProcesses@alm_bncs_output@@AAE_NABVQString@@@Z$14 1001a177 f   alm_bncs_output.obj
 0001:00019180       __unwindfunclet$?loadProcesses@alm_bncs_output@@AAE_NABVQString@@@Z$15 1001a180 f   alm_bncs_output.obj
 0001:00019189       __unwindfunclet$?loadProcesses@alm_bncs_output@@AAE_NABVQString@@@Z$16 1001a189 f   alm_bncs_output.obj
 0001:00019193       __unwindfunclet$?loadProcesses@alm_bncs_output@@AAE_NABVQString@@@Z$17 1001a193 f   alm_bncs_output.obj
 0001:0001919c       __ehhandler$?loadProcesses@alm_bncs_output@@AAE_NABVQString@@@Z 1001a19c f   alm_bncs_output.obj
 0001:000191ba       __unwindfunclet$?loadTemplates@alm_bncs_output@@AAEXABVQStringList@@ABV?$QMap@VQString@@V1@@@@Z$0 1001a1ba f   alm_bncs_output.obj
 0001:000191c3       __unwindfunclet$?loadTemplates@alm_bncs_output@@AAEXABVQStringList@@ABV?$QMap@VQString@@V1@@@@Z$1 1001a1c3 f   alm_bncs_output.obj
 0001:000191cd       __unwindfunclet$?loadTemplates@alm_bncs_output@@AAEXABVQStringList@@ABV?$QMap@VQString@@V1@@@@Z$2 1001a1cd f   alm_bncs_output.obj
 0001:000191d6       __unwindfunclet$?loadTemplates@alm_bncs_output@@AAEXABVQStringList@@ABV?$QMap@VQString@@V1@@@@Z$3 1001a1d6 f   alm_bncs_output.obj
 0001:000191df       __unwindfunclet$?loadTemplates@alm_bncs_output@@AAEXABVQStringList@@ABV?$QMap@VQString@@V1@@@@Z$4 1001a1df f   alm_bncs_output.obj
 0001:000191e8       __unwindfunclet$?loadTemplates@alm_bncs_output@@AAEXABVQStringList@@ABV?$QMap@VQString@@V1@@@@Z$5 1001a1e8 f   alm_bncs_output.obj
 0001:000191f1       __unwindfunclet$?loadTemplates@alm_bncs_output@@AAEXABVQStringList@@ABV?$QMap@VQString@@V1@@@@Z$6 1001a1f1 f   alm_bncs_output.obj
 0001:000191fa       __unwindfunclet$?loadTemplates@alm_bncs_output@@AAEXABVQStringList@@ABV?$QMap@VQString@@V1@@@@Z$7 1001a1fa f   alm_bncs_output.obj
 0001:00019203       __unwindfunclet$?loadTemplates@alm_bncs_output@@AAEXABVQStringList@@ABV?$QMap@VQString@@V1@@@@Z$8 1001a203 f   alm_bncs_output.obj
 0001:0001920c       __unwindfunclet$?loadTemplates@alm_bncs_output@@AAEXABVQStringList@@ABV?$QMap@VQString@@V1@@@@Z$9 1001a20c f   alm_bncs_output.obj
 0001:00019215       __unwindfunclet$?loadTemplates@alm_bncs_output@@AAEXABVQStringList@@ABV?$QMap@VQString@@V1@@@@Z$10 1001a215 f   alm_bncs_output.obj
 0001:0001921e       __unwindfunclet$?loadTemplates@alm_bncs_output@@AAEXABVQStringList@@ABV?$QMap@VQString@@V1@@@@Z$11 1001a21e f   alm_bncs_output.obj
 0001:00019227       __unwindfunclet$?loadTemplates@alm_bncs_output@@AAEXABVQStringList@@ABV?$QMap@VQString@@V1@@@@Z$12 1001a227 f   alm_bncs_output.obj
 0001:00019230       __unwindfunclet$?loadTemplates@alm_bncs_output@@AAEXABVQStringList@@ABV?$QMap@VQString@@V1@@@@Z$13 1001a230 f   alm_bncs_output.obj
 0001:00019239       __unwindfunclet$?loadTemplates@alm_bncs_output@@AAEXABVQStringList@@ABV?$QMap@VQString@@V1@@@@Z$14 1001a239 f   alm_bncs_output.obj
 0001:00019242       __unwindfunclet$?loadTemplates@alm_bncs_output@@AAEXABVQStringList@@ABV?$QMap@VQString@@V1@@@@Z$15 1001a242 f   alm_bncs_output.obj
 0001:0001924b       __unwindfunclet$?loadTemplates@alm_bncs_output@@AAEXABVQStringList@@ABV?$QMap@VQString@@V1@@@@Z$16 1001a24b f   alm_bncs_output.obj
 0001:00019254       __ehhandler$?loadTemplates@alm_bncs_output@@AAEXABVQStringList@@ABV?$QMap@VQString@@V1@@@@Z 1001a254 f   alm_bncs_output.obj
 0001:00019272       __unwindfunclet$?lockDevDesc@alm_bncs_output@@AAEXABVQString@@@Z$0 1001a272 f   alm_bncs_output.obj
 0001:00019272       __unwindfunclet$?replyUpload@alm_bncs_output@@AAEXPAVresponse@@@Z$0 1001a272 f   alm_bncs_output.obj
 0001:0001927b       __ehhandler$?replyUpload@alm_bncs_output@@AAEXPAVresponse@@@Z 1001a27b f   alm_bncs_output.obj
 0001:0001927b       __ehhandler$?lockDevDesc@alm_bncs_output@@AAEXABVQString@@@Z 1001a27b f   alm_bncs_output.obj
 0001:00019296       __unwindfunclet$?manageTemplate@alm_bncs_output@@QAEXXZ$0 1001a296 f   alm_bncs_output.obj
 0001:000192a0       __unwindfunclet$?manageTemplate@alm_bncs_output@@QAEXXZ$1 1001a2a0 f   alm_bncs_output.obj
 0001:000192a8       __unwindfunclet$?manageTemplate@alm_bncs_output@@QAEXXZ$2 1001a2a8 f   alm_bncs_output.obj
 0001:000192b1       __unwindfunclet$?manageTemplate@alm_bncs_output@@QAEXXZ$3 1001a2b1 f   alm_bncs_output.obj
 0001:000192ba       __unwindfunclet$?manageTemplate@alm_bncs_output@@QAEXXZ$4 1001a2ba f   alm_bncs_output.obj
 0001:000192c3       __unwindfunclet$?manageTemplate@alm_bncs_output@@QAEXXZ$5 1001a2c3 f   alm_bncs_output.obj
 0001:000192cc       __unwindfunclet$?manageTemplate@alm_bncs_output@@QAEXXZ$6 1001a2cc f   alm_bncs_output.obj
 0001:000192d5       __unwindfunclet$?manageTemplate@alm_bncs_output@@QAEXXZ$7 1001a2d5 f   alm_bncs_output.obj
 0001:000192de       __unwindfunclet$?manageTemplate@alm_bncs_output@@QAEXXZ$8 1001a2de f   alm_bncs_output.obj
 0001:000192e7       __unwindfunclet$?manageTemplate@alm_bncs_output@@QAEXXZ$9 1001a2e7 f   alm_bncs_output.obj
 0001:000192ef       __unwindfunclet$?manageTemplate@alm_bncs_output@@QAEXXZ$10 1001a2ef f   alm_bncs_output.obj
 0001:000192f8       __unwindfunclet$?manageTemplate@alm_bncs_output@@QAEXXZ$11 1001a2f8 f   alm_bncs_output.obj
 0001:00019301       __unwindfunclet$?manageTemplate@alm_bncs_output@@QAEXXZ$12 1001a301 f   alm_bncs_output.obj
 0001:0001930a       __unwindfunclet$?manageTemplate@alm_bncs_output@@QAEXXZ$13 1001a30a f   alm_bncs_output.obj
 0001:00019313       __unwindfunclet$?manageTemplate@alm_bncs_output@@QAEXXZ$14 1001a313 f   alm_bncs_output.obj
 0001:0001931c       __unwindfunclet$?manageTemplate@alm_bncs_output@@QAEXXZ$15 1001a31c f   alm_bncs_output.obj
 0001:00019325       __unwindfunclet$?manageTemplate@alm_bncs_output@@QAEXXZ$16 1001a325 f   alm_bncs_output.obj
 0001:0001932e       __unwindfunclet$?manageTemplate@alm_bncs_output@@QAEXXZ$17 1001a32e f   alm_bncs_output.obj
 0001:00019337       __unwindfunclet$?manageTemplate@alm_bncs_output@@QAEXXZ$18 1001a337 f   alm_bncs_output.obj
 0001:00019340       __ehhandler$?manageTemplate@alm_bncs_output@@QAEXXZ 1001a340 f   alm_bncs_output.obj
 0001:0001935b       __unwindfunclet$?markDirty@alm_bncs_output@@QAEXXZ$0 1001a35b f   alm_bncs_output.obj
 0001:00019364       __ehhandler$?markDirty@alm_bncs_output@@QAEXXZ 1001a364 f   alm_bncs_output.obj
 0001:0001937f       __unwindfunclet$?menuDeleteFile@alm_bncs_output@@QAEXXZ$0 1001a37f f   alm_bncs_output.obj
 0001:00019388       __unwindfunclet$?menuDeleteFile@alm_bncs_output@@QAEXXZ$1 1001a388 f   alm_bncs_output.obj
 0001:00019391       __unwindfunclet$?menuDeleteFile@alm_bncs_output@@QAEXXZ$2 1001a391 f   alm_bncs_output.obj
 0001:0001939a       __unwindfunclet$?menuDeleteFile@alm_bncs_output@@QAEXXZ$3 1001a39a f   alm_bncs_output.obj
 0001:000193a3       __unwindfunclet$?menuDeleteFile@alm_bncs_output@@QAEXXZ$4 1001a3a3 f   alm_bncs_output.obj
 0001:000193ac       __unwindfunclet$?menuDeleteFile@alm_bncs_output@@QAEXXZ$5 1001a3ac f   alm_bncs_output.obj
 0001:000193b5       __unwindfunclet$?menuDeleteFile@alm_bncs_output@@QAEXXZ$6 1001a3b5 f   alm_bncs_output.obj
 0001:000193be       __ehhandler$?menuDeleteFile@alm_bncs_output@@QAEXXZ 1001a3be f   alm_bncs_output.obj
 0001:000193d9       __unwindfunclet$?menuDuplicateFile@alm_bncs_output@@QAEXXZ$0 1001a3d9 f   alm_bncs_output.obj
 0001:000193e2       __unwindfunclet$?menuDuplicateFile@alm_bncs_output@@QAEXXZ$1 1001a3e2 f   alm_bncs_output.obj
 0001:000193eb       __unwindfunclet$?menuDuplicateFile@alm_bncs_output@@QAEXXZ$2 1001a3eb f   alm_bncs_output.obj
 0001:000193f4       __unwindfunclet$?menuDuplicateFile@alm_bncs_output@@QAEXXZ$3 1001a3f4 f   alm_bncs_output.obj
 0001:000193fd       __unwindfunclet$?menuDuplicateFile@alm_bncs_output@@QAEXXZ$4 1001a3fd f   alm_bncs_output.obj
 0001:00019406       __unwindfunclet$?menuDuplicateFile@alm_bncs_output@@QAEXXZ$5 1001a406 f   alm_bncs_output.obj
 0001:0001940f       __unwindfunclet$?menuDuplicateFile@alm_bncs_output@@QAEXXZ$6 1001a40f f   alm_bncs_output.obj
 0001:00019418       __unwindfunclet$?menuDuplicateFile@alm_bncs_output@@QAEXXZ$7 1001a418 f   alm_bncs_output.obj
 0001:00019421       __unwindfunclet$?menuDuplicateFile@alm_bncs_output@@QAEXXZ$8 1001a421 f   alm_bncs_output.obj
 0001:0001942a       __unwindfunclet$?menuDuplicateFile@alm_bncs_output@@QAEXXZ$9 1001a42a f   alm_bncs_output.obj
 0001:00019433       __unwindfunclet$?menuDuplicateFile@alm_bncs_output@@QAEXXZ$10 1001a433 f   alm_bncs_output.obj
 0001:0001943c       __unwindfunclet$?menuDuplicateFile@alm_bncs_output@@QAEXXZ$11 1001a43c f   alm_bncs_output.obj
 0001:00019445       __unwindfunclet$?menuDuplicateFile@alm_bncs_output@@QAEXXZ$12 1001a445 f   alm_bncs_output.obj
 0001:0001944f       __unwindfunclet$?menuDuplicateFile@alm_bncs_output@@QAEXXZ$13 1001a44f f   alm_bncs_output.obj
 0001:00019469       __unwindfunclet$?menuDuplicateFile@alm_bncs_output@@QAEXXZ$14 1001a469 f   alm_bncs_output.obj
 0001:00019473       __unwindfunclet$?menuDuplicateFile@alm_bncs_output@@QAEXXZ$15 1001a473 f   alm_bncs_output.obj
 0001:0001947c       __unwindfunclet$?menuDuplicateFile@alm_bncs_output@@QAEXXZ$16 1001a47c f   alm_bncs_output.obj
 0001:00019485       __unwindfunclet$?menuDuplicateFile@alm_bncs_output@@QAEXXZ$17 1001a485 f   alm_bncs_output.obj
 0001:0001948e       __unwindfunclet$?menuDuplicateFile@alm_bncs_output@@QAEXXZ$18 1001a48e f   alm_bncs_output.obj
 0001:00019497       __unwindfunclet$?menuDuplicateFile@alm_bncs_output@@QAEXXZ$19 1001a497 f   alm_bncs_output.obj
 0001:000194a0       __unwindfunclet$?menuDuplicateFile@alm_bncs_output@@QAEXXZ$20 1001a4a0 f   alm_bncs_output.obj
 0001:000194a9       __unwindfunclet$?menuDuplicateFile@alm_bncs_output@@QAEXXZ$21 1001a4a9 f   alm_bncs_output.obj
 0001:000194b2       __ehhandler$?menuDuplicateFile@alm_bncs_output@@QAEXXZ 1001a4b2 f   alm_bncs_output.obj
 0001:000194cd       __unwindfunclet$?menus@alm_bncs_output@@UAE?AVQPopupMenuList@@XZ$0 1001a4cd f   alm_bncs_output.obj
 0001:000194e6       __ehhandler$?menus@alm_bncs_output@@UAE?AVQPopupMenuList@@XZ 1001a4e6 f   alm_bncs_output.obj
 0001:00019501       __unwindfunclet$?navigate@alm_bncs_output@@UAEXABVQString@@0@Z$0 1001a501 f   alm_bncs_output.obj
 0001:0001950a       __unwindfunclet$?navigate@alm_bncs_output@@UAEXABVQString@@0@Z$1 1001a50a f   alm_bncs_output.obj
 0001:00019513       __unwindfunclet$?navigate@alm_bncs_output@@UAEXABVQString@@0@Z$2 1001a513 f   alm_bncs_output.obj
 0001:0001951c       __unwindfunclet$?navigate@alm_bncs_output@@UAEXABVQString@@0@Z$3 1001a51c f   alm_bncs_output.obj
 0001:00019525       __unwindfunclet$?navigate@alm_bncs_output@@UAEXABVQString@@0@Z$4 1001a525 f   alm_bncs_output.obj
 0001:0001952e       __unwindfunclet$?navigate@alm_bncs_output@@UAEXABVQString@@0@Z$5 1001a52e f   alm_bncs_output.obj
 0001:00019537       __unwindfunclet$?navigate@alm_bncs_output@@UAEXABVQString@@0@Z$6 1001a537 f   alm_bncs_output.obj
 0001:00019551       __unwindfunclet$?navigate@alm_bncs_output@@UAEXABVQString@@0@Z$7 1001a551 f   alm_bncs_output.obj
 0001:0001956b       __unwindfunclet$?navigate@alm_bncs_output@@UAEXABVQString@@0@Z$8 1001a56b f   alm_bncs_output.obj
 0001:00019574       __unwindfunclet$?navigate@alm_bncs_output@@UAEXABVQString@@0@Z$9 1001a574 f   alm_bncs_output.obj
 0001:0001957d       __unwindfunclet$?navigate@alm_bncs_output@@UAEXABVQString@@0@Z$10 1001a57d f   alm_bncs_output.obj
 0001:00019586       __unwindfunclet$?navigate@alm_bncs_output@@UAEXABVQString@@0@Z$11 1001a586 f   alm_bncs_output.obj
 0001:0001958f       __unwindfunclet$?navigate@alm_bncs_output@@UAEXABVQString@@0@Z$12 1001a58f f   alm_bncs_output.obj
 0001:00019598       __unwindfunclet$?navigate@alm_bncs_output@@UAEXABVQString@@0@Z$13 1001a598 f   alm_bncs_output.obj
 0001:000195a1       __unwindfunclet$?navigate@alm_bncs_output@@UAEXABVQString@@0@Z$14 1001a5a1 f   alm_bncs_output.obj
 0001:000195aa       __unwindfunclet$?navigate@alm_bncs_output@@UAEXABVQString@@0@Z$15 1001a5aa f   alm_bncs_output.obj
 0001:000195b3       __ehhandler$?navigate@alm_bncs_output@@UAEXABVQString@@0@Z 1001a5b3 f   alm_bncs_output.obj
 0001:000195ce       __unwindfunclet$?newFile@alm_bncs_output@@AAEXABVQString@@@Z$0 1001a5ce f   alm_bncs_output.obj
 0001:000195d7       __unwindfunclet$?newFile@alm_bncs_output@@AAEXABVQString@@@Z$1 1001a5d7 f   alm_bncs_output.obj
 0001:000195e0       __unwindfunclet$?newFile@alm_bncs_output@@AAEXABVQString@@@Z$2 1001a5e0 f   alm_bncs_output.obj
 0001:000195ea       __unwindfunclet$?newFile@alm_bncs_output@@AAEXABVQString@@@Z$3 1001a5ea f   alm_bncs_output.obj
 0001:00019604       __unwindfunclet$?newFile@alm_bncs_output@@AAEXABVQString@@@Z$4 1001a604 f   alm_bncs_output.obj
 0001:0001960e       __unwindfunclet$?newFile@alm_bncs_output@@AAEXABVQString@@@Z$5 1001a60e f   alm_bncs_output.obj
 0001:00019617       __unwindfunclet$?newFile@alm_bncs_output@@AAEXABVQString@@@Z$6 1001a617 f   alm_bncs_output.obj
 0001:00019620       __unwindfunclet$?newFile@alm_bncs_output@@AAEXABVQString@@@Z$7 1001a620 f   alm_bncs_output.obj
 0001:00019629       __unwindfunclet$?newFile@alm_bncs_output@@AAEXABVQString@@@Z$8 1001a629 f   alm_bncs_output.obj
 0001:00019632       __unwindfunclet$?newFile@alm_bncs_output@@AAEXABVQString@@@Z$9 1001a632 f   alm_bncs_output.obj
 0001:0001963b       __unwindfunclet$?newFile@alm_bncs_output@@AAEXABVQString@@@Z$10 1001a63b f   alm_bncs_output.obj
 0001:00019644       __unwindfunclet$?newFile@alm_bncs_output@@AAEXABVQString@@@Z$11 1001a644 f   alm_bncs_output.obj
 0001:0001964d       __unwindfunclet$?newFile@alm_bncs_output@@AAEXABVQString@@@Z$13 1001a64d f   alm_bncs_output.obj
 0001:00019656       __unwindfunclet$?newFile@alm_bncs_output@@AAEXABVQString@@@Z$14 1001a656 f   alm_bncs_output.obj
 0001:0001965f       __unwindfunclet$?newFile@alm_bncs_output@@AAEXABVQString@@@Z$15 1001a65f f   alm_bncs_output.obj
 0001:00019668       __unwindfunclet$?newFile@alm_bncs_output@@AAEXABVQString@@@Z$16 1001a668 f   alm_bncs_output.obj
 0001:00019671       __unwindfunclet$?newFile@alm_bncs_output@@AAEXABVQString@@@Z$17 1001a671 f   alm_bncs_output.obj
 0001:0001967a       __unwindfunclet$?newFile@alm_bncs_output@@AAEXABVQString@@@Z$18 1001a67a f   alm_bncs_output.obj
 0001:00019683       __unwindfunclet$?newFile@alm_bncs_output@@AAEXABVQString@@@Z$19 1001a683 f   alm_bncs_output.obj
 0001:0001968c       __unwindfunclet$?newFile@alm_bncs_output@@AAEXABVQString@@@Z$20 1001a68c f   alm_bncs_output.obj
 0001:00019695       __unwindfunclet$?newFile@alm_bncs_output@@AAEXABVQString@@@Z$21 1001a695 f   alm_bncs_output.obj
 0001:0001969e       __unwindfunclet$?newFile@alm_bncs_output@@AAEXABVQString@@@Z$22 1001a69e f   alm_bncs_output.obj
 0001:000196a7       __unwindfunclet$?newFile@alm_bncs_output@@AAEXABVQString@@@Z$23 1001a6a7 f   alm_bncs_output.obj
 0001:000196b0       __unwindfunclet$?newFile@alm_bncs_output@@AAEXABVQString@@@Z$24 1001a6b0 f   alm_bncs_output.obj
 0001:000196b9       __unwindfunclet$?newFile@alm_bncs_output@@AAEXABVQString@@@Z$25 1001a6b9 f   alm_bncs_output.obj
 0001:000196c2       __ehhandler$?newFile@alm_bncs_output@@AAEXABVQString@@@Z 1001a6c2 f   alm_bncs_output.obj
 0001:000196dd       __unwindfunclet$?renameModule@alm_bncs_output@@QAEXPAVQListViewItem@@HABVQString@@@Z$0 1001a6dd f   alm_bncs_output.obj
 0001:000196e6       __unwindfunclet$?renameModule@alm_bncs_output@@QAEXPAVQListViewItem@@HABVQString@@@Z$1 1001a6e6 f   alm_bncs_output.obj
 0001:000196ef       __unwindfunclet$?renameModule@alm_bncs_output@@QAEXPAVQListViewItem@@HABVQString@@@Z$2 1001a6ef f   alm_bncs_output.obj
 0001:000196f8       __unwindfunclet$?renameModule@alm_bncs_output@@QAEXPAVQListViewItem@@HABVQString@@@Z$3 1001a6f8 f   alm_bncs_output.obj
 0001:00019701       __unwindfunclet$?renameModule@alm_bncs_output@@QAEXPAVQListViewItem@@HABVQString@@@Z$4 1001a701 f   alm_bncs_output.obj
 0001:0001970a       __unwindfunclet$?renameModule@alm_bncs_output@@QAEXPAVQListViewItem@@HABVQString@@@Z$5 1001a70a f   alm_bncs_output.obj
 0001:00019713       __unwindfunclet$?renameModule@alm_bncs_output@@QAEXPAVQListViewItem@@HABVQString@@@Z$6 1001a713 f   alm_bncs_output.obj
 0001:0001971c       __unwindfunclet$?renameModule@alm_bncs_output@@QAEXPAVQListViewItem@@HABVQString@@@Z$7 1001a71c f   alm_bncs_output.obj
 0001:00019725       __unwindfunclet$?renameModule@alm_bncs_output@@QAEXPAVQListViewItem@@HABVQString@@@Z$8 1001a725 f   alm_bncs_output.obj
 0001:0001972e       __unwindfunclet$?renameModule@alm_bncs_output@@QAEXPAVQListViewItem@@HABVQString@@@Z$9 1001a72e f   alm_bncs_output.obj
 0001:00019737       __ehhandler$?renameModule@alm_bncs_output@@QAEXPAVQListViewItem@@HABVQString@@@Z 1001a737 f   alm_bncs_output.obj
 0001:00019752       __unwindfunclet$?replyDownload@alm_bncs_output@@AAEXPAVresponse@@@Z$0 1001a752 f   alm_bncs_output.obj
 0001:0001975b       __unwindfunclet$?replyDownload@alm_bncs_output@@AAEXPAVresponse@@@Z$1 1001a75b f   alm_bncs_output.obj
 0001:00019764       __unwindfunclet$?replyDownload@alm_bncs_output@@AAEXPAVresponse@@@Z$2 1001a764 f   alm_bncs_output.obj
 0001:0001976d       __ehhandler$?replyDownload@alm_bncs_output@@AAEXPAVresponse@@@Z 1001a76d f   alm_bncs_output.obj
 0001:00019788       __unwindfunclet$?replyLock@alm_bncs_output@@AAEXPAVresponse@@@Z$0 1001a788 f   alm_bncs_output.obj
 0001:00019791       __unwindfunclet$?replyLock@alm_bncs_output@@AAEXPAVresponse@@@Z$1 1001a791 f   alm_bncs_output.obj
 0001:0001979a       __unwindfunclet$?replyLock@alm_bncs_output@@AAEXPAVresponse@@@Z$2 1001a79a f   alm_bncs_output.obj
 0001:000197a3       __unwindfunclet$?replyLock@alm_bncs_output@@AAEXPAVresponse@@@Z$3 1001a7a3 f   alm_bncs_output.obj
 0001:000197ac       __unwindfunclet$?replyLock@alm_bncs_output@@AAEXPAVresponse@@@Z$4 1001a7ac f   alm_bncs_output.obj
 0001:000197b5       __unwindfunclet$?replyLock@alm_bncs_output@@AAEXPAVresponse@@@Z$5 1001a7b5 f   alm_bncs_output.obj
 0001:000197be       __unwindfunclet$?replyLock@alm_bncs_output@@AAEXPAVresponse@@@Z$6 1001a7be f   alm_bncs_output.obj
 0001:000197c7       __unwindfunclet$?replyLock@alm_bncs_output@@AAEXPAVresponse@@@Z$7 1001a7c7 f   alm_bncs_output.obj
 0001:000197d0       __unwindfunclet$?replyLock@alm_bncs_output@@AAEXPAVresponse@@@Z$8 1001a7d0 f   alm_bncs_output.obj
 0001:000197d9       __unwindfunclet$?replyLock@alm_bncs_output@@AAEXPAVresponse@@@Z$9 1001a7d9 f   alm_bncs_output.obj
 0001:000197e2       __unwindfunclet$?replyLock@alm_bncs_output@@AAEXPAVresponse@@@Z$10 1001a7e2 f   alm_bncs_output.obj
 0001:000197eb       __unwindfunclet$?replyLock@alm_bncs_output@@AAEXPAVresponse@@@Z$11 1001a7eb f   alm_bncs_output.obj
 0001:000197f4       __unwindfunclet$?replyLock@alm_bncs_output@@AAEXPAVresponse@@@Z$12 1001a7f4 f   alm_bncs_output.obj
 0001:000197fd       __unwindfunclet$?replyLock@alm_bncs_output@@AAEXPAVresponse@@@Z$13 1001a7fd f   alm_bncs_output.obj
 0001:00019806       __ehhandler$?replyLock@alm_bncs_output@@AAEXPAVresponse@@@Z 1001a806 f   alm_bncs_output.obj
 0001:00019821       __unwindfunclet$?saveFile@alm_bncs_output@@AAE_NQAVcOutputFile@@_N1@Z$0 1001a821 f   alm_bncs_output.obj
 0001:0001982a       __unwindfunclet$?saveFile@alm_bncs_output@@AAE_NQAVcOutputFile@@_N1@Z$1 1001a82a f   alm_bncs_output.obj
 0001:00019833       __unwindfunclet$?saveFile@alm_bncs_output@@AAE_NQAVcOutputFile@@_N1@Z$2 1001a833 f   alm_bncs_output.obj
 0001:0001983f       __unwindfunclet$?saveFile@alm_bncs_output@@AAE_NQAVcOutputFile@@_N1@Z$3 1001a83f f   alm_bncs_output.obj
 0001:00019848       __unwindfunclet$?saveFile@alm_bncs_output@@AAE_NQAVcOutputFile@@_N1@Z$4 1001a848 f   alm_bncs_output.obj
 0001:00019851       __unwindfunclet$?saveFile@alm_bncs_output@@AAE_NQAVcOutputFile@@_N1@Z$5 1001a851 f   alm_bncs_output.obj
 0001:0001985a       __unwindfunclet$?saveFile@alm_bncs_output@@AAE_NQAVcOutputFile@@_N1@Z$6 1001a85a f   alm_bncs_output.obj
 0001:00019863       __unwindfunclet$?saveFile@alm_bncs_output@@AAE_NQAVcOutputFile@@_N1@Z$7 1001a863 f   alm_bncs_output.obj
 0001:0001986c       __unwindfunclet$?saveFile@alm_bncs_output@@AAE_NQAVcOutputFile@@_N1@Z$8 1001a86c f   alm_bncs_output.obj
 0001:00019875       __unwindfunclet$?saveFile@alm_bncs_output@@AAE_NQAVcOutputFile@@_N1@Z$9 1001a875 f   alm_bncs_output.obj
 0001:0001987e       __unwindfunclet$?saveFile@alm_bncs_output@@AAE_NQAVcOutputFile@@_N1@Z$10 1001a87e f   alm_bncs_output.obj
 0001:00019887       __unwindfunclet$?saveFile@alm_bncs_output@@AAE_NQAVcOutputFile@@_N1@Z$11 1001a887 f   alm_bncs_output.obj
 0001:00019890       __unwindfunclet$?saveFile@alm_bncs_output@@AAE_NQAVcOutputFile@@_N1@Z$12 1001a890 f   alm_bncs_output.obj
 0001:00019899       __unwindfunclet$?saveFile@alm_bncs_output@@AAE_NQAVcOutputFile@@_N1@Z$13 1001a899 f   alm_bncs_output.obj
 0001:000198a2       __unwindfunclet$?saveFile@alm_bncs_output@@AAE_NQAVcOutputFile@@_N1@Z$14 1001a8a2 f   alm_bncs_output.obj
 0001:000198ab       __unwindfunclet$?saveFile@alm_bncs_output@@AAE_NQAVcOutputFile@@_N1@Z$15 1001a8ab f   alm_bncs_output.obj
 0001:000198b4       __unwindfunclet$?saveFile@alm_bncs_output@@AAE_NQAVcOutputFile@@_N1@Z$16 1001a8b4 f   alm_bncs_output.obj
 0001:000198bd       __unwindfunclet$?saveFile@alm_bncs_output@@AAE_NQAVcOutputFile@@_N1@Z$17 1001a8bd f   alm_bncs_output.obj
 0001:000198c6       __unwindfunclet$?saveFile@alm_bncs_output@@AAE_NQAVcOutputFile@@_N1@Z$18 1001a8c6 f   alm_bncs_output.obj
 0001:000198cf       __ehhandler$?saveFile@alm_bncs_output@@AAE_NQAVcOutputFile@@_N1@Z 1001a8cf f   alm_bncs_output.obj
 0001:000198ed       __unwindfunclet$?saveTemplates@alm_bncs_output@@AAEXPBVcOutputFile@@_NAAVQString@@2@Z$0 1001a8ed f   alm_bncs_output.obj
 0001:000198f8       __unwindfunclet$?saveTemplates@alm_bncs_output@@AAEXPBVcOutputFile@@_NAAVQString@@2@Z$1 1001a8f8 f   alm_bncs_output.obj
 0001:00019901       __unwindfunclet$?saveTemplates@alm_bncs_output@@AAEXPBVcOutputFile@@_NAAVQString@@2@Z$2 1001a901 f   alm_bncs_output.obj
 0001:0001990a       __unwindfunclet$?saveTemplates@alm_bncs_output@@AAEXPBVcOutputFile@@_NAAVQString@@2@Z$3 1001a90a f   alm_bncs_output.obj
 0001:00019913       __unwindfunclet$?saveTemplates@alm_bncs_output@@AAEXPBVcOutputFile@@_NAAVQString@@2@Z$4 1001a913 f   alm_bncs_output.obj
 0001:0001991c       __unwindfunclet$?saveTemplates@alm_bncs_output@@AAEXPBVcOutputFile@@_NAAVQString@@2@Z$5 1001a91c f   alm_bncs_output.obj
 0001:00019925       __unwindfunclet$?saveTemplates@alm_bncs_output@@AAEXPBVcOutputFile@@_NAAVQString@@2@Z$6 1001a925 f   alm_bncs_output.obj
 0001:0001992e       __unwindfunclet$?saveTemplates@alm_bncs_output@@AAEXPBVcOutputFile@@_NAAVQString@@2@Z$7 1001a92e f   alm_bncs_output.obj
 0001:00019937       __unwindfunclet$?saveTemplates@alm_bncs_output@@AAEXPBVcOutputFile@@_NAAVQString@@2@Z$8 1001a937 f   alm_bncs_output.obj
 0001:00019940       __unwindfunclet$?saveTemplates@alm_bncs_output@@AAEXPBVcOutputFile@@_NAAVQString@@2@Z$9 1001a940 f   alm_bncs_output.obj
 0001:00019949       __unwindfunclet$?saveTemplates@alm_bncs_output@@AAEXPBVcOutputFile@@_NAAVQString@@2@Z$10 1001a949 f   alm_bncs_output.obj
 0001:00019955       __unwindfunclet$?saveTemplates@alm_bncs_output@@AAEXPBVcOutputFile@@_NAAVQString@@2@Z$11 1001a955 f   alm_bncs_output.obj
 0001:0001995e       __unwindfunclet$?saveTemplates@alm_bncs_output@@AAEXPBVcOutputFile@@_NAAVQString@@2@Z$12 1001a95e f   alm_bncs_output.obj
 0001:00019967       __unwindfunclet$?saveTemplates@alm_bncs_output@@AAEXPBVcOutputFile@@_NAAVQString@@2@Z$13 1001a967 f   alm_bncs_output.obj
 0001:00019970       __unwindfunclet$?saveTemplates@alm_bncs_output@@AAEXPBVcOutputFile@@_NAAVQString@@2@Z$14 1001a970 f   alm_bncs_output.obj
 0001:00019979       __unwindfunclet$?saveTemplates@alm_bncs_output@@AAEXPBVcOutputFile@@_NAAVQString@@2@Z$15 1001a979 f   alm_bncs_output.obj
 0001:00019982       __unwindfunclet$?saveTemplates@alm_bncs_output@@AAEXPBVcOutputFile@@_NAAVQString@@2@Z$16 1001a982 f   alm_bncs_output.obj
 0001:0001998b       __unwindfunclet$?saveTemplates@alm_bncs_output@@AAEXPBVcOutputFile@@_NAAVQString@@2@Z$17 1001a98b f   alm_bncs_output.obj
 0001:00019994       __unwindfunclet$?saveTemplates@alm_bncs_output@@AAEXPBVcOutputFile@@_NAAVQString@@2@Z$18 1001a994 f   alm_bncs_output.obj
 0001:0001999d       __unwindfunclet$?saveTemplates@alm_bncs_output@@AAEXPBVcOutputFile@@_NAAVQString@@2@Z$19 1001a99d f   alm_bncs_output.obj
 0001:000199a6       __unwindfunclet$?saveTemplates@alm_bncs_output@@AAEXPBVcOutputFile@@_NAAVQString@@2@Z$20 1001a9a6 f   alm_bncs_output.obj
 0001:000199af       __unwindfunclet$?saveTemplates@alm_bncs_output@@AAEXPBVcOutputFile@@_NAAVQString@@2@Z$21 1001a9af f   alm_bncs_output.obj
 0001:000199b8       __unwindfunclet$?saveTemplates@alm_bncs_output@@AAEXPBVcOutputFile@@_NAAVQString@@2@Z$22 1001a9b8 f   alm_bncs_output.obj
 0001:000199c1       __unwindfunclet$?saveTemplates@alm_bncs_output@@AAEXPBVcOutputFile@@_NAAVQString@@2@Z$23 1001a9c1 f   alm_bncs_output.obj
 0001:000199ca       __unwindfunclet$?saveTemplates@alm_bncs_output@@AAEXPBVcOutputFile@@_NAAVQString@@2@Z$24 1001a9ca f   alm_bncs_output.obj
 0001:000199d3       __unwindfunclet$?saveTemplates@alm_bncs_output@@AAEXPBVcOutputFile@@_NAAVQString@@2@Z$25 1001a9d3 f   alm_bncs_output.obj
 0001:000199dc       __unwindfunclet$?saveTemplates@alm_bncs_output@@AAEXPBVcOutputFile@@_NAAVQString@@2@Z$28 1001a9dc f   alm_bncs_output.obj
 0001:000199e5       __unwindfunclet$?saveTemplates@alm_bncs_output@@AAEXPBVcOutputFile@@_NAAVQString@@2@Z$29 1001a9e5 f   alm_bncs_output.obj
 0001:000199ee       __unwindfunclet$?saveTemplates@alm_bncs_output@@AAEXPBVcOutputFile@@_NAAVQString@@2@Z$26 1001a9ee f   alm_bncs_output.obj
 0001:000199f7       __unwindfunclet$?saveTemplates@alm_bncs_output@@AAEXPBVcOutputFile@@_NAAVQString@@2@Z$27 1001a9f7 f   alm_bncs_output.obj
 0001:00019a00       __ehhandler$?saveTemplates@alm_bncs_output@@AAEXPBVcOutputFile@@_NAAVQString@@2@Z 1001aa00 f   alm_bncs_output.obj
 0001:00019a1e       __unwindfunclet$?selectFile@alm_bncs_output@@QAEXPAVQListViewItem@@@Z$0 1001aa1e f   alm_bncs_output.obj
 0001:00019a27       __unwindfunclet$?selectFile@alm_bncs_output@@QAEXPAVQListViewItem@@@Z$1 1001aa27 f   alm_bncs_output.obj
 0001:00019a30       __unwindfunclet$?selectFile@alm_bncs_output@@QAEXPAVQListViewItem@@@Z$2 1001aa30 f   alm_bncs_output.obj
 0001:00019a39       __unwindfunclet$?selectFile@alm_bncs_output@@QAEXPAVQListViewItem@@@Z$3 1001aa39 f   alm_bncs_output.obj
 0001:00019a42       __unwindfunclet$?selectFile@alm_bncs_output@@QAEXPAVQListViewItem@@@Z$4 1001aa42 f   alm_bncs_output.obj
 0001:00019a4b       __unwindfunclet$?selectFile@alm_bncs_output@@QAEXPAVQListViewItem@@@Z$5 1001aa4b f   alm_bncs_output.obj
 0001:00019a54       __unwindfunclet$?selectFile@alm_bncs_output@@QAEXPAVQListViewItem@@@Z$6 1001aa54 f   alm_bncs_output.obj
 0001:00019a5d       __unwindfunclet$?selectFile@alm_bncs_output@@QAEXPAVQListViewItem@@@Z$7 1001aa5d f   alm_bncs_output.obj
 0001:00019a66       __unwindfunclet$?selectFile@alm_bncs_output@@QAEXPAVQListViewItem@@@Z$8 1001aa66 f   alm_bncs_output.obj
 0001:00019a6f       __ehhandler$?selectFile@alm_bncs_output@@QAEXPAVQListViewItem@@@Z 1001aa6f f   alm_bncs_output.obj
 0001:00019a8a       __unwindfunclet$?selectSystem@alm_bncs_output@@IAEXABVQString@@@Z$0 1001aa8a f   alm_bncs_output.obj
 0001:00019a93       __unwindfunclet$?selectSystem@alm_bncs_output@@IAEXABVQString@@@Z$1 1001aa93 f   alm_bncs_output.obj
 0001:00019a9c       __unwindfunclet$?selectSystem@alm_bncs_output@@IAEXABVQString@@@Z$2 1001aa9c f   alm_bncs_output.obj
 0001:00019aa5       __unwindfunclet$?selectSystem@alm_bncs_output@@IAEXABVQString@@@Z$3 1001aaa5 f   alm_bncs_output.obj
 0001:00019aae       __unwindfunclet$?selectSystem@alm_bncs_output@@IAEXABVQString@@@Z$4 1001aaae f   alm_bncs_output.obj
 0001:00019ab7       __unwindfunclet$?selectSystem@alm_bncs_output@@IAEXABVQString@@@Z$5 1001aab7 f   alm_bncs_output.obj
 0001:00019ac0       __unwindfunclet$?selectSystem@alm_bncs_output@@IAEXABVQString@@@Z$7 1001aac0 f   alm_bncs_output.obj
 0001:00019ac9       __unwindfunclet$?selectSystem@alm_bncs_output@@IAEXABVQString@@@Z$8 1001aac9 f   alm_bncs_output.obj
 0001:00019ad2       __unwindfunclet$?selectSystem@alm_bncs_output@@IAEXABVQString@@@Z$9 1001aad2 f   alm_bncs_output.obj
 0001:00019adb       __unwindfunclet$?selectSystem@alm_bncs_output@@IAEXABVQString@@@Z$10 1001aadb f   alm_bncs_output.obj
 0001:00019ae4       __unwindfunclet$?selectSystem@alm_bncs_output@@IAEXABVQString@@@Z$11 1001aae4 f   alm_bncs_output.obj
 0001:00019aed       __unwindfunclet$?selectSystem@alm_bncs_output@@IAEXABVQString@@@Z$12 1001aaed f   alm_bncs_output.obj
 0001:00019af6       __unwindfunclet$?selectSystem@alm_bncs_output@@IAEXABVQString@@@Z$13 1001aaf6 f   alm_bncs_output.obj
 0001:00019aff       __ehhandler$?selectSystem@alm_bncs_output@@IAEXABVQString@@@Z 1001aaff f   alm_bncs_output.obj
 0001:00019b1a       __unwindfunclet$?sendCommand@alm_bncs_output@@UAEXABVQString@@0@Z$0 1001ab1a f   alm_bncs_output.obj
 0001:00019b23       __ehhandler$?sendCommand@alm_bncs_output@@UAEXABVQString@@0@Z 1001ab23 f   alm_bncs_output.obj
 0001:00019b3e       __unwindfunclet$?showLockedDevDescFileList@alm_bncs_output@@AAEXXZ$0 1001ab3e f   alm_bncs_output.obj
 0001:00019b47       __unwindfunclet$?showLockedDevDescFileList@alm_bncs_output@@AAEXXZ$1 1001ab47 f   alm_bncs_output.obj
 0001:00019b50       __unwindfunclet$?showLockedDevDescFileList@alm_bncs_output@@AAEXXZ$2 1001ab50 f   alm_bncs_output.obj
 0001:00019b59       __unwindfunclet$?showLockedDevDescFileList@alm_bncs_output@@AAEXXZ$3 1001ab59 f   alm_bncs_output.obj
 0001:00019b62       __ehhandler$?showLockedDevDescFileList@alm_bncs_output@@AAEXXZ 1001ab62 f   alm_bncs_output.obj
 0001:00019b7d       __unwindfunclet$?toolbars@alm_bncs_output@@UAE?AVQDockWindowList@@XZ$0 1001ab7d f   alm_bncs_output.obj
 0001:00019b96       __ehhandler$?toolbars@alm_bncs_output@@UAE?AVQDockWindowList@@XZ 1001ab96 f   alm_bncs_output.obj
 0001:00019bb1       __unwindfunclet$?updateFileList@alm_bncs_output@@AAEXXZ$0 1001abb1 f   alm_bncs_output.obj
 0001:00019bbd       __unwindfunclet$?updateFileList@alm_bncs_output@@AAEXXZ$1 1001abbd f   alm_bncs_output.obj
 0001:00019bc9       __unwindfunclet$?updateFileList@alm_bncs_output@@AAEXXZ$2 1001abc9 f   alm_bncs_output.obj
 0001:00019bd5       __unwindfunclet$?updateFileList@alm_bncs_output@@AAEXXZ$3 1001abd5 f   alm_bncs_output.obj
 0001:00019be1       __unwindfunclet$?updateFileList@alm_bncs_output@@AAEXXZ$4 1001abe1 f   alm_bncs_output.obj
 0001:00019bed       __unwindfunclet$?updateFileList@alm_bncs_output@@AAEXXZ$5 1001abed f   alm_bncs_output.obj
 0001:00019bf9       __unwindfunclet$?updateFileList@alm_bncs_output@@AAEXXZ$6 1001abf9 f   alm_bncs_output.obj
 0001:00019c05       __unwindfunclet$?updateFileList@alm_bncs_output@@AAEXXZ$7 1001ac05 f   alm_bncs_output.obj
 0001:00019c11       __unwindfunclet$?updateFileList@alm_bncs_output@@AAEXXZ$8 1001ac11 f   alm_bncs_output.obj
 0001:00019c1c       __unwindfunclet$?updateFileList@alm_bncs_output@@AAEXXZ$9 1001ac1c f   alm_bncs_output.obj
 0001:00019c28       __unwindfunclet$?updateFileList@alm_bncs_output@@AAEXXZ$10 1001ac28 f   alm_bncs_output.obj
 0001:00019c34       __unwindfunclet$?updateFileList@alm_bncs_output@@AAEXXZ$11 1001ac34 f   alm_bncs_output.obj
 0001:00019c40       __unwindfunclet$?updateFileList@alm_bncs_output@@AAEXXZ$12 1001ac40 f   alm_bncs_output.obj
 0001:00019c4c       __unwindfunclet$?updateFileList@alm_bncs_output@@AAEXXZ$13 1001ac4c f   alm_bncs_output.obj
 0001:00019c58       __unwindfunclet$?updateFileList@alm_bncs_output@@AAEXXZ$14 1001ac58 f   alm_bncs_output.obj
 0001:00019c64       __unwindfunclet$?updateFileList@alm_bncs_output@@AAEXXZ$15 1001ac64 f   alm_bncs_output.obj
 0001:00019c70       __unwindfunclet$?updateFileList@alm_bncs_output@@AAEXXZ$16 1001ac70 f   alm_bncs_output.obj
 0001:00019c7c       __unwindfunclet$?updateFileList@alm_bncs_output@@AAEXXZ$17 1001ac7c f   alm_bncs_output.obj
 0001:00019c88       __unwindfunclet$?updateFileList@alm_bncs_output@@AAEXXZ$18 1001ac88 f   alm_bncs_output.obj
 0001:00019c94       __unwindfunclet$?updateFileList@alm_bncs_output@@AAEXXZ$19 1001ac94 f   alm_bncs_output.obj
 0001:00019ca0       __unwindfunclet$?updateFileList@alm_bncs_output@@AAEXXZ$20 1001aca0 f   alm_bncs_output.obj
 0001:00019cad       __unwindfunclet$?updateFileList@alm_bncs_output@@AAEXXZ$21 1001acad f   alm_bncs_output.obj
 0001:00019cb9       __unwindfunclet$?updateFileList@alm_bncs_output@@AAEXXZ$22 1001acb9 f   alm_bncs_output.obj
 0001:00019cc5       __unwindfunclet$?updateFileList@alm_bncs_output@@AAEXXZ$23 1001acc5 f   alm_bncs_output.obj
 0001:00019cd1       __unwindfunclet$?updateFileList@alm_bncs_output@@AAEXXZ$24 1001acd1 f   alm_bncs_output.obj
 0001:00019cdd       __unwindfunclet$?updateFileList@alm_bncs_output@@AAEXXZ$25 1001acdd f   alm_bncs_output.obj
 0001:00019ce9       __unwindfunclet$?updateFileList@alm_bncs_output@@AAEXXZ$26 1001ace9 f   alm_bncs_output.obj
 0001:00019cf5       __unwindfunclet$?updateFileList@alm_bncs_output@@AAEXXZ$27 1001acf5 f   alm_bncs_output.obj
 0001:00019d01       __unwindfunclet$?updateFileList@alm_bncs_output@@AAEXXZ$29 1001ad01 f   alm_bncs_output.obj
 0001:00019d0d       __unwindfunclet$?updateFileList@alm_bncs_output@@AAEXXZ$30 1001ad0d f   alm_bncs_output.obj
 0001:00019d19       __unwindfunclet$?updateFileList@alm_bncs_output@@AAEXXZ$31 1001ad19 f   alm_bncs_output.obj
 0001:00019d26       __unwindfunclet$?updateFileList@alm_bncs_output@@AAEXXZ$32 1001ad26 f   alm_bncs_output.obj
 0001:00019d32       __unwindfunclet$?updateFileList@alm_bncs_output@@AAEXXZ$33 1001ad32 f   alm_bncs_output.obj
 0001:00019d3e       __unwindfunclet$?updateFileList@alm_bncs_output@@AAEXXZ$34 1001ad3e f   alm_bncs_output.obj
 0001:00019d4b       __unwindfunclet$?updateFileList@alm_bncs_output@@AAEXXZ$35 1001ad4b f   alm_bncs_output.obj
 0001:00019d57       __unwindfunclet$?updateFileList@alm_bncs_output@@AAEXXZ$36 1001ad57 f   alm_bncs_output.obj
 0001:00019d63       __unwindfunclet$?updateFileList@alm_bncs_output@@AAEXXZ$37 1001ad63 f   alm_bncs_output.obj
 0001:00019d6f       __unwindfunclet$?updateFileList@alm_bncs_output@@AAEXXZ$38 1001ad6f f   alm_bncs_output.obj
 0001:00019d7b       __unwindfunclet$?updateFileList@alm_bncs_output@@AAEXXZ$39 1001ad7b f   alm_bncs_output.obj
 0001:00019d87       __unwindfunclet$?updateFileList@alm_bncs_output@@AAEXXZ$40 1001ad87 f   alm_bncs_output.obj
 0001:00019d93       __unwindfunclet$?updateFileList@alm_bncs_output@@AAEXXZ$41 1001ad93 f   alm_bncs_output.obj
 0001:00019d9f       __ehhandler$?updateFileList@alm_bncs_output@@AAEXXZ 1001ad9f f   alm_bncs_output.obj
 0001:00019dc7       __unwindfunclet$?writeDefaultDevicetypesFile@alm_bncs_output@@AAEXXZ$0 1001adc7 f   alm_bncs_output.obj
 0001:00019dd0       __unwindfunclet$?writeDefaultDevicetypesFile@alm_bncs_output@@AAEXXZ$1 1001add0 f   alm_bncs_output.obj
 0001:00019dd9       __unwindfunclet$?writeDefaultDevicetypesFile@alm_bncs_output@@AAEXXZ$2 1001add9 f   alm_bncs_output.obj
 0001:00019de2       __unwindfunclet$?writeDefaultDevicetypesFile@alm_bncs_output@@AAEXXZ$3 1001ade2 f   alm_bncs_output.obj
 0001:00019deb       __unwindfunclet$?writeDefaultDevicetypesFile@alm_bncs_output@@AAEXXZ$4 1001adeb f   alm_bncs_output.obj
 0001:00019df4       __unwindfunclet$?writeDefaultDevicetypesFile@alm_bncs_output@@AAEXXZ$5 1001adf4 f   alm_bncs_output.obj
 0001:00019dfd       __unwindfunclet$?writeDefaultDevicetypesFile@alm_bncs_output@@AAEXXZ$6 1001adfd f   alm_bncs_output.obj
 0001:00019e06       __unwindfunclet$?writeDefaultDevicetypesFile@alm_bncs_output@@AAEXXZ$7 1001ae06 f   alm_bncs_output.obj
 0001:00019e0f       __unwindfunclet$?writeDefaultDevicetypesFile@alm_bncs_output@@AAEXXZ$9 1001ae0f f   alm_bncs_output.obj
 0001:00019e18       __unwindfunclet$?writeDefaultDevicetypesFile@alm_bncs_output@@AAEXXZ$10 1001ae18 f   alm_bncs_output.obj
 0001:00019e21       __unwindfunclet$?writeDefaultDevicetypesFile@alm_bncs_output@@AAEXXZ$11 1001ae21 f   alm_bncs_output.obj
 0001:00019e2a       __unwindfunclet$?writeDefaultDevicetypesFile@alm_bncs_output@@AAEXXZ$12 1001ae2a f   alm_bncs_output.obj
 0001:00019e33       __unwindfunclet$?writeDefaultDevicetypesFile@alm_bncs_output@@AAEXXZ$13 1001ae33 f   alm_bncs_output.obj
 0001:00019e3c       __unwindfunclet$?writeDefaultDevicetypesFile@alm_bncs_output@@AAEXXZ$14 1001ae3c f   alm_bncs_output.obj
 0001:00019e44       __unwindfunclet$?writeDefaultDevicetypesFile@alm_bncs_output@@AAEXXZ$15 1001ae44 f   alm_bncs_output.obj
 0001:00019e4d       __unwindfunclet$?writeDefaultDevicetypesFile@alm_bncs_output@@AAEXXZ$16 1001ae4d f   alm_bncs_output.obj
 0001:00019e56       __unwindfunclet$?writeDefaultDevicetypesFile@alm_bncs_output@@AAEXXZ$17 1001ae56 f   alm_bncs_output.obj
 0001:00019e5f       __unwindfunclet$?writeDefaultDevicetypesFile@alm_bncs_output@@AAEXXZ$18 1001ae5f f   alm_bncs_output.obj
 0001:00019e68       __unwindfunclet$?writeDefaultDevicetypesFile@alm_bncs_output@@AAEXXZ$19 1001ae68 f   alm_bncs_output.obj
 0001:00019e71       __unwindfunclet$?writeDefaultDevicetypesFile@alm_bncs_output@@AAEXXZ$20 1001ae71 f   alm_bncs_output.obj
 0001:00019e7a       __unwindfunclet$?writeDefaultDevicetypesFile@alm_bncs_output@@AAEXXZ$22 1001ae7a f   alm_bncs_output.obj
 0001:00019e83       __unwindfunclet$?writeDefaultDevicetypesFile@alm_bncs_output@@AAEXXZ$23 1001ae83 f   alm_bncs_output.obj
 0001:00019e8c       __unwindfunclet$?writeDefaultDevicetypesFile@alm_bncs_output@@AAEXXZ$24 1001ae8c f   alm_bncs_output.obj
 0001:00019e95       __unwindfunclet$?writeDefaultDevicetypesFile@alm_bncs_output@@AAEXXZ$25 1001ae95 f   alm_bncs_output.obj
 0001:00019e9e       __unwindfunclet$?writeDefaultDevicetypesFile@alm_bncs_output@@AAEXXZ$26 1001ae9e f   alm_bncs_output.obj
 0001:00019ea7       __unwindfunclet$?writeDefaultDevicetypesFile@alm_bncs_output@@AAEXXZ$27 1001aea7 f   alm_bncs_output.obj
 0001:00019eb0       __ehhandler$?writeDefaultDevicetypesFile@alm_bncs_output@@AAEXXZ 1001aeb0 f   alm_bncs_output.obj
 0001:00019ecc       __unwindfunclet$?writeDevDescFile@alm_bncs_output@@AAEXQBVcOutputFile@@_N@Z$0 1001aecc f   alm_bncs_output.obj
 0001:00019ed5       __unwindfunclet$?writeDevDescFile@alm_bncs_output@@AAEXQBVcOutputFile@@_N@Z$1 1001aed5 f   alm_bncs_output.obj
 0001:00019ede       __unwindfunclet$?writeDevDescFile@alm_bncs_output@@AAEXQBVcOutputFile@@_N@Z$2 1001aede f   alm_bncs_output.obj
 0001:00019ee7       __unwindfunclet$?writeDevDescFile@alm_bncs_output@@AAEXQBVcOutputFile@@_N@Z$3 1001aee7 f   alm_bncs_output.obj
 0001:00019ef0       __unwindfunclet$?writeDevDescFile@alm_bncs_output@@AAEXQBVcOutputFile@@_N@Z$4 1001aef0 f   alm_bncs_output.obj
 0001:00019ef9       __unwindfunclet$?writeDevDescFile@alm_bncs_output@@AAEXQBVcOutputFile@@_N@Z$5 1001aef9 f   alm_bncs_output.obj
 0001:00019f02       __unwindfunclet$?writeDevDescFile@alm_bncs_output@@AAEXQBVcOutputFile@@_N@Z$6 1001af02 f   alm_bncs_output.obj
 0001:00019f0b       __unwindfunclet$?writeDevDescFile@alm_bncs_output@@AAEXQBVcOutputFile@@_N@Z$7 1001af0b f   alm_bncs_output.obj
 0001:00019f14       __unwindfunclet$?writeDevDescFile@alm_bncs_output@@AAEXQBVcOutputFile@@_N@Z$8 1001af14 f   alm_bncs_output.obj
 0001:00019f1d       __unwindfunclet$?writeDevDescFile@alm_bncs_output@@AAEXQBVcOutputFile@@_N@Z$9 1001af1d f   alm_bncs_output.obj
 0001:00019f26       __unwindfunclet$?writeDevDescFile@alm_bncs_output@@AAEXQBVcOutputFile@@_N@Z$10 1001af26 f   alm_bncs_output.obj
 0001:00019f2f       __unwindfunclet$?writeDevDescFile@alm_bncs_output@@AAEXQBVcOutputFile@@_N@Z$11 1001af2f f   alm_bncs_output.obj
 0001:00019f38       __unwindfunclet$?writeDevDescFile@alm_bncs_output@@AAEXQBVcOutputFile@@_N@Z$12 1001af38 f   alm_bncs_output.obj
 0001:00019f41       __unwindfunclet$?writeDevDescFile@alm_bncs_output@@AAEXQBVcOutputFile@@_N@Z$13 1001af41 f   alm_bncs_output.obj
 0001:00019f4a       __unwindfunclet$?writeDevDescFile@alm_bncs_output@@AAEXQBVcOutputFile@@_N@Z$14 1001af4a f   alm_bncs_output.obj
 0001:00019f53       __unwindfunclet$?writeDevDescFile@alm_bncs_output@@AAEXQBVcOutputFile@@_N@Z$15 1001af53 f   alm_bncs_output.obj
 0001:00019f5f       __unwindfunclet$?writeDevDescFile@alm_bncs_output@@AAEXQBVcOutputFile@@_N@Z$16 1001af5f f   alm_bncs_output.obj
 0001:00019f68       __unwindfunclet$?writeDevDescFile@alm_bncs_output@@AAEXQBVcOutputFile@@_N@Z$17 1001af68 f   alm_bncs_output.obj
 0001:00019f71       __unwindfunclet$?writeDevDescFile@alm_bncs_output@@AAEXQBVcOutputFile@@_N@Z$18 1001af71 f   alm_bncs_output.obj
 0001:00019f7a       __unwindfunclet$?writeDevDescFile@alm_bncs_output@@AAEXQBVcOutputFile@@_N@Z$19 1001af7a f   alm_bncs_output.obj
 0001:00019f83       __unwindfunclet$?writeDevDescFile@alm_bncs_output@@AAEXQBVcOutputFile@@_N@Z$20 1001af83 f   alm_bncs_output.obj
 0001:00019f8c       __unwindfunclet$?writeDevDescFile@alm_bncs_output@@AAEXQBVcOutputFile@@_N@Z$21 1001af8c f   alm_bncs_output.obj
 0001:00019f95       __unwindfunclet$?writeDevDescFile@alm_bncs_output@@AAEXQBVcOutputFile@@_N@Z$22 1001af95 f   alm_bncs_output.obj
 0001:00019f9e       __unwindfunclet$?writeDevDescFile@alm_bncs_output@@AAEXQBVcOutputFile@@_N@Z$23 1001af9e f   alm_bncs_output.obj
 0001:00019fa7       __unwindfunclet$?writeDevDescFile@alm_bncs_output@@AAEXQBVcOutputFile@@_N@Z$24 1001afa7 f   alm_bncs_output.obj
 0001:00019fb3       __unwindfunclet$?writeDevDescFile@alm_bncs_output@@AAEXQBVcOutputFile@@_N@Z$25 1001afb3 f   alm_bncs_output.obj
 0001:00019fbc       __unwindfunclet$?writeDevDescFile@alm_bncs_output@@AAEXQBVcOutputFile@@_N@Z$26 1001afbc f   alm_bncs_output.obj
 0001:00019fc5       __unwindfunclet$?writeDevDescFile@alm_bncs_output@@AAEXQBVcOutputFile@@_N@Z$27 1001afc5 f   alm_bncs_output.obj
 0001:00019fce       __unwindfunclet$?writeDevDescFile@alm_bncs_output@@AAEXQBVcOutputFile@@_N@Z$28 1001afce f   alm_bncs_output.obj
 0001:00019fd7       __unwindfunclet$?writeDevDescFile@alm_bncs_output@@AAEXQBVcOutputFile@@_N@Z$29 1001afd7 f   alm_bncs_output.obj
 0001:00019fe0       __unwindfunclet$?writeDevDescFile@alm_bncs_output@@AAEXQBVcOutputFile@@_N@Z$30 1001afe0 f   alm_bncs_output.obj
 0001:00019fe9       __unwindfunclet$?writeDevDescFile@alm_bncs_output@@AAEXQBVcOutputFile@@_N@Z$31 1001afe9 f   alm_bncs_output.obj
 0001:00019ff2       __unwindfunclet$?writeDevDescFile@alm_bncs_output@@AAEXQBVcOutputFile@@_N@Z$32 1001aff2 f   alm_bncs_output.obj
 0001:00019ffb       __unwindfunclet$?writeDevDescFile@alm_bncs_output@@AAEXQBVcOutputFile@@_N@Z$33 1001affb f   alm_bncs_output.obj
 0001:0001a004       __unwindfunclet$?writeDevDescFile@alm_bncs_output@@AAEXQBVcOutputFile@@_N@Z$34 1001b004 f   alm_bncs_output.obj
 0001:0001a00d       __unwindfunclet$?writeDevDescFile@alm_bncs_output@@AAEXQBVcOutputFile@@_N@Z$35 1001b00d f   alm_bncs_output.obj
 0001:0001a016       __unwindfunclet$?writeDevDescFile@alm_bncs_output@@AAEXQBVcOutputFile@@_N@Z$36 1001b016 f   alm_bncs_output.obj
 0001:0001a01f       __unwindfunclet$?writeDevDescFile@alm_bncs_output@@AAEXQBVcOutputFile@@_N@Z$37 1001b01f f   alm_bncs_output.obj
 0001:0001a028       __unwindfunclet$?writeDevDescFile@alm_bncs_output@@AAEXQBVcOutputFile@@_N@Z$38 1001b028 f   alm_bncs_output.obj
 0001:0001a031       __unwindfunclet$?writeDevDescFile@alm_bncs_output@@AAEXQBVcOutputFile@@_N@Z$39 1001b031 f   alm_bncs_output.obj
 0001:0001a03a       __unwindfunclet$?writeDevDescFile@alm_bncs_output@@AAEXQBVcOutputFile@@_N@Z$40 1001b03a f   alm_bncs_output.obj
 0001:0001a043       __unwindfunclet$?writeDevDescFile@alm_bncs_output@@AAEXQBVcOutputFile@@_N@Z$41 1001b043 f   alm_bncs_output.obj
 0001:0001a04c       __ehhandler$?writeDevDescFile@alm_bncs_output@@AAEXQBVcOutputFile@@_N@Z 1001b04c f   alm_bncs_output.obj
 0001:0001a06a       __unwindfunclet$?writeDeviceTypesFile@alm_bncs_output@@AAE_NQBVcOutputFile@@@Z$0 1001b06a f   alm_bncs_output.obj
 0001:0001a073       __unwindfunclet$?writeDeviceTypesFile@alm_bncs_output@@AAE_NQBVcOutputFile@@@Z$1 1001b073 f   alm_bncs_output.obj
 0001:0001a07c       __unwindfunclet$?writeDeviceTypesFile@alm_bncs_output@@AAE_NQBVcOutputFile@@@Z$2 1001b07c f   alm_bncs_output.obj
 0001:0001a088       __unwindfunclet$?writeDeviceTypesFile@alm_bncs_output@@AAE_NQBVcOutputFile@@@Z$3 1001b088 f   alm_bncs_output.obj
 0001:0001a091       __unwindfunclet$?writeDeviceTypesFile@alm_bncs_output@@AAE_NQBVcOutputFile@@@Z$4 1001b091 f   alm_bncs_output.obj
 0001:0001a09a       __unwindfunclet$?writeDeviceTypesFile@alm_bncs_output@@AAE_NQBVcOutputFile@@@Z$5 1001b09a f   alm_bncs_output.obj
 0001:0001a0a3       __unwindfunclet$?writeDeviceTypesFile@alm_bncs_output@@AAE_NQBVcOutputFile@@@Z$6 1001b0a3 f   alm_bncs_output.obj
 0001:0001a0ac       __unwindfunclet$?writeDeviceTypesFile@alm_bncs_output@@AAE_NQBVcOutputFile@@@Z$7 1001b0ac f   alm_bncs_output.obj
 0001:0001a0b5       __unwindfunclet$?writeDeviceTypesFile@alm_bncs_output@@AAE_NQBVcOutputFile@@@Z$8 1001b0b5 f   alm_bncs_output.obj
 0001:0001a0be       __unwindfunclet$?writeDeviceTypesFile@alm_bncs_output@@AAE_NQBVcOutputFile@@@Z$9 1001b0be f   alm_bncs_output.obj
 0001:0001a0c7       __unwindfunclet$?writeDeviceTypesFile@alm_bncs_output@@AAE_NQBVcOutputFile@@@Z$10 1001b0c7 f   alm_bncs_output.obj
 0001:0001a0d0       __unwindfunclet$?writeDeviceTypesFile@alm_bncs_output@@AAE_NQBVcOutputFile@@@Z$11 1001b0d0 f   alm_bncs_output.obj
 0001:0001a0d9       __unwindfunclet$?writeDeviceTypesFile@alm_bncs_output@@AAE_NQBVcOutputFile@@@Z$12 1001b0d9 f   alm_bncs_output.obj
 0001:0001a0e2       __unwindfunclet$?writeDeviceTypesFile@alm_bncs_output@@AAE_NQBVcOutputFile@@@Z$13 1001b0e2 f   alm_bncs_output.obj
 0001:0001a0eb       __unwindfunclet$?writeDeviceTypesFile@alm_bncs_output@@AAE_NQBVcOutputFile@@@Z$14 1001b0eb f   alm_bncs_output.obj
 0001:0001a0f4       __unwindfunclet$?writeDeviceTypesFile@alm_bncs_output@@AAE_NQBVcOutputFile@@@Z$15 1001b0f4 f   alm_bncs_output.obj
 0001:0001a0fd       __unwindfunclet$?writeDeviceTypesFile@alm_bncs_output@@AAE_NQBVcOutputFile@@@Z$16 1001b0fd f   alm_bncs_output.obj
 0001:0001a106       __unwindfunclet$?writeDeviceTypesFile@alm_bncs_output@@AAE_NQBVcOutputFile@@@Z$17 1001b106 f   alm_bncs_output.obj
 0001:0001a10f       __unwindfunclet$?writeDeviceTypesFile@alm_bncs_output@@AAE_NQBVcOutputFile@@@Z$18 1001b10f f   alm_bncs_output.obj
 0001:0001a11a       __unwindfunclet$?writeDeviceTypesFile@alm_bncs_output@@AAE_NQBVcOutputFile@@@Z$19 1001b11a f   alm_bncs_output.obj
 0001:0001a123       __unwindfunclet$?writeDeviceTypesFile@alm_bncs_output@@AAE_NQBVcOutputFile@@@Z$20 1001b123 f   alm_bncs_output.obj
 0001:0001a12c       __unwindfunclet$?writeDeviceTypesFile@alm_bncs_output@@AAE_NQBVcOutputFile@@@Z$21 1001b12c f   alm_bncs_output.obj
 0001:0001a135       __unwindfunclet$?writeDeviceTypesFile@alm_bncs_output@@AAE_NQBVcOutputFile@@@Z$22 1001b135 f   alm_bncs_output.obj
 0001:0001a13e       __unwindfunclet$?writeDeviceTypesFile@alm_bncs_output@@AAE_NQBVcOutputFile@@@Z$23 1001b13e f   alm_bncs_output.obj
 0001:0001a147       __unwindfunclet$?writeDeviceTypesFile@alm_bncs_output@@AAE_NQBVcOutputFile@@@Z$24 1001b147 f   alm_bncs_output.obj
 0001:0001a150       __unwindfunclet$?writeDeviceTypesFile@alm_bncs_output@@AAE_NQBVcOutputFile@@@Z$25 1001b150 f   alm_bncs_output.obj
 0001:0001a159       __unwindfunclet$?writeDeviceTypesFile@alm_bncs_output@@AAE_NQBVcOutputFile@@@Z$26 1001b159 f   alm_bncs_output.obj
 0001:0001a162       __unwindfunclet$?writeDeviceTypesFile@alm_bncs_output@@AAE_NQBVcOutputFile@@@Z$27 1001b162 f   alm_bncs_output.obj
 0001:0001a16b       __unwindfunclet$?writeDeviceTypesFile@alm_bncs_output@@AAE_NQBVcOutputFile@@@Z$28 1001b16b f   alm_bncs_output.obj
 0001:0001a174       __unwindfunclet$?writeDeviceTypesFile@alm_bncs_output@@AAE_NQBVcOutputFile@@@Z$29 1001b174 f   alm_bncs_output.obj
 0001:0001a17d       __unwindfunclet$?writeDeviceTypesFile@alm_bncs_output@@AAE_NQBVcOutputFile@@@Z$30 1001b17d f   alm_bncs_output.obj
 0001:0001a186       __unwindfunclet$?writeDeviceTypesFile@alm_bncs_output@@AAE_NQBVcOutputFile@@@Z$31 1001b186 f   alm_bncs_output.obj
 0001:0001a192       __unwindfunclet$?writeDeviceTypesFile@alm_bncs_output@@AAE_NQBVcOutputFile@@@Z$32 1001b192 f   alm_bncs_output.obj
 0001:0001a19b       __unwindfunclet$?writeDeviceTypesFile@alm_bncs_output@@AAE_NQBVcOutputFile@@@Z$33 1001b19b f   alm_bncs_output.obj
 0001:0001a1a4       __unwindfunclet$?writeDeviceTypesFile@alm_bncs_output@@AAE_NQBVcOutputFile@@@Z$34 1001b1a4 f   alm_bncs_output.obj
 0001:0001a1ad       __unwindfunclet$?writeDeviceTypesFile@alm_bncs_output@@AAE_NQBVcOutputFile@@@Z$35 1001b1ad f   alm_bncs_output.obj
 0001:0001a1b6       __unwindfunclet$?writeDeviceTypesFile@alm_bncs_output@@AAE_NQBVcOutputFile@@@Z$36 1001b1b6 f   alm_bncs_output.obj
 0001:0001a1bf       __unwindfunclet$?writeDeviceTypesFile@alm_bncs_output@@AAE_NQBVcOutputFile@@@Z$37 1001b1bf f   alm_bncs_output.obj
 0001:0001a1c8       __unwindfunclet$?writeDeviceTypesFile@alm_bncs_output@@AAE_NQBVcOutputFile@@@Z$38 1001b1c8 f   alm_bncs_output.obj
 0001:0001a1d4       __unwindfunclet$?writeDeviceTypesFile@alm_bncs_output@@AAE_NQBVcOutputFile@@@Z$39 1001b1d4 f   alm_bncs_output.obj
 0001:0001a1dd       __unwindfunclet$?writeDeviceTypesFile@alm_bncs_output@@AAE_NQBVcOutputFile@@@Z$40 1001b1dd f   alm_bncs_output.obj
 0001:0001a1e9       __unwindfunclet$?writeDeviceTypesFile@alm_bncs_output@@AAE_NQBVcOutputFile@@@Z$41 1001b1e9 f   alm_bncs_output.obj
 0001:0001a1f2       __unwindfunclet$?writeDeviceTypesFile@alm_bncs_output@@AAE_NQBVcOutputFile@@@Z$42 1001b1f2 f   alm_bncs_output.obj
 0001:0001a1fe       __unwindfunclet$?writeDeviceTypesFile@alm_bncs_output@@AAE_NQBVcOutputFile@@@Z$43 1001b1fe f   alm_bncs_output.obj
 0001:0001a207       __unwindfunclet$?writeDeviceTypesFile@alm_bncs_output@@AAE_NQBVcOutputFile@@@Z$44 1001b207 f   alm_bncs_output.obj
 0001:0001a210       __unwindfunclet$?writeDeviceTypesFile@alm_bncs_output@@AAE_NQBVcOutputFile@@@Z$45 1001b210 f   alm_bncs_output.obj
 0001:0001a219       __unwindfunclet$?writeDeviceTypesFile@alm_bncs_output@@AAE_NQBVcOutputFile@@@Z$46 1001b219 f   alm_bncs_output.obj
 0001:0001a222       __unwindfunclet$?writeDeviceTypesFile@alm_bncs_output@@AAE_NQBVcOutputFile@@@Z$47 1001b222 f   alm_bncs_output.obj
 0001:0001a22e       __unwindfunclet$?writeDeviceTypesFile@alm_bncs_output@@AAE_NQBVcOutputFile@@@Z$48 1001b22e f   alm_bncs_output.obj
 0001:0001a23a       __unwindfunclet$?writeDeviceTypesFile@alm_bncs_output@@AAE_NQBVcOutputFile@@@Z$49 1001b23a f   alm_bncs_output.obj
 0001:0001a243       __unwindfunclet$?writeDeviceTypesFile@alm_bncs_output@@AAE_NQBVcOutputFile@@@Z$50 1001b243 f   alm_bncs_output.obj
 0001:0001a24c       __unwindfunclet$?writeDeviceTypesFile@alm_bncs_output@@AAE_NQBVcOutputFile@@@Z$51 1001b24c f   alm_bncs_output.obj
 0001:0001a255       __unwindfunclet$?writeDeviceTypesFile@alm_bncs_output@@AAE_NQBVcOutputFile@@@Z$52 1001b255 f   alm_bncs_output.obj
 0001:0001a25e       __unwindfunclet$?writeDeviceTypesFile@alm_bncs_output@@AAE_NQBVcOutputFile@@@Z$53 1001b25e f   alm_bncs_output.obj
 0001:0001a267       __unwindfunclet$?writeDeviceTypesFile@alm_bncs_output@@AAE_NQBVcOutputFile@@@Z$54 1001b267 f   alm_bncs_output.obj
 0001:0001a270       __unwindfunclet$?writeDeviceTypesFile@alm_bncs_output@@AAE_NQBVcOutputFile@@@Z$55 1001b270 f   alm_bncs_output.obj
 0001:0001a279       __unwindfunclet$?writeDeviceTypesFile@alm_bncs_output@@AAE_NQBVcOutputFile@@@Z$56 1001b279 f   alm_bncs_output.obj
 0001:0001a282       __unwindfunclet$?writeDeviceTypesFile@alm_bncs_output@@AAE_NQBVcOutputFile@@@Z$57 1001b282 f   alm_bncs_output.obj
 0001:0001a28b       __unwindfunclet$?writeDeviceTypesFile@alm_bncs_output@@AAE_NQBVcOutputFile@@@Z$58 1001b28b f   alm_bncs_output.obj
 0001:0001a294       __unwindfunclet$?writeDeviceTypesFile@alm_bncs_output@@AAE_NQBVcOutputFile@@@Z$59 1001b294 f   alm_bncs_output.obj
 0001:0001a29d       __unwindfunclet$?writeDeviceTypesFile@alm_bncs_output@@AAE_NQBVcOutputFile@@@Z$60 1001b29d f   alm_bncs_output.obj
 0001:0001a2a6       __unwindfunclet$?writeDeviceTypesFile@alm_bncs_output@@AAE_NQBVcOutputFile@@@Z$61 1001b2a6 f   alm_bncs_output.obj
 0001:0001a2af       __ehhandler$?writeDeviceTypesFile@alm_bncs_output@@AAE_NQBVcOutputFile@@@Z 1001b2af f   alm_bncs_output.obj
 0001:0001a2cd       __unwindfunclet$?writeDomDoc@alm_bncs_output@@EBEXAAVQDomDocument@@ABVQString@@@Z$0 1001b2cd f   alm_bncs_output.obj
 0001:0001a2d6       __unwindfunclet$?writeDomDoc@alm_bncs_output@@EBEXAAVQDomDocument@@ABVQString@@@Z$1 1001b2d6 f   alm_bncs_output.obj
 0001:0001a2df       __unwindfunclet$?writeDomDoc@alm_bncs_output@@EBEXAAVQDomDocument@@ABVQString@@@Z$2 1001b2df f   alm_bncs_output.obj
 0001:0001a2e8       __unwindfunclet$?writeDomDoc@alm_bncs_output@@EBEXAAVQDomDocument@@ABVQString@@@Z$3 1001b2e8 f   alm_bncs_output.obj
 0001:0001a2f1       __unwindfunclet$?writeDomDoc@alm_bncs_output@@EBEXAAVQDomDocument@@ABVQString@@@Z$4 1001b2f1 f   alm_bncs_output.obj
 0001:0001a2fa       __unwindfunclet$?writeDomDoc@alm_bncs_output@@EBEXAAVQDomDocument@@ABVQString@@@Z$5 1001b2fa f   alm_bncs_output.obj
 0001:0001a303       __unwindfunclet$?writeDomDoc@alm_bncs_output@@EBEXAAVQDomDocument@@ABVQString@@@Z$6 1001b303 f   alm_bncs_output.obj
 0001:0001a30f       __ehhandler$?writeDomDoc@alm_bncs_output@@EBEXAAVQDomDocument@@ABVQString@@@Z 1001b30f f   alm_bncs_output.obj
 0001:0001a32d       __unwindfunclet$?writeEmptyDevicetypesFile@alm_bncs_output@@AAEXABVQString@@@Z$0 1001b32d f   alm_bncs_output.obj
 0001:0001a336       __unwindfunclet$?writeEmptyDevicetypesFile@alm_bncs_output@@AAEXABVQString@@@Z$1 1001b336 f   alm_bncs_output.obj
 0001:0001a33f       __unwindfunclet$?writeEmptyDevicetypesFile@alm_bncs_output@@AAEXABVQString@@@Z$2 1001b33f f   alm_bncs_output.obj
 0001:0001a348       __unwindfunclet$?writeEmptyDevicetypesFile@alm_bncs_output@@AAEXABVQString@@@Z$3 1001b348 f   alm_bncs_output.obj
 0001:0001a351       __unwindfunclet$?writeEmptyDevicetypesFile@alm_bncs_output@@AAEXABVQString@@@Z$4 1001b351 f   alm_bncs_output.obj
 0001:0001a35a       __unwindfunclet$?writeEmptyDevicetypesFile@alm_bncs_output@@AAEXABVQString@@@Z$5 1001b35a f   alm_bncs_output.obj
 0001:0001a363       __unwindfunclet$?writeEmptyDevicetypesFile@alm_bncs_output@@AAEXABVQString@@@Z$7 1001b363 f   alm_bncs_output.obj
 0001:0001a36c       __unwindfunclet$?writeEmptyDevicetypesFile@alm_bncs_output@@AAEXABVQString@@@Z$8 1001b36c f   alm_bncs_output.obj
 0001:0001a375       __unwindfunclet$?writeEmptyDevicetypesFile@alm_bncs_output@@AAEXABVQString@@@Z$9 1001b375 f   alm_bncs_output.obj
 0001:0001a37e       __unwindfunclet$?writeEmptyDevicetypesFile@alm_bncs_output@@AAEXABVQString@@@Z$10 1001b37e f   alm_bncs_output.obj
 0001:0001a387       __unwindfunclet$?writeEmptyDevicetypesFile@alm_bncs_output@@AAEXABVQString@@@Z$11 1001b387 f   alm_bncs_output.obj
 0001:0001a390       __unwindfunclet$?writeEmptyDevicetypesFile@alm_bncs_output@@AAEXABVQString@@@Z$12 1001b390 f   alm_bncs_output.obj
 0001:0001a399       __ehhandler$?writeEmptyDevicetypesFile@alm_bncs_output@@AAEXABVQString@@@Z 1001b399 f   alm_bncs_output.obj
 0001:0001a3b4       __unwindfunclet$?writeEmptyInstancesFile@alm_bncs_output@@AAEXABVQString@@@Z$0 1001b3b4 f   alm_bncs_output.obj
 0001:0001a3bd       __unwindfunclet$?writeEmptyInstancesFile@alm_bncs_output@@AAEXABVQString@@@Z$1 1001b3bd f   alm_bncs_output.obj
 0001:0001a3c6       __unwindfunclet$?writeEmptyInstancesFile@alm_bncs_output@@AAEXABVQString@@@Z$2 1001b3c6 f   alm_bncs_output.obj
 0001:0001a3cf       __unwindfunclet$?writeEmptyInstancesFile@alm_bncs_output@@AAEXABVQString@@@Z$3 1001b3cf f   alm_bncs_output.obj
 0001:0001a3d8       __unwindfunclet$?writeEmptyInstancesFile@alm_bncs_output@@AAEXABVQString@@@Z$4 1001b3d8 f   alm_bncs_output.obj
 0001:0001a3e1       __unwindfunclet$?writeEmptyInstancesFile@alm_bncs_output@@AAEXABVQString@@@Z$5 1001b3e1 f   alm_bncs_output.obj
 0001:0001a3ea       __unwindfunclet$?writeEmptyInstancesFile@alm_bncs_output@@AAEXABVQString@@@Z$7 1001b3ea f   alm_bncs_output.obj
 0001:0001a3f3       __unwindfunclet$?writeEmptyInstancesFile@alm_bncs_output@@AAEXABVQString@@@Z$8 1001b3f3 f   alm_bncs_output.obj
 0001:0001a3fc       __unwindfunclet$?writeEmptyInstancesFile@alm_bncs_output@@AAEXABVQString@@@Z$9 1001b3fc f   alm_bncs_output.obj
 0001:0001a405       __unwindfunclet$?writeEmptyInstancesFile@alm_bncs_output@@AAEXABVQString@@@Z$10 1001b405 f   alm_bncs_output.obj
 0001:0001a40e       __unwindfunclet$?writeEmptyInstancesFile@alm_bncs_output@@AAEXABVQString@@@Z$11 1001b40e f   alm_bncs_output.obj
 0001:0001a417       __unwindfunclet$?writeEmptyInstancesFile@alm_bncs_output@@AAEXABVQString@@@Z$12 1001b417 f   alm_bncs_output.obj
 0001:0001a420       __unwindfunclet$?writeEmptyInstancesFile@alm_bncs_output@@AAEXABVQString@@@Z$13 1001b420 f   alm_bncs_output.obj
 0001:0001a429       __unwindfunclet$?writeEmptyInstancesFile@alm_bncs_output@@AAEXABVQString@@@Z$14 1001b429 f   alm_bncs_output.obj
 0001:0001a432       __unwindfunclet$?writeEmptyInstancesFile@alm_bncs_output@@AAEXABVQString@@@Z$15 1001b432 f   alm_bncs_output.obj
 0001:0001a43b       __ehhandler$?writeEmptyInstancesFile@alm_bncs_output@@AAEXABVQString@@@Z 1001b43b f   alm_bncs_output.obj
 0001:0001a456       __unwindfunclet$?writeInstances@alm_bncs_output@@AAE_NXZ$0 1001b456 f   alm_bncs_output.obj
 0001:0001a45f       __unwindfunclet$?writeInstances@alm_bncs_output@@AAE_NXZ$1 1001b45f f   alm_bncs_output.obj
 0001:0001a468       __unwindfunclet$?writeInstances@alm_bncs_output@@AAE_NXZ$2 1001b468 f   alm_bncs_output.obj
 0001:0001a474       __unwindfunclet$?writeInstances@alm_bncs_output@@AAE_NXZ$3 1001b474 f   alm_bncs_output.obj
 0001:0001a47d       __unwindfunclet$?writeInstances@alm_bncs_output@@AAE_NXZ$4 1001b47d f   alm_bncs_output.obj
 0001:0001a486       __unwindfunclet$?writeInstances@alm_bncs_output@@AAE_NXZ$5 1001b486 f   alm_bncs_output.obj
 0001:0001a48f       __unwindfunclet$?writeInstances@alm_bncs_output@@AAE_NXZ$6 1001b48f f   alm_bncs_output.obj
 0001:0001a498       __unwindfunclet$?writeInstances@alm_bncs_output@@AAE_NXZ$7 1001b498 f   alm_bncs_output.obj
 0001:0001a4a1       __unwindfunclet$?writeInstances@alm_bncs_output@@AAE_NXZ$8 1001b4a1 f   alm_bncs_output.obj
 0001:0001a4aa       __unwindfunclet$?writeInstances@alm_bncs_output@@AAE_NXZ$9 1001b4aa f   alm_bncs_output.obj
 0001:0001a4b3       __unwindfunclet$?writeInstances@alm_bncs_output@@AAE_NXZ$10 1001b4b3 f   alm_bncs_output.obj
 0001:0001a4bf       __unwindfunclet$?writeInstances@alm_bncs_output@@AAE_NXZ$11 1001b4bf f   alm_bncs_output.obj
 0001:0001a4c8       __unwindfunclet$?writeInstances@alm_bncs_output@@AAE_NXZ$12 1001b4c8 f   alm_bncs_output.obj
 0001:0001a4d0       __unwindfunclet$?writeInstances@alm_bncs_output@@AAE_NXZ$13 1001b4d0 f   alm_bncs_output.obj
 0001:0001a4d9       __unwindfunclet$?writeInstances@alm_bncs_output@@AAE_NXZ$14 1001b4d9 f   alm_bncs_output.obj
 0001:0001a4e2       __unwindfunclet$?writeInstances@alm_bncs_output@@AAE_NXZ$15 1001b4e2 f   alm_bncs_output.obj
 0001:0001a4eb       __unwindfunclet$?writeInstances@alm_bncs_output@@AAE_NXZ$16 1001b4eb f   alm_bncs_output.obj
 0001:0001a4f4       __unwindfunclet$?writeInstances@alm_bncs_output@@AAE_NXZ$17 1001b4f4 f   alm_bncs_output.obj
 0001:0001a4fd       __unwindfunclet$?writeInstances@alm_bncs_output@@AAE_NXZ$18 1001b4fd f   alm_bncs_output.obj
 0001:0001a509       __unwindfunclet$?writeInstances@alm_bncs_output@@AAE_NXZ$19 1001b509 f   alm_bncs_output.obj
 0001:0001a512       __unwindfunclet$?writeInstances@alm_bncs_output@@AAE_NXZ$20 1001b512 f   alm_bncs_output.obj
 0001:0001a51b       __unwindfunclet$?writeInstances@alm_bncs_output@@AAE_NXZ$21 1001b51b f   alm_bncs_output.obj
 0001:0001a527       __unwindfunclet$?writeInstances@alm_bncs_output@@AAE_NXZ$22 1001b527 f   alm_bncs_output.obj
 0001:0001a533       __unwindfunclet$?writeInstances@alm_bncs_output@@AAE_NXZ$23 1001b533 f   alm_bncs_output.obj
 0001:0001a53c       __unwindfunclet$?writeInstances@alm_bncs_output@@AAE_NXZ$24 1001b53c f   alm_bncs_output.obj
 0001:0001a545       __unwindfunclet$?writeInstances@alm_bncs_output@@AAE_NXZ$25 1001b545 f   alm_bncs_output.obj
 0001:0001a551       __unwindfunclet$?writeInstances@alm_bncs_output@@AAE_NXZ$26 1001b551 f   alm_bncs_output.obj
 0001:0001a55d       __unwindfunclet$?writeInstances@alm_bncs_output@@AAE_NXZ$27 1001b55d f   alm_bncs_output.obj
 0001:0001a569       __unwindfunclet$?writeInstances@alm_bncs_output@@AAE_NXZ$28 1001b569 f   alm_bncs_output.obj
 0001:0001a575       __unwindfunclet$?writeInstances@alm_bncs_output@@AAE_NXZ$29 1001b575 f   alm_bncs_output.obj
 0001:0001a581       __unwindfunclet$?writeInstances@alm_bncs_output@@AAE_NXZ$30 1001b581 f   alm_bncs_output.obj
 0001:0001a58a       __unwindfunclet$?writeInstances@alm_bncs_output@@AAE_NXZ$31 1001b58a f   alm_bncs_output.obj
 0001:0001a596       __unwindfunclet$?writeInstances@alm_bncs_output@@AAE_NXZ$32 1001b596 f   alm_bncs_output.obj
 0001:0001a59f       __unwindfunclet$?writeInstances@alm_bncs_output@@AAE_NXZ$33 1001b59f f   alm_bncs_output.obj
 0001:0001a5ab       __unwindfunclet$?writeInstances@alm_bncs_output@@AAE_NXZ$34 1001b5ab f   alm_bncs_output.obj
 0001:0001a5b4       __unwindfunclet$?writeInstances@alm_bncs_output@@AAE_NXZ$35 1001b5b4 f   alm_bncs_output.obj
 0001:0001a5c0       __unwindfunclet$?writeInstances@alm_bncs_output@@AAE_NXZ$36 1001b5c0 f   alm_bncs_output.obj
 0001:0001a5cc       __unwindfunclet$?writeInstances@alm_bncs_output@@AAE_NXZ$37 1001b5cc f   alm_bncs_output.obj
 0001:0001a5d8       __unwindfunclet$?writeInstances@alm_bncs_output@@AAE_NXZ$38 1001b5d8 f   alm_bncs_output.obj
 0001:0001a5e1       __unwindfunclet$?writeInstances@alm_bncs_output@@AAE_NXZ$39 1001b5e1 f   alm_bncs_output.obj
 0001:0001a5ea       __unwindfunclet$?writeInstances@alm_bncs_output@@AAE_NXZ$40 1001b5ea f   alm_bncs_output.obj
 0001:0001a5f6       __unwindfunclet$?writeInstances@alm_bncs_output@@AAE_NXZ$41 1001b5f6 f   alm_bncs_output.obj
 0001:0001a602       __unwindfunclet$?writeInstances@alm_bncs_output@@AAE_NXZ$42 1001b602 f   alm_bncs_output.obj
 0001:0001a60b       __unwindfunclet$?writeInstances@alm_bncs_output@@AAE_NXZ$43 1001b60b f   alm_bncs_output.obj
 0001:0001a614       __unwindfunclet$?writeInstances@alm_bncs_output@@AAE_NXZ$44 1001b614 f   alm_bncs_output.obj
 0001:0001a620       __unwindfunclet$?writeInstances@alm_bncs_output@@AAE_NXZ$45 1001b620 f   alm_bncs_output.obj
 0001:0001a629       __unwindfunclet$?writeInstances@alm_bncs_output@@AAE_NXZ$46 1001b629 f   alm_bncs_output.obj
 0001:0001a632       __unwindfunclet$?writeInstances@alm_bncs_output@@AAE_NXZ$47 1001b632 f   alm_bncs_output.obj
 0001:0001a63b       __unwindfunclet$?writeInstances@alm_bncs_output@@AAE_NXZ$48 1001b63b f   alm_bncs_output.obj
 0001:0001a644       __unwindfunclet$?writeInstances@alm_bncs_output@@AAE_NXZ$49 1001b644 f   alm_bncs_output.obj
 0001:0001a64d       __unwindfunclet$?writeInstances@alm_bncs_output@@AAE_NXZ$50 1001b64d f   alm_bncs_output.obj
 0001:0001a656       __unwindfunclet$?writeInstances@alm_bncs_output@@AAE_NXZ$51 1001b656 f   alm_bncs_output.obj
 0001:0001a65f       __unwindfunclet$?writeInstances@alm_bncs_output@@AAE_NXZ$52 1001b65f f   alm_bncs_output.obj
 0001:0001a668       __unwindfunclet$?writeInstances@alm_bncs_output@@AAE_NXZ$53 1001b668 f   alm_bncs_output.obj
 0001:0001a671       __unwindfunclet$?writeInstances@alm_bncs_output@@AAE_NXZ$54 1001b671 f   alm_bncs_output.obj
 0001:0001a67a       __unwindfunclet$?writeInstances@alm_bncs_output@@AAE_NXZ$55 1001b67a f   alm_bncs_output.obj
 0001:0001a683       __unwindfunclet$?writeInstances@alm_bncs_output@@AAE_NXZ$56 1001b683 f   alm_bncs_output.obj
 0001:0001a68c       __unwindfunclet$?writeInstances@alm_bncs_output@@AAE_NXZ$57 1001b68c f   alm_bncs_output.obj
 0001:0001a695       __unwindfunclet$?writeInstances@alm_bncs_output@@AAE_NXZ$58 1001b695 f   alm_bncs_output.obj
 0001:0001a69e       __unwindfunclet$?writeInstances@alm_bncs_output@@AAE_NXZ$59 1001b69e f   alm_bncs_output.obj
 0001:0001a6a7       __unwindfunclet$?writeInstances@alm_bncs_output@@AAE_NXZ$60 1001b6a7 f   alm_bncs_output.obj
 0001:0001a6b0       __unwindfunclet$?writeInstances@alm_bncs_output@@AAE_NXZ$61 1001b6b0 f   alm_bncs_output.obj
 0001:0001a6b9       __ehhandler$?writeInstances@alm_bncs_output@@AAE_NXZ 1001b6b9 f   alm_bncs_output.obj
 0001:0001a6d7       __unwindfunclet$?writeNewInstanceFile@alm_bncs_output@@AAEXXZ$0 1001b6d7 f   alm_bncs_output.obj
 0001:0001a6e0       __unwindfunclet$?writeNewInstanceFile@alm_bncs_output@@AAEXXZ$1 1001b6e0 f   alm_bncs_output.obj
 0001:0001a6e9       __unwindfunclet$?writeNewInstanceFile@alm_bncs_output@@AAEXXZ$2 1001b6e9 f   alm_bncs_output.obj
 0001:0001a6f2       __unwindfunclet$?writeNewInstanceFile@alm_bncs_output@@AAEXXZ$3 1001b6f2 f   alm_bncs_output.obj
 0001:0001a6fb       __unwindfunclet$?writeNewInstanceFile@alm_bncs_output@@AAEXXZ$4 1001b6fb f   alm_bncs_output.obj
 0001:0001a704       __unwindfunclet$?writeNewInstanceFile@alm_bncs_output@@AAEXXZ$5 1001b704 f   alm_bncs_output.obj
 0001:0001a70d       __unwindfunclet$?writeNewInstanceFile@alm_bncs_output@@AAEXXZ$6 1001b70d f   alm_bncs_output.obj
 0001:0001a716       __unwindfunclet$?writeNewInstanceFile@alm_bncs_output@@AAEXXZ$7 1001b716 f   alm_bncs_output.obj
 0001:0001a71f       __unwindfunclet$?writeNewInstanceFile@alm_bncs_output@@AAEXXZ$8 1001b71f f   alm_bncs_output.obj
 0001:0001a72b       __unwindfunclet$?writeNewInstanceFile@alm_bncs_output@@AAEXXZ$10 1001b72b f   alm_bncs_output.obj
 0001:0001a734       __unwindfunclet$?writeNewInstanceFile@alm_bncs_output@@AAEXXZ$11 1001b734 f   alm_bncs_output.obj
 0001:0001a73d       __unwindfunclet$?writeNewInstanceFile@alm_bncs_output@@AAEXXZ$12 1001b73d f   alm_bncs_output.obj
 0001:0001a746       __unwindfunclet$?writeNewInstanceFile@alm_bncs_output@@AAEXXZ$13 1001b746 f   alm_bncs_output.obj
 0001:0001a74f       __unwindfunclet$?writeNewInstanceFile@alm_bncs_output@@AAEXXZ$14 1001b74f f   alm_bncs_output.obj
 0001:0001a758       __unwindfunclet$?writeNewInstanceFile@alm_bncs_output@@AAEXXZ$15 1001b758 f   alm_bncs_output.obj
 0001:0001a761       __unwindfunclet$?writeNewInstanceFile@alm_bncs_output@@AAEXXZ$16 1001b761 f   alm_bncs_output.obj
 0001:0001a76a       __unwindfunclet$?writeNewInstanceFile@alm_bncs_output@@AAEXXZ$17 1001b76a f   alm_bncs_output.obj
 0001:0001a773       __unwindfunclet$?writeNewInstanceFile@alm_bncs_output@@AAEXXZ$18 1001b773 f   alm_bncs_output.obj
 0001:0001a77e       __unwindfunclet$?writeNewInstanceFile@alm_bncs_output@@AAEXXZ$19 1001b77e f   alm_bncs_output.obj
 0001:0001a787       __unwindfunclet$?writeNewInstanceFile@alm_bncs_output@@AAEXXZ$20 1001b787 f   alm_bncs_output.obj
 0001:0001a790       __unwindfunclet$?writeNewInstanceFile@alm_bncs_output@@AAEXXZ$21 1001b790 f   alm_bncs_output.obj
 0001:0001a799       __unwindfunclet$?writeNewInstanceFile@alm_bncs_output@@AAEXXZ$22 1001b799 f   alm_bncs_output.obj
 0001:0001a7a2       __unwindfunclet$?writeNewInstanceFile@alm_bncs_output@@AAEXXZ$23 1001b7a2 f   alm_bncs_output.obj
 0001:0001a7ad       __unwindfunclet$?writeNewInstanceFile@alm_bncs_output@@AAEXXZ$24 1001b7ad f   alm_bncs_output.obj
 0001:0001a7b9       __unwindfunclet$?writeNewInstanceFile@alm_bncs_output@@AAEXXZ$25 1001b7b9 f   alm_bncs_output.obj
 0001:0001a7c2       __unwindfunclet$?writeNewInstanceFile@alm_bncs_output@@AAEXXZ$26 1001b7c2 f   alm_bncs_output.obj
 0001:0001a7cb       __unwindfunclet$?writeNewInstanceFile@alm_bncs_output@@AAEXXZ$27 1001b7cb f   alm_bncs_output.obj
 0001:0001a7d4       __unwindfunclet$?writeNewInstanceFile@alm_bncs_output@@AAEXXZ$28 1001b7d4 f   alm_bncs_output.obj
 0001:0001a7dd       __unwindfunclet$?writeNewInstanceFile@alm_bncs_output@@AAEXXZ$29 1001b7dd f   alm_bncs_output.obj
 0001:0001a7e6       __unwindfunclet$?writeNewInstanceFile@alm_bncs_output@@AAEXXZ$30 1001b7e6 f   alm_bncs_output.obj
 0001:0001a7ef       __unwindfunclet$?writeNewInstanceFile@alm_bncs_output@@AAEXXZ$31 1001b7ef f   alm_bncs_output.obj
 0001:0001a7f8       __unwindfunclet$?writeNewInstanceFile@alm_bncs_output@@AAEXXZ$33 1001b7f8 f   alm_bncs_output.obj
 0001:0001a801       __unwindfunclet$?writeNewInstanceFile@alm_bncs_output@@AAEXXZ$34 1001b801 f   alm_bncs_output.obj
 0001:0001a80a       __unwindfunclet$?writeNewInstanceFile@alm_bncs_output@@AAEXXZ$35 1001b80a f   alm_bncs_output.obj
 0001:0001a813       __unwindfunclet$?writeNewInstanceFile@alm_bncs_output@@AAEXXZ$36 1001b813 f   alm_bncs_output.obj
 0001:0001a81c       __unwindfunclet$?writeNewInstanceFile@alm_bncs_output@@AAEXXZ$37 1001b81c f   alm_bncs_output.obj
 0001:0001a828       __unwindfunclet$?writeNewInstanceFile@alm_bncs_output@@AAEXXZ$38 1001b828 f   alm_bncs_output.obj
 0001:0001a834       __unwindfunclet$?writeNewInstanceFile@alm_bncs_output@@AAEXXZ$39 1001b834 f   alm_bncs_output.obj
 0001:0001a83d       __unwindfunclet$?writeNewInstanceFile@alm_bncs_output@@AAEXXZ$40 1001b83d f   alm_bncs_output.obj
 0001:0001a846       __unwindfunclet$?writeNewInstanceFile@alm_bncs_output@@AAEXXZ$41 1001b846 f   alm_bncs_output.obj
 0001:0001a84f       __unwindfunclet$?writeNewInstanceFile@alm_bncs_output@@AAEXXZ$42 1001b84f f   alm_bncs_output.obj
 0001:0001a858       __ehhandler$?writeNewInstanceFile@alm_bncs_output@@AAEXXZ 1001b858 f   alm_bncs_output.obj
 0001:0001a876       __unwindfunclet$??0cOutputFile@@QAE@ABVQString@@00@Z$0 1001b876 f   cOutputFile.obj
 0001:0001a876       __unwindfunclet$??0cOutputFile@@QAE@XZ$0 1001b876 f   cOutputFile.obj
 0001:0001a876       __unwindfunclet$??1cOutputFile@@UAE@XZ$0 1001b876 f   cOutputFile.obj
 0001:0001a882       __unwindfunclet$??0cOutputFile@@QAE@ABVQString@@00@Z$1 1001b882 f   cOutputFile.obj
 0001:0001a882       __unwindfunclet$??1cOutputFile@@UAE@XZ$1 1001b882 f   cOutputFile.obj
 0001:0001a882       __unwindfunclet$??0cOutputFile@@QAE@XZ$1 1001b882 f   cOutputFile.obj
 0001:0001a88e       __ehhandler$??0cOutputFile@@QAE@ABVQString@@00@Z 1001b88e f   cOutputFile.obj
 0001:0001a88e       __ehhandler$??0cOutputFile@@QAE@XZ 1001b88e f   cOutputFile.obj
 0001:0001a88e       __ehhandler$??1cOutputFile@@UAE@XZ 1001b88e f   cOutputFile.obj
 0001:0001a8a9       __unwindfunclet$??0devTemplate@@QAE@ABVQString@@@Z$0 1001b8a9 f   devTemplate.obj
 0001:0001a8b5       __unwindfunclet$??0devTemplate@@QAE@ABVQString@@@Z$1 1001b8b5 f   devTemplate.obj
 0001:0001a8c1       __unwindfunclet$??0devTemplate@@QAE@ABVQString@@@Z$2 1001b8c1 f   devTemplate.obj
 0001:0001a8cd       __unwindfunclet$??0devTemplate@@QAE@ABVQString@@@Z$3 1001b8cd f   devTemplate.obj
 0001:0001a8d9       __unwindfunclet$??0devTemplate@@QAE@ABVQString@@@Z$4 1001b8d9 f   devTemplate.obj
 0001:0001a8e2       __unwindfunclet$??0devTemplate@@QAE@ABVQString@@@Z$5 1001b8e2 f   devTemplate.obj
 0001:0001a8eb       __unwindfunclet$??0devTemplate@@QAE@ABVQString@@@Z$6 1001b8eb f   devTemplate.obj
 0001:0001a8f4       __unwindfunclet$??0devTemplate@@QAE@ABVQString@@@Z$7 1001b8f4 f   devTemplate.obj
 0001:0001a90e       __unwindfunclet$??0devTemplate@@QAE@ABVQString@@@Z$8 1001b90e f   devTemplate.obj
 0001:0001a928       __unwindfunclet$??0devTemplate@@QAE@ABVQString@@@Z$9 1001b928 f   devTemplate.obj
 0001:0001a931       __unwindfunclet$??0devTemplate@@QAE@ABVQString@@@Z$10 1001b931 f   devTemplate.obj
 0001:0001a93a       __unwindfunclet$??0devTemplate@@QAE@ABVQString@@@Z$11 1001b93a f   devTemplate.obj
 0001:0001a943       __ehhandler$??0devTemplate@@QAE@ABVQString@@@Z 1001b943 f   devTemplate.obj
 0001:0001a95e       __unwindfunclet$??1?$QDict@VdevTemplate@@@@UAE@XZ$0 1001b95e f   devTemplate.obj
 0001:0001a967       __ehhandler$??1?$QDict@VdevTemplate@@@@UAE@XZ 1001b967 f   devTemplate.obj
 0001:0001a982       __unwindfunclet$??1devTemplate@@UAE@XZ$0 1001b982 f   devTemplate.obj
 0001:0001a98e       __unwindfunclet$??1devTemplate@@UAE@XZ$1 1001b98e f   devTemplate.obj
 0001:0001a99a       __unwindfunclet$??1devTemplate@@UAE@XZ$2 1001b99a f   devTemplate.obj
 0001:0001a9a6       __ehhandler$??1devTemplate@@UAE@XZ 1001b9a6 f   devTemplate.obj
 0001:0001a9c1       __unwindfunclet$?loadDevDesc@devTemplate@@QAE_NABVQString@@0@Z$0 1001b9c1 f   devTemplate.obj
 0001:0001a9ca       __unwindfunclet$?loadDevDesc@devTemplate@@QAE_NABVQString@@0@Z$1 1001b9ca f   devTemplate.obj
 0001:0001a9d3       __unwindfunclet$?loadDevDesc@devTemplate@@QAE_NABVQString@@0@Z$2 1001b9d3 f   devTemplate.obj
 0001:0001a9dc       __unwindfunclet$?loadDevDesc@devTemplate@@QAE_NABVQString@@0@Z$3 1001b9dc f   devTemplate.obj
 0001:0001a9e5       __unwindfunclet$?loadDevDesc@devTemplate@@QAE_NABVQString@@0@Z$4 1001b9e5 f   devTemplate.obj
 0001:0001a9ee       __unwindfunclet$?loadDevDesc@devTemplate@@QAE_NABVQString@@0@Z$5 1001b9ee f   devTemplate.obj
 0001:0001a9f7       __unwindfunclet$?loadDevDesc@devTemplate@@QAE_NABVQString@@0@Z$6 1001b9f7 f   devTemplate.obj
 0001:0001aa00       __unwindfunclet$?loadDevDesc@devTemplate@@QAE_NABVQString@@0@Z$7 1001ba00 f   devTemplate.obj
 0001:0001aa09       __unwindfunclet$?loadDevDesc@devTemplate@@QAE_NABVQString@@0@Z$8 1001ba09 f   devTemplate.obj
 0001:0001aa12       __unwindfunclet$?loadDevDesc@devTemplate@@QAE_NABVQString@@0@Z$9 1001ba12 f   devTemplate.obj
 0001:0001aa1b       __unwindfunclet$?loadDevDesc@devTemplate@@QAE_NABVQString@@0@Z$10 1001ba1b f   devTemplate.obj
 0001:0001aa24       __unwindfunclet$?loadDevDesc@devTemplate@@QAE_NABVQString@@0@Z$11 1001ba24 f   devTemplate.obj
 0001:0001aa2d       __unwindfunclet$?loadDevDesc@devTemplate@@QAE_NABVQString@@0@Z$12 1001ba2d f   devTemplate.obj
 0001:0001aa36       __unwindfunclet$?loadDevDesc@devTemplate@@QAE_NABVQString@@0@Z$13 1001ba36 f   devTemplate.obj
 0001:0001aa3f       __unwindfunclet$?loadDevDesc@devTemplate@@QAE_NABVQString@@0@Z$14 1001ba3f f   devTemplate.obj
 0001:0001aa48       __unwindfunclet$?loadDevDesc@devTemplate@@QAE_NABVQString@@0@Z$15 1001ba48 f   devTemplate.obj
 0001:0001aa51       __unwindfunclet$?loadDevDesc@devTemplate@@QAE_NABVQString@@0@Z$16 1001ba51 f   devTemplate.obj
 0001:0001aa5a       __unwindfunclet$?loadDevDesc@devTemplate@@QAE_NABVQString@@0@Z$17 1001ba5a f   devTemplate.obj
 0001:0001aa63       __ehhandler$?loadDevDesc@devTemplate@@QAE_NABVQString@@0@Z 1001ba63 f   devTemplate.obj
 0001:0001aa7e       __unwindfunclet$?saveFile@devTemplate@@QBE_NABVQString@@0QBVIDomDoc@@QAVIGetDocuments@@@Z$0 1001ba7e f   devTemplate.obj
 0001:0001aa87       __unwindfunclet$?saveFile@devTemplate@@QBE_NABVQString@@0QBVIDomDoc@@QAVIGetDocuments@@@Z$1 1001ba87 f   devTemplate.obj
 0001:0001aa90       __unwindfunclet$?saveFile@devTemplate@@QBE_NABVQString@@0QBVIDomDoc@@QAVIGetDocuments@@@Z$2 1001ba90 f   devTemplate.obj
 0001:0001aa99       __unwindfunclet$?saveFile@devTemplate@@QBE_NABVQString@@0QBVIDomDoc@@QAVIGetDocuments@@@Z$3 1001ba99 f   devTemplate.obj
 0001:0001aaa2       __unwindfunclet$?saveFile@devTemplate@@QBE_NABVQString@@0QBVIDomDoc@@QAVIGetDocuments@@@Z$4 1001baa2 f   devTemplate.obj
 0001:0001aaae       __unwindfunclet$?saveFile@devTemplate@@QBE_NABVQString@@0QBVIDomDoc@@QAVIGetDocuments@@@Z$5 1001baae f   devTemplate.obj
 0001:0001aab7       __unwindfunclet$?saveFile@devTemplate@@QBE_NABVQString@@0QBVIDomDoc@@QAVIGetDocuments@@@Z$6 1001bab7 f   devTemplate.obj
 0001:0001aac0       __unwindfunclet$?saveFile@devTemplate@@QBE_NABVQString@@0QBVIDomDoc@@QAVIGetDocuments@@@Z$7 1001bac0 f   devTemplate.obj
 0001:0001aac9       __unwindfunclet$?saveFile@devTemplate@@QBE_NABVQString@@0QBVIDomDoc@@QAVIGetDocuments@@@Z$8 1001bac9 f   devTemplate.obj
 0001:0001aad2       __unwindfunclet$?saveFile@devTemplate@@QBE_NABVQString@@0QBVIDomDoc@@QAVIGetDocuments@@@Z$9 1001bad2 f   devTemplate.obj
 0001:0001aadb       __unwindfunclet$?saveFile@devTemplate@@QBE_NABVQString@@0QBVIDomDoc@@QAVIGetDocuments@@@Z$10 1001badb f   devTemplate.obj
 0001:0001aae4       __unwindfunclet$?saveFile@devTemplate@@QBE_NABVQString@@0QBVIDomDoc@@QAVIGetDocuments@@@Z$11 1001bae4 f   devTemplate.obj
 0001:0001aaed       __unwindfunclet$?saveFile@devTemplate@@QBE_NABVQString@@0QBVIDomDoc@@QAVIGetDocuments@@@Z$12 1001baed f   devTemplate.obj
 0001:0001aaf6       __unwindfunclet$?saveFile@devTemplate@@QBE_NABVQString@@0QBVIDomDoc@@QAVIGetDocuments@@@Z$13 1001baf6 f   devTemplate.obj
 0001:0001aaff       __unwindfunclet$?saveFile@devTemplate@@QBE_NABVQString@@0QBVIDomDoc@@QAVIGetDocuments@@@Z$14 1001baff f   devTemplate.obj
 0001:0001ab08       __unwindfunclet$?saveFile@devTemplate@@QBE_NABVQString@@0QBVIDomDoc@@QAVIGetDocuments@@@Z$15 1001bb08 f   devTemplate.obj
 0001:0001ab11       __unwindfunclet$?saveFile@devTemplate@@QBE_NABVQString@@0QBVIDomDoc@@QAVIGetDocuments@@@Z$16 1001bb11 f   devTemplate.obj
 0001:0001ab1a       __unwindfunclet$?saveFile@devTemplate@@QBE_NABVQString@@0QBVIDomDoc@@QAVIGetDocuments@@@Z$17 1001bb1a f   devTemplate.obj
 0001:0001ab23       __unwindfunclet$?saveFile@devTemplate@@QBE_NABVQString@@0QBVIDomDoc@@QAVIGetDocuments@@@Z$18 1001bb23 f   devTemplate.obj
 0001:0001ab2c       __unwindfunclet$?saveFile@devTemplate@@QBE_NABVQString@@0QBVIDomDoc@@QAVIGetDocuments@@@Z$19 1001bb2c f   devTemplate.obj
 0001:0001ab35       __ehhandler$?saveFile@devTemplate@@QBE_NABVQString@@0QBVIDomDoc@@QAVIGetDocuments@@@Z 1001bb35 f   devTemplate.obj
 0001:0001ab53       __unwindfunclet$??0dialog@@QAE@PAVIGetDocuments@@PAVQWidget@@PBDI@Z$0 1001bb53 f   dialogimpl.obj
 0001:0001ab5b       __unwindfunclet$??0dialog@@QAE@PAVIGetDocuments@@PAVQWidget@@PBDI@Z$1 1001bb5b f   dialogimpl.obj
 0001:0001ab6a       __unwindfunclet$??0dialog@@QAE@PAVIGetDocuments@@PAVQWidget@@PBDI@Z$2 1001bb6a f   dialogimpl.obj
 0001:0001ab73       __unwindfunclet$??0dialog@@QAE@PAVIGetDocuments@@PAVQWidget@@PBDI@Z$3 1001bb73 f   dialogimpl.obj
 0001:0001ab7c       __unwindfunclet$??0dialog@@QAE@PAVIGetDocuments@@PAVQWidget@@PBDI@Z$4 1001bb7c f   dialogimpl.obj
 0001:0001ab85       __unwindfunclet$??0dialog@@QAE@PAVIGetDocuments@@PAVQWidget@@PBDI@Z$5 1001bb85 f   dialogimpl.obj
 0001:0001ab8e       __unwindfunclet$??0dialog@@QAE@PAVIGetDocuments@@PAVQWidget@@PBDI@Z$6 1001bb8e f   dialogimpl.obj
 0001:0001ab97       __unwindfunclet$??0dialog@@QAE@PAVIGetDocuments@@PAVQWidget@@PBDI@Z$7 1001bb97 f   dialogimpl.obj
 0001:0001aba0       __unwindfunclet$??0dialog@@QAE@PAVIGetDocuments@@PAVQWidget@@PBDI@Z$8 1001bba0 f   dialogimpl.obj
 0001:0001aba9       __unwindfunclet$??0dialog@@QAE@PAVIGetDocuments@@PAVQWidget@@PBDI@Z$9 1001bba9 f   dialogimpl.obj
 0001:0001abb3       __unwindfunclet$??0dialog@@QAE@PAVIGetDocuments@@PAVQWidget@@PBDI@Z$10 1001bbb3 f   dialogimpl.obj
 0001:0001abcd       __unwindfunclet$??0dialog@@QAE@PAVIGetDocuments@@PAVQWidget@@PBDI@Z$11 1001bbcd f   dialogimpl.obj
 0001:0001abe7       __unwindfunclet$??0dialog@@QAE@PAVIGetDocuments@@PAVQWidget@@PBDI@Z$12 1001bbe7 f   dialogimpl.obj
 0001:0001ac01       __unwindfunclet$??0dialog@@QAE@PAVIGetDocuments@@PAVQWidget@@PBDI@Z$13 1001bc01 f   dialogimpl.obj
 0001:0001ac1b       __unwindfunclet$??0dialog@@QAE@PAVIGetDocuments@@PAVQWidget@@PBDI@Z$15 1001bc1b f   dialogimpl.obj
 0001:0001ac25       __unwindfunclet$??0dialog@@QAE@PAVIGetDocuments@@PAVQWidget@@PBDI@Z$16 1001bc25 f   dialogimpl.obj
 0001:0001ac3f       __unwindfunclet$??0dialog@@QAE@PAVIGetDocuments@@PAVQWidget@@PBDI@Z$17 1001bc3f f   dialogimpl.obj
 0001:0001ac59       __unwindfunclet$??0dialog@@QAE@PAVIGetDocuments@@PAVQWidget@@PBDI@Z$18 1001bc59 f   dialogimpl.obj
 0001:0001ac73       __unwindfunclet$??0dialog@@QAE@PAVIGetDocuments@@PAVQWidget@@PBDI@Z$19 1001bc73 f   dialogimpl.obj
 0001:0001ac92       __ehhandler$??0dialog@@QAE@PAVIGetDocuments@@PAVQWidget@@PBDI@Z 1001bc92 f   dialogimpl.obj
 0001:0001acad       __unwindfunclet$??1dialog@@UAE@XZ$0 1001bcad f   dialogimpl.obj
 0001:0001acb5       __unwindfunclet$??1dialog@@UAE@XZ$1 1001bcb5 f   dialogimpl.obj
 0001:0001acc4       __unwindfunclet$??1dialog@@UAE@XZ$2 1001bcc4 f   dialogimpl.obj
 0001:0001accd       __unwindfunclet$??1dialog@@UAE@XZ$3 1001bccd f   dialogimpl.obj
 0001:0001acd6       __ehhandler$??1dialog@@UAE@XZ 1001bcd6 f   dialogimpl.obj
 0001:0001acf1       __unwindfunclet$?autoNumber@dialog@@QAEXXZ$0 1001bcf1 f   dialogimpl.obj
 0001:0001acfa       __unwindfunclet$?autoNumber@dialog@@QAEXXZ$1 1001bcfa f   dialogimpl.obj
 0001:0001ad04       __unwindfunclet$?autoNumber@dialog@@QAEXXZ$2 1001bd04 f   dialogimpl.obj
 0001:0001ad0d       __unwindfunclet$?autoNumber@dialog@@QAEXXZ$3 1001bd0d f   dialogimpl.obj
 0001:0001ad16       __unwindfunclet$?autoNumber@dialog@@QAEXXZ$4 1001bd16 f   dialogimpl.obj
 0001:0001ad1f       __unwindfunclet$?autoNumber@dialog@@QAEXXZ$5 1001bd1f f   dialogimpl.obj
 0001:0001ad28       __unwindfunclet$?autoNumber@dialog@@QAEXXZ$6 1001bd28 f   dialogimpl.obj
 0001:0001ad31       __unwindfunclet$?autoNumber@dialog@@QAEXXZ$7 1001bd31 f   dialogimpl.obj
 0001:0001ad3a       __unwindfunclet$?autoNumber@dialog@@QAEXXZ$10 1001bd3a f   dialogimpl.obj
 0001:0001ad43       __unwindfunclet$?autoNumber@dialog@@QAEXXZ$9 1001bd43 f   dialogimpl.obj
 0001:0001ad4c       __unwindfunclet$?autoNumber@dialog@@QAEXXZ$8 1001bd4c f   dialogimpl.obj
 0001:0001ad55       __unwindfunclet$?autoNumber@dialog@@QAEXXZ$11 1001bd55 f   dialogimpl.obj
 0001:0001ad5e       __ehhandler$?autoNumber@dialog@@QAEXXZ 1001bd5e f   dialogimpl.obj
 0001:0001ad79       __unwindfunclet$?changeSelection@dialog@@QAEXXZ$0 1001bd79 f   dialogimpl.obj
 0001:0001ad82       __unwindfunclet$?changeSelection@dialog@@QAEXXZ$1 1001bd82 f   dialogimpl.obj
 0001:0001ad8b       __ehhandler$?changeSelection@dialog@@QAEXXZ 1001bd8b f   dialogimpl.obj
 0001:0001ada6       __unwindfunclet$?checkForDuplicates@dialog@@QAE_NXZ$0 1001bda6 f   dialogimpl.obj
 0001:0001adae       __unwindfunclet$?checkForDuplicates@dialog@@QAE_NXZ$2 1001bdae f   dialogimpl.obj
 0001:0001adb7       __unwindfunclet$?checkForDuplicates@dialog@@QAE_NXZ$4 1001bdb7 f   dialogimpl.obj
 0001:0001adc0       __unwindfunclet$?checkForDuplicates@dialog@@QAE_NXZ$5 1001bdc0 f   dialogimpl.obj
 0001:0001adc9       __unwindfunclet$?checkForDuplicates@dialog@@QAE_NXZ$6 1001bdc9 f   dialogimpl.obj
 0001:0001add2       __unwindfunclet$?checkForDuplicates@dialog@@QAE_NXZ$7 1001bdd2 f   dialogimpl.obj
 0001:0001addb       __ehhandler$?checkForDuplicates@dialog@@QAE_NXZ 1001bddb f   dialogimpl.obj
 0001:0001adf6       __unwindfunclet$?clearSelectedSlots@dialog@@QAEXXZ$0 1001bdf6 f   dialogimpl.obj
 0001:0001adf6       __unwindfunclet$?clearSelectableSlots@dialog@@QAEXXZ$0 1001bdf6 f   dialogimpl.obj
 0001:0001adf6       __unwindfunclet$?clearAllSlots@dialog@@QAEXXZ$0 1001bdf6 f   dialogimpl.obj
 0001:0001adff       __unwindfunclet$?clearSelectedSlots@dialog@@QAEXXZ$1 1001bdff f   dialogimpl.obj
 0001:0001adff       __unwindfunclet$?clearSelectableSlots@dialog@@QAEXXZ$1 1001bdff f   dialogimpl.obj
 0001:0001adff       __unwindfunclet$?clearAllSlots@dialog@@QAEXXZ$1 1001bdff f   dialogimpl.obj
 0001:0001ae08       __unwindfunclet$?clearSelectableSlots@dialog@@QAEXXZ$2 1001be08 f   dialogimpl.obj
 0001:0001ae08       __unwindfunclet$?clearSelectedSlots@dialog@@QAEXXZ$2 1001be08 f   dialogimpl.obj
 0001:0001ae08       __unwindfunclet$?clearAllSlots@dialog@@QAEXXZ$2 1001be08 f   dialogimpl.obj
 0001:0001ae11       __unwindfunclet$?clearAllSlots@dialog@@QAEXXZ$3 1001be11 f   dialogimpl.obj
 0001:0001ae11       __unwindfunclet$?clearSelectableSlots@dialog@@QAEXXZ$3 1001be11 f   dialogimpl.obj
 0001:0001ae11       __unwindfunclet$?clearSelectedSlots@dialog@@QAEXXZ$3 1001be11 f   dialogimpl.obj
 0001:0001ae1a       __ehhandler$?clearAllSlots@dialog@@QAEXXZ 1001be1a f   dialogimpl.obj
 0001:0001ae1a       __ehhandler$?clearSelectableSlots@dialog@@QAEXXZ 1001be1a f   dialogimpl.obj
 0001:0001ae1a       __ehhandler$?clearSelectedSlots@dialog@@QAEXXZ 1001be1a f   dialogimpl.obj
 0001:0001ae35       __unwindfunclet$?clearSlots@dialog@@QAEXXZ$1 1001be35 f   dialogimpl.obj
 0001:0001ae3e       __unwindfunclet$?clearSlots@dialog@@QAEXXZ$2 1001be3e f   dialogimpl.obj
 0001:0001ae47       __unwindfunclet$?clearSlots@dialog@@QAEXXZ$3 1001be47 f   dialogimpl.obj
 0001:0001ae50       __unwindfunclet$?clearSlots@dialog@@QAEXXZ$4 1001be50 f   dialogimpl.obj
 0001:0001ae59       __unwindfunclet$?clearSlots@dialog@@QAEXXZ$5 1001be59 f   dialogimpl.obj
 0001:0001ae62       __unwindfunclet$?clearSlots@dialog@@QAEXXZ$6 1001be62 f   dialogimpl.obj
 0001:0001ae6b       __unwindfunclet$?clearSlots@dialog@@QAEXXZ$7 1001be6b f   dialogimpl.obj
 0001:0001ae74       __unwindfunclet$?clearSlots@dialog@@QAEXXZ$8 1001be74 f   dialogimpl.obj
 0001:0001ae7d       __ehhandler$?clearSlots@dialog@@QAEXXZ 1001be7d f   dialogimpl.obj
 0001:0001ae98       __unwindfunclet$?clipboardDataChange@dialog@@QAEXXZ$0 1001be98 f   dialogimpl.obj
 0001:0001aea1       __unwindfunclet$?clipboardDataChange@dialog@@QAEXXZ$1 1001bea1 f   dialogimpl.obj
 0001:0001aeaa       __unwindfunclet$?clipboardDataChange@dialog@@QAEXXZ$2 1001beaa f   dialogimpl.obj
 0001:0001aeb3       __unwindfunclet$?clipboardDataChange@dialog@@QAEXXZ$3 1001beb3 f   dialogimpl.obj
 0001:0001aebc       __unwindfunclet$?clipboardDataChange@dialog@@QAEXXZ$4 1001bebc f   dialogimpl.obj
 0001:0001aec5       __unwindfunclet$?clipboardDataChange@dialog@@QAEXXZ$5 1001bec5 f   dialogimpl.obj
 0001:0001aece       __unwindfunclet$?clipboardDataChange@dialog@@QAEXXZ$6 1001bece f   dialogimpl.obj
 0001:0001aed7       __ehhandler$?clipboardDataChange@dialog@@QAEXXZ 1001bed7 f   dialogimpl.obj
 0001:0001aef2       __unwindfunclet$?copyData@dialog@@QAEXXZ$0 1001bef2 f   dialogimpl.obj
 0001:0001aefb       __unwindfunclet$?copyData@dialog@@QAEXXZ$1 1001befb f   dialogimpl.obj
 0001:0001af04       __unwindfunclet$?copyData@dialog@@QAEXXZ$2 1001bf04 f   dialogimpl.obj
 0001:0001af0d       __unwindfunclet$?copyData@dialog@@QAEXXZ$3 1001bf0d f   dialogimpl.obj
 0001:0001af16       __unwindfunclet$?copyData@dialog@@QAEXXZ$4 1001bf16 f   dialogimpl.obj
 0001:0001af1f       __unwindfunclet$?copyData@dialog@@QAEXXZ$5 1001bf1f f   dialogimpl.obj
 0001:0001af28       __ehhandler$?copyData@dialog@@QAEXXZ 1001bf28 f   dialogimpl.obj
 0001:0001af43       __unwindfunclet$?pasteData@dialog@@QAEXXZ$0 1001bf43 f   dialogimpl.obj
 0001:0001af4c       __unwindfunclet$?pasteData@dialog@@QAEXXZ$1 1001bf4c f   dialogimpl.obj
 0001:0001af55       __unwindfunclet$?pasteData@dialog@@QAEXXZ$2 1001bf55 f   dialogimpl.obj
 0001:0001af5e       __unwindfunclet$?pasteData@dialog@@QAEXXZ$3 1001bf5e f   dialogimpl.obj
 0001:0001af67       __unwindfunclet$?pasteData@dialog@@QAEXXZ$4 1001bf67 f   dialogimpl.obj
 0001:0001af70       __unwindfunclet$?pasteData@dialog@@QAEXXZ$5 1001bf70 f   dialogimpl.obj
 0001:0001af79       __unwindfunclet$?pasteData@dialog@@QAEXXZ$6 1001bf79 f   dialogimpl.obj
 0001:0001af82       __unwindfunclet$?pasteData@dialog@@QAEXXZ$7 1001bf82 f   dialogimpl.obj
 0001:0001af8b       __unwindfunclet$?pasteData@dialog@@QAEXXZ$8 1001bf8b f   dialogimpl.obj
 0001:0001af94       __unwindfunclet$?pasteData@dialog@@QAEXXZ$9 1001bf94 f   dialogimpl.obj
 0001:0001afae       __unwindfunclet$?pasteData@dialog@@QAEXXZ$10 1001bfae f   dialogimpl.obj
 0001:0001afb7       __unwindfunclet$?pasteData@dialog@@QAEXXZ$11 1001bfb7 f   dialogimpl.obj
 0001:0001afc0       __unwindfunclet$?pasteData@dialog@@QAEXXZ$12 1001bfc0 f   dialogimpl.obj
 0001:0001afc9       __unwindfunclet$?pasteData@dialog@@QAEXXZ$13 1001bfc9 f   dialogimpl.obj
 0001:0001afd2       __unwindfunclet$?pasteData@dialog@@QAEXXZ$14 1001bfd2 f   dialogimpl.obj
 0001:0001afdb       __unwindfunclet$?pasteData@dialog@@QAEXXZ$15 1001bfdb f   dialogimpl.obj
 0001:0001afe4       __unwindfunclet$?pasteData@dialog@@QAEXXZ$16 1001bfe4 f   dialogimpl.obj
 0001:0001afed       __unwindfunclet$?pasteData@dialog@@QAEXXZ$17 1001bfed f   dialogimpl.obj
 0001:0001aff6       __ehhandler$?pasteData@dialog@@QAEXXZ 1001bff6 f   dialogimpl.obj
 0001:0001b011       __unwindfunclet$?selectProc@dialog@@QAEXPAVQListViewItem@@@Z$0 1001c011 f   dialogimpl.obj
 0001:0001b01a       __ehhandler$?selectProc@dialog@@QAEXPAVQListViewItem@@@Z 1001c01a f   dialogimpl.obj
 0001:0001b035       __unwindfunclet$?slotChange@dialog@@QAEXPAVQListViewItem@@HABVQString@@@Z$0 1001c035 f   dialogimpl.obj
 0001:0001b03e       __unwindfunclet$?slotChange@dialog@@QAEXPAVQListViewItem@@HABVQString@@@Z$2 1001c03e f   dialogimpl.obj
 0001:0001b047       __unwindfunclet$?slotChange@dialog@@QAEXPAVQListViewItem@@HABVQString@@@Z$3 1001c047 f   dialogimpl.obj
 0001:0001b050       __unwindfunclet$?slotChange@dialog@@QAEXPAVQListViewItem@@HABVQString@@@Z$4 1001c050 f   dialogimpl.obj
 0001:0001b059       __unwindfunclet$?slotChange@dialog@@QAEXPAVQListViewItem@@HABVQString@@@Z$1 1001c059 f   dialogimpl.obj
 0001:0001b062       __unwindfunclet$?slotChange@dialog@@QAEXPAVQListViewItem@@HABVQString@@@Z$5 1001c062 f   dialogimpl.obj
 0001:0001b06b       __ehhandler$?slotChange@dialog@@QAEXPAVQListViewItem@@HABVQString@@@Z 1001c06b f   dialogimpl.obj
 0001:0001b086       __unwindfunclet$??0manage_tempBase@@QAE@PAVQWidget@@PBD_NI@Z$0 1001c086 f   manage_temp.obj
 0001:0001b08f       __unwindfunclet$??0manage_tempBase@@QAE@PAVQWidget@@PBD_NI@Z$1 1001c08f f   manage_temp.obj
 0001:0001b099       __unwindfunclet$??0manage_tempBase@@QAE@PAVQWidget@@PBD_NI@Z$2 1001c099 f   manage_temp.obj
 0001:0001b0a3       __unwindfunclet$??0manage_tempBase@@QAE@PAVQWidget@@PBD_NI@Z$3 1001c0a3 f   manage_temp.obj
 0001:0001b0ad       __unwindfunclet$??0manage_tempBase@@QAE@PAVQWidget@@PBD_NI@Z$4 1001c0ad f   manage_temp.obj
 0001:0001b0b7       __unwindfunclet$??0manage_tempBase@@QAE@PAVQWidget@@PBD_NI@Z$5 1001c0b7 f   manage_temp.obj
 0001:0001b0c1       __unwindfunclet$??0manage_tempBase@@QAE@PAVQWidget@@PBD_NI@Z$6 1001c0c1 f   manage_temp.obj
 0001:0001b0cb       __unwindfunclet$??0manage_tempBase@@QAE@PAVQWidget@@PBD_NI@Z$7 1001c0cb f   manage_temp.obj
 0001:0001b0d5       __unwindfunclet$??0manage_tempBase@@QAE@PAVQWidget@@PBD_NI@Z$8 1001c0d5 f   manage_temp.obj
 0001:0001b0df       __unwindfunclet$??0manage_tempBase@@QAE@PAVQWidget@@PBD_NI@Z$9 1001c0df f   manage_temp.obj
 0001:0001b0e9       __unwindfunclet$??0manage_tempBase@@QAE@PAVQWidget@@PBD_NI@Z$10 1001c0e9 f   manage_temp.obj
 0001:0001b0f3       __unwindfunclet$??0manage_tempBase@@QAE@PAVQWidget@@PBD_NI@Z$11 1001c0f3 f   manage_temp.obj
 0001:0001b0fd       __unwindfunclet$??0manage_tempBase@@QAE@PAVQWidget@@PBD_NI@Z$12 1001c0fd f   manage_temp.obj
 0001:0001b107       __unwindfunclet$??0manage_tempBase@@QAE@PAVQWidget@@PBD_NI@Z$13 1001c107 f   manage_temp.obj
 0001:0001b111       __unwindfunclet$??0manage_tempBase@@QAE@PAVQWidget@@PBD_NI@Z$14 1001c111 f   manage_temp.obj
 0001:0001b11b       __unwindfunclet$??0manage_tempBase@@QAE@PAVQWidget@@PBD_NI@Z$15 1001c11b f   manage_temp.obj
 0001:0001b125       __unwindfunclet$??0manage_tempBase@@QAE@PAVQWidget@@PBD_NI@Z$16 1001c125 f   manage_temp.obj
 0001:0001b12f       __unwindfunclet$??0manage_tempBase@@QAE@PAVQWidget@@PBD_NI@Z$17 1001c12f f   manage_temp.obj
 0001:0001b139       __unwindfunclet$??0manage_tempBase@@QAE@PAVQWidget@@PBD_NI@Z$18 1001c139 f   manage_temp.obj
 0001:0001b143       __unwindfunclet$??0manage_tempBase@@QAE@PAVQWidget@@PBD_NI@Z$19 1001c143 f   manage_temp.obj
 0001:0001b14d       __unwindfunclet$??0manage_tempBase@@QAE@PAVQWidget@@PBD_NI@Z$20 1001c14d f   manage_temp.obj
 0001:0001b157       __unwindfunclet$??0manage_tempBase@@QAE@PAVQWidget@@PBD_NI@Z$21 1001c157 f   manage_temp.obj
 0001:0001b161       __unwindfunclet$??0manage_tempBase@@QAE@PAVQWidget@@PBD_NI@Z$22 1001c161 f   manage_temp.obj
 0001:0001b16b       __unwindfunclet$??0manage_tempBase@@QAE@PAVQWidget@@PBD_NI@Z$23 1001c16b f   manage_temp.obj
 0001:0001b174       __unwindfunclet$??0manage_tempBase@@QAE@PAVQWidget@@PBD_NI@Z$24 1001c174 f   manage_temp.obj
 0001:0001b17d       __unwindfunclet$??0manage_tempBase@@QAE@PAVQWidget@@PBD_NI@Z$25 1001c17d f   manage_temp.obj
 0001:0001b187       __unwindfunclet$??0manage_tempBase@@QAE@PAVQWidget@@PBD_NI@Z$26 1001c187 f   manage_temp.obj
 0001:0001b191       __unwindfunclet$??0manage_tempBase@@QAE@PAVQWidget@@PBD_NI@Z$27 1001c191 f   manage_temp.obj
 0001:0001b19b       __unwindfunclet$??0manage_tempBase@@QAE@PAVQWidget@@PBD_NI@Z$28 1001c19b f   manage_temp.obj
 0001:0001b1a5       __unwindfunclet$??0manage_tempBase@@QAE@PAVQWidget@@PBD_NI@Z$29 1001c1a5 f   manage_temp.obj
 0001:0001b1ae       __unwindfunclet$??0manage_tempBase@@QAE@PAVQWidget@@PBD_NI@Z$30 1001c1ae f   manage_temp.obj
 0001:0001b1b8       __unwindfunclet$??0manage_tempBase@@QAE@PAVQWidget@@PBD_NI@Z$31 1001c1b8 f   manage_temp.obj
 0001:0001b1c2       __unwindfunclet$??0manage_tempBase@@QAE@PAVQWidget@@PBD_NI@Z$32 1001c1c2 f   manage_temp.obj
 0001:0001b1cc       __unwindfunclet$??0manage_tempBase@@QAE@PAVQWidget@@PBD_NI@Z$33 1001c1cc f   manage_temp.obj
 0001:0001b1d5       __unwindfunclet$??0manage_tempBase@@QAE@PAVQWidget@@PBD_NI@Z$34 1001c1d5 f   manage_temp.obj
 0001:0001b1de       __unwindfunclet$??0manage_tempBase@@QAE@PAVQWidget@@PBD_NI@Z$35 1001c1de f   manage_temp.obj
 0001:0001b1e8       __unwindfunclet$??0manage_tempBase@@QAE@PAVQWidget@@PBD_NI@Z$36 1001c1e8 f   manage_temp.obj
 0001:0001b1f2       __unwindfunclet$??0manage_tempBase@@QAE@PAVQWidget@@PBD_NI@Z$37 1001c1f2 f   manage_temp.obj
 0001:0001b1fc       __unwindfunclet$??0manage_tempBase@@QAE@PAVQWidget@@PBD_NI@Z$38 1001c1fc f   manage_temp.obj
 0001:0001b206       __unwindfunclet$??0manage_tempBase@@QAE@PAVQWidget@@PBD_NI@Z$39 1001c206 f   manage_temp.obj
 0001:0001b210       __unwindfunclet$??0manage_tempBase@@QAE@PAVQWidget@@PBD_NI@Z$40 1001c210 f   manage_temp.obj
 0001:0001b21a       __unwindfunclet$??0manage_tempBase@@QAE@PAVQWidget@@PBD_NI@Z$41 1001c21a f   manage_temp.obj
 0001:0001b223       __ehhandler$??0manage_tempBase@@QAE@PAVQWidget@@PBD_NI@Z 1001c223 f   manage_temp.obj
 0001:0001b23e       __unwindfunclet$?languageChange@manage_tempBase@@MAEXXZ$0 1001c23e f   manage_temp.obj
 0001:0001b247       __unwindfunclet$?languageChange@manage_tempBase@@MAEXXZ$1 1001c247 f   manage_temp.obj
 0001:0001b250       __unwindfunclet$?languageChange@manage_tempBase@@MAEXXZ$2 1001c250 f   manage_temp.obj
 0001:0001b259       __unwindfunclet$?languageChange@manage_tempBase@@MAEXXZ$3 1001c259 f   manage_temp.obj
 0001:0001b262       __unwindfunclet$?languageChange@manage_tempBase@@MAEXXZ$4 1001c262 f   manage_temp.obj
 0001:0001b26b       __unwindfunclet$?languageChange@manage_tempBase@@MAEXXZ$5 1001c26b f   manage_temp.obj
 0001:0001b274       __unwindfunclet$?languageChange@manage_tempBase@@MAEXXZ$6 1001c274 f   manage_temp.obj
 0001:0001b27d       __unwindfunclet$?languageChange@manage_tempBase@@MAEXXZ$7 1001c27d f   manage_temp.obj
 0001:0001b286       __unwindfunclet$?languageChange@manage_tempBase@@MAEXXZ$8 1001c286 f   manage_temp.obj
 0001:0001b28f       __unwindfunclet$?languageChange@manage_tempBase@@MAEXXZ$9 1001c28f f   manage_temp.obj
 0001:0001b298       __unwindfunclet$?languageChange@manage_tempBase@@MAEXXZ$10 1001c298 f   manage_temp.obj
 0001:0001b2a1       __unwindfunclet$?languageChange@manage_tempBase@@MAEXXZ$11 1001c2a1 f   manage_temp.obj
 0001:0001b2aa       __unwindfunclet$?languageChange@manage_tempBase@@MAEXXZ$12 1001c2aa f   manage_temp.obj
 0001:0001b2b3       __unwindfunclet$?languageChange@manage_tempBase@@MAEXXZ$13 1001c2b3 f   manage_temp.obj
 0001:0001b2bc       __unwindfunclet$?languageChange@manage_tempBase@@MAEXXZ$14 1001c2bc f   manage_temp.obj
 0001:0001b2c5       __unwindfunclet$?languageChange@manage_tempBase@@MAEXXZ$15 1001c2c5 f   manage_temp.obj
 0001:0001b2ce       __unwindfunclet$?languageChange@manage_tempBase@@MAEXXZ$16 1001c2ce f   manage_temp.obj
 0001:0001b2d7       __unwindfunclet$?languageChange@manage_tempBase@@MAEXXZ$17 1001c2d7 f   manage_temp.obj
 0001:0001b2e0       __unwindfunclet$?languageChange@manage_tempBase@@MAEXXZ$18 1001c2e0 f   manage_temp.obj
 0001:0001b2e9       __unwindfunclet$?languageChange@manage_tempBase@@MAEXXZ$19 1001c2e9 f   manage_temp.obj
 0001:0001b2f2       __unwindfunclet$?languageChange@manage_tempBase@@MAEXXZ$20 1001c2f2 f   manage_temp.obj
 0001:0001b2fb       __unwindfunclet$?languageChange@manage_tempBase@@MAEXXZ$21 1001c2fb f   manage_temp.obj
 0001:0001b304       __unwindfunclet$?languageChange@manage_tempBase@@MAEXXZ$22 1001c304 f   manage_temp.obj
 0001:0001b30d       __ehhandler$?languageChange@manage_tempBase@@MAEXXZ 1001c30d f   manage_temp.obj
 0001:0001b328       __unwindfunclet$??0manage_temp@@QAE@ABVQStringList@@QBVTemplateList@@QAVIGetDocuments@@PAVQWidget@@PBD_NI@Z$0 1001c328 f   manage_tempimpl.obj
 0001:0001b330       __unwindfunclet$??0manage_temp@@QAE@ABVQStringList@@QBVTemplateList@@QAVIGetDocuments@@PAVQWidget@@PBD_NI@Z$1 1001c330 f   manage_tempimpl.obj
 0001:0001b33e       __unwindfunclet$??0manage_temp@@QAE@ABVQStringList@@QBVTemplateList@@QAVIGetDocuments@@PAVQWidget@@PBD_NI@Z$2 1001c33e f   manage_tempimpl.obj
 0001:0001b347       __unwindfunclet$??0manage_temp@@QAE@ABVQStringList@@QBVTemplateList@@QAVIGetDocuments@@PAVQWidget@@PBD_NI@Z$3 1001c347 f   manage_tempimpl.obj
 0001:0001b350       __unwindfunclet$??0manage_temp@@QAE@ABVQStringList@@QBVTemplateList@@QAVIGetDocuments@@PAVQWidget@@PBD_NI@Z$4 1001c350 f   manage_tempimpl.obj
 0001:0001b359       __unwindfunclet$??0manage_temp@@QAE@ABVQStringList@@QBVTemplateList@@QAVIGetDocuments@@PAVQWidget@@PBD_NI@Z$5 1001c359 f   manage_tempimpl.obj
 0001:0001b362       __unwindfunclet$??0manage_temp@@QAE@ABVQStringList@@QBVTemplateList@@QAVIGetDocuments@@PAVQWidget@@PBD_NI@Z$6 1001c362 f   manage_tempimpl.obj
 0001:0001b36b       __unwindfunclet$??0manage_temp@@QAE@ABVQStringList@@QBVTemplateList@@QAVIGetDocuments@@PAVQWidget@@PBD_NI@Z$7 1001c36b f   manage_tempimpl.obj
 0001:0001b374       __ehhandler$??0manage_temp@@QAE@ABVQStringList@@QBVTemplateList@@QAVIGetDocuments@@PAVQWidget@@PBD_NI@Z 1001c374 f   manage_tempimpl.obj
 0001:0001b38f       __unwindfunclet$??1manage_temp@@UAE@XZ$0 1001c38f f   manage_tempimpl.obj
 0001:0001b397       __unwindfunclet$??1manage_temp@@UAE@XZ$1 1001c397 f   manage_tempimpl.obj
 0001:0001b3a5       __unwindfunclet$??1manage_temp@@UAE@XZ$2 1001c3a5 f   manage_tempimpl.obj
 0001:0001b3ae       __unwindfunclet$??1manage_temp@@UAE@XZ$3 1001c3ae f   manage_tempimpl.obj
 0001:0001b3b7       __unwindfunclet$??1manage_temp@@UAE@XZ$4 1001c3b7 f   manage_tempimpl.obj
 0001:0001b3c0       __unwindfunclet$??1manage_temp@@UAE@XZ$5 1001c3c0 f   manage_tempimpl.obj
 0001:0001b3c9       __unwindfunclet$??1manage_temp@@UAE@XZ$6 1001c3c9 f   manage_tempimpl.obj
 0001:0001b3d2       __unwindfunclet$??1manage_temp@@UAE@XZ$7 1001c3d2 f   manage_tempimpl.obj
 0001:0001b3db       __ehhandler$??1manage_temp@@UAE@XZ 1001c3db f   manage_tempimpl.obj
 0001:0001b3f6       __unwindfunclet$?autoNumberSlots@manage_temp@@QAEXXZ$0 1001c3f6 f   manage_tempimpl.obj
 0001:0001b3ff       __unwindfunclet$?autoNumberSlots@manage_temp@@QAEXXZ$1 1001c3ff f   manage_tempimpl.obj
 0001:0001b408       __unwindfunclet$?autoNumberSlots@manage_temp@@QAEXXZ$2 1001c408 f   manage_tempimpl.obj
 0001:0001b411       __ehhandler$?autoNumberSlots@manage_temp@@QAEXXZ 1001c411 f   manage_tempimpl.obj
 0001:0001b42c       __unwindfunclet$?changePrefix@manage_temp@@QAEXABVQString@@@Z$0 1001c42c f   manage_tempimpl.obj
 0001:0001b435       __unwindfunclet$?changePrefix@manage_temp@@QAEXABVQString@@@Z$1 1001c435 f   manage_tempimpl.obj
 0001:0001b43e       __unwindfunclet$?changePrefix@manage_temp@@QAEXABVQString@@@Z$2 1001c43e f   manage_tempimpl.obj
 0001:0001b448       __unwindfunclet$?changePrefix@manage_temp@@QAEXABVQString@@@Z$3 1001c448 f   manage_tempimpl.obj
 0001:0001b451       __unwindfunclet$?changePrefix@manage_temp@@QAEXABVQString@@@Z$4 1001c451 f   manage_tempimpl.obj
 0001:0001b45a       __unwindfunclet$?changePrefix@manage_temp@@QAEXABVQString@@@Z$5 1001c45a f   manage_tempimpl.obj
 0001:0001b463       __unwindfunclet$?changePrefix@manage_temp@@QAEXABVQString@@@Z$6 1001c463 f   manage_tempimpl.obj
 0001:0001b46c       __unwindfunclet$?changePrefix@manage_temp@@QAEXABVQString@@@Z$7 1001c46c f   manage_tempimpl.obj
 0001:0001b475       __unwindfunclet$?changePrefix@manage_temp@@QAEXABVQString@@@Z$8 1001c475 f   manage_tempimpl.obj
 0001:0001b47e       __unwindfunclet$?changePrefix@manage_temp@@QAEXABVQString@@@Z$9 1001c47e f   manage_tempimpl.obj
 0001:0001b487       __unwindfunclet$?changePrefix@manage_temp@@QAEXABVQString@@@Z$11 1001c487 f   manage_tempimpl.obj
 0001:0001b490       __ehhandler$?changePrefix@manage_temp@@QAEXABVQString@@@Z 1001c490 f   manage_tempimpl.obj
 0001:0001b4ab       __unwindfunclet$?clearSlots@manage_temp@@QAEXXZ$0 1001c4ab f   manage_tempimpl.obj
 0001:0001b4b4       __unwindfunclet$?clearSlots@manage_temp@@QAEXXZ$1 1001c4b4 f   manage_tempimpl.obj
 0001:0001b4bd       __unwindfunclet$?clearSlots@manage_temp@@QAEXXZ$2 1001c4bd f   manage_tempimpl.obj
 0001:0001b4c6       __ehhandler$?clearSlots@manage_temp@@QAEXXZ 1001c4c6 f   manage_tempimpl.obj
 0001:0001b4e1       __unwindfunclet$?getTemplates@manage_temp@@QAEXQAVTemplateList@@@Z$0 1001c4e1 f   manage_tempimpl.obj
 0001:0001b4e9       __unwindfunclet$?getTemplates@manage_temp@@QAEXQAVTemplateList@@@Z$1 1001c4e9 f   manage_tempimpl.obj
 0001:0001b4f2       __unwindfunclet$?getTemplates@manage_temp@@QAEXQAVTemplateList@@@Z$2 1001c4f2 f   manage_tempimpl.obj
 0001:0001b4fc       __ehhandler$?getTemplates@manage_temp@@QAEXQAVTemplateList@@@Z 1001c4fc f   manage_tempimpl.obj
 0001:0001b517       __unwindfunclet$?loadTemplates@manage_temp@@AAEXABVQStringList@@QBVTemplateList@@@Z$0 1001c517 f   manage_tempimpl.obj
 0001:0001b51f       __unwindfunclet$?loadTemplates@manage_temp@@AAEXABVQStringList@@QBVTemplateList@@@Z$1 1001c51f f   manage_tempimpl.obj
 0001:0001b528       __unwindfunclet$?loadTemplates@manage_temp@@AAEXABVQStringList@@QBVTemplateList@@@Z$2 1001c528 f   manage_tempimpl.obj
 0001:0001b532       __unwindfunclet$?loadTemplates@manage_temp@@AAEXABVQStringList@@QBVTemplateList@@@Z$3 1001c532 f   manage_tempimpl.obj
 0001:0001b53a       __unwindfunclet$?loadTemplates@manage_temp@@AAEXABVQStringList@@QBVTemplateList@@@Z$4 1001c53a f   manage_tempimpl.obj
 0001:0001b543       __unwindfunclet$?loadTemplates@manage_temp@@AAEXABVQStringList@@QBVTemplateList@@@Z$5 1001c543 f   manage_tempimpl.obj
 0001:0001b54c       __ehhandler$?loadTemplates@manage_temp@@AAEXABVQStringList@@QBVTemplateList@@@Z 1001c54c f   manage_tempimpl.obj
 0001:0001b567       __unwindfunclet$?newTemplate@manage_temp@@QAEXXZ$0 1001c567 f   manage_tempimpl.obj
 0001:0001b570       __unwindfunclet$?newTemplate@manage_temp@@QAEXXZ$1 1001c570 f   manage_tempimpl.obj
 0001:0001b579       __unwindfunclet$?newTemplate@manage_temp@@QAEXXZ$2 1001c579 f   manage_tempimpl.obj
 0001:0001b582       __unwindfunclet$?newTemplate@manage_temp@@QAEXXZ$3 1001c582 f   manage_tempimpl.obj
 0001:0001b58b       __unwindfunclet$?newTemplate@manage_temp@@QAEXXZ$4 1001c58b f   manage_tempimpl.obj
 0001:0001b594       __unwindfunclet$?newTemplate@manage_temp@@QAEXXZ$5 1001c594 f   manage_tempimpl.obj
 0001:0001b59d       __unwindfunclet$?newTemplate@manage_temp@@QAEXXZ$6 1001c59d f   manage_tempimpl.obj
 0001:0001b5a7       __unwindfunclet$?newTemplate@manage_temp@@QAEXXZ$7 1001c5a7 f   manage_tempimpl.obj
 0001:0001b5b0       __ehhandler$?newTemplate@manage_temp@@QAEXXZ 1001c5b0 f   manage_tempimpl.obj
 0001:0001b5cb       __unwindfunclet$?saveCurrentTemplate@manage_temp@@QAEXXZ$0 1001c5cb f   manage_tempimpl.obj
 0001:0001b5d4       __unwindfunclet$?saveCurrentTemplate@manage_temp@@QAEXXZ$1 1001c5d4 f   manage_tempimpl.obj
 0001:0001b5dd       __unwindfunclet$?saveCurrentTemplate@manage_temp@@QAEXXZ$2 1001c5dd f   manage_tempimpl.obj
 0001:0001b5e6       __unwindfunclet$?saveCurrentTemplate@manage_temp@@QAEXXZ$3 1001c5e6 f   manage_tempimpl.obj
 0001:0001b5ef       __ehhandler$?saveCurrentTemplate@manage_temp@@QAEXXZ 1001c5ef f   manage_tempimpl.obj
 0001:0001b60a       __unwindfunclet$?selectTemplate@manage_temp@@QAEXABVQString@@@Z$0 1001c60a f   manage_tempimpl.obj
 0001:0001b613       __unwindfunclet$?selectTemplate@manage_temp@@QAEXABVQString@@@Z$1 1001c613 f   manage_tempimpl.obj
 0001:0001b61c       __unwindfunclet$?selectTemplate@manage_temp@@QAEXABVQString@@@Z$2 1001c61c f   manage_tempimpl.obj
 0001:0001b625       __ehhandler$?selectTemplate@manage_temp@@QAEXABVQString@@@Z 1001c625 f   manage_tempimpl.obj
 0001:0001b640       __unwindfunclet$?updateInstanceDisplay@manage_temp@@AAEXXZ$0 1001c640 f   manage_tempimpl.obj
 0001:0001b649       __unwindfunclet$?updateInstanceDisplay@manage_temp@@AAEXXZ$1 1001c649 f   manage_tempimpl.obj
 0001:0001b652       __unwindfunclet$?updateInstanceDisplay@manage_temp@@AAEXXZ$2 1001c652 f   manage_tempimpl.obj
 0001:0001b65b       __unwindfunclet$?updateInstanceDisplay@manage_temp@@AAEXXZ$3 1001c65b f   manage_tempimpl.obj
 0001:0001b664       __unwindfunclet$?updateInstanceDisplay@manage_temp@@AAEXXZ$4 1001c664 f   manage_tempimpl.obj
 0001:0001b66d       __unwindfunclet$?updateInstanceDisplay@manage_temp@@AAEXXZ$5 1001c66d f   manage_tempimpl.obj
 0001:0001b676       __unwindfunclet$?updateInstanceDisplay@manage_temp@@AAEXXZ$6 1001c676 f   manage_tempimpl.obj
 0001:0001b67f       __unwindfunclet$?updateInstanceDisplay@manage_temp@@AAEXXZ$7 1001c67f f   manage_tempimpl.obj
 0001:0001b689       __unwindfunclet$?updateInstanceDisplay@manage_temp@@AAEXXZ$8 1001c689 f   manage_tempimpl.obj
 0001:0001b6a3       __ehhandler$?updateInstanceDisplay@manage_temp@@AAEXXZ 1001c6a3 f   manage_tempimpl.obj
 0001:0001b6be       __unwindfunclet$?keys@plugindesc@@UAE?AVQStringList@@ABVQString@@0@Z$0 1001c6be f   plugindesc.obj
 0001:0001b6d8       __unwindfunclet$?keys@plugindesc@@UAE?AVQStringList@@ABVQString@@0@Z$1 1001c6d8 f   plugindesc.obj
 0001:0001b6e1       __ehhandler$?keys@plugindesc@@UAE?AVQStringList@@ABVQString@@0@Z 1001c6e1 f   plugindesc.obj
 0001:0001b6fc       __unwindfunclet$??0processItem@@QAE@PAVQListView@@VQString@@1@Z$0 1001c6fc f   processItem.obj
 0001:0001b705       __unwindfunclet$??0processItem@@QAE@PAVQListView@@VQString@@1@Z$1 1001c705 f   processItem.obj
 0001:0001b70e       __unwindfunclet$??0processItem@@QAE@PAVQListView@@VQString@@1@Z$2 1001c70e f   processItem.obj
 0001:0001b717       __unwindfunclet$??0processItem@@QAE@PAVQListView@@VQString@@1@Z$3 1001c717 f   processItem.obj
 0001:0001b720       __unwindfunclet$??0processItem@@QAE@PAVQListView@@VQString@@1@Z$4 1001c720 f   processItem.obj
 0001:0001b729       __unwindfunclet$??0processItem@@QAE@PAVQListView@@VQString@@1@Z$5 1001c729 f   processItem.obj
 0001:0001b732       __unwindfunclet$??0processItem@@QAE@PAVQListView@@VQString@@1@Z$6 1001c732 f   processItem.obj
 0001:0001b73b       __unwindfunclet$??0processItem@@QAE@PAVQListView@@VQString@@1@Z$7 1001c73b f   processItem.obj
 0001:0001b744       __unwindfunclet$??0processItem@@QAE@PAVQListView@@VQString@@1@Z$8 1001c744 f   processItem.obj
 0001:0001b74d       __ehhandler$??0processItem@@QAE@PAVQListView@@VQString@@1@Z 1001c74d f   processItem.obj
 0001:0001b768       __unwindfunclet$?compare@processItem@@UBEHPAVQListViewItem@@H_N@Z$0 1001c768 f   processItem.obj
 0001:0001b771       __unwindfunclet$?compare@processItem@@UBEHPAVQListViewItem@@H_N@Z$1 1001c771 f   processItem.obj
 0001:0001b77a       __unwindfunclet$?compare@processItem@@UBEHPAVQListViewItem@@H_N@Z$2 1001c77a f   processItem.obj
 0001:0001b783       __unwindfunclet$?compare@processItem@@UBEHPAVQListViewItem@@H_N@Z$3 1001c783 f   processItem.obj
 0001:0001b78c       __ehhandler$?compare@processItem@@UBEHPAVQListViewItem@@H_N@Z 1001c78c f   processItem.obj
 0001:0001b7a7       __unwindfunclet$?paintCell@processItem@@UAEXPAVQPainter@@ABVQColorGroup@@HHH@Z$0 1001c7a7 f   processItem.obj
 0001:0001b7b0       __ehhandler$?paintCell@processItem@@UAEXPAVQPainter@@ABVQColorGroup@@HHH@Z 1001c7b0 f   processItem.obj
 0001:0001b7cb       __unwindfunclet$??0autoNumberDialogBase@@QAE@PAVQWidget@@PBD_NI@Z$0 1001c7cb f   autonumberdialog.obj
 0001:0001b7d4       __unwindfunclet$??0autoNumberDialogBase@@QAE@PAVQWidget@@PBD_NI@Z$1 1001c7d4 f   autonumberdialog.obj
 0001:0001b7de       __unwindfunclet$??0autoNumberDialogBase@@QAE@PAVQWidget@@PBD_NI@Z$2 1001c7de f   autonumberdialog.obj
 0001:0001b7e8       __unwindfunclet$??0autoNumberDialogBase@@QAE@PAVQWidget@@PBD_NI@Z$3 1001c7e8 f   autonumberdialog.obj
 0001:0001b7f2       __unwindfunclet$??0autoNumberDialogBase@@QAE@PAVQWidget@@PBD_NI@Z$4 1001c7f2 f   autonumberdialog.obj
 0001:0001b7fc       __unwindfunclet$??0autoNumberDialogBase@@QAE@PAVQWidget@@PBD_NI@Z$5 1001c7fc f   autonumberdialog.obj
 0001:0001b806       __unwindfunclet$??0autoNumberDialogBase@@QAE@PAVQWidget@@PBD_NI@Z$6 1001c806 f   autonumberdialog.obj
 0001:0001b810       __unwindfunclet$??0autoNumberDialogBase@@QAE@PAVQWidget@@PBD_NI@Z$7 1001c810 f   autonumberdialog.obj
 0001:0001b81a       __unwindfunclet$??0autoNumberDialogBase@@QAE@PAVQWidget@@PBD_NI@Z$8 1001c81a f   autonumberdialog.obj
 0001:0001b824       __unwindfunclet$??0autoNumberDialogBase@@QAE@PAVQWidget@@PBD_NI@Z$9 1001c824 f   autonumberdialog.obj
 0001:0001b82e       __unwindfunclet$??0autoNumberDialogBase@@QAE@PAVQWidget@@PBD_NI@Z$10 1001c82e f   autonumberdialog.obj
 0001:0001b838       __unwindfunclet$??0autoNumberDialogBase@@QAE@PAVQWidget@@PBD_NI@Z$11 1001c838 f   autonumberdialog.obj
 0001:0001b842       __unwindfunclet$??0autoNumberDialogBase@@QAE@PAVQWidget@@PBD_NI@Z$12 1001c842 f   autonumberdialog.obj
 0001:0001b84c       __unwindfunclet$??0autoNumberDialogBase@@QAE@PAVQWidget@@PBD_NI@Z$13 1001c84c f   autonumberdialog.obj
 0001:0001b856       __unwindfunclet$??0autoNumberDialogBase@@QAE@PAVQWidget@@PBD_NI@Z$14 1001c856 f   autonumberdialog.obj
 0001:0001b860       __unwindfunclet$??0autoNumberDialogBase@@QAE@PAVQWidget@@PBD_NI@Z$15 1001c860 f   autonumberdialog.obj
 0001:0001b86a       __unwindfunclet$??0autoNumberDialogBase@@QAE@PAVQWidget@@PBD_NI@Z$16 1001c86a f   autonumberdialog.obj
 0001:0001b874       __unwindfunclet$??0autoNumberDialogBase@@QAE@PAVQWidget@@PBD_NI@Z$17 1001c874 f   autonumberdialog.obj
 0001:0001b87e       __ehhandler$??0autoNumberDialogBase@@QAE@PAVQWidget@@PBD_NI@Z 1001c87e f   autonumberdialog.obj
 0001:0001b899       __unwindfunclet$?languageChange@autoNumberDialogBase@@MAEXXZ$0 1001c899 f   autonumberdialog.obj
 0001:0001b8a2       __unwindfunclet$?languageChange@autoNumberDialogBase@@MAEXXZ$1 1001c8a2 f   autonumberdialog.obj
 0001:0001b8ab       __unwindfunclet$?languageChange@autoNumberDialogBase@@MAEXXZ$2 1001c8ab f   autonumberdialog.obj
 0001:0001b8b4       __unwindfunclet$?languageChange@autoNumberDialogBase@@MAEXXZ$3 1001c8b4 f   autonumberdialog.obj
 0001:0001b8bd       __unwindfunclet$?languageChange@autoNumberDialogBase@@MAEXXZ$4 1001c8bd f   autonumberdialog.obj
 0001:0001b8c6       __unwindfunclet$?languageChange@autoNumberDialogBase@@MAEXXZ$5 1001c8c6 f   autonumberdialog.obj
 0001:0001b8cf       __unwindfunclet$?languageChange@autoNumberDialogBase@@MAEXXZ$6 1001c8cf f   autonumberdialog.obj
 0001:0001b8d8       __unwindfunclet$?languageChange@autoNumberDialogBase@@MAEXXZ$7 1001c8d8 f   autonumberdialog.obj
 0001:0001b8e1       __unwindfunclet$?languageChange@autoNumberDialogBase@@MAEXXZ$8 1001c8e1 f   autonumberdialog.obj
 0001:0001b8ea       __unwindfunclet$?languageChange@autoNumberDialogBase@@MAEXXZ$9 1001c8ea f   autonumberdialog.obj
 0001:0001b8f3       __unwindfunclet$?languageChange@autoNumberDialogBase@@MAEXXZ$10 1001c8f3 f   autonumberdialog.obj
 0001:0001b8fc       __unwindfunclet$?languageChange@autoNumberDialogBase@@MAEXXZ$11 1001c8fc f   autonumberdialog.obj
 0001:0001b905       __unwindfunclet$?languageChange@autoNumberDialogBase@@MAEXXZ$12 1001c905 f   autonumberdialog.obj
 0001:0001b90e       __unwindfunclet$?languageChange@autoNumberDialogBase@@MAEXXZ$13 1001c90e f   autonumberdialog.obj
 0001:0001b917       __ehhandler$?languageChange@autoNumberDialogBase@@MAEXXZ 1001c917 f   autonumberdialog.obj
 0001:0001b932       __unwindfunclet$??0dialogBase@@QAE@PAVQWidget@@PBDI@Z$0 1001c932 f   dialog.obj
 0001:0001b93b       __unwindfunclet$??0dialogBase@@QAE@PAVQWidget@@PBDI@Z$1 1001c93b f   dialog.obj
 0001:0001b945       __unwindfunclet$??0dialogBase@@QAE@PAVQWidget@@PBDI@Z$2 1001c945 f   dialog.obj
 0001:0001b94f       __unwindfunclet$??0dialogBase@@QAE@PAVQWidget@@PBDI@Z$3 1001c94f f   dialog.obj
 0001:0001b959       __unwindfunclet$??0dialogBase@@QAE@PAVQWidget@@PBDI@Z$4 1001c959 f   dialog.obj
 0001:0001b963       __unwindfunclet$??0dialogBase@@QAE@PAVQWidget@@PBDI@Z$5 1001c963 f   dialog.obj
 0001:0001b96c       __unwindfunclet$??0dialogBase@@QAE@PAVQWidget@@PBDI@Z$6 1001c96c f   dialog.obj
 0001:0001b975       __unwindfunclet$??0dialogBase@@QAE@PAVQWidget@@PBDI@Z$7 1001c975 f   dialog.obj
 0001:0001b97e       __unwindfunclet$??0dialogBase@@QAE@PAVQWidget@@PBDI@Z$8 1001c97e f   dialog.obj
 0001:0001b987       __unwindfunclet$??0dialogBase@@QAE@PAVQWidget@@PBDI@Z$9 1001c987 f   dialog.obj
 0001:0001b990       __unwindfunclet$??0dialogBase@@QAE@PAVQWidget@@PBDI@Z$10 1001c990 f   dialog.obj
 0001:0001b99a       __unwindfunclet$??0dialogBase@@QAE@PAVQWidget@@PBDI@Z$11 1001c99a f   dialog.obj
 0001:0001b9a4       __unwindfunclet$??0dialogBase@@QAE@PAVQWidget@@PBDI@Z$12 1001c9a4 f   dialog.obj
 0001:0001b9ae       __unwindfunclet$??0dialogBase@@QAE@PAVQWidget@@PBDI@Z$13 1001c9ae f   dialog.obj
 0001:0001b9b8       __unwindfunclet$??0dialogBase@@QAE@PAVQWidget@@PBDI@Z$14 1001c9b8 f   dialog.obj
 0001:0001b9c2       __unwindfunclet$??0dialogBase@@QAE@PAVQWidget@@PBDI@Z$15 1001c9c2 f   dialog.obj
 0001:0001b9cc       __unwindfunclet$??0dialogBase@@QAE@PAVQWidget@@PBDI@Z$16 1001c9cc f   dialog.obj
 0001:0001b9d6       __unwindfunclet$??0dialogBase@@QAE@PAVQWidget@@PBDI@Z$17 1001c9d6 f   dialog.obj
 0001:0001b9e0       __unwindfunclet$??0dialogBase@@QAE@PAVQWidget@@PBDI@Z$18 1001c9e0 f   dialog.obj
 0001:0001b9ea       __unwindfunclet$??0dialogBase@@QAE@PAVQWidget@@PBDI@Z$19 1001c9ea f   dialog.obj
 0001:0001b9f4       __unwindfunclet$??0dialogBase@@QAE@PAVQWidget@@PBDI@Z$20 1001c9f4 f   dialog.obj
 0001:0001b9fe       __unwindfunclet$??0dialogBase@@QAE@PAVQWidget@@PBDI@Z$21 1001c9fe f   dialog.obj
 0001:0001ba08       __unwindfunclet$??0dialogBase@@QAE@PAVQWidget@@PBDI@Z$22 1001ca08 f   dialog.obj
 0001:0001ba12       __unwindfunclet$??0dialogBase@@QAE@PAVQWidget@@PBDI@Z$23 1001ca12 f   dialog.obj
 0001:0001ba1c       __unwindfunclet$??0dialogBase@@QAE@PAVQWidget@@PBDI@Z$24 1001ca1c f   dialog.obj
 0001:0001ba26       __unwindfunclet$??0dialogBase@@QAE@PAVQWidget@@PBDI@Z$25 1001ca26 f   dialog.obj
 0001:0001ba30       __unwindfunclet$??0dialogBase@@QAE@PAVQWidget@@PBDI@Z$26 1001ca30 f   dialog.obj
 0001:0001ba3a       __unwindfunclet$??0dialogBase@@QAE@PAVQWidget@@PBDI@Z$27 1001ca3a f   dialog.obj
 0001:0001ba44       __unwindfunclet$??0dialogBase@@QAE@PAVQWidget@@PBDI@Z$28 1001ca44 f   dialog.obj
 0001:0001ba4e       __unwindfunclet$??0dialogBase@@QAE@PAVQWidget@@PBDI@Z$29 1001ca4e f   dialog.obj
 0001:0001ba58       __ehhandler$??0dialogBase@@QAE@PAVQWidget@@PBDI@Z 1001ca58 f   dialog.obj
 0001:0001ba73       __unwindfunclet$?languageChange@dialogBase@@MAEXXZ$0 1001ca73 f   dialog.obj
 0001:0001ba7c       __unwindfunclet$?languageChange@dialogBase@@MAEXXZ$1 1001ca7c f   dialog.obj
 0001:0001ba85       __unwindfunclet$?languageChange@dialogBase@@MAEXXZ$2 1001ca85 f   dialog.obj
 0001:0001ba8e       __unwindfunclet$?languageChange@dialogBase@@MAEXXZ$3 1001ca8e f   dialog.obj
 0001:0001ba97       __unwindfunclet$?languageChange@dialogBase@@MAEXXZ$4 1001ca97 f   dialog.obj
 0001:0001baa0       __unwindfunclet$?languageChange@dialogBase@@MAEXXZ$5 1001caa0 f   dialog.obj
 0001:0001baa9       __unwindfunclet$?languageChange@dialogBase@@MAEXXZ$6 1001caa9 f   dialog.obj
 0001:0001bab2       __unwindfunclet$?languageChange@dialogBase@@MAEXXZ$7 1001cab2 f   dialog.obj
 0001:0001babb       __unwindfunclet$?languageChange@dialogBase@@MAEXXZ$8 1001cabb f   dialog.obj
 0001:0001bac4       __unwindfunclet$?languageChange@dialogBase@@MAEXXZ$9 1001cac4 f   dialog.obj
 0001:0001bacd       __unwindfunclet$?languageChange@dialogBase@@MAEXXZ$10 1001cacd f   dialog.obj
 0001:0001bad6       __unwindfunclet$?languageChange@dialogBase@@MAEXXZ$11 1001cad6 f   dialog.obj
 0001:0001badf       __unwindfunclet$?languageChange@dialogBase@@MAEXXZ$12 1001cadf f   dialog.obj
 0001:0001bae8       __unwindfunclet$?languageChange@dialogBase@@MAEXXZ$13 1001cae8 f   dialog.obj
 0001:0001baf1       __unwindfunclet$?languageChange@dialogBase@@MAEXXZ$14 1001caf1 f   dialog.obj
 0001:0001bafa       __unwindfunclet$?languageChange@dialogBase@@MAEXXZ$15 1001cafa f   dialog.obj
 0001:0001bb03       __unwindfunclet$?languageChange@dialogBase@@MAEXXZ$16 1001cb03 f   dialog.obj
 0001:0001bb0c       __unwindfunclet$?languageChange@dialogBase@@MAEXXZ$17 1001cb0c f   dialog.obj
 0001:0001bb15       __unwindfunclet$?languageChange@dialogBase@@MAEXXZ$18 1001cb15 f   dialog.obj
 0001:0001bb1e       __unwindfunclet$?languageChange@dialogBase@@MAEXXZ$19 1001cb1e f   dialog.obj
 0001:0001bb27       __unwindfunclet$?languageChange@dialogBase@@MAEXXZ$20 1001cb27 f   dialog.obj
 0001:0001bb30       __unwindfunclet$?languageChange@dialogBase@@MAEXXZ$21 1001cb30 f   dialog.obj
 0001:0001bb39       __unwindfunclet$?languageChange@dialogBase@@MAEXXZ$22 1001cb39 f   dialog.obj
 0001:0001bb42       __unwindfunclet$?languageChange@dialogBase@@MAEXXZ$23 1001cb42 f   dialog.obj
 0001:0001bb4b       __unwindfunclet$?languageChange@dialogBase@@MAEXXZ$24 1001cb4b f   dialog.obj
 0001:0001bb54       __unwindfunclet$?languageChange@dialogBase@@MAEXXZ$25 1001cb54 f   dialog.obj
 0001:0001bb5d       __unwindfunclet$?languageChange@dialogBase@@MAEXXZ$26 1001cb5d f   dialog.obj
 0001:0001bb66       __unwindfunclet$?languageChange@dialogBase@@MAEXXZ$27 1001cb66 f   dialog.obj
 0001:0001bb6f       __unwindfunclet$?languageChange@dialogBase@@MAEXXZ$28 1001cb6f f   dialog.obj
 0001:0001bb78       __unwindfunclet$?languageChange@dialogBase@@MAEXXZ$29 1001cb78 f   dialog.obj
 0001:0001bb81       __unwindfunclet$?languageChange@dialogBase@@MAEXXZ$30 1001cb81 f   dialog.obj
 0001:0001bb8a       __unwindfunclet$?languageChange@dialogBase@@MAEXXZ$31 1001cb8a f   dialog.obj
 0001:0001bb93       __unwindfunclet$?languageChange@dialogBase@@MAEXXZ$32 1001cb93 f   dialog.obj
 0001:0001bb9c       __unwindfunclet$?languageChange@dialogBase@@MAEXXZ$33 1001cb9c f   dialog.obj
 0001:0001bba5       __unwindfunclet$?languageChange@dialogBase@@MAEXXZ$34 1001cba5 f   dialog.obj
 0001:0001bbae       __unwindfunclet$?languageChange@dialogBase@@MAEXXZ$35 1001cbae f   dialog.obj
 0001:0001bbb7       __unwindfunclet$?languageChange@dialogBase@@MAEXXZ$36 1001cbb7 f   dialog.obj
 0001:0001bbc0       __unwindfunclet$?languageChange@dialogBase@@MAEXXZ$37 1001cbc0 f   dialog.obj
 0001:0001bbc9       __ehhandler$?languageChange@dialogBase@@MAEXXZ 1001cbc9 f   dialog.obj
 0001:0001bbe4       __unwindfunclet$?command@alm_bncs_output@@IAEXVQString@@0@Z$0 1001cbe4 f   moc_alm_bncs_output.obj
 0001:0001bbed       __unwindfunclet$?command@alm_bncs_output@@IAEXVQString@@0@Z$1 1001cbed f   moc_alm_bncs_output.obj
 0001:0001bbf6       __unwindfunclet$?command@alm_bncs_output@@IAEXVQString@@0@Z$2 1001cbf6 f   moc_alm_bncs_output.obj
 0001:0001bc0a       __ehhandler$?command@alm_bncs_output@@IAEXVQString@@0@Z 1001cc0a f   moc_alm_bncs_output.obj
 0001:0001bc2f       __unwindfunclet$?qt_emit@alm_bncs_output@@UAE_NHPAUQUObject@@@Z$0 1001cc2f f   moc_alm_bncs_output.obj
 0001:0001bc38       __ehhandler$?qt_emit@alm_bncs_output@@UAE_NHPAUQUObject@@@Z 1001cc38 f   moc_alm_bncs_output.obj
 0001:0001bc53       __unwindfunclet$?qt_invoke@dialog@@UAE_NHPAUQUObject@@@Z$0 1001cc53 f   moc_alm_bncs_output.obj
 0001:0001bc53       __unwindfunclet$?menuNewFile@alm_bncs_output@@QAEXXZ$0 1001cc53 f   moc_alm_bncs_output.obj
 0001:0001bc53       __unwindfunclet$?qt_invoke@alm_bncs_output@@UAE_NHPAUQUObject@@@Z$0 1001cc53 f   moc_alm_bncs_output.obj
 0001:0001bc5c       __ehhandler$?qt_invoke@dialog@@UAE_NHPAUQUObject@@@Z 1001cc5c f   moc_alm_bncs_output.obj
 0001:0001bc5c       __ehhandler$?qt_invoke@alm_bncs_output@@UAE_NHPAUQUObject@@@Z 1001cc5c f   moc_alm_bncs_output.obj
 0001:0001bc5c       __ehhandler$?menuNewFile@alm_bncs_output@@QAEXXZ 1001cc5c f   moc_alm_bncs_output.obj
 0001:0001bc77       __unwindfunclet$?loadState@cfg_Settings@@SA?AVQString@@ABV2@@Z$0 1001cc77 f   cfg_widgets001:cfg_Settings.obj
 0001:0001bc80       __unwindfunclet$?loadState@cfg_Settings@@SA?AVQString@@ABV2@@Z$1 1001cc80 f   cfg_widgets001:cfg_Settings.obj
 0001:0001bc89       __unwindfunclet$?loadState@cfg_Settings@@SA?AVQString@@ABV2@@Z$2 1001cc89 f   cfg_widgets001:cfg_Settings.obj
 0001:0001bc92       __unwindfunclet$?loadState@cfg_Settings@@SA?AVQString@@ABV2@@Z$3 1001cc92 f   cfg_widgets001:cfg_Settings.obj
 0001:0001bcac       __ehhandler$?loadState@cfg_Settings@@SA?AVQString@@ABV2@@Z 1001ccac f   cfg_widgets001:cfg_Settings.obj
 0001:0001bcc7       __unwindfunclet$?loadState@cfg_Settings@@SAXAAVQPoint@@AAVQSize@@AA_NABVQString@@@Z$0 1001ccc7 f   cfg_widgets001:cfg_Settings.obj
 0001:0001bcd0       __unwindfunclet$?loadState@cfg_Settings@@SAXAAVQPoint@@AAVQSize@@AA_NABVQString@@@Z$1 1001ccd0 f   cfg_widgets001:cfg_Settings.obj
 0001:0001bcd9       __ehhandler$?loadState@cfg_Settings@@SAXAAVQPoint@@AAVQSize@@AA_NABVQString@@@Z 1001ccd9 f   cfg_widgets001:cfg_Settings.obj
 0001:0001bcf4       __unwindfunclet$?loadState@cfg_Settings@@SAXQAVQListView@@ABVQString@@@Z$0 1001ccf4 f   cfg_widgets001:cfg_Settings.obj
 0001:0001bcf4       __unwindfunclet$?loadState@cfg_Settings@@SAXQAVQTable@@ABVQString@@@Z$0 1001ccf4 f   cfg_widgets001:cfg_Settings.obj
 0001:0001bcfd       __unwindfunclet$?loadState@cfg_Settings@@SAXQAVQListView@@ABVQString@@@Z$1 1001ccfd f   cfg_widgets001:cfg_Settings.obj
 0001:0001bcfd       __unwindfunclet$?loadState@cfg_Settings@@SAXQAVQTable@@ABVQString@@@Z$1 1001ccfd f   cfg_widgets001:cfg_Settings.obj
 0001:0001bd06       __ehhandler$?loadState@cfg_Settings@@SAXQAVQListView@@ABVQString@@@Z 1001cd06 f   cfg_widgets001:cfg_Settings.obj
 0001:0001bd06       __ehhandler$?loadState@cfg_Settings@@SAXQAVQTable@@ABVQString@@@Z 1001cd06 f   cfg_widgets001:cfg_Settings.obj
 0001:0001bd21       __unwindfunclet$?saveState@cfg_Settings@@SAXABVQPoint@@ABVQSize@@AB_NABVQString@@@Z$0 1001cd21 f   cfg_widgets001:cfg_Settings.obj
 0001:0001bd2a       __unwindfunclet$?saveState@cfg_Settings@@SAXABVQPoint@@ABVQSize@@AB_NABVQString@@@Z$1 1001cd2a f   cfg_widgets001:cfg_Settings.obj
 0001:0001bd33       __unwindfunclet$?saveState@cfg_Settings@@SAXABVQPoint@@ABVQSize@@AB_NABVQString@@@Z$2 1001cd33 f   cfg_widgets001:cfg_Settings.obj
 0001:0001bd3c       __unwindfunclet$?saveState@cfg_Settings@@SAXABVQPoint@@ABVQSize@@AB_NABVQString@@@Z$3 1001cd3c f   cfg_widgets001:cfg_Settings.obj
 0001:0001bd45       __unwindfunclet$?saveState@cfg_Settings@@SAXABVQPoint@@ABVQSize@@AB_NABVQString@@@Z$4 1001cd45 f   cfg_widgets001:cfg_Settings.obj
 0001:0001bd4e       __unwindfunclet$?saveState@cfg_Settings@@SAXABVQPoint@@ABVQSize@@AB_NABVQString@@@Z$5 1001cd4e f   cfg_widgets001:cfg_Settings.obj
 0001:0001bd57       __unwindfunclet$?saveState@cfg_Settings@@SAXABVQPoint@@ABVQSize@@AB_NABVQString@@@Z$6 1001cd57 f   cfg_widgets001:cfg_Settings.obj
 0001:0001bd60       __ehhandler$?saveState@cfg_Settings@@SAXABVQPoint@@ABVQSize@@AB_NABVQString@@@Z 1001cd60 f   cfg_widgets001:cfg_Settings.obj
 0001:0001bd7b       __unwindfunclet$?saveState@cfg_Settings@@SAXABVQString@@0@Z$0 1001cd7b f   cfg_widgets001:cfg_Settings.obj
 0001:0001bd84       __unwindfunclet$?saveState@cfg_Settings@@SAXABVQString@@0@Z$1 1001cd84 f   cfg_widgets001:cfg_Settings.obj
 0001:0001bd8d       __unwindfunclet$?saveState@cfg_Settings@@SAXABVQString@@0@Z$2 1001cd8d f   cfg_widgets001:cfg_Settings.obj
 0001:0001bd96       __ehhandler$?saveState@cfg_Settings@@SAXABVQString@@0@Z 1001cd96 f   cfg_widgets001:cfg_Settings.obj
 0001:0001bdb1       __unwindfunclet$?saveState@cfg_Settings@@SAXQBVQTable@@ABVQString@@@Z$0 1001cdb1 f   cfg_widgets001:cfg_Settings.obj
 0001:0001bdb1       __unwindfunclet$?saveState@cfg_Settings@@SAXQBVQListView@@ABVQString@@@Z$0 1001cdb1 f   cfg_widgets001:cfg_Settings.obj
 0001:0001bdba       __unwindfunclet$?saveState@cfg_Settings@@SAXQBVQListView@@ABVQString@@@Z$1 1001cdba f   cfg_widgets001:cfg_Settings.obj
 0001:0001bdba       __unwindfunclet$?saveState@cfg_Settings@@SAXQBVQTable@@ABVQString@@@Z$1 1001cdba f   cfg_widgets001:cfg_Settings.obj
 0001:0001bdc3       __unwindfunclet$?saveState@cfg_Settings@@SAXQBVQTable@@ABVQString@@@Z$2 1001cdc3 f   cfg_widgets001:cfg_Settings.obj
 0001:0001bdc3       __unwindfunclet$?saveState@cfg_Settings@@SAXQBVQListView@@ABVQString@@@Z$2 1001cdc3 f   cfg_widgets001:cfg_Settings.obj
 0001:0001bdcc       __unwindfunclet$?saveState@cfg_Settings@@SAXQBVQListView@@ABVQString@@@Z$3 1001cdcc f   cfg_widgets001:cfg_Settings.obj
 0001:0001bdcc       __unwindfunclet$?saveState@cfg_Settings@@SAXQBVQTable@@ABVQString@@@Z$3 1001cdcc f   cfg_widgets001:cfg_Settings.obj
 0001:0001bdd5       __ehhandler$?saveState@cfg_Settings@@SAXQBVQTable@@ABVQString@@@Z 1001cdd5 f   cfg_widgets001:cfg_Settings.obj
 0001:0001bdd5       __ehhandler$?saveState@cfg_Settings@@SAXQBVQListView@@ABVQString@@@Z 1001cdd5 f   cfg_widgets001:cfg_Settings.obj
 0001:0001bdf0       __unwindfunclet$??0Document_BncsSystem@@QAE@XZ$0 1001cdf0 f   config_alarm_utilities:Document.obj
 0001:0001bdf9       __unwindfunclet$??0Document_BncsSystem@@QAE@XZ$1 1001cdf9 f   config_alarm_utilities:Document.obj
 0001:0001be01       __ehhandler$??0Document_BncsSystem@@QAE@XZ 1001ce01 f   config_alarm_utilities:Document.obj
 0001:0001be20       __unwindfunclet$?load@Document_BncsSystem@@QAE_NXZ$0 1001ce20 f   config_alarm_utilities:Document.obj
 0001:0001be2c       __unwindfunclet$?load@Document_BncsSystem@@QAE_NXZ$1 1001ce2c f   config_alarm_utilities:Document.obj
 0001:0001be38       __ehhandler$?load@Document_BncsSystem@@QAE_NXZ 1001ce38 f   config_alarm_utilities:Document.obj
 0001:0001be60       __unwindfunclet$??1FileLoad@@UAE@XZ$0 1001ce60 f   config_alarm_utilities:Loaders.obj
 0001:0001be60       __unwindfunclet$??0FileLoad@@IAE@ABVQString@@@Z$0 1001ce60 f   config_alarm_utilities:Loaders.obj
 0001:0001be6c       __ehhandler$??0FileLoad@@IAE@ABVQString@@@Z 1001ce6c f   config_alarm_utilities:Loaders.obj
 0001:0001be6c       __ehhandler$??1FileLoad@@UAE@XZ 1001ce6c f   config_alarm_utilities:Loaders.obj
 0001:0001be90       __unwindfunclet$??0Loaders@@QAE@XZ$0 1001ce90 f   config_alarm_utilities:Loaders.obj
 0001:0001be9b       __ehhandler$??0Loaders@@QAE@XZ 1001ce9b f   config_alarm_utilities:Loaders.obj
 0001:0001bec0       __unwindfunclet$??1Loaders@@UAE@XZ$0 1001cec0 f   config_alarm_utilities:Loaders.obj
 0001:0001becb       __unwindfunclet$??1Loaders@@UAE@XZ$1 1001cecb f   config_alarm_utilities:Loaders.obj
 0001:0001bed6       __unwindfunclet$??1Loaders@@UAE@XZ$2 1001ced6 f   config_alarm_utilities:Loaders.obj
 0001:0001bedf       __unwindfunclet$??1Loaders@@UAE@XZ$3 1001cedf f   config_alarm_utilities:Loaders.obj
 0001:0001bee8       __ehhandler$??1Loaders@@UAE@XZ 1001cee8 f   config_alarm_utilities:Loaders.obj
 0001:0001bf10       __unwindfunclet$??_G?$QPtrList@VDirLoad@@@@UAEPAXI@Z$0 1001cf10 f   config_alarm_utilities:Loaders.obj
 0001:0001bf10       __unwindfunclet$??1?$QPtrList@VFileLoad@@@@UAE@XZ$0 1001cf10 f   config_alarm_utilities:Loaders.obj
 0001:0001bf10       __unwindfunclet$??_G?$QPtrList@VFileLoad@@@@UAEPAXI@Z$0 1001cf10 f   config_alarm_utilities:Loaders.obj
 0001:0001bf10       __unwindfunclet$??1?$QPtrList@VDirLoad@@@@UAE@XZ$0 1001cf10 f   config_alarm_utilities:Loaders.obj
 0001:0001bf19       __ehhandler$??1?$QPtrList@VDirLoad@@@@UAE@XZ 1001cf19 f   config_alarm_utilities:Loaders.obj
 0001:0001bf19       __ehhandler$??_G?$QPtrList@VFileLoad@@@@UAEPAXI@Z 1001cf19 f   config_alarm_utilities:Loaders.obj
 0001:0001bf19       __ehhandler$??1?$QPtrList@VFileLoad@@@@UAE@XZ 1001cf19 f   config_alarm_utilities:Loaders.obj
 0001:0001bf19       __ehhandler$??_G?$QPtrList@VDirLoad@@@@UAEPAXI@Z 1001cf19 f   config_alarm_utilities:Loaders.obj
 0001:0001bf40       __unwindfunclet$?matches@FileLoad@@QAE_NABVQString@@@Z$0 1001cf40 f   config_alarm_utilities:Loaders.obj
 0001:0001bf49       __unwindfunclet$?matches@FileLoad@@QAE_NABVQString@@@Z$1 1001cf49 f   config_alarm_utilities:Loaders.obj
 0001:0001bf52       __unwindfunclet$?matches@FileLoad@@QAE_NABVQString@@@Z$2 1001cf52 f   config_alarm_utilities:Loaders.obj
 0001:0001bf5b       __ehhandler$?matches@FileLoad@@QAE_NABVQString@@@Z 1001cf5b f   config_alarm_utilities:Loaders.obj
 0001:0001bf80       __unwindfunclet$?request@FileLoad@@QAEXPAVISendCommand@@@Z$0 1001cf80 f   config_alarm_utilities:Loaders.obj
 0001:0001bf89       __unwindfunclet$?request@FileLoad@@QAEXPAVISendCommand@@@Z$1 1001cf89 f   config_alarm_utilities:Loaders.obj
 0001:0001bf92       __ehhandler$?request@FileLoad@@QAEXPAVISendCommand@@@Z 1001cf92 f   config_alarm_utilities:Loaders.obj
 0001:0001bfb0       ??__F?sm_sDomEncoding@alm_bncs_output@@0VQString@@B@@YAXXZ 1001cfb0 f   alm_bncs_output.obj
 0001:0001bfcf       ??__FcleanUp_manage_tempBase@@YAXXZ 1001cfcf f   moc_manage_temp.obj
 0001:0001bfda       ??__FcleanUp_manage_temp@@YAXXZ 1001cfda f   moc_manage_tempimpl.obj
 0001:0001bfe5       ??__FcleanUp_alm_bncs_output@@YAXXZ 1001cfe5 f   moc_alm_bncs_output.obj
 0001:0001bff0       ??__FcleanUp_autoNumberDialogBase@@YAXXZ 1001cff0 f   moc_autonumberdialog.obj
 0001:0001bffb       ??__FcleanUp_autoNumberDialog@@YAXXZ 1001cffb f   moc_autonumberdialogimpl.obj
 0001:0001c006       ??__FcleanUp_dialogBase@@YAXXZ 1001d006 f   moc_dialog.obj
 0001:0001c011       ??__FcleanUp_dialog@@YAXXZ 1001d011 f   moc_dialogimpl.obj
 0001:0001c020       ??__F?sm_sSystemFolder@Document@@1VQString@@A@@YAXXZ 1001d020 f   config_alarm_utilities:Document.obj
 0002:00001360       ?sm_sDomEncoding$initializer$@alm_bncs_output@@0P6AXXZA 1001f360     alm_bncs_output.obj
 0002:00001364       _cleanUp_manage_tempBase$initializer$ 1001f364     moc_manage_temp.obj
 0002:00001368       _cleanUp_manage_temp$initializer$ 1001f368     moc_manage_tempimpl.obj
 0002:0000136c       _cleanUp_alm_bncs_output$initializer$ 1001f36c     moc_alm_bncs_output.obj
 0002:00001370       _cleanUp_autoNumberDialogBase$initializer$ 1001f370     moc_autonumberdialog.obj
 0002:00001374       _cleanUp_autoNumberDialog$initializer$ 1001f374     moc_autonumberdialogimpl.obj
 0002:00001378       _cleanUp_dialogBase$initializer$ 1001f378     moc_dialog.obj
 0002:0000137c       _cleanUp_dialog$initializer$ 1001f37c     moc_dialogimpl.obj
 0002:00001380       ?sm_sSystemFolder$initializer$@Document@@1P6AXXZA 1001f380     config_alarm_utilities:Document.obj
 0002:0000138c       _pcinit                    1001f38c     MSVCRT:crtdll.obj
 0002:00001390       _pinit                     1001f390     MSVCRT:atonexit.obj
 0002:000071bc       ?slot_0@?3??staticMetaObject@manage_tempBase@@SAPAVQMetaObject@@XZ@4UQUMethod@@B 100251bc     moc_manage_temp.obj
 0002:000071d8       ?slot_tbl@?3??staticMetaObject@manage_tempBase@@SAPAVQMetaObject@@XZ@4QBUQMetaData@@B 100251d8     moc_manage_temp.obj
 0002:00007204       ?slot_0@?3??staticMetaObject@manage_temp@@SAPAVQMetaObject@@XZ@4UQUMethod@@B 10025204     moc_manage_tempimpl.obj
 0002:00007218       ?slot_1@?3??staticMetaObject@manage_temp@@SAPAVQMetaObject@@XZ@4UQUMethod@@B 10025218     moc_manage_tempimpl.obj
 0002:00007238       ?slot_2@?3??staticMetaObject@manage_temp@@SAPAVQMetaObject@@XZ@4UQUMethod@@B 10025238     moc_manage_tempimpl.obj
 0002:0000725c       ?slot_3@?3??staticMetaObject@manage_temp@@SAPAVQMetaObject@@XZ@4UQUMethod@@B 1002525c     moc_manage_tempimpl.obj
 0002:00007280       ?slot_4@?3??staticMetaObject@manage_temp@@SAPAVQMetaObject@@XZ@4UQUMethod@@B 10025280     moc_manage_tempimpl.obj
 0002:000072a8       ?slot_5@?3??staticMetaObject@manage_temp@@SAPAVQMetaObject@@XZ@4UQUMethod@@B 100252a8     moc_manage_tempimpl.obj
 0002:000072c8       ?slot_6@?3??staticMetaObject@manage_temp@@SAPAVQMetaObject@@XZ@4UQUMethod@@B 100252c8     moc_manage_tempimpl.obj
 0002:000072e0       ?slot_7@?3??staticMetaObject@manage_temp@@SAPAVQMetaObject@@XZ@4UQUMethod@@B 100252e0     moc_manage_tempimpl.obj
 0002:00007310       ?slot_8@?3??staticMetaObject@manage_temp@@SAPAVQMetaObject@@XZ@4UQUMethod@@B 10025310     moc_manage_tempimpl.obj
 0002:00007330       ?slot_9@?3??staticMetaObject@manage_temp@@SAPAVQMetaObject@@XZ@4UQUMethod@@B 10025330     moc_manage_tempimpl.obj
 0002:00007350       ?slot_10@?3??staticMetaObject@manage_temp@@SAPAVQMetaObject@@XZ@4UQUMethod@@B 10025350     moc_manage_tempimpl.obj
 0002:00007378       ?slot_11@?3??staticMetaObject@manage_temp@@SAPAVQMetaObject@@XZ@4UQUMethod@@B 10025378     moc_manage_tempimpl.obj
 0002:00007394       ?slot_12@?3??staticMetaObject@manage_temp@@SAPAVQMetaObject@@XZ@4UQUMethod@@B 10025394     moc_manage_tempimpl.obj
 0002:000073b0       ?slot_13@?3??staticMetaObject@manage_temp@@SAPAVQMetaObject@@XZ@4UQUMethod@@B 100253b0     moc_manage_tempimpl.obj
 0002:000073ec       ?slot_14@?3??staticMetaObject@manage_temp@@SAPAVQMetaObject@@XZ@4UQUMethod@@B 100253ec     moc_manage_tempimpl.obj
 0002:00007408       ?slot_tbl@?3??staticMetaObject@manage_temp@@SAPAVQMetaObject@@XZ@4QBUQMetaData@@B 10025408     moc_manage_tempimpl.obj
 0002:000089a8       ?slot_0@?3??staticMetaObject@alm_bncs_output@@SAPAVQMetaObject@@XZ@4UQUMethod@@B 100269a8     moc_alm_bncs_output.obj
 0002:000089b4       ?slot_1@?3??staticMetaObject@alm_bncs_output@@SAPAVQMetaObject@@XZ@4UQUMethod@@B 100269b4     moc_alm_bncs_output.obj
 0002:000089d0       ?slot_2@?3??staticMetaObject@alm_bncs_output@@SAPAVQMetaObject@@XZ@4UQUMethod@@B 100269d0     moc_alm_bncs_output.obj
 0002:000089ec       ?slot_3@?3??staticMetaObject@alm_bncs_output@@SAPAVQMetaObject@@XZ@4UQUMethod@@B 100269ec     moc_alm_bncs_output.obj
 0002:00008a00       ?slot_4@?3??staticMetaObject@alm_bncs_output@@SAPAVQMetaObject@@XZ@4UQUMethod@@B 10026a00     moc_alm_bncs_output.obj
 0002:00008a14       ?slot_5@?3??staticMetaObject@alm_bncs_output@@SAPAVQMetaObject@@XZ@4UQUMethod@@B 10026a14     moc_alm_bncs_output.obj
 0002:00008a28       ?slot_6@?3??staticMetaObject@alm_bncs_output@@SAPAVQMetaObject@@XZ@4UQUMethod@@B 10026a28     moc_alm_bncs_output.obj
 0002:00008a40       ?slot_7@?3??staticMetaObject@alm_bncs_output@@SAPAVQMetaObject@@XZ@4UQUMethod@@B 10026a40     moc_alm_bncs_output.obj
 0002:00008a5c       ?slot_8@?3??staticMetaObject@alm_bncs_output@@SAPAVQMetaObject@@XZ@4UQUMethod@@B 10026a5c     moc_alm_bncs_output.obj
 0002:00008a7c       ?slot_9@?3??staticMetaObject@alm_bncs_output@@SAPAVQMetaObject@@XZ@4UQUMethod@@B 10026a7c     moc_alm_bncs_output.obj
 0002:00008a94       ?slot_10@?3??staticMetaObject@alm_bncs_output@@SAPAVQMetaObject@@XZ@4UQUMethod@@B 10026a94     moc_alm_bncs_output.obj
 0002:00008aac       ?slot_11@?3??staticMetaObject@alm_bncs_output@@SAPAVQMetaObject@@XZ@4UQUMethod@@B 10026aac     moc_alm_bncs_output.obj
 0002:00008ad8       ?slot_12@?3??staticMetaObject@alm_bncs_output@@SAPAVQMetaObject@@XZ@4UQUMethod@@B 10026ad8     moc_alm_bncs_output.obj
 0002:00008af4       ?slot_13@?3??staticMetaObject@alm_bncs_output@@SAPAVQMetaObject@@XZ@4UQUMethod@@B 10026af4     moc_alm_bncs_output.obj
 0002:00008b14       ?slot_14@?3??staticMetaObject@alm_bncs_output@@SAPAVQMetaObject@@XZ@4UQUMethod@@B 10026b14     moc_alm_bncs_output.obj
 0002:00008b34       ?slot_15@?3??staticMetaObject@alm_bncs_output@@SAPAVQMetaObject@@XZ@4UQUMethod@@B 10026b34     moc_alm_bncs_output.obj
 0002:00008b50       ?slot_16@?3??staticMetaObject@alm_bncs_output@@SAPAVQMetaObject@@XZ@4UQUMethod@@B 10026b50     moc_alm_bncs_output.obj
 0002:00008b70       ?slot_tbl@?3??staticMetaObject@alm_bncs_output@@SAPAVQMetaObject@@XZ@4QBUQMetaData@@B 10026b70     moc_alm_bncs_output.obj
 0002:00008d94       ?signal_0@?3??staticMetaObject@alm_bncs_output@@SAPAVQMetaObject@@XZ@4UQUMethod@@B 10026d94     moc_alm_bncs_output.obj
 0002:00008da8       ?signal_tbl@?3??staticMetaObject@alm_bncs_output@@SAPAVQMetaObject@@XZ@4QBUQMetaData@@B 10026da8     moc_alm_bncs_output.obj
 0002:00008df8       ?slot_0@?3??staticMetaObject@autoNumberDialogBase@@SAPAVQMetaObject@@XZ@4UQUMethod@@B 10026df8     moc_autonumberdialog.obj
 0002:00008e04       ?slot_tbl@?3??staticMetaObject@autoNumberDialogBase@@SAPAVQMetaObject@@XZ@4QBUQMetaData@@B 10026e04     moc_autonumberdialog.obj
 0002:00008e24       ?slot_0@?3??staticMetaObject@dialogBase@@SAPAVQMetaObject@@XZ@4UQUMethod@@B 10026e24     moc_dialog.obj
 0002:00008e30       ?slot_tbl@?3??staticMetaObject@dialogBase@@SAPAVQMetaObject@@XZ@4QBUQMetaData@@B 10026e30     moc_dialog.obj
 0002:00008e3c       ?slot_0@?3??staticMetaObject@dialog@@SAPAVQMetaObject@@XZ@4UQUMethod@@B 10026e3c     moc_dialogimpl.obj
 0002:00008e48       ?slot_1@?3??staticMetaObject@dialog@@SAPAVQMetaObject@@XZ@4UQUMethod@@B 10026e48     moc_dialogimpl.obj
 0002:00008e64       ?slot_2@?3??staticMetaObject@dialog@@SAPAVQMetaObject@@XZ@4UQUMethod@@B 10026e64     moc_dialogimpl.obj
 0002:00008e70       ?slot_3@?3??staticMetaObject@dialog@@SAPAVQMetaObject@@XZ@4UQUMethod@@B 10026e70     moc_dialogimpl.obj
 0002:00008e94       ?slot_4@?3??staticMetaObject@dialog@@SAPAVQMetaObject@@XZ@4UQUMethod@@B 10026e94     moc_dialogimpl.obj
 0002:00008ebc       ?slot_5@?3??staticMetaObject@dialog@@SAPAVQMetaObject@@XZ@4UQUMethod@@B 10026ebc     moc_dialogimpl.obj
 0002:00008ed0       ?slot_6@?3??staticMetaObject@dialog@@SAPAVQMetaObject@@XZ@4UQUMethod@@B 10026ed0     moc_dialogimpl.obj
 0002:00008eec       ?slot_7@?3??staticMetaObject@dialog@@SAPAVQMetaObject@@XZ@4UQUMethod@@B 10026eec     moc_dialogimpl.obj
 0002:00008f04       ?slot_8@?3??staticMetaObject@dialog@@SAPAVQMetaObject@@XZ@4UQUMethod@@B 10026f04     moc_dialogimpl.obj
 0002:00008f20       ?slot_9@?3??staticMetaObject@dialog@@SAPAVQMetaObject@@XZ@4UQUMethod@@B 10026f20     moc_dialogimpl.obj
 0002:00008f40       ?slot_10@?3??staticMetaObject@dialog@@SAPAVQMetaObject@@XZ@4UQUMethod@@B 10026f40     moc_dialogimpl.obj
 0002:00008f4c       ?slot_11@?3??staticMetaObject@dialog@@SAPAVQMetaObject@@XZ@4UQUMethod@@B 10026f4c     moc_dialogimpl.obj
 0002:00008f64       ?slot_12@?3??staticMetaObject@dialog@@SAPAVQMetaObject@@XZ@4UQUMethod@@B 10026f64     moc_dialogimpl.obj
 0002:00008f84       ?slot_13@?3??staticMetaObject@dialog@@SAPAVQMetaObject@@XZ@4UQUMethod@@B 10026f84     moc_dialogimpl.obj
 0002:00008f9c       ?slot_14@?3??staticMetaObject@dialog@@SAPAVQMetaObject@@XZ@4UQUMethod@@B 10026f9c     moc_dialogimpl.obj
 0002:00008fb4       ?slot_15@?3??staticMetaObject@dialog@@SAPAVQMetaObject@@XZ@4UQUMethod@@B 10026fb4     moc_dialogimpl.obj
 0002:00008fcc       ?slot_16@?3??staticMetaObject@dialog@@SAPAVQMetaObject@@XZ@4UQUMethod@@B 10026fcc     moc_dialogimpl.obj
 0002:00008fd8       ?slot_17@?3??staticMetaObject@dialog@@SAPAVQMetaObject@@XZ@4UQUMethod@@B 10026fd8     moc_dialogimpl.obj
 0002:00008fe4       ?slot_18@?3??staticMetaObject@dialog@@SAPAVQMetaObject@@XZ@4UQUMethod@@B 10026fe4     moc_dialogimpl.obj
 0002:00009008       ?slot_tbl@?3??staticMetaObject@dialog@@SAPAVQMetaObject@@XZ@4QBUQMetaData@@B 10027008     moc_dialogimpl.obj
 0002:0000920c       ?signal_0@?3??staticMetaObject@dialog@@SAPAVQMetaObject@@XZ@4UQUMethod@@B 1002720c     moc_dialogimpl.obj
 0002:00009228       ?signal_tbl@?3??staticMetaObject@dialog@@SAPAVQMetaObject@@XZ@4QBUQMetaData@@B 10027228     moc_dialogimpl.obj
 0002:00009350       _GS_ExceptionPointers      10027350     MSVCRT:gs_report.obj
 0002:0000ae08       __unwindtable$??1QDockWindowList@@UAE@XZ 10028e08     alm_bncs_output.obj
 0002:0000ae18       __ehfuncinfo$??1QDockWindowList@@UAE@XZ 10028e18     alm_bncs_output.obj
 0002:0000ae3c       __unwindtable$??1QPopupMenuList@@UAE@XZ 10028e3c     alm_bncs_output.obj
 0002:0000ae44       __ehfuncinfo$??1QPopupMenuList@@UAE@XZ 10028e44     alm_bncs_output.obj
 0002:0000ae68       __unwindtable$??0config_plugin_base@@QAE@ABVQString@@00@Z 10028e68     alm_bncs_output.obj
 0002:0000ae88       __ehfuncinfo$??0config_plugin_base@@QAE@ABVQString@@00@Z 10028e88     alm_bncs_output.obj
 0002:0000aeac       __unwindtable$??1config_plugin_base@@UAE@XZ 10028eac     alm_bncs_output.obj
 0002:0000aec4       __ehfuncinfo$??1config_plugin_base@@UAE@XZ 10028ec4     alm_bncs_output.obj
 0002:0000aee8       __unwindtable$?about@config_plugin_base@@UAE?AVQString@@XZ 10028ee8     alm_bncs_output.obj
 0002:0000aef8       __ehfuncinfo$?about@config_plugin_base@@UAE?AVQString@@XZ 10028ef8     alm_bncs_output.obj
 0002:0000af1c       __ehfuncinfo$??0alm_bncs_output@@QAE@ABVQString@@00@Z 10028f1c     alm_bncs_output.obj
 0002:0000af40       __unwindtable$??0alm_bncs_output@@QAE@ABVQString@@00@Z 10028f40     alm_bncs_output.obj
 0002:0000b158       __ehfuncinfo$??1alm_bncs_output@@UAE@XZ 10029158     alm_bncs_output.obj
 0002:0000b17c       __unwindtable$??1alm_bncs_output@@UAE@XZ 1002917c     alm_bncs_output.obj
 0002:0000b1fc       __unwindtable$?toolbars@alm_bncs_output@@UAE?AVQDockWindowList@@XZ 100291fc     alm_bncs_output.obj
 0002:0000b204       __ehfuncinfo$?toolbars@alm_bncs_output@@UAE?AVQDockWindowList@@XZ 10029204     alm_bncs_output.obj
 0002:0000b228       __unwindtable$?menus@alm_bncs_output@@UAE?AVQPopupMenuList@@XZ 10029228     alm_bncs_output.obj
 0002:0000b230       __ehfuncinfo$?menus@alm_bncs_output@@UAE?AVQPopupMenuList@@XZ 10029230     alm_bncs_output.obj
 0002:0000b254       __ehfuncinfo$?navigate@alm_bncs_output@@UAEXABVQString@@0@Z 10029254     alm_bncs_output.obj
 0002:0000b278       __unwindtable$?navigate@alm_bncs_output@@UAEXABVQString@@0@Z 10029278     alm_bncs_output.obj
 0002:0000b300       __ehfuncinfo$?activate@alm_bncs_output@@UAEX_N@Z 10029300     alm_bncs_output.obj
 0002:0000b324       __unwindtable$?activate@alm_bncs_output@@UAEX_N@Z 10029324     alm_bncs_output.obj
 0002:0000b354       __unwindtable$?closeEvent@alm_bncs_output@@UAEXPAVQCloseEvent@@@Z 10029354     alm_bncs_output.obj
 0002:0000b374       __ehfuncinfo$?closeEvent@alm_bncs_output@@UAEXPAVQCloseEvent@@@Z 10029374     alm_bncs_output.obj
 0002:0000b398       __unwindtable$?sendCommand@alm_bncs_output@@UAEXABVQString@@0@Z 10029398     alm_bncs_output.obj
 0002:0000b3a0       __ehfuncinfo$?sendCommand@alm_bncs_output@@UAEXABVQString@@0@Z 100293a0     alm_bncs_output.obj
 0002:0000b3c4       __ehfuncinfo$?applyTemplates@alm_bncs_output@@QAEXXZ 100293c4     alm_bncs_output.obj
 0002:0000b3e8       __unwindtable$?applyTemplates@alm_bncs_output@@QAEXXZ 100293e8     alm_bncs_output.obj
 0002:0000b468       __ehfuncinfo$?manageTemplate@alm_bncs_output@@QAEXXZ 10029468     alm_bncs_output.obj
 0002:0000b48c       __unwindtable$?manageTemplate@alm_bncs_output@@QAEXXZ 1002948c     alm_bncs_output.obj
 0002:0000b574       __unwindtable$?about@alm_bncs_output@@UAE?AVQString@@XZ 10029574     alm_bncs_output.obj
 0002:0000b57c       __ehfuncinfo$?about@alm_bncs_output@@UAE?AVQString@@XZ 1002957c     alm_bncs_output.obj
 0002:0000b5a0       __unwindtable$?apply@alm_bncs_output@@UAEXXZ 100295a0     alm_bncs_output.obj
 0002:0000b5c0       __ehfuncinfo$?apply@alm_bncs_output@@UAEXXZ 100295c0     alm_bncs_output.obj
 0002:0000b5e4       __unwindtable$?markDirty@alm_bncs_output@@QAEXXZ 100295e4     alm_bncs_output.obj
 0002:0000b5ec       __ehfuncinfo$?markDirty@alm_bncs_output@@QAEXXZ 100295ec     alm_bncs_output.obj
 0002:0000b610       __ehfuncinfo$?menuDeleteFile@alm_bncs_output@@QAEXXZ 10029610     alm_bncs_output.obj
 0002:0000b634       __unwindtable$?menuDeleteFile@alm_bncs_output@@QAEXXZ 10029634     alm_bncs_output.obj
 0002:0000b66c       __ehfuncinfo$?menuDuplicateFile@alm_bncs_output@@QAEXXZ 1002966c     alm_bncs_output.obj
 0002:0000b690       __unwindtable$?menuDuplicateFile@alm_bncs_output@@QAEXXZ 10029690     alm_bncs_output.obj
 0002:0000b748       __unwindtable$?EditProcess@alm_bncs_output@@QAEXXZ 10029748     alm_bncs_output.obj
 0002:0000b768       __ehfuncinfo$?EditProcess@alm_bncs_output@@QAEXXZ 10029768     alm_bncs_output.obj
 0002:0000b78c       __ehfuncinfo$?renameModule@alm_bncs_output@@QAEXPAVQListViewItem@@HABVQString@@@Z 1002978c     alm_bncs_output.obj
 0002:0000b7b0       __unwindtable$?renameModule@alm_bncs_output@@QAEXPAVQListViewItem@@HABVQString@@@Z 100297b0     alm_bncs_output.obj
 0002:0000b810       __ehfuncinfo$?selectFile@alm_bncs_output@@QAEXPAVQListViewItem@@@Z 10029810     alm_bncs_output.obj
 0002:0000b834       __unwindtable$?selectFile@alm_bncs_output@@QAEXPAVQListViewItem@@@Z 10029834     alm_bncs_output.obj
 0002:0000b8a4       __ehfuncinfo$?selectSystem@alm_bncs_output@@IAEXABVQString@@@Z 100298a4     alm_bncs_output.obj
 0002:0000b8c8       __unwindtable$?selectSystem@alm_bncs_output@@IAEXABVQString@@@Z 100298c8     alm_bncs_output.obj
 0002:0000b968       __unwindtable$??0FileLoad_BncsSystem@alm_bncs_output@@QAE@PAV1@@Z 10029968     alm_bncs_output.obj
 0002:0000b988       __ehfuncinfo$??0FileLoad_BncsSystem@alm_bncs_output@@QAE@PAV1@@Z 10029988     alm_bncs_output.obj
 0002:0000b9ac       __unwindtable$??1FileLoad_BncsSystem@alm_bncs_output@@UAE@XZ 100299ac     alm_bncs_output.obj
 0002:0000b9b4       __ehfuncinfo$??1FileLoad_BncsSystem@alm_bncs_output@@UAE@XZ 100299b4     alm_bncs_output.obj
 0002:0000b9d8       __ehfuncinfo$?writeDeviceTypesFile@alm_bncs_output@@AAE_NQBVcOutputFile@@@Z 100299d8     alm_bncs_output.obj
 0002:0000b9fc       __unwindtable$?writeDeviceTypesFile@alm_bncs_output@@AAE_NQBVcOutputFile@@@Z 100299fc     alm_bncs_output.obj
 0002:0000bc44       __ehfuncinfo$?writeDefaultDevicetypesFile@alm_bncs_output@@AAEXXZ 10029c44     alm_bncs_output.obj
 0002:0000bc68       __unwindtable$?writeDefaultDevicetypesFile@alm_bncs_output@@AAEXXZ 10029c68     alm_bncs_output.obj
 0002:0000bd58       __ehfuncinfo$?extractParam@alm_bncs_output@@AAE?AVQString@@ABV2@0PA_N@Z 10029d58     alm_bncs_output.obj
 0002:0000bd7c       __unwindtable$?extractParam@alm_bncs_output@@AAE?AVQString@@ABV2@0PA_N@Z 10029d7c     alm_bncs_output.obj
 0002:0000bdb4       __ehfuncinfo$?writeInstances@alm_bncs_output@@AAE_NXZ 10029db4     alm_bncs_output.obj
 0002:0000bdd8       __unwindtable$?writeInstances@alm_bncs_output@@AAE_NXZ 10029dd8     alm_bncs_output.obj
 0002:0000bfe0       __ehfuncinfo$?writeNewInstanceFile@alm_bncs_output@@AAEXXZ 10029fe0     alm_bncs_output.obj
 0002:0000c004       __unwindtable$?writeNewInstanceFile@alm_bncs_output@@AAEXXZ 1002a004     alm_bncs_output.obj
 0002:0000c194       __ehfuncinfo$?insertModifiedInstances@alm_bncs_output@@AAE?AVQString@@PAV?$QDictIterator@VdevTemplate@@@@ABV2@11@Z 1002a194     alm_bncs_output.obj
 0002:0000c1b8       __unwindtable$?insertModifiedInstances@alm_bncs_output@@AAE?AVQString@@PAV?$QDictIterator@VdevTemplate@@@@ABV2@11@Z 1002a1b8     alm_bncs_output.obj
 0002:0000c298       __ehfuncinfo$?enableControls@alm_bncs_output@@AAEXXZ 1002a298     alm_bncs_output.obj
 0002:0000c2bc       __unwindtable$?enableControls@alm_bncs_output@@AAEXXZ 1002a2bc     alm_bncs_output.obj
 0002:0000c2f4       __unwindtable$?lockDevDesc@alm_bncs_output@@AAEXABVQString@@@Z 1002a2f4     alm_bncs_output.obj
 0002:0000c2f4       __unwindtable$?replyUpload@alm_bncs_output@@AAEXPAVresponse@@@Z 1002a2f4     alm_bncs_output.obj
 0002:0000c2fc       __ehfuncinfo$?lockDevDesc@alm_bncs_output@@AAEXABVQString@@@Z 1002a2fc     alm_bncs_output.obj
 0002:0000c2fc       __ehfuncinfo$?replyUpload@alm_bncs_output@@AAEXPAVresponse@@@Z 1002a2fc     alm_bncs_output.obj
 0002:0000c320       __unwindtable$?showLockedDevDescFileList@alm_bncs_output@@AAEXXZ 1002a320     alm_bncs_output.obj
 0002:0000c340       __ehfuncinfo$?showLockedDevDescFileList@alm_bncs_output@@AAEXXZ 1002a340     alm_bncs_output.obj
 0002:0000c364       __unwindtable$?changeDevType@alm_bncs_output@@AAEXABVQString@@0@Z 1002a364     alm_bncs_output.obj
 0002:0000c384       __ehfuncinfo$?changeDevType@alm_bncs_output@@AAEXABVQString@@0@Z 1002a384     alm_bncs_output.obj
 0002:0000c3a8       __ehfuncinfo$?deleteAndLockDevDescs@alm_bncs_output@@AAEXABVQString@@0@Z 1002a3a8     alm_bncs_output.obj
 0002:0000c3cc       __unwindtable$?deleteAndLockDevDescs@alm_bncs_output@@AAEXABVQString@@0@Z 1002a3cc     alm_bncs_output.obj
 0002:0000c52c       __ehfuncinfo$?changeDevTypeInstances@alm_bncs_output@@AAEXABVQString@@0@Z 1002a52c     alm_bncs_output.obj
 0002:0000c550       __unwindtable$?changeDevTypeInstances@alm_bncs_output@@AAEXABVQString@@0@Z 1002a550     alm_bncs_output.obj
 0002:0000c718       __ehfuncinfo$?writeEmptyInstancesFile@alm_bncs_output@@AAEXABVQString@@@Z 1002a718     alm_bncs_output.obj
 0002:0000c73c       __unwindtable$?writeEmptyInstancesFile@alm_bncs_output@@AAEXABVQString@@@Z 1002a73c     alm_bncs_output.obj
 0002:0000c7bc       __ehfuncinfo$?changeDevTypeDevicetypes@alm_bncs_output@@AAEXABVQString@@0@Z 1002a7bc     alm_bncs_output.obj
 0002:0000c7e0       __unwindtable$?changeDevTypeDevicetypes@alm_bncs_output@@AAEXABVQString@@0@Z 1002a7e0     alm_bncs_output.obj
 0002:0000c960       __ehfuncinfo$?writeEmptyDevicetypesFile@alm_bncs_output@@AAEXABVQString@@@Z 1002a960     alm_bncs_output.obj
 0002:0000c984       __unwindtable$?writeEmptyDevicetypesFile@alm_bncs_output@@AAEXABVQString@@@Z 1002a984     alm_bncs_output.obj
 0002:0000c9ec       __ehfuncinfo$?createEmptyDomDoc@alm_bncs_output@@EBEXABVQString@@0AAVQDomDocument@@@Z 1002a9ec     alm_bncs_output.obj
 0002:0000ca10       __unwindtable$?createEmptyDomDoc@alm_bncs_output@@EBEXABVQString@@0AAVQDomDocument@@@Z 1002aa10     alm_bncs_output.obj
 0002:0000ca68       __ehfuncinfo$?writeDomDoc@alm_bncs_output@@EBEXAAVQDomDocument@@ABVQString@@@Z 1002aa68     alm_bncs_output.obj
 0002:0000ca8c       __unwindtable$?writeDomDoc@alm_bncs_output@@EBEXAAVQDomDocument@@ABVQString@@@Z 1002aa8c     alm_bncs_output.obj
 0002:0000cad4       __ehfuncinfo$?writeDevDescFile@alm_bncs_output@@AAEXQBVcOutputFile@@_N@Z 1002aad4     alm_bncs_output.obj
 0002:0000caf8       __unwindtable$?writeDevDescFile@alm_bncs_output@@AAEXQBVcOutputFile@@_N@Z 1002aaf8     alm_bncs_output.obj
 0002:0000cc80       __ehfuncinfo$?ensureFolderExists@alm_bncs_output@@AAE_NABVQString@@@Z 1002ac80     alm_bncs_output.obj
 0002:0000cca4       __unwindtable$?ensureFolderExists@alm_bncs_output@@AAE_NABVQString@@@Z 1002aca4     alm_bncs_output.obj
 0002:0000ccdc       __ehfuncinfo$?updateFileList@alm_bncs_output@@AAEXXZ 1002acdc     alm_bncs_output.obj
 0002:0000cd00       __unwindtable$?updateFileList@alm_bncs_output@@AAEXXZ 1002ad00     alm_bncs_output.obj
 0002:0000ce88       __ehfuncinfo$?loadFile@alm_bncs_output@@AAE_NABVQString@@@Z 1002ae88     alm_bncs_output.obj
 0002:0000ceac       __unwindtable$?loadFile@alm_bncs_output@@AAE_NABVQString@@@Z 1002aeac     alm_bncs_output.obj
 0002:0000cffc       __ehfuncinfo$?saveTemplates@alm_bncs_output@@AAEXPBVcOutputFile@@_NAAVQString@@2@Z 1002affc     alm_bncs_output.obj
 0002:0000d020       __unwindtable$?saveTemplates@alm_bncs_output@@AAEXPBVcOutputFile@@_NAAVQString@@2@Z 1002b020     alm_bncs_output.obj
 0002:0000d140       __ehfuncinfo$?loadTemplates@alm_bncs_output@@AAEXABVQStringList@@ABV?$QMap@VQString@@V1@@@@Z 1002b140     alm_bncs_output.obj
 0002:0000d164       __unwindtable$?loadTemplates@alm_bncs_output@@AAEXABVQStringList@@ABV?$QMap@VQString@@V1@@@@Z 1002b164     alm_bncs_output.obj
 0002:0000d214       __ehfuncinfo$?saveFile@alm_bncs_output@@AAE_NQAVcOutputFile@@_N1@Z 1002b214     alm_bncs_output.obj
 0002:0000d238       __unwindtable$?saveFile@alm_bncs_output@@AAE_NQAVcOutputFile@@_N1@Z 1002b238     alm_bncs_output.obj
 0002:0000d2d0       __ehfuncinfo$?newFile@alm_bncs_output@@AAEXABVQString@@@Z 1002b2d0     alm_bncs_output.obj
 0002:0000d2f4       __unwindtable$?newFile@alm_bncs_output@@AAEXABVQString@@@Z 1002b2f4     alm_bncs_output.obj
 0002:0000d3ec       __ehfuncinfo$?loadProcesses@alm_bncs_output@@AAE_NABVQString@@@Z 1002b3ec     alm_bncs_output.obj
 0002:0000d410       __unwindtable$?loadProcesses@alm_bncs_output@@AAE_NABVQString@@@Z 1002b410     alm_bncs_output.obj
 0002:0000d498       __unwindtable$?replyDownload@alm_bncs_output@@AAEXPAVresponse@@@Z 1002b498     alm_bncs_output.obj
 0002:0000d4b0       __ehfuncinfo$?replyDownload@alm_bncs_output@@AAEXPAVresponse@@@Z 1002b4b0     alm_bncs_output.obj
 0002:0000d4d4       __ehfuncinfo$?doDownloadRead@alm_bncs_output@@AAEXPAVresponse@@@Z 1002b4d4     alm_bncs_output.obj
 0002:0000d4f8       __unwindtable$?doDownloadRead@alm_bncs_output@@AAEXPAVresponse@@@Z 1002b4f8     alm_bncs_output.obj
 0002:0000d620       __ehfuncinfo$?doDone@alm_bncs_output@@AAEXPAVresponse@@@Z 1002b620     alm_bncs_output.obj
 0002:0000d644       __unwindtable$?doDone@alm_bncs_output@@AAEXPAVresponse@@@Z 1002b644     alm_bncs_output.obj
 0002:0000d6f4       __ehfuncinfo$?replyLock@alm_bncs_output@@AAEXPAVresponse@@@Z 1002b6f4     alm_bncs_output.obj
 0002:0000d718       __unwindtable$?replyLock@alm_bncs_output@@AAEXPAVresponse@@@Z 1002b718     alm_bncs_output.obj
 0002:0000d7a0       __ehfuncinfo$?allocateCfgFileName@alm_bncs_output@@AAEXAAVQString@@0@Z 1002b7a0     alm_bncs_output.obj
 0002:0000d7c4       __unwindtable$?allocateCfgFileName@alm_bncs_output@@AAEXAAVQString@@0@Z 1002b7c4     alm_bncs_output.obj
 0002:0000d7fc       __unwindtable$?allocateModuleName@alm_bncs_output@@AAEXAAVQString@@@Z 1002b7fc     alm_bncs_output.obj
 0002:0000d80c       __ehfuncinfo$?allocateModuleName@alm_bncs_output@@AAEXAAVQString@@@Z 1002b80c     alm_bncs_output.obj
 0002:0000d830       __unwindtable$??1?$QPtrList@VcOutputFile@@@@UAE@XZ 1002b830     alm_bncs_output.obj
 0002:0000d830       __unwindtable$??1?$QPtrList@VQPopupMenu@@@@UAE@XZ 1002b830     alm_bncs_output.obj
 0002:0000d838       __ehfuncinfo$??1?$QPtrList@VQPopupMenu@@@@UAE@XZ 1002b838     alm_bncs_output.obj
 0002:0000d838       __ehfuncinfo$??1?$QPtrList@VcOutputFile@@@@UAE@XZ 1002b838     alm_bncs_output.obj
 0002:0000d85c       __unwindtable$??4?$QGuardedPtr@VQPopupMenu@@@@QAEAAV0@PAVQPopupMenu@@@Z 1002b85c     alm_bncs_output.obj
 0002:0000d85c       __unwindtable$?create@plugindesc@@UAEPAVconfig_plugin_base@@ABVQString@@00@Z 1002b85c     alm_bncs_output.obj
 0002:0000d85c       __unwindtable$??0?$QMapPrivate@VQString@@W4ESection@@@@QAE@XZ 1002b85c     alm_bncs_output.obj
 0002:0000d85c       __unwindtable$??0?$QGuardedPtr@VQPopupMenu@@@@QAE@XZ 1002b85c     alm_bncs_output.obj
 0002:0000d85c       __unwindtable$?insert@?$QMapPrivate@VQString@@W4ESection@@@@QAE?AV?$QMapIterator@VQString@@W4ESection@@@@PAUQMapNodeBase@@0ABVQString@@@Z 1002b85c     alm_bncs_output.obj
 0002:0000d85c       __unwindtable$??4?$QGuardedPtr@VQDockWindow@@@@QAEAAV0@PAVQDockWindow@@@Z 1002b85c     alm_bncs_output.obj
 0002:0000d85c       __unwindtable$??0?$QMap@VQString@@W4ESection@@@@QAE@XZ 1002b85c     alm_bncs_output.obj
 0002:0000d85c       __unwindtable$?detachInternal@?$QMap@VQString@@W4ESection@@@@AAEXXZ 1002b85c     alm_bncs_output.obj
 0002:0000d85c       __unwindtable$??0?$QGuardedPtr@VQDockWindow@@@@QAE@XZ 1002b85c     alm_bncs_output.obj
 0002:0000d864       __ehfuncinfo$??0?$QMap@VQString@@W4ESection@@@@QAE@XZ 1002b864     alm_bncs_output.obj
 0002:0000d864       __ehfuncinfo$?detachInternal@?$QMap@VQString@@W4ESection@@@@AAEXXZ 1002b864     alm_bncs_output.obj
 0002:0000d864       __ehfuncinfo$??0?$QMapPrivate@VQString@@W4ESection@@@@QAE@XZ 1002b864     alm_bncs_output.obj
 0002:0000d864       __ehfuncinfo$??0?$QGuardedPtr@VQDockWindow@@@@QAE@XZ 1002b864     alm_bncs_output.obj
 0002:0000d864       __ehfuncinfo$?create@plugindesc@@UAEPAVconfig_plugin_base@@ABVQString@@00@Z 1002b864     alm_bncs_output.obj
 0002:0000d864       __ehfuncinfo$??0?$QGuardedPtr@VQPopupMenu@@@@QAE@XZ 1002b864     alm_bncs_output.obj
 0002:0000d864       __ehfuncinfo$?insert@?$QMapPrivate@VQString@@W4ESection@@@@QAE?AV?$QMapIterator@VQString@@W4ESection@@@@PAUQMapNodeBase@@0ABVQString@@@Z 1002b864     alm_bncs_output.obj
 0002:0000d864       __ehfuncinfo$??4?$QGuardedPtr@VQDockWindow@@@@QAEAAV0@PAVQDockWindow@@@Z 1002b864     alm_bncs_output.obj
 0002:0000d864       __ehfuncinfo$??4?$QGuardedPtr@VQPopupMenu@@@@QAEAAV0@PAVQPopupMenu@@@Z 1002b864     alm_bncs_output.obj
 0002:0000d888       __unwindtable$?copy@?$QMapPrivate@VQString@@W4ESection@@@@QAEPAU?$QMapNode@VQString@@W4ESection@@@@PAU2@@Z 1002b888     alm_bncs_output.obj
 0002:0000d888       __unwindtable$??0?$QMapPrivate@VQString@@W4ESection@@@@QAE@PBV0@@Z 1002b888     alm_bncs_output.obj
 0002:0000d890       __ehfuncinfo$??0?$QMapPrivate@VQString@@W4ESection@@@@QAE@PBV0@@Z 1002b890     alm_bncs_output.obj
 0002:0000d890       __ehfuncinfo$?copy@?$QMapPrivate@VQString@@W4ESection@@@@QAEPAU?$QMapNode@VQString@@W4ESection@@@@PAU2@@Z 1002b890     alm_bncs_output.obj
 0002:0000d8b4       __unwindtable$??0?$QMapNode@VQString@@W4ESection@@@@QAE@ABU0@@Z 1002b8b4     alm_bncs_output.obj
 0002:0000d8b4       __unwindtable$??0?$QMapNode@VQString@@W4ESection@@@@QAE@ABVQString@@@Z 1002b8b4     alm_bncs_output.obj
 0002:0000d8bc       __ehfuncinfo$??0?$QMapNode@VQString@@W4ESection@@@@QAE@ABU0@@Z 1002b8bc     alm_bncs_output.obj
 0002:0000d8bc       __ehfuncinfo$??0?$QMapNode@VQString@@W4ESection@@@@QAE@ABVQString@@@Z 1002b8bc     alm_bncs_output.obj
 0002:0000d8e0       __unwindtable$??0cOutputFile@@QAE@XZ 1002b8e0     cOutputFile.obj
 0002:0000d8e0       __unwindtable$??1cOutputFile@@UAE@XZ 1002b8e0     cOutputFile.obj
 0002:0000d8e0       __unwindtable$??0cOutputFile@@QAE@ABVQString@@00@Z 1002b8e0     cOutputFile.obj
 0002:0000d8f0       __ehfuncinfo$??0cOutputFile@@QAE@XZ 1002b8f0     cOutputFile.obj
 0002:0000d8f0       __ehfuncinfo$??1cOutputFile@@UAE@XZ 1002b8f0     cOutputFile.obj
 0002:0000d8f0       __ehfuncinfo$??0cOutputFile@@QAE@ABVQString@@00@Z 1002b8f0     cOutputFile.obj
 0002:0000d914       __ehfuncinfo$??0devTemplate@@QAE@ABVQString@@@Z 1002b914     devTemplate.obj
 0002:0000d938       __unwindtable$??0devTemplate@@QAE@ABVQString@@@Z 1002b938     devTemplate.obj
 0002:0000d998       __unwindtable$??1devTemplate@@UAE@XZ 1002b998     devTemplate.obj
 0002:0000d9b0       __ehfuncinfo$??1devTemplate@@UAE@XZ 1002b9b0     devTemplate.obj
 0002:0000d9d4       __ehfuncinfo$?saveFile@devTemplate@@QBE_NABVQString@@0QBVIDomDoc@@QAVIGetDocuments@@@Z 1002b9d4     devTemplate.obj
 0002:0000d9f8       __unwindtable$?saveFile@devTemplate@@QBE_NABVQString@@0QBVIDomDoc@@QAVIGetDocuments@@@Z 1002b9f8     devTemplate.obj
 0002:0000da98       __ehfuncinfo$?loadDevDesc@devTemplate@@QAE_NABVQString@@0@Z 1002ba98     devTemplate.obj
 0002:0000dabc       __unwindtable$?loadDevDesc@devTemplate@@QAE_NABVQString@@0@Z 1002babc     devTemplate.obj
 0002:0000db54       __unwindtable$??1?$QDict@VdevTemplate@@@@UAE@XZ 1002bb54     devTemplate.obj
 0002:0000db5c       __ehfuncinfo$??1?$QDict@VdevTemplate@@@@UAE@XZ 1002bb5c     devTemplate.obj
 0002:0000db80       __ehfuncinfo$??0dialog@@QAE@PAVIGetDocuments@@PAVQWidget@@PBDI@Z 1002bb80     dialogimpl.obj
 0002:0000dba4       __unwindtable$??0dialog@@QAE@PAVIGetDocuments@@PAVQWidget@@PBDI@Z 1002bba4     dialogimpl.obj
 0002:0000dc7c       __unwindtable$??1dialog@@UAE@XZ 1002bc7c     dialogimpl.obj
 0002:0000dc9c       __ehfuncinfo$??1dialog@@UAE@XZ 1002bc9c     dialogimpl.obj
 0002:0000dcc0       __unwindtable$?clearSelectableSlots@dialog@@QAEXXZ 1002bcc0     dialogimpl.obj
 0002:0000dcc0       __unwindtable$?clearSelectedSlots@dialog@@QAEXXZ 1002bcc0     dialogimpl.obj
 0002:0000dcc0       __unwindtable$?clearAllSlots@dialog@@QAEXXZ 1002bcc0     dialogimpl.obj
 0002:0000dce0       __ehfuncinfo$?clearAllSlots@dialog@@QAEXXZ 1002bce0     dialogimpl.obj
 0002:0000dce0       __ehfuncinfo$?clearSelectedSlots@dialog@@QAEXXZ 1002bce0     dialogimpl.obj
 0002:0000dce0       __ehfuncinfo$?clearSelectableSlots@dialog@@QAEXXZ 1002bce0     dialogimpl.obj
 0002:0000dd04       __ehfuncinfo$?clearSlots@dialog@@QAEXXZ 1002bd04     dialogimpl.obj
 0002:0000dd28       __unwindtable$?clearSlots@dialog@@QAEXXZ 1002bd28     dialogimpl.obj
 0002:0000dd68       __unwindtable$?changeSelection@dialog@@QAEXXZ 1002bd68     dialogimpl.obj
 0002:0000dd78       __ehfuncinfo$?changeSelection@dialog@@QAEXXZ 1002bd78     dialogimpl.obj
 0002:0000dd9c       __ehfuncinfo$?autoNumber@dialog@@QAEXXZ 1002bd9c     dialogimpl.obj
 0002:0000ddc0       __unwindtable$?autoNumber@dialog@@QAEXXZ 1002bdc0     dialogimpl.obj
 0002:0000de20       __ehfuncinfo$?clipboardDataChange@dialog@@QAEXXZ 1002be20     dialogimpl.obj
 0002:0000de44       __unwindtable$?clipboardDataChange@dialog@@QAEXXZ 1002be44     dialogimpl.obj
 0002:0000de7c       __ehfuncinfo$?pasteData@dialog@@QAEXXZ 1002be7c     dialogimpl.obj
 0002:0000dea0       __unwindtable$?pasteData@dialog@@QAEXXZ 1002bea0     dialogimpl.obj
 0002:0000df30       __ehfuncinfo$?copyData@dialog@@QAEXXZ 1002bf30     dialogimpl.obj
 0002:0000df54       __unwindtable$?copyData@dialog@@QAEXXZ 1002bf54     dialogimpl.obj
 0002:0000df84       __unwindtable$?selectProc@dialog@@QAEXPAVQListViewItem@@@Z 1002bf84     dialogimpl.obj
 0002:0000df8c       __ehfuncinfo$?selectProc@dialog@@QAEXPAVQListViewItem@@@Z 1002bf8c     dialogimpl.obj
 0002:0000dfb0       __ehfuncinfo$?slotChange@dialog@@QAEXPAVQListViewItem@@HABVQString@@@Z 1002bfb0     dialogimpl.obj
 0002:0000dfd4       __unwindtable$?slotChange@dialog@@QAEXPAVQListViewItem@@HABVQString@@@Z 1002bfd4     dialogimpl.obj
 0002:0000e004       __ehfuncinfo$?checkForDuplicates@dialog@@QAE_NXZ 1002c004     dialogimpl.obj
 0002:0000e028       __unwindtable$?checkForDuplicates@dialog@@QAE_NXZ 1002c028     dialogimpl.obj
 0002:0000e058       __ehfuncinfo$??0manage_tempBase@@QAE@PAVQWidget@@PBD_NI@Z 1002c058     manage_temp.obj
 0002:0000e07c       __unwindtable$??0manage_tempBase@@QAE@PAVQWidget@@PBD_NI@Z 1002c07c     manage_temp.obj
 0002:0000e1cc       __ehfuncinfo$?languageChange@manage_tempBase@@MAEXXZ 1002c1cc     manage_temp.obj
 0002:0000e1f0       __unwindtable$?languageChange@manage_tempBase@@MAEXXZ 1002c1f0     manage_temp.obj
 0002:0000e2a8       __ehfuncinfo$??0manage_temp@@QAE@ABVQStringList@@QBVTemplateList@@QAVIGetDocuments@@PAVQWidget@@PBD_NI@Z 1002c2a8     manage_tempimpl.obj
 0002:0000e2cc       __unwindtable$??0manage_temp@@QAE@ABVQStringList@@QBVTemplateList@@QAVIGetDocuments@@PAVQWidget@@PBD_NI@Z 1002c2cc     manage_tempimpl.obj
 0002:0000e30c       __ehfuncinfo$??1manage_temp@@UAE@XZ 1002c30c     manage_tempimpl.obj
 0002:0000e330       __unwindtable$??1manage_temp@@UAE@XZ 1002c330     manage_tempimpl.obj
 0002:0000e370       __ehfuncinfo$?newTemplate@manage_temp@@QAEXXZ 1002c370     manage_tempimpl.obj
 0002:0000e394       __unwindtable$?newTemplate@manage_temp@@QAEXXZ 1002c394     manage_tempimpl.obj
 0002:0000e3e4       __unwindtable$?saveCurrentTemplate@manage_temp@@QAEXXZ 1002c3e4     manage_tempimpl.obj
 0002:0000e404       __ehfuncinfo$?saveCurrentTemplate@manage_temp@@QAEXXZ 1002c404     manage_tempimpl.obj
 0002:0000e428       __ehfuncinfo$?changePrefix@manage_temp@@QAEXABVQString@@@Z 1002c428     manage_tempimpl.obj
 0002:0000e44c       __unwindtable$?changePrefix@manage_temp@@QAEXABVQString@@@Z 1002c44c     manage_tempimpl.obj
 0002:0000e4a4       __unwindtable$?selectTemplate@manage_temp@@QAEXABVQString@@@Z 1002c4a4     manage_tempimpl.obj
 0002:0000e4bc       __ehfuncinfo$?selectTemplate@manage_temp@@QAEXABVQString@@@Z 1002c4bc     manage_tempimpl.obj
 0002:0000e4e0       __unwindtable$?autoNumberSlots@manage_temp@@QAEXXZ 1002c4e0     manage_tempimpl.obj
 0002:0000e4f8       __ehfuncinfo$?autoNumberSlots@manage_temp@@QAEXXZ 1002c4f8     manage_tempimpl.obj
 0002:0000e51c       __unwindtable$?clearSlots@manage_temp@@QAEXXZ 1002c51c     manage_tempimpl.obj
 0002:0000e534       __ehfuncinfo$?clearSlots@manage_temp@@QAEXXZ 1002c534     manage_tempimpl.obj
 0002:0000e558       __unwindtable$?getTemplates@manage_temp@@QAEXQAVTemplateList@@@Z 1002c558     manage_tempimpl.obj
 0002:0000e570       __ehfuncinfo$?getTemplates@manage_temp@@QAEXQAVTemplateList@@@Z 1002c570     manage_tempimpl.obj
 0002:0000e594       __ehfuncinfo$?loadTemplates@manage_temp@@AAEXABVQStringList@@QBVTemplateList@@@Z 1002c594     manage_tempimpl.obj
 0002:0000e5b8       __unwindtable$?loadTemplates@manage_temp@@AAEXABVQStringList@@QBVTemplateList@@@Z 1002c5b8     manage_tempimpl.obj
 0002:0000e5e8       __ehfuncinfo$?updateInstanceDisplay@manage_temp@@AAEXXZ 1002c5e8     manage_tempimpl.obj
 0002:0000e60c       __unwindtable$?updateInstanceDisplay@manage_temp@@AAEXXZ 1002c60c     manage_tempimpl.obj
 0002:0000e65c       __unwindtable$?keys@plugindesc@@UAE?AVQStringList@@ABVQString@@0@Z 1002c65c     plugindesc.obj
 0002:0000e66c       __ehfuncinfo$?keys@plugindesc@@UAE?AVQStringList@@ABVQString@@0@Z 1002c66c     plugindesc.obj
 0002:0000e690       __ehfuncinfo$??0processItem@@QAE@PAVQListView@@VQString@@1@Z 1002c690     processItem.obj
 0002:0000e6b4       __unwindtable$??0processItem@@QAE@PAVQListView@@VQString@@1@Z 1002c6b4     processItem.obj
 0002:0000e6fc       __unwindtable$?paintCell@processItem@@UAEXPAVQPainter@@ABVQColorGroup@@HHH@Z 1002c6fc     processItem.obj
 0002:0000e704       __ehfuncinfo$?paintCell@processItem@@UAEXPAVQPainter@@ABVQColorGroup@@HHH@Z 1002c704     processItem.obj
 0002:0000e728       __unwindtable$?compare@processItem@@UBEHPAVQListViewItem@@H_N@Z 1002c728     processItem.obj
 0002:0000e748       __ehfuncinfo$?compare@processItem@@UBEHPAVQListViewItem@@H_N@Z 1002c748     processItem.obj
 0002:0000e76c       __ehfuncinfo$??0autoNumberDialogBase@@QAE@PAVQWidget@@PBD_NI@Z 1002c76c     autonumberdialog.obj
 0002:0000e790       __unwindtable$??0autoNumberDialogBase@@QAE@PAVQWidget@@PBD_NI@Z 1002c790     autonumberdialog.obj
 0002:0000e820       __ehfuncinfo$?languageChange@autoNumberDialogBase@@MAEXXZ 1002c820     autonumberdialog.obj
 0002:0000e844       __unwindtable$?languageChange@autoNumberDialogBase@@MAEXXZ 1002c844     autonumberdialog.obj
 0002:0000e8b4       __ehfuncinfo$??0dialogBase@@QAE@PAVQWidget@@PBDI@Z 1002c8b4     dialog.obj
 0002:0000e8d8       __unwindtable$??0dialogBase@@QAE@PAVQWidget@@PBDI@Z 1002c8d8     dialog.obj
 0002:0000e9c8       __ehfuncinfo$?languageChange@dialogBase@@MAEXXZ 1002c9c8     dialog.obj
 0002:0000e9ec       __unwindtable$?languageChange@dialogBase@@MAEXXZ 1002c9ec     dialog.obj
 0002:0000eb1c       __unwindtable$?menuNewFile@alm_bncs_output@@QAEXXZ 1002cb1c     moc_alm_bncs_output.obj
 0002:0000eb1c       __unwindtable$?qt_invoke@dialog@@UAE_NHPAUQUObject@@@Z 1002cb1c     moc_alm_bncs_output.obj
 0002:0000eb1c       __unwindtable$?qt_invoke@alm_bncs_output@@UAE_NHPAUQUObject@@@Z 1002cb1c     moc_alm_bncs_output.obj
 0002:0000eb24       __ehfuncinfo$?qt_invoke@dialog@@UAE_NHPAUQUObject@@@Z 1002cb24     moc_alm_bncs_output.obj
 0002:0000eb24       __ehfuncinfo$?qt_invoke@alm_bncs_output@@UAE_NHPAUQUObject@@@Z 1002cb24     moc_alm_bncs_output.obj
 0002:0000eb24       __ehfuncinfo$?menuNewFile@alm_bncs_output@@QAEXXZ 1002cb24     moc_alm_bncs_output.obj
 0002:0000eb48       __unwindtable$?qt_emit@alm_bncs_output@@UAE_NHPAUQUObject@@@Z 1002cb48     moc_alm_bncs_output.obj
 0002:0000eb50       __ehfuncinfo$?qt_emit@alm_bncs_output@@UAE_NHPAUQUObject@@@Z 1002cb50     moc_alm_bncs_output.obj
 0002:0000eb74       __unwindtable$?command@alm_bncs_output@@IAEXVQString@@0@Z 1002cb74     moc_alm_bncs_output.obj
 0002:0000eb8c       __ehfuncinfo$?command@alm_bncs_output@@IAEXVQString@@0@Z 1002cb8c     moc_alm_bncs_output.obj
 0002:0000ebb0       __unwindtable$?saveState@cfg_Settings@@SAXABVQString@@0@Z 1002cbb0     cfg_widgets001:cfg_Settings.obj
 0002:0000ebc8       __ehfuncinfo$?saveState@cfg_Settings@@SAXABVQString@@0@Z 1002cbc8     cfg_widgets001:cfg_Settings.obj
 0002:0000ebec       __ehfuncinfo$?saveState@cfg_Settings@@SAXQBVQTable@@ABVQString@@@Z 1002cbec     cfg_widgets001:cfg_Settings.obj
 0002:0000ebec       __ehfuncinfo$?saveState@cfg_Settings@@SAXQBVQListView@@ABVQString@@@Z 1002cbec     cfg_widgets001:cfg_Settings.obj
 0002:0000ec10       __unwindtable$?saveState@cfg_Settings@@SAXQBVQTable@@ABVQString@@@Z 1002cc10     cfg_widgets001:cfg_Settings.obj
 0002:0000ec10       __unwindtable$?saveState@cfg_Settings@@SAXQBVQListView@@ABVQString@@@Z 1002cc10     cfg_widgets001:cfg_Settings.obj
 0002:0000ec38       __ehfuncinfo$?saveState@cfg_Settings@@SAXABVQPoint@@ABVQSize@@AB_NABVQString@@@Z 1002cc38     cfg_widgets001:cfg_Settings.obj
 0002:0000ec5c       __unwindtable$?saveState@cfg_Settings@@SAXABVQPoint@@ABVQSize@@AB_NABVQString@@@Z 1002cc5c     cfg_widgets001:cfg_Settings.obj
 0002:0000ec94       __unwindtable$?loadState@cfg_Settings@@SA?AVQString@@ABV2@@Z 1002cc94     cfg_widgets001:cfg_Settings.obj
 0002:0000ecb4       __ehfuncinfo$?loadState@cfg_Settings@@SA?AVQString@@ABV2@@Z 1002ccb4     cfg_widgets001:cfg_Settings.obj
 0002:0000ecd8       __unwindtable$?loadState@cfg_Settings@@SAXQAVQListView@@ABVQString@@@Z 1002ccd8     cfg_widgets001:cfg_Settings.obj
 0002:0000ecd8       __unwindtable$?loadState@cfg_Settings@@SAXQAVQTable@@ABVQString@@@Z 1002ccd8     cfg_widgets001:cfg_Settings.obj
 0002:0000ece8       __ehfuncinfo$?loadState@cfg_Settings@@SAXQAVQListView@@ABVQString@@@Z 1002cce8     cfg_widgets001:cfg_Settings.obj
 0002:0000ece8       __ehfuncinfo$?loadState@cfg_Settings@@SAXQAVQTable@@ABVQString@@@Z 1002cce8     cfg_widgets001:cfg_Settings.obj
 0002:0000ed0c       __unwindtable$?loadState@cfg_Settings@@SAXAAVQPoint@@AAVQSize@@AA_NABVQString@@@Z 1002cd0c     cfg_widgets001:cfg_Settings.obj
 0002:0000ed1c       __ehfuncinfo$?loadState@cfg_Settings@@SAXAAVQPoint@@AAVQSize@@AA_NABVQString@@@Z 1002cd1c     cfg_widgets001:cfg_Settings.obj
 0002:0000ed40       __unwindtable$??0Document_BncsSystem@@QAE@XZ 1002cd40     config_alarm_utilities:Document.obj
 0002:0000ed58       __ehfuncinfo$??0Document_BncsSystem@@QAE@XZ 1002cd58     config_alarm_utilities:Document.obj
 0002:0000ed7c       __unwindtable$?load@Document_BncsSystem@@QAE_NXZ 1002cd7c     config_alarm_utilities:Document.obj
 0002:0000ed94       __ehfuncinfo$?load@Document_BncsSystem@@QAE_NXZ 1002cd94     config_alarm_utilities:Document.obj
 0002:0000edb8       __unwindtable$??0FileLoad@@IAE@ABVQString@@@Z 1002cdb8     config_alarm_utilities:Loaders.obj
 0002:0000edb8       __unwindtable$??1FileLoad@@UAE@XZ 1002cdb8     config_alarm_utilities:Loaders.obj
 0002:0000edc0       __ehfuncinfo$??0FileLoad@@IAE@ABVQString@@@Z 1002cdc0     config_alarm_utilities:Loaders.obj
 0002:0000edc0       __ehfuncinfo$??1FileLoad@@UAE@XZ 1002cdc0     config_alarm_utilities:Loaders.obj
 0002:0000ede4       __unwindtable$?matches@FileLoad@@QAE_NABVQString@@@Z 1002cde4     config_alarm_utilities:Loaders.obj
 0002:0000edfc       __ehfuncinfo$?matches@FileLoad@@QAE_NABVQString@@@Z 1002cdfc     config_alarm_utilities:Loaders.obj
 0002:0000ee20       __unwindtable$?request@FileLoad@@QAEXPAVISendCommand@@@Z 1002ce20     config_alarm_utilities:Loaders.obj
 0002:0000ee30       __ehfuncinfo$?request@FileLoad@@QAEXPAVISendCommand@@@Z 1002ce30     config_alarm_utilities:Loaders.obj
 0002:0000ee54       __unwindtable$??0Loaders@@QAE@XZ 1002ce54     config_alarm_utilities:Loaders.obj
 0002:0000ee5c       __ehfuncinfo$??0Loaders@@QAE@XZ 1002ce5c     config_alarm_utilities:Loaders.obj
 0002:0000ee80       __unwindtable$??1Loaders@@UAE@XZ 1002ce80     config_alarm_utilities:Loaders.obj
 0002:0000eea0       __ehfuncinfo$??1Loaders@@UAE@XZ 1002cea0     config_alarm_utilities:Loaders.obj
 0002:0000eec4       __unwindtable$??1?$QPtrList@VFileLoad@@@@UAE@XZ 1002cec4     config_alarm_utilities:Loaders.obj
 0002:0000eec4       __unwindtable$??1?$QPtrList@VDirLoad@@@@UAE@XZ 1002cec4     config_alarm_utilities:Loaders.obj
 0002:0000eec4       __unwindtable$??_G?$QPtrList@VFileLoad@@@@UAEPAXI@Z 1002cec4     config_alarm_utilities:Loaders.obj
 0002:0000eec4       __unwindtable$??_G?$QPtrList@VDirLoad@@@@UAEPAXI@Z 1002cec4     config_alarm_utilities:Loaders.obj
 0002:0000eecc       __ehfuncinfo$??1?$QPtrList@VDirLoad@@@@UAE@XZ 1002cecc     config_alarm_utilities:Loaders.obj
 0002:0000eecc       __ehfuncinfo$??1?$QPtrList@VFileLoad@@@@UAE@XZ 1002cecc     config_alarm_utilities:Loaders.obj
 0002:0000eecc       __ehfuncinfo$??_G?$QPtrList@VDirLoad@@@@UAEPAXI@Z 1002cecc     config_alarm_utilities:Loaders.obj
 0002:0000eecc       __ehfuncinfo$??_G?$QPtrList@VFileLoad@@@@UAEPAXI@Z 1002cecc     config_alarm_utilities:Loaders.obj
 0002:0000eef0       __sehtable$__onexit        1002cef0     MSVCRT:atonexit.obj
 0002:0000ef10       __sehtable$??_L@YGXPAXIHP6EX0@Z1@Z 1002cf10     MSVCRT:ehvecctr.obj
 0002:0000ef30       __sehtable$??_M@YGXPAXIHP6EX0@Z@Z 1002cf30     MSVCRT:ehvecdtr.obj
 0002:0000ef50       __sehtable$?__ArrayUnwind@@YGXPAXIHP6EX0@Z@Z 1002cf50     MSVCRT:ehvecdtr.obj
 0002:0000ef70       __sehtable$___DllMainCRTStartup 1002cf70     MSVCRT:crtdll.obj
 0002:0000ef98       __sehtable$__IsNonwritableInCurrentImage 1002cf98     MSVCRT:pesect.obj
 0002:0000efc0       .edata                     1002cfc0     config_alm_bncs_output.exp
 0002:0000efe8       rgpv                       1002cfe8     config_alm_bncs_output.exp
 0002:0000efec       rgszName                   1002cfec     config_alm_bncs_output.exp
 0002:0000eff0       rgwOrd                     1002cff0     config_alm_bncs_output.exp
 0002:0000eff2       szName                     1002cff2     config_alm_bncs_output.exp
 0002:0000f00d       $N00001                    1002d00d     config_alm_bncs_output.exp
 0002:00010434       .idata$6                   1002e434     config_icons:config_icons.dll
 0002:0001c6b8       .idata$6                   1003a6b8     qt-mt323:qt-mt323.dll
 0002:0001c89e       .idata$6                   1003a89e     alm_sys_select:alm_sys_select.dll
 0002:0001c8ce       .idata$6                   1003a8ce     kernel32:KERNEL32.dll
 0002:0001c930       .idata$6                   1003a930     MSVCRT:MSVCR120.dll
 0002:0001cab2       .idata$6                   1003aab2     msvcprt:MSVCP120.dll
 0003:00000000       ?iBase@?1??autoNumber@dialog@@QAEXXZ@4HA 1003b000     dialogimpl.obj
 0003:00000004       ?param_slot_10@?3??staticMetaObject@manage_temp@@SAPAVQMetaObject@@XZ@4QBUQUParameter@@B 1003b004     moc_manage_tempimpl.obj
 0003:00000014       ?param_slot_11@?3??staticMetaObject@manage_temp@@SAPAVQMetaObject@@XZ@4QBUQUParameter@@B 1003b014     moc_manage_tempimpl.obj
 0003:00000024       ?param_slot_14@?3??staticMetaObject@manage_temp@@SAPAVQMetaObject@@XZ@4QBUQUParameter@@B 1003b024     moc_manage_tempimpl.obj
 0003:00000038       _filesave                  1003b038     plugindesc.obj
 0003:00000084       ?param_slot_12@?3??staticMetaObject@alm_bncs_output@@SAPAVQMetaObject@@XZ@4QBUQUParameter@@B 1003b084     moc_alm_bncs_output.obj
 0003:000000b4       ?param_slot_14@?3??staticMetaObject@alm_bncs_output@@SAPAVQMetaObject@@XZ@4QBUQUParameter@@B 1003b0b4     moc_alm_bncs_output.obj
 0003:000000e4       ?param_slot_16@?3??staticMetaObject@alm_bncs_output@@SAPAVQMetaObject@@XZ@4QBUQUParameter@@B 1003b0e4     moc_alm_bncs_output.obj
 0003:000000f4       ?param_slot_5@?3??staticMetaObject@dialog@@SAPAVQMetaObject@@XZ@4QBUQUParameter@@B 1003b0f4     moc_dialogimpl.obj
 0003:00000104       ?param_slot_10@?3??staticMetaObject@dialog@@SAPAVQMetaObject@@XZ@4QBUQUParameter@@B 1003b104     moc_dialogimpl.obj
 0003:00000114       ?param_slot_16@?3??staticMetaObject@dialog@@SAPAVQMetaObject@@XZ@4QBUQUParameter@@B 1003b114     moc_dialogimpl.obj
 0003:00000124       ?param_slot_17@?3??staticMetaObject@dialog@@SAPAVQMetaObject@@XZ@4QBUQUParameter@@B 1003b124     moc_dialogimpl.obj
 0003:000009bc       _allocator_arg             1003b9bc     dialogimpl.obj
 0003:000009bd       _piecewise_construct       1003b9bd     dialogimpl.obj
 0003:000009c0       ?iOffset@?1??autoNumber@dialog@@QAEXXZ@4HA 1003b9c0     dialogimpl.obj
 0003:000009c8       _cleanUp_manage_tempBase   1003b9c8     moc_manage_temp.obj
 0003:000009d0       _cleanUp_manage_temp       1003b9d0     moc_manage_tempimpl.obj
 0003:000009d4       ?param_slot_6@?3??staticMetaObject@manage_temp@@SAPAVQMetaObject@@XZ@4QBUQUParameter@@B 1003b9d4     moc_manage_tempimpl.obj
 0003:000009e4       ?$S1@?3??staticMetaObject@manage_temp@@SAPAVQMetaObject@@XZ@4IA 1003b9e4     moc_manage_tempimpl.obj
 0003:000009e8       ?param_slot_8@?3??staticMetaObject@manage_temp@@SAPAVQMetaObject@@XZ@4QBUQUParameter@@B 1003b9e8     moc_manage_tempimpl.obj
 0003:000009f8       ?param_slot_9@?3??staticMetaObject@manage_temp@@SAPAVQMetaObject@@XZ@4QBUQUParameter@@B 1003b9f8     moc_manage_tempimpl.obj
 0003:00000a2c       _cleanUp_alm_bncs_output   1003ba2c     moc_alm_bncs_output.obj
 0003:00000a30       ?param_slot_3@?3??staticMetaObject@alm_bncs_output@@SAPAVQMetaObject@@XZ@4QBUQUParameter@@B 1003ba30     moc_alm_bncs_output.obj
 0003:00000a40       ?$S1@?3??staticMetaObject@alm_bncs_output@@SAPAVQMetaObject@@XZ@4IA 1003ba40     moc_alm_bncs_output.obj
 0003:00000a44       ?param_slot_4@?3??staticMetaObject@alm_bncs_output@@SAPAVQMetaObject@@XZ@4QBUQUParameter@@B 1003ba44     moc_alm_bncs_output.obj
 0003:00000a54       ?param_slot_13@?3??staticMetaObject@alm_bncs_output@@SAPAVQMetaObject@@XZ@4QBUQUParameter@@B 1003ba54     moc_alm_bncs_output.obj
 0003:00000a64       ?param_signal_0@?3??staticMetaObject@alm_bncs_output@@SAPAVQMetaObject@@XZ@4QBUQUParameter@@B 1003ba64     moc_alm_bncs_output.obj
 0003:00000a88       _cleanUp_autoNumberDialogBase 1003ba88     moc_autonumberdialog.obj
 0003:00000a90       _cleanUp_autoNumberDialog  1003ba90     moc_autonumberdialogimpl.obj
 0003:00000a98       _cleanUp_dialogBase        1003ba98     moc_dialog.obj
 0003:00000aa0       _cleanUp_dialog            1003baa0     moc_dialogimpl.obj
 0003:00000aa4       ?$S1@?3??staticMetaObject@dialog@@SAPAVQMetaObject@@XZ@4IA 1003baa4     moc_dialogimpl.obj
 0003:00000aa8       ?param_slot_15@?3??staticMetaObject@dialog@@SAPAVQMetaObject@@XZ@4QBUQUParameter@@B 1003baa8     moc_dialogimpl.obj
 0003:00000ab8       ?param_slot_18@?3??staticMetaObject@dialog@@SAPAVQMetaObject@@XZ@4QBUQUParameter@@B 1003bab8     moc_dialogimpl.obj
 0003:00000acc       ___proc_attached           1003bacc     MSVCRT:crtdll.obj
 0003:00000ad0       _GS_ExceptionRecord        1003bad0     MSVCRT:gs_report.obj
 0003:00000b20       _GS_ContextRecord          1003bb20     MSVCRT:gs_report.obj
 0003:00000dec       _DebuggerWasPresent        1003bdec     MSVCRT:gs_report.obj
 0004:000000a0       $R000000                   1003c0a0     version.res
 0004:00000540       $R0004A0                   1003c540     version.res
